LX51 LINKER/LOCATER V4.66.30.0                                                          07/27/2019  23:22:19  PAGE 1


LX51 LINKER/LOCATER V4.66.30.0, INVOKED BY:
C:\SILICONLABS\SIMPLICITYSTUDIO\V4\DEVELOPER\TOOLCHAINS\KEIL_8051\9.53\BIN\LX51.EXE ./src/SILABS_STARTUP.OBJ, ./src/gat_
>> nametag_main.OBJ, ./src/InitDevice.OBJ, ./src/Interrupts.OBJ, ./src/fw.OBJ, ./src/driver/efm8_smb1.OBJ, ./src/driver/
>> oled_ssd1306.OBJ, ./src/disp/draw_ssd1306.OBJ, ./src/disp/hsv2rgb.OBJ, ./src/led/rgbled.OBJ, ./src/disp/font.OBJ, ./l
>> ib/efm8ub2/peripheralDrivers/src/pwr.OBJ, ./lib/efm8_assert/assert.OBJ, ./src/user_config.OBJ, ./src/disp/font_table.
>> OBJ, ./src/driver/efm8_spi.OBJ, ./src/driver/efm8ub2_hwid.OBJ, ./src/driver/efm8ub2_userflash.OBJ, ./src/led/rgbled_p
>> rog.OBJ, ./src/math/checksum.OBJ, ./src/math/i8atan2.OBJ, ./src/math/rand16.OBJ, ./src/math/sin7.OBJ, ./src/sensor/ad
>> xl.OBJ, ./src/sensor/lightlevel.OBJ, ./src/ui/btn.OBJ, ./src/ui/menu.OBJ, ./src/ui/menu_0_fn.OBJ, ./src/ui/menu_1_fn.
>> OBJ, ./src/ui/menu_2_fn.OBJ, ./src/ui/menu_5_fn.OBJ, ./src/ui/menu_6_fn.OBJ, ./src/ui/menu_def.OBJ TO GAT_NAMETAG.OMF
>> .CRBUILD REMOVEUNUSED PRINT (.\gat_nametag.m51) PAGEWIDTH (120) PAGELENGTH (65) DISABLEWARNING (15) CLASSES (ECODE (C
>> :0X0-C:0XFBFE), HCONST (C:0X0-C:0XFBFE), XDATA (X:0X0-X:0XFFF), HDATA (X:0X0-X:0XFFF))


CPU MODE:     8051 MODE
MEMORY MODEL: SMALL


INPUT MODULES INCLUDED:
  ./src/SILABS_STARTUP.OBJ (?C_STARTUP)
         COMMENT TYPE 0: AX51 V3.12.0.0
  ./src/gat_nametag_main.OBJ (GAT_NAMETAG_MAIN)
         COMMENT TYPE 0: C51 V9.53.0.0
  ./src/InitDevice.OBJ (INITDEVICE)
         COMMENT TYPE 0: C51 V9.53.0.0
  ./src/Interrupts.OBJ (INTERRUPTS)
         COMMENT TYPE 0: C51 V9.53.0.0
  ./src/fw.OBJ (FW)
         COMMENT TYPE 0: C51 V9.53.0.0
  ./src/driver/efm8_smb1.OBJ (EFM8_SMB1)
         COMMENT TYPE 0: C51 V9.53.0.0
  ./src/driver/oled_ssd1306.OBJ (OLED_SSD1306)
         COMMENT TYPE 0: C51 V9.53.0.0
  ./src/disp/draw_ssd1306.OBJ (DRAW_SSD1306)
         COMMENT TYPE 0: C51 V9.53.0.0
  ./src/disp/hsv2rgb.OBJ (HSV2RGB)
         COMMENT TYPE 0: C51 V9.53.0.0
  ./src/led/rgbled.OBJ (RGBLED)
         COMMENT TYPE 0: C51 V9.53.0.0
  ./src/disp/font.OBJ (FONT)
         COMMENT TYPE 0: C51 V9.53.0.0
  ./lib/efm8ub2/peripheralDrivers/src/pwr.OBJ (PWR)
         COMMENT TYPE 0: C51 V9.53.0.0
  ./lib/efm8_assert/assert.OBJ (ASSERT)
         COMMENT TYPE 0: C51 V9.53.0.0
  ./src/user_config.OBJ (USER_CONFIG)
         COMMENT TYPE 0: C51 V9.53.0.0
  ./src/disp/font_table.OBJ (FONT_TABLE)
         COMMENT TYPE 0: C51 V9.53.0.0
  ./src/driver/efm8_spi.OBJ (EFM8_SPI)
         COMMENT TYPE 0: C51 V9.53.0.0
  ./src/driver/efm8ub2_hwid.OBJ (EFM8UB2_HWID)
         COMMENT TYPE 0: C51 V9.53.0.0
  ./src/driver/efm8ub2_userflash.OBJ (EFM8UB2_USERFLASH)
         COMMENT TYPE 0: C51 V9.53.0.0
  ./src/led/rgbled_prog.OBJ (RGBLED_PROG)
         COMMENT TYPE 0: C51 V9.53.0.0
  ./src/math/checksum.OBJ (CHECKSUM)
         COMMENT TYPE 0: C51 V9.53.0.0
  ./src/math/i8atan2.OBJ (I8ATAN2)
         COMMENT TYPE 0: C51 V9.53.0.0
  ./src/math/rand16.OBJ (RAND16)
         COMMENT TYPE 0: AX51 V3.12.0.0
  ./src/math/sin7.OBJ (SIN7)
LX51 LINKER/LOCATER V4.66.30.0                                                        07/27/2019  23:22:19  PAGE 2


         COMMENT TYPE 0: C51 V9.53.0.0
  ./src/sensor/adxl.OBJ (ADXL)
         COMMENT TYPE 0: C51 V9.53.0.0
  ./src/sensor/lightlevel.OBJ (LIGHTLEVEL)
         COMMENT TYPE 0: C51 V9.53.0.0
  ./src/ui/btn.OBJ (BTN)
         COMMENT TYPE 0: C51 V9.53.0.0
  ./src/ui/menu.OBJ (MENU)
         COMMENT TYPE 0: C51 V9.53.0.0
  ./src/ui/menu_0_fn.OBJ (MENU_0_FN)
         COMMENT TYPE 0: C51 V9.53.0.0
  ./src/ui/menu_1_fn.OBJ (MENU_1_FN)
         COMMENT TYPE 0: C51 V9.53.0.0
  ./src/ui/menu_2_fn.OBJ (MENU_2_FN)
         COMMENT TYPE 0: C51 V9.53.0.0
  ./src/ui/menu_5_fn.OBJ (MENU_5_FN)
         COMMENT TYPE 0: C51 V9.53.0.0
  ./src/ui/menu_6_fn.OBJ (MENU_6_FN)
         COMMENT TYPE 0: C51 V9.53.0.0
  ./src/ui/menu_def.OBJ (MENU_DEF)
         COMMENT TYPE 0: C51 V9.53.0.0
  C:\SILICONLABS\SIMPLICITYSTUDIO\V4\DEVELOPER\TOOLCHAINS\KEIL_8051\9.53\LIB\C51S.LIB (?C_INIT)
         COMMENT TYPE 1: A51 / ASM51 Assembler
  C:\SILICONLABS\SIMPLICITYSTUDIO\V4\DEVELOPER\TOOLCHAINS\KEIL_8051\9.53\LIB\C51S.LIB (?C?CLDPTR)
         COMMENT TYPE 1: A51 / ASM51 Assembler
  C:\SILICONLABS\SIMPLICITYSTUDIO\V4\DEVELOPER\TOOLCHAINS\KEIL_8051\9.53\LIB\C51S.LIB (?C?CLDOPTR)
         COMMENT TYPE 1: A51 / ASM51 Assembler
  C:\SILICONLABS\SIMPLICITYSTUDIO\V4\DEVELOPER\TOOLCHAINS\KEIL_8051\9.53\LIB\C51S.LIB (?C?CILDPTR)
         COMMENT TYPE 1: A51 / ASM51 Assembler
  C:\SILICONLABS\SIMPLICITYSTUDIO\V4\DEVELOPER\TOOLCHAINS\KEIL_8051\9.53\LIB\C51S.LIB (?C?CILDOPTR)
         COMMENT TYPE 1: A51 / ASM51 Assembler
  C:\SILICONLABS\SIMPLICITYSTUDIO\V4\DEVELOPER\TOOLCHAINS\KEIL_8051\9.53\LIB\C51S.LIB (?C?CSTPTR)
         COMMENT TYPE 1: A51 / ASM51 Assembler
  C:\SILICONLABS\SIMPLICITYSTUDIO\V4\DEVELOPER\TOOLCHAINS\KEIL_8051\9.53\LIB\C51S.LIB (?C?CSTOPTR)
         COMMENT TYPE 1: A51 / ASM51 Assembler
  C:\SILICONLABS\SIMPLICITYSTUDIO\V4\DEVELOPER\TOOLCHAINS\KEIL_8051\9.53\LIB\C51S.LIB (?C?IMUL)
         COMMENT TYPE 1: A51 / ASM51 Assembler
  C:\SILICONLABS\SIMPLICITYSTUDIO\V4\DEVELOPER\TOOLCHAINS\KEIL_8051\9.53\LIB\C51S.LIB (?C?UIDIV)
         COMMENT TYPE 1: A51 / ASM51 Assembler
  C:\SILICONLABS\SIMPLICITYSTUDIO\V4\DEVELOPER\TOOLCHAINS\KEIL_8051\9.53\LIB\C51S.LIB (?C?SIDIV)
         COMMENT TYPE 1: A51 / ASM51 Assembler
  C:\SILICONLABS\SIMPLICITYSTUDIO\V4\DEVELOPER\TOOLCHAINS\KEIL_8051\9.53\LIB\C51S.LIB (?C?IILDX)
         COMMENT TYPE 1: A51 / ASM51 Assembler
  C:\SILICONLABS\SIMPLICITYSTUDIO\V4\DEVELOPER\TOOLCHAINS\KEIL_8051\9.53\LIB\C51S.LIB (?C?ILDPTR)
         COMMENT TYPE 1: A51 / ASM51 Assembler
  C:\SILICONLABS\SIMPLICITYSTUDIO\V4\DEVELOPER\TOOLCHAINS\KEIL_8051\9.53\LIB\C51S.LIB (?C?ILDOPTR)
         COMMENT TYPE 1: A51 / ASM51 Assembler
  C:\SILICONLABS\SIMPLICITYSTUDIO\V4\DEVELOPER\TOOLCHAINS\KEIL_8051\9.53\LIB\C51S.LIB (?C?ISTPTR)
         COMMENT TYPE 1: A51 / ASM51 Assembler
  C:\SILICONLABS\SIMPLICITYSTUDIO\V4\DEVELOPER\TOOLCHAINS\KEIL_8051\9.53\LIB\C51S.LIB (?C?ISTOPTR)
         COMMENT TYPE 1: A51 / ASM51 Assembler
  C:\SILICONLABS\SIMPLICITYSTUDIO\V4\DEVELOPER\TOOLCHAINS\KEIL_8051\9.53\LIB\C51S.LIB (?C?ULDIV)
         COMMENT TYPE 1: A51 / ASM51 Assembler
  C:\SILICONLABS\SIMPLICITYSTUDIO\V4\DEVELOPER\TOOLCHAINS\KEIL_8051\9.53\LIB\C51S.LIB (?C?ULCMP)
         COMMENT TYPE 1: A51 / ASM51 Assembler
  C:\SILICONLABS\SIMPLICITYSTUDIO\V4\DEVELOPER\TOOLCHAINS\KEIL_8051\9.53\LIB\C51S.LIB (?C?ULSHR)
         COMMENT TYPE 1: A51 / ASM51 Assembler
  C:\SILICONLABS\SIMPLICITYSTUDIO\V4\DEVELOPER\TOOLCHAINS\KEIL_8051\9.53\LIB\C51S.LIB (?C?LLDXDATA)
         COMMENT TYPE 1: A51 / ASM51 Assembler
  C:\SILICONLABS\SIMPLICITYSTUDIO\V4\DEVELOPER\TOOLCHAINS\KEIL_8051\9.53\LIB\C51S.LIB (?C?LSTXDATA)
         COMMENT TYPE 1: A51 / ASM51 Assembler
  C:\SILICONLABS\SIMPLICITYSTUDIO\V4\DEVELOPER\TOOLCHAINS\KEIL_8051\9.53\LIB\C51S.LIB (?C?OFFXADD)
LX51 LINKER/LOCATER V4.66.30.0                                                        07/27/2019  23:22:19  PAGE 3


         COMMENT TYPE 1: A51 / ASM51 Assembler
  C:\SILICONLABS\SIMPLICITYSTUDIO\V4\DEVELOPER\TOOLCHAINS\KEIL_8051\9.53\LIB\C51S.LIB (?C?PLDIIDATA)
         COMMENT TYPE 1: A51 / ASM51 Assembler
  C:\SILICONLABS\SIMPLICITYSTUDIO\V4\DEVELOPER\TOOLCHAINS\KEIL_8051\9.53\LIB\C51S.LIB (?C?PLDXDATA)
         COMMENT TYPE 1: A51 / ASM51 Assembler
  C:\SILICONLABS\SIMPLICITYSTUDIO\V4\DEVELOPER\TOOLCHAINS\KEIL_8051\9.53\LIB\C51S.LIB (?C?PSTXDATA)
         COMMENT TYPE 1: A51 / ASM51 Assembler
  C:\SILICONLABS\SIMPLICITYSTUDIO\V4\DEVELOPER\TOOLCHAINS\KEIL_8051\9.53\LIB\C51S.LIB (?C?PLDPDATA)
         COMMENT TYPE 1: A51 / ASM51 Assembler
  C:\SILICONLABS\SIMPLICITYSTUDIO\V4\DEVELOPER\TOOLCHAINS\KEIL_8051\9.53\LIB\C51S.LIB (?C?PSTPDATA)
         COMMENT TYPE 1: A51 / ASM51 Assembler
  C:\SILICONLABS\SIMPLICITYSTUDIO\V4\DEVELOPER\TOOLCHAINS\KEIL_8051\9.53\LIB\C51S.LIB (?C?PLDCODE)
         COMMENT TYPE 1: A51 / ASM51 Assembler
  C:\SILICONLABS\SIMPLICITYSTUDIO\V4\DEVELOPER\TOOLCHAINS\KEIL_8051\9.53\LIB\C51S.LIB (?C?CCASE)
         COMMENT TYPE 1: A51 / ASM51 Assembler
  C:\SILICONLABS\SIMPLICITYSTUDIO\V4\DEVELOPER\TOOLCHAINS\KEIL_8051\9.53\LIB\C51S.LIB (?C?ICALL)
         COMMENT TYPE 1: A51 / ASM51 Assembler
  C:\SILICONLABS\SIMPLICITYSTUDIO\V4\DEVELOPER\TOOLCHAINS\KEIL_8051\9.53\LIB\C51S.LIB (PRINTF)
         COMMENT TYPE 1: A51 / ASM51 Assembler
  C:\SILICONLABS\SIMPLICITYSTUDIO\V4\DEVELOPER\TOOLCHAINS\KEIL_8051\9.53\LIB\C51S.LIB (ABS)
         COMMENT TYPE 1: A51 / ASM51 Assembler
  C:\SILICONLABS\SIMPLICITYSTUDIO\V4\DEVELOPER\TOOLCHAINS\KEIL_8051\9.53\LIB\C51S.LIB (?C?STRCPY)
         COMMENT TYPE 1: A51 / ASM51 Assembler
  C:\SILICONLABS\SIMPLICITYSTUDIO\V4\DEVELOPER\TOOLCHAINS\KEIL_8051\9.53\LIB\C51S.LIB (STRLEN)
         COMMENT TYPE 1: A51 / ASM51 Assembler
  C:\SILICONLABS\SIMPLICITYSTUDIO\V4\DEVELOPER\TOOLCHAINS\KEIL_8051\9.53\LIB\C51S.LIB (?C?MEMSET)
         COMMENT TYPE 1: A51 / ASM51 Assembler
  C:\SILICONLABS\SIMPLICITYSTUDIO\V4\DEVELOPER\TOOLCHAINS\KEIL_8051\9.53\LIB\C51S.LIB (PUTCHAR)
         COMMENT TYPE 1: A51 / ASM51 Assembler


ACTIVE MEMORY CLASSES OF MODULE:  GAT_NAMETAG.OMF.CRBUILD (?C_STARTUP)

BASE        START       END         USED      MEMORY CLASS
==========================================================
C:000000H   C:000000H   C:00FBFEH             ECODE
B00:0000H   C:000000H   C:00FBFEH             HCONST
X:000000H   X:000000H   X:000FFFH   000495H   XDATA
X:000000H   X:000000H   X:000FFFH             HDATA
C:000000H   C:000000H   C:00FFFFH   005BB3H   CODE
I:000000H   I:000000H   I:0000FFH   000029H   IDATA
I:000000H   I:000000H   I:00007FH   000063H   DATA
C:000000H   C:000000H   C:00FFFFH   0074D4H   CONST
I:000020H.0 I:000020H.0 I:00002FH.7 000001H.4 BIT
X:000000H   X:000000H   X:0000FFH   00002BH   PDATA


MEMORY MAP OF MODULE:  GAT_NAMETAG.OMF.CRBUILD (?C_STARTUP)


START     STOP      LENGTH    ALIGN  RELOC    MEMORY CLASS   SEGMENT NAME
=========================================================================

* * * * * * * * * * *   D A T A   M E M O R Y   * * * * * * * * * * * * *
000000H   000007H   000008H   ---    AT..     DATA           "REG BANK 0"
000008H   000012H   00000BH   BYTE   UNIT     DATA           ?DT?EFM8_SMB1
000013H   000017H   000005H   BYTE   UNIT     DATA           ?DT?FW
000018H   00001BH   000004H   BYTE   UNIT     DATA           ?DT?MENU
00001CH   00001EH   000003H   BYTE   UNIT     DATA           ?DT?DRAW_SSD1306
00001FH   00001FH   000001H   BYTE   UNIT     DATA           ?DT?USER_CONFIG
000020H.0 000021H.0 000001H.1 BIT    UNIT     BIT            _BIT_GROUP_
000021H.1 000021H.2 000000H.2 BIT    UNIT     BIT            ?BI?FW
LX51 LINKER/LOCATER V4.66.30.0                                                        07/27/2019  23:22:19  PAGE 4


000021H.3 000021H.3 000000H.1 BIT    UNIT     BIT            ?BI?OLED_SSD1306
000021H.4 000021H   000000H.4 ---    ---      **GAP**
000022H   00005EH   00003DH   BYTE   UNIT     DATA           _DATA_GROUP_
00005FH   000060H   000002H   BYTE   UNIT     DATA           ?DT?EFM8UB2_HWID
000061H   000062H   000002H   BYTE   UNIT     DATA           ?DT?EFM8UB2_USERFLASH
000063H   000064H   000002H   BYTE   UNIT     DATA           ?DT?MENU_6_FN
000065H   000080H   00001CH   BYTE   UNIT     IDATA          ?ID?RGBLED
000081H   000083H   000003H   BYTE   UNIT     IDATA          ?ID?FW
000084H   000085H   000002H   BYTE   UNIT     IDATA          ?ID?USER_CONFIG
000086H   000087H   000002H   BYTE   UNIT     IDATA          ?ID?RGBLED_PROG
000088H   000089H   000002H   BYTE   UNIT     IDATA          ?ID?MENU_2_FN
00008AH   00008AH   000001H   BYTE   UNIT     IDATA          ?ID?EFM8_SMB1
00008BH   00008BH   000001H   BYTE   UNIT     IDATA          ?ID?LIGHTLEVEL
00008CH   00008CH   000001H   BYTE   UNIT     IDATA          ?ID?MENU_0_FN
00008DH   00008DH   000001H   BYTE   UNIT     IDATA          ?STACK

* * * * * * * * * * *   C O D E   M E M O R Y   * * * * * * * * * * * * *
000000H   000002H   000003H   ---    OFFS..   CODE           ?CO?SILABS_STARTUP?3
000003H   000005H   000003H   BYTE   OFFS..   CODE           ?INTERRUPTS?00003
000006H   00008BH   000086H   BYTE   UNIT     CODE           ?PR?_LEDPROG_CCROSS?RGBLED_PROG
00008CH   000092H   000007H   BYTE   UNIT     CODE           ?PR?SMBUS_1_ENTER_DEFAULTMODE_FROM_RESET?INITDEVICE
000093H   000095H   000003H   BYTE   OFFS..   CODE           ?INTERRUPTS?00093
000096H   0000A2H   00000DH   BYTE   UNIT     CODE           ?PR?PCA_0_ENTER_DEFAULTMODE_FROM_RESET?INITDEVICE
0000A3H   0000A5H   000003H   BYTE   OFFS..   CODE           ?INTERRUPTS?000A3
0000A6H   00062CH   000587H   BYTE   UNIT     CODE           ?PR?_MENU_6_DISP?MENU_6_FN
00062DH   000AF4H   0004C8H   BYTE   UNIT     CODE           ?C?LIB_CODE
000AF5H   000E5AH   000366H   BYTE   UNIT     CODE           ?PR?_MENU_NONE_DISP?MENU_0_FN
000E5BH   0011B8H   00035EH   BYTE   UNIT     CODE           ?PR?_SSD1306FB_DRAW_RAW?DRAW_SSD1306
0011B9H   001514H   00035CH   BYTE   UNIT     CODE           ?PR?PRINTF?PRINTF
001515H   00185AH   000346H   BYTE   UNIT     CODE           ?PR?_MENU_2_DISP?MENU_2_FN
00185BH   001B7BH   000321H   BYTE   UNIT     CODE           ?PR?_SSD1306FB_COPY?DRAW_SSD1306
001B7CH   001E79H   0002FEH   BYTE   UNIT     CODE           ?PR?_MENU_1_DISP?MENU_1_FN
001E7AH   002154H   0002DBH   BYTE   UNIT     CODE           ?PR?_MENU_DRAW_BUTTONS?MENU
002155H   002367H   000213H   BYTE   UNIT     CODE           ?PR?_SSD1306FB_ROTATE?DRAW_SSD1306
002368H   002523H   0001BCH   BYTE   UNIT     CODE           ?PR?_SSD1306FB_INTERNAL_STR?DRAW_SSD1306
002524H   0026D1H   0001AEH   BYTE   UNIT     CODE           ?PR?_SSD1306FB_DRAW_VLINE?DRAW_SSD1306
0026D2H   00287AH   0001A9H   BYTE   UNIT     CODE           ?PR?FW_TICK_CRITICAL?FW
00287BH   0029F7H   00017DH   BYTE   UNIT     CODE           ?CO?RGBLED_PROG
0029F8H   002B59H   000162H   BYTE   UNIT     CODE           ?PR?BTN_CALLBACK?BTN
002B5AH   002CB9H   000160H   BYTE   UNIT     CODE           ?PR?_HSV2RGB_8B?HSV2RGB
002CBAH   002E06H   00014DH   BYTE   UNIT     CODE           ?PR?SMB1_INTERRUPT?EFM8_SMB1
002E07H   002F4EH   000148H   BYTE   UNIT     CODE           ?PR?_RGBLED_UPDATE?RGBLED
002F4FH   003071H   000123H   BYTE   UNIT     CODE           ?PR?_MENU_5_DISP?MENU_5_FN
003072H   003192H   000121H   BYTE   UNIT     CODE           ?PR?BTN_TICK?BTN
003193H   0032A5H   000113H   BYTE   UNIT     CODE           ?PR?_LEDPROG_PFADE1?RGBLED_PROG
0032A6H   0033B8H   000113H   BYTE   UNIT     CODE           ?CO?MENU_6_FN
0033B9H   0034BCH   000104H   BYTE   UNIT     CODE           ?PR?_LEDPROG_FLICKER?RGBLED_PROG
0034BDH   0035B5H   0000F9H   BYTE   UNIT     CODE           ?PR?_MENU_0_DISP?MENU_0_FN
0035B6H   0036A4H   0000EFH   BYTE   UNIT     CODE           ?PR?_LEDPROG_RANDOMCOLOR?RGBLED_PROG
0036A5H   003792H   0000EEH   BYTE   UNIT     CODE           ?PR?_SSD1306FB_DRAW_HLINE?DRAW_SSD1306
003793H   003876H   0000E4H   BYTE   UNIT     CODE           ?PR?_LEDPROG_RAINBOW?RGBLED_PROG
003877H   003952H   0000DCH   BYTE   UNIT     CODE           ?PR?FW_OLED_UPDATE_DONE?FW
003953H   003A2CH   0000DAH   BYTE   UNIT     CODE           ?PR?MENU_1_NAME_EDIT?MENU_1_FN
003A2DH   003B01H   0000D5H   BYTE   UNIT     CODE           ?PR?_SSD1306FB_DRAW_CIRCLE?DRAW_SSD1306
003B02H   003BD5H   0000D4H   BYTE   UNIT     CODE           ?CO?MENU_0_FN
003BD6H   003CA4H   0000CFH   BYTE   UNIT     CODE           ?PR?_I8ATAN2?I8ATAN2
003CA5H   003D70H   0000CCH   BYTE   UNIT     CODE           ?CO?MENU_1_FN
003D71H   003E38H   0000C8H   BYTE   UNIT     CODE           ?PR?UCONF_WRITE?USER_CONFIG
003E39H   003EFFH   0000C7H   BYTE   UNIT     CODE           ?PR?_SSD1306FB_DRAW_LINE?DRAW_SSD1306
003F00H   003FC0H   0000C1H   BYTE   UNIT     CODE           ?PR?_LEDPROG_CMIRROR?RGBLED_PROG
003FC1H   004079H   0000B9H   BYTE   UNIT     CODE           ?PR?_LEDPROG_CFLIP?RGBLED_PROG
00407AH   004131H   0000B8H   BYTE   UNIT     CODE           ?PR?_LEDPROG_SOLID?RGBLED_PROG
LX51 LINKER/LOCATER V4.66.30.0                                                        07/27/2019  23:22:19  PAGE 5


004132H   0041E9H   0000B8H   BYTE   UNIT     CODE           ?PR?_LEDPROG_RANDOM?RGBLED_PROG
0041EAH   00429AH   0000B1H   BYTE   UNIT     CODE           ?PR?_MENU_1_ENTER?MENU_1_FN
00429BH   004349H   0000AFH   BYTE   UNIT     CODE           ?PR?_LEDPROG_CALT?RGBLED_PROG
00434AH   0043F8H   0000AFH   BYTE   UNIT     CODE           ?PR?MENU_1_BTN_NEXT?MENU_1_FN
0043F9H   0044A6H   0000AEH   BYTE   UNIT     CODE           ?PR?_MENU_2_BTN_USE?MENU_2_FN
0044A7H   004553H   0000ADH   BYTE   UNIT     CODE           ?PR?MENU_1_BTN_USE?MENU_1_FN
004554H   0045F1H   00009EH   BYTE   UNIT     CODE           ?PR?MENU_1_BTN_PREV?MENU_1_FN
0045F2H   004689H   000098H   BYTE   UNIT     CODE           ?PR?_SSD1306FB_DRAW_PIX?DRAW_SSD1306
00468AH   00471CH   000093H   BYTE   UNIT     CODE           ?PR?MENU_BTN_USE_STD?MENU
00471DH   0047ACH   000090H   BYTE   UNIT     CODE           ?PR?_LEDPROG_CIRCLER?RGBLED_PROG
0047ADH   00483BH   00008FH   BYTE   UNIT     CODE           ?C_C51STARTUP
00483CH   0048CAH   00008FH   BYTE   UNIT     CODE           ?PR?BTN_INIT?BTN
0048CBH   00494FH   000085H   BYTE   UNIT     CODE           ?PR?FW_TICK_MAINLOOP?FW
004950H   0049D1H   000082H   BYTE   UNIT     CODE           ?PR?_SSD1306FB_GET_STR_WIDTH?DRAW_SSD1306
0049D2H   004A50H   00007FH   BYTE   UNIT     CODE           ?PR?FW_INIT?FW
004A51H   004ACFH   00007FH   BYTE   UNIT     CODE           ?PR?_MENU_DRAW_TABS?MENU
004AD0H   004B4AH   00007BH   BYTE   UNIT     CODE           ?CO?FONT_TABLE
004B4BH   004BC2H   000078H   BYTE   UNIT     CODE           ?PR?_ADXL345_GET_AXES?ADXL
004BC3H   004C25H   000063H   BYTE   UNIT     CODE           ?CO?MENU_2_FN
004C26H   004C86H   000061H   BYTE   UNIT     CODE           ?PR?HWID_GET_MODEL?EFM8UB2_HWID
004C87H   004CE7H   000061H   BYTE   UNIT     CODE           ?PR?ADXL345_TICK?ADXL
004CE8H   004D47H   000060H   BYTE   UNIT     CODE           ?PR?MENU_1_BTN_EXIT?MENU_1_FN
004D48H   004DA5H   00005EH   BYTE   UNIT     CODE           ?PR?UCONF_LOAD?USER_CONFIG
004DA6H   004E03H   00005EH   BYTE   UNIT     CODE           ?PR?MENU_TICK?MENU
004E04H   004E60H   00005DH   BYTE   UNIT     CODE           ?PR?_SSD1306_INIT?OLED_SSD1306
004E61H   004EBDH   00005DH   BYTE   UNIT     CODE           ?PR?SSD1306_UPDATE?OLED_SSD1306
004EBEH   004F18H   00005BH   BYTE   UNIT     CODE           ?PR?UCONF_DEFAULTS?USER_CONFIG
004F19H   004F72H   00005AH   BYTE   UNIT     CODE           ?CO?MENU
004F73H   004FCCH   00005AH   BYTE   UNIT     CODE           ?PR?_MENU_2_ENTER?MENU_2_FN
004FCDH   00501CH   000050H   BYTE   UNIT     CODE           ?PR?_SSD1306_SET_FLIP?OLED_SSD1306
00501DH   00506CH   000050H   BYTE   UNIT     CODE           ?PR?_SSD1306_SET_MIRROR?OLED_SSD1306
00506DH   0050BBH   00004FH   BYTE   UNIT     CODE           ?PR?ENTER_DEFAULTMODE_FROM_RESET?INITDEVICE
0050BCH   00510AH   00004FH   BYTE   UNIT     CODE           ?PR?MENU_2_BTN_NEXT?MENU_2_FN
00510BH   005159H   00004FH   BYTE   UNIT     CODE           ?PR?MENU_2_BTN_PREV?MENU_2_FN
00515AH   0051A7H   00004EH   BYTE   UNIT     CODE           ?PR?_UCONF_VALIDATE?USER_CONFIG
0051A8H   0051F4H   00004DH   BYTE   UNIT     CODE           ?PR?_SSD1306_CLS?OLED_SSD1306
0051F5H   00523FH   00004BH   BYTE   UNIT     CODE           ?PR?_BTN_CHECK?BTN
005240H   00528AH   00004BH   BYTE   UNIT     CODE           ?PR?_MENU_NONE_PRINT_ERROR?MENU_0_FN
00528BH   0052D0H   000046H   BYTE   UNIT     CODE           ?PR?TIMER5_ISR?INTERRUPTS
0052D1H   005316H   000046H   BYTE   UNIT     CODE           ?PR?_SPI0_XFER?EFM8_SPI
005317H   00535AH   000044H   BYTE   UNIT     CODE           ?PR?_MENU_5_ENTER?MENU_5_FN
00535BH   00539CH   000042H   BYTE   UNIT     CODE           ?PR?ADXL345_INIT?ADXL
00539DH   0053D9H   00003DH   BYTE   UNIT     CODE           ?CO?MENU_5_FN
0053DAH   005416H   00003DH   BYTE   UNIT     CODE           ?PR?MENU_6_BTN_USE?MENU_6_FN
005417H   005452H   00003CH   BYTE   UNIT     CODE           ?PR?_SSD1306_SET_DISPLAY?OLED_SSD1306
005453H   00548DH   00003BH   BYTE   UNIT     CODE           ?PR?SMBUS1_ISR?INTERRUPTS
00548EH   0054C7H   00003AH   BYTE   UNIT     CODE           ?PR?_SIN7?SIN7
0054C8H   005500H   000039H   BYTE   UNIT     CODE           ?PR?RAND16?RAND16
005501H   005539H   000039H   BYTE   UNIT     CODE           ?PR?MENU_NONE_INIT?MENU_0_FN
00553AH   005572H   000039H   BYTE   UNIT     CODE           ?PR?_MENU_0_ENTER?MENU_0_FN
005573H   0055AAH   000038H   BYTE   UNIT     CODE           ?PR?_MENU_6_FONT_GLYPH?MENU_6_FN
0055ABH   0055E0H   000036H   BYTE   UNIT     CODE           ?PR?MENU_BTN_EXIT?MENU
0055E1H   005615H   000035H   BYTE   UNIT     CODE           ?C_INITSEG
005616H   005646H   000031H   BYTE   UNIT     CODE           ?PR?_USERFLASH_WRITE?EFM8UB2_USERFLASH
005647H   005676H   000030H   BYTE   UNIT     CODE           ?PR?_SSD1306FB_DRAW_RECT?DRAW_SSD1306
005677H   0056A4H   00002EH   BYTE   UNIT     CODE           ?PR?MENU_BTN_USE_NONE?MENU
0056A5H   0056D0H   00002CH   BYTE   UNIT     CODE           ?PR?_IAT2?I8ATAN2
0056D1H   0056FBH   00002BH   BYTE   UNIT     CODE           ?PR?_SSD1306FB_DRAW_STR?DRAW_SSD1306
0056FCH   005726H   00002BH   BYTE   UNIT     CODE           ?PR?_USERFLASH_READ?EFM8UB2_USERFLASH
005727H   005751H   00002BH   BYTE   UNIT     CODE           ?PR?MENU_BTN_ENTER?MENU
005752H   005778H   000027H   BYTE   UNIT     CODE           ?PR?PUTCHAR?PUTCHAR
005779H   00579EH   000026H   BYTE   UNIT     CODE           ?PR?_SMB1_MWRITE?EFM8_SMB1
LX51 LINKER/LOCATER V4.66.30.0                                                        07/27/2019  23:22:19  PAGE 6


00579FH   0057C2H   000024H   BYTE   UNIT     CODE           ?PR?SSD1306_IDLE_WAIT?OLED_SSD1306
0057C3H   0057E6H   000024H   BYTE   UNIT     CODE           ?PR?MENU_1_FONT_NEXT?MENU_1_FN
0057E7H   005807H   000021H   BYTE   UNIT     CODE           ?PR?_ADXL345_GET_ROTATION?ADXL
005808H   005827H   000020H   BYTE   UNIT     CODE           ?PR?_USERFLASH_WRITE_BYTE?EFM8UB2_USERFLASH
005828H   005846H   00001FH   BYTE   UNIT     CODE           ?PR?_SSD1306FB_SET_COLOR?DRAW_SSD1306
005847H   005865H   00001FH   BYTE   UNIT     CODE           ?PR?_MENU_NONE_SET_FLIPMIRROR?MENU_0_FN
005866H   005883H   00001EH   BYTE   UNIT     CODE           ?PR?_LSENS_PULSE?LIGHTLEVEL
005884H   0058A0H   00001DH   BYTE   UNIT     CODE           ?PR?SSD1306_INIT_STEP3?OLED_SSD1306
0058A1H   0058BDH   00001DH   BYTE   UNIT     CODE           ?PR?_USERFLASH_RESERVE_PAGES?EFM8UB2_USERFLASH
0058BEH   0058DAH   00001DH   BYTE   UNIT     CODE           ?PR?_CHECKSUM_GEN?CHECKSUM
0058DBH   0058F4H   00001AH   BYTE   UNIT     CODE           ?PR?_MENU_6_FONT_INDEX?MENU_6_FN
0058F5H   00590DH   000019H   BYTE   UNIT     CODE           ?PR?_MENU_NONE_SET_HALFWIDTH?MENU_0_FN
00590EH   005923H   000016H   BYTE   UNIT     CODE           ?PR?TIMER16_5_ENTER_DEFAULTMODE_FROM_RESET?INITDEVICE
005924H   005939H   000016H   BYTE   UNIT     CODE           ?PR?SSD1306_INIT_STEP2?OLED_SSD1306
00593AH   00594EH   000015H   BYTE   UNIT     CODE           ?PR?TIMER_SETUP_0_ENTER_DEFAULTMODE_FROM_RESET?INITDEVICE
00594FH   005963H   000015H   BYTE   UNIT     CODE           ?PR?_COS7?SIN7
005964H   005978H   000015H   BYTE   UNIT     CODE           ?PR?MENU_BTN_NEXT?MENU
005979H   00598DH   000015H   BYTE   UNIT     CODE           ?PR?_STRLEN?STRLEN
00598EH   0059A1H   000014H   BYTE   UNIT     CODE           ?PR?_SSD1306FB_SET_CURSOR?DRAW_SSD1306
0059A2H   0059B4H   000013H   BYTE   UNIT     CODE           ?PR?MAIN?GAT_NAMETAG_MAIN
0059B5H   0059C7H   000013H   BYTE   UNIT     CODE           ?PR?TIMER16_2_ENTER_DEFAULTMODE_FROM_RESET?INITDEVICE
0059C8H   0059DAH   000013H   BYTE   UNIT     CODE           ?PR?TIMER01_0_ENTER_DEFAULTMODE_FROM_RESET?INITDEVICE
0059DBH   0059EDH   000013H   BYTE   UNIT     CODE           ?PR?MENU_6_FONT_NEXT?MENU_6_FN
0059EEH   005A00H   000013H   BYTE   UNIT     CODE           ?PR?MENU_6_FONT_PREV?MENU_6_FN
005A01H   005A12H   000012H   BYTE   UNIT     CODE           ?PR?LSENS_TICK?LIGHTLEVEL
005A13H   005A24H   000012H   BYTE   UNIT     CODE           ?PR?_MENU_START?MENU
005A25H   005A36H   000012H   BYTE   UNIT     CODE           ?PR?MENU_BTN_PREV?MENU
005A37H   005A48H   000012H   BYTE   UNIT     CODE           ?PR?MENU_1_BTN_ENTER?MENU_1_FN
005A49H   005A59H   000011H   BYTE   UNIT     CODE           ?PR?USERFLASH_INIT?EFM8UB2_USERFLASH
005A5AH   005A69H   000010H   BYTE   UNIT     CODE           ?PR?SPI_0_ENTER_DEFAULTMODE_FROM_RESET?INITDEVICE
005A6AH   005A79H   000010H   BYTE   UNIT     CODE           ?PR?_SSD1306_SET_FLIPMIRROR?OLED_SSD1306
005A7AH   005A88H   00000FH   BYTE   UNIT     CODE           ?PR?_MENU_2_VAL_INC?MENU_2_FN
005A89H   005A96H   00000EH   BYTE   UNIT     CODE           ?PR?PWR_ENTERIDLE?PWR
005A97H   005AA4H   00000EH   BYTE   UNIT     CODE           ?PR?_MENU_2_VAL_DEC?MENU_2_FN
005AA5H   005AB1H   00000DH   BYTE   UNIT     CODE           ?PR?PORTS_0_ENTER_DEFAULTMODE_FROM_RESET?INITDEVICE
005AB2H   005ABEH   00000DH   BYTE   UNIT     CODE           ?PR?PORTS_2_ENTER_DEFAULTMODE_FROM_RESET?INITDEVICE
005ABFH   005ACBH   00000DH   BYTE   UNIT     CODE           ?PR?_SPI0_XFER_BYTE?EFM8_SPI
005ACCH   005AD8H   00000DH   BYTE   UNIT     CODE           ?PR?_RAND16_INIT?RAND16
005AD9H   005AE4H   00000CH   BYTE   UNIT     CODE           ?PR?_ABS?ABS
005AE5H   005AEEH   00000AH   BYTE   UNIT     CODE           ?PR?PCACH_0_ENTER_DEFAULTMODE_FROM_RESET?INITDEVICE
005AEFH   005AF8H   00000AH   BYTE   UNIT     CODE           ?PR?PCACH_1_ENTER_DEFAULTMODE_FROM_RESET?INITDEVICE
005AF9H   005B02H   00000AH   BYTE   UNIT     CODE           ?PR?PCACH_2_ENTER_DEFAULTMODE_FROM_RESET?INITDEVICE
005B03H   005B0CH   00000AH   BYTE   UNIT     CODE           ?PR?PCACH_3_ENTER_DEFAULTMODE_FROM_RESET?INITDEVICE
005B0DH   005B16H   00000AH   BYTE   UNIT     CODE           ?PR?PORTS_1_ENTER_DEFAULTMODE_FROM_RESET?INITDEVICE
005B17H   005B20H   00000AH   BYTE   UNIT     CODE           ?PR?PBCFG_0_ENTER_DEFAULTMODE_FROM_RESET?INITDEVICE
005B21H   005B2AH   00000AH   BYTE   UNIT     CODE           ?PR?ADC_0_ENTER_DEFAULTMODE_FROM_RESET?INITDEVICE
005B2BH   005B34H   00000AH   BYTE   UNIT     CODE           ?PR?INTERRUPT_0_ENTER_DEFAULTMODE_FROM_RESET?INITDEVICE
005B35H   005B3EH   00000AH   BYTE   UNIT     CODE           ?PR?SMBUS_0_ENTER_DEFAULTMODE_FROM_RESET?INITDEVICE
005B3FH   005B48H   00000AH   BYTE   UNIT     CODE           ?PR?SMB1_STOP?EFM8_SMB1
005B49H   005B51H   000009H   BYTE   UNIT     CODE           ?PR?SSD1306_CB_GET?OLED_SSD1306
005B52H   005B5AH   000009H   BYTE   UNIT     CODE           ?PR?_SSD1306FB_GET_FONT_HEIGHT?DRAW_SSD1306
005B5BH   005B63H   000009H   BYTE   UNIT     CODE           ?PR?_MENU_STOP?MENU
005B64H   005B6BH   000008H   BYTE   UNIT     CODE           ?PR?_SSD1306_CB?OLED_SSD1306
005B6CH   005B73H   000008H   BYTE   UNIT     CODE           ?PR?_USERFLASH_ERASE_PAGE?EFM8UB2_USERFLASH
005B74H   005B7AH   000007H   BYTE   UNIT     CODE           ?PR?PCACH_4_ENTER_DEFAULTMODE_FROM_RESET?INITDEVICE
005B7BH   005B81H   000007H   BYTE   UNIT     CODE           ?PR?_SSD1306FB_SET_TARGET?DRAW_SSD1306
005B82H   005B88H   000007H   BYTE   UNIT     CODE           ?PR?HWID_INIT?EFM8UB2_HWID
005B89H   005B8FH   000007H   BYTE   UNIT     CODE           ?PR?MENU_2_BTN_EXIT?MENU_2_FN
005B90H   005B94H   000005H   BYTE   UNIT     CODE           ?CO?USER_CONFIG
005B95H   005B99H   000005H   BYTE   UNIT     CODE           ?PR?USERFLASH_GET_BASEADDR?EFM8UB2_USERFLASH
005B9AH   005B9DH   000004H   BYTE   UNIT     CODE           ?PR?HFOSC_0_ENTER_DEFAULTMODE_FROM_RESET?INITDEVICE
005B9EH   005BA1H   000004H   BYTE   UNIT     CODE           ?PR?CLOCK_0_ENTER_DEFAULTMODE_FROM_RESET?INITDEVICE
LX51 LINKER/LOCATER V4.66.30.0                                                        07/27/2019  23:22:19  PAGE 7


005BA2H   005BA5H   000004H   BYTE   UNIT     CODE           ?PR?EXTINT_0_ENTER_DEFAULTMODE_FROM_RESET?INITDEVICE
005BA6H   005BA9H   000004H   BYTE   UNIT     CODE           ?PR?UART_0_ENTER_DEFAULTMODE_FROM_RESET?INITDEVICE
005BAAH   005BACH   000003H   BYTE   UNIT     CODE           ?PR?INT0_ISR?INTERRUPTS
005BADH   005BAFH   000003H   BYTE   UNIT     CODE           ?PR?SMB1_GET_STATE?EFM8_SMB1
005BB0H   005BB0H   000001H   BYTE   UNIT     CODE           ?PR?SILABS_STARTUP?GAT_NAMETAG_MAIN
005BB1H   005BB1H   000001H   BYTE   UNIT     CODE           ?PR?PORTS_3_ENTER_DEFAULTMODE_FROM_RESET?INITDEVICE
005BB2H   005BB2H   000001H   BYTE   UNIT     CODE           ?PR?_LEDPROG_SOLID_EDIT?RGBLED_PROG
005BB3H   00CFF6H   007444H   BYTE   UNIT     CONST          ?CO?FONT
00CFF7H   00D03EH   000048H   BYTE   UNIT     CONST          ?CO?MENU_DEF
00D03FH   00D05FH   000021H   BYTE   UNIT     CONST          ?CO?SIN7
00D060H   00D07FH   000020H   BYTE   UNIT     CONST          ?CO?OLED_SSD1306
00D080H   00D086H   000007H   BYTE   UNIT     CONST          ?CO?FW

* * * * * * * * * * *  X D A T A   M E M O R Y  * * * * * * * * * * * * *
000000H   000022H   000023H   BYTE   INPAGE   PDATA          _PDATA_GROUP_
000023H   00002AH   000008H   BYTE   INPAGE   PDATA          ?PD?OLED_SSD1306
00002BH   000238H   00020EH   BYTE   UNIT     XDATA          ?XD?OLED_SSD1306
000239H   000392H   00015AH   BYTE   UNIT     XDATA          ?XD?MENU_0_FN
000393H   000412H   000080H   BYTE   UNIT     XDATA          ?XD?USER_CONFIG
000413H   000460H   00004EH   BYTE   UNIT     XDATA          _XDATA_GROUP_
000461H   0004A4H   000044H   BYTE   UNIT     XDATA          ?XD?BTN
0004A5H   0004B7H   000013H   BYTE   UNIT     XDATA          ?XD?ADXL
0004B8H   0004BBH   000004H   BYTE   UNIT     XDATA          ?XD?RAND16
0004BCH   0004BEH   000003H   BYTE   UNIT     XDATA          ?XD?MENU_1_FN
0004BFH   0004BFH   000001H   BYTE   UNIT     XDATA          ?XD?RGBLED_PROG

* * * * * * * * *   R E M O V E D     S E G M E N T S   * * * * * * * *
   *DEL*:           000009H   BYTE   UNIT     CODE           ?PR?LFOSC_0_ENTER_DEFAULTMODE_FROM_RESET?INITDEVICE
   *DEL*:           000004H   BYTE   UNIT     CODE           ?PR?CIP51_0_ENTER_DEFAULTMODE_FROM_RESET?INITDEVICE
   *DEL*:           000013H   BYTE   UNIT     CODE           ?PR?TIMER16_4_ENTER_DEFAULTMODE_FROM_RESET?INITDEVICE
   *DEL*:           000026H   BYTE   UNIT     CODE           ?PR?_SMB1_MREAD?EFM8_SMB1
   *DEL*:           000009H   BYTE   UNIT     DATA           ?DT?_SMB1_MREAD?EFM8_SMB1
   *DEL*:           000033H   BYTE   UNIT     CODE           ?PR?_SSD1306_CMD?OLED_SSD1306
   *DEL*:           00003CH   BYTE   UNIT     CODE           ?PR?_SSD1306_SET_INVERT?OLED_SSD1306
   *DEL*:           000043H   BYTE   UNIT     CODE           ?PR?_SSD1306_SET_CONTRAST?OLED_SSD1306
   *DEL*:           000028H   BYTE   UNIT     CODE           ?PR?_SSD1306FB_DRAW_RECT_FILL?DRAW_SSD1306
   *DEL*:           000004H   BYTE   UNIT     DATA           ?DT?_SSD1306FB_DRAW_RECT_FILL?DRAW_SSD1306
   *DEL*:           00000FH   BYTE   UNIT     CODE           ?PR?PWR_ENTERSTOP?PWR
   *DEL*:           00001BH   BYTE   UNIT     CODE           ?PR?PWR_ENTERSUSPEND?PWR
   *DEL*:           000009H   BYTE   UNIT     CODE           ?PR?PWR_ENTERSHUTDOWN?PWR
   *DEL*:           000002H   BYTE   UNIT     CODE           ?PR?SLAB_ASSERT?ASSERT
   *DEL*:           000016H   BYTE   UNIT     CODE           ?PR?_HWID_GET_BYTE?EFM8UB2_HWID
   *DEL*:           000001H   BYTE   UNIT     CODE           ?PR?_LEDPROG_NONE?RGBLED_PROG
   *DEL*:           00000CH   BYTE   UNIT     CODE           ?PR?_CHECKSUM_VERIFY?CHECKSUM
   *DEL*:           000005H   BYTE   UNIT     DATA           ?DT?_CHECKSUM_VERIFY?CHECKSUM
   *DEL*:           000001H   BYTE   UNIT     CODE           ?PR?_ADXL345_SET_INTERRUPT?ADXL
   *DEL*:           00001EH   BYTE   UNIT     CODE           ?PR?ADXL345_GET_INTERRUPT?ADXL
   *DEL*:           000001H   BYTE   UNIT     CODE           ?PR?LSENS_READ?LIGHTLEVEL
   *DEL*:           00003DH   BYTE   UNIT     CODE           ?PR?MENU_1_GET_OFFSET?MENU_1_FN



OVERLAY MAP OF MODULE:   GAT_NAMETAG.OMF.CRBUILD (?C_STARTUP)


FUNCTION/MODULE                                BIT_GROUP   DATA_GROUP   PDATA_GROUP  XDATA_GROUP
--> CALLED FUNCTION/MODULE                    START  STOP  START  STOP  START  STOP  START  STOP
================================================================================================
?C_C51STARTUP                                 ----- -----  ----- -----  ----- -----  ----- -----
  +--> SILABS_STARTUP/GAT_NAMETAG_MAIN
  +--> MAIN/GAT_NAMETAG_MAIN
  +--> ?C_INITSEG
LX51 LINKER/LOCATER V4.66.30.0                                                        07/27/2019  23:22:19  PAGE 8



SILABS_STARTUP/GAT_NAMETAG_MAIN               ----- -----  ----- -----  ----- -----  ----- -----

MAIN/GAT_NAMETAG_MAIN                         ----- -----  ----- -----  ----- -----  ----- -----
  +--> ENTER_DEFAULTMODE_FROM_RESET/INITDEVICE
  +--> FW_INIT/FW
  +--> PWR_ENTERIDLE/PWR
  +--> FW_TICK_MAINLOOP/FW

ENTER_DEFAULTMODE_FROM_RESET/INITDEVICE       ----- -----  0022H 0022H  ----- -----  ----- -----
  +--> PCA_0_ENTER_DEFAULTMODE_FROM_RESET/INITDEVICE
  +--> PCACH_0_ENTER_DEFAULTMODE_FROM_RESET/INITDEVICE
  +--> PCACH_1_ENTER_DEFAULTMODE_FROM_RESET/INITDEVICE
  +--> PCACH_2_ENTER_DEFAULTMODE_FROM_RESET/INITDEVICE
  +--> PCACH_3_ENTER_DEFAULTMODE_FROM_RESET/INITDEVICE
  +--> PCACH_4_ENTER_DEFAULTMODE_FROM_RESET/INITDEVICE
  +--> PORTS_0_ENTER_DEFAULTMODE_FROM_RESET/INITDEVICE
  +--> PORTS_1_ENTER_DEFAULTMODE_FROM_RESET/INITDEVICE
  +--> PORTS_2_ENTER_DEFAULTMODE_FROM_RESET/INITDEVICE
  +--> PORTS_3_ENTER_DEFAULTMODE_FROM_RESET/INITDEVICE
  +--> PBCFG_0_ENTER_DEFAULTMODE_FROM_RESET/INITDEVICE
  +--> ADC_0_ENTER_DEFAULTMODE_FROM_RESET/INITDEVICE
  +--> HFOSC_0_ENTER_DEFAULTMODE_FROM_RESET/INITDEVICE
  +--> CLOCK_0_ENTER_DEFAULTMODE_FROM_RESET/INITDEVICE
  +--> TIMER01_0_ENTER_DEFAULTMODE_FROM_RESET/INITDEVICE
  +--> TIMER16_2_ENTER_DEFAULTMODE_FROM_RESET/INITDEVICE
  +--> TIMER16_5_ENTER_DEFAULTMODE_FROM_RESET/INITDEVICE
  +--> TIMER_SETUP_0_ENTER_DEFAULTMODE_FROM_RESET/INITDEVICE
  +--> SMBUS_0_ENTER_DEFAULTMODE_FROM_RESET/INITDEVICE
  +--> SMBUS_1_ENTER_DEFAULTMODE_FROM_RESET/INITDEVICE
  +--> SPI_0_ENTER_DEFAULTMODE_FROM_RESET/INITDEVICE
  +--> UART_0_ENTER_DEFAULTMODE_FROM_RESET/INITDEVICE
  +--> EXTINT_0_ENTER_DEFAULTMODE_FROM_RESET/INITDEVICE
  +--> INTERRUPT_0_ENTER_DEFAULTMODE_FROM_RESET/INITDEVICE

PCA_0_ENTER_DEFAULTMODE_FROM_RESET/INITD+     ----- -----  ----- -----  ----- -----  ----- -----
... EVICE

PCACH_0_ENTER_DEFAULTMODE_FROM_RESET/INI+     ----- -----  ----- -----  ----- -----  ----- -----
... TDEVICE

PCACH_1_ENTER_DEFAULTMODE_FROM_RESET/INI+     ----- -----  ----- -----  ----- -----  ----- -----
... TDEVICE

PCACH_2_ENTER_DEFAULTMODE_FROM_RESET/INI+     ----- -----  ----- -----  ----- -----  ----- -----
... TDEVICE

PCACH_3_ENTER_DEFAULTMODE_FROM_RESET/INI+     ----- -----  ----- -----  ----- -----  ----- -----
... TDEVICE

PCACH_4_ENTER_DEFAULTMODE_FROM_RESET/INI+     ----- -----  ----- -----  ----- -----  ----- -----
... TDEVICE

PORTS_0_ENTER_DEFAULTMODE_FROM_RESET/INI+     ----- -----  ----- -----  ----- -----  ----- -----
... TDEVICE

PORTS_1_ENTER_DEFAULTMODE_FROM_RESET/INI+     ----- -----  ----- -----  ----- -----  ----- -----
... TDEVICE

PORTS_2_ENTER_DEFAULTMODE_FROM_RESET/INI+     ----- -----  ----- -----  ----- -----  ----- -----
... TDEVICE

LX51 LINKER/LOCATER V4.66.30.0                                                        07/27/2019  23:22:19  PAGE 9


PORTS_3_ENTER_DEFAULTMODE_FROM_RESET/INI+     ----- -----  ----- -----  ----- -----  ----- -----
... TDEVICE

PBCFG_0_ENTER_DEFAULTMODE_FROM_RESET/INI+     ----- -----  ----- -----  ----- -----  ----- -----
... TDEVICE

ADC_0_ENTER_DEFAULTMODE_FROM_RESET/INITD+     ----- -----  ----- -----  ----- -----  ----- -----
... EVICE

HFOSC_0_ENTER_DEFAULTMODE_FROM_RESET/INI+     ----- -----  ----- -----  ----- -----  ----- -----
... TDEVICE

CLOCK_0_ENTER_DEFAULTMODE_FROM_RESET/INI+     ----- -----  ----- -----  ----- -----  ----- -----
... TDEVICE

TIMER01_0_ENTER_DEFAULTMODE_FROM_RESET/I+     ----- -----  ----- -----  ----- -----  ----- -----
... NITDEVICE

TIMER16_2_ENTER_DEFAULTMODE_FROM_RESET/I+     ----- -----  ----- -----  ----- -----  ----- -----
... NITDEVICE

TIMER16_5_ENTER_DEFAULTMODE_FROM_RESET/I+     ----- -----  ----- -----  ----- -----  ----- -----
... NITDEVICE

TIMER_SETUP_0_ENTER_DEFAULTMODE_FROM_RES+     ----- -----  ----- -----  ----- -----  ----- -----
... ET/INITDEVICE

SMBUS_0_ENTER_DEFAULTMODE_FROM_RESET/INI+     ----- -----  ----- -----  ----- -----  ----- -----
... TDEVICE

SMBUS_1_ENTER_DEFAULTMODE_FROM_RESET/INI+     ----- -----  ----- -----  ----- -----  ----- -----
... TDEVICE

SPI_0_ENTER_DEFAULTMODE_FROM_RESET/INITD+     ----- -----  ----- -----  ----- -----  ----- -----
... EVICE

UART_0_ENTER_DEFAULTMODE_FROM_RESET/INIT+     ----- -----  ----- -----  ----- -----  ----- -----
... DEVICE

EXTINT_0_ENTER_DEFAULTMODE_FROM_RESET/IN+     ----- -----  ----- -----  ----- -----  ----- -----
... ITDEVICE

INTERRUPT_0_ENTER_DEFAULTMODE_FROM_RESET+     ----- -----  ----- -----  ----- -----  ----- -----
... /INITDEVICE

FW_INIT/FW                                    ----- -----  ----- -----  ----- -----  ----- -----
  +--> ADXL345_INIT/ADXL
  +--> ADXL345_TICK/ADXL
  +--> _RAND16_INIT/RAND16
  +--> HWID_INIT/EFM8UB2_HWID
  +--> BTN_INIT/BTN
  +--> UCONF_LOAD/USER_CONFIG
  +--> SMB1_STOP/EFM8_SMB1
  +--> _SSD1306FB_SET_TARGET/DRAW_SSD1306
  +--> _SSD1306_INIT/OLED_SSD1306
  +--> _LSENS_PULSE/LIGHTLEVEL
  +--> _MENU_STOP/MENU

ADXL345_INIT/ADXL                             ----- -----  ----- -----  ----- -----  ----- -----
  +--> _SPI0_XFER/EFM8_SPI

_SPI0_XFER/EFM8_SPI                           ----- -----  0046H 004CH  ----- -----  ----- -----
LX51 LINKER/LOCATER V4.66.30.0                                                        07/27/2019  23:22:19  PAGE 10


  +--> _SPI0_XFER_BYTE/EFM8_SPI

_SPI0_XFER_BYTE/EFM8_SPI                      ----- -----  ----- -----  ----- -----  ----- -----

ADXL345_TICK/ADXL                             ----- -----  ----- -----  ----- -----  ----- -----
  +--> _ADXL345_GET_AXES/ADXL

_ADXL345_GET_AXES/ADXL                        ----- -----  0043H 0045H  ----- -----  ----- -----
  +--> _SPI0_XFER/EFM8_SPI

_RAND16_INIT/RAND16                           ----- -----  ----- -----  ----- -----  ----- -----
  +--> RAND16/RAND16

RAND16/RAND16                                 ----- -----  ----- -----  ----- -----  ----- -----

HWID_INIT/EFM8UB2_HWID                        ----- -----  ----- -----  ----- -----  ----- -----

BTN_INIT/BTN                                  ----- -----  ----- -----  ----- -----  ----- -----

UCONF_LOAD/USER_CONFIG                        ----- -----  0022H 0027H  ----- -----  ----- -----
  +--> _USERFLASH_RESERVE_PAGES/EFM8UB2_USERFLASH
  +--> _UCONF_VALIDATE/USER_CONFIG
  +--> _USERFLASH_READ/EFM8UB2_USERFLASH
  +--> UCONF_DEFAULTS/USER_CONFIG

_USERFLASH_RESERVE_PAGES/EFM8UB2_USERFLA+     ----- -----  0028H 0028H  ----- -----  ----- -----
... SH
  +--> USERFLASH_INIT/EFM8UB2_USERFLASH

USERFLASH_INIT/EFM8UB2_USERFLASH              ----- -----  ----- -----  ----- -----  ----- -----
  +--> HWID_GET_MODEL/EFM8UB2_HWID

HWID_GET_MODEL/EFM8UB2_HWID                   ----- -----  0029H 002AH  ----- -----  ----- -----

_UCONF_VALIDATE/USER_CONFIG                   ----- -----  0028H 002AH  ----- -----  ----- -----
  +--> USERFLASH_GET_BASEADDR/EFM8UB2_USERFLASH
  +--> _CHECKSUM_GEN/CHECKSUM

USERFLASH_GET_BASEADDR/EFM8UB2_USERFLASH      ----- -----  ----- -----  ----- -----  ----- -----

_CHECKSUM_GEN/CHECKSUM                        ----- -----  002BH 002DH  ----- -----  ----- -----

_USERFLASH_READ/EFM8UB2_USERFLASH             ----- -----  0028H 0029H  ----- -----  ----- -----

UCONF_DEFAULTS/USER_CONFIG                    ----- -----  ----- -----  ----- -----  ----- -----
  +--> ?CO?USER_CONFIG
  +--> _CHECKSUM_GEN/CHECKSUM

?CO?USER_CONFIG                               ----- -----  ----- -----  ----- -----  ----- -----

SMB1_STOP/EFM8_SMB1                           ----- -----  ----- -----  ----- -----  ----- -----

_SSD1306FB_SET_TARGET/DRAW_SSD1306            ----- -----  ----- -----  ----- -----  ----- -----

_SSD1306_INIT/OLED_SSD1306                    ----- -----  0022H 0022H  ----- -----  ----- -----
  +--> _SSD1306_SET_DISPLAY/OLED_SSD1306
  +--> _SSD1306_CB/OLED_SSD1306
  +--> ?CO?OLED_SSD1306
  +--> _SMB1_MWRITE/EFM8_SMB1
  +--> SSD1306_INIT_STEP2/OLED_SSD1306
  +--> SSD1306_INIT_STEP3/OLED_SSD1306

LX51 LINKER/LOCATER V4.66.30.0                                                        07/27/2019  23:22:19  PAGE 11


_SSD1306_SET_DISPLAY/OLED_SSD1306             ----- -----  ----- -----  ----- -----  ----- -----
  +--> _SMB1_MWRITE/EFM8_SMB1
  +--> SSD1306_IDLE_WAIT/OLED_SSD1306

_SMB1_MWRITE/EFM8_SMB1                        ----- -----  002EH 0036H  ----- -----  ----- -----

SSD1306_IDLE_WAIT/OLED_SSD1306                ----- -----  002EH 002FH  ----- -----  ----- -----
  +--> SMB1_GET_STATE/EFM8_SMB1

SMB1_GET_STATE/EFM8_SMB1                      ----- -----  ----- -----  ----- -----  ----- -----

_SSD1306_CB/OLED_SSD1306                      ----- -----  ----- -----  ----- -----  ----- -----

?CO?OLED_SSD1306                              ----- -----  ----- -----  ----- -----  ----- -----

SSD1306_INIT_STEP2/OLED_SSD1306               ----- -----  ----- -----  ----- -----  ----- -----
  +--> _SSD1306_CLS/OLED_SSD1306
  +--> SSD1306_UPDATE/OLED_SSD1306
  +--> SSD1306_INIT_STEP3/OLED_SSD1306

_SSD1306_CLS/OLED_SSD1306                     ----- -----  002AH 002BH  ----- -----  ----- -----

SSD1306_UPDATE/OLED_SSD1306                   ----- -----  ----- -----  ----- -----  ----- -----
  +--> ?CO?OLED_SSD1306
  +--> _SMB1_MWRITE/EFM8_SMB1
  +--> SSD1306_IDLE_WAIT/OLED_SSD1306
  +--> _SSD1306_CB/OLED_SSD1306

SSD1306_INIT_STEP3/OLED_SSD1306               ----- -----  ----- -----  ----- -----  ----- -----
  +--> _SSD1306_SET_DISPLAY/OLED_SSD1306

_LSENS_PULSE/LIGHTLEVEL                       ----- -----  ----- -----  ----- -----  ----- -----

_MENU_STOP/MENU                               ----- -----  ----- -----  ----- -----  ----- -----
  +--> ?CO?MENU_DEF
  +--> MENU_BTN_USE_NONE/MENU

?CO?MENU_DEF                                  ----- -----  ----- -----  ----- -----  ----- -----
  +--> _MENU_NONE_DISP/MENU_0_FN
  +--> _MENU_START/MENU
  +--> _MENU_0_DISP/MENU_0_FN
  +--> _MENU_0_ENTER/MENU_0_FN
  +--> _MENU_1_DISP/MENU_1_FN
  +--> _MENU_1_ENTER/MENU_1_FN
  +--> _MENU_2_DISP/MENU_2_FN
  +--> _MENU_2_ENTER/MENU_2_FN
  +--> _MENU_5_DISP/MENU_5_FN
  +--> _MENU_5_ENTER/MENU_5_FN
  +--> _MENU_6_DISP/MENU_6_FN

_MENU_NONE_DISP/MENU_0_FN                     ----- -----  0022H 0029H  ----- -----  0413H 0414H
  +--> MENU_NONE_INIT/MENU_0_FN
  +--> _MENU_NONE_SET_HALFWIDTH/MENU_0_FN
  +--> _SSD1306FB_SET_TARGET/DRAW_SSD1306
  +--> ?CO?FONT_TABLE
  +--> _STRLEN/STRLEN
  +--> _SSD1306FB_GET_STR_WIDTH/DRAW_SSD1306
  +--> ?CO?MENU_0_FN
  +--> _MENU_NONE_PRINT_ERROR/MENU_0_FN
  +--> _SSD1306FB_GET_FONT_HEIGHT/DRAW_SSD1306
  +--> _ADXL345_GET_ROTATION/ADXL
  +--> _MENU_NONE_SET_FLIPMIRROR/MENU_0_FN
LX51 LINKER/LOCATER V4.66.30.0                                                        07/27/2019  23:22:19  PAGE 12


  +--> _SSD1306FB_SET_CURSOR/DRAW_SSD1306
  +--> _SSD1306FB_DRAW_STR/DRAW_SSD1306
  +--> _COS7/SIN7
  +--> _SSD1306_SET_FLIPMIRROR/OLED_SSD1306
  +--> _SSD1306FB_SET_COLOR/DRAW_SSD1306
  +--> _SSD1306_CLS/OLED_SSD1306
  +--> _SSD1306FB_ROTATE/DRAW_SSD1306
  +--> _SSD1306FB_COPY/DRAW_SSD1306
  +--> PRINTF/PRINTF
  +--> ?CO?FONT

MENU_NONE_INIT/MENU_0_FN                      ----- -----  ----- -----  ----- -----  ----- -----

_MENU_NONE_SET_HALFWIDTH/MENU_0_FN            ----- -----  ----- -----  ----- -----  ----- -----

?CO?FONT_TABLE                                ----- -----  ----- -----  ----- -----  ----- -----
  +--> ?CO?FONT

?CO?FONT                                      ----- -----  ----- -----  ----- -----  ----- -----

_STRLEN/STRLEN                                ----- -----  ----- -----  ----- -----  ----- -----

_SSD1306FB_GET_STR_WIDTH/DRAW_SSD1306         ----- -----  002AH 0034H  ----- -----  ----- -----

?CO?MENU_0_FN                                 ----- -----  ----- -----  ----- -----  ----- -----

_MENU_NONE_PRINT_ERROR/MENU_0_FN              ----- -----  002AH 0032H  ----- -----  ----- -----
  +--> _SSD1306FB_SET_CURSOR/DRAW_SSD1306
  +--> ?CO?FONT
  +--> _SSD1306FB_DRAW_STR/DRAW_SSD1306

_SSD1306FB_SET_CURSOR/DRAW_SSD1306            ----- -----  ----- -----  ----- -----  ----- -----

_SSD1306FB_DRAW_STR/DRAW_SSD1306              ----- -----  0033H 0039H  ----- -----  ----- -----
  +--> _STRLEN/STRLEN
  +--> _SSD1306FB_INTERNAL_STR/DRAW_SSD1306

_SSD1306FB_INTERNAL_STR/DRAW_SSD1306          ----- -----  003AH 003DH  0000H 000EH  ----- -----
  +--> _SSD1306FB_DRAW_RAW/DRAW_SSD1306

_SSD1306FB_DRAW_RAW/DRAW_SSD1306              ----- -----  003EH 0042H  000FH 0022H  ----- -----

_SSD1306FB_GET_FONT_HEIGHT/DRAW_SSD1306       ----- -----  ----- -----  ----- -----  ----- -----

_ADXL345_GET_ROTATION/ADXL                    ----- -----  ----- -----  ----- -----  ----- -----
  +--> _I8ATAN2/I8ATAN2

_I8ATAN2/I8ATAN2                              ----- -----  002AH 002AH  ----- -----  ----- -----
  +--> _IAT2/I8ATAN2

_IAT2/I8ATAN2                                 ----- -----  ----- -----  ----- -----  ----- -----

_MENU_NONE_SET_FLIPMIRROR/MENU_0_FN           ----- -----  ----- -----  ----- -----  ----- -----
  +--> _SSD1306_SET_FLIPMIRROR/OLED_SSD1306

_SSD1306_SET_FLIPMIRROR/OLED_SSD1306          ----- -----  002AH 002CH  ----- -----  ----- -----
  +--> _SSD1306_SET_FLIP/OLED_SSD1306
  +--> _SSD1306_SET_MIRROR/OLED_SSD1306

_SSD1306_SET_FLIP/OLED_SSD1306                ----- -----  002DH 002DH  ----- -----  ----- -----
  +--> _SMB1_MWRITE/EFM8_SMB1
  +--> SSD1306_IDLE_WAIT/OLED_SSD1306
LX51 LINKER/LOCATER V4.66.30.0                                                        07/27/2019  23:22:19  PAGE 13



_SSD1306_SET_MIRROR/OLED_SSD1306              ----- -----  002DH 002DH  ----- -----  ----- -----
  +--> _SMB1_MWRITE/EFM8_SMB1
  +--> SSD1306_IDLE_WAIT/OLED_SSD1306

_COS7/SIN7                                    ----- -----  ----- -----  ----- -----  ----- -----
  +--> _SIN7/SIN7

_SIN7/SIN7                                    ----- -----  ----- -----  ----- -----  ----- -----
  +--> ?CO?SIN7

?CO?SIN7                                      ----- -----  ----- -----  ----- -----  ----- -----

_SSD1306FB_SET_COLOR/DRAW_SSD1306             ----- -----  ----- -----  ----- -----  ----- -----

_SSD1306FB_ROTATE/DRAW_SSD1306                ----- -----  002AH 0040H  ----- -----  ----- -----
  +--> _SIN7/SIN7
  +--> _COS7/SIN7

_SSD1306FB_COPY/DRAW_SSD1306                  ----- -----  002AH 002FH  0000H 000FH  ----- -----

PRINTF/PRINTF                                 20H.0 21H.0  002AH 003DH  ----- -----  ----- -----
  +--> PUTCHAR/PUTCHAR

PUTCHAR/PUTCHAR                               ----- -----  ----- -----  ----- -----  ----- -----

_MENU_START/MENU                              ----- -----  ----- -----  ----- -----  ----- -----
  +--> ?CO?MENU_DEF
  +--> MENU_BTN_USE_STD/MENU

MENU_BTN_USE_STD/MENU                         ----- -----  ----- -----  ----- -----  ----- -----
  +--> MENU_BTN_NEXT/MENU
  +--> MENU_BTN_EXIT/MENU
  +--> MENU_BTN_ENTER/MENU
  +--> MENU_BTN_PREV/MENU

MENU_BTN_NEXT/MENU                            ----- -----  ----- -----  ----- -----  ----- -----

MENU_BTN_EXIT/MENU                            ----- -----  ----- -----  ----- -----  ----- -----
  +--> UCONF_WRITE/USER_CONFIG

UCONF_WRITE/USER_CONFIG                       ----- -----  0026H 0028H  ----- -----  ----- -----
  +--> USERFLASH_GET_BASEADDR/EFM8UB2_USERFLASH
  +--> _USERFLASH_ERASE_PAGE/EFM8UB2_USERFLASH
  +--> _CHECKSUM_GEN/CHECKSUM
  +--> _USERFLASH_WRITE/EFM8UB2_USERFLASH

_USERFLASH_ERASE_PAGE/EFM8UB2_USERFLASH       ----- -----  ----- -----  ----- -----  ----- -----
  +--> _USERFLASH_WRITE_BYTE/EFM8UB2_USERFLASH

_USERFLASH_WRITE_BYTE/EFM8UB2_USERFLASH       20H.0 20H.0  ----- -----  ----- -----  ----- -----

_USERFLASH_WRITE/EFM8UB2_USERFLASH            ----- -----  0029H 002CH  ----- -----  ----- -----
  +--> _USERFLASH_WRITE_BYTE/EFM8UB2_USERFLASH

MENU_BTN_ENTER/MENU                           ----- -----  ----- -----  ----- -----  ----- -----

MENU_BTN_PREV/MENU                            ----- -----  ----- -----  ----- -----  ----- -----

_MENU_0_DISP/MENU_0_FN                        ----- -----  0022H 0023H  ----- -----  0413H 041EH
  +--> _SSD1306FB_SET_COLOR/DRAW_SSD1306
  +--> _SSD1306FB_DRAW_CIRCLE/DRAW_SSD1306
LX51 LINKER/LOCATER V4.66.30.0                                                        07/27/2019  23:22:19  PAGE 14


  +--> _SSD1306FB_SET_CURSOR/DRAW_SSD1306
  +--> ?CO?MENU_0_FN
  +--> ?CO?FONT
  +--> _SSD1306FB_DRAW_STR/DRAW_SSD1306
  +--> _STRLEN/STRLEN
  +--> _SSD1306FB_GET_STR_WIDTH/DRAW_SSD1306
  +--> _SSD1306FB_DRAW_HLINE/DRAW_SSD1306
  +--> _MENU_DRAW_TABS/MENU
  +--> _MENU_DRAW_BUTTONS/MENU

_SSD1306FB_DRAW_CIRCLE/DRAW_SSD1306           ----- -----  0025H 0029H  ----- -----  ----- -----
  +--> _SSD1306FB_DRAW_PIX/DRAW_SSD1306

_SSD1306FB_DRAW_PIX/DRAW_SSD1306              ----- -----  002FH 0032H  ----- -----  ----- -----

_SSD1306FB_DRAW_HLINE/DRAW_SSD1306            ----- -----  002DH 0031H  ----- -----  ----- -----

_MENU_DRAW_TABS/MENU                          ----- -----  0026H 002CH  ----- -----  ----- -----
  +--> _SSD1306FB_DRAW_HLINE/DRAW_SSD1306
  +--> _SSD1306FB_DRAW_VLINE/DRAW_SSD1306

_SSD1306FB_DRAW_VLINE/DRAW_SSD1306            ----- -----  002DH 0034H  ----- -----  ----- -----

_MENU_DRAW_BUTTONS/MENU                       ----- -----  0026H 0029H  ----- -----  0423H 0452H
  +--> ?CO?MENU
  +--> _SSD1306FB_SET_CURSOR/DRAW_SSD1306
  +--> ?CO?FONT
  +--> _SSD1306FB_DRAW_STR/DRAW_SSD1306
  +--> _STRLEN/STRLEN
  +--> _SSD1306FB_GET_STR_WIDTH/DRAW_SSD1306
  +--> _SSD1306FB_DRAW_HLINE/DRAW_SSD1306

?CO?MENU                                      ----- -----  ----- -----  ----- -----  ----- -----

_MENU_0_ENTER/MENU_0_FN                       ----- -----  ----- -----  ----- -----  ----- -----
  +--> _MENU_STOP/MENU
  +--> ?CO?MENU_DEF

_MENU_1_DISP/MENU_1_FN                        ----- -----  0022H 0024H  ----- -----  0413H 0422H
  +--> MENU_1_BTN_USE/MENU_1_FN
  +--> MENU_1_NAME_EDIT/MENU_1_FN
  +--> _SSD1306FB_SET_CURSOR/DRAW_SSD1306
  +--> ?CO?FONT_TABLE
  +--> ?CO?MENU_1_FN
  +--> _SSD1306FB_DRAW_STR/DRAW_SSD1306
  +--> _SSD1306FB_GET_FONT_HEIGHT/DRAW_SSD1306
  +--> PRINTF/PRINTF
  +--> _STRLEN/STRLEN
  +--> _SSD1306FB_GET_STR_WIDTH/DRAW_SSD1306
  +--> _SSD1306FB_DRAW_RECT/DRAW_SSD1306
  +--> _MENU_DRAW_TABS/MENU
  +--> _MENU_DRAW_BUTTONS/MENU

MENU_1_BTN_USE/MENU_1_FN                      ----- -----  ----- -----  ----- -----  ----- -----
  +--> MENU_1_BTN_PREV/MENU_1_FN
  +--> MENU_1_BTN_EXIT/MENU_1_FN
  +--> MENU_1_BTN_ENTER/MENU_1_FN
  +--> MENU_1_BTN_NEXT/MENU_1_FN

MENU_1_BTN_PREV/MENU_1_FN                     ----- -----  0025H 0026H  ----- -----  ----- -----
  +--> _STRLEN/STRLEN
  +--> ?CO?FONT_TABLE
LX51 LINKER/LOCATER V4.66.30.0                                                        07/27/2019  23:22:19  PAGE 15



MENU_1_BTN_EXIT/MENU_1_FN                     ----- -----  0025H 0025H  ----- -----  ----- -----
  +--> MENU_BTN_USE_STD/MENU
  +--> _STRLEN/STRLEN

MENU_1_BTN_ENTER/MENU_1_FN                    ----- -----  ----- -----  ----- -----  ----- -----

MENU_1_BTN_NEXT/MENU_1_FN                     ----- -----  0025H 0026H  ----- -----  ----- -----
  +--> _STRLEN/STRLEN
  +--> ?CO?FONT_TABLE

MENU_1_NAME_EDIT/MENU_1_FN                    ----- -----  ----- -----  ----- -----  0423H 042CH
  +--> _SSD1306FB_SET_CURSOR/DRAW_SSD1306
  +--> ?CO?FONT_TABLE
  +--> _SSD1306FB_DRAW_STR/DRAW_SSD1306
  +--> _SSD1306FB_DRAW_CIRCLE/DRAW_SSD1306
  +--> _SSD1306FB_DRAW_HLINE/DRAW_SSD1306
  +--> _STRLEN/STRLEN
  +--> ?CO?MENU_1_FN
  +--> PRINTF/PRINTF
  +--> _SSD1306FB_GET_STR_WIDTH/DRAW_SSD1306

?CO?MENU_1_FN                                 ----- -----  ----- -----  ----- -----  ----- -----

_SSD1306FB_DRAW_RECT/DRAW_SSD1306             ----- -----  0026H 0029H  ----- -----  ----- -----
  +--> _SSD1306FB_DRAW_VLINE/DRAW_SSD1306
  +--> _SSD1306FB_DRAW_HLINE/DRAW_SSD1306

_MENU_1_ENTER/MENU_1_FN                       ----- -----  ----- -----  ----- -----  ----- -----
  +--> MENU_1_FONT_NEXT/MENU_1_FN

MENU_1_FONT_NEXT/MENU_1_FN                    ----- -----  ----- -----  ----- -----  ----- -----
  +--> ?CO?FONT_TABLE

_MENU_2_DISP/MENU_2_FN                        ----- -----  0022H 0025H  ----- -----  0413H 041EH
  +--> _MENU_2_BTN_USE/MENU_2_FN
  +--> _SSD1306FB_SET_CURSOR/DRAW_SSD1306
  +--> ?CO?FONT_TABLE
  +--> ?CO?MENU_2_FN
  +--> _SSD1306FB_DRAW_STR/DRAW_SSD1306
  +--> ?CO?RGBLED_PROG
  +--> PRINTF/PRINTF
  +--> _SSD1306FB_DRAW_VLINE/DRAW_SSD1306
  +--> _SSD1306FB_DRAW_HLINE/DRAW_SSD1306
  +--> _SSD1306FB_DRAW_LINE/DRAW_SSD1306
  +--> _STRLEN/STRLEN
  +--> _SSD1306FB_GET_STR_WIDTH/DRAW_SSD1306
  +--> _SSD1306FB_DRAW_RECT/DRAW_SSD1306
  +--> _MENU_DRAW_TABS/MENU
  +--> _MENU_DRAW_BUTTONS/MENU

_MENU_2_BTN_USE/MENU_2_FN                     ----- -----  ----- -----  ----- -----  ----- -----
  +--> MENU_2_BTN_PREV/MENU_2_FN
  +--> MENU_2_BTN_EXIT/MENU_2_FN
  +--> MENU_2_BTN_NEXT/MENU_2_FN

MENU_2_BTN_PREV/MENU_2_FN                     ----- -----  ----- -----  ----- -----  ----- -----
  +--> _MENU_2_VAL_DEC/MENU_2_FN

_MENU_2_VAL_DEC/MENU_2_FN                     ----- -----  ----- -----  ----- -----  ----- -----

MENU_2_BTN_EXIT/MENU_2_FN                     ----- -----  ----- -----  ----- -----  ----- -----
LX51 LINKER/LOCATER V4.66.30.0                                                        07/27/2019  23:22:19  PAGE 16


  +--> MENU_BTN_USE_STD/MENU

MENU_2_BTN_NEXT/MENU_2_FN                     ----- -----  ----- -----  ----- -----  ----- -----
  +--> _MENU_2_VAL_INC/MENU_2_FN

_MENU_2_VAL_INC/MENU_2_FN                     ----- -----  ----- -----  ----- -----  ----- -----

?CO?MENU_2_FN                                 ----- -----  ----- -----  ----- -----  ----- -----

?CO?RGBLED_PROG                               ----- -----  ----- -----  ----- -----  ----- -----
  +--> _LEDPROG_SOLID/RGBLED_PROG
  +--> _LEDPROG_SOLID_EDIT/RGBLED_PROG
  +--> _LEDPROG_FLICKER/RGBLED_PROG
  +--> _LEDPROG_CIRCLER/RGBLED_PROG
  +--> _LEDPROG_RANDOM/RGBLED_PROG
  +--> _LEDPROG_RANDOMCOLOR/RGBLED_PROG
  +--> _LEDPROG_CCROSS/RGBLED_PROG
  +--> _LEDPROG_CFLIP/RGBLED_PROG
  +--> _LEDPROG_CMIRROR/RGBLED_PROG
  +--> _LEDPROG_CALT/RGBLED_PROG
  +--> _LEDPROG_PFADE1/RGBLED_PROG
  +--> _LEDPROG_RAINBOW/RGBLED_PROG

_LEDPROG_SOLID/RGBLED_PROG                    ----- -----  0043H 0047H  ----- -----  ----- -----

_LEDPROG_SOLID_EDIT/RGBLED_PROG               ----- -----  ----- -----  ----- -----  ----- -----

_LEDPROG_FLICKER/RGBLED_PROG                  ----- -----  0043H 0049H  ----- -----  ----- -----
  +--> RAND16/RAND16

_LEDPROG_CIRCLER/RGBLED_PROG                  ----- -----  0043H 0044H  ----- -----  ----- -----

_LEDPROG_RANDOM/RGBLED_PROG                   ----- -----  0043H 0049H  ----- -----  ----- -----
  +--> RAND16/RAND16

_LEDPROG_RANDOMCOLOR/RGBLED_PROG              ----- -----  0043H 0049H  ----- -----  ----- -----
  +--> RAND16/RAND16

_LEDPROG_CCROSS/RGBLED_PROG                   ----- -----  0043H 0045H  ----- -----  ----- -----

_LEDPROG_CFLIP/RGBLED_PROG                    ----- -----  0043H 0045H  ----- -----  ----- -----

_LEDPROG_CMIRROR/RGBLED_PROG                  ----- -----  0043H 0045H  ----- -----  ----- -----

_LEDPROG_CALT/RGBLED_PROG                     ----- -----  0043H 0045H  ----- -----  ----- -----

_LEDPROG_PFADE1/RGBLED_PROG                   ----- -----  0043H 0048H  ----- -----  ----- -----

_LEDPROG_RAINBOW/RGBLED_PROG                  ----- -----  0043H 0045H  ----- -----  ----- -----

_SSD1306FB_DRAW_LINE/DRAW_SSD1306             ----- -----  0026H 002EH  ----- -----  ----- -----
  +--> _ABS/ABS
  +--> _SSD1306FB_DRAW_PIX/DRAW_SSD1306

_ABS/ABS                                      ----- -----  ----- -----  ----- -----  ----- -----

_MENU_2_ENTER/MENU_2_FN                       ----- -----  0022H 0022H  ----- -----  ----- -----
  +--> MENU_BTN_USE_STD/MENU

_MENU_5_DISP/MENU_5_FN                        ----- -----  0022H 0024H  ----- -----  0413H 041EH
  +--> _SSD1306FB_SET_CURSOR/DRAW_SSD1306
  +--> ?CO?FONT_TABLE
LX51 LINKER/LOCATER V4.66.30.0                                                        07/27/2019  23:22:19  PAGE 17


  +--> ?CO?MENU_5_FN
  +--> _SSD1306FB_DRAW_STR/DRAW_SSD1306
  +--> _STRLEN/STRLEN
  +--> _SSD1306FB_GET_STR_WIDTH/DRAW_SSD1306
  +--> _SSD1306FB_DRAW_RECT/DRAW_SSD1306
  +--> _MENU_DRAW_TABS/MENU
  +--> _MENU_DRAW_BUTTONS/MENU

?CO?MENU_5_FN                                 ----- -----  ----- -----  ----- -----  ----- -----

_MENU_5_ENTER/MENU_5_FN                       ----- -----  ----- -----  ----- -----  ----- -----

_MENU_6_DISP/MENU_6_FN                        ----- -----  0022H 0023H  ----- -----  0413H 041EH
  +--> _SSD1306FB_SET_CURSOR/DRAW_SSD1306
  +--> ?CO?FONT
  +--> ?CO?MENU_6_FN
  +--> _SSD1306FB_DRAW_STR/DRAW_SSD1306
  +--> ?CO?FW
  +--> PRINTF/PRINTF
  +--> _SSD1306FB_DRAW_LINE/DRAW_SSD1306
  +--> _SSD1306FB_SET_COLOR/DRAW_SSD1306
  +--> _SSD1306FB_DRAW_CIRCLE/DRAW_SSD1306
  +--> HWID_GET_MODEL/EFM8UB2_HWID
  +--> _SSD1306FB_DRAW_RECT/DRAW_SSD1306
  +--> ?CO?FONT_TABLE
  +--> _MENU_DRAW_TABS/MENU
  +--> MENU_BTN_USE_STD/MENU
  +--> MENU_6_BTN_USE/MENU_6_FN
  +--> _MENU_DRAW_BUTTONS/MENU

?CO?MENU_6_FN                                 ----- -----  ----- -----  ----- -----  ----- -----

?CO?FW                                        ----- -----  ----- -----  ----- -----  ----- -----

MENU_6_BTN_USE/MENU_6_FN                      ----- -----  ----- -----  ----- -----  ----- -----
  +--> MENU_6_FONT_PREV/MENU_6_FN
  +--> MENU_6_FONT_NEXT/MENU_6_FN

MENU_6_FONT_PREV/MENU_6_FN                    ----- -----  ----- -----  ----- -----  ----- -----
  +--> _MENU_6_FONT_INDEX/MENU_6_FN
  +--> _MENU_6_FONT_GLYPH/MENU_6_FN

_MENU_6_FONT_INDEX/MENU_6_FN                  ----- -----  ----- -----  ----- -----  ----- -----

_MENU_6_FONT_GLYPH/MENU_6_FN                  ----- -----  ----- -----  ----- -----  ----- -----
  +--> ?CO?FONT_TABLE

MENU_6_FONT_NEXT/MENU_6_FN                    ----- -----  ----- -----  ----- -----  ----- -----
  +--> _MENU_6_FONT_INDEX/MENU_6_FN
  +--> _MENU_6_FONT_GLYPH/MENU_6_FN

MENU_BTN_USE_NONE/MENU                        ----- -----  ----- -----  ----- -----  ----- -----
  +--> MENU_BTN_ENTER/MENU

PWR_ENTERIDLE/PWR                             ----- -----  ----- -----  ----- -----  ----- -----

FW_TICK_MAINLOOP/FW                           ----- -----  ----- -----  ----- -----  ----- -----
  +--> _SSD1306_INIT/OLED_SSD1306
  +--> BTN_CALLBACK/BTN
  +--> SSD1306_CB_GET/OLED_SSD1306
  +--> FW_OLED_UPDATE_DONE/FW
  +--> SSD1306_UPDATE/OLED_SSD1306
LX51 LINKER/LOCATER V4.66.30.0                                                        07/27/2019  23:22:19  PAGE 18


  +--> LSENS_TICK/LIGHTLEVEL
  +--> RAND16/RAND16

BTN_CALLBACK/BTN                              ----- -----  0022H 0023H  ----- -----  ----- -----

SSD1306_CB_GET/OLED_SSD1306                   20H.0 20H.0  ----- -----  ----- -----  ----- -----

FW_OLED_UPDATE_DONE/FW                        ----- -----  ----- -----  ----- -----  ----- -----
  +--> _SSD1306_CLS/OLED_SSD1306
  +--> _SSD1306FB_SET_COLOR/DRAW_SSD1306
  +--> _ADXL345_GET_ROTATION/ADXL
  +--> MENU_TICK/MENU

MENU_TICK/MENU                                ----- -----  ----- -----  ----- -----  ----- -----
  +--> ?CO?MENU_DEF
  +--> _SSD1306_SET_FLIPMIRROR/OLED_SSD1306

LSENS_TICK/LIGHTLEVEL                         ----- -----  ----- -----  ----- -----  ----- -----

?C_INITSEG                                    ----- -----  ----- -----  ----- -----  ----- -----

*** NEW ROOT ********************************

INT0_ISR/INTERRUPTS                           ----- -----  ----- -----  ----- -----  ----- -----

*** NEW ROOT ********************************

TIMER5_ISR/INTERRUPTS                         ----- -----  ----- -----  ----- -----  ----- -----
  +--> FW_TICK_CRITICAL/FW

FW_TICK_CRITICAL/FW                           ----- -----  ----- -----  ----- -----  0453H 0460H
  +--> _RGBLED_UPDATE/RGBLED
  +--> ADXL345_TICK/ADXL
  +--> BTN_TICK/BTN
  +--> ?CO?RGBLED_PROG

_RGBLED_UPDATE/RGBLED                         ----- -----  0043H 0048H  ----- -----  ----- -----
  +--> _HSV2RGB_8B/HSV2RGB

_HSV2RGB_8B/HSV2RGB                           ----- -----  0049H 005DH  ----- -----  ----- -----

BTN_TICK/BTN                                  ----- -----  ----- -----  ----- -----  ----- -----
  +--> _BTN_CHECK/BTN

_BTN_CHECK/BTN                                ----- -----  ----- -----  ----- -----  ----- -----

*** NEW ROOT ********************************

SMBUS1_ISR/INTERRUPTS                         ----- -----  ----- -----  ----- -----  ----- -----
  +--> SMB1_INTERRUPT/EFM8_SMB1

SMB1_INTERRUPT/EFM8_SMB1                      ----- -----  005EH 005EH  ----- -----  ----- -----



PUBLIC SYMBOLS OF MODULE:  GAT_NAMETAG.OMF.CRBUILD (?C_STARTUP)


      VALUE       CLASS    TYPE      PUBLIC SYMBOL NAME
      =================================================
*DEL*:00000000H   DATA     BYTE      ?_checksum_verify?BYTE
      00000049H   DATA     BYTE      ?_hsv2rgb_8b?BYTE
LX51 LINKER/LOCATER V4.66.30.0                                                        07/27/2019  23:22:19  PAGE 19


      0000002AH   DATA     ---       ?_PRINTF517?BYTE
      0000002AH   DATA     ---       ?_PRINTF?BYTE
*DEL*:00000000H   DATA     BYTE      ?_smb1_mread?BYTE
      0000002EH   DATA     BYTE      ?_smb1_mwrite?BYTE
      00000046H   DATA     BYTE      ?_spi0_xfer?BYTE
      0000002AH   DATA     ---       ?_SPRINTF517?BYTE
      0000002AH   DATA     ---       ?_SPRINTF?BYTE
      02000000H   PDATA    BYTE      ?_ssd1306fb_copy?BYTE
      00000026H   DATA     BYTE      ?_ssd1306fb_draw_line?BYTE
      0200000FH   PDATA    BYTE      ?_ssd1306fb_draw_raw?BYTE
      00000026H   DATA     BYTE      ?_ssd1306fb_draw_rect?BYTE
*DEL*:00000000H   DATA     BYTE      ?_ssd1306fb_draw_rect_fill?BYTE
      00000033H   DATA     BYTE      ?_ssd1306fb_draw_str?BYTE
      0000002AH   DATA     BYTE      ?_ssd1306fb_get_str_width?BYTE
      02000000H   PDATA    BYTE      ?_ssd1306fb_internal_str?BYTE
      0000002AH   DATA     BYTE      ?_ssd1306fb_rotate?BYTE
      010009B4H   CODE     ---       ?C?CCASE
      01000695H   CODE     ---       ?C?CILDOPTR
      01000673H   CODE     ---       ?C?CILDPTR
      01000646H   CODE     ---       ?C?CLDOPTR
      0100062DH   CODE     ---       ?C?CLDPTR
      00000000H   NUMBER   ---       ?C?CODESEG
      010006DAH   CODE     ---       ?C?CSTOPTR
      010006C8H   CODE     ---       ?C?CSTPTR
      010009DAH   CODE     ---       ?C?ICALL
      010009DEH   CODE     ---       ?C?ICALL2
      01000799H   CODE     ---       ?C?IILDX
      010007DAH   CODE     ---       ?C?ILDOPTR
      010007AFH   CODE     ---       ?C?ILDPTR
      010006FCH   CODE     ---       ?C?IMUL
      01000831H   CODE     ---       ?C?ISTOPTR
      01000812H   CODE     ---       ?C?ISTPTR
      01000950H   CODE     ---       ?C?LLDXDATA
      0100095CH   CODE     ---       ?C?LSTXDATA
      01000AC9H   CODE     ---       ?C?MEMSET
      01000968H   CODE     ---       ?C?OFFXADD
      010009A8H   CODE     ---       ?C?PLDCODE
      01000974H   CODE     ---       ?C?PLDIIDATA
      01000996H   CODE     ---       ?C?PLDPDATA
      01000984H   CODE     ---       ?C?PLDXDATA
      0100099FH   CODE     ---       ?C?PSTPDATA
      0100098DH   CODE     ---       ?C?PSTXDATA
      01000763H   CODE     ---       ?C?SIDIV
      01000AACH   CODE     ---       ?C?STRCPY
      0100070EH   CODE     ---       ?C?UIDIV
      0100092CH   CODE     ---       ?C?ULCMP
      0100089AH   CODE     ---       ?C?ULDIV
      0100093DH   CODE     ---       ?C?ULSHR
      00000000H   NUMBER   ---       ?C?XDATASEG
      010047F7H   CODE     ---       ?C_START
      01000000H   CODE     NEAR LAB  ?C_STARTUP
      01005AD9H   CODE     ---       _ABS
      01004B4BH   CODE     ---       _adxl345_get_axes
      010057E7H   CODE     ---       _adxl345_get_rotation
*DEL*:00000000H   CODE     ---       _adxl345_set_interrupt
      010058BEH   CODE     ---       _checksum_gen
*DEL*:00000000H   CODE     ---       _checksum_verify
      0100594FH   CODE     ---       _cos7
      01002B5AH   CODE     ---       _hsv2rgb_8b
*DEL*:00000000H   CODE     ---       _hwid_get_byte
      01003BD6H   CODE     ---       _i8atan2
      0100429BH   CODE     ---       _ledprog_calt
LX51 LINKER/LOCATER V4.66.30.0                                                        07/27/2019  23:22:19  PAGE 20


      01000006H   CODE     ---       _ledprog_ccross
      01003FC1H   CODE     ---       _ledprog_cflip
      0100471DH   CODE     ---       _ledprog_circler
      01003F00H   CODE     ---       _ledprog_cmirror
      010033B9H   CODE     ---       _ledprog_flicker
*DEL*:00000000H   CODE     ---       _ledprog_none
      01003193H   CODE     ---       _ledprog_pfade1
      01003793H   CODE     ---       _ledprog_rainbow
      01004132H   CODE     ---       _ledprog_random
      010035B6H   CODE     ---       _ledprog_randomcolor
      0100407AH   CODE     ---       _ledprog_solid
      01005BB2H   CODE     ---       _ledprog_solid_edit
      01005866H   CODE     ---       _lsens_pulse
      010034BDH   CODE     ---       _menu_0_disp
      0100553AH   CODE     ---       _menu_0_enter
      01001B7CH   CODE     ---       _menu_1_disp
      010041EAH   CODE     ---       _menu_1_enter
      010043F9H   CODE     ---       _menu_2_btn_use
      01001515H   CODE     ---       _menu_2_disp
      01004F73H   CODE     ---       _menu_2_enter
      01002F4FH   CODE     ---       _menu_5_disp
      01005317H   CODE     ---       _menu_5_enter
      010000A6H   CODE     ---       _menu_6_disp
      01005573H   CODE     ---       _menu_6_font_glyph
      010058DBH   CODE     ---       _menu_6_font_index
      01001E7AH   CODE     ---       _menu_draw_buttons
      01004A51H   CODE     ---       _menu_draw_tabs
      01000AF5H   CODE     ---       _menu_none_disp
      01005A13H   CODE     ---       _menu_start
      01005B5BH   CODE     ---       _menu_stop
      0100121BH   CODE     ---       _PRINTF
      0100121BH   CODE     ---       _PRINTF517
      01005752H   CODE     ---       _PUTCHAR
      01005ACCH   CODE     NEAR LAB  _rand16_init
      01002E07H   CODE     ---       _rgbled_update
      0100548EH   CODE     ---       _sin7
*DEL*:00000000H   CODE     ---       _smb1_mread
      01005779H   CODE     ---       _smb1_mwrite
      010052D1H   CODE     ---       _spi0_xfer
      01005ABFH   CODE     ---       _spi0_xfer_byte
      01001215H   CODE     ---       _SPRINTF
      01001215H   CODE     ---       _SPRINTF517
      01005B64H   CODE     ---       _ssd1306_cb
      010051A8H   CODE     ---       _ssd1306_cls
*DEL*:00000000H   CODE     ---       _ssd1306_cmd
      01004E04H   CODE     ---       _ssd1306_init
*DEL*:00000000H   CODE     ---       _ssd1306_set_contrast
      01005417H   CODE     ---       _ssd1306_set_display
      01004FCDH   CODE     ---       _ssd1306_set_flip
      01005A6AH   CODE     ---       _ssd1306_set_flipmirror
*DEL*:00000000H   CODE     ---       _ssd1306_set_invert
      0100501DH   CODE     ---       _ssd1306_set_mirror
      0100185BH   CODE     ---       _ssd1306fb_copy
      01003A2DH   CODE     ---       _ssd1306fb_draw_circle
      010036A5H   CODE     ---       _ssd1306fb_draw_hline
      01003E39H   CODE     ---       _ssd1306fb_draw_line
      010045F8H   CODE     ---       _ssd1306fb_draw_pix
      01000E5BH   CODE     ---       _ssd1306fb_draw_raw
      01005647H   CODE     ---       _ssd1306fb_draw_rect
*DEL*:00000000H   CODE     ---       _ssd1306fb_draw_rect_fill
      010056D1H   CODE     ---       _ssd1306fb_draw_str
      01002524H   CODE     ---       _ssd1306fb_draw_vline
LX51 LINKER/LOCATER V4.66.30.0                                                        07/27/2019  23:22:19  PAGE 21


      01005B52H   CODE     ---       _ssd1306fb_get_font_height
      01004950H   CODE     ---       _ssd1306fb_get_str_width
      01002368H   CODE     ---       _ssd1306fb_internal_str
      01002155H   CODE     ---       _ssd1306fb_rotate
      01005828H   CODE     ---       _ssd1306fb_set_color
      0100598EH   CODE     ---       _ssd1306fb_set_cursor
      01005B7BH   CODE     ---       _ssd1306fb_set_target
      01005979H   CODE     ---       _STRLEN
      01005B6CH   CODE     ---       _userflash_erase_page
      010056FCH   CODE     ---       _userflash_read
      010058A1H   CODE     ---       _userflash_reserve_pages
      01005616H   CODE     ---       _userflash_write
      01005808H   CODE     ---       _userflash_write_byte
*SFR* 000000E0H   DATA     BYTE      ACC
*SFR* 000000E0H   DATA     BIT       ACC_ACC0
*SFR* 000000E0H.1 DATA     BIT       ACC_ACC1
*SFR* 000000E0H.2 DATA     BIT       ACC_ACC2
*SFR* 000000E0H.3 DATA     BIT       ACC_ACC3
*SFR* 000000E0H.4 DATA     BIT       ACC_ACC4
*SFR* 000000E0H.5 DATA     BIT       ACC_ACC5
*SFR* 000000E0H.6 DATA     BIT       ACC_ACC6
*SFR* 000000E0H.7 DATA     BIT       ACC_ACC7
*SFR* 000000BDH   DATA     WORD      ADC0
*SFR* 000000BCH   DATA     BYTE      ADC0CF
*SFR* 000000E8H   DATA     BYTE      ADC0CN0
*SFR* 000000E8H.4 DATA     BIT       ADC0CN0_ADBUSY
*SFR* 000000E8H   DATA     BIT       ADC0CN0_ADCM0
*SFR* 000000E8H.1 DATA     BIT       ADC0CN0_ADCM1
*SFR* 000000E8H.2 DATA     BIT       ADC0CN0_ADCM2
*SFR* 000000E8H.7 DATA     BIT       ADC0CN0_ADEN
*SFR* 000000E8H.5 DATA     BIT       ADC0CN0_ADINT
*SFR* 000000E8H.6 DATA     BIT       ADC0CN0_ADTM
*SFR* 000000E8H.3 DATA     BIT       ADC0CN0_ADWINT
*SFR* 000000C3H   DATA     WORD      ADC0GT
*SFR* 000000C4H   DATA     BYTE      ADC0GTH
*SFR* 000000C3H   DATA     BYTE      ADC0GTL
*SFR* 000000BEH   DATA     BYTE      ADC0H
*SFR* 000000BDH   DATA     BYTE      ADC0L
*SFR* 000000C5H   DATA     WORD      ADC0LT
*SFR* 000000C6H   DATA     BYTE      ADC0LTH
*SFR* 000000C5H   DATA     BYTE      ADC0LTL
      01005B21H   CODE     ---       ADC_0_enter_DefaultMode_from_RESET
      020004A5H   XDATA    ---       adxl
*DEL*:00000000H   CODE     ---       adxl345_get_interrupt
      0100535BH   CODE     ---       adxl345_init
      01004C87H   CODE     ---       adxl345_tick
      020004B2H   XDATA    ---       adxl_smoothing
*SFR* 000000BAH   DATA     BYTE      AMX0N
*SFR* 000000BBH   DATA     BYTE      AMX0P
*SFR* 000000F0H   DATA     BYTE      B
*SFR* 000000F0H   DATA     BIT       B_B0
*SFR* 000000F0H.1 DATA     BIT       B_B1
*SFR* 000000F0H.2 DATA     BIT       B_B2
*SFR* 000000F0H.3 DATA     BIT       B_B3
*SFR* 000000F0H.4 DATA     BIT       B_B4
*SFR* 000000F0H.5 DATA     BIT       B_B5
*SFR* 000000F0H.6 DATA     BIT       B_B6
*SFR* 000000F0H.7 DATA     BIT       B_B7
      02000461H   XDATA    ---       btn
      010029F8H   CODE     ---       btn_callback
      0100483CH   CODE     ---       btn_init
      01003072H   CODE     ---       btn_tick
LX51 LINKER/LOCATER V4.66.30.0                                                        07/27/2019  23:22:19  PAGE 22


      020004ABH   XDATA    ---       buf
*DEL*:00000000H   CODE     ---       CIP51_0_enter_DefaultMode_from_RESET
*SFR* 0000008EH   DATA     BYTE      CKCON0
*SFR* 000000E4H   DATA     BYTE      CKCON1
*SFR* 000000A9H   DATA     BYTE      CLKSEL
      01005B9EH   CODE     ---       CLOCK_0_enter_DefaultMode_from_RESET
*SFR* 0000009BH   DATA     BYTE      CMP0CN0
*SFR* 0000009DH   DATA     BYTE      CMP0MD
*SFR* 0000009FH   DATA     BYTE      CMP0MX
*SFR* 0000009AH   DATA     BYTE      CMP1CN0
*SFR* 0000009CH   DATA     BYTE      CMP1MD
*SFR* 0000009EH   DATA     BYTE      CMP1MX
      00000082H   IDATA    BYTE      cpu_max
      00000083H   IDATA    BYTE      cpu_use
*SFR* 00000082H   DATA     WORD      DP
*SFR* 00000083H   DATA     BYTE      DPH
*SFR* 00000082H   DATA     BYTE      DPL
      00000061H   DATA     WORD      ee_baseaddr
*SFR* 000000E6H   DATA     BYTE      EIE1
*SFR* 000000E7H   DATA     BYTE      EIE2
*SFR* 000000F6H   DATA     BYTE      EIP1
*SFR* 000000F7H   DATA     BYTE      EIP2
*SFR* 00000085H   DATA     BYTE      EMI0CF
*SFR* 000000AAH   DATA     BYTE      EMI0CN
*SFR* 00000084H   DATA     BYTE      EMI0TC
      0100506DH   CODE     ---       enter_DefaultMode_from_RESET
      01003B8DH   CODE     ---       err_namelong_1
      01003B9BH   CODE     ---       err_namelong_2
      01003BB5H   CODE     ---       err_namelong_3
      01003B47H   CODE     ---       err_namewide_1
      01003B55H   CODE     ---       err_namewide_2
      01003B6EH   CODE     ---       err_namewide_3
      01005BA2H   CODE     ---       EXTINT_0_enter_DefaultMode_from_RESET
*SFR* 000000B7H   DATA     BYTE      FLKEY
*SFR* 000000B6H   DATA     BYTE      FLSCL
      010089C4H   CONST    ---       font_Chewy_24
      01009994H   CONST    ---       font_Crushed_25
      0100601EH   CONST    ---       font_DejaVu_Sans_Mono_Bold_11
      01005BB3H   CONST    ---       font_Dialog_plain_8
      01007670H   CONST    ---       font_DialogInput_Bold_24
      00000064H   DATA     BYTE      font_glyph
      00000063H   DATA     BYTE      font_index
      01006636H   CONST    ---       font_Nimbus_Mono_L_Bold_20
      0100A794H   CONST    ---       font_Nimbus_Sans_L_25
      0100B6E0H   CONST    ---       font_Orbitron_28
      01004B23H   CODE     ---       font_table
      010049D2H   CODE     ---       fw_init
      00000021H.2 BIT      BIT       fw_interrupt
      00000021H.1 BIT      BIT       fw_loop_busy
      01003877H   CODE     ---       fw_oled_update_done
      010026D2H   CODE     ---       fw_tick_critical
      010048CBH   CODE     ---       fw_tick_mainloop
*SFR* 000000B3H   DATA     BYTE      HFO0CAL
*SFR* 000000B2H   DATA     BYTE      HFO0CN
      01005B9AH   CODE     ---       HFOSC_0_enter_DefaultMode_from_RESET
      00000071H   IDATA    ---       hsv
      0000005FH   DATA     ---       hwid
      01004C26H   CODE     ---       hwid_get_model
      01005B82H   CODE     ---       hwid_init
*SFR* 000000A8H   DATA     BYTE      IE
*SFR* 000000A8H.7 DATA     BIT       IE_EA
*SFR* 000000A8H.4 DATA     BIT       IE_ES0
LX51 LINKER/LOCATER V4.66.30.0                                                        07/27/2019  23:22:19  PAGE 23


*SFR* 000000A8H.6 DATA     BIT       IE_ESPI0
*SFR* 000000A8H.1 DATA     BIT       IE_ET0
*SFR* 000000A8H.3 DATA     BIT       IE_ET1
*SFR* 000000A8H.5 DATA     BIT       IE_ET2
*SFR* 000000A8H   DATA     BIT       IE_EX0
*SFR* 000000A8H.2 DATA     BIT       IE_EX1
      01005BAAH   CODE     ---       INT0_ISR
      01005B2BH   CODE     ---       INTERRUPT_0_enter_DefaultMode_from_RESET
*SFR* 000000B8H   DATA     BYTE      IP
*SFR* 000000B8H.4 DATA     BIT       IP_PS0
*SFR* 000000B8H.6 DATA     BIT       IP_PSPI0
*SFR* 000000B8H.1 DATA     BIT       IP_PT0
*SFR* 000000B8H.3 DATA     BIT       IP_PT1
*SFR* 000000B8H.5 DATA     BIT       IP_PT2
*SFR* 000000B8H   DATA     BIT       IP_PX0
*SFR* 000000B8H.2 DATA     BIT       IP_PX1
*SFR* 000000E4H   DATA     BYTE      IT01CF
      00000085H   IDATA    BYTE      last_empty_offset
      00000084H   IDATA    BYTE      last_valid_offset
      01002971H   CODE     ---       ledprog
*SFR* 00000086H   DATA     BYTE      LFO0CN
*DEL*:00000000H   CODE     ---       LFOSC_0_enter_DefaultMode_from_RESET
*DEL*:00000000H   CODE     ---       lsens_read
      01005A01H   CODE     ---       lsens_tick
      0000008BH   IDATA    BYTE      lsens_timeout
      010059A2H   CODE     ---       main
      00000019H   DATA     ---       menu
      0100D003H   CONST    ---       menu_0
      0100D00FH   CONST    ---       menu_1
      01005A37H   CODE     ---       menu_1_btn_enter
      01004CE8H   CODE     ---       menu_1_btn_exit
      0100434AH   CODE     ---       menu_1_btn_next
      01004554H   CODE     ---       menu_1_btn_prev
      010044A7H   CODE     ---       menu_1_btn_use
      010057C3H   CODE     ---       menu_1_font_next
*DEL*:00000000H   CODE     ---       menu_1_get_offset
      01003953H   CODE     ---       menu_1_name_edit
      0100D01BH   CONST    ---       menu_2
      01005B89H   CODE     ---       menu_2_btn_exit
      010050BCH   CODE     ---       menu_2_btn_next
      0100510BH   CODE     ---       menu_2_btn_prev
      0100D027H   CONST    ---       menu_5
      0100D033H   CONST    ---       menu_6
      010053DAH   CODE     ---       menu_6_btn_use
      010059DBH   CODE     ---       menu_6_font_next
      010059EEH   CODE     ---       menu_6_font_prev
      01005727H   CODE     ---       menu_btn_enter
      010055ABH   CODE     ---       menu_btn_exit
      01005964H   CODE     ---       menu_btn_next
      01005A25H   CODE     ---       menu_btn_prev
      01005677H   CODE     ---       menu_btn_use_none
      0100468AH   CODE     ---       menu_btn_use_std
      0000001BH   DATA     BYTE      menu_idx
      0100CFF7H   CONST    ---       menu_none
      01004DA6H   CODE     ---       menu_tick
      00000081H   IDATA    BYTE      missed
      00000018H   DATA     BYTE      mtick
      0000001CH   DATA     ---       o
      0200002BH   XDATA    ---       oled
      02000038H   XDATA    ---       oled_fb
*SFR* 00000080H   DATA     BYTE      P0
*SFR* 00000080H   DATA     BIT       P0_B0
LX51 LINKER/LOCATER V4.66.30.0                                                        07/27/2019  23:22:19  PAGE 24


*SFR* 00000080H.1 DATA     BIT       P0_B1
*SFR* 00000080H.2 DATA     BIT       P0_B2
*SFR* 00000080H.3 DATA     BIT       P0_B3
*SFR* 00000080H.4 DATA     BIT       P0_B4
*SFR* 00000080H.5 DATA     BIT       P0_B5
*SFR* 00000080H.6 DATA     BIT       P0_B6
*SFR* 00000080H.7 DATA     BIT       P0_B7
*SFR* 000000F1H   DATA     BYTE      P0MDIN
*SFR* 000000A4H   DATA     BYTE      P0MDOUT
*SFR* 000000D4H   DATA     BYTE      P0SKIP
*SFR* 00000090H   DATA     BYTE      P1
*SFR* 00000090H   DATA     BIT       P1_B0
*SFR* 00000090H.1 DATA     BIT       P1_B1
*SFR* 00000090H.2 DATA     BIT       P1_B2
*SFR* 00000090H.3 DATA     BIT       P1_B3
*SFR* 00000090H.4 DATA     BIT       P1_B4
*SFR* 00000090H.5 DATA     BIT       P1_B5
*SFR* 00000090H.6 DATA     BIT       P1_B6
*SFR* 00000090H.7 DATA     BIT       P1_B7
*SFR* 000000F2H   DATA     BYTE      P1MDIN
*SFR* 000000A5H   DATA     BYTE      P1MDOUT
*SFR* 000000D5H   DATA     BYTE      P1SKIP
*SFR* 000000A0H   DATA     BYTE      P2
*SFR* 000000A0H   DATA     BIT       P2_B0
*SFR* 000000A0H.1 DATA     BIT       P2_B1
*SFR* 000000A0H.2 DATA     BIT       P2_B2
*SFR* 000000A0H.3 DATA     BIT       P2_B3
*SFR* 000000A0H.4 DATA     BIT       P2_B4
*SFR* 000000A0H.5 DATA     BIT       P2_B5
*SFR* 000000A0H.6 DATA     BIT       P2_B6
*SFR* 000000A0H.7 DATA     BIT       P2_B7
*SFR* 000000F3H   DATA     BYTE      P2MDIN
*SFR* 000000A6H   DATA     BYTE      P2MDOUT
*SFR* 000000D6H   DATA     BYTE      P2SKIP
*SFR* 000000B0H   DATA     BYTE      P3
*SFR* 000000B0H   DATA     BIT       P3_B0
*SFR* 000000B0H.1 DATA     BIT       P3_B1
*SFR* 000000B0H.2 DATA     BIT       P3_B2
*SFR* 000000B0H.3 DATA     BIT       P3_B3
*SFR* 000000B0H.4 DATA     BIT       P3_B4
*SFR* 000000B0H.5 DATA     BIT       P3_B5
*SFR* 000000B0H.6 DATA     BIT       P3_B6
*SFR* 000000B0H.7 DATA     BIT       P3_B7
*SFR* 000000F4H   DATA     BYTE      P3MDIN
*SFR* 000000A7H   DATA     BYTE      P3MDOUT
*SFR* 000000DFH   DATA     BYTE      P3SKIP
*SFR* 000000C7H   DATA     BYTE      P4
*SFR* 000000F5H   DATA     BYTE      P4MDIN
*SFR* 000000AEH   DATA     BYTE      P4MDOUT
      01005B17H   CODE     ---       PBCFG_0_enter_DefaultMode_from_RESET
*SFR* 000000F9H   DATA     WORD      PCA0
*SFR* 000000D8H   DATA     BYTE      PCA0CN0
*SFR* 000000D8H   DATA     BIT       PCA0CN0_CCF0
*SFR* 000000D8H.1 DATA     BIT       PCA0CN0_CCF1
*SFR* 000000D8H.2 DATA     BIT       PCA0CN0_CCF2
*SFR* 000000D8H.3 DATA     BIT       PCA0CN0_CCF3
*SFR* 000000D8H.4 DATA     BIT       PCA0CN0_CCF4
*SFR* 000000D8H.7 DATA     BIT       PCA0CN0_CF
*SFR* 000000D8H.6 DATA     BIT       PCA0CN0_CR
*SFR* 000000FBH   DATA     WORD      PCA0CP0
*SFR* 000000E9H   DATA     WORD      PCA0CP1
*SFR* 000000EBH   DATA     WORD      PCA0CP2
LX51 LINKER/LOCATER V4.66.30.0                                                        07/27/2019  23:22:19  PAGE 25


*SFR* 000000EDH   DATA     WORD      PCA0CP3
*SFR* 000000FDH   DATA     WORD      PCA0CP4
*SFR* 000000FCH   DATA     BYTE      PCA0CPH0
*SFR* 000000EAH   DATA     BYTE      PCA0CPH1
*SFR* 000000ECH   DATA     BYTE      PCA0CPH2
*SFR* 000000EEH   DATA     BYTE      PCA0CPH3
*SFR* 000000FEH   DATA     BYTE      PCA0CPH4
*SFR* 000000FBH   DATA     BYTE      PCA0CPL0
*SFR* 000000E9H   DATA     BYTE      PCA0CPL1
*SFR* 000000EBH   DATA     BYTE      PCA0CPL2
*SFR* 000000EDH   DATA     BYTE      PCA0CPL3
*SFR* 000000FDH   DATA     BYTE      PCA0CPL4
*SFR* 000000DAH   DATA     BYTE      PCA0CPM0
*SFR* 000000DBH   DATA     BYTE      PCA0CPM1
*SFR* 000000DCH   DATA     BYTE      PCA0CPM2
*SFR* 000000DDH   DATA     BYTE      PCA0CPM3
*SFR* 000000DEH   DATA     BYTE      PCA0CPM4
*SFR* 000000FAH   DATA     BYTE      PCA0H
*SFR* 000000F9H   DATA     BYTE      PCA0L
*SFR* 000000D9H   DATA     BYTE      PCA0MD
      01000096H   CODE     ---       PCA_0_enter_DefaultMode_from_RESET
      01005AE5H   CODE     ---       PCACH_0_enter_DefaultMode_from_RESET
      01005AEFH   CODE     ---       PCACH_1_enter_DefaultMode_from_RESET
      01005AF9H   CODE     ---       PCACH_2_enter_DefaultMode_from_RESET
      01005B03H   CODE     ---       PCACH_3_enter_DefaultMode_from_RESET
      01005B74H   CODE     ---       PCACH_4_enter_DefaultMode_from_RESET
*SFR* 00000087H   DATA     BYTE      PCON0
*SFR* 000000AFH   DATA     BYTE      PFE0CN
      01005AA5H   CODE     ---       PORTS_0_enter_DefaultMode_from_RESET
      01005B0DH   CODE     ---       PORTS_1_enter_DefaultMode_from_RESET
      01005AB2H   CODE     ---       PORTS_2_enter_DefaultMode_from_RESET
      01005BB1H   CODE     ---       PORTS_3_enter_DefaultMode_from_RESET
*SFR* 000000A0H   DATA     BYTE      PPAGE_SFR
*SFR* 0000008FH   DATA     BYTE      PSCTL
*SFR* 000000D0H   DATA     BYTE      PSW
*SFR* 000000D0H.6 DATA     BIT       PSW_AC
*SFR* 000000D0H.7 DATA     BIT       PSW_CY
*SFR* 000000D0H.5 DATA     BIT       PSW_F0
*SFR* 000000D0H.1 DATA     BIT       PSW_F1
*SFR* 000000D0H.2 DATA     BIT       PSW_OV
*SFR* 000000D0H   DATA     BIT       PSW_PARITY
*SFR* 000000D0H.3 DATA     BIT       PSW_RS0
*SFR* 000000D0H.4 DATA     BIT       PSW_RS1
      01005A89H   CODE     ---       PWR_enterIdle
*DEL*:00000000H   CODE     ---       PWR_enterShutdown
*DEL*:00000000H   CODE     ---       PWR_enterStop
*DEL*:00000000H   CODE     ---       PWR_enterSuspend
      010054C8H   CODE     NEAR LAB  rand16
*SFR* 000000D1H   DATA     BYTE      REF0CN
*SFR* 000000C9H   DATA     BYTE      REG01CN
      00000065H   IDATA    ---       rgb
      02000245H   XDATA    ---       rotdst
      020002F2H   XDATA    ---       rotdst_fb
      02000239H   XDATA    ---       rotsrc
      02000251H   XDATA    ---       rotsrc_fb
*SFR* 000000EFH   DATA     BYTE      RSTSRC
*SFR* 000000ACH   DATA     BYTE      SBCON1
*SFR* 000000B4H   DATA     WORD      SBRL1
*SFR* 000000B5H   DATA     BYTE      SBRLH1
*SFR* 000000B4H   DATA     BYTE      SBRLL1
*SFR* 00000099H   DATA     BYTE      SBUF0
*SFR* 000000D3H   DATA     BYTE      SBUF1
LX51 LINKER/LOCATER V4.66.30.0                                                        07/27/2019  23:22:19  PAGE 26


*SFR* 00000098H   DATA     BYTE      SCON0
*SFR* 00000098H.5 DATA     BIT       SCON0_MCE
*SFR* 00000098H.2 DATA     BIT       SCON0_RB8
*SFR* 00000098H.4 DATA     BIT       SCON0_REN
*SFR* 00000098H   DATA     BIT       SCON0_RI
*SFR* 00000098H.7 DATA     BIT       SCON0_SMODE
*SFR* 00000098H.3 DATA     BIT       SCON0_TB8
*SFR* 00000098H.1 DATA     BIT       SCON0_TI
*SFR* 000000D2H   DATA     BYTE      SCON1
*SFR* 000000BFH   DATA     BYTE      SFRPAGE
      01005BB0H   CODE     ---       SILABS_STARTUP
      0100D03FH   CONST    ---       sin90
*DEL*:00000000H   CODE     ---       slab_Assert
*SFR* 000000CEH   DATA     BYTE      SMB0ADM
*SFR* 000000CFH   DATA     BYTE      SMB0ADR
*SFR* 000000C1H   DATA     BYTE      SMB0CF
*SFR* 000000C0H   DATA     BYTE      SMB0CN0
*SFR* 000000C0H.1 DATA     BIT       SMB0CN0_ACK
*SFR* 000000C0H.3 DATA     BIT       SMB0CN0_ACKRQ
*SFR* 000000C0H.2 DATA     BIT       SMB0CN0_ARBLOST
*SFR* 000000C0H.7 DATA     BIT       SMB0CN0_MASTER
*SFR* 000000C0H   DATA     BIT       SMB0CN0_SI
*SFR* 000000C0H.5 DATA     BIT       SMB0CN0_STA
*SFR* 000000C0H.4 DATA     BIT       SMB0CN0_STO
*SFR* 000000C0H.6 DATA     BIT       SMB0CN0_TXMODE
*SFR* 000000C2H   DATA     BYTE      SMB0DAT
      01005BADH   CODE     ---       smb1_get_state
      01002CBAH   CODE     ---       smb1_interrupt
      00000012H   DATA     BYTE      smb1_state
      01005B3FH   CODE     ---       smb1_stop
*SFR* 000000CEH   DATA     BYTE      SMB1ADM
*SFR* 000000CFH   DATA     BYTE      SMB1ADR
*SFR* 000000C1H   DATA     BYTE      SMB1CF
*SFR* 000000C0H   DATA     BYTE      SMB1CN0
*SFR* 000000C0H.1 DATA     BIT       SMB1CN0_ACK
*SFR* 000000C0H.3 DATA     BIT       SMB1CN0_ACKRQ
*SFR* 000000C0H.2 DATA     BIT       SMB1CN0_ARBLOST
*SFR* 000000C0H.7 DATA     BIT       SMB1CN0_MASTER
*SFR* 000000C0H   DATA     BIT       SMB1CN0_SI
*SFR* 000000C0H.5 DATA     BIT       SMB1CN0_STA
*SFR* 000000C0H.4 DATA     BIT       SMB1CN0_STO
*SFR* 000000C0H.6 DATA     BIT       SMB1CN0_TXMODE
*SFR* 000000C2H   DATA     BYTE      SMB1DAT
*SFR* 000000B9H   DATA     BYTE      SMBTC
      01005453H   CODE     ---       SMBUS1_ISR
      01005B35H   CODE     ---       SMBUS_0_enter_DefaultMode_from_RESET
      0100008CH   CODE     ---       SMBUS_1_enter_DefaultMode_from_RESET
*SFR* 000000E5H   DATA     BYTE      SMOD1
*SFR* 00000081H   DATA     BYTE      SP
*SFR* 000000A1H   DATA     BYTE      SPI0CFG
*SFR* 000000A2H   DATA     BYTE      SPI0CKR
*SFR* 000000F8H   DATA     BYTE      SPI0CN0
*SFR* 000000F8H.5 DATA     BIT       SPI0CN0_MODF
*SFR* 000000F8H.2 DATA     BIT       SPI0CN0_NSSMD0
*SFR* 000000F8H.3 DATA     BIT       SPI0CN0_NSSMD1
*SFR* 000000F8H.4 DATA     BIT       SPI0CN0_RXOVRN
*SFR* 000000F8H   DATA     BIT       SPI0CN0_SPIEN
*SFR* 000000F8H.7 DATA     BIT       SPI0CN0_SPIF
*SFR* 000000F8H.1 DATA     BIT       SPI0CN0_TXBMT
*SFR* 000000F8H.6 DATA     BIT       SPI0CN0_WCOL
*SFR* 000000A3H   DATA     BYTE      SPI0DAT
      01005A5AH   CODE     ---       SPI_0_enter_DefaultMode_from_RESET
LX51 LINKER/LOCATER V4.66.30.0                                                        07/27/2019  23:22:19  PAGE 27


      02000023H   PDATA    ---       ssd1306_buf
      01005B49H   CODE     ---       ssd1306_cb_get
      00000021H.3 BIT      BIT       ssd1306_cb_pending
      02000037H   XDATA    BYTE      ssd1306_cb_state
      0100D079H   CONST    ---       ssd1306_cmd_disp_window_def
      0100D060H   CONST    ---       ssd1306_cmd_init
      0100579FH   CODE     ---       ssd1306_idle_wait
      01005924H   CODE     ---       ssd1306_init_step2
      01005884H   CODE     ---       ssd1306_init_step3
      01004E61H   CODE     ---       ssd1306_update
      0000001FH   DATA     BYTE      sysflags
*SFR* 00000088H   DATA     BYTE      TCON
*SFR* 00000088H.1 DATA     BIT       TCON_IE0
*SFR* 00000088H.3 DATA     BIT       TCON_IE1
*SFR* 00000088H   DATA     BIT       TCON_IT0
*SFR* 00000088H.2 DATA     BIT       TCON_IT1
*SFR* 00000088H.5 DATA     BIT       TCON_TF0
*SFR* 00000088H.7 DATA     BIT       TCON_TF1
*SFR* 00000088H.4 DATA     BIT       TCON_TR0
*SFR* 00000088H.6 DATA     BIT       TCON_TR1
*SFR* 0000008CH   DATA     BYTE      TH0
*SFR* 0000008DH   DATA     BYTE      TH1
      00000017H   DATA     BYTE      tick_ctr
      010059C8H   CODE     ---       TIMER01_0_enter_DefaultMode_from_RESET
      010059B5H   CODE     ---       TIMER16_2_enter_DefaultMode_from_RESET
*DEL*:00000000H   CODE     ---       TIMER16_4_enter_DefaultMode_from_RESET
      0100590EH   CODE     ---       TIMER16_5_enter_DefaultMode_from_RESET
      0100528BH   CODE     ---       TIMER5_ISR
      0100593AH   CODE     ---       TIMER_SETUP_0_enter_DefaultMode_from_RESET
*SFR* 0000008AH   DATA     BYTE      TL0
*SFR* 0000008BH   DATA     BYTE      TL1
*SFR* 00000089H   DATA     BYTE      TMOD
*SFR* 000000CCH   DATA     WORD      TMR2
*SFR* 000000C8H   DATA     BYTE      TMR2CN0
*SFR* 000000C8H.1 DATA     BIT       TMR2CN0_T2CSS
*SFR* 000000C8H.3 DATA     BIT       TMR2CN0_T2SPLIT
*SFR* 000000C8H   DATA     BIT       TMR2CN0_T2XCLK
*SFR* 000000C8H.4 DATA     BIT       TMR2CN0_TF2CEN
*SFR* 000000C8H.7 DATA     BIT       TMR2CN0_TF2H
*SFR* 000000C8H.6 DATA     BIT       TMR2CN0_TF2L
*SFR* 000000C8H.5 DATA     BIT       TMR2CN0_TF2LEN
*SFR* 000000C8H.2 DATA     BIT       TMR2CN0_TR2
*SFR* 000000CDH   DATA     BYTE      TMR2H
*SFR* 000000CCH   DATA     BYTE      TMR2L
*SFR* 000000CAH   DATA     WORD      TMR2RL
*SFR* 000000CBH   DATA     BYTE      TMR2RLH
*SFR* 000000CAH   DATA     BYTE      TMR2RLL
*SFR* 00000094H   DATA     WORD      TMR3
*SFR* 00000091H   DATA     BYTE      TMR3CN0
*SFR* 00000095H   DATA     BYTE      TMR3H
*SFR* 00000094H   DATA     BYTE      TMR3L
*SFR* 00000092H   DATA     WORD      TMR3RL
*SFR* 00000093H   DATA     BYTE      TMR3RLH
*SFR* 00000092H   DATA     BYTE      TMR3RLL
*SFR* 00000094H   DATA     WORD      TMR4
*SFR* 00000091H   DATA     BYTE      TMR4CN0
*SFR* 00000095H   DATA     BYTE      TMR4H
*SFR* 00000094H   DATA     BYTE      TMR4L
*SFR* 00000092H   DATA     WORD      TMR4RL
*SFR* 00000093H   DATA     BYTE      TMR4RLH
*SFR* 00000092H   DATA     BYTE      TMR4RLL
*SFR* 000000CCH   DATA     WORD      TMR5
LX51 LINKER/LOCATER V4.66.30.0                                                        07/27/2019  23:22:19  PAGE 28


*SFR* 000000C8H   DATA     BYTE      TMR5CN0
*SFR* 000000C8H.3 DATA     BIT       TMR5CN0_T5SPLIT
*SFR* 000000C8H   DATA     BIT       TMR5CN0_T5XCLK
*SFR* 000000C8H.7 DATA     BIT       TMR5CN0_TF5H
*SFR* 000000C8H.6 DATA     BIT       TMR5CN0_TF5L
*SFR* 000000C8H.5 DATA     BIT       TMR5CN0_TF5LEN
*SFR* 000000C8H.2 DATA     BIT       TMR5CN0_TR5
*SFR* 000000CDH   DATA     BYTE      TMR5H
*SFR* 000000CCH   DATA     BYTE      TMR5L
*SFR* 000000CAH   DATA     WORD      TMR5RL
*SFR* 000000CBH   DATA     BYTE      TMR5RLH
*SFR* 000000CAH   DATA     BYTE      TMR5RLL
      01005BA6H   CODE     ---       UART_0_enter_DefaultMode_from_RESET
      02000393H   XDATA    ---       uconf
      01004D48H   CODE     ---       uconf_load
      01003D71H   CODE     ---       uconf_write
      00000013H   DATA     DWORD     uptime
*SFR* 00000096H   DATA     BYTE      USB0ADR
*SFR* 00000097H   DATA     BYTE      USB0DAT
*SFR* 000000D7H   DATA     BYTE      USB0XCN
      01005B95H   CODE     ---       userflash_get_baseaddr
      01005A49H   CODE     ---       userflash_init
*SFR* 000000FFH   DATA     BYTE      VDM0CN
      0100D080H   CONST    ---       ver
      0000008CH   IDATA    BYTE      wiggle
*SFR* 000000E1H   DATA     BYTE      XBR0
*SFR* 000000E2H   DATA     BYTE      XBR1
*SFR* 000000E3H   DATA     BYTE      XBR2
*SFR* 000000B1H   DATA     BYTE      XOSC0CN



SYMBOL TABLE OF MODULE:  GAT_NAMETAG.OMF.CRBUILD (?C_STARTUP)

      VALUE       REP       CLASS    TYPE      SYMBOL NAME
      ====================================================
      ---         MODULE    ---      ---       ?C_STARTUP
      01000000H   PUBLIC    CODE     NEAR LAB  ?C_STARTUP
      000000E0H   SFRSYM    DATA     BYTE      ACC
      000000F0H   SFRSYM    DATA     BYTE      B
      00000083H   SFRSYM    DATA     BYTE      DPH
      00000082H   SFRSYM    DATA     BYTE      DPL
      000000A0H   SFRSYM    DATA     BYTE      PPAGE_SFR
      00000081H   SFRSYM    DATA     BYTE      SP
      00000000H   SYMBOL    NUMBER   ---       IBPSTACK
      00000100H   SYMBOL    NUMBER   ---       IBPSTACKTOP
      00000080H   SYMBOL    NUMBER   ---       IDATALEN
      010047B3H   SYMBOL    CODE     NEAR LAB  IDATALOOP
      00000000H   SYMBOL    NUMBER   ---       PBPSTACK
      00000100H   SYMBOL    NUMBER   ---       PBPSTACKTOP
      00000000H   SYMBOL    NUMBER   ---       PDATALEN
      00000000H   SYMBOL    NUMBER   ---       PDATASTART
      00000000H   SYMBOL    NUMBER   ---       PPAGE
      00000000H   SYMBOL    NUMBER   ---       PPAGEENABLE
      010047ADH   SYMBOL    CODE     NEAR LAB  STARTUP1
      00000000H   SYMBOL    NUMBER   ---       XBPSTACK
      00010000H   SYMBOL    NUMBER   ---       XBPSTACKTOP
      00000000H   SYMBOL    NUMBER   ---       XDATALEN
      00000000H   SYMBOL    NUMBER   ---       XDATASTART

      01000000H   BLOCK     CODE     NEAR LAB  LVL=0
      01000000H   LINE      CODE     ---       #126
LX51 LINKER/LOCATER V4.66.30.0                                                        07/27/2019  23:22:19  PAGE 29


      ---         BLOCKEND  ---      ---       LVL=0

      010047ADH   BLOCK     CODE     NEAR LAB  LVL=0
      010047ADH   LINE      CODE     ---       #134
      010047B0H   LINE      CODE     ---       #138
      010047B2H   LINE      CODE     ---       #139
      010047B3H   LINE      CODE     ---       #140
      010047B4H   LINE      CODE     ---       #141
      010047B6H   LINE      CODE     ---       #190
      010047B9H   LINE      CODE     ---       #201
      ---         BLOCKEND  ---      ---       LVL=0

      ---         MODULE    ---      ---       GAT_NAMETAG_MAIN
      010059A2H   PUBLIC    CODE     ---       main
      01005BB0H   PUBLIC    CODE     ---       SiLabs_Startup
      000000A2H   SFRSYM    DATA     BYTE      SPI0CKR
      00000080H   SFRSYM    DATA     BYTE      P0
      000000D0H.2 SFRSYM    DATA     BIT       PSW_OV
      000000B1H   SFRSYM    DATA     BYTE      XOSC0CN
      00000090H   SFRSYM    DATA     BYTE      P1
      000000A0H   SFRSYM    DATA     BYTE      P2
      000000B0H   SFRSYM    DATA     BYTE      P3
      000000BCH   SFRSYM    DATA     BYTE      ADC0CF
      000000C8H   SFRSYM    DATA     BIT       TMR2CN0_T2XCLK
      000000C7H   SFRSYM    DATA     BYTE      P4
      000000C0H.7 SFRSYM    DATA     BIT       SMB0CN0_MASTER
      000000F9H   SFRSYM    DATA     WORD      PCA0
      000000E6H   SFRSYM    DATA     BYTE      EIE1
      000000C0H.7 SFRSYM    DATA     BIT       SMB1CN0_MASTER
      000000C0H.1 SFRSYM    DATA     BIT       SMB0CN0_ACK
      000000D7H   SFRSYM    DATA     BYTE      USB0XCN
      000000E7H   SFRSYM    DATA     BYTE      EIE2
      000000C0H.1 SFRSYM    DATA     BIT       SMB1CN0_ACK
      0000008FH   SFRSYM    DATA     BYTE      PSCTL
      000000E4H   SFRSYM    DATA     BYTE      IT01CF
      000000C8H   SFRSYM    DATA     BIT       TMR5CN0_T5XCLK
      000000C0H.6 SFRSYM    DATA     BIT       SMB0CN0_TXMODE
      000000C0H.6 SFRSYM    DATA     BIT       SMB1CN0_TXMODE
      000000BFH   SFRSYM    DATA     BYTE      SFRPAGE
      000000A4H   SFRSYM    DATA     BYTE      P0MDOUT
      000000A5H   SFRSYM    DATA     BYTE      P1MDOUT
      000000E8H.5 SFRSYM    DATA     BIT       ADC0CN0_ADINT
      000000CBH   SFRSYM    DATA     BYTE      TMR2RLH
      000000A6H   SFRSYM    DATA     BYTE      P2MDOUT
      000000A8H   SFRSYM    DATA     BYTE      IE
      00000093H   SFRSYM    DATA     BYTE      TMR3RLH
      000000A7H   SFRSYM    DATA     BYTE      P3MDOUT
      00000093H   SFRSYM    DATA     BYTE      TMR4RLH
      000000AEH   SFRSYM    DATA     BYTE      P4MDOUT
      000000F6H   SFRSYM    DATA     BYTE      EIP1
      000000CBH   SFRSYM    DATA     BYTE      TMR5RLH
      000000F7H   SFRSYM    DATA     BYTE      EIP2
      00000098H.2 SFRSYM    DATA     BIT       SCON0_RB8
      000000CAH   SFRSYM    DATA     BYTE      TMR2RLL
      000000FCH   SFRSYM    DATA     BYTE      PCA0CPH0
      00000092H   SFRSYM    DATA     BYTE      TMR3RLL
      000000EAH   SFRSYM    DATA     BYTE      PCA0CPH1
      00000098H.3 SFRSYM    DATA     BIT       SCON0_TB8
      000000F0H   SFRSYM    DATA     BIT       B_B0
      00000082H   SFRSYM    DATA     WORD      DP
      00000092H   SFRSYM    DATA     BYTE      TMR4RLL
      000000ECH   SFRSYM    DATA     BYTE      PCA0CPH2
LX51 LINKER/LOCATER V4.66.30.0                                                        07/27/2019  23:22:19  PAGE 30


      000000F0H.1 SFRSYM    DATA     BIT       B_B1
      000000C3H   SFRSYM    DATA     WORD      ADC0GT
      000000CAH   SFRSYM    DATA     BYTE      TMR5RLL
      000000EEH   SFRSYM    DATA     BYTE      PCA0CPH3
      000000F0H.2 SFRSYM    DATA     BIT       B_B2
      000000FBH   SFRSYM    DATA     BYTE      PCA0CPL0
      000000FEH   SFRSYM    DATA     BYTE      PCA0CPH4
      00000085H   SFRSYM    DATA     BYTE      EMI0CF
      000000F0H.3 SFRSYM    DATA     BIT       B_B3
      000000D9H   SFRSYM    DATA     BYTE      PCA0MD
      000000DAH   SFRSYM    DATA     BYTE      PCA0CPM0
      000000E9H   SFRSYM    DATA     BYTE      PCA0CPL1
      000000F0H.4 SFRSYM    DATA     BIT       B_B4
      000000DBH   SFRSYM    DATA     BYTE      PCA0CPM1
      000000EBH   SFRSYM    DATA     BYTE      PCA0CPL2
      000000F0H.5 SFRSYM    DATA     BIT       B_B5
      000000DCH   SFRSYM    DATA     BYTE      PCA0CPM2
      000000EDH   SFRSYM    DATA     BYTE      PCA0CPL3
      000000B8H   SFRSYM    DATA     BYTE      IP
      000000F0H.6 SFRSYM    DATA     BIT       B_B6
      000000C5H   SFRSYM    DATA     WORD      ADC0LT
      000000DDH   SFRSYM    DATA     BYTE      PCA0CPM3
      000000FDH   SFRSYM    DATA     BYTE      PCA0CPL4
      00000098H.5 SFRSYM    DATA     BIT       SCON0_MCE
      000000F0H.7 SFRSYM    DATA     BIT       B_B7
      000000DEH   SFRSYM    DATA     BYTE      PCA0CPM4
      000000E1H   SFRSYM    DATA     BYTE      XBR0
      000000C1H   SFRSYM    DATA     BYTE      SMB0CF
      000000E2H   SFRSYM    DATA     BYTE      XBR1
      000000C1H   SFRSYM    DATA     BYTE      SMB1CF
      000000AFH   SFRSYM    DATA     BYTE      PFE0CN
      000000AAH   SFRSYM    DATA     BYTE      EMI0CN
      000000C0H.5 SFRSYM    DATA     BIT       SMB0CN0_STA
      000000E3H   SFRSYM    DATA     BYTE      XBR2
      000000C0H.5 SFRSYM    DATA     BIT       SMB1CN0_STA
      000000E0H   SFRSYM    DATA     BIT       ACC_ACC0
      000000D1H   SFRSYM    DATA     BYTE      REF0CN
      000000B2H   SFRSYM    DATA     BYTE      HFO0CN
      0000008EH   SFRSYM    DATA     BYTE      CKCON0
      000000E0H.1 SFRSYM    DATA     BIT       ACC_ACC1
      000000E4H   SFRSYM    DATA     BYTE      CKCON1
      000000C8H.2 SFRSYM    DATA     BIT       TMR2CN0_TR2
      000000E0H.2 SFRSYM    DATA     BIT       ACC_ACC2
      000000E0H.3 SFRSYM    DATA     BIT       ACC_ACC3
      00000081H   SFRSYM    DATA     BYTE      SP
      0000009DH   SFRSYM    DATA     BYTE      CMP0MD
      000000E0H.4 SFRSYM    DATA     BIT       ACC_ACC4
      00000086H   SFRSYM    DATA     BYTE      LFO0CN
      00000084H   SFRSYM    DATA     BYTE      EMI0TC
      0000009CH   SFRSYM    DATA     BYTE      CMP1MD
      000000D8H   SFRSYM    DATA     BIT       PCA0CN0_CCF0
      000000E0H.5 SFRSYM    DATA     BIT       ACC_ACC5
      000000D8H.1 SFRSYM    DATA     BIT       PCA0CN0_CCF1
      000000E0H.6 SFRSYM    DATA     BIT       ACC_ACC6
      000000CCH   SFRSYM    DATA     WORD      TMR2
      000000D8H.2 SFRSYM    DATA     BIT       PCA0CN0_CCF2
      000000E0H.7 SFRSYM    DATA     BIT       ACC_ACC7
      00000094H   SFRSYM    DATA     WORD      TMR3
      000000C8H.2 SFRSYM    DATA     BIT       TMR5CN0_TR5
      000000D8H.3 SFRSYM    DATA     BIT       PCA0CN0_CCF3
      00000094H   SFRSYM    DATA     WORD      TMR4
      000000ACH   SFRSYM    DATA     BYTE      SBCON1
LX51 LINKER/LOCATER V4.66.30.0                                                        07/27/2019  23:22:19  PAGE 31


      000000D8H.4 SFRSYM    DATA     BIT       PCA0CN0_CCF4
      000000CCH   SFRSYM    DATA     WORD      TMR5
      000000C0H.3 SFRSYM    DATA     BIT       SMB0CN0_ACKRQ
      000000FFH   SFRSYM    DATA     BYTE      VDM0CN
      000000F1H   SFRSYM    DATA     BYTE      P0MDIN
      000000C0H.3 SFRSYM    DATA     BIT       SMB1CN0_ACKRQ
      00000098H.4 SFRSYM    DATA     BIT       SCON0_REN
      000000F2H   SFRSYM    DATA     BYTE      P1MDIN
      000000F3H   SFRSYM    DATA     BYTE      P2MDIN
      000000C0H.4 SFRSYM    DATA     BIT       SMB0CN0_STO
      000000F4H   SFRSYM    DATA     BYTE      P3MDIN
      000000C0H.4 SFRSYM    DATA     BIT       SMB1CN0_STO
      000000B5H   SFRSYM    DATA     BYTE      SBRLH1
      000000F5H   SFRSYM    DATA     BYTE      P4MDIN
      000000D0H.3 SFRSYM    DATA     BIT       PSW_RS0
      000000D8H.7 SFRSYM    DATA     BIT       PCA0CN0_CF
      000000F8H.4 SFRSYM    DATA     BIT       SPI0CN0_RXOVRN
      000000D0H.4 SFRSYM    DATA     BIT       PSW_RS1
      000000B4H   SFRSYM    DATA     BYTE      SBRLL1
      000000E8H.7 SFRSYM    DATA     BIT       ADC0CN0_ADEN
      00000089H   SFRSYM    DATA     BYTE      TMOD
      00000088H   SFRSYM    DATA     BYTE      TCON
      000000D0H   SFRSYM    DATA     BIT       PSW_PARITY
      000000A8H.4 SFRSYM    DATA     BIT       IE_ES0
      0000009FH   SFRSYM    DATA     BYTE      CMP0MX
      000000A8H.1 SFRSYM    DATA     BIT       IE_ET0
      0000009EH   SFRSYM    DATA     BYTE      CMP1MX
      000000A8H.3 SFRSYM    DATA     BIT       IE_ET1
      000000D4H   SFRSYM    DATA     BYTE      P0SKIP
      000000C8H.1 SFRSYM    DATA     BIT       TMR2CN0_T2CSS
      000000A8H.5 SFRSYM    DATA     BIT       IE_ET2
      000000D5H   SFRSYM    DATA     BYTE      P1SKIP
      000000D6H   SFRSYM    DATA     BYTE      P2SKIP
      000000E8H   SFRSYM    DATA     BYTE      ADC0CN0
      000000A8H   SFRSYM    DATA     BIT       IE_EX0
      000000DFH   SFRSYM    DATA     BYTE      P3SKIP
      000000D8H.6 SFRSYM    DATA     BIT       PCA0CN0_CR
      000000A8H.2 SFRSYM    DATA     BIT       IE_EX1
      00000098H.7 SFRSYM    DATA     BIT       SCON0_SMODE
      000000A9H   SFRSYM    DATA     BYTE      CLKSEL
      000000F8H   SFRSYM    DATA     BIT       SPI0CN0_SPIEN
      000000F0H   SFRSYM    DATA     BYTE      B
      000000BEH   SFRSYM    DATA     BYTE      ADC0H
      000000E8H.6 SFRSYM    DATA     BIT       ADC0CN0_ADTM
      000000CAH   SFRSYM    DATA     WORD      TMR2RL
      000000BDH   SFRSYM    DATA     BYTE      ADC0L
      00000092H   SFRSYM    DATA     WORD      TMR3RL
      00000092H   SFRSYM    DATA     WORD      TMR4RL
      000000D8H   SFRSYM    DATA     BYTE      PCA0CN0
      000000E0H   SFRSYM    DATA     BYTE      ACC
      000000CAH   SFRSYM    DATA     WORD      TMR5RL
      000000FBH   SFRSYM    DATA     WORD      PCA0CP0
      000000E9H   SFRSYM    DATA     WORD      PCA0CP1
      000000EBH   SFRSYM    DATA     WORD      PCA0CP2
      000000EDH   SFRSYM    DATA     WORD      PCA0CP3
      0000008CH   SFRSYM    DATA     BYTE      TH0
      000000B8H.4 SFRSYM    DATA     BIT       IP_PS0
      000000FDH   SFRSYM    DATA     WORD      PCA0CP4
      0000008DH   SFRSYM    DATA     BYTE      TH1
      000000FAH   SFRSYM    DATA     BYTE      PCA0H
      000000B8H.1 SFRSYM    DATA     BIT       IP_PT0
      000000B8H.3 SFRSYM    DATA     BIT       IP_PT1
LX51 LINKER/LOCATER V4.66.30.0                                                        07/27/2019  23:22:19  PAGE 32


      000000C0H.2 SFRSYM    DATA     BIT       SMB0CN0_ARBLOST
      000000B8H.5 SFRSYM    DATA     BIT       IP_PT2
      0000008AH   SFRSYM    DATA     BYTE      TL0
      000000F8H.1 SFRSYM    DATA     BIT       SPI0CN0_TXBMT
      000000C0H.2 SFRSYM    DATA     BIT       SMB1CN0_ARBLOST
      000000D0H.5 SFRSYM    DATA     BIT       PSW_F0
      000000A8H.6 SFRSYM    DATA     BIT       IE_ESPI0
      0000008BH   SFRSYM    DATA     BYTE      TL1
      000000F9H   SFRSYM    DATA     BYTE      PCA0L
      000000C0H   SFRSYM    DATA     BIT       SMB0CN0_SI
      000000D0H.1 SFRSYM    DATA     BIT       PSW_F1
      00000080H   SFRSYM    DATA     BIT       P0_B0
      000000B8H   SFRSYM    DATA     BIT       IP_PX0
      000000C9H   SFRSYM    DATA     BYTE      REG01CN
      000000C0H   SFRSYM    DATA     BIT       SMB1CN0_SI
      00000090H   SFRSYM    DATA     BIT       P1_B0
      00000080H.1 SFRSYM    DATA     BIT       P0_B1
      000000B8H.2 SFRSYM    DATA     BIT       IP_PX1
      0000009BH   SFRSYM    DATA     BYTE      CMP0CN0
      00000088H.1 SFRSYM    DATA     BIT       TCON_IE0
      000000A0H   SFRSYM    DATA     BIT       P2_B0
      00000090H.1 SFRSYM    DATA     BIT       P1_B1
      00000080H.2 SFRSYM    DATA     BIT       P0_B2
      0000009AH   SFRSYM    DATA     BYTE      CMP1CN0
      00000088H.3 SFRSYM    DATA     BIT       TCON_IE1
      000000B0H   SFRSYM    DATA     BIT       P3_B0
      000000A0H.1 SFRSYM    DATA     BIT       P2_B1
      00000090H.2 SFRSYM    DATA     BIT       P1_B2
      00000080H.3 SFRSYM    DATA     BIT       P0_B3
      000000C0H   SFRSYM    DATA     BYTE      SMB0CN0
      000000B0H.1 SFRSYM    DATA     BIT       P3_B1
      000000A0H.2 SFRSYM    DATA     BIT       P2_B2
      00000090H.3 SFRSYM    DATA     BIT       P1_B3
      00000080H.4 SFRSYM    DATA     BIT       P0_B4
      000000C0H   SFRSYM    DATA     BYTE      SMB1CN0
      000000B0H.2 SFRSYM    DATA     BIT       P3_B2
      000000A0H.3 SFRSYM    DATA     BIT       P2_B3
      00000090H.4 SFRSYM    DATA     BIT       P1_B4
      00000080H.5 SFRSYM    DATA     BIT       P0_B5
      000000B0H.3 SFRSYM    DATA     BIT       P3_B3
      000000A0H.4 SFRSYM    DATA     BIT       P2_B4
      00000090H.5 SFRSYM    DATA     BIT       P1_B5
      00000080H.6 SFRSYM    DATA     BIT       P0_B6
      000000B0H.4 SFRSYM    DATA     BIT       P3_B4
      000000A0H.5 SFRSYM    DATA     BIT       P2_B5
      00000090H.6 SFRSYM    DATA     BIT       P1_B6
      00000080H.7 SFRSYM    DATA     BIT       P0_B7
      000000B0H.5 SFRSYM    DATA     BIT       P3_B5
      000000A0H.6 SFRSYM    DATA     BIT       P2_B6
      00000090H.7 SFRSYM    DATA     BIT       P1_B7
      000000B0H.6 SFRSYM    DATA     BIT       P3_B6
      000000A0H.7 SFRSYM    DATA     BIT       P2_B7
      000000B0H.7 SFRSYM    DATA     BIT       P3_B7
      00000083H   SFRSYM    DATA     BYTE      DPH
      000000C4H   SFRSYM    DATA     BYTE      ADC0GTH
      000000C8H.7 SFRSYM    DATA     BIT       TMR2CN0_TF2H
      000000C8H.3 SFRSYM    DATA     BIT       TMR2CN0_T2SPLIT
      000000D0H.6 SFRSYM    DATA     BIT       PSW_AC
      000000F8H   SFRSYM    DATA     BYTE      SPI0CN0
      000000B3H   SFRSYM    DATA     BYTE      HFO0CAL
      00000088H.5 SFRSYM    DATA     BIT       TCON_TF0
      00000098H   SFRSYM    DATA     BIT       SCON0_RI
LX51 LINKER/LOCATER V4.66.30.0                                                        07/27/2019  23:22:19  PAGE 33


      00000082H   SFRSYM    DATA     BYTE      DPL
      00000088H.7 SFRSYM    DATA     BIT       TCON_TF1
      00000099H   SFRSYM    DATA     BYTE      SBUF0
      00000087H   SFRSYM    DATA     BYTE      PCON0
      000000C3H   SFRSYM    DATA     BYTE      ADC0GTL
      000000C8H.6 SFRSYM    DATA     BIT       TMR2CN0_TF2L
      00000098H.1 SFRSYM    DATA     BIT       SCON0_TI
      000000E8H   SFRSYM    DATA     BIT       ADC0CN0_ADCM0
      000000D3H   SFRSYM    DATA     BYTE      SBUF1
      000000C6H   SFRSYM    DATA     BYTE      ADC0LTH
      00000088H   SFRSYM    DATA     BIT       TCON_IT0
      000000E8H.1 SFRSYM    DATA     BIT       ADC0CN0_ADCM1
      000000EFH   SFRSYM    DATA     BYTE      RSTSRC
      000000C8H.7 SFRSYM    DATA     BIT       TMR5CN0_TF5H
      000000C8H.3 SFRSYM    DATA     BIT       TMR5CN0_T5SPLIT
      00000088H.2 SFRSYM    DATA     BIT       TCON_IT1
      000000E8H.2 SFRSYM    DATA     BIT       ADC0CN0_ADCM2
      00000098H   SFRSYM    DATA     BYTE      SCON0
      000000E8H.3 SFRSYM    DATA     BIT       ADC0CN0_ADWINT
      000000B4H   SFRSYM    DATA     WORD      SBRL1
      000000E5H   SFRSYM    DATA     BYTE      SMOD1
      000000D2H   SFRSYM    DATA     BYTE      SCON1
      000000BAH   SFRSYM    DATA     BYTE      AMX0N
      000000E8H.4 SFRSYM    DATA     BIT       ADC0CN0_ADBUSY
      000000CEH   SFRSYM    DATA     BYTE      SMB0ADM
      000000C5H   SFRSYM    DATA     BYTE      ADC0LTL
      000000F8H.5 SFRSYM    DATA     BIT       SPI0CN0_MODF
      000000B8H.6 SFRSYM    DATA     BIT       IP_PSPI0
      000000CEH   SFRSYM    DATA     BYTE      SMB1ADM
      000000BBH   SFRSYM    DATA     BYTE      AMX0P
      000000C8H.6 SFRSYM    DATA     BIT       TMR5CN0_TF5L
      000000C8H   SFRSYM    DATA     BYTE      TMR2CN0
      00000091H   SFRSYM    DATA     BYTE      TMR3CN0
      00000091H   SFRSYM    DATA     BYTE      TMR4CN0
      000000C8H   SFRSYM    DATA     BYTE      TMR5CN0
      000000CFH   SFRSYM    DATA     BYTE      SMB0ADR
      00000088H.4 SFRSYM    DATA     BIT       TCON_TR0
      000000CFH   SFRSYM    DATA     BYTE      SMB1ADR
      000000C8H.4 SFRSYM    DATA     BIT       TMR2CN0_TF2CEN
      00000088H.6 SFRSYM    DATA     BIT       TCON_TR1
      000000C2H   SFRSYM    DATA     BYTE      SMB0DAT
      000000CDH   SFRSYM    DATA     BYTE      TMR2H
      000000A1H   SFRSYM    DATA     BYTE      SPI0CFG
      000000C2H   SFRSYM    DATA     BYTE      SMB1DAT
      00000095H   SFRSYM    DATA     BYTE      TMR3H
      00000095H   SFRSYM    DATA     BYTE      TMR4H
      000000CDH   SFRSYM    DATA     BYTE      TMR5H
      000000CCH   SFRSYM    DATA     BYTE      TMR2L
      000000F8H.7 SFRSYM    DATA     BIT       SPI0CN0_SPIF
      00000096H   SFRSYM    DATA     BYTE      USB0ADR
      00000094H   SFRSYM    DATA     BYTE      TMR3L
      000000A8H.7 SFRSYM    DATA     BIT       IE_EA
      00000094H   SFRSYM    DATA     BYTE      TMR4L
      00000097H   SFRSYM    DATA     BYTE      USB0DAT
      000000CCH   SFRSYM    DATA     BYTE      TMR5L
      000000B6H   SFRSYM    DATA     BYTE      FLSCL
      000000C8H.5 SFRSYM    DATA     BIT       TMR2CN0_TF2LEN
      000000F8H.6 SFRSYM    DATA     BIT       SPI0CN0_WCOL
      000000F8H.2 SFRSYM    DATA     BIT       SPI0CN0_NSSMD0
      000000D0H.7 SFRSYM    DATA     BIT       PSW_CY
      000000A3H   SFRSYM    DATA     BYTE      SPI0DAT
      000000F8H.3 SFRSYM    DATA     BIT       SPI0CN0_NSSMD1
LX51 LINKER/LOCATER V4.66.30.0                                                        07/27/2019  23:22:19  PAGE 34


      000000BDH   SFRSYM    DATA     WORD      ADC0
      000000B9H   SFRSYM    DATA     BYTE      SMBTC
      000000D0H   SFRSYM    DATA     BYTE      PSW
      000000C8H.5 SFRSYM    DATA     BIT       TMR5CN0_TF5LEN
      000000B7H   SFRSYM    DATA     BYTE      FLKEY

      01005BB0H   BLOCK     CODE     ---       LVL=0
      01005BB0H   LINE      CODE     ---       #27
      01005BB0H   LINE      CODE     ---       #30
      ---         BLOCKEND  ---      ---       LVL=0

      010059A2H   BLOCK     CODE     ---       LVL=0
      010059A2H   LINE      CODE     ---       #35
      010059A2H   LINE      CODE     ---       #37
      010059A5H   LINE      CODE     ---       #39
      010059A8H   LINE      CODE     ---       #41
      010059A8H   LINE      CODE     ---       #44
      010059ABH   LINE      CODE     ---       #46
      010059AEH   LINE      CODE     ---       #47
      010059B0H   LINE      CODE     ---       #48
      010059B3H   LINE      CODE     ---       #49
      010059B3H   LINE      CODE     ---       #50
      ---         BLOCKEND  ---      ---       LVL=0

      ---         MODULE    ---      ---       INITDEVICE
      01005BA6H   PUBLIC    CODE     ---       UART_0_enter_DefaultMode_from_RESET
      010059C8H   PUBLIC    CODE     ---       TIMER01_0_enter_DefaultMode_from_RESET
      01005B74H   PUBLIC    CODE     ---       PCACH_4_enter_DefaultMode_from_RESET
      010059B5H   PUBLIC    CODE     ---       TIMER16_2_enter_DefaultMode_from_RESET
      0100008CH   PUBLIC    CODE     ---       SMBUS_1_enter_DefaultMode_from_RESET
      01005B35H   PUBLIC    CODE     ---       SMBUS_0_enter_DefaultMode_from_RESET
      0100593AH   PUBLIC    CODE     ---       TIMER_SETUP_0_enter_DefaultMode_from_RESET
      0100590EH   PUBLIC    CODE     ---       TIMER16_5_enter_DefaultMode_from_RESET
      01005B2BH   PUBLIC    CODE     ---       INTERRUPT_0_enter_DefaultMode_from_RESET
      01005BA2H   PUBLIC    CODE     ---       EXTINT_0_enter_DefaultMode_from_RESET
      01005A5AH   PUBLIC    CODE     ---       SPI_0_enter_DefaultMode_from_RESET
      01005B9EH   PUBLIC    CODE     ---       CLOCK_0_enter_DefaultMode_from_RESET
      01005B9AH   PUBLIC    CODE     ---       HFOSC_0_enter_DefaultMode_from_RESET
      01005B21H   PUBLIC    CODE     ---       ADC_0_enter_DefaultMode_from_RESET
      01005B17H   PUBLIC    CODE     ---       PBCFG_0_enter_DefaultMode_from_RESET
      01005BB1H   PUBLIC    CODE     ---       PORTS_3_enter_DefaultMode_from_RESET
      01005AB2H   PUBLIC    CODE     ---       PORTS_2_enter_DefaultMode_from_RESET
      01005B0DH   PUBLIC    CODE     ---       PORTS_1_enter_DefaultMode_from_RESET
      01005AA5H   PUBLIC    CODE     ---       PORTS_0_enter_DefaultMode_from_RESET
      01005B03H   PUBLIC    CODE     ---       PCACH_3_enter_DefaultMode_from_RESET
      01005AF9H   PUBLIC    CODE     ---       PCACH_2_enter_DefaultMode_from_RESET
      01005AEFH   PUBLIC    CODE     ---       PCACH_1_enter_DefaultMode_from_RESET
      01005AE5H   PUBLIC    CODE     ---       PCACH_0_enter_DefaultMode_from_RESET
      01000096H   PUBLIC    CODE     ---       PCA_0_enter_DefaultMode_from_RESET
      0100506DH   PUBLIC    CODE     ---       enter_DefaultMode_from_RESET
      000000A2H   SFRSYM    DATA     BYTE      SPI0CKR
      00000080H   SFRSYM    DATA     BYTE      P0
      000000D0H.2 SFRSYM    DATA     BIT       PSW_OV
      000000B1H   SFRSYM    DATA     BYTE      XOSC0CN
      00000090H   SFRSYM    DATA     BYTE      P1
      000000A0H   SFRSYM    DATA     BYTE      P2
      000000B0H   SFRSYM    DATA     BYTE      P3
      000000BCH   SFRSYM    DATA     BYTE      ADC0CF
      000000C8H   SFRSYM    DATA     BIT       TMR2CN0_T2XCLK
      000000C7H   SFRSYM    DATA     BYTE      P4
      000000C0H.7 SFRSYM    DATA     BIT       SMB0CN0_MASTER
      000000F9H   SFRSYM    DATA     WORD      PCA0
LX51 LINKER/LOCATER V4.66.30.0                                                        07/27/2019  23:22:19  PAGE 35


      000000E6H   SFRSYM    DATA     BYTE      EIE1
      000000C0H.7 SFRSYM    DATA     BIT       SMB1CN0_MASTER
      000000C0H.1 SFRSYM    DATA     BIT       SMB0CN0_ACK
      000000D7H   SFRSYM    DATA     BYTE      USB0XCN
      000000E7H   SFRSYM    DATA     BYTE      EIE2
      000000C0H.1 SFRSYM    DATA     BIT       SMB1CN0_ACK
      0000008FH   SFRSYM    DATA     BYTE      PSCTL
      000000E4H   SFRSYM    DATA     BYTE      IT01CF
      000000C8H   SFRSYM    DATA     BIT       TMR5CN0_T5XCLK
      000000C0H.6 SFRSYM    DATA     BIT       SMB0CN0_TXMODE
      000000C0H.6 SFRSYM    DATA     BIT       SMB1CN0_TXMODE
      000000BFH   SFRSYM    DATA     BYTE      SFRPAGE
      000000A4H   SFRSYM    DATA     BYTE      P0MDOUT
      000000A5H   SFRSYM    DATA     BYTE      P1MDOUT
      000000E8H.5 SFRSYM    DATA     BIT       ADC0CN0_ADINT
      000000CBH   SFRSYM    DATA     BYTE      TMR2RLH
      000000A6H   SFRSYM    DATA     BYTE      P2MDOUT
      000000A8H   SFRSYM    DATA     BYTE      IE
      00000093H   SFRSYM    DATA     BYTE      TMR3RLH
      000000A7H   SFRSYM    DATA     BYTE      P3MDOUT
      00000093H   SFRSYM    DATA     BYTE      TMR4RLH
      000000AEH   SFRSYM    DATA     BYTE      P4MDOUT
      000000F6H   SFRSYM    DATA     BYTE      EIP1
      000000CBH   SFRSYM    DATA     BYTE      TMR5RLH
      000000F7H   SFRSYM    DATA     BYTE      EIP2
      00000098H.2 SFRSYM    DATA     BIT       SCON0_RB8
      000000CAH   SFRSYM    DATA     BYTE      TMR2RLL
      000000FCH   SFRSYM    DATA     BYTE      PCA0CPH0
      00000092H   SFRSYM    DATA     BYTE      TMR3RLL
      000000EAH   SFRSYM    DATA     BYTE      PCA0CPH1
      00000098H.3 SFRSYM    DATA     BIT       SCON0_TB8
      000000F0H   SFRSYM    DATA     BIT       B_B0
      00000082H   SFRSYM    DATA     WORD      DP
      00000092H   SFRSYM    DATA     BYTE      TMR4RLL
      000000ECH   SFRSYM    DATA     BYTE      PCA0CPH2
      000000F0H.1 SFRSYM    DATA     BIT       B_B1
      000000C3H   SFRSYM    DATA     WORD      ADC0GT
      000000CAH   SFRSYM    DATA     BYTE      TMR5RLL
      000000EEH   SFRSYM    DATA     BYTE      PCA0CPH3
      000000F0H.2 SFRSYM    DATA     BIT       B_B2
      000000FBH   SFRSYM    DATA     BYTE      PCA0CPL0
      000000FEH   SFRSYM    DATA     BYTE      PCA0CPH4
      00000085H   SFRSYM    DATA     BYTE      EMI0CF
      000000F0H.3 SFRSYM    DATA     BIT       B_B3
      000000D9H   SFRSYM    DATA     BYTE      PCA0MD
      000000DAH   SFRSYM    DATA     BYTE      PCA0CPM0
      000000E9H   SFRSYM    DATA     BYTE      PCA0CPL1
      000000F0H.4 SFRSYM    DATA     BIT       B_B4
      000000DBH   SFRSYM    DATA     BYTE      PCA0CPM1
      000000EBH   SFRSYM    DATA     BYTE      PCA0CPL2
      000000F0H.5 SFRSYM    DATA     BIT       B_B5
      000000DCH   SFRSYM    DATA     BYTE      PCA0CPM2
      000000EDH   SFRSYM    DATA     BYTE      PCA0CPL3
      000000B8H   SFRSYM    DATA     BYTE      IP
      000000F0H.6 SFRSYM    DATA     BIT       B_B6
      000000C5H   SFRSYM    DATA     WORD      ADC0LT
      000000DDH   SFRSYM    DATA     BYTE      PCA0CPM3
      000000FDH   SFRSYM    DATA     BYTE      PCA0CPL4
      00000098H.5 SFRSYM    DATA     BIT       SCON0_MCE
      000000F0H.7 SFRSYM    DATA     BIT       B_B7
      000000DEH   SFRSYM    DATA     BYTE      PCA0CPM4
      000000E1H   SFRSYM    DATA     BYTE      XBR0
LX51 LINKER/LOCATER V4.66.30.0                                                        07/27/2019  23:22:19  PAGE 36


      000000C1H   SFRSYM    DATA     BYTE      SMB0CF
      000000E2H   SFRSYM    DATA     BYTE      XBR1
      000000C1H   SFRSYM    DATA     BYTE      SMB1CF
      000000AFH   SFRSYM    DATA     BYTE      PFE0CN
      000000AAH   SFRSYM    DATA     BYTE      EMI0CN
      000000C0H.5 SFRSYM    DATA     BIT       SMB0CN0_STA
      000000E3H   SFRSYM    DATA     BYTE      XBR2
      000000C0H.5 SFRSYM    DATA     BIT       SMB1CN0_STA
      000000E0H   SFRSYM    DATA     BIT       ACC_ACC0
      000000D1H   SFRSYM    DATA     BYTE      REF0CN
      000000B2H   SFRSYM    DATA     BYTE      HFO0CN
      0000008EH   SFRSYM    DATA     BYTE      CKCON0
      000000E0H.1 SFRSYM    DATA     BIT       ACC_ACC1
      000000E4H   SFRSYM    DATA     BYTE      CKCON1
      000000C8H.2 SFRSYM    DATA     BIT       TMR2CN0_TR2
      000000E0H.2 SFRSYM    DATA     BIT       ACC_ACC2
      000000E0H.3 SFRSYM    DATA     BIT       ACC_ACC3
      00000081H   SFRSYM    DATA     BYTE      SP
      0000009DH   SFRSYM    DATA     BYTE      CMP0MD
      000000E0H.4 SFRSYM    DATA     BIT       ACC_ACC4
      00000086H   SFRSYM    DATA     BYTE      LFO0CN
      00000084H   SFRSYM    DATA     BYTE      EMI0TC
      0000009CH   SFRSYM    DATA     BYTE      CMP1MD
      000000D8H   SFRSYM    DATA     BIT       PCA0CN0_CCF0
      000000E0H.5 SFRSYM    DATA     BIT       ACC_ACC5
      000000D8H.1 SFRSYM    DATA     BIT       PCA0CN0_CCF1
      000000E0H.6 SFRSYM    DATA     BIT       ACC_ACC6
      000000CCH   SFRSYM    DATA     WORD      TMR2
      000000D8H.2 SFRSYM    DATA     BIT       PCA0CN0_CCF2
      000000E0H.7 SFRSYM    DATA     BIT       ACC_ACC7
      00000094H   SFRSYM    DATA     WORD      TMR3
      000000C8H.2 SFRSYM    DATA     BIT       TMR5CN0_TR5
      000000D8H.3 SFRSYM    DATA     BIT       PCA0CN0_CCF3
      00000094H   SFRSYM    DATA     WORD      TMR4
      000000ACH   SFRSYM    DATA     BYTE      SBCON1
      000000D8H.4 SFRSYM    DATA     BIT       PCA0CN0_CCF4
      000000CCH   SFRSYM    DATA     WORD      TMR5
      000000C0H.3 SFRSYM    DATA     BIT       SMB0CN0_ACKRQ
      000000FFH   SFRSYM    DATA     BYTE      VDM0CN
      000000F1H   SFRSYM    DATA     BYTE      P0MDIN
      000000C0H.3 SFRSYM    DATA     BIT       SMB1CN0_ACKRQ
      00000098H.4 SFRSYM    DATA     BIT       SCON0_REN
      000000F2H   SFRSYM    DATA     BYTE      P1MDIN
      000000F3H   SFRSYM    DATA     BYTE      P2MDIN
      000000C0H.4 SFRSYM    DATA     BIT       SMB0CN0_STO
      000000F4H   SFRSYM    DATA     BYTE      P3MDIN
      000000C0H.4 SFRSYM    DATA     BIT       SMB1CN0_STO
      000000B5H   SFRSYM    DATA     BYTE      SBRLH1
      000000F5H   SFRSYM    DATA     BYTE      P4MDIN
      000000D0H.3 SFRSYM    DATA     BIT       PSW_RS0
      000000D8H.7 SFRSYM    DATA     BIT       PCA0CN0_CF
      000000F8H.4 SFRSYM    DATA     BIT       SPI0CN0_RXOVRN
      000000D0H.4 SFRSYM    DATA     BIT       PSW_RS1
      000000B4H   SFRSYM    DATA     BYTE      SBRLL1
      000000E8H.7 SFRSYM    DATA     BIT       ADC0CN0_ADEN
      00000089H   SFRSYM    DATA     BYTE      TMOD
      00000088H   SFRSYM    DATA     BYTE      TCON
      000000D0H   SFRSYM    DATA     BIT       PSW_PARITY
      000000A8H.4 SFRSYM    DATA     BIT       IE_ES0
      0000009FH   SFRSYM    DATA     BYTE      CMP0MX
      000000A8H.1 SFRSYM    DATA     BIT       IE_ET0
      0000009EH   SFRSYM    DATA     BYTE      CMP1MX
LX51 LINKER/LOCATER V4.66.30.0                                                        07/27/2019  23:22:19  PAGE 37


      000000A8H.3 SFRSYM    DATA     BIT       IE_ET1
      000000D4H   SFRSYM    DATA     BYTE      P0SKIP
      000000C8H.1 SFRSYM    DATA     BIT       TMR2CN0_T2CSS
      000000A8H.5 SFRSYM    DATA     BIT       IE_ET2
      000000D5H   SFRSYM    DATA     BYTE      P1SKIP
      000000D6H   SFRSYM    DATA     BYTE      P2SKIP
      000000E8H   SFRSYM    DATA     BYTE      ADC0CN0
      000000A8H   SFRSYM    DATA     BIT       IE_EX0
      000000DFH   SFRSYM    DATA     BYTE      P3SKIP
      000000D8H.6 SFRSYM    DATA     BIT       PCA0CN0_CR
      000000A8H.2 SFRSYM    DATA     BIT       IE_EX1
      00000098H.7 SFRSYM    DATA     BIT       SCON0_SMODE
      000000A9H   SFRSYM    DATA     BYTE      CLKSEL
      000000F8H   SFRSYM    DATA     BIT       SPI0CN0_SPIEN
      000000F0H   SFRSYM    DATA     BYTE      B
      000000BEH   SFRSYM    DATA     BYTE      ADC0H
      000000E8H.6 SFRSYM    DATA     BIT       ADC0CN0_ADTM
      000000CAH   SFRSYM    DATA     WORD      TMR2RL
      000000BDH   SFRSYM    DATA     BYTE      ADC0L
      00000092H   SFRSYM    DATA     WORD      TMR3RL
      00000092H   SFRSYM    DATA     WORD      TMR4RL
      000000D8H   SFRSYM    DATA     BYTE      PCA0CN0
      000000E0H   SFRSYM    DATA     BYTE      ACC
      000000CAH   SFRSYM    DATA     WORD      TMR5RL
      000000FBH   SFRSYM    DATA     WORD      PCA0CP0
      000000E9H   SFRSYM    DATA     WORD      PCA0CP1
      000000EBH   SFRSYM    DATA     WORD      PCA0CP2
      000000EDH   SFRSYM    DATA     WORD      PCA0CP3
      0000008CH   SFRSYM    DATA     BYTE      TH0
      000000B8H.4 SFRSYM    DATA     BIT       IP_PS0
      000000FDH   SFRSYM    DATA     WORD      PCA0CP4
      0000008DH   SFRSYM    DATA     BYTE      TH1
      000000FAH   SFRSYM    DATA     BYTE      PCA0H
      000000B8H.1 SFRSYM    DATA     BIT       IP_PT0
      000000B8H.3 SFRSYM    DATA     BIT       IP_PT1
      000000C0H.2 SFRSYM    DATA     BIT       SMB0CN0_ARBLOST
      000000B8H.5 SFRSYM    DATA     BIT       IP_PT2
      0000008AH   SFRSYM    DATA     BYTE      TL0
      000000F8H.1 SFRSYM    DATA     BIT       SPI0CN0_TXBMT
      000000C0H.2 SFRSYM    DATA     BIT       SMB1CN0_ARBLOST
      000000D0H.5 SFRSYM    DATA     BIT       PSW_F0
      000000A8H.6 SFRSYM    DATA     BIT       IE_ESPI0
      0000008BH   SFRSYM    DATA     BYTE      TL1
      000000F9H   SFRSYM    DATA     BYTE      PCA0L
      000000C0H   SFRSYM    DATA     BIT       SMB0CN0_SI
      000000D0H.1 SFRSYM    DATA     BIT       PSW_F1
      00000080H   SFRSYM    DATA     BIT       P0_B0
      000000B8H   SFRSYM    DATA     BIT       IP_PX0
      000000C9H   SFRSYM    DATA     BYTE      REG01CN
      000000C0H   SFRSYM    DATA     BIT       SMB1CN0_SI
      00000090H   SFRSYM    DATA     BIT       P1_B0
      00000080H.1 SFRSYM    DATA     BIT       P0_B1
      000000B8H.2 SFRSYM    DATA     BIT       IP_PX1
      0000009BH   SFRSYM    DATA     BYTE      CMP0CN0
      00000088H.1 SFRSYM    DATA     BIT       TCON_IE0
      000000A0H   SFRSYM    DATA     BIT       P2_B0
      00000090H.1 SFRSYM    DATA     BIT       P1_B1
      00000080H.2 SFRSYM    DATA     BIT       P0_B2
      0000009AH   SFRSYM    DATA     BYTE      CMP1CN0
      00000088H.3 SFRSYM    DATA     BIT       TCON_IE1
      000000B0H   SFRSYM    DATA     BIT       P3_B0
      000000A0H.1 SFRSYM    DATA     BIT       P2_B1
LX51 LINKER/LOCATER V4.66.30.0                                                        07/27/2019  23:22:19  PAGE 38


      00000090H.2 SFRSYM    DATA     BIT       P1_B2
      00000080H.3 SFRSYM    DATA     BIT       P0_B3
      000000C0H   SFRSYM    DATA     BYTE      SMB0CN0
      000000B0H.1 SFRSYM    DATA     BIT       P3_B1
      000000A0H.2 SFRSYM    DATA     BIT       P2_B2
      00000090H.3 SFRSYM    DATA     BIT       P1_B3
      00000080H.4 SFRSYM    DATA     BIT       P0_B4
      000000C0H   SFRSYM    DATA     BYTE      SMB1CN0
      000000B0H.2 SFRSYM    DATA     BIT       P3_B2
      000000A0H.3 SFRSYM    DATA     BIT       P2_B3
      00000090H.4 SFRSYM    DATA     BIT       P1_B4
      00000080H.5 SFRSYM    DATA     BIT       P0_B5
      000000B0H.3 SFRSYM    DATA     BIT       P3_B3
      000000A0H.4 SFRSYM    DATA     BIT       P2_B4
      00000090H.5 SFRSYM    DATA     BIT       P1_B5
      00000080H.6 SFRSYM    DATA     BIT       P0_B6
      000000B0H.4 SFRSYM    DATA     BIT       P3_B4
      000000A0H.5 SFRSYM    DATA     BIT       P2_B5
      00000090H.6 SFRSYM    DATA     BIT       P1_B6
      00000080H.7 SFRSYM    DATA     BIT       P0_B7
      000000B0H.5 SFRSYM    DATA     BIT       P3_B5
      000000A0H.6 SFRSYM    DATA     BIT       P2_B6
      00000090H.7 SFRSYM    DATA     BIT       P1_B7
      000000B0H.6 SFRSYM    DATA     BIT       P3_B6
      000000A0H.7 SFRSYM    DATA     BIT       P2_B7
      000000B0H.7 SFRSYM    DATA     BIT       P3_B7
      00000083H   SFRSYM    DATA     BYTE      DPH
      000000C4H   SFRSYM    DATA     BYTE      ADC0GTH
      000000C8H.7 SFRSYM    DATA     BIT       TMR2CN0_TF2H
      000000C8H.3 SFRSYM    DATA     BIT       TMR2CN0_T2SPLIT
      000000D0H.6 SFRSYM    DATA     BIT       PSW_AC
      000000F8H   SFRSYM    DATA     BYTE      SPI0CN0
      000000B3H   SFRSYM    DATA     BYTE      HFO0CAL
      00000088H.5 SFRSYM    DATA     BIT       TCON_TF0
      00000098H   SFRSYM    DATA     BIT       SCON0_RI
      00000082H   SFRSYM    DATA     BYTE      DPL
      00000088H.7 SFRSYM    DATA     BIT       TCON_TF1
      00000099H   SFRSYM    DATA     BYTE      SBUF0
      00000087H   SFRSYM    DATA     BYTE      PCON0
      000000C3H   SFRSYM    DATA     BYTE      ADC0GTL
      000000C8H.6 SFRSYM    DATA     BIT       TMR2CN0_TF2L
      00000098H.1 SFRSYM    DATA     BIT       SCON0_TI
      000000E8H   SFRSYM    DATA     BIT       ADC0CN0_ADCM0
      000000D3H   SFRSYM    DATA     BYTE      SBUF1
      000000C6H   SFRSYM    DATA     BYTE      ADC0LTH
      00000088H   SFRSYM    DATA     BIT       TCON_IT0
      000000E8H.1 SFRSYM    DATA     BIT       ADC0CN0_ADCM1
      000000EFH   SFRSYM    DATA     BYTE      RSTSRC
      000000C8H.7 SFRSYM    DATA     BIT       TMR5CN0_TF5H
      000000C8H.3 SFRSYM    DATA     BIT       TMR5CN0_T5SPLIT
      00000088H.2 SFRSYM    DATA     BIT       TCON_IT1
      000000E8H.2 SFRSYM    DATA     BIT       ADC0CN0_ADCM2
      00000098H   SFRSYM    DATA     BYTE      SCON0
      000000E8H.3 SFRSYM    DATA     BIT       ADC0CN0_ADWINT
      000000B4H   SFRSYM    DATA     WORD      SBRL1
      000000E5H   SFRSYM    DATA     BYTE      SMOD1
      000000D2H   SFRSYM    DATA     BYTE      SCON1
      000000BAH   SFRSYM    DATA     BYTE      AMX0N
      000000E8H.4 SFRSYM    DATA     BIT       ADC0CN0_ADBUSY
      000000CEH   SFRSYM    DATA     BYTE      SMB0ADM
      000000C5H   SFRSYM    DATA     BYTE      ADC0LTL
      000000F8H.5 SFRSYM    DATA     BIT       SPI0CN0_MODF
LX51 LINKER/LOCATER V4.66.30.0                                                        07/27/2019  23:22:19  PAGE 39


      000000B8H.6 SFRSYM    DATA     BIT       IP_PSPI0
      000000CEH   SFRSYM    DATA     BYTE      SMB1ADM
      000000BBH   SFRSYM    DATA     BYTE      AMX0P
      000000C8H.6 SFRSYM    DATA     BIT       TMR5CN0_TF5L
      000000C8H   SFRSYM    DATA     BYTE      TMR2CN0
      00000091H   SFRSYM    DATA     BYTE      TMR3CN0
      00000091H   SFRSYM    DATA     BYTE      TMR4CN0
      000000C8H   SFRSYM    DATA     BYTE      TMR5CN0
      000000CFH   SFRSYM    DATA     BYTE      SMB0ADR
      00000088H.4 SFRSYM    DATA     BIT       TCON_TR0
      000000CFH   SFRSYM    DATA     BYTE      SMB1ADR
      000000C8H.4 SFRSYM    DATA     BIT       TMR2CN0_TF2CEN
      00000088H.6 SFRSYM    DATA     BIT       TCON_TR1
      000000C2H   SFRSYM    DATA     BYTE      SMB0DAT
      000000CDH   SFRSYM    DATA     BYTE      TMR2H
      000000A1H   SFRSYM    DATA     BYTE      SPI0CFG
      000000C2H   SFRSYM    DATA     BYTE      SMB1DAT
      00000095H   SFRSYM    DATA     BYTE      TMR3H
      00000095H   SFRSYM    DATA     BYTE      TMR4H
      000000CDH   SFRSYM    DATA     BYTE      TMR5H
      000000CCH   SFRSYM    DATA     BYTE      TMR2L
      000000F8H.7 SFRSYM    DATA     BIT       SPI0CN0_SPIF
      00000096H   SFRSYM    DATA     BYTE      USB0ADR
      00000094H   SFRSYM    DATA     BYTE      TMR3L
      000000A8H.7 SFRSYM    DATA     BIT       IE_EA
      00000094H   SFRSYM    DATA     BYTE      TMR4L
      00000097H   SFRSYM    DATA     BYTE      USB0DAT
      000000CCH   SFRSYM    DATA     BYTE      TMR5L
      000000B6H   SFRSYM    DATA     BYTE      FLSCL
      000000C8H.5 SFRSYM    DATA     BIT       TMR2CN0_TF2LEN
      000000F8H.6 SFRSYM    DATA     BIT       SPI0CN0_WCOL
      000000F8H.2 SFRSYM    DATA     BIT       SPI0CN0_NSSMD0
      000000D0H.7 SFRSYM    DATA     BIT       PSW_CY
      000000A3H   SFRSYM    DATA     BYTE      SPI0DAT
      000000F8H.3 SFRSYM    DATA     BIT       SPI0CN0_NSSMD1
      000000BDH   SFRSYM    DATA     WORD      ADC0
      000000B9H   SFRSYM    DATA     BYTE      SMBTC
      000000D0H   SFRSYM    DATA     BYTE      PSW
      000000C8H.5 SFRSYM    DATA     BIT       TMR5CN0_TF5LEN
      000000B7H   SFRSYM    DATA     BYTE      FLKEY

      0100506DH   BLOCK     CODE     ---       LVL=0
      0100506DH   BLOCK     CODE     NEAR LAB  LVL=1
      00000022H   SYMBOL    DATA     BYTE      SFRPAGE_save
      ---         BLOCKEND  ---      ---       LVL=1
      0100506DH   LINE      CODE     ---       #22
      0100506DH   LINE      CODE     ---       #25
      01005070H   LINE      CODE     ---       #26
      01005073H   LINE      CODE     ---       #27
      01005076H   LINE      CODE     ---       #28
      01005079H   LINE      CODE     ---       #29
      0100507CH   LINE      CODE     ---       #30
      0100507FH   LINE      CODE     ---       #31
      01005082H   LINE      CODE     ---       #32
      01005085H   LINE      CODE     ---       #33
      01005088H   LINE      CODE     ---       #34
      0100508BH   LINE      CODE     ---       #35
      0100508EH   LINE      CODE     ---       #36
      01005091H   LINE      CODE     ---       #37
      01005094H   LINE      CODE     ---       #38
      01005097H   LINE      CODE     ---       #39
      0100509AH   LINE      CODE     ---       #40
LX51 LINKER/LOCATER V4.66.30.0                                                        07/27/2019  23:22:19  PAGE 40


      0100509DH   LINE      CODE     ---       #41
      010050A0H   LINE      CODE     ---       #42
      010050A3H   LINE      CODE     ---       #43
      010050A6H   LINE      CODE     ---       #44
      010050A9H   LINE      CODE     ---       #45
      010050ACH   LINE      CODE     ---       #46
      010050AFH   LINE      CODE     ---       #47
      010050B2H   LINE      CODE     ---       #48
      010050B5H   LINE      CODE     ---       #49
      010050B8H   LINE      CODE     ---       #51
      010050BBH   LINE      CODE     ---       #54
      ---         BLOCKEND  ---      ---       LVL=0

      01000096H   BLOCK     CODE     ---       LVL=0
      01000096H   LINE      CODE     ---       #56
      01000096H   LINE      CODE     ---       #67
      01000099H   LINE      CODE     ---       #68
      0100009CH   LINE      CODE     ---       #69
      0100009FH   LINE      CODE     ---       #84
      010000A2H   LINE      CODE     ---       #87
      ---         BLOCKEND  ---      ---       LVL=0

      01005AE5H   BLOCK     CODE     ---       LVL=0
      01005AE5H   LINE      CODE     ---       #89
      01005AE5H   LINE      CODE     ---       #101
      01005AE8H   LINE      CODE     ---       #111
      01005AEBH   LINE      CODE     ---       #118
      01005AEEH   LINE      CODE     ---       #124
      ---         BLOCKEND  ---      ---       LVL=0

      01005AEFH   BLOCK     CODE     ---       LVL=0
      01005AEFH   LINE      CODE     ---       #126
      01005AEFH   LINE      CODE     ---       #138
      01005AF2H   LINE      CODE     ---       #148
      01005AF5H   LINE      CODE     ---       #155
      01005AF8H   LINE      CODE     ---       #161
      ---         BLOCKEND  ---      ---       LVL=0

      01005AF9H   BLOCK     CODE     ---       LVL=0
      01005AF9H   LINE      CODE     ---       #163
      01005AF9H   LINE      CODE     ---       #175
      01005AFCH   LINE      CODE     ---       #185
      01005AFFH   LINE      CODE     ---       #192
      01005B02H   LINE      CODE     ---       #198
      ---         BLOCKEND  ---      ---       LVL=0

      01005B03H   BLOCK     CODE     ---       LVL=0
      01005B03H   LINE      CODE     ---       #200
      01005B03H   LINE      CODE     ---       #212
      01005B06H   LINE      CODE     ---       #222
      01005B09H   LINE      CODE     ---       #229
      01005B0CH   LINE      CODE     ---       #235
      ---         BLOCKEND  ---      ---       LVL=0

      01005AA5H   BLOCK     CODE     ---       LVL=0
      01005AA5H   LINE      CODE     ---       #237
      01005AA5H   LINE      CODE     ---       #249
      01005AA8H   LINE      CODE     ---       #264
      01005AABH   LINE      CODE     ---       #281
      01005AAEH   LINE      CODE     ---       #297
      01005AB1H   LINE      CODE     ---       #302
      ---         BLOCKEND  ---      ---       LVL=0
LX51 LINKER/LOCATER V4.66.30.0                                                        07/27/2019  23:22:19  PAGE 41



      01005B0DH   BLOCK     CODE     ---       LVL=0
      01005B0DH   LINE      CODE     ---       #304
      01005B0DH   LINE      CODE     ---       #316
      01005B10H   LINE      CODE     ---       #331
      01005B13H   LINE      CODE     ---       #351
      01005B16H   LINE      CODE     ---       #357
      ---         BLOCKEND  ---      ---       LVL=0

      01005AB2H   BLOCK     CODE     ---       LVL=0
      01005AB2H   LINE      CODE     ---       #359
      01005AB2H   LINE      CODE     ---       #371
      01005AB5H   LINE      CODE     ---       #386
      01005AB8H   LINE      CODE     ---       #403
      01005ABBH   LINE      CODE     ---       #419
      01005ABEH   LINE      CODE     ---       #425
      ---         BLOCKEND  ---      ---       LVL=0

      01005BB1H   BLOCK     CODE     ---       LVL=0
      01005BB1H   LINE      CODE     ---       #427
      01005BB1H   LINE      CODE     ---       #440
      ---         BLOCKEND  ---      ---       LVL=0

      01005B17H   BLOCK     CODE     ---       LVL=0
      01005B17H   LINE      CODE     ---       #442
      01005B17H   LINE      CODE     ---       #452
      01005B1AH   LINE      CODE     ---       #468
      01005B1DH   LINE      CODE     ---       #478
      01005B20H   LINE      CODE     ---       #481
      ---         BLOCKEND  ---      ---       LVL=0

      01005B21H   BLOCK     CODE     ---       LVL=0
      01005B21H   LINE      CODE     ---       #483
      01005B21H   LINE      CODE     ---       #489
      01005B24H   LINE      CODE     ---       #508
      01005B27H   LINE      CODE     ---       #515
      01005B2AH   LINE      CODE     ---       #521
      ---         BLOCKEND  ---      ---       LVL=0

      01005B9AH   BLOCK     CODE     ---       LVL=0
      01005B9AH   LINE      CODE     ---       #523
      01005B9AH   LINE      CODE     ---       #528
      01005B9DH   LINE      CODE     ---       #531
      ---         BLOCKEND  ---      ---       LVL=0

      01005B9EH   BLOCK     CODE     ---       LVL=0
      01005B9EH   LINE      CODE     ---       #549
      01005B9EH   LINE      CODE     ---       #557
      01005BA1H   LINE      CODE     ---       #561
      ---         BLOCKEND  ---      ---       LVL=0

      01005A5AH   BLOCK     CODE     ---       LVL=0
      01005A5AH   LINE      CODE     ---       #574
      01005A5AH   LINE      CODE     ---       #579
      01005A5DH   LINE      CODE     ---       #580
      01005A60H   LINE      CODE     ---       #589
      01005A63H   LINE      CODE     ---       #598
      01005A66H   LINE      CODE     ---       #599
      01005A69H   LINE      CODE     ---       #602
      ---         BLOCKEND  ---      ---       LVL=0

      01005BA2H   BLOCK     CODE     ---       LVL=0
LX51 LINKER/LOCATER V4.66.30.0                                                        07/27/2019  23:22:19  PAGE 42


      01005BA2H   LINE      CODE     ---       #604
      01005BA2H   LINE      CODE     ---       #612
      01005BA5H   LINE      CODE     ---       #616
      ---         BLOCKEND  ---      ---       LVL=0

      01005B2BH   BLOCK     CODE     ---       LVL=0
      01005B2BH   LINE      CODE     ---       #618
      01005B2BH   LINE      CODE     ---       #636
      01005B2EH   LINE      CODE     ---       #652
      01005B31H   LINE      CODE     ---       #664
      01005B34H   LINE      CODE     ---       #668
      ---         BLOCKEND  ---      ---       LVL=0

      0100590EH   BLOCK     CODE     ---       LVL=0
      0100590EH   BLOCK     CODE     NEAR LAB  LVL=1
      00000007H   SYMBOL    DATA     BYTE      TMR5CN0_TR5_save
      ---         BLOCKEND  ---      ---       LVL=1
      0100590EH   LINE      CODE     ---       #670
      0100590EH   LINE      CODE     ---       #674
      01005911H   LINE      CODE     ---       #675
      01005915H   LINE      CODE     ---       #677
      01005918H   LINE      CODE     ---       #693
      0100591BH   LINE      CODE     ---       #700
      0100591EH   LINE      CODE     ---       #707
      01005921H   LINE      CODE     ---       #712
      01005923H   LINE      CODE     ---       #715
      ---         BLOCKEND  ---      ---       LVL=0

      0100593AH   BLOCK     CODE     ---       LVL=0
      0100593AH   LINE      CODE     ---       #717
      0100593AH   LINE      CODE     ---       #728
      0100593DH   LINE      CODE     ---       #729
      01005940H   LINE      CODE     ---       #742
      01005943H   LINE      CODE     ---       #743
      01005946H   LINE      CODE     ---       #756
      01005948H   LINE      CODE     ---       #757
      0100594BH   LINE      CODE     ---       #767
      0100594EH   LINE      CODE     ---       #770
      ---         BLOCKEND  ---      ---       LVL=0

      01005B35H   BLOCK     CODE     ---       LVL=0
      01005B35H   LINE      CODE     ---       #772
      01005B35H   LINE      CODE     ---       #778
      01005B38H   LINE      CODE     ---       #787
      01005B3BH   LINE      CODE     ---       #797
      01005B3EH   LINE      CODE     ---       #801
      ---         BLOCKEND  ---      ---       LVL=0

      0100008CH   BLOCK     CODE     ---       LVL=0
      0100008CH   LINE      CODE     ---       #803
      0100008CH   LINE      CODE     ---       #817
      0100008FH   LINE      CODE     ---       #818
      01000092H   LINE      CODE     ---       #822
      ---         BLOCKEND  ---      ---       LVL=0
      00000007H   SYMBOL    DATA     BYTE      TMR4CN0_TR4_save

      010059B5H   BLOCK     CODE     ---       LVL=0
      010059B5H   BLOCK     CODE     NEAR LAB  LVL=1
      00000007H   SYMBOL    DATA     BYTE      TMR2CN0_TR2_save
      ---         BLOCKEND  ---      ---       LVL=1
      010059B5H   LINE      CODE     ---       #867
      010059B5H   LINE      CODE     ---       #871
LX51 LINKER/LOCATER V4.66.30.0                                                        07/27/2019  23:22:19  PAGE 43


      010059B9H   LINE      CODE     ---       #873
      010059BCH   LINE      CODE     ---       #889
      010059BFH   LINE      CODE     ---       #896
      010059C2H   LINE      CODE     ---       #903
      010059C5H   LINE      CODE     ---       #908
      010059C7H   LINE      CODE     ---       #911
      ---         BLOCKEND  ---      ---       LVL=0

      01005B74H   BLOCK     CODE     ---       LVL=0
      01005B74H   LINE      CODE     ---       #913
      01005B74H   LINE      CODE     ---       #925
      01005B77H   LINE      CODE     ---       #935
      01005B7AH   LINE      CODE     ---       #941
      ---         BLOCKEND  ---      ---       LVL=0

      010059C8H   BLOCK     CODE     ---       LVL=0
      010059C8H   BLOCK     CODE     NEAR LAB  LVL=1
      00000007H   SYMBOL    DATA     BYTE      TCON_save
      ---         BLOCKEND  ---      ---       LVL=1
      010059C8H   LINE      CODE     ---       #943
      010059C8H   LINE      CODE     ---       #947
      010059CAH   LINE      CODE     ---       #949
      010059CDH   LINE      CODE     ---       #963
      010059D0H   LINE      CODE     ---       #971
      010059DAH   LINE      CODE     ---       #975
      ---         BLOCKEND  ---      ---       LVL=0

      01005BA6H   BLOCK     CODE     ---       LVL=0
      01005BA6H   LINE      CODE     ---       #977
      01005BA6H   LINE      CODE     ---       #982
      01005BA9H   LINE      CODE     ---       #985
      ---         BLOCKEND  ---      ---       LVL=0

      ---         MODULE    ---      ---       INTERRUPTS
      01005453H   PUBLIC    CODE     ---       SMBUS1_ISR
      0100528BH   PUBLIC    CODE     ---       TIMER5_ISR
      01005BAAH   PUBLIC    CODE     ---       INT0_ISR
      000000A2H   SFRSYM    DATA     BYTE      SPI0CKR
      00000080H   SFRSYM    DATA     BYTE      P0
      000000D0H.2 SFRSYM    DATA     BIT       PSW_OV
      000000B1H   SFRSYM    DATA     BYTE      XOSC0CN
      00000090H   SFRSYM    DATA     BYTE      P1
      000000A0H   SFRSYM    DATA     BYTE      P2
      000000B0H   SFRSYM    DATA     BYTE      P3
      000000BCH   SFRSYM    DATA     BYTE      ADC0CF
      000000C8H   SFRSYM    DATA     BIT       TMR2CN0_T2XCLK
      000000C7H   SFRSYM    DATA     BYTE      P4
      000000C0H.7 SFRSYM    DATA     BIT       SMB0CN0_MASTER
      000000F9H   SFRSYM    DATA     WORD      PCA0
      000000E6H   SFRSYM    DATA     BYTE      EIE1
      000000C0H.7 SFRSYM    DATA     BIT       SMB1CN0_MASTER
      000000C0H.1 SFRSYM    DATA     BIT       SMB0CN0_ACK
      000000D7H   SFRSYM    DATA     BYTE      USB0XCN
      000000E7H   SFRSYM    DATA     BYTE      EIE2
      000000C0H.1 SFRSYM    DATA     BIT       SMB1CN0_ACK
      0000008FH   SFRSYM    DATA     BYTE      PSCTL
      000000E4H   SFRSYM    DATA     BYTE      IT01CF
      000000C8H   SFRSYM    DATA     BIT       TMR5CN0_T5XCLK
      000000C0H.6 SFRSYM    DATA     BIT       SMB0CN0_TXMODE
      000000C0H.6 SFRSYM    DATA     BIT       SMB1CN0_TXMODE
      000000BFH   SFRSYM    DATA     BYTE      SFRPAGE
      000000A4H   SFRSYM    DATA     BYTE      P0MDOUT
LX51 LINKER/LOCATER V4.66.30.0                                                        07/27/2019  23:22:19  PAGE 44


      000000A5H   SFRSYM    DATA     BYTE      P1MDOUT
      000000E8H.5 SFRSYM    DATA     BIT       ADC0CN0_ADINT
      000000CBH   SFRSYM    DATA     BYTE      TMR2RLH
      000000A6H   SFRSYM    DATA     BYTE      P2MDOUT
      000000A8H   SFRSYM    DATA     BYTE      IE
      00000093H   SFRSYM    DATA     BYTE      TMR3RLH
      000000A7H   SFRSYM    DATA     BYTE      P3MDOUT
      00000093H   SFRSYM    DATA     BYTE      TMR4RLH
      000000AEH   SFRSYM    DATA     BYTE      P4MDOUT
      000000F6H   SFRSYM    DATA     BYTE      EIP1
      000000CBH   SFRSYM    DATA     BYTE      TMR5RLH
      000000F7H   SFRSYM    DATA     BYTE      EIP2
      00000098H.2 SFRSYM    DATA     BIT       SCON0_RB8
      000000CAH   SFRSYM    DATA     BYTE      TMR2RLL
      000000FCH   SFRSYM    DATA     BYTE      PCA0CPH0
      00000092H   SFRSYM    DATA     BYTE      TMR3RLL
      000000EAH   SFRSYM    DATA     BYTE      PCA0CPH1
      00000098H.3 SFRSYM    DATA     BIT       SCON0_TB8
      000000F0H   SFRSYM    DATA     BIT       B_B0
      00000082H   SFRSYM    DATA     WORD      DP
      00000092H   SFRSYM    DATA     BYTE      TMR4RLL
      000000ECH   SFRSYM    DATA     BYTE      PCA0CPH2
      000000F0H.1 SFRSYM    DATA     BIT       B_B1
      000000C3H   SFRSYM    DATA     WORD      ADC0GT
      000000CAH   SFRSYM    DATA     BYTE      TMR5RLL
      000000EEH   SFRSYM    DATA     BYTE      PCA0CPH3
      000000F0H.2 SFRSYM    DATA     BIT       B_B2
      000000FBH   SFRSYM    DATA     BYTE      PCA0CPL0
      000000FEH   SFRSYM    DATA     BYTE      PCA0CPH4
      00000085H   SFRSYM    DATA     BYTE      EMI0CF
      000000F0H.3 SFRSYM    DATA     BIT       B_B3
      000000D9H   SFRSYM    DATA     BYTE      PCA0MD
      000000DAH   SFRSYM    DATA     BYTE      PCA0CPM0
      000000E9H   SFRSYM    DATA     BYTE      PCA0CPL1
      000000F0H.4 SFRSYM    DATA     BIT       B_B4
      000000DBH   SFRSYM    DATA     BYTE      PCA0CPM1
      000000EBH   SFRSYM    DATA     BYTE      PCA0CPL2
      000000F0H.5 SFRSYM    DATA     BIT       B_B5
      000000DCH   SFRSYM    DATA     BYTE      PCA0CPM2
      000000EDH   SFRSYM    DATA     BYTE      PCA0CPL3
      000000B8H   SFRSYM    DATA     BYTE      IP
      000000F0H.6 SFRSYM    DATA     BIT       B_B6
      000000C5H   SFRSYM    DATA     WORD      ADC0LT
      000000DDH   SFRSYM    DATA     BYTE      PCA0CPM3
      000000FDH   SFRSYM    DATA     BYTE      PCA0CPL4
      00000098H.5 SFRSYM    DATA     BIT       SCON0_MCE
      000000F0H.7 SFRSYM    DATA     BIT       B_B7
      000000DEH   SFRSYM    DATA     BYTE      PCA0CPM4
      000000E1H   SFRSYM    DATA     BYTE      XBR0
      000000C1H   SFRSYM    DATA     BYTE      SMB0CF
      000000E2H   SFRSYM    DATA     BYTE      XBR1
      000000C1H   SFRSYM    DATA     BYTE      SMB1CF
      000000AFH   SFRSYM    DATA     BYTE      PFE0CN
      000000AAH   SFRSYM    DATA     BYTE      EMI0CN
      000000C0H.5 SFRSYM    DATA     BIT       SMB0CN0_STA
      000000E3H   SFRSYM    DATA     BYTE      XBR2
      000000C0H.5 SFRSYM    DATA     BIT       SMB1CN0_STA
      000000E0H   SFRSYM    DATA     BIT       ACC_ACC0
      000000D1H   SFRSYM    DATA     BYTE      REF0CN
      000000B2H   SFRSYM    DATA     BYTE      HFO0CN
      0000008EH   SFRSYM    DATA     BYTE      CKCON0
      000000E0H.1 SFRSYM    DATA     BIT       ACC_ACC1
LX51 LINKER/LOCATER V4.66.30.0                                                        07/27/2019  23:22:19  PAGE 45


      000000E4H   SFRSYM    DATA     BYTE      CKCON1
      000000C8H.2 SFRSYM    DATA     BIT       TMR2CN0_TR2
      000000E0H.2 SFRSYM    DATA     BIT       ACC_ACC2
      000000E0H.3 SFRSYM    DATA     BIT       ACC_ACC3
      00000081H   SFRSYM    DATA     BYTE      SP
      0000009DH   SFRSYM    DATA     BYTE      CMP0MD
      000000E0H.4 SFRSYM    DATA     BIT       ACC_ACC4
      00000086H   SFRSYM    DATA     BYTE      LFO0CN
      00000084H   SFRSYM    DATA     BYTE      EMI0TC
      0000009CH   SFRSYM    DATA     BYTE      CMP1MD
      000000D8H   SFRSYM    DATA     BIT       PCA0CN0_CCF0
      000000E0H.5 SFRSYM    DATA     BIT       ACC_ACC5
      000000D8H.1 SFRSYM    DATA     BIT       PCA0CN0_CCF1
      000000E0H.6 SFRSYM    DATA     BIT       ACC_ACC6
      000000CCH   SFRSYM    DATA     WORD      TMR2
      000000D8H.2 SFRSYM    DATA     BIT       PCA0CN0_CCF2
      000000E0H.7 SFRSYM    DATA     BIT       ACC_ACC7
      00000094H   SFRSYM    DATA     WORD      TMR3
      000000C8H.2 SFRSYM    DATA     BIT       TMR5CN0_TR5
      000000D8H.3 SFRSYM    DATA     BIT       PCA0CN0_CCF3
      00000094H   SFRSYM    DATA     WORD      TMR4
      000000ACH   SFRSYM    DATA     BYTE      SBCON1
      000000D8H.4 SFRSYM    DATA     BIT       PCA0CN0_CCF4
      000000CCH   SFRSYM    DATA     WORD      TMR5
      000000C0H.3 SFRSYM    DATA     BIT       SMB0CN0_ACKRQ
      000000FFH   SFRSYM    DATA     BYTE      VDM0CN
      000000F1H   SFRSYM    DATA     BYTE      P0MDIN
      000000C0H.3 SFRSYM    DATA     BIT       SMB1CN0_ACKRQ
      00000098H.4 SFRSYM    DATA     BIT       SCON0_REN
      000000F2H   SFRSYM    DATA     BYTE      P1MDIN
      000000F3H   SFRSYM    DATA     BYTE      P2MDIN
      000000C0H.4 SFRSYM    DATA     BIT       SMB0CN0_STO
      000000F4H   SFRSYM    DATA     BYTE      P3MDIN
      000000C0H.4 SFRSYM    DATA     BIT       SMB1CN0_STO
      000000B5H   SFRSYM    DATA     BYTE      SBRLH1
      000000F5H   SFRSYM    DATA     BYTE      P4MDIN
      000000D0H.3 SFRSYM    DATA     BIT       PSW_RS0
      000000D8H.7 SFRSYM    DATA     BIT       PCA0CN0_CF
      000000F8H.4 SFRSYM    DATA     BIT       SPI0CN0_RXOVRN
      000000D0H.4 SFRSYM    DATA     BIT       PSW_RS1
      000000B4H   SFRSYM    DATA     BYTE      SBRLL1
      000000E8H.7 SFRSYM    DATA     BIT       ADC0CN0_ADEN
      00000089H   SFRSYM    DATA     BYTE      TMOD
      00000088H   SFRSYM    DATA     BYTE      TCON
      000000D0H   SFRSYM    DATA     BIT       PSW_PARITY
      000000A8H.4 SFRSYM    DATA     BIT       IE_ES0
      0000009FH   SFRSYM    DATA     BYTE      CMP0MX
      000000A8H.1 SFRSYM    DATA     BIT       IE_ET0
      0000009EH   SFRSYM    DATA     BYTE      CMP1MX
      000000A8H.3 SFRSYM    DATA     BIT       IE_ET1
      000000D4H   SFRSYM    DATA     BYTE      P0SKIP
      000000C8H.1 SFRSYM    DATA     BIT       TMR2CN0_T2CSS
      000000A8H.5 SFRSYM    DATA     BIT       IE_ET2
      000000D5H   SFRSYM    DATA     BYTE      P1SKIP
      000000D6H   SFRSYM    DATA     BYTE      P2SKIP
      000000E8H   SFRSYM    DATA     BYTE      ADC0CN0
      000000A8H   SFRSYM    DATA     BIT       IE_EX0
      000000DFH   SFRSYM    DATA     BYTE      P3SKIP
      000000D8H.6 SFRSYM    DATA     BIT       PCA0CN0_CR
      000000A8H.2 SFRSYM    DATA     BIT       IE_EX1
      00000098H.7 SFRSYM    DATA     BIT       SCON0_SMODE
      000000A9H   SFRSYM    DATA     BYTE      CLKSEL
LX51 LINKER/LOCATER V4.66.30.0                                                        07/27/2019  23:22:19  PAGE 46


      000000F8H   SFRSYM    DATA     BIT       SPI0CN0_SPIEN
      000000F0H   SFRSYM    DATA     BYTE      B
      000000BEH   SFRSYM    DATA     BYTE      ADC0H
      000000E8H.6 SFRSYM    DATA     BIT       ADC0CN0_ADTM
      000000CAH   SFRSYM    DATA     WORD      TMR2RL
      000000BDH   SFRSYM    DATA     BYTE      ADC0L
      00000092H   SFRSYM    DATA     WORD      TMR3RL
      00000092H   SFRSYM    DATA     WORD      TMR4RL
      000000D8H   SFRSYM    DATA     BYTE      PCA0CN0
      000000E0H   SFRSYM    DATA     BYTE      ACC
      000000CAH   SFRSYM    DATA     WORD      TMR5RL
      000000FBH   SFRSYM    DATA     WORD      PCA0CP0
      000000E9H   SFRSYM    DATA     WORD      PCA0CP1
      000000EBH   SFRSYM    DATA     WORD      PCA0CP2
      000000EDH   SFRSYM    DATA     WORD      PCA0CP3
      0000008CH   SFRSYM    DATA     BYTE      TH0
      000000B8H.4 SFRSYM    DATA     BIT       IP_PS0
      000000FDH   SFRSYM    DATA     WORD      PCA0CP4
      0000008DH   SFRSYM    DATA     BYTE      TH1
      000000FAH   SFRSYM    DATA     BYTE      PCA0H
      000000B8H.1 SFRSYM    DATA     BIT       IP_PT0
      000000B8H.3 SFRSYM    DATA     BIT       IP_PT1
      000000C0H.2 SFRSYM    DATA     BIT       SMB0CN0_ARBLOST
      000000B8H.5 SFRSYM    DATA     BIT       IP_PT2
      0000008AH   SFRSYM    DATA     BYTE      TL0
      000000F8H.1 SFRSYM    DATA     BIT       SPI0CN0_TXBMT
      000000C0H.2 SFRSYM    DATA     BIT       SMB1CN0_ARBLOST
      000000D0H.5 SFRSYM    DATA     BIT       PSW_F0
      000000A8H.6 SFRSYM    DATA     BIT       IE_ESPI0
      0000008BH   SFRSYM    DATA     BYTE      TL1
      000000F9H   SFRSYM    DATA     BYTE      PCA0L
      000000C0H   SFRSYM    DATA     BIT       SMB0CN0_SI
      000000D0H.1 SFRSYM    DATA     BIT       PSW_F1
      00000080H   SFRSYM    DATA     BIT       P0_B0
      000000B8H   SFRSYM    DATA     BIT       IP_PX0
      000000C9H   SFRSYM    DATA     BYTE      REG01CN
      000000C0H   SFRSYM    DATA     BIT       SMB1CN0_SI
      00000090H   SFRSYM    DATA     BIT       P1_B0
      00000080H.1 SFRSYM    DATA     BIT       P0_B1
      000000B8H.2 SFRSYM    DATA     BIT       IP_PX1
      0000009BH   SFRSYM    DATA     BYTE      CMP0CN0
      00000088H.1 SFRSYM    DATA     BIT       TCON_IE0
      000000A0H   SFRSYM    DATA     BIT       P2_B0
      00000090H.1 SFRSYM    DATA     BIT       P1_B1
      00000080H.2 SFRSYM    DATA     BIT       P0_B2
      0000009AH   SFRSYM    DATA     BYTE      CMP1CN0
      00000088H.3 SFRSYM    DATA     BIT       TCON_IE1
      000000B0H   SFRSYM    DATA     BIT       P3_B0
      000000A0H.1 SFRSYM    DATA     BIT       P2_B1
      00000090H.2 SFRSYM    DATA     BIT       P1_B2
      00000080H.3 SFRSYM    DATA     BIT       P0_B3
      000000C0H   SFRSYM    DATA     BYTE      SMB0CN0
      000000B0H.1 SFRSYM    DATA     BIT       P3_B1
      000000A0H.2 SFRSYM    DATA     BIT       P2_B2
      00000090H.3 SFRSYM    DATA     BIT       P1_B3
      00000080H.4 SFRSYM    DATA     BIT       P0_B4
      000000C0H   SFRSYM    DATA     BYTE      SMB1CN0
      000000B0H.2 SFRSYM    DATA     BIT       P3_B2
      000000A0H.3 SFRSYM    DATA     BIT       P2_B3
      00000090H.4 SFRSYM    DATA     BIT       P1_B4
      00000080H.5 SFRSYM    DATA     BIT       P0_B5
      000000B0H.3 SFRSYM    DATA     BIT       P3_B3
LX51 LINKER/LOCATER V4.66.30.0                                                        07/27/2019  23:22:19  PAGE 47


      000000A0H.4 SFRSYM    DATA     BIT       P2_B4
      00000090H.5 SFRSYM    DATA     BIT       P1_B5
      00000080H.6 SFRSYM    DATA     BIT       P0_B6
      000000B0H.4 SFRSYM    DATA     BIT       P3_B4
      000000A0H.5 SFRSYM    DATA     BIT       P2_B5
      00000090H.6 SFRSYM    DATA     BIT       P1_B6
      00000080H.7 SFRSYM    DATA     BIT       P0_B7
      000000B0H.5 SFRSYM    DATA     BIT       P3_B5
      000000A0H.6 SFRSYM    DATA     BIT       P2_B6
      00000090H.7 SFRSYM    DATA     BIT       P1_B7
      000000B0H.6 SFRSYM    DATA     BIT       P3_B6
      000000A0H.7 SFRSYM    DATA     BIT       P2_B7
      000000B0H.7 SFRSYM    DATA     BIT       P3_B7
      00000083H   SFRSYM    DATA     BYTE      DPH
      000000C4H   SFRSYM    DATA     BYTE      ADC0GTH
      000000C8H.7 SFRSYM    DATA     BIT       TMR2CN0_TF2H
      000000C8H.3 SFRSYM    DATA     BIT       TMR2CN0_T2SPLIT
      000000D0H.6 SFRSYM    DATA     BIT       PSW_AC
      000000F8H   SFRSYM    DATA     BYTE      SPI0CN0
      000000B3H   SFRSYM    DATA     BYTE      HFO0CAL
      00000088H.5 SFRSYM    DATA     BIT       TCON_TF0
      00000098H   SFRSYM    DATA     BIT       SCON0_RI
      00000082H   SFRSYM    DATA     BYTE      DPL
      00000088H.7 SFRSYM    DATA     BIT       TCON_TF1
      00000099H   SFRSYM    DATA     BYTE      SBUF0
      00000087H   SFRSYM    DATA     BYTE      PCON0
      000000C3H   SFRSYM    DATA     BYTE      ADC0GTL
      000000C8H.6 SFRSYM    DATA     BIT       TMR2CN0_TF2L
      00000098H.1 SFRSYM    DATA     BIT       SCON0_TI
      000000E8H   SFRSYM    DATA     BIT       ADC0CN0_ADCM0
      000000D3H   SFRSYM    DATA     BYTE      SBUF1
      000000C6H   SFRSYM    DATA     BYTE      ADC0LTH
      00000088H   SFRSYM    DATA     BIT       TCON_IT0
      000000E8H.1 SFRSYM    DATA     BIT       ADC0CN0_ADCM1
      000000EFH   SFRSYM    DATA     BYTE      RSTSRC
      000000C8H.7 SFRSYM    DATA     BIT       TMR5CN0_TF5H
      000000C8H.3 SFRSYM    DATA     BIT       TMR5CN0_T5SPLIT
      00000088H.2 SFRSYM    DATA     BIT       TCON_IT1
      000000E8H.2 SFRSYM    DATA     BIT       ADC0CN0_ADCM2
      00000098H   SFRSYM    DATA     BYTE      SCON0
      000000E8H.3 SFRSYM    DATA     BIT       ADC0CN0_ADWINT
      000000B4H   SFRSYM    DATA     WORD      SBRL1
      000000E5H   SFRSYM    DATA     BYTE      SMOD1
      000000D2H   SFRSYM    DATA     BYTE      SCON1
      000000BAH   SFRSYM    DATA     BYTE      AMX0N
      000000E8H.4 SFRSYM    DATA     BIT       ADC0CN0_ADBUSY
      000000CEH   SFRSYM    DATA     BYTE      SMB0ADM
      000000C5H   SFRSYM    DATA     BYTE      ADC0LTL
      000000F8H.5 SFRSYM    DATA     BIT       SPI0CN0_MODF
      000000B8H.6 SFRSYM    DATA     BIT       IP_PSPI0
      000000CEH   SFRSYM    DATA     BYTE      SMB1ADM
      000000BBH   SFRSYM    DATA     BYTE      AMX0P
      000000C8H.6 SFRSYM    DATA     BIT       TMR5CN0_TF5L
      000000C8H   SFRSYM    DATA     BYTE      TMR2CN0
      00000091H   SFRSYM    DATA     BYTE      TMR3CN0
      00000091H   SFRSYM    DATA     BYTE      TMR4CN0
      000000C8H   SFRSYM    DATA     BYTE      TMR5CN0
      000000CFH   SFRSYM    DATA     BYTE      SMB0ADR
      00000088H.4 SFRSYM    DATA     BIT       TCON_TR0
      000000CFH   SFRSYM    DATA     BYTE      SMB1ADR
      000000C8H.4 SFRSYM    DATA     BIT       TMR2CN0_TF2CEN
      00000088H.6 SFRSYM    DATA     BIT       TCON_TR1
LX51 LINKER/LOCATER V4.66.30.0                                                        07/27/2019  23:22:19  PAGE 48


      000000C2H   SFRSYM    DATA     BYTE      SMB0DAT
      000000CDH   SFRSYM    DATA     BYTE      TMR2H
      000000A1H   SFRSYM    DATA     BYTE      SPI0CFG
      000000C2H   SFRSYM    DATA     BYTE      SMB1DAT
      00000095H   SFRSYM    DATA     BYTE      TMR3H
      00000095H   SFRSYM    DATA     BYTE      TMR4H
      000000CDH   SFRSYM    DATA     BYTE      TMR5H
      000000CCH   SFRSYM    DATA     BYTE      TMR2L
      000000F8H.7 SFRSYM    DATA     BIT       SPI0CN0_SPIF
      00000096H   SFRSYM    DATA     BYTE      USB0ADR
      00000094H   SFRSYM    DATA     BYTE      TMR3L
      000000A8H.7 SFRSYM    DATA     BIT       IE_EA
      00000094H   SFRSYM    DATA     BYTE      TMR4L
      00000097H   SFRSYM    DATA     BYTE      USB0DAT
      000000CCH   SFRSYM    DATA     BYTE      TMR5L
      000000B6H   SFRSYM    DATA     BYTE      FLSCL
      000000C8H.5 SFRSYM    DATA     BIT       TMR2CN0_TF2LEN
      000000F8H.6 SFRSYM    DATA     BIT       SPI0CN0_WCOL
      000000F8H.2 SFRSYM    DATA     BIT       SPI0CN0_NSSMD0
      000000D0H.7 SFRSYM    DATA     BIT       PSW_CY
      000000A3H   SFRSYM    DATA     BYTE      SPI0DAT
      000000F8H.3 SFRSYM    DATA     BIT       SPI0CN0_NSSMD1
      000000BDH   SFRSYM    DATA     WORD      ADC0
      000000B9H   SFRSYM    DATA     BYTE      SMBTC
      000000D0H   SFRSYM    DATA     BYTE      PSW
      000000C8H.5 SFRSYM    DATA     BIT       TMR5CN0_TF5LEN
      000000B7H   SFRSYM    DATA     BYTE      FLKEY

      01005BAAH   BLOCK     CODE     ---       LVL=0
      01005BAAH   LINE      CODE     ---       #23
      01005BAAH   LINE      CODE     ---       #25
      01005BACH   LINE      CODE     ---       #26
      ---         BLOCKEND  ---      ---       LVL=0

      0100528BH   BLOCK     CODE     ---       LVL=0
      010052A8H   BLOCK     CODE     NEAR LAB  LVL=1
      00000007H   SYMBOL    DATA     BYTE      sfrsave
      ---         BLOCKEND  ---      ---       LVL=1
      0100528BH   LINE      CODE     ---       #37
      010052A8H   LINE      CODE     ---       #41
      010052AAH   LINE      CODE     ---       #42
      010052ADH   LINE      CODE     ---       #44
      010052AFH   LINE      CODE     ---       #45
      010052B2H   LINE      CODE     ---       #48
      010052B4H   LINE      CODE     ---       #50
      010052B6H   LINE      CODE     ---       #51
      ---         BLOCKEND  ---      ---       LVL=0

      01005453H   BLOCK     CODE     ---       LVL=0
      01005453H   LINE      CODE     ---       #60
      01005470H   LINE      CODE     ---       #62
      01005473H   LINE      CODE     ---       #63
      ---         BLOCKEND  ---      ---       LVL=0

      ---         MODULE    ---      ---       FW
      00000083H   PUBLIC    IDATA    BYTE      cpu_use
      00000082H   PUBLIC    IDATA    BYTE      cpu_max
      00000017H   PUBLIC    DATA     BYTE      tick_ctr
      00000021H.2 PUBLIC    BIT      BIT       fw_interrupt
      00000021H.1 PUBLIC    BIT      BIT       fw_loop_busy
      00000013H   PUBLIC    DATA     DWORD     uptime
      00000081H   PUBLIC    IDATA    BYTE      missed
LX51 LINKER/LOCATER V4.66.30.0                                                        07/27/2019  23:22:19  PAGE 49


      0100D080H   PUBLIC    CONST    ---       ver
      010048CBH   PUBLIC    CODE     ---       fw_tick_mainloop
      010026D2H   PUBLIC    CODE     ---       fw_tick_critical
      010049D2H   PUBLIC    CODE     ---       fw_init
      01003877H   PUBLIC    CODE     ---       fw_oled_update_done
      000000A2H   SFRSYM    DATA     BYTE      SPI0CKR
      00000080H   SFRSYM    DATA     BYTE      P0
      000000D0H.2 SFRSYM    DATA     BIT       PSW_OV
      000000B1H   SFRSYM    DATA     BYTE      XOSC0CN
      00000090H   SFRSYM    DATA     BYTE      P1
      000000A0H   SFRSYM    DATA     BYTE      P2
      000000B0H   SFRSYM    DATA     BYTE      P3
      000000BCH   SFRSYM    DATA     BYTE      ADC0CF
      000000C8H   SFRSYM    DATA     BIT       TMR2CN0_T2XCLK
      000000C7H   SFRSYM    DATA     BYTE      P4
      000000C0H.7 SFRSYM    DATA     BIT       SMB0CN0_MASTER
      000000F9H   SFRSYM    DATA     WORD      PCA0
      000000E6H   SFRSYM    DATA     BYTE      EIE1
      000000C0H.7 SFRSYM    DATA     BIT       SMB1CN0_MASTER
      000000C0H.1 SFRSYM    DATA     BIT       SMB0CN0_ACK
      000000D7H   SFRSYM    DATA     BYTE      USB0XCN
      000000E7H   SFRSYM    DATA     BYTE      EIE2
      000000C0H.1 SFRSYM    DATA     BIT       SMB1CN0_ACK
      0000008FH   SFRSYM    DATA     BYTE      PSCTL
      000000E4H   SFRSYM    DATA     BYTE      IT01CF
      000000C8H   SFRSYM    DATA     BIT       TMR5CN0_T5XCLK
      000000C0H.6 SFRSYM    DATA     BIT       SMB0CN0_TXMODE
      000000C0H.6 SFRSYM    DATA     BIT       SMB1CN0_TXMODE
      000000BFH   SFRSYM    DATA     BYTE      SFRPAGE
      000000A4H   SFRSYM    DATA     BYTE      P0MDOUT
      000000A5H   SFRSYM    DATA     BYTE      P1MDOUT
      000000E8H.5 SFRSYM    DATA     BIT       ADC0CN0_ADINT
      000000CBH   SFRSYM    DATA     BYTE      TMR2RLH
      000000A6H   SFRSYM    DATA     BYTE      P2MDOUT
      000000A8H   SFRSYM    DATA     BYTE      IE
      00000093H   SFRSYM    DATA     BYTE      TMR3RLH
      000000A7H   SFRSYM    DATA     BYTE      P3MDOUT
      00000093H   SFRSYM    DATA     BYTE      TMR4RLH
      000000AEH   SFRSYM    DATA     BYTE      P4MDOUT
      000000F6H   SFRSYM    DATA     BYTE      EIP1
      000000CBH   SFRSYM    DATA     BYTE      TMR5RLH
      000000F7H   SFRSYM    DATA     BYTE      EIP2
      00000098H.2 SFRSYM    DATA     BIT       SCON0_RB8
      000000CAH   SFRSYM    DATA     BYTE      TMR2RLL
      000000FCH   SFRSYM    DATA     BYTE      PCA0CPH0
      00000092H   SFRSYM    DATA     BYTE      TMR3RLL
      000000EAH   SFRSYM    DATA     BYTE      PCA0CPH1
      00000098H.3 SFRSYM    DATA     BIT       SCON0_TB8
      000000F0H   SFRSYM    DATA     BIT       B_B0
      00000082H   SFRSYM    DATA     WORD      DP
      00000092H   SFRSYM    DATA     BYTE      TMR4RLL
      000000ECH   SFRSYM    DATA     BYTE      PCA0CPH2
      000000F0H.1 SFRSYM    DATA     BIT       B_B1
      000000C3H   SFRSYM    DATA     WORD      ADC0GT
      000000CAH   SFRSYM    DATA     BYTE      TMR5RLL
      000000EEH   SFRSYM    DATA     BYTE      PCA0CPH3
      000000F0H.2 SFRSYM    DATA     BIT       B_B2
      000000FBH   SFRSYM    DATA     BYTE      PCA0CPL0
      000000FEH   SFRSYM    DATA     BYTE      PCA0CPH4
      00000085H   SFRSYM    DATA     BYTE      EMI0CF
      000000F0H.3 SFRSYM    DATA     BIT       B_B3
      000000D9H   SFRSYM    DATA     BYTE      PCA0MD
LX51 LINKER/LOCATER V4.66.30.0                                                        07/27/2019  23:22:19  PAGE 50


      000000DAH   SFRSYM    DATA     BYTE      PCA0CPM0
      000000E9H   SFRSYM    DATA     BYTE      PCA0CPL1
      000000F0H.4 SFRSYM    DATA     BIT       B_B4
      000000DBH   SFRSYM    DATA     BYTE      PCA0CPM1
      000000EBH   SFRSYM    DATA     BYTE      PCA0CPL2
      000000F0H.5 SFRSYM    DATA     BIT       B_B5
      000000DCH   SFRSYM    DATA     BYTE      PCA0CPM2
      000000EDH   SFRSYM    DATA     BYTE      PCA0CPL3
      000000B8H   SFRSYM    DATA     BYTE      IP
      000000F0H.6 SFRSYM    DATA     BIT       B_B6
      000000C5H   SFRSYM    DATA     WORD      ADC0LT
      000000DDH   SFRSYM    DATA     BYTE      PCA0CPM3
      000000FDH   SFRSYM    DATA     BYTE      PCA0CPL4
      00000098H.5 SFRSYM    DATA     BIT       SCON0_MCE
      000000F0H.7 SFRSYM    DATA     BIT       B_B7
      000000DEH   SFRSYM    DATA     BYTE      PCA0CPM4
      000000E1H   SFRSYM    DATA     BYTE      XBR0
      000000C1H   SFRSYM    DATA     BYTE      SMB0CF
      000000E2H   SFRSYM    DATA     BYTE      XBR1
      000000C1H   SFRSYM    DATA     BYTE      SMB1CF
      000000AFH   SFRSYM    DATA     BYTE      PFE0CN
      000000AAH   SFRSYM    DATA     BYTE      EMI0CN
      000000C0H.5 SFRSYM    DATA     BIT       SMB0CN0_STA
      000000E3H   SFRSYM    DATA     BYTE      XBR2
      000000C0H.5 SFRSYM    DATA     BIT       SMB1CN0_STA
      000000E0H   SFRSYM    DATA     BIT       ACC_ACC0
      000000D1H   SFRSYM    DATA     BYTE      REF0CN
      000000B2H   SFRSYM    DATA     BYTE      HFO0CN
      0000008EH   SFRSYM    DATA     BYTE      CKCON0
      000000E0H.1 SFRSYM    DATA     BIT       ACC_ACC1
      000000E4H   SFRSYM    DATA     BYTE      CKCON1
      000000C8H.2 SFRSYM    DATA     BIT       TMR2CN0_TR2
      000000E0H.2 SFRSYM    DATA     BIT       ACC_ACC2
      000000E0H.3 SFRSYM    DATA     BIT       ACC_ACC3
      00000081H   SFRSYM    DATA     BYTE      SP
      0000009DH   SFRSYM    DATA     BYTE      CMP0MD
      000000E0H.4 SFRSYM    DATA     BIT       ACC_ACC4
      00000086H   SFRSYM    DATA     BYTE      LFO0CN
      00000084H   SFRSYM    DATA     BYTE      EMI0TC
      0000009CH   SFRSYM    DATA     BYTE      CMP1MD
      000000D8H   SFRSYM    DATA     BIT       PCA0CN0_CCF0
      000000E0H.5 SFRSYM    DATA     BIT       ACC_ACC5
      000000D8H.1 SFRSYM    DATA     BIT       PCA0CN0_CCF1
      000000E0H.6 SFRSYM    DATA     BIT       ACC_ACC6
      000000CCH   SFRSYM    DATA     WORD      TMR2
      000000D8H.2 SFRSYM    DATA     BIT       PCA0CN0_CCF2
      000000E0H.7 SFRSYM    DATA     BIT       ACC_ACC7
      00000094H   SFRSYM    DATA     WORD      TMR3
      000000C8H.2 SFRSYM    DATA     BIT       TMR5CN0_TR5
      000000D8H.3 SFRSYM    DATA     BIT       PCA0CN0_CCF3
      00000094H   SFRSYM    DATA     WORD      TMR4
      000000ACH   SFRSYM    DATA     BYTE      SBCON1
      000000D8H.4 SFRSYM    DATA     BIT       PCA0CN0_CCF4
      000000CCH   SFRSYM    DATA     WORD      TMR5
      000000C0H.3 SFRSYM    DATA     BIT       SMB0CN0_ACKRQ
      000000FFH   SFRSYM    DATA     BYTE      VDM0CN
      000000F1H   SFRSYM    DATA     BYTE      P0MDIN
      000000C0H.3 SFRSYM    DATA     BIT       SMB1CN0_ACKRQ
      00000098H.4 SFRSYM    DATA     BIT       SCON0_REN
      000000F2H   SFRSYM    DATA     BYTE      P1MDIN
      000000F3H   SFRSYM    DATA     BYTE      P2MDIN
      000000C0H.4 SFRSYM    DATA     BIT       SMB0CN0_STO
LX51 LINKER/LOCATER V4.66.30.0                                                        07/27/2019  23:22:19  PAGE 51


      000000F4H   SFRSYM    DATA     BYTE      P3MDIN
      000000C0H.4 SFRSYM    DATA     BIT       SMB1CN0_STO
      000000B5H   SFRSYM    DATA     BYTE      SBRLH1
      000000F5H   SFRSYM    DATA     BYTE      P4MDIN
      000000D0H.3 SFRSYM    DATA     BIT       PSW_RS0
      000000D8H.7 SFRSYM    DATA     BIT       PCA0CN0_CF
      000000F8H.4 SFRSYM    DATA     BIT       SPI0CN0_RXOVRN
      000000D0H.4 SFRSYM    DATA     BIT       PSW_RS1
      000000B4H   SFRSYM    DATA     BYTE      SBRLL1
      000000E8H.7 SFRSYM    DATA     BIT       ADC0CN0_ADEN
      00000089H   SFRSYM    DATA     BYTE      TMOD
      00000088H   SFRSYM    DATA     BYTE      TCON
      000000D0H   SFRSYM    DATA     BIT       PSW_PARITY
      000000A8H.4 SFRSYM    DATA     BIT       IE_ES0
      0000009FH   SFRSYM    DATA     BYTE      CMP0MX
      000000A8H.1 SFRSYM    DATA     BIT       IE_ET0
      0000009EH   SFRSYM    DATA     BYTE      CMP1MX
      000000A8H.3 SFRSYM    DATA     BIT       IE_ET1
      000000D4H   SFRSYM    DATA     BYTE      P0SKIP
      000000C8H.1 SFRSYM    DATA     BIT       TMR2CN0_T2CSS
      000000A8H.5 SFRSYM    DATA     BIT       IE_ET2
      000000D5H   SFRSYM    DATA     BYTE      P1SKIP
      000000D6H   SFRSYM    DATA     BYTE      P2SKIP
      000000E8H   SFRSYM    DATA     BYTE      ADC0CN0
      000000A8H   SFRSYM    DATA     BIT       IE_EX0
      000000DFH   SFRSYM    DATA     BYTE      P3SKIP
      000000D8H.6 SFRSYM    DATA     BIT       PCA0CN0_CR
      000000A8H.2 SFRSYM    DATA     BIT       IE_EX1
      00000098H.7 SFRSYM    DATA     BIT       SCON0_SMODE
      000000A9H   SFRSYM    DATA     BYTE      CLKSEL
      000000F8H   SFRSYM    DATA     BIT       SPI0CN0_SPIEN
      000000F0H   SFRSYM    DATA     BYTE      B
      000000BEH   SFRSYM    DATA     BYTE      ADC0H
      000000E8H.6 SFRSYM    DATA     BIT       ADC0CN0_ADTM
      000000CAH   SFRSYM    DATA     WORD      TMR2RL
      000000BDH   SFRSYM    DATA     BYTE      ADC0L
      00000092H   SFRSYM    DATA     WORD      TMR3RL
      00000092H   SFRSYM    DATA     WORD      TMR4RL
      000000D8H   SFRSYM    DATA     BYTE      PCA0CN0
      000000E0H   SFRSYM    DATA     BYTE      ACC
      000000CAH   SFRSYM    DATA     WORD      TMR5RL
      000000FBH   SFRSYM    DATA     WORD      PCA0CP0
      000000E9H   SFRSYM    DATA     WORD      PCA0CP1
      000000EBH   SFRSYM    DATA     WORD      PCA0CP2
      000000EDH   SFRSYM    DATA     WORD      PCA0CP3
      0000008CH   SFRSYM    DATA     BYTE      TH0
      000000B8H.4 SFRSYM    DATA     BIT       IP_PS0
      000000FDH   SFRSYM    DATA     WORD      PCA0CP4
      0000008DH   SFRSYM    DATA     BYTE      TH1
      000000FAH   SFRSYM    DATA     BYTE      PCA0H
      000000B8H.1 SFRSYM    DATA     BIT       IP_PT0
      000000B8H.3 SFRSYM    DATA     BIT       IP_PT1
      000000C0H.2 SFRSYM    DATA     BIT       SMB0CN0_ARBLOST
      000000B8H.5 SFRSYM    DATA     BIT       IP_PT2
      0000008AH   SFRSYM    DATA     BYTE      TL0
      000000F8H.1 SFRSYM    DATA     BIT       SPI0CN0_TXBMT
      000000C0H.2 SFRSYM    DATA     BIT       SMB1CN0_ARBLOST
      000000D0H.5 SFRSYM    DATA     BIT       PSW_F0
      000000A8H.6 SFRSYM    DATA     BIT       IE_ESPI0
      0000008BH   SFRSYM    DATA     BYTE      TL1
      000000F9H   SFRSYM    DATA     BYTE      PCA0L
      000000C0H   SFRSYM    DATA     BIT       SMB0CN0_SI
LX51 LINKER/LOCATER V4.66.30.0                                                        07/27/2019  23:22:19  PAGE 52


      000000D0H.1 SFRSYM    DATA     BIT       PSW_F1
      00000080H   SFRSYM    DATA     BIT       P0_B0
      000000B8H   SFRSYM    DATA     BIT       IP_PX0
      000000C9H   SFRSYM    DATA     BYTE      REG01CN
      000000C0H   SFRSYM    DATA     BIT       SMB1CN0_SI
      00000090H   SFRSYM    DATA     BIT       P1_B0
      00000080H.1 SFRSYM    DATA     BIT       P0_B1
      000000B8H.2 SFRSYM    DATA     BIT       IP_PX1
      0000009BH   SFRSYM    DATA     BYTE      CMP0CN0
      00000088H.1 SFRSYM    DATA     BIT       TCON_IE0
      000000A0H   SFRSYM    DATA     BIT       P2_B0
      00000090H.1 SFRSYM    DATA     BIT       P1_B1
      00000080H.2 SFRSYM    DATA     BIT       P0_B2
      0000009AH   SFRSYM    DATA     BYTE      CMP1CN0
      00000088H.3 SFRSYM    DATA     BIT       TCON_IE1
      000000B0H   SFRSYM    DATA     BIT       P3_B0
      000000A0H.1 SFRSYM    DATA     BIT       P2_B1
      00000090H.2 SFRSYM    DATA     BIT       P1_B2
      00000080H.3 SFRSYM    DATA     BIT       P0_B3
      000000C0H   SFRSYM    DATA     BYTE      SMB0CN0
      000000B0H.1 SFRSYM    DATA     BIT       P3_B1
      000000A0H.2 SFRSYM    DATA     BIT       P2_B2
      00000090H.3 SFRSYM    DATA     BIT       P1_B3
      00000080H.4 SFRSYM    DATA     BIT       P0_B4
      000000C0H   SFRSYM    DATA     BYTE      SMB1CN0
      000000B0H.2 SFRSYM    DATA     BIT       P3_B2
      000000A0H.3 SFRSYM    DATA     BIT       P2_B3
      00000090H.4 SFRSYM    DATA     BIT       P1_B4
      00000080H.5 SFRSYM    DATA     BIT       P0_B5
      000000B0H.3 SFRSYM    DATA     BIT       P3_B3
      000000A0H.4 SFRSYM    DATA     BIT       P2_B4
      00000090H.5 SFRSYM    DATA     BIT       P1_B5
      00000080H.6 SFRSYM    DATA     BIT       P0_B6
      000000B0H.4 SFRSYM    DATA     BIT       P3_B4
      000000A0H.5 SFRSYM    DATA     BIT       P2_B5
      00000090H.6 SFRSYM    DATA     BIT       P1_B6
      00000080H.7 SFRSYM    DATA     BIT       P0_B7
      000000B0H.5 SFRSYM    DATA     BIT       P3_B5
      000000A0H.6 SFRSYM    DATA     BIT       P2_B6
      00000090H.7 SFRSYM    DATA     BIT       P1_B7
      000000B0H.6 SFRSYM    DATA     BIT       P3_B6
      000000A0H.7 SFRSYM    DATA     BIT       P2_B7
      000000B0H.7 SFRSYM    DATA     BIT       P3_B7
      00000083H   SFRSYM    DATA     BYTE      DPH
      000000C4H   SFRSYM    DATA     BYTE      ADC0GTH
      000000C8H.7 SFRSYM    DATA     BIT       TMR2CN0_TF2H
      000000C8H.3 SFRSYM    DATA     BIT       TMR2CN0_T2SPLIT
      000000D0H.6 SFRSYM    DATA     BIT       PSW_AC
      000000F8H   SFRSYM    DATA     BYTE      SPI0CN0
      000000B3H   SFRSYM    DATA     BYTE      HFO0CAL
      00000088H.5 SFRSYM    DATA     BIT       TCON_TF0
      00000098H   SFRSYM    DATA     BIT       SCON0_RI
      00000082H   SFRSYM    DATA     BYTE      DPL
      00000088H.7 SFRSYM    DATA     BIT       TCON_TF1
      00000099H   SFRSYM    DATA     BYTE      SBUF0
      00000087H   SFRSYM    DATA     BYTE      PCON0
      000000C3H   SFRSYM    DATA     BYTE      ADC0GTL
      000000C8H.6 SFRSYM    DATA     BIT       TMR2CN0_TF2L
      00000098H.1 SFRSYM    DATA     BIT       SCON0_TI
      000000E8H   SFRSYM    DATA     BIT       ADC0CN0_ADCM0
      000000D3H   SFRSYM    DATA     BYTE      SBUF1
      000000C6H   SFRSYM    DATA     BYTE      ADC0LTH
LX51 LINKER/LOCATER V4.66.30.0                                                        07/27/2019  23:22:19  PAGE 53


      00000088H   SFRSYM    DATA     BIT       TCON_IT0
      000000E8H.1 SFRSYM    DATA     BIT       ADC0CN0_ADCM1
      000000EFH   SFRSYM    DATA     BYTE      RSTSRC
      000000C8H.7 SFRSYM    DATA     BIT       TMR5CN0_TF5H
      000000C8H.3 SFRSYM    DATA     BIT       TMR5CN0_T5SPLIT
      00000088H.2 SFRSYM    DATA     BIT       TCON_IT1
      000000E8H.2 SFRSYM    DATA     BIT       ADC0CN0_ADCM2
      00000098H   SFRSYM    DATA     BYTE      SCON0
      000000E8H.3 SFRSYM    DATA     BIT       ADC0CN0_ADWINT
      000000B4H   SFRSYM    DATA     WORD      SBRL1
      000000E5H   SFRSYM    DATA     BYTE      SMOD1
      000000D2H   SFRSYM    DATA     BYTE      SCON1
      000000BAH   SFRSYM    DATA     BYTE      AMX0N
      000000E8H.4 SFRSYM    DATA     BIT       ADC0CN0_ADBUSY
      000000CEH   SFRSYM    DATA     BYTE      SMB0ADM
      000000C5H   SFRSYM    DATA     BYTE      ADC0LTL
      000000F8H.5 SFRSYM    DATA     BIT       SPI0CN0_MODF
      000000B8H.6 SFRSYM    DATA     BIT       IP_PSPI0
      000000CEH   SFRSYM    DATA     BYTE      SMB1ADM
      000000BBH   SFRSYM    DATA     BYTE      AMX0P
      000000C8H.6 SFRSYM    DATA     BIT       TMR5CN0_TF5L
      000000C8H   SFRSYM    DATA     BYTE      TMR2CN0
      00000091H   SFRSYM    DATA     BYTE      TMR3CN0
      00000091H   SFRSYM    DATA     BYTE      TMR4CN0
      000000C8H   SFRSYM    DATA     BYTE      TMR5CN0
      000000CFH   SFRSYM    DATA     BYTE      SMB0ADR
      00000088H.4 SFRSYM    DATA     BIT       TCON_TR0
      000000CFH   SFRSYM    DATA     BYTE      SMB1ADR
      000000C8H.4 SFRSYM    DATA     BIT       TMR2CN0_TF2CEN
      00000088H.6 SFRSYM    DATA     BIT       TCON_TR1
      000000C2H   SFRSYM    DATA     BYTE      SMB0DAT
      000000CDH   SFRSYM    DATA     BYTE      TMR2H
      000000A1H   SFRSYM    DATA     BYTE      SPI0CFG
      000000C2H   SFRSYM    DATA     BYTE      SMB1DAT
      00000095H   SFRSYM    DATA     BYTE      TMR3H
      00000095H   SFRSYM    DATA     BYTE      TMR4H
      000000CDH   SFRSYM    DATA     BYTE      TMR5H
      000000CCH   SFRSYM    DATA     BYTE      TMR2L
      000000F8H.7 SFRSYM    DATA     BIT       SPI0CN0_SPIF
      00000096H   SFRSYM    DATA     BYTE      USB0ADR
      00000094H   SFRSYM    DATA     BYTE      TMR3L
      000000A8H.7 SFRSYM    DATA     BIT       IE_EA
      00000094H   SFRSYM    DATA     BYTE      TMR4L
      00000097H   SFRSYM    DATA     BYTE      USB0DAT
      000000CCH   SFRSYM    DATA     BYTE      TMR5L
      000000B6H   SFRSYM    DATA     BYTE      FLSCL
      000000C8H.5 SFRSYM    DATA     BIT       TMR2CN0_TF2LEN
      000000F8H.6 SFRSYM    DATA     BIT       SPI0CN0_WCOL
      000000F8H.2 SFRSYM    DATA     BIT       SPI0CN0_NSSMD0
      000000D0H.7 SFRSYM    DATA     BIT       PSW_CY
      000000A3H   SFRSYM    DATA     BYTE      SPI0DAT
      000000F8H.3 SFRSYM    DATA     BIT       SPI0CN0_NSSMD1
      000000BDH   SFRSYM    DATA     WORD      ADC0
      000000B9H   SFRSYM    DATA     BYTE      SMBTC
      000000D0H   SFRSYM    DATA     BYTE      PSW
      000000C8H.5 SFRSYM    DATA     BIT       TMR5CN0_TF5LEN
      000000B7H   SFRSYM    DATA     BYTE      FLKEY

      01003877H   BLOCK     CODE     ---       LVL=0
      01003877H   BLOCK     CODE     NEAR LAB  LVL=1
      00000006H   SYMBOL    DATA     INT       a
      00000007H   SYMBOL    DATA     CHAR      rot
LX51 LINKER/LOCATER V4.66.30.0                                                        07/27/2019  23:22:19  PAGE 54


      ---         BLOCKEND  ---      ---       LVL=1
      01003877H   LINE      CODE     ---       #80
      01003877H   LINE      CODE     ---       #81
      01003877H   LINE      CODE     ---       #87
      01003883H   LINE      CODE     ---       #88
      0100388AH   LINE      CODE     ---       #89
      0100388FH   LINE      CODE     ---       #90
      01003896H   LINE      CODE     ---       #94
      0100389FH   LINE      CODE     ---       #96
      010038AFH   LINE      CODE     ---       #97
      010038B2H   LINE      CODE     ---       #98
      010038C3H   LINE      CODE     ---       #99
      010038C6H   LINE      CODE     ---       #100
      010038C6H   LINE      CODE     ---       #102
      010038D5H   LINE      CODE     ---       #103
      010038D8H   LINE      CODE     ---       #104
      010038E9H   LINE      CODE     ---       #105
      010038ECH   LINE      CODE     ---       #106
      010038ECH   LINE      CODE     ---       #108
      010038FCH   LINE      CODE     ---       #109
      010038FFH   LINE      CODE     ---       #110
      01003910H   LINE      CODE     ---       #111
      01003913H   LINE      CODE     ---       #112
      01003913H   LINE      CODE     ---       #116
      01003916H   LINE      CODE     ---       #120
      01003927H   LINE      CODE     ---       #122
      0100392EH   LINE      CODE     ---       #125
      01003936H   LINE      CODE     ---       #126
      01003936H   LINE      CODE     ---       #128
      01003944H   LINE      CODE     ---       #129
      0100394AH   LINE      CODE     ---       #130
      0100394AH   LINE      CODE     ---       #131
      0100394EH   LINE      CODE     ---       #135
      01003952H   LINE      CODE     ---       #136
      ---         BLOCKEND  ---      ---       LVL=0

      010049D2H   BLOCK     CODE     ---       LVL=0
      010049D2H   BLOCK     CODE     NEAR LAB  LVL=1
      00000007H   SYMBOL    DATA     BYTE      i
      ---         BLOCKEND  ---      ---       LVL=1
      010049D2H   LINE      CODE     ---       #140
      010049D2H   LINE      CODE     ---       #141
      010049D2H   LINE      CODE     ---       #145
      010049D4H   LINE      CODE     ---       #146
      010049E0H   LINE      CODE     ---       #147
      010049F4H   LINE      CODE     ---       #148
      010049F8H   LINE      CODE     ---       #151
      010049FBH   LINE      CODE     ---       #152
      010049FEH   LINE      CODE     ---       #155
      01004A26H   LINE      CODE     ---       #158
      01004A29H   LINE      CODE     ---       #159
      01004A2CH   LINE      CODE     ---       #162
      01004A2FH   LINE      CODE     ---       #165
      01004A32H   LINE      CODE     ---       #166
      01004A35H   LINE      CODE     ---       #167
      01004A3EH   LINE      CODE     ---       #169
      01004A43H   LINE      CODE     ---       #172
      01004A48H   LINE      CODE     ---       #176
      01004A4DH   LINE      CODE     ---       #179
      01004A50H   LINE      CODE     ---       #180
      ---         BLOCKEND  ---      ---       LVL=0

LX51 LINKER/LOCATER V4.66.30.0                                                        07/27/2019  23:22:19  PAGE 55


      010026D2H   BLOCK     CODE     ---       LVL=0
      010026D2H   BLOCK     CODE     NEAR LAB  LVL=1
      02000453H   SYMBOL    XDATA    ---       led
      ---         BLOCKEND  ---      ---       LVL=1
      010026D2H   LINE      CODE     ---       #186
      010026D2H   LINE      CODE     ---       #187
      010026D2H   LINE      CODE     ---       #192
      010026D4H   LINE      CODE     ---       #193
      010026D8H   LINE      CODE     ---       #194
      010026F0H   LINE      CODE     ---       #195
      010026F0H   LINE      CODE     ---       #197
      010026F3H   LINE      CODE     ---       #198
      010026F6H   LINE      CODE     ---       #199
      010026F6H   LINE      CODE     ---       #205
      010026FDH   LINE      CODE     ---       #207
      01002703H   LINE      CODE     ---       #210
      0100270BH   LINE      CODE     ---       #213
      01002712H   LINE      CODE     ---       #214
      01002715H   LINE      CODE     ---       #215
      01002715H   LINE      CODE     ---       #218
      0100271EH   LINE      CODE     ---       #219
      01002727H   LINE      CODE     ---       #220
      01002741H   LINE      CODE     ---       #221
      01002743H   LINE      CODE     ---       #223
      01002749H   LINE      CODE     ---       #224
      01002749H   LINE      CODE     ---       #230
      0100274FH   LINE      CODE     ---       #231
      01002752H   LINE      CODE     ---       #232
      01002752H   LINE      CODE     ---       #237
      01002755H   LINE      CODE     ---       #244
      0100275AH   LINE      CODE     ---       #245
      01002762H   LINE      CODE     ---       #246
      0100276AH   LINE      CODE     ---       #247
      01002772H   LINE      CODE     ---       #248
      0100277AH   LINE      CODE     ---       #249
      01002782H   LINE      CODE     ---       #250
      0100278AH   LINE      CODE     ---       #251
      0100278EH   LINE      CODE     ---       #252
      0100279CH   LINE      CODE     ---       #253
      010027A2H   LINE      CODE     ---       #254
      010027A6H   LINE      CODE     ---       #257
      010027C6H   LINE      CODE     ---       #258
      010027C6H   LINE      CODE     ---       #259
      010027CCH   LINE      CODE     ---       #260
      010027CEH   LINE      CODE     ---       #261
      010027CEH   LINE      CODE     ---       #262
      010027CEH   LINE      CODE     ---       #263
      010027D4H   LINE      CODE     ---       #264
      010027D6H   LINE      CODE     ---       #265
      010027D6H   LINE      CODE     ---       #266
      010027D6H   LINE      CODE     ---       #267
      010027DCH   LINE      CODE     ---       #268
      010027DEH   LINE      CODE     ---       #269
      010027DEH   LINE      CODE     ---       #270
      010027DEH   LINE      CODE     ---       #271
      010027E6H   LINE      CODE     ---       #272
      010027E8H   LINE      CODE     ---       #273
      010027E8H   LINE      CODE     ---       #274
      010027E8H   LINE      CODE     ---       #275
      010027EDH   LINE      CODE     ---       #276
      010027F2H   LINE      CODE     ---       #277
      010027F2H   LINE      CODE     ---       #278
LX51 LINKER/LOCATER V4.66.30.0                                                        07/27/2019  23:22:19  PAGE 56


      010027F4H   LINE      CODE     ---       #279
      010027F4H   LINE      CODE     ---       #280
      010027F4H   LINE      CODE     ---       #281
      010027F9H   LINE      CODE     ---       #282
      010027FFH   LINE      CODE     ---       #283
      01002804H   LINE      CODE     ---       #284
      01002808H   LINE      CODE     ---       #285
      0100280CH   LINE      CODE     ---       #286
      01002810H   LINE      CODE     ---       #287
      01002812H   LINE      CODE     ---       #288
      01002812H   LINE      CODE     ---       #289
      01002812H   LINE      CODE     ---       #290
      01002818H   LINE      CODE     ---       #291
      01002829H   LINE      CODE     ---       #292
      01002829H   LINE      CODE     ---       #293
      01002829H   LINE      CODE     ---       #294
      01002829H   LINE      CODE     ---       #297
      0100282FH   LINE      CODE     ---       #298
      01002834H   LINE      CODE     ---       #299
      01002834H   LINE      CODE     ---       #301
      01002850H   LINE      CODE     ---       #302
      0100287AH   LINE      CODE     ---       #303
      0100287AH   LINE      CODE     ---       #304
      ---         BLOCKEND  ---      ---       LVL=0

      010048CBH   BLOCK     CODE     ---       LVL=0
      010048CBH   LINE      CODE     ---       #309
      010048CBH   LINE      CODE     ---       #310
      010048CBH   LINE      CODE     ---       #311
      010048CDH   LINE      CODE     ---       #317
      010048ECH   LINE      CODE     ---       #318
      010048F9H   LINE      CODE     ---       #319
      010048FDH   LINE      CODE     ---       #320
      010048FDH   LINE      CODE     ---       #321
      01004900H   LINE      CODE     ---       #323
      01004900H   LINE      CODE     ---       #326
      01004903H   LINE      CODE     ---       #331
      01004915H   LINE      CODE     ---       #332
      0100491AH   LINE      CODE     ---       #333
      01004923H   LINE      CODE     ---       #334
      01004923H   LINE      CODE     ---       #335
      01004923H   LINE      CODE     ---       #338
      01004931H   LINE      CODE     ---       #340
      01004938H   LINE      CODE     ---       #341
      01004944H   LINE      CODE     ---       #342
      01004944H   LINE      CODE     ---       #343
      01004947H   LINE      CODE     ---       #344
      01004947H   LINE      CODE     ---       #349
      0100494AH   LINE      CODE     ---       #354
      0100494DH   LINE      CODE     ---       #358
      0100494FH   LINE      CODE     ---       #359
      ---         BLOCKEND  ---      ---       LVL=0

      ---         MODULE    ---      ---       EFM8_SMB1
      00000012H   PUBLIC    DATA     BYTE      smb1_state
      01002CBAH   PUBLIC    CODE     ---       smb1_interrupt
      01005BADH   PUBLIC    CODE     ---       smb1_get_state
      01005B3FH   PUBLIC    CODE     ---       smb1_stop
      0000002EH   PUBLIC    DATA     BYTE      ?_smb1_mwrite?BYTE
      01005779H   PUBLIC    CODE     ---       _smb1_mwrite
      000000A2H   SFRSYM    DATA     BYTE      SPI0CKR
      00000080H   SFRSYM    DATA     BYTE      P0
LX51 LINKER/LOCATER V4.66.30.0                                                        07/27/2019  23:22:19  PAGE 57


      000000D0H.2 SFRSYM    DATA     BIT       PSW_OV
      000000B1H   SFRSYM    DATA     BYTE      XOSC0CN
      00000090H   SFRSYM    DATA     BYTE      P1
      000000A0H   SFRSYM    DATA     BYTE      P2
      000000B0H   SFRSYM    DATA     BYTE      P3
      000000BCH   SFRSYM    DATA     BYTE      ADC0CF
      000000C8H   SFRSYM    DATA     BIT       TMR2CN0_T2XCLK
      000000C7H   SFRSYM    DATA     BYTE      P4
      000000C0H.7 SFRSYM    DATA     BIT       SMB0CN0_MASTER
      000000F9H   SFRSYM    DATA     WORD      PCA0
      000000E6H   SFRSYM    DATA     BYTE      EIE1
      000000C0H.7 SFRSYM    DATA     BIT       SMB1CN0_MASTER
      000000C0H.1 SFRSYM    DATA     BIT       SMB0CN0_ACK
      000000D7H   SFRSYM    DATA     BYTE      USB0XCN
      000000E7H   SFRSYM    DATA     BYTE      EIE2
      000000C0H.1 SFRSYM    DATA     BIT       SMB1CN0_ACK
      0000008FH   SFRSYM    DATA     BYTE      PSCTL
      000000E4H   SFRSYM    DATA     BYTE      IT01CF
      000000C8H   SFRSYM    DATA     BIT       TMR5CN0_T5XCLK
      000000C0H.6 SFRSYM    DATA     BIT       SMB0CN0_TXMODE
      000000C0H.6 SFRSYM    DATA     BIT       SMB1CN0_TXMODE
      000000BFH   SFRSYM    DATA     BYTE      SFRPAGE
      000000A4H   SFRSYM    DATA     BYTE      P0MDOUT
      000000A5H   SFRSYM    DATA     BYTE      P1MDOUT
      000000E8H.5 SFRSYM    DATA     BIT       ADC0CN0_ADINT
      000000CBH   SFRSYM    DATA     BYTE      TMR2RLH
      000000A6H   SFRSYM    DATA     BYTE      P2MDOUT
      000000A8H   SFRSYM    DATA     BYTE      IE
      00000093H   SFRSYM    DATA     BYTE      TMR3RLH
      000000A7H   SFRSYM    DATA     BYTE      P3MDOUT
      00000093H   SFRSYM    DATA     BYTE      TMR4RLH
      000000AEH   SFRSYM    DATA     BYTE      P4MDOUT
      000000F6H   SFRSYM    DATA     BYTE      EIP1
      000000CBH   SFRSYM    DATA     BYTE      TMR5RLH
      000000F7H   SFRSYM    DATA     BYTE      EIP2
      00000098H.2 SFRSYM    DATA     BIT       SCON0_RB8
      000000CAH   SFRSYM    DATA     BYTE      TMR2RLL
      000000FCH   SFRSYM    DATA     BYTE      PCA0CPH0
      00000092H   SFRSYM    DATA     BYTE      TMR3RLL
      000000EAH   SFRSYM    DATA     BYTE      PCA0CPH1
      00000098H.3 SFRSYM    DATA     BIT       SCON0_TB8
      000000F0H   SFRSYM    DATA     BIT       B_B0
      00000082H   SFRSYM    DATA     WORD      DP
      00000092H   SFRSYM    DATA     BYTE      TMR4RLL
      000000ECH   SFRSYM    DATA     BYTE      PCA0CPH2
      000000F0H.1 SFRSYM    DATA     BIT       B_B1
      000000C3H   SFRSYM    DATA     WORD      ADC0GT
      000000CAH   SFRSYM    DATA     BYTE      TMR5RLL
      000000EEH   SFRSYM    DATA     BYTE      PCA0CPH3
      000000F0H.2 SFRSYM    DATA     BIT       B_B2
      000000FBH   SFRSYM    DATA     BYTE      PCA0CPL0
      000000FEH   SFRSYM    DATA     BYTE      PCA0CPH4
      00000085H   SFRSYM    DATA     BYTE      EMI0CF
      000000F0H.3 SFRSYM    DATA     BIT       B_B3
      000000D9H   SFRSYM    DATA     BYTE      PCA0MD
      000000DAH   SFRSYM    DATA     BYTE      PCA0CPM0
      000000E9H   SFRSYM    DATA     BYTE      PCA0CPL1
      000000F0H.4 SFRSYM    DATA     BIT       B_B4
      000000DBH   SFRSYM    DATA     BYTE      PCA0CPM1
      000000EBH   SFRSYM    DATA     BYTE      PCA0CPL2
      000000F0H.5 SFRSYM    DATA     BIT       B_B5
      000000DCH   SFRSYM    DATA     BYTE      PCA0CPM2
LX51 LINKER/LOCATER V4.66.30.0                                                        07/27/2019  23:22:19  PAGE 58


      000000EDH   SFRSYM    DATA     BYTE      PCA0CPL3
      000000B8H   SFRSYM    DATA     BYTE      IP
      000000F0H.6 SFRSYM    DATA     BIT       B_B6
      000000C5H   SFRSYM    DATA     WORD      ADC0LT
      000000DDH   SFRSYM    DATA     BYTE      PCA0CPM3
      000000FDH   SFRSYM    DATA     BYTE      PCA0CPL4
      00000098H.5 SFRSYM    DATA     BIT       SCON0_MCE
      000000F0H.7 SFRSYM    DATA     BIT       B_B7
      000000DEH   SFRSYM    DATA     BYTE      PCA0CPM4
      000000E1H   SFRSYM    DATA     BYTE      XBR0
      000000C1H   SFRSYM    DATA     BYTE      SMB0CF
      000000E2H   SFRSYM    DATA     BYTE      XBR1
      000000C1H   SFRSYM    DATA     BYTE      SMB1CF
      000000AFH   SFRSYM    DATA     BYTE      PFE0CN
      000000AAH   SFRSYM    DATA     BYTE      EMI0CN
      000000C0H.5 SFRSYM    DATA     BIT       SMB0CN0_STA
      000000E3H   SFRSYM    DATA     BYTE      XBR2
      000000C0H.5 SFRSYM    DATA     BIT       SMB1CN0_STA
      000000E0H   SFRSYM    DATA     BIT       ACC_ACC0
      000000D1H   SFRSYM    DATA     BYTE      REF0CN
      000000B2H   SFRSYM    DATA     BYTE      HFO0CN
      0000008EH   SFRSYM    DATA     BYTE      CKCON0
      000000E0H.1 SFRSYM    DATA     BIT       ACC_ACC1
      000000E4H   SFRSYM    DATA     BYTE      CKCON1
      000000C8H.2 SFRSYM    DATA     BIT       TMR2CN0_TR2
      000000E0H.2 SFRSYM    DATA     BIT       ACC_ACC2
      000000E0H.3 SFRSYM    DATA     BIT       ACC_ACC3
      00000081H   SFRSYM    DATA     BYTE      SP
      0000009DH   SFRSYM    DATA     BYTE      CMP0MD
      000000E0H.4 SFRSYM    DATA     BIT       ACC_ACC4
      00000086H   SFRSYM    DATA     BYTE      LFO0CN
      00000084H   SFRSYM    DATA     BYTE      EMI0TC
      0000009CH   SFRSYM    DATA     BYTE      CMP1MD
      000000D8H   SFRSYM    DATA     BIT       PCA0CN0_CCF0
      000000E0H.5 SFRSYM    DATA     BIT       ACC_ACC5
      000000D8H.1 SFRSYM    DATA     BIT       PCA0CN0_CCF1
      000000E0H.6 SFRSYM    DATA     BIT       ACC_ACC6
      000000CCH   SFRSYM    DATA     WORD      TMR2
      000000D8H.2 SFRSYM    DATA     BIT       PCA0CN0_CCF2
      000000E0H.7 SFRSYM    DATA     BIT       ACC_ACC7
      00000094H   SFRSYM    DATA     WORD      TMR3
      000000C8H.2 SFRSYM    DATA     BIT       TMR5CN0_TR5
      000000D8H.3 SFRSYM    DATA     BIT       PCA0CN0_CCF3
      00000094H   SFRSYM    DATA     WORD      TMR4
      000000ACH   SFRSYM    DATA     BYTE      SBCON1
      000000D8H.4 SFRSYM    DATA     BIT       PCA0CN0_CCF4
      000000CCH   SFRSYM    DATA     WORD      TMR5
      000000C0H.3 SFRSYM    DATA     BIT       SMB0CN0_ACKRQ
      000000FFH   SFRSYM    DATA     BYTE      VDM0CN
      000000F1H   SFRSYM    DATA     BYTE      P0MDIN
      000000C0H.3 SFRSYM    DATA     BIT       SMB1CN0_ACKRQ
      00000098H.4 SFRSYM    DATA     BIT       SCON0_REN
      000000F2H   SFRSYM    DATA     BYTE      P1MDIN
      000000F3H   SFRSYM    DATA     BYTE      P2MDIN
      000000C0H.4 SFRSYM    DATA     BIT       SMB0CN0_STO
      000000F4H   SFRSYM    DATA     BYTE      P3MDIN
      000000C0H.4 SFRSYM    DATA     BIT       SMB1CN0_STO
      000000B5H   SFRSYM    DATA     BYTE      SBRLH1
      000000F5H   SFRSYM    DATA     BYTE      P4MDIN
      000000D0H.3 SFRSYM    DATA     BIT       PSW_RS0
      000000D8H.7 SFRSYM    DATA     BIT       PCA0CN0_CF
      000000F8H.4 SFRSYM    DATA     BIT       SPI0CN0_RXOVRN
LX51 LINKER/LOCATER V4.66.30.0                                                        07/27/2019  23:22:19  PAGE 59


      000000D0H.4 SFRSYM    DATA     BIT       PSW_RS1
      000000B4H   SFRSYM    DATA     BYTE      SBRLL1
      000000E8H.7 SFRSYM    DATA     BIT       ADC0CN0_ADEN
      00000089H   SFRSYM    DATA     BYTE      TMOD
      00000088H   SFRSYM    DATA     BYTE      TCON
      000000D0H   SFRSYM    DATA     BIT       PSW_PARITY
      000000A8H.4 SFRSYM    DATA     BIT       IE_ES0
      0000009FH   SFRSYM    DATA     BYTE      CMP0MX
      000000A8H.1 SFRSYM    DATA     BIT       IE_ET0
      0000009EH   SFRSYM    DATA     BYTE      CMP1MX
      000000A8H.3 SFRSYM    DATA     BIT       IE_ET1
      000000D4H   SFRSYM    DATA     BYTE      P0SKIP
      000000C8H.1 SFRSYM    DATA     BIT       TMR2CN0_T2CSS
      000000A8H.5 SFRSYM    DATA     BIT       IE_ET2
      000000D5H   SFRSYM    DATA     BYTE      P1SKIP
      000000D6H   SFRSYM    DATA     BYTE      P2SKIP
      000000E8H   SFRSYM    DATA     BYTE      ADC0CN0
      000000A8H   SFRSYM    DATA     BIT       IE_EX0
      000000DFH   SFRSYM    DATA     BYTE      P3SKIP
      000000D8H.6 SFRSYM    DATA     BIT       PCA0CN0_CR
      000000A8H.2 SFRSYM    DATA     BIT       IE_EX1
      00000098H.7 SFRSYM    DATA     BIT       SCON0_SMODE
      000000A9H   SFRSYM    DATA     BYTE      CLKSEL
      000000F8H   SFRSYM    DATA     BIT       SPI0CN0_SPIEN
      000000F0H   SFRSYM    DATA     BYTE      B
      000000BEH   SFRSYM    DATA     BYTE      ADC0H
      000000E8H.6 SFRSYM    DATA     BIT       ADC0CN0_ADTM
      000000CAH   SFRSYM    DATA     WORD      TMR2RL
      000000BDH   SFRSYM    DATA     BYTE      ADC0L
      00000092H   SFRSYM    DATA     WORD      TMR3RL
      00000092H   SFRSYM    DATA     WORD      TMR4RL
      000000D8H   SFRSYM    DATA     BYTE      PCA0CN0
      000000E0H   SFRSYM    DATA     BYTE      ACC
      000000CAH   SFRSYM    DATA     WORD      TMR5RL
      000000FBH   SFRSYM    DATA     WORD      PCA0CP0
      000000E9H   SFRSYM    DATA     WORD      PCA0CP1
      000000EBH   SFRSYM    DATA     WORD      PCA0CP2
      000000EDH   SFRSYM    DATA     WORD      PCA0CP3
      0000008CH   SFRSYM    DATA     BYTE      TH0
      000000B8H.4 SFRSYM    DATA     BIT       IP_PS0
      000000FDH   SFRSYM    DATA     WORD      PCA0CP4
      0000008DH   SFRSYM    DATA     BYTE      TH1
      000000FAH   SFRSYM    DATA     BYTE      PCA0H
      000000B8H.1 SFRSYM    DATA     BIT       IP_PT0
      000000B8H.3 SFRSYM    DATA     BIT       IP_PT1
      000000C0H.2 SFRSYM    DATA     BIT       SMB0CN0_ARBLOST
      000000B8H.5 SFRSYM    DATA     BIT       IP_PT2
      0000008AH   SFRSYM    DATA     BYTE      TL0
      000000F8H.1 SFRSYM    DATA     BIT       SPI0CN0_TXBMT
      000000C0H.2 SFRSYM    DATA     BIT       SMB1CN0_ARBLOST
      000000D0H.5 SFRSYM    DATA     BIT       PSW_F0
      000000A8H.6 SFRSYM    DATA     BIT       IE_ESPI0
      0000008BH   SFRSYM    DATA     BYTE      TL1
      000000F9H   SFRSYM    DATA     BYTE      PCA0L
      000000C0H   SFRSYM    DATA     BIT       SMB0CN0_SI
      000000D0H.1 SFRSYM    DATA     BIT       PSW_F1
      00000080H   SFRSYM    DATA     BIT       P0_B0
      000000B8H   SFRSYM    DATA     BIT       IP_PX0
      000000C9H   SFRSYM    DATA     BYTE      REG01CN
      000000C0H   SFRSYM    DATA     BIT       SMB1CN0_SI
      00000090H   SFRSYM    DATA     BIT       P1_B0
      00000080H.1 SFRSYM    DATA     BIT       P0_B1
LX51 LINKER/LOCATER V4.66.30.0                                                        07/27/2019  23:22:19  PAGE 60


      000000B8H.2 SFRSYM    DATA     BIT       IP_PX1
      0000009BH   SFRSYM    DATA     BYTE      CMP0CN0
      00000088H.1 SFRSYM    DATA     BIT       TCON_IE0
      000000A0H   SFRSYM    DATA     BIT       P2_B0
      00000090H.1 SFRSYM    DATA     BIT       P1_B1
      00000080H.2 SFRSYM    DATA     BIT       P0_B2
      0000009AH   SFRSYM    DATA     BYTE      CMP1CN0
      00000088H.3 SFRSYM    DATA     BIT       TCON_IE1
      000000B0H   SFRSYM    DATA     BIT       P3_B0
      000000A0H.1 SFRSYM    DATA     BIT       P2_B1
      00000090H.2 SFRSYM    DATA     BIT       P1_B2
      00000080H.3 SFRSYM    DATA     BIT       P0_B3
      000000C0H   SFRSYM    DATA     BYTE      SMB0CN0
      000000B0H.1 SFRSYM    DATA     BIT       P3_B1
      000000A0H.2 SFRSYM    DATA     BIT       P2_B2
      00000090H.3 SFRSYM    DATA     BIT       P1_B3
      00000080H.4 SFRSYM    DATA     BIT       P0_B4
      000000C0H   SFRSYM    DATA     BYTE      SMB1CN0
      000000B0H.2 SFRSYM    DATA     BIT       P3_B2
      000000A0H.3 SFRSYM    DATA     BIT       P2_B3
      00000090H.4 SFRSYM    DATA     BIT       P1_B4
      00000080H.5 SFRSYM    DATA     BIT       P0_B5
      000000B0H.3 SFRSYM    DATA     BIT       P3_B3
      000000A0H.4 SFRSYM    DATA     BIT       P2_B4
      00000090H.5 SFRSYM    DATA     BIT       P1_B5
      00000080H.6 SFRSYM    DATA     BIT       P0_B6
      000000B0H.4 SFRSYM    DATA     BIT       P3_B4
      000000A0H.5 SFRSYM    DATA     BIT       P2_B5
      00000090H.6 SFRSYM    DATA     BIT       P1_B6
      00000080H.7 SFRSYM    DATA     BIT       P0_B7
      000000B0H.5 SFRSYM    DATA     BIT       P3_B5
      000000A0H.6 SFRSYM    DATA     BIT       P2_B6
      00000090H.7 SFRSYM    DATA     BIT       P1_B7
      000000B0H.6 SFRSYM    DATA     BIT       P3_B6
      000000A0H.7 SFRSYM    DATA     BIT       P2_B7
      000000B0H.7 SFRSYM    DATA     BIT       P3_B7
      00000083H   SFRSYM    DATA     BYTE      DPH
      000000C4H   SFRSYM    DATA     BYTE      ADC0GTH
      000000C8H.7 SFRSYM    DATA     BIT       TMR2CN0_TF2H
      000000C8H.3 SFRSYM    DATA     BIT       TMR2CN0_T2SPLIT
      000000D0H.6 SFRSYM    DATA     BIT       PSW_AC
      000000F8H   SFRSYM    DATA     BYTE      SPI0CN0
      000000B3H   SFRSYM    DATA     BYTE      HFO0CAL
      00000088H.5 SFRSYM    DATA     BIT       TCON_TF0
      00000098H   SFRSYM    DATA     BIT       SCON0_RI
      00000082H   SFRSYM    DATA     BYTE      DPL
      00000088H.7 SFRSYM    DATA     BIT       TCON_TF1
      00000099H   SFRSYM    DATA     BYTE      SBUF0
      00000087H   SFRSYM    DATA     BYTE      PCON0
      000000C3H   SFRSYM    DATA     BYTE      ADC0GTL
      000000C8H.6 SFRSYM    DATA     BIT       TMR2CN0_TF2L
      00000098H.1 SFRSYM    DATA     BIT       SCON0_TI
      000000E8H   SFRSYM    DATA     BIT       ADC0CN0_ADCM0
      000000D3H   SFRSYM    DATA     BYTE      SBUF1
      000000C6H   SFRSYM    DATA     BYTE      ADC0LTH
      00000088H   SFRSYM    DATA     BIT       TCON_IT0
      000000E8H.1 SFRSYM    DATA     BIT       ADC0CN0_ADCM1
      000000EFH   SFRSYM    DATA     BYTE      RSTSRC
      000000C8H.7 SFRSYM    DATA     BIT       TMR5CN0_TF5H
      000000C8H.3 SFRSYM    DATA     BIT       TMR5CN0_T5SPLIT
      00000088H.2 SFRSYM    DATA     BIT       TCON_IT1
      000000E8H.2 SFRSYM    DATA     BIT       ADC0CN0_ADCM2
LX51 LINKER/LOCATER V4.66.30.0                                                        07/27/2019  23:22:19  PAGE 61


      00000098H   SFRSYM    DATA     BYTE      SCON0
      000000E8H.3 SFRSYM    DATA     BIT       ADC0CN0_ADWINT
      000000B4H   SFRSYM    DATA     WORD      SBRL1
      000000E5H   SFRSYM    DATA     BYTE      SMOD1
      000000D2H   SFRSYM    DATA     BYTE      SCON1
      000000BAH   SFRSYM    DATA     BYTE      AMX0N
      000000E8H.4 SFRSYM    DATA     BIT       ADC0CN0_ADBUSY
      000000CEH   SFRSYM    DATA     BYTE      SMB0ADM
      000000C5H   SFRSYM    DATA     BYTE      ADC0LTL
      000000F8H.5 SFRSYM    DATA     BIT       SPI0CN0_MODF
      000000B8H.6 SFRSYM    DATA     BIT       IP_PSPI0
      000000CEH   SFRSYM    DATA     BYTE      SMB1ADM
      000000BBH   SFRSYM    DATA     BYTE      AMX0P
      000000C8H.6 SFRSYM    DATA     BIT       TMR5CN0_TF5L
      000000C8H   SFRSYM    DATA     BYTE      TMR2CN0
      00000091H   SFRSYM    DATA     BYTE      TMR3CN0
      00000091H   SFRSYM    DATA     BYTE      TMR4CN0
      000000C8H   SFRSYM    DATA     BYTE      TMR5CN0
      000000CFH   SFRSYM    DATA     BYTE      SMB0ADR
      00000088H.4 SFRSYM    DATA     BIT       TCON_TR0
      000000CFH   SFRSYM    DATA     BYTE      SMB1ADR
      000000C8H.4 SFRSYM    DATA     BIT       TMR2CN0_TF2CEN
      00000088H.6 SFRSYM    DATA     BIT       TCON_TR1
      000000C2H   SFRSYM    DATA     BYTE      SMB0DAT
      000000CDH   SFRSYM    DATA     BYTE      TMR2H
      000000A1H   SFRSYM    DATA     BYTE      SPI0CFG
      000000C2H   SFRSYM    DATA     BYTE      SMB1DAT
      00000095H   SFRSYM    DATA     BYTE      TMR3H
      00000095H   SFRSYM    DATA     BYTE      TMR4H
      000000CDH   SFRSYM    DATA     BYTE      TMR5H
      000000CCH   SFRSYM    DATA     BYTE      TMR2L
      000000F8H.7 SFRSYM    DATA     BIT       SPI0CN0_SPIF
      00000096H   SFRSYM    DATA     BYTE      USB0ADR
      00000094H   SFRSYM    DATA     BYTE      TMR3L
      000000A8H.7 SFRSYM    DATA     BIT       IE_EA
      00000094H   SFRSYM    DATA     BYTE      TMR4L
      00000097H   SFRSYM    DATA     BYTE      USB0DAT
      000000CCH   SFRSYM    DATA     BYTE      TMR5L
      000000B6H   SFRSYM    DATA     BYTE      FLSCL
      000000C8H.5 SFRSYM    DATA     BIT       TMR2CN0_TF2LEN
      000000F8H.6 SFRSYM    DATA     BIT       SPI0CN0_WCOL
      000000F8H.2 SFRSYM    DATA     BIT       SPI0CN0_NSSMD0
      000000D0H.7 SFRSYM    DATA     BIT       PSW_CY
      000000A3H   SFRSYM    DATA     BYTE      SPI0DAT
      000000F8H.3 SFRSYM    DATA     BIT       SPI0CN0_NSSMD1
      000000BDH   SFRSYM    DATA     WORD      ADC0
      000000B9H   SFRSYM    DATA     BYTE      SMBTC
      000000D0H   SFRSYM    DATA     BYTE      PSW
      000000C8H.5 SFRSYM    DATA     BIT       TMR5CN0_TF5LEN
      000000B7H   SFRSYM    DATA     BYTE      FLKEY
      00000008H   SYMBOL    DATA     ---       smb1_buf
      0000000BH   SYMBOL    DATA     ---       _smb1_cb
      0000000EH   SYMBOL    DATA     WORD      smb1_buf_len
      00000010H   SYMBOL    DATA     WORD      smb1_buf_idx
      0000008AH   SYMBOL    IDATA    BYTE      smb1_slave_addr

      01005779H   BLOCK     CODE     ---       LVL=0
      00000007H   SYMBOL    DATA     BYTE      slave
      00000001H   SYMBOL    DATA     ---       buf
      00000032H   SYMBOL    DATA     WORD      bytes
      00000034H   SYMBOL    DATA     ---       completed_callback
      01005779H   BLOCK     CODE     NEAR LAB  LVL=1
LX51 LINKER/LOCATER V4.66.30.0                                                        07/27/2019  23:22:19  PAGE 62


      00000007H   SYMBOL    DATA     BYTE      sfrsave
      ---         BLOCKEND  ---      ---       LVL=1
      01005779H   LINE      CODE     ---       #27
      01005779H   LINE      CODE     ---       #28
      01005779H   LINE      CODE     ---       #31
      0100577DH   LINE      CODE     ---       #32
      01005783H   LINE      CODE     ---       #33
      01005789H   LINE      CODE     ---       #34
      01005792H   LINE      CODE     ---       #36
      01005795H   LINE      CODE     ---       #38
      01005797H   LINE      CODE     ---       #39
      0100579AH   LINE      CODE     ---       #41
      0100579CH   LINE      CODE     ---       #43
      0100579EH   LINE      CODE     ---       #44
      ---         BLOCKEND  ---      ---       LVL=0
      00000007H   SYMBOL    DATA     BYTE      slave
      00000001H   SYMBOL    DATA     ---       buf
      00000007H   SYMBOL    DATA     BYTE      sfrsave

      01005B3FH   BLOCK     CODE     ---       LVL=0
      01005B3FH   BLOCK     CODE     NEAR LAB  LVL=1
      00000007H   SYMBOL    DATA     BYTE      sfrsave
      ---         BLOCKEND  ---      ---       LVL=1
      01005B3FH   LINE      CODE     ---       #68
      01005B3FH   LINE      CODE     ---       #69
      01005B3FH   LINE      CODE     ---       #72
      01005B41H   LINE      CODE     ---       #73
      01005B44H   LINE      CODE     ---       #75
      01005B46H   LINE      CODE     ---       #77
      01005B48H   LINE      CODE     ---       #78
      ---         BLOCKEND  ---      ---       LVL=0

      01005BADH   BLOCK     CODE     ---       LVL=0
      01005BADH   LINE      CODE     ---       #80
      01005BADH   LINE      CODE     ---       #81
      01005BADH   LINE      CODE     ---       #82
      01005BAFH   LINE      CODE     ---       #83
      ---         BLOCKEND  ---      ---       LVL=0

      01002CBAH   BLOCK     CODE     ---       LVL=0
      01002CBAH   BLOCK     CODE     NEAR LAB  LVL=1
      0000005EH   SYMBOL    DATA     BYTE      sfrsave
      ---         BLOCKEND  ---      ---       LVL=1
      01002CBAH   LINE      CODE     ---       #86
      01002CBAH   LINE      CODE     ---       #87
      01002CBAH   LINE      CODE     ---       #90
      01002CBDH   LINE      CODE     ---       #91
      01002CC0H   LINE      CODE     ---       #93
      01002CE1H   LINE      CODE     ---       #94
      01002CE1H   LINE      CODE     ---       #97
      01002CE1H   LINE      CODE     ---       #98
      01002CE4H   LINE      CODE     ---       #100
      01002CE6H   LINE      CODE     ---       #101
      01002CE9H   LINE      CODE     ---       #103
      01002CFAH   LINE      CODE     ---       #104
      01002CFAH   LINE      CODE     ---       #105
      01002CFAH   LINE      CODE     ---       #107
      01002CFDH   LINE      CODE     ---       #108
      01002CFDH   LINE      CODE     ---       #110
      01002D08H   LINE      CODE     ---       #112
      01002D0AH   LINE      CODE     ---       #113
      01002D0DH   LINE      CODE     ---       #115
LX51 LINKER/LOCATER V4.66.30.0                                                        07/27/2019  23:22:19  PAGE 63


      01002D1EH   LINE      CODE     ---       #116
      01002D1EH   LINE      CODE     ---       #117
      01002D1EH   LINE      CODE     ---       #119
      01002D21H   LINE      CODE     ---       #120
      01002D21H   LINE      CODE     ---       #122
      01002D3BH   LINE      CODE     ---       #124
      01002D3EH   LINE      CODE     ---       #125
      01002D3EH   LINE      CODE     ---       #127
      01002D3EH   LINE      CODE     ---       #128
      01002D40H   LINE      CODE     ---       #129
      01002D42H   LINE      CODE     ---       #131
      01002D49H   LINE      CODE     ---       #132
      01002D4CH   LINE      CODE     ---       #133
      01002D4FH   LINE      CODE     ---       #134
      01002D4FH   LINE      CODE     ---       #137
      01002D4FH   LINE      CODE     ---       #138
      01002D52H   LINE      CODE     ---       #140
      01002D54H   LINE      CODE     ---       #141
      01002D54H   LINE      CODE     ---       #142
      01002D56H   LINE      CODE     ---       #143
      01002D56H   LINE      CODE     ---       #145
      01002D61H   LINE      CODE     ---       #146
      01002D67H   LINE      CODE     ---       #148
      01002D6AH   LINE      CODE     ---       #150
      01002D6DH   LINE      CODE     ---       #151
      01002D6DH   LINE      CODE     ---       #155
      01002D6DH   LINE      CODE     ---       #156
      01002D6FH   LINE      CODE     ---       #157
      01002D71H   LINE      CODE     ---       #158
      01002D7AH   LINE      CODE     ---       #160
      01002D7DH   LINE      CODE     ---       #161
      01002D7FH   LINE      CODE     ---       #163
      01002D82H   LINE      CODE     ---       #164
      01002D82H   LINE      CODE     ---       #167
      01002D82H   LINE      CODE     ---       #168
      01002D85H   LINE      CODE     ---       #170
      01002D87H   LINE      CODE     ---       #171
      01002D8AH   LINE      CODE     ---       #173
      01002D8CH   LINE      CODE     ---       #174
      01002D8CH   LINE      CODE     ---       #176
      01002D94H   LINE      CODE     ---       #178
      01002D96H   LINE      CODE     ---       #179
      01002D98H   LINE      CODE     ---       #181
      01002D9AH   LINE      CODE     ---       #182
      01002D9AH   LINE      CODE     ---       #184
      01002D9FH   LINE      CODE     ---       #185
      01002DA2H   LINE      CODE     ---       #187
      01002DA4H   LINE      CODE     ---       #188
      01002DA4H   LINE      CODE     ---       #191
      01002DA4H   LINE      CODE     ---       #192
      01002DBEH   LINE      CODE     ---       #194
      01002DC9H   LINE      CODE     ---       #196
      01002DCBH   LINE      CODE     ---       #197
      01002DCDH   LINE      CODE     ---       #198
      01002DD0H   LINE      CODE     ---       #200
      01002DDEH   LINE      CODE     ---       #201
      01002DE7H   LINE      CODE     ---       #202
      01002DE7H   LINE      CODE     ---       #204
      01002DE9H   LINE      CODE     ---       #205
      01002DE9H   LINE      CODE     ---       #207
      01002DFBH   LINE      CODE     ---       #208
      01002DFDH   LINE      CODE     ---       #209
LX51 LINKER/LOCATER V4.66.30.0                                                        07/27/2019  23:22:19  PAGE 64


      01002DFFH   LINE      CODE     ---       #210
      01002E01H   LINE      CODE     ---       #211
      01002E01H   LINE      CODE     ---       #213
      01002E01H   LINE      CODE     ---       #214
      01002E01H   LINE      CODE     ---       #215
      01002E01H   LINE      CODE     ---       #218
      01002E03H   LINE      CODE     ---       #220
      01002E06H   LINE      CODE     ---       #221
      ---         BLOCKEND  ---      ---       LVL=0

      ---         MODULE    ---      ---       OLED_SSD1306
      02000038H   PUBLIC    XDATA    ---       oled_fb
      02000037H   PUBLIC    XDATA    BYTE      ssd1306_cb_state
      02000023H   PUBLIC    PDATA    ---       ssd1306_buf
      0200002BH   PUBLIC    XDATA    ---       oled
      00000021H.3 PUBLIC    BIT      BIT       ssd1306_cb_pending
      0100D079H   PUBLIC    CONST    ---       ssd1306_cmd_disp_window_def
      0100D060H   PUBLIC    CONST    ---       ssd1306_cmd_init
      01005A6AH   PUBLIC    CODE     ---       _ssd1306_set_flipmirror
      0100501DH   PUBLIC    CODE     ---       _ssd1306_set_mirror
      01004FCDH   PUBLIC    CODE     ---       _ssd1306_set_flip
      01005417H   PUBLIC    CODE     ---       _ssd1306_set_display
      010051A8H   PUBLIC    CODE     ---       _ssd1306_cls
      01004E61H   PUBLIC    CODE     ---       ssd1306_update
      01004E04H   PUBLIC    CODE     ---       _ssd1306_init
      01005924H   PUBLIC    CODE     ---       ssd1306_init_step2
      01005884H   PUBLIC    CODE     ---       ssd1306_init_step3
      0100579FH   PUBLIC    CODE     ---       ssd1306_idle_wait
      01005B49H   PUBLIC    CODE     ---       ssd1306_cb_get
      01005B64H   PUBLIC    CODE     ---       _ssd1306_cb
      000000A2H   SFRSYM    DATA     BYTE      SPI0CKR
      00000080H   SFRSYM    DATA     BYTE      P0
      000000D0H.2 SFRSYM    DATA     BIT       PSW_OV
      000000B1H   SFRSYM    DATA     BYTE      XOSC0CN
      00000090H   SFRSYM    DATA     BYTE      P1
      000000A0H   SFRSYM    DATA     BYTE      P2
      000000B0H   SFRSYM    DATA     BYTE      P3
      000000BCH   SFRSYM    DATA     BYTE      ADC0CF
      000000C8H   SFRSYM    DATA     BIT       TMR2CN0_T2XCLK
      000000C7H   SFRSYM    DATA     BYTE      P4
      000000C0H.7 SFRSYM    DATA     BIT       SMB0CN0_MASTER
      000000F9H   SFRSYM    DATA     WORD      PCA0
      000000E6H   SFRSYM    DATA     BYTE      EIE1
      000000C0H.7 SFRSYM    DATA     BIT       SMB1CN0_MASTER
      000000C0H.1 SFRSYM    DATA     BIT       SMB0CN0_ACK
      000000D7H   SFRSYM    DATA     BYTE      USB0XCN
      000000E7H   SFRSYM    DATA     BYTE      EIE2
      000000C0H.1 SFRSYM    DATA     BIT       SMB1CN0_ACK
      0000008FH   SFRSYM    DATA     BYTE      PSCTL
      000000E4H   SFRSYM    DATA     BYTE      IT01CF
      000000C8H   SFRSYM    DATA     BIT       TMR5CN0_T5XCLK
      000000C0H.6 SFRSYM    DATA     BIT       SMB0CN0_TXMODE
      000000C0H.6 SFRSYM    DATA     BIT       SMB1CN0_TXMODE
      000000BFH   SFRSYM    DATA     BYTE      SFRPAGE
      000000A4H   SFRSYM    DATA     BYTE      P0MDOUT
      000000A5H   SFRSYM    DATA     BYTE      P1MDOUT
      000000E8H.5 SFRSYM    DATA     BIT       ADC0CN0_ADINT
      000000CBH   SFRSYM    DATA     BYTE      TMR2RLH
      000000A6H   SFRSYM    DATA     BYTE      P2MDOUT
      000000A8H   SFRSYM    DATA     BYTE      IE
      00000093H   SFRSYM    DATA     BYTE      TMR3RLH
      000000A7H   SFRSYM    DATA     BYTE      P3MDOUT
LX51 LINKER/LOCATER V4.66.30.0                                                        07/27/2019  23:22:19  PAGE 65


      00000093H   SFRSYM    DATA     BYTE      TMR4RLH
      000000AEH   SFRSYM    DATA     BYTE      P4MDOUT
      000000F6H   SFRSYM    DATA     BYTE      EIP1
      000000CBH   SFRSYM    DATA     BYTE      TMR5RLH
      000000F7H   SFRSYM    DATA     BYTE      EIP2
      00000098H.2 SFRSYM    DATA     BIT       SCON0_RB8
      000000CAH   SFRSYM    DATA     BYTE      TMR2RLL
      000000FCH   SFRSYM    DATA     BYTE      PCA0CPH0
      00000092H   SFRSYM    DATA     BYTE      TMR3RLL
      000000EAH   SFRSYM    DATA     BYTE      PCA0CPH1
      00000098H.3 SFRSYM    DATA     BIT       SCON0_TB8
      000000F0H   SFRSYM    DATA     BIT       B_B0
      00000082H   SFRSYM    DATA     WORD      DP
      00000092H   SFRSYM    DATA     BYTE      TMR4RLL
      000000ECH   SFRSYM    DATA     BYTE      PCA0CPH2
      000000F0H.1 SFRSYM    DATA     BIT       B_B1
      000000C3H   SFRSYM    DATA     WORD      ADC0GT
      000000CAH   SFRSYM    DATA     BYTE      TMR5RLL
      000000EEH   SFRSYM    DATA     BYTE      PCA0CPH3
      000000F0H.2 SFRSYM    DATA     BIT       B_B2
      000000FBH   SFRSYM    DATA     BYTE      PCA0CPL0
      000000FEH   SFRSYM    DATA     BYTE      PCA0CPH4
      00000085H   SFRSYM    DATA     BYTE      EMI0CF
      000000F0H.3 SFRSYM    DATA     BIT       B_B3
      000000D9H   SFRSYM    DATA     BYTE      PCA0MD
      000000DAH   SFRSYM    DATA     BYTE      PCA0CPM0
      000000E9H   SFRSYM    DATA     BYTE      PCA0CPL1
      000000F0H.4 SFRSYM    DATA     BIT       B_B4
      000000DBH   SFRSYM    DATA     BYTE      PCA0CPM1
      000000EBH   SFRSYM    DATA     BYTE      PCA0CPL2
      000000F0H.5 SFRSYM    DATA     BIT       B_B5
      000000DCH   SFRSYM    DATA     BYTE      PCA0CPM2
      000000EDH   SFRSYM    DATA     BYTE      PCA0CPL3
      000000B8H   SFRSYM    DATA     BYTE      IP
      000000F0H.6 SFRSYM    DATA     BIT       B_B6
      000000C5H   SFRSYM    DATA     WORD      ADC0LT
      000000DDH   SFRSYM    DATA     BYTE      PCA0CPM3
      000000FDH   SFRSYM    DATA     BYTE      PCA0CPL4
      00000098H.5 SFRSYM    DATA     BIT       SCON0_MCE
      000000F0H.7 SFRSYM    DATA     BIT       B_B7
      000000DEH   SFRSYM    DATA     BYTE      PCA0CPM4
      000000E1H   SFRSYM    DATA     BYTE      XBR0
      000000C1H   SFRSYM    DATA     BYTE      SMB0CF
      000000E2H   SFRSYM    DATA     BYTE      XBR1
      000000C1H   SFRSYM    DATA     BYTE      SMB1CF
      000000AFH   SFRSYM    DATA     BYTE      PFE0CN
      000000AAH   SFRSYM    DATA     BYTE      EMI0CN
      000000C0H.5 SFRSYM    DATA     BIT       SMB0CN0_STA
      000000E3H   SFRSYM    DATA     BYTE      XBR2
      000000C0H.5 SFRSYM    DATA     BIT       SMB1CN0_STA
      000000E0H   SFRSYM    DATA     BIT       ACC_ACC0
      000000D1H   SFRSYM    DATA     BYTE      REF0CN
      000000B2H   SFRSYM    DATA     BYTE      HFO0CN
      0000008EH   SFRSYM    DATA     BYTE      CKCON0
      000000E0H.1 SFRSYM    DATA     BIT       ACC_ACC1
      000000E4H   SFRSYM    DATA     BYTE      CKCON1
      000000C8H.2 SFRSYM    DATA     BIT       TMR2CN0_TR2
      000000E0H.2 SFRSYM    DATA     BIT       ACC_ACC2
      000000E0H.3 SFRSYM    DATA     BIT       ACC_ACC3
      00000081H   SFRSYM    DATA     BYTE      SP
      0000009DH   SFRSYM    DATA     BYTE      CMP0MD
      000000E0H.4 SFRSYM    DATA     BIT       ACC_ACC4
LX51 LINKER/LOCATER V4.66.30.0                                                        07/27/2019  23:22:19  PAGE 66


      00000086H   SFRSYM    DATA     BYTE      LFO0CN
      00000084H   SFRSYM    DATA     BYTE      EMI0TC
      0000009CH   SFRSYM    DATA     BYTE      CMP1MD
      000000D8H   SFRSYM    DATA     BIT       PCA0CN0_CCF0
      000000E0H.5 SFRSYM    DATA     BIT       ACC_ACC5
      000000D8H.1 SFRSYM    DATA     BIT       PCA0CN0_CCF1
      000000E0H.6 SFRSYM    DATA     BIT       ACC_ACC6
      000000CCH   SFRSYM    DATA     WORD      TMR2
      000000D8H.2 SFRSYM    DATA     BIT       PCA0CN0_CCF2
      000000E0H.7 SFRSYM    DATA     BIT       ACC_ACC7
      00000094H   SFRSYM    DATA     WORD      TMR3
      000000C8H.2 SFRSYM    DATA     BIT       TMR5CN0_TR5
      000000D8H.3 SFRSYM    DATA     BIT       PCA0CN0_CCF3
      00000094H   SFRSYM    DATA     WORD      TMR4
      000000ACH   SFRSYM    DATA     BYTE      SBCON1
      000000D8H.4 SFRSYM    DATA     BIT       PCA0CN0_CCF4
      000000CCH   SFRSYM    DATA     WORD      TMR5
      000000C0H.3 SFRSYM    DATA     BIT       SMB0CN0_ACKRQ
      000000FFH   SFRSYM    DATA     BYTE      VDM0CN
      000000F1H   SFRSYM    DATA     BYTE      P0MDIN
      000000C0H.3 SFRSYM    DATA     BIT       SMB1CN0_ACKRQ
      00000098H.4 SFRSYM    DATA     BIT       SCON0_REN
      000000F2H   SFRSYM    DATA     BYTE      P1MDIN
      000000F3H   SFRSYM    DATA     BYTE      P2MDIN
      000000C0H.4 SFRSYM    DATA     BIT       SMB0CN0_STO
      000000F4H   SFRSYM    DATA     BYTE      P3MDIN
      000000C0H.4 SFRSYM    DATA     BIT       SMB1CN0_STO
      000000B5H   SFRSYM    DATA     BYTE      SBRLH1
      000000F5H   SFRSYM    DATA     BYTE      P4MDIN
      000000D0H.3 SFRSYM    DATA     BIT       PSW_RS0
      000000D8H.7 SFRSYM    DATA     BIT       PCA0CN0_CF
      000000F8H.4 SFRSYM    DATA     BIT       SPI0CN0_RXOVRN
      000000D0H.4 SFRSYM    DATA     BIT       PSW_RS1
      000000B4H   SFRSYM    DATA     BYTE      SBRLL1
      000000E8H.7 SFRSYM    DATA     BIT       ADC0CN0_ADEN
      00000089H   SFRSYM    DATA     BYTE      TMOD
      00000088H   SFRSYM    DATA     BYTE      TCON
      000000D0H   SFRSYM    DATA     BIT       PSW_PARITY
      000000A8H.4 SFRSYM    DATA     BIT       IE_ES0
      0000009FH   SFRSYM    DATA     BYTE      CMP0MX
      000000A8H.1 SFRSYM    DATA     BIT       IE_ET0
      0000009EH   SFRSYM    DATA     BYTE      CMP1MX
      000000A8H.3 SFRSYM    DATA     BIT       IE_ET1
      000000D4H   SFRSYM    DATA     BYTE      P0SKIP
      000000C8H.1 SFRSYM    DATA     BIT       TMR2CN0_T2CSS
      000000A8H.5 SFRSYM    DATA     BIT       IE_ET2
      000000D5H   SFRSYM    DATA     BYTE      P1SKIP
      000000D6H   SFRSYM    DATA     BYTE      P2SKIP
      000000E8H   SFRSYM    DATA     BYTE      ADC0CN0
      000000A8H   SFRSYM    DATA     BIT       IE_EX0
      000000DFH   SFRSYM    DATA     BYTE      P3SKIP
      000000D8H.6 SFRSYM    DATA     BIT       PCA0CN0_CR
      000000A8H.2 SFRSYM    DATA     BIT       IE_EX1
      00000098H.7 SFRSYM    DATA     BIT       SCON0_SMODE
      000000A9H   SFRSYM    DATA     BYTE      CLKSEL
      000000F8H   SFRSYM    DATA     BIT       SPI0CN0_SPIEN
      000000F0H   SFRSYM    DATA     BYTE      B
      000000BEH   SFRSYM    DATA     BYTE      ADC0H
      000000E8H.6 SFRSYM    DATA     BIT       ADC0CN0_ADTM
      000000CAH   SFRSYM    DATA     WORD      TMR2RL
      000000BDH   SFRSYM    DATA     BYTE      ADC0L
      00000092H   SFRSYM    DATA     WORD      TMR3RL
LX51 LINKER/LOCATER V4.66.30.0                                                        07/27/2019  23:22:19  PAGE 67


      00000092H   SFRSYM    DATA     WORD      TMR4RL
      000000D8H   SFRSYM    DATA     BYTE      PCA0CN0
      000000E0H   SFRSYM    DATA     BYTE      ACC
      000000CAH   SFRSYM    DATA     WORD      TMR5RL
      000000FBH   SFRSYM    DATA     WORD      PCA0CP0
      000000E9H   SFRSYM    DATA     WORD      PCA0CP1
      000000EBH   SFRSYM    DATA     WORD      PCA0CP2
      000000EDH   SFRSYM    DATA     WORD      PCA0CP3
      0000008CH   SFRSYM    DATA     BYTE      TH0
      000000B8H.4 SFRSYM    DATA     BIT       IP_PS0
      000000FDH   SFRSYM    DATA     WORD      PCA0CP4
      0000008DH   SFRSYM    DATA     BYTE      TH1
      000000FAH   SFRSYM    DATA     BYTE      PCA0H
      000000B8H.1 SFRSYM    DATA     BIT       IP_PT0
      000000B8H.3 SFRSYM    DATA     BIT       IP_PT1
      000000C0H.2 SFRSYM    DATA     BIT       SMB0CN0_ARBLOST
      000000B8H.5 SFRSYM    DATA     BIT       IP_PT2
      0000008AH   SFRSYM    DATA     BYTE      TL0
      000000F8H.1 SFRSYM    DATA     BIT       SPI0CN0_TXBMT
      000000C0H.2 SFRSYM    DATA     BIT       SMB1CN0_ARBLOST
      000000D0H.5 SFRSYM    DATA     BIT       PSW_F0
      000000A8H.6 SFRSYM    DATA     BIT       IE_ESPI0
      0000008BH   SFRSYM    DATA     BYTE      TL1
      000000F9H   SFRSYM    DATA     BYTE      PCA0L
      000000C0H   SFRSYM    DATA     BIT       SMB0CN0_SI
      000000D0H.1 SFRSYM    DATA     BIT       PSW_F1
      00000080H   SFRSYM    DATA     BIT       P0_B0
      000000B8H   SFRSYM    DATA     BIT       IP_PX0
      000000C9H   SFRSYM    DATA     BYTE      REG01CN
      000000C0H   SFRSYM    DATA     BIT       SMB1CN0_SI
      00000090H   SFRSYM    DATA     BIT       P1_B0
      00000080H.1 SFRSYM    DATA     BIT       P0_B1
      000000B8H.2 SFRSYM    DATA     BIT       IP_PX1
      0000009BH   SFRSYM    DATA     BYTE      CMP0CN0
      00000088H.1 SFRSYM    DATA     BIT       TCON_IE0
      000000A0H   SFRSYM    DATA     BIT       P2_B0
      00000090H.1 SFRSYM    DATA     BIT       P1_B1
      00000080H.2 SFRSYM    DATA     BIT       P0_B2
      0000009AH   SFRSYM    DATA     BYTE      CMP1CN0
      00000088H.3 SFRSYM    DATA     BIT       TCON_IE1
      000000B0H   SFRSYM    DATA     BIT       P3_B0
      000000A0H.1 SFRSYM    DATA     BIT       P2_B1
      00000090H.2 SFRSYM    DATA     BIT       P1_B2
      00000080H.3 SFRSYM    DATA     BIT       P0_B3
      000000C0H   SFRSYM    DATA     BYTE      SMB0CN0
      000000B0H.1 SFRSYM    DATA     BIT       P3_B1
      000000A0H.2 SFRSYM    DATA     BIT       P2_B2
      00000090H.3 SFRSYM    DATA     BIT       P1_B3
      00000080H.4 SFRSYM    DATA     BIT       P0_B4
      000000C0H   SFRSYM    DATA     BYTE      SMB1CN0
      000000B0H.2 SFRSYM    DATA     BIT       P3_B2
      000000A0H.3 SFRSYM    DATA     BIT       P2_B3
      00000090H.4 SFRSYM    DATA     BIT       P1_B4
      00000080H.5 SFRSYM    DATA     BIT       P0_B5
      000000B0H.3 SFRSYM    DATA     BIT       P3_B3
      000000A0H.4 SFRSYM    DATA     BIT       P2_B4
      00000090H.5 SFRSYM    DATA     BIT       P1_B5
      00000080H.6 SFRSYM    DATA     BIT       P0_B6
      000000B0H.4 SFRSYM    DATA     BIT       P3_B4
      000000A0H.5 SFRSYM    DATA     BIT       P2_B5
      00000090H.6 SFRSYM    DATA     BIT       P1_B6
      00000080H.7 SFRSYM    DATA     BIT       P0_B7
LX51 LINKER/LOCATER V4.66.30.0                                                        07/27/2019  23:22:19  PAGE 68


      000000B0H.5 SFRSYM    DATA     BIT       P3_B5
      000000A0H.6 SFRSYM    DATA     BIT       P2_B6
      00000090H.7 SFRSYM    DATA     BIT       P1_B7
      000000B0H.6 SFRSYM    DATA     BIT       P3_B6
      000000A0H.7 SFRSYM    DATA     BIT       P2_B7
      000000B0H.7 SFRSYM    DATA     BIT       P3_B7
      00000083H   SFRSYM    DATA     BYTE      DPH
      000000C4H   SFRSYM    DATA     BYTE      ADC0GTH
      000000C8H.7 SFRSYM    DATA     BIT       TMR2CN0_TF2H
      000000C8H.3 SFRSYM    DATA     BIT       TMR2CN0_T2SPLIT
      000000D0H.6 SFRSYM    DATA     BIT       PSW_AC
      000000F8H   SFRSYM    DATA     BYTE      SPI0CN0
      000000B3H   SFRSYM    DATA     BYTE      HFO0CAL
      00000088H.5 SFRSYM    DATA     BIT       TCON_TF0
      00000098H   SFRSYM    DATA     BIT       SCON0_RI
      00000082H   SFRSYM    DATA     BYTE      DPL
      00000088H.7 SFRSYM    DATA     BIT       TCON_TF1
      00000099H   SFRSYM    DATA     BYTE      SBUF0
      00000087H   SFRSYM    DATA     BYTE      PCON0
      000000C3H   SFRSYM    DATA     BYTE      ADC0GTL
      000000C8H.6 SFRSYM    DATA     BIT       TMR2CN0_TF2L
      00000098H.1 SFRSYM    DATA     BIT       SCON0_TI
      000000E8H   SFRSYM    DATA     BIT       ADC0CN0_ADCM0
      000000D3H   SFRSYM    DATA     BYTE      SBUF1
      000000C6H   SFRSYM    DATA     BYTE      ADC0LTH
      00000088H   SFRSYM    DATA     BIT       TCON_IT0
      000000E8H.1 SFRSYM    DATA     BIT       ADC0CN0_ADCM1
      000000EFH   SFRSYM    DATA     BYTE      RSTSRC
      000000C8H.7 SFRSYM    DATA     BIT       TMR5CN0_TF5H
      000000C8H.3 SFRSYM    DATA     BIT       TMR5CN0_T5SPLIT
      00000088H.2 SFRSYM    DATA     BIT       TCON_IT1
      000000E8H.2 SFRSYM    DATA     BIT       ADC0CN0_ADCM2
      00000098H   SFRSYM    DATA     BYTE      SCON0
      000000E8H.3 SFRSYM    DATA     BIT       ADC0CN0_ADWINT
      000000B4H   SFRSYM    DATA     WORD      SBRL1
      000000E5H   SFRSYM    DATA     BYTE      SMOD1
      000000D2H   SFRSYM    DATA     BYTE      SCON1
      000000BAH   SFRSYM    DATA     BYTE      AMX0N
      000000E8H.4 SFRSYM    DATA     BIT       ADC0CN0_ADBUSY
      000000CEH   SFRSYM    DATA     BYTE      SMB0ADM
      000000C5H   SFRSYM    DATA     BYTE      ADC0LTL
      000000F8H.5 SFRSYM    DATA     BIT       SPI0CN0_MODF
      000000B8H.6 SFRSYM    DATA     BIT       IP_PSPI0
      000000CEH   SFRSYM    DATA     BYTE      SMB1ADM
      000000BBH   SFRSYM    DATA     BYTE      AMX0P
      000000C8H.6 SFRSYM    DATA     BIT       TMR5CN0_TF5L
      000000C8H   SFRSYM    DATA     BYTE      TMR2CN0
      00000091H   SFRSYM    DATA     BYTE      TMR3CN0
      00000091H   SFRSYM    DATA     BYTE      TMR4CN0
      000000C8H   SFRSYM    DATA     BYTE      TMR5CN0
      000000CFH   SFRSYM    DATA     BYTE      SMB0ADR
      00000088H.4 SFRSYM    DATA     BIT       TCON_TR0
      000000CFH   SFRSYM    DATA     BYTE      SMB1ADR
      000000C8H.4 SFRSYM    DATA     BIT       TMR2CN0_TF2CEN
      00000088H.6 SFRSYM    DATA     BIT       TCON_TR1
      000000C2H   SFRSYM    DATA     BYTE      SMB0DAT
      000000CDH   SFRSYM    DATA     BYTE      TMR2H
      000000A1H   SFRSYM    DATA     BYTE      SPI0CFG
      000000C2H   SFRSYM    DATA     BYTE      SMB1DAT
      00000095H   SFRSYM    DATA     BYTE      TMR3H
      00000095H   SFRSYM    DATA     BYTE      TMR4H
      000000CDH   SFRSYM    DATA     BYTE      TMR5H
LX51 LINKER/LOCATER V4.66.30.0                                                        07/27/2019  23:22:19  PAGE 69


      000000CCH   SFRSYM    DATA     BYTE      TMR2L
      000000F8H.7 SFRSYM    DATA     BIT       SPI0CN0_SPIF
      00000096H   SFRSYM    DATA     BYTE      USB0ADR
      00000094H   SFRSYM    DATA     BYTE      TMR3L
      000000A8H.7 SFRSYM    DATA     BIT       IE_EA
      00000094H   SFRSYM    DATA     BYTE      TMR4L
      00000097H   SFRSYM    DATA     BYTE      USB0DAT
      000000CCH   SFRSYM    DATA     BYTE      TMR5L
      000000B6H   SFRSYM    DATA     BYTE      FLSCL
      000000C8H.5 SFRSYM    DATA     BIT       TMR2CN0_TF2LEN
      000000F8H.6 SFRSYM    DATA     BIT       SPI0CN0_WCOL
      000000F8H.2 SFRSYM    DATA     BIT       SPI0CN0_NSSMD0
      000000D0H.7 SFRSYM    DATA     BIT       PSW_CY
      000000A3H   SFRSYM    DATA     BYTE      SPI0DAT
      000000F8H.3 SFRSYM    DATA     BIT       SPI0CN0_NSSMD1
      000000BDH   SFRSYM    DATA     WORD      ADC0
      000000B9H   SFRSYM    DATA     BYTE      SMBTC
      000000D0H   SFRSYM    DATA     BYTE      PSW
      000000C8H.5 SFRSYM    DATA     BIT       TMR5CN0_TF5LEN
      000000B7H   SFRSYM    DATA     BYTE      FLKEY

      01005B64H   BLOCK     CODE     ---       LVL=0
      00000007H   SYMBOL    DATA     BYTE      p
      01005B64H   LINE      CODE     ---       #59
      01005B64H   LINE      CODE     ---       #60
      01005B64H   LINE      CODE     ---       #61
      01005B66H   LINE      CODE     ---       #62
      01005B6BH   LINE      CODE     ---       #63
      ---         BLOCKEND  ---      ---       LVL=0

      01005B49H   BLOCK     CODE     ---       LVL=0
      01005B49H   BLOCK     CODE     NEAR LAB  LVL=1
      00000020H.0 SYMBOL    BIT      BIT       ret
      ---         BLOCKEND  ---      ---       LVL=1
      01005B49H   LINE      CODE     ---       #65
      01005B49H   LINE      CODE     ---       #66
      01005B49H   LINE      CODE     ---       #69
      01005B4DH   LINE      CODE     ---       #70
      01005B4FH   LINE      CODE     ---       #72
      01005B51H   LINE      CODE     ---       #73
      ---         BLOCKEND  ---      ---       LVL=0

      0100579FH   BLOCK     CODE     ---       LVL=0
      0100579FH   BLOCK     CODE     NEAR LAB  LVL=1
      0000002EH   SYMBOL    DATA     WORD      timeout
      ---         BLOCKEND  ---      ---       LVL=1
      0100579FH   LINE      CODE     ---       #77
      0100579FH   LINE      CODE     ---       #78
      0100579FH   LINE      CODE     ---       #80
      010057A5H   LINE      CODE     ---       #83
      010057AFH   LINE      CODE     ---       #85
      010057B7H   LINE      CODE     ---       #86
      010057BDH   LINE      CODE     ---       #87
      010057C0H   LINE      CODE     ---       #88
      010057C0H   LINE      CODE     ---       #90
      010057C2H   LINE      CODE     ---       #91
      ---         BLOCKEND  ---      ---       LVL=0
      00000007H   SYMBOL    DATA     BYTE      cmd
      00000004H   SYMBOL    DATA     ---       b

      01005884H   BLOCK     CODE     ---       LVL=0
      01005884H   LINE      CODE     ---       #115
LX51 LINKER/LOCATER V4.66.30.0                                                        07/27/2019  23:22:19  PAGE 70


      01005884H   LINE      CODE     ---       #116
      01005884H   LINE      CODE     ---       #117
      01005889H   LINE      CODE     ---       #118
      0100588EH   LINE      CODE     ---       #119
      0100589AH   LINE      CODE     ---       #120
      010058A0H   LINE      CODE     ---       #121
      ---         BLOCKEND  ---      ---       LVL=0

      01005924H   BLOCK     CODE     ---       LVL=0
      01005924H   LINE      CODE     ---       #122
      01005924H   LINE      CODE     ---       #123
      01005924H   LINE      CODE     ---       #124
      0100592BH   LINE      CODE     ---       #125
      0100592EH   LINE      CODE     ---       #126
      ---         BLOCKEND  ---      ---       LVL=0

      01004E04H   BLOCK     CODE     ---       LVL=0
      00000022H   SYMBOL    DATA     BYTE      display_off_during_init
      01004E04H   LINE      CODE     ---       #128
      01004E06H   LINE      CODE     ---       #129
      01004E06H   LINE      CODE     ---       #130
      01004E0CH   LINE      CODE     ---       #131
      01004E10H   LINE      CODE     ---       #132
      01004E15H   LINE      CODE     ---       #133
      01004E1FH   LINE      CODE     ---       #134
      01004E27H   LINE      CODE     ---       #136
      01004E2BH   LINE      CODE     ---       #137
      01004E30H   LINE      CODE     ---       #138
      01004E30H   LINE      CODE     ---       #140
      01004E4AH   LINE      CODE     ---       #142
      01004E50H   LINE      CODE     ---       #143
      01004E54H   LINE      CODE     ---       #144
      01004E56H   LINE      CODE     ---       #145
      01004E60H   LINE      CODE     ---       #146
      01004E60H   LINE      CODE     ---       #147
      ---         BLOCKEND  ---      ---       LVL=0

      01004E61H   BLOCK     CODE     ---       LVL=0
      01004E61H   LINE      CODE     ---       #149
      01004E61H   LINE      CODE     ---       #150
      01004E61H   LINE      CODE     ---       #152
      01004E7BH   LINE      CODE     ---       #153
      01004E7EH   LINE      CODE     ---       #161
      01004E8DH   LINE      CODE     ---       #162
      ---         BLOCKEND  ---      ---       LVL=0

      010051A8H   BLOCK     CODE     ---       LVL=0
      00000004H   SYMBOL    DATA     ---       o
      010051ACH   BLOCK     CODE     NEAR LAB  LVL=1
      0000002AH   SYMBOL    DATA     WORD      len
      00000006H   SYMBOL    DATA     ---       buf
      ---         BLOCKEND  ---      ---       LVL=1
      010051A8H   LINE      CODE     ---       #165
      010051ACH   LINE      CODE     ---       #166
      010051ACH   LINE      CODE     ---       #170
      010051C9H   LINE      CODE     ---       #171
      010051D7H   LINE      CODE     ---       #173
      010051E4H   LINE      CODE     ---       #174
      010051F2H   LINE      CODE     ---       #175
      010051F4H   LINE      CODE     ---       #176
      ---         BLOCKEND  ---      ---       LVL=0

LX51 LINKER/LOCATER V4.66.30.0                                                        07/27/2019  23:22:19  PAGE 71


      01005417H   BLOCK     CODE     ---       LVL=0
      00000007H   SYMBOL    DATA     BYTE      display
      01005417H   BLOCK     CODE     NEAR LAB  LVL=1
      00000004H   SYMBOL    DATA     ---       b
      ---         BLOCKEND  ---      ---       LVL=1
      01005417H   LINE      CODE     ---       #178
      01005417H   LINE      CODE     ---       #179
      01005417H   LINE      CODE     ---       #182
      0100541BH   LINE      CODE     ---       #184
      01005429H   LINE      CODE     ---       #185
      01005436H   LINE      CODE     ---       #187
      01005450H   LINE      CODE     ---       #188
      ---         BLOCKEND  ---      ---       LVL=0
      00000007H   SYMBOL    DATA     BYTE      invert
      00000004H   SYMBOL    DATA     ---       b
      00000007H   SYMBOL    DATA     BYTE      contrast
      00000004H   SYMBOL    DATA     ---       b

      01004FCDH   BLOCK     CODE     ---       LVL=0
      0000002DH   SYMBOL    DATA     BYTE      flip
      01004FCFH   BLOCK     CODE     NEAR LAB  LVL=1
      00000006H   SYMBOL    DATA     ---       b
      ---         BLOCKEND  ---      ---       LVL=1
      01004FCDH   LINE      CODE     ---       #218
      01004FCFH   LINE      CODE     ---       #219
      01004FCFH   LINE      CODE     ---       #222
      01004FD3H   LINE      CODE     ---       #224
      01004FE1H   LINE      CODE     ---       #225
      01004FEFH   LINE      CODE     ---       #227
      01005009H   LINE      CODE     ---       #228
      0100500CH   LINE      CODE     ---       #230
      01005013H   LINE      CODE     ---       #231
      01005017H   LINE      CODE     ---       #232
      01005018H   LINE      CODE     ---       #233
      0100501CH   LINE      CODE     ---       #234
      0100501CH   LINE      CODE     ---       #235
      ---         BLOCKEND  ---      ---       LVL=0

      0100501DH   BLOCK     CODE     ---       LVL=0
      0000002DH   SYMBOL    DATA     BYTE      mirror
      0100501FH   BLOCK     CODE     NEAR LAB  LVL=1
      00000006H   SYMBOL    DATA     ---       b
      ---         BLOCKEND  ---      ---       LVL=1
      0100501DH   LINE      CODE     ---       #237
      0100501FH   LINE      CODE     ---       #238
      0100501FH   LINE      CODE     ---       #241
      01005023H   LINE      CODE     ---       #243
      01005031H   LINE      CODE     ---       #244
      0100503FH   LINE      CODE     ---       #246
      01005059H   LINE      CODE     ---       #247
      0100505CH   LINE      CODE     ---       #249
      01005063H   LINE      CODE     ---       #250
      01005067H   LINE      CODE     ---       #251
      01005068H   LINE      CODE     ---       #252
      0100506CH   LINE      CODE     ---       #253
      0100506CH   LINE      CODE     ---       #254
      ---         BLOCKEND  ---      ---       LVL=0

      01005A6AH   BLOCK     CODE     ---       LVL=0
      0000002AH   SYMBOL    DATA     BYTE      flipm
      01005A6CH   BLOCK     CODE     NEAR LAB  LVL=1
      0000002BH   SYMBOL    DATA     ---       b
LX51 LINKER/LOCATER V4.66.30.0                                                        07/27/2019  23:22:19  PAGE 72


      ---         BLOCKEND  ---      ---       LVL=1
      01005A6AH   LINE      CODE     ---       #256
      01005A6CH   LINE      CODE     ---       #257
      01005A6CH   LINE      CODE     ---       #260
      01005A72H   LINE      CODE     ---       #262
      01005A75H   LINE      CODE     ---       #263
      ---         BLOCKEND  ---      ---       LVL=0

      ---         MODULE    ---      ---       DRAW_SSD1306
      0000001CH   PUBLIC    DATA     ---       o
      00000033H   PUBLIC    DATA     BYTE      ?_ssd1306fb_draw_str?BYTE
      010056D1H   PUBLIC    CODE     ---       _ssd1306fb_draw_str
      02000000H   PUBLIC    PDATA    BYTE      ?_ssd1306fb_internal_str?BYTE
      01002368H   PUBLIC    CODE     ---       _ssd1306fb_internal_str
      01005B52H   PUBLIC    CODE     ---       _ssd1306fb_get_font_height
      0000002AH   PUBLIC    DATA     BYTE      ?_ssd1306fb_get_str_width?BYTE
      01004950H   PUBLIC    CODE     ---       _ssd1306fb_get_str_width
      01003A2DH   PUBLIC    CODE     ---       _ssd1306fb_draw_circle
      00000026H   PUBLIC    DATA     BYTE      ?_ssd1306fb_draw_rect?BYTE
      01005647H   PUBLIC    CODE     ---       _ssd1306fb_draw_rect
      00000026H   PUBLIC    DATA     BYTE      ?_ssd1306fb_draw_line?BYTE
      01003E39H   PUBLIC    CODE     ---       _ssd1306fb_draw_line
      01002524H   PUBLIC    CODE     ---       _ssd1306fb_draw_vline
      010036A5H   PUBLIC    CODE     ---       _ssd1306fb_draw_hline
      010045F8H   PUBLIC    CODE     ---       _ssd1306fb_draw_pix
      0200000FH   PUBLIC    PDATA    BYTE      ?_ssd1306fb_draw_raw?BYTE
      01000E5BH   PUBLIC    CODE     ---       _ssd1306fb_draw_raw
      02000000H   PUBLIC    PDATA    BYTE      ?_ssd1306fb_copy?BYTE
      0100185BH   PUBLIC    CODE     ---       _ssd1306fb_copy
      0000002AH   PUBLIC    DATA     BYTE      ?_ssd1306fb_rotate?BYTE
      01002155H   PUBLIC    CODE     ---       _ssd1306fb_rotate
      01005828H   PUBLIC    CODE     ---       _ssd1306fb_set_color
      0100598EH   PUBLIC    CODE     ---       _ssd1306fb_set_cursor
      01005B7BH   PUBLIC    CODE     ---       _ssd1306fb_set_target
      000000A2H   SFRSYM    DATA     BYTE      SPI0CKR
      00000080H   SFRSYM    DATA     BYTE      P0
      000000D0H.2 SFRSYM    DATA     BIT       PSW_OV
      000000B1H   SFRSYM    DATA     BYTE      XOSC0CN
      00000090H   SFRSYM    DATA     BYTE      P1
      000000A0H   SFRSYM    DATA     BYTE      P2
      000000B0H   SFRSYM    DATA     BYTE      P3
      000000BCH   SFRSYM    DATA     BYTE      ADC0CF
      000000C8H   SFRSYM    DATA     BIT       TMR2CN0_T2XCLK
      000000C7H   SFRSYM    DATA     BYTE      P4
      000000C0H.7 SFRSYM    DATA     BIT       SMB0CN0_MASTER
      000000F9H   SFRSYM    DATA     WORD      PCA0
      000000E6H   SFRSYM    DATA     BYTE      EIE1
      000000C0H.7 SFRSYM    DATA     BIT       SMB1CN0_MASTER
      000000C0H.1 SFRSYM    DATA     BIT       SMB0CN0_ACK
      000000D7H   SFRSYM    DATA     BYTE      USB0XCN
      000000E7H   SFRSYM    DATA     BYTE      EIE2
      000000C0H.1 SFRSYM    DATA     BIT       SMB1CN0_ACK
      0000008FH   SFRSYM    DATA     BYTE      PSCTL
      000000E4H   SFRSYM    DATA     BYTE      IT01CF
      000000C8H   SFRSYM    DATA     BIT       TMR5CN0_T5XCLK
      000000C0H.6 SFRSYM    DATA     BIT       SMB0CN0_TXMODE
      000000C0H.6 SFRSYM    DATA     BIT       SMB1CN0_TXMODE
      000000BFH   SFRSYM    DATA     BYTE      SFRPAGE
      000000A4H   SFRSYM    DATA     BYTE      P0MDOUT
      000000A5H   SFRSYM    DATA     BYTE      P1MDOUT
      000000E8H.5 SFRSYM    DATA     BIT       ADC0CN0_ADINT
      000000CBH   SFRSYM    DATA     BYTE      TMR2RLH
LX51 LINKER/LOCATER V4.66.30.0                                                        07/27/2019  23:22:19  PAGE 73


      000000A6H   SFRSYM    DATA     BYTE      P2MDOUT
      000000A8H   SFRSYM    DATA     BYTE      IE
      00000093H   SFRSYM    DATA     BYTE      TMR3RLH
      000000A7H   SFRSYM    DATA     BYTE      P3MDOUT
      00000093H   SFRSYM    DATA     BYTE      TMR4RLH
      000000AEH   SFRSYM    DATA     BYTE      P4MDOUT
      000000F6H   SFRSYM    DATA     BYTE      EIP1
      000000CBH   SFRSYM    DATA     BYTE      TMR5RLH
      000000F7H   SFRSYM    DATA     BYTE      EIP2
      00000098H.2 SFRSYM    DATA     BIT       SCON0_RB8
      000000CAH   SFRSYM    DATA     BYTE      TMR2RLL
      000000FCH   SFRSYM    DATA     BYTE      PCA0CPH0
      00000092H   SFRSYM    DATA     BYTE      TMR3RLL
      000000EAH   SFRSYM    DATA     BYTE      PCA0CPH1
      00000098H.3 SFRSYM    DATA     BIT       SCON0_TB8
      000000F0H   SFRSYM    DATA     BIT       B_B0
      00000082H   SFRSYM    DATA     WORD      DP
      00000092H   SFRSYM    DATA     BYTE      TMR4RLL
      000000ECH   SFRSYM    DATA     BYTE      PCA0CPH2
      000000F0H.1 SFRSYM    DATA     BIT       B_B1
      000000C3H   SFRSYM    DATA     WORD      ADC0GT
      000000CAH   SFRSYM    DATA     BYTE      TMR5RLL
      000000EEH   SFRSYM    DATA     BYTE      PCA0CPH3
      000000F0H.2 SFRSYM    DATA     BIT       B_B2
      000000FBH   SFRSYM    DATA     BYTE      PCA0CPL0
      000000FEH   SFRSYM    DATA     BYTE      PCA0CPH4
      00000085H   SFRSYM    DATA     BYTE      EMI0CF
      000000F0H.3 SFRSYM    DATA     BIT       B_B3
      000000D9H   SFRSYM    DATA     BYTE      PCA0MD
      000000DAH   SFRSYM    DATA     BYTE      PCA0CPM0
      000000E9H   SFRSYM    DATA     BYTE      PCA0CPL1
      000000F0H.4 SFRSYM    DATA     BIT       B_B4
      000000DBH   SFRSYM    DATA     BYTE      PCA0CPM1
      000000EBH   SFRSYM    DATA     BYTE      PCA0CPL2
      000000F0H.5 SFRSYM    DATA     BIT       B_B5
      000000DCH   SFRSYM    DATA     BYTE      PCA0CPM2
      000000EDH   SFRSYM    DATA     BYTE      PCA0CPL3
      000000B8H   SFRSYM    DATA     BYTE      IP
      000000F0H.6 SFRSYM    DATA     BIT       B_B6
      000000C5H   SFRSYM    DATA     WORD      ADC0LT
      000000DDH   SFRSYM    DATA     BYTE      PCA0CPM3
      000000FDH   SFRSYM    DATA     BYTE      PCA0CPL4
      00000098H.5 SFRSYM    DATA     BIT       SCON0_MCE
      000000F0H.7 SFRSYM    DATA     BIT       B_B7
      000000DEH   SFRSYM    DATA     BYTE      PCA0CPM4
      000000E1H   SFRSYM    DATA     BYTE      XBR0
      000000C1H   SFRSYM    DATA     BYTE      SMB0CF
      000000E2H   SFRSYM    DATA     BYTE      XBR1
      000000C1H   SFRSYM    DATA     BYTE      SMB1CF
      000000AFH   SFRSYM    DATA     BYTE      PFE0CN
      000000AAH   SFRSYM    DATA     BYTE      EMI0CN
      000000C0H.5 SFRSYM    DATA     BIT       SMB0CN0_STA
      000000E3H   SFRSYM    DATA     BYTE      XBR2
      000000C0H.5 SFRSYM    DATA     BIT       SMB1CN0_STA
      000000E0H   SFRSYM    DATA     BIT       ACC_ACC0
      000000D1H   SFRSYM    DATA     BYTE      REF0CN
      000000B2H   SFRSYM    DATA     BYTE      HFO0CN
      0000008EH   SFRSYM    DATA     BYTE      CKCON0
      000000E0H.1 SFRSYM    DATA     BIT       ACC_ACC1
      000000E4H   SFRSYM    DATA     BYTE      CKCON1
      000000C8H.2 SFRSYM    DATA     BIT       TMR2CN0_TR2
      000000E0H.2 SFRSYM    DATA     BIT       ACC_ACC2
LX51 LINKER/LOCATER V4.66.30.0                                                        07/27/2019  23:22:19  PAGE 74


      000000E0H.3 SFRSYM    DATA     BIT       ACC_ACC3
      00000081H   SFRSYM    DATA     BYTE      SP
      0000009DH   SFRSYM    DATA     BYTE      CMP0MD
      000000E0H.4 SFRSYM    DATA     BIT       ACC_ACC4
      00000086H   SFRSYM    DATA     BYTE      LFO0CN
      00000084H   SFRSYM    DATA     BYTE      EMI0TC
      0000009CH   SFRSYM    DATA     BYTE      CMP1MD
      000000D8H   SFRSYM    DATA     BIT       PCA0CN0_CCF0
      000000E0H.5 SFRSYM    DATA     BIT       ACC_ACC5
      000000D8H.1 SFRSYM    DATA     BIT       PCA0CN0_CCF1
      000000E0H.6 SFRSYM    DATA     BIT       ACC_ACC6
      000000CCH   SFRSYM    DATA     WORD      TMR2
      000000D8H.2 SFRSYM    DATA     BIT       PCA0CN0_CCF2
      000000E0H.7 SFRSYM    DATA     BIT       ACC_ACC7
      00000094H   SFRSYM    DATA     WORD      TMR3
      000000C8H.2 SFRSYM    DATA     BIT       TMR5CN0_TR5
      000000D8H.3 SFRSYM    DATA     BIT       PCA0CN0_CCF3
      00000094H   SFRSYM    DATA     WORD      TMR4
      000000ACH   SFRSYM    DATA     BYTE      SBCON1
      000000D8H.4 SFRSYM    DATA     BIT       PCA0CN0_CCF4
      000000CCH   SFRSYM    DATA     WORD      TMR5
      000000C0H.3 SFRSYM    DATA     BIT       SMB0CN0_ACKRQ
      000000FFH   SFRSYM    DATA     BYTE      VDM0CN
      000000F1H   SFRSYM    DATA     BYTE      P0MDIN
      000000C0H.3 SFRSYM    DATA     BIT       SMB1CN0_ACKRQ
      00000098H.4 SFRSYM    DATA     BIT       SCON0_REN
      000000F2H   SFRSYM    DATA     BYTE      P1MDIN
      000000F3H   SFRSYM    DATA     BYTE      P2MDIN
      000000C0H.4 SFRSYM    DATA     BIT       SMB0CN0_STO
      000000F4H   SFRSYM    DATA     BYTE      P3MDIN
      000000C0H.4 SFRSYM    DATA     BIT       SMB1CN0_STO
      000000B5H   SFRSYM    DATA     BYTE      SBRLH1
      000000F5H   SFRSYM    DATA     BYTE      P4MDIN
      000000D0H.3 SFRSYM    DATA     BIT       PSW_RS0
      000000D8H.7 SFRSYM    DATA     BIT       PCA0CN0_CF
      000000F8H.4 SFRSYM    DATA     BIT       SPI0CN0_RXOVRN
      000000D0H.4 SFRSYM    DATA     BIT       PSW_RS1
      000000B4H   SFRSYM    DATA     BYTE      SBRLL1
      000000E8H.7 SFRSYM    DATA     BIT       ADC0CN0_ADEN
      00000089H   SFRSYM    DATA     BYTE      TMOD
      00000088H   SFRSYM    DATA     BYTE      TCON
      000000D0H   SFRSYM    DATA     BIT       PSW_PARITY
      000000A8H.4 SFRSYM    DATA     BIT       IE_ES0
      0000009FH   SFRSYM    DATA     BYTE      CMP0MX
      000000A8H.1 SFRSYM    DATA     BIT       IE_ET0
      0000009EH   SFRSYM    DATA     BYTE      CMP1MX
      000000A8H.3 SFRSYM    DATA     BIT       IE_ET1
      000000D4H   SFRSYM    DATA     BYTE      P0SKIP
      000000C8H.1 SFRSYM    DATA     BIT       TMR2CN0_T2CSS
      000000A8H.5 SFRSYM    DATA     BIT       IE_ET2
      000000D5H   SFRSYM    DATA     BYTE      P1SKIP
      000000D6H   SFRSYM    DATA     BYTE      P2SKIP
      000000E8H   SFRSYM    DATA     BYTE      ADC0CN0
      000000A8H   SFRSYM    DATA     BIT       IE_EX0
      000000DFH   SFRSYM    DATA     BYTE      P3SKIP
      000000D8H.6 SFRSYM    DATA     BIT       PCA0CN0_CR
      000000A8H.2 SFRSYM    DATA     BIT       IE_EX1
      00000098H.7 SFRSYM    DATA     BIT       SCON0_SMODE
      000000A9H   SFRSYM    DATA     BYTE      CLKSEL
      000000F8H   SFRSYM    DATA     BIT       SPI0CN0_SPIEN
      000000F0H   SFRSYM    DATA     BYTE      B
      000000BEH   SFRSYM    DATA     BYTE      ADC0H
LX51 LINKER/LOCATER V4.66.30.0                                                        07/27/2019  23:22:19  PAGE 75


      000000E8H.6 SFRSYM    DATA     BIT       ADC0CN0_ADTM
      000000CAH   SFRSYM    DATA     WORD      TMR2RL
      000000BDH   SFRSYM    DATA     BYTE      ADC0L
      00000092H   SFRSYM    DATA     WORD      TMR3RL
      00000092H   SFRSYM    DATA     WORD      TMR4RL
      000000D8H   SFRSYM    DATA     BYTE      PCA0CN0
      000000E0H   SFRSYM    DATA     BYTE      ACC
      000000CAH   SFRSYM    DATA     WORD      TMR5RL
      000000FBH   SFRSYM    DATA     WORD      PCA0CP0
      000000E9H   SFRSYM    DATA     WORD      PCA0CP1
      000000EBH   SFRSYM    DATA     WORD      PCA0CP2
      000000EDH   SFRSYM    DATA     WORD      PCA0CP3
      0000008CH   SFRSYM    DATA     BYTE      TH0
      000000B8H.4 SFRSYM    DATA     BIT       IP_PS0
      000000FDH   SFRSYM    DATA     WORD      PCA0CP4
      0000008DH   SFRSYM    DATA     BYTE      TH1
      000000FAH   SFRSYM    DATA     BYTE      PCA0H
      000000B8H.1 SFRSYM    DATA     BIT       IP_PT0
      000000B8H.3 SFRSYM    DATA     BIT       IP_PT1
      000000C0H.2 SFRSYM    DATA     BIT       SMB0CN0_ARBLOST
      000000B8H.5 SFRSYM    DATA     BIT       IP_PT2
      0000008AH   SFRSYM    DATA     BYTE      TL0
      000000F8H.1 SFRSYM    DATA     BIT       SPI0CN0_TXBMT
      000000C0H.2 SFRSYM    DATA     BIT       SMB1CN0_ARBLOST
      000000D0H.5 SFRSYM    DATA     BIT       PSW_F0
      000000A8H.6 SFRSYM    DATA     BIT       IE_ESPI0
      0000008BH   SFRSYM    DATA     BYTE      TL1
      000000F9H   SFRSYM    DATA     BYTE      PCA0L
      000000C0H   SFRSYM    DATA     BIT       SMB0CN0_SI
      000000D0H.1 SFRSYM    DATA     BIT       PSW_F1
      00000080H   SFRSYM    DATA     BIT       P0_B0
      000000B8H   SFRSYM    DATA     BIT       IP_PX0
      000000C9H   SFRSYM    DATA     BYTE      REG01CN
      000000C0H   SFRSYM    DATA     BIT       SMB1CN0_SI
      00000090H   SFRSYM    DATA     BIT       P1_B0
      00000080H.1 SFRSYM    DATA     BIT       P0_B1
      000000B8H.2 SFRSYM    DATA     BIT       IP_PX1
      0000009BH   SFRSYM    DATA     BYTE      CMP0CN0
      00000088H.1 SFRSYM    DATA     BIT       TCON_IE0
      000000A0H   SFRSYM    DATA     BIT       P2_B0
      00000090H.1 SFRSYM    DATA     BIT       P1_B1
      00000080H.2 SFRSYM    DATA     BIT       P0_B2
      0000009AH   SFRSYM    DATA     BYTE      CMP1CN0
      00000088H.3 SFRSYM    DATA     BIT       TCON_IE1
      000000B0H   SFRSYM    DATA     BIT       P3_B0
      000000A0H.1 SFRSYM    DATA     BIT       P2_B1
      00000090H.2 SFRSYM    DATA     BIT       P1_B2
      00000080H.3 SFRSYM    DATA     BIT       P0_B3
      000000C0H   SFRSYM    DATA     BYTE      SMB0CN0
      000000B0H.1 SFRSYM    DATA     BIT       P3_B1
      000000A0H.2 SFRSYM    DATA     BIT       P2_B2
      00000090H.3 SFRSYM    DATA     BIT       P1_B3
      00000080H.4 SFRSYM    DATA     BIT       P0_B4
      000000C0H   SFRSYM    DATA     BYTE      SMB1CN0
      000000B0H.2 SFRSYM    DATA     BIT       P3_B2
      000000A0H.3 SFRSYM    DATA     BIT       P2_B3
      00000090H.4 SFRSYM    DATA     BIT       P1_B4
      00000080H.5 SFRSYM    DATA     BIT       P0_B5
      000000B0H.3 SFRSYM    DATA     BIT       P3_B3
      000000A0H.4 SFRSYM    DATA     BIT       P2_B4
      00000090H.5 SFRSYM    DATA     BIT       P1_B5
      00000080H.6 SFRSYM    DATA     BIT       P0_B6
LX51 LINKER/LOCATER V4.66.30.0                                                        07/27/2019  23:22:19  PAGE 76


      000000B0H.4 SFRSYM    DATA     BIT       P3_B4
      000000A0H.5 SFRSYM    DATA     BIT       P2_B5
      00000090H.6 SFRSYM    DATA     BIT       P1_B6
      00000080H.7 SFRSYM    DATA     BIT       P0_B7
      000000B0H.5 SFRSYM    DATA     BIT       P3_B5
      000000A0H.6 SFRSYM    DATA     BIT       P2_B6
      00000090H.7 SFRSYM    DATA     BIT       P1_B7
      000000B0H.6 SFRSYM    DATA     BIT       P3_B6
      000000A0H.7 SFRSYM    DATA     BIT       P2_B7
      000000B0H.7 SFRSYM    DATA     BIT       P3_B7
      00000083H   SFRSYM    DATA     BYTE      DPH
      000000C4H   SFRSYM    DATA     BYTE      ADC0GTH
      000000C8H.7 SFRSYM    DATA     BIT       TMR2CN0_TF2H
      000000C8H.3 SFRSYM    DATA     BIT       TMR2CN0_T2SPLIT
      000000D0H.6 SFRSYM    DATA     BIT       PSW_AC
      000000F8H   SFRSYM    DATA     BYTE      SPI0CN0
      000000B3H   SFRSYM    DATA     BYTE      HFO0CAL
      00000088H.5 SFRSYM    DATA     BIT       TCON_TF0
      00000098H   SFRSYM    DATA     BIT       SCON0_RI
      00000082H   SFRSYM    DATA     BYTE      DPL
      00000088H.7 SFRSYM    DATA     BIT       TCON_TF1
      00000099H   SFRSYM    DATA     BYTE      SBUF0
      00000087H   SFRSYM    DATA     BYTE      PCON0
      000000C3H   SFRSYM    DATA     BYTE      ADC0GTL
      000000C8H.6 SFRSYM    DATA     BIT       TMR2CN0_TF2L
      00000098H.1 SFRSYM    DATA     BIT       SCON0_TI
      000000E8H   SFRSYM    DATA     BIT       ADC0CN0_ADCM0
      000000D3H   SFRSYM    DATA     BYTE      SBUF1
      000000C6H   SFRSYM    DATA     BYTE      ADC0LTH
      00000088H   SFRSYM    DATA     BIT       TCON_IT0
      000000E8H.1 SFRSYM    DATA     BIT       ADC0CN0_ADCM1
      000000EFH   SFRSYM    DATA     BYTE      RSTSRC
      000000C8H.7 SFRSYM    DATA     BIT       TMR5CN0_TF5H
      000000C8H.3 SFRSYM    DATA     BIT       TMR5CN0_T5SPLIT
      00000088H.2 SFRSYM    DATA     BIT       TCON_IT1
      000000E8H.2 SFRSYM    DATA     BIT       ADC0CN0_ADCM2
      00000098H   SFRSYM    DATA     BYTE      SCON0
      000000E8H.3 SFRSYM    DATA     BIT       ADC0CN0_ADWINT
      000000B4H   SFRSYM    DATA     WORD      SBRL1
      000000E5H   SFRSYM    DATA     BYTE      SMOD1
      000000D2H   SFRSYM    DATA     BYTE      SCON1
      000000BAH   SFRSYM    DATA     BYTE      AMX0N
      000000E8H.4 SFRSYM    DATA     BIT       ADC0CN0_ADBUSY
      000000CEH   SFRSYM    DATA     BYTE      SMB0ADM
      000000C5H   SFRSYM    DATA     BYTE      ADC0LTL
      000000F8H.5 SFRSYM    DATA     BIT       SPI0CN0_MODF
      000000B8H.6 SFRSYM    DATA     BIT       IP_PSPI0
      000000CEH   SFRSYM    DATA     BYTE      SMB1ADM
      000000BBH   SFRSYM    DATA     BYTE      AMX0P
      000000C8H.6 SFRSYM    DATA     BIT       TMR5CN0_TF5L
      000000C8H   SFRSYM    DATA     BYTE      TMR2CN0
      00000091H   SFRSYM    DATA     BYTE      TMR3CN0
      00000091H   SFRSYM    DATA     BYTE      TMR4CN0
      000000C8H   SFRSYM    DATA     BYTE      TMR5CN0
      000000CFH   SFRSYM    DATA     BYTE      SMB0ADR
      00000088H.4 SFRSYM    DATA     BIT       TCON_TR0
      000000CFH   SFRSYM    DATA     BYTE      SMB1ADR
      000000C8H.4 SFRSYM    DATA     BIT       TMR2CN0_TF2CEN
      00000088H.6 SFRSYM    DATA     BIT       TCON_TR1
      000000C2H   SFRSYM    DATA     BYTE      SMB0DAT
      000000CDH   SFRSYM    DATA     BYTE      TMR2H
      000000A1H   SFRSYM    DATA     BYTE      SPI0CFG
LX51 LINKER/LOCATER V4.66.30.0                                                        07/27/2019  23:22:19  PAGE 77


      000000C2H   SFRSYM    DATA     BYTE      SMB1DAT
      00000095H   SFRSYM    DATA     BYTE      TMR3H
      00000095H   SFRSYM    DATA     BYTE      TMR4H
      000000CDH   SFRSYM    DATA     BYTE      TMR5H
      000000CCH   SFRSYM    DATA     BYTE      TMR2L
      000000F8H.7 SFRSYM    DATA     BIT       SPI0CN0_SPIF
      00000096H   SFRSYM    DATA     BYTE      USB0ADR
      00000094H   SFRSYM    DATA     BYTE      TMR3L
      000000A8H.7 SFRSYM    DATA     BIT       IE_EA
      00000094H   SFRSYM    DATA     BYTE      TMR4L
      00000097H   SFRSYM    DATA     BYTE      USB0DAT
      000000CCH   SFRSYM    DATA     BYTE      TMR5L
      000000B6H   SFRSYM    DATA     BYTE      FLSCL
      000000C8H.5 SFRSYM    DATA     BIT       TMR2CN0_TF2LEN
      000000F8H.6 SFRSYM    DATA     BIT       SPI0CN0_WCOL
      000000F8H.2 SFRSYM    DATA     BIT       SPI0CN0_NSSMD0
      000000D0H.7 SFRSYM    DATA     BIT       PSW_CY
      000000A3H   SFRSYM    DATA     BYTE      SPI0DAT
      000000F8H.3 SFRSYM    DATA     BIT       SPI0CN0_NSSMD1
      000000BDH   SFRSYM    DATA     WORD      ADC0
      000000B9H   SFRSYM    DATA     BYTE      SMBTC
      000000D0H   SFRSYM    DATA     BYTE      PSW
      000000C8H.5 SFRSYM    DATA     BIT       TMR5CN0_TF5LEN
      000000B7H   SFRSYM    DATA     BYTE      FLKEY

      01005B7BH   BLOCK     CODE     ---       LVL=0
      00000001H   SYMBOL    DATA     ---       target
      01005B7BH   LINE      CODE     ---       #25
      01005B7BH   LINE      CODE     ---       #26
      01005B7BH   LINE      CODE     ---       #27
      01005B81H   LINE      CODE     ---       #28
      ---         BLOCKEND  ---      ---       LVL=0

      0100598EH   BLOCK     CODE     ---       LVL=0
      00000007H   SYMBOL    DATA     CHAR      x
      00000005H   SYMBOL    DATA     CHAR      y
      0100598EH   LINE      CODE     ---       #31
      0100598EH   LINE      CODE     ---       #32
      0100598EH   LINE      CODE     ---       #33
      0100599BH   LINE      CODE     ---       #34
      ---         BLOCKEND  ---      ---       LVL=0

      01005828H   BLOCK     CODE     ---       LVL=0
      00000007H   SYMBOL    DATA     BYTE      color
      01005828H   LINE      CODE     ---       #37
      01005828H   LINE      CODE     ---       #38
      01005828H   LINE      CODE     ---       #39
      01005836H   LINE      CODE     ---       #40
      ---         BLOCKEND  ---      ---       LVL=0

      01002155H   BLOCK     CODE     ---       LVL=0
      00000001H   SYMBOL    DATA     ---       src
      0000002DH   SYMBOL    DATA     ---       dst
      00000030H   SYMBOL    DATA     CHAR      rot
      01002155H   BLOCK     CODE     NEAR LAB  LVL=1
      00000031H   SYMBOL    DATA     CHAR      x
      00000032H   SYMBOL    DATA     CHAR      y
      00000033H   SYMBOL    DATA     CHAR      nx
      00000007H   SYMBOL    DATA     CHAR      ny
      00000034H   SYMBOL    DATA     CHAR      startx
      00000035H   SYMBOL    DATA     CHAR      starty
      00000036H   SYMBOL    DATA     CHAR      endx
LX51 LINKER/LOCATER V4.66.30.0                                                        07/27/2019  23:22:19  PAGE 78


      00000037H   SYMBOL    DATA     CHAR      endy
      00000038H   SYMBOL    DATA     CHAR      yoff
      00000039H   SYMBOL    DATA     CHAR      xoff
      00000007H   SYMBOL    DATA     CHAR      dxoff
      0000003AH   SYMBOL    DATA     CHAR      dyoff
      0000003BH   SYMBOL    DATA     ---       s
      0000003EH   SYMBOL    DATA     ---       d
      ---         BLOCKEND  ---      ---       LVL=1
      01002155H   LINE      CODE     ---       #50
      01002155H   LINE      CODE     ---       #51
      01002155H   LINE      CODE     ---       #63
      01002164H   LINE      CODE     ---       #64
      01002179H   LINE      CODE     ---       #66
      01002186H   LINE      CODE     ---       #67
      0100218AH   LINE      CODE     ---       #68
      01002190H   LINE      CODE     ---       #70
      0100219BH   LINE      CODE     ---       #71
      0100219FH   LINE      CODE     ---       #72
      010021A5H   LINE      CODE     ---       #74
      010021B8H   LINE      CODE     ---       #75
      010021C2H   LINE      CODE     ---       #76
      010021DCH   LINE      CODE     ---       #78
      010021EFH   LINE      CODE     ---       #79
      0100223BH   LINE      CODE     ---       #80
      01002285H   LINE      CODE     ---       #81
      010022C7H   LINE      CODE     ---       #83
      010022E4H   LINE      CODE     ---       #84
      010022FCH   LINE      CODE     ---       #85
      01002305H   LINE      CODE     ---       #86
      0100231EH   LINE      CODE     ---       #87
      0100235DH   LINE      CODE     ---       #88
      0100235DH   LINE      CODE     ---       #89
      0100235DH   LINE      CODE     ---       #90
      0100235DH   LINE      CODE     ---       #91
      01002362H   LINE      CODE     ---       #92
      01002367H   LINE      CODE     ---       #93
      ---         BLOCKEND  ---      ---       LVL=0

      0100185BH   BLOCK     CODE     ---       LVL=0
      02000000H   SYMBOL    PDATA    CHAR      x
      02000001H   SYMBOL    PDATA    CHAR      y
      02000002H   SYMBOL    PDATA    BYTE      width
      02000003H   SYMBOL    PDATA    BYTE      height
      02000004H   SYMBOL    PDATA    ---       dat
      01001866H   BLOCK     CODE     NEAR LAB  LVL=1
      0000002AH   SYMBOL    DATA     WORD      i
      0000002CH   SYMBOL    DATA     BYTE      d
      0000002DH   SYMBOL    DATA     BYTE      w
      02000007H   SYMBOL    PDATA    BYTE      xp
      00000006H   SYMBOL    DATA     WORD      yp
      02000008H   SYMBOL    PDATA    INT       pos
      0000002EH   SYMBOL    DATA     BYTE      rh
      0000002FH   SYMBOL    DATA     CHAR      yoff
      0200000AH   SYMBOL    PDATA    WORD      bytes
      0200000CH   SYMBOL    PDATA    ---       fb
      0200000EH   SYMBOL    PDATA    INT       fb_siz
      ---         BLOCKEND  ---      ---       LVL=1
      0100185BH   LINE      CODE     ---       #99
      01001866H   LINE      CODE     ---       #120
      01001885H   LINE      CODE     ---       #121
      010018A1H   LINE      CODE     ---       #123
      010018B6H   LINE      CODE     ---       #124
LX51 LINKER/LOCATER V4.66.30.0                                                        07/27/2019  23:22:19  PAGE 79


      010018D6H   LINE      CODE     ---       #126
      010018E2H   LINE      CODE     ---       #127
      010018E9H   LINE      CODE     ---       #129
      010018F9H   LINE      CODE     ---       #131
      010018FBH   LINE      CODE     ---       #133
      01001901H   LINE      CODE     ---       #134
      01001904H   LINE      CODE     ---       #136
      01001917H   LINE      CODE     ---       #137
      01001927H   LINE      CODE     ---       #139
      0100193AH   LINE      CODE     ---       #140
      01001972H   LINE      CODE     ---       #142
      0100197DH   LINE      CODE     ---       #145
      01001989H   LINE      CODE     ---       #146
      01001994H   LINE      CODE     ---       #147
      01001998H   LINE      CODE     ---       #148
      0100199CH   LINE      CODE     ---       #150
      010019A0H   LINE      CODE     ---       #151
      010019B3H   LINE      CODE     ---       #152
      010019B6H   LINE      CODE     ---       #153
      010019B6H   LINE      CODE     ---       #154
      010019B6H   LINE      CODE     ---       #155
      010019B6H   LINE      CODE     ---       #157
      010019D3H   LINE      CODE     ---       #159
      010019F9H   LINE      CODE     ---       #160
      01001A05H   LINE      CODE     ---       #161
      01001A10H   LINE      CODE     ---       #162
      01001A1DH   LINE      CODE     ---       #163
      01001A40H   LINE      CODE     ---       #164
      01001A46H   LINE      CODE     ---       #165
      01001A6BH   LINE      CODE     ---       #166
      01001A6DH   LINE      CODE     ---       #167
      01001A93H   LINE      CODE     ---       #168
      01001A93H   LINE      CODE     ---       #169
      01001A93H   LINE      CODE     ---       #171
      01001AC6H   LINE      CODE     ---       #172
      01001ACCH   LINE      CODE     ---       #173
      01001AFFH   LINE      CODE     ---       #174
      01001B07H   LINE      CODE     ---       #175
      01001B3AH   LINE      CODE     ---       #176
      01001B3CH   LINE      CODE     ---       #177
      01001B70H   LINE      CODE     ---       #178
      01001B70H   LINE      CODE     ---       #179
      01001B70H   LINE      CODE     ---       #180
      01001B70H   LINE      CODE     ---       #181
      01001B70H   LINE      CODE     ---       #182
      01001B7BH   LINE      CODE     ---       #183
      ---         BLOCKEND  ---      ---       LVL=0

      01000E5BH   BLOCK     CODE     ---       LVL=0
      0200000FH   SYMBOL    PDATA    CHAR      x
      02000010H   SYMBOL    PDATA    CHAR      y
      02000011H   SYMBOL    PDATA    BYTE      width
      02000012H   SYMBOL    PDATA    BYTE      height
      02000013H   SYMBOL    PDATA    ---       dat
      02000016H   SYMBOL    PDATA    WORD      dat_offset
      02000018H   SYMBOL    PDATA    WORD      bytes
      01000E66H   BLOCK     CODE     NEAR LAB  LVL=1
      0000003EH   SYMBOL    DATA     WORD      i
      00000040H   SYMBOL    DATA     BYTE      d
      0200001AH   SYMBOL    PDATA    BYTE      xp
      00000006H   SYMBOL    DATA     WORD      yp
      0200001BH   SYMBOL    PDATA    INT       pos
LX51 LINKER/LOCATER V4.66.30.0                                                        07/27/2019  23:22:19  PAGE 80


      00000041H   SYMBOL    DATA     BYTE      rh
      00000042H   SYMBOL    DATA     CHAR      yoff
      0200001DH   SYMBOL    PDATA    CHAR      y_init
      0200001EH   SYMBOL    PDATA    CHAR      yoff_init
      0200001FH   SYMBOL    PDATA    ---       fb
      02000021H   SYMBOL    PDATA    INT       fb_siz
      ---         BLOCKEND  ---      ---       LVL=1
      01000E5BH   LINE      CODE     ---       #188
      01000E66H   LINE      CODE     ---       #207
      01000E85H   LINE      CODE     ---       #208
      01000EA1H   LINE      CODE     ---       #210
      01000EB0H   LINE      CODE     ---       #211
      01000ED0H   LINE      CODE     ---       #213
      01000EDCH   LINE      CODE     ---       #214
      01000EE4H   LINE      CODE     ---       #216
      01000F05H   LINE      CODE     ---       #218
      01000F09H   LINE      CODE     ---       #219
      01000F0DH   LINE      CODE     ---       #221
      01000F13H   LINE      CODE     ---       #222
      01000F16H   LINE      CODE     ---       #224
      01000F29H   LINE      CODE     ---       #226
      01000F40H   LINE      CODE     ---       #227
      01000F46H   LINE      CODE     ---       #228
      01000F4BH   LINE      CODE     ---       #229
      01000F4BH   LINE      CODE     ---       #231
      01000F64H   LINE      CODE     ---       #233
      01000F77H   LINE      CODE     ---       #234
      01000FAFH   LINE      CODE     ---       #236
      01000FBAH   LINE      CODE     ---       #239
      01000FC6H   LINE      CODE     ---       #240
      01000FD1H   LINE      CODE     ---       #241
      01000FD5H   LINE      CODE     ---       #242
      01000FD9H   LINE      CODE     ---       #244
      01000FDDH   LINE      CODE     ---       #245
      01000FF0H   LINE      CODE     ---       #246
      01000FF3H   LINE      CODE     ---       #247
      01000FF3H   LINE      CODE     ---       #248
      01000FF3H   LINE      CODE     ---       #249
      01000FF3H   LINE      CODE     ---       #251
      01001010H   LINE      CODE     ---       #253
      01001036H   LINE      CODE     ---       #254
      01001042H   LINE      CODE     ---       #255
      0100104DH   LINE      CODE     ---       #256
      0100105AH   LINE      CODE     ---       #257
      0100107DH   LINE      CODE     ---       #258
      01001083H   LINE      CODE     ---       #259
      010010A8H   LINE      CODE     ---       #260
      010010AAH   LINE      CODE     ---       #261
      010010D0H   LINE      CODE     ---       #262
      010010D0H   LINE      CODE     ---       #263
      010010D0H   LINE      CODE     ---       #265
      01001103H   LINE      CODE     ---       #266
      01001109H   LINE      CODE     ---       #267
      0100113CH   LINE      CODE     ---       #268
      01001144H   LINE      CODE     ---       #269
      01001177H   LINE      CODE     ---       #270
      01001179H   LINE      CODE     ---       #271
      010011ADH   LINE      CODE     ---       #272
      010011ADH   LINE      CODE     ---       #273
      010011ADH   LINE      CODE     ---       #274
      010011ADH   LINE      CODE     ---       #275
      010011ADH   LINE      CODE     ---       #276
LX51 LINKER/LOCATER V4.66.30.0                                                        07/27/2019  23:22:19  PAGE 81


      010011B8H   LINE      CODE     ---       #277
      ---         BLOCKEND  ---      ---       LVL=0

      010045F2H   BLOCK     CODE     ---       LVL=0
      ---         BLOCKEND  ---      ---       LVL=0

      010045F8H   BLOCK     CODE     ---       LVL=0
      0000002FH   SYMBOL    DATA     BYTE      x
      00000030H   SYMBOL    DATA     BYTE      y
      00000031H   SYMBOL    DATA     ---       fb
      010045FCH   BLOCK     CODE     NEAR LAB  LVL=1
      00000031H   SYMBOL    DATA     ---       fb
      ---         BLOCKEND  ---      ---       LVL=1
      010045F8H   LINE      CODE     ---       #279
      010045FCH   LINE      CODE     ---       #280
      010045FCH   LINE      CODE     ---       #283
      0100460FH   LINE      CODE     ---       #284
      0100461CH   LINE      CODE     ---       #286
      01004627H   LINE      CODE     ---       #287
      0100463CH   LINE      CODE     ---       #288
      01004647H   LINE      CODE     ---       #290
      01004659H   LINE      CODE     ---       #292
      01004660H   LINE      CODE     ---       #293
      0100466AH   LINE      CODE     ---       #294
      0100466FH   LINE      CODE     ---       #295
      01004679H   LINE      CODE     ---       #296
      0100467AH   LINE      CODE     ---       #297
      01004689H   LINE      CODE     ---       #298
      01004689H   LINE      CODE     ---       #299
      ---         BLOCKEND  ---      ---       LVL=0

      010036A5H   BLOCK     CODE     ---       LVL=0
      0000002DH   SYMBOL    DATA     BYTE      x1
      0000002EH   SYMBOL    DATA     BYTE      x2
      0000002FH   SYMBOL    DATA     BYTE      y
      010036ABH   BLOCK     CODE     NEAR LAB  LVL=1
      00000006H   SYMBOL    DATA     BYTE      t
      00000030H   SYMBOL    DATA     ---       fb
      ---         BLOCKEND  ---      ---       LVL=1
      010036A5H   LINE      CODE     ---       #301
      010036ABH   LINE      CODE     ---       #302
      010036ABH   LINE      CODE     ---       #306
      010036C1H   LINE      CODE     ---       #307
      010036CAH   LINE      CODE     ---       #308
      010036DAH   LINE      CODE     ---       #310
      010036E1H   LINE      CODE     ---       #311
      010036E8H   LINE      CODE     ---       #312
      010036E8H   LINE      CODE     ---       #314
      010036F3H   LINE      CODE     ---       #315
      0100370FH   LINE      CODE     ---       #316
      0100371AH   LINE      CODE     ---       #318
      0100372CH   LINE      CODE     ---       #319
      01003733H   LINE      CODE     ---       #321
      0100373AH   LINE      CODE     ---       #322
      01003755H   LINE      CODE     ---       #323
      01003759H   LINE      CODE     ---       #324
      01003774H   LINE      CODE     ---       #325
      01003774H   LINE      CODE     ---       #326
      01003777H   LINE      CODE     ---       #327
      01003792H   LINE      CODE     ---       #328
      01003792H   LINE      CODE     ---       #329
      ---         BLOCKEND  ---      ---       LVL=0
LX51 LINKER/LOCATER V4.66.30.0                                                        07/27/2019  23:22:19  PAGE 82



      01002524H   BLOCK     CODE     ---       LVL=0
      0000002DH   SYMBOL    DATA     BYTE      x
      0000002EH   SYMBOL    DATA     BYTE      y1
      0000002FH   SYMBOL    DATA     BYTE      y2
      0100252AH   BLOCK     CODE     NEAR LAB  LVL=1
      00000006H   SYMBOL    DATA     BYTE      t
      00000030H   SYMBOL    DATA     BYTE      draw
      00000031H   SYMBOL    DATA     ---       fb
      00000033H   SYMBOL    DATA     CHAR      yoff
      00000034H   SYMBOL    DATA     CHAR      len
      ---         BLOCKEND  ---      ---       LVL=1
      01002524H   LINE      CODE     ---       #331
      0100252AH   LINE      CODE     ---       #332
      0100252AH   LINE      CODE     ---       #338
      01002540H   LINE      CODE     ---       #339
      01002550H   LINE      CODE     ---       #340
      01002559H   LINE      CODE     ---       #342
      01002560H   LINE      CODE     ---       #343
      01002567H   LINE      CODE     ---       #344
      01002567H   LINE      CODE     ---       #346
      0100256DH   LINE      CODE     ---       #348
      01002578H   LINE      CODE     ---       #349
      0100258DH   LINE      CODE     ---       #350
      01002598H   LINE      CODE     ---       #352
      010025A0H   LINE      CODE     ---       #355
      010025A7H   LINE      CODE     ---       #356
      010025AEH   LINE      CODE     ---       #358
      010025BDH   LINE      CODE     ---       #360
      010025CAH   LINE      CODE     ---       #361
      010025DDH   LINE      CODE     ---       #362
      010025DDH   LINE      CODE     ---       #364
      010025EAH   LINE      CODE     ---       #365
      010025F4H   LINE      CODE     ---       #366
      010025FAH   LINE      CODE     ---       #367
      01002604H   LINE      CODE     ---       #368
      01002606H   LINE      CODE     ---       #369
      01002615H   LINE      CODE     ---       #370
      01002615H   LINE      CODE     ---       #372
      01002625H   LINE      CODE     ---       #374
      0100262AH   LINE      CODE     ---       #375
      0100262AH   LINE      CODE     ---       #376
      0100262CH   LINE      CODE     ---       #379
      01002635H   LINE      CODE     ---       #380
      01002642H   LINE      CODE     ---       #381
      0100264BH   LINE      CODE     ---       #382
      01002651H   LINE      CODE     ---       #383
      0100265EH   LINE      CODE     ---       #384
      01002660H   LINE      CODE     ---       #385
      01002668H   LINE      CODE     ---       #386
      01002668H   LINE      CODE     ---       #388
      0100266EH   LINE      CODE     ---       #389
      0100267DH   LINE      CODE     ---       #390
      0100267FH   LINE      CODE     ---       #393
      01002688H   LINE      CODE     ---       #394
      0100269BH   LINE      CODE     ---       #396
      010026A8H   LINE      CODE     ---       #397
      010026B2H   LINE      CODE     ---       #398
      010026B7H   LINE      CODE     ---       #399
      010026C1H   LINE      CODE     ---       #400
      010026C2H   LINE      CODE     ---       #401
      010026D1H   LINE      CODE     ---       #402
LX51 LINKER/LOCATER V4.66.30.0                                                        07/27/2019  23:22:19  PAGE 83


      010026D1H   LINE      CODE     ---       #403
      010026D1H   LINE      CODE     ---       #404
      ---         BLOCKEND  ---      ---       LVL=0

      01003E39H   BLOCK     CODE     ---       LVL=0
      00000026H   SYMBOL    DATA     BYTE      x1
      00000027H   SYMBOL    DATA     BYTE      y1
      00000028H   SYMBOL    DATA     BYTE      x2
      00000029H   SYMBOL    DATA     BYTE      y2
      01003E3FH   BLOCK     CODE     NEAR LAB  LVL=1
      0000002AH   SYMBOL    DATA     CHAR      t
      0000002BH   SYMBOL    DATA     CHAR      dx
      0000002CH   SYMBOL    DATA     CHAR      dy
      00000004H   SYMBOL    DATA     CHAR      err
      0000002DH   SYMBOL    DATA     CHAR      ystep
      0000002EH   SYMBOL    DATA     CHAR      steep
      ---         BLOCKEND  ---      ---       LVL=1
      01003E39H   LINE      CODE     ---       #406
      01003E3FH   LINE      CODE     ---       #407
      01003E3FH   LINE      CODE     ---       #413
      01003E73H   LINE      CODE     ---       #415
      01003E77H   LINE      CODE     ---       #416
      01003E80H   LINE      CODE     ---       #417
      01003E89H   LINE      CODE     ---       #418
      01003E89H   LINE      CODE     ---       #420
      01003E90H   LINE      CODE     ---       #421
      01003E99H   LINE      CODE     ---       #422
      01003EA2H   LINE      CODE     ---       #423
      01003EA2H   LINE      CODE     ---       #425
      01003EA9H   LINE      CODE     ---       #426
      01003EB8H   LINE      CODE     ---       #428
      01003EBEH   LINE      CODE     ---       #430
      01003EC5H   LINE      CODE     ---       #431
      01003EC8H   LINE      CODE     ---       #432
      01003ECAH   LINE      CODE     ---       #433
      01003ECDH   LINE      CODE     ---       #434
      01003ECDH   LINE      CODE     ---       #436
      01003ED4H   LINE      CODE     ---       #437
      01003ED8H   LINE      CODE     ---       #438
      01003EDCH   LINE      CODE     ---       #439
      01003EDEH   LINE      CODE     ---       #440
      01003EE5H   LINE      CODE     ---       #441
      01003EE5H   LINE      CODE     ---       #443
      01003EEAH   LINE      CODE     ---       #445
      01003EF1H   LINE      CODE     ---       #446
      01003EF7H   LINE      CODE     ---       #447
      01003EFBH   LINE      CODE     ---       #448
      01003EFBH   LINE      CODE     ---       #449
      01003EFFH   LINE      CODE     ---       #450
      ---         BLOCKEND  ---      ---       LVL=0

      01005647H   BLOCK     CODE     ---       LVL=0
      00000026H   SYMBOL    DATA     BYTE      x1
      00000027H   SYMBOL    DATA     BYTE      y1
      00000028H   SYMBOL    DATA     BYTE      x2
      00000029H   SYMBOL    DATA     BYTE      y2
      01005647H   LINE      CODE     ---       #452
      0100564DH   LINE      CODE     ---       #453
      0100564DH   LINE      CODE     ---       #454
      01005658H   LINE      CODE     ---       #455
      01005661H   LINE      CODE     ---       #456
      0100566AH   LINE      CODE     ---       #457
LX51 LINKER/LOCATER V4.66.30.0                                                        07/27/2019  23:22:19  PAGE 84


      ---         BLOCKEND  ---      ---       LVL=0
      00000007H   SYMBOL    DATA     BYTE      t

      01003A2DH   BLOCK     CODE     ---       LVL=0
      00000025H   SYMBOL    DATA     CHAR      x
      00000004H   SYMBOL    DATA     CHAR      y
      00000026H   SYMBOL    DATA     BYTE      radius
      01003A33H   BLOCK     CODE     NEAR LAB  LVL=1
      00000027H   SYMBOL    DATA     CHAR      xs
      00000028H   SYMBOL    DATA     CHAR      ys
      00000029H   SYMBOL    DATA     CHAR      dp
      ---         BLOCKEND  ---      ---       LVL=1
      01003A2DH   LINE      CODE     ---       #475
      01003A33H   LINE      CODE     ---       #476
      01003A33H   LINE      CODE     ---       #477
      01003A36H   LINE      CODE     ---       #478
      01003A39H   LINE      CODE     ---       #479
      01003A3FH   LINE      CODE     ---       #481
      01003A3FH   LINE      CODE     ---       #482
      01003A4AH   LINE      CODE     ---       #483
      01003A55H   LINE      CODE     ---       #484
      01003A57H   LINE      CODE     ---       #485
      01003A6EH   LINE      CODE     ---       #486
      01003A6EH   LINE      CODE     ---       #488
      01003A7AH   LINE      CODE     ---       #489
      01003A87H   LINE      CODE     ---       #490
      01003A8EH   LINE      CODE     ---       #491
      01003A96H   LINE      CODE     ---       #492
      01003AA2H   LINE      CODE     ---       #493
      01003AAFH   LINE      CODE     ---       #494
      01003ABCH   LINE      CODE     ---       #495
      01003ACAH   LINE      CODE     ---       #496
      01003ADAH   LINE      CODE     ---       #498
      01003AE4H   LINE      CODE     ---       #499
      01003AEDH   LINE      CODE     ---       #500
      01003AF8H   LINE      CODE     ---       #501
      ---         BLOCKEND  ---      ---       LVL=0

      01004950H   BLOCK     CODE     ---       LVL=0
      0000002AH   SYMBOL    DATA     ---       font
      0000002CH   SYMBOL    DATA     ---       str
      0000002FH   SYMBOL    DATA     BYTE      len
      00000030H   SYMBOL    DATA     CHAR      extra_spacing
      0100495AH   BLOCK     CODE     NEAR LAB  LVL=1
      00000031H   SYMBOL    DATA     BYTE      first
      00000032H   SYMBOL    DATA     BYTE      chr_width
      00000033H   SYMBOL    DATA     BYTE      str_width
      00000034H   SYMBOL    DATA     BYTE      w
      ---         BLOCKEND  ---      ---       LVL=1
      01004950H   LINE      CODE     ---       #507
      0100495AH   LINE      CODE     ---       #508
      0100495AH   LINE      CODE     ---       #509
      01004963H   LINE      CODE     ---       #511
      01004966H   LINE      CODE     ---       #514
      01004969H   LINE      CODE     ---       #516
      01004970H   LINE      CODE     ---       #517
      010049ABH   LINE      CODE     ---       #519
      010049B7H   LINE      CODE     ---       #520
      010049BDH   LINE      CODE     ---       #521
      010049BDH   LINE      CODE     ---       #523
      010049C3H   LINE      CODE     ---       #524
      010049C5H   LINE      CODE     ---       #526
LX51 LINKER/LOCATER V4.66.30.0                                                        07/27/2019  23:22:19  PAGE 85


      010049D0H   LINE      CODE     ---       #528
      010049D1H   LINE      CODE     ---       #529
      ---         BLOCKEND  ---      ---       LVL=0

      01005B52H   BLOCK     CODE     ---       LVL=0
      00000082H   SYMBOL    DATA     ---       font
      01005B52H   LINE      CODE     ---       #531
      01005B56H   LINE      CODE     ---       #532
      01005B56H   LINE      CODE     ---       #533
      01005B5AH   LINE      CODE     ---       #534
      ---         BLOCKEND  ---      ---       LVL=0

      01002368H   BLOCK     CODE     ---       LVL=0
      02000000H   SYMBOL    PDATA    ---       font
      02000002H   SYMBOL    PDATA    ---       str
      02000005H   SYMBOL    PDATA    BYTE      len
      02000006H   SYMBOL    PDATA    CHAR      spacing
      01002373H   BLOCK     CODE     NEAR LAB  LVL=1
      0000003AH   SYMBOL    DATA     BYTE      height
      02000007H   SYMBOL    PDATA    BYTE      first
      02000008H   SYMBOL    PDATA    WORD      jt_siz
      0200000AH   SYMBOL    PDATA    WORD      last
      0000003BH   SYMBOL    DATA     BYTE      i
      00000007H   SYMBOL    DATA     BYTE      c
      0200000CH   SYMBOL    PDATA    BYTE      offset
      0200000DH   SYMBOL    PDATA    ---       jtdata
      0000003CH   SYMBOL    DATA     WORD      pos
      ---         BLOCKEND  ---      ---       LVL=1
      01002368H   LINE      CODE     ---       #536
      01002373H   LINE      CODE     ---       #538
      01002382H   LINE      CODE     ---       #539
      01002389H   LINE      CODE     ---       #540
      010023A4H   LINE      CODE     ---       #541
      010023ADH   LINE      CODE     ---       #551
      010023B5H   LINE      CODE     ---       #553
      010023C5H   LINE      CODE     ---       #554
      010023EAH   LINE      CODE     ---       #556
      010023F9H   LINE      CODE     ---       #559
      01002415H   LINE      CODE     ---       #560
      0100241AH   LINE      CODE     ---       #563
      01002437H   LINE      CODE     ---       #565
      01002452H   LINE      CODE     ---       #566
      0100247CH   LINE      CODE     ---       #571
      010024D6H   LINE      CODE     ---       #579
      010024D6H   LINE      CODE     ---       #581
      010024E6H   LINE      CODE     ---       #583
      010024F2H   LINE      CODE     ---       #584
      010024F6H   LINE      CODE     ---       #585
      010024F6H   LINE      CODE     ---       #587
      010024FFH   LINE      CODE     ---       #589
      01002510H   LINE      CODE     ---       #590
      0100251EH   LINE      CODE     ---       #591
      0100251EH   LINE      CODE     ---       #592
      0100251EH   LINE      CODE     ---       #593
      01002523H   LINE      CODE     ---       #594
      ---         BLOCKEND  ---      ---       LVL=0

      010056D1H   BLOCK     CODE     ---       LVL=0
      00000033H   SYMBOL    DATA     ---       font
      00000035H   SYMBOL    DATA     ---       str
      00000038H   SYMBOL    DATA     CHAR      extra_spacing
      010056DBH   BLOCK     CODE     NEAR LAB  LVL=1
LX51 LINKER/LOCATER V4.66.30.0                                                        07/27/2019  23:22:19  PAGE 86


      00000039H   SYMBOL    DATA     BYTE      lh
      00000007H   SYMBOL    DATA     BYTE      len
      ---         BLOCKEND  ---      ---       LVL=1
      010056D1H   LINE      CODE     ---       #596
      010056DBH   LINE      CODE     ---       #597
      010056DBH   LINE      CODE     ---       #601
      010056E4H   LINE      CODE     ---       #602
      010056E7H   LINE      CODE     ---       #604
      ---         BLOCKEND  ---      ---       LVL=0

      ---         MODULE    ---      ---       HSV2RGB
      00000049H   PUBLIC    DATA     BYTE      ?_hsv2rgb_8b?BYTE
      01002B5AH   PUBLIC    CODE     ---       _hsv2rgb_8b

      01002B5AH   BLOCK     CODE     ---       LVL=0
      00000049H   SYMBOL    DATA     WORD      h
      0000004BH   SYMBOL    DATA     BYTE      s
      0000004CH   SYMBOL    DATA     BYTE      v
      0000004DH   SYMBOL    DATA     ---       r
      00000050H   SYMBOL    DATA     ---       g
      00000053H   SYMBOL    DATA     ---       b
      01002B62H   BLOCK     CODE     NEAR LAB  LVL=1
      00000056H   SYMBOL    DATA     BYTE      sextant
      00000057H   SYMBOL    DATA     BYTE      bb
      00000058H   SYMBOL    DATA     WORD      ww
      0000005AH   SYMBOL    DATA     BYTE      h_fraction
      01002B91H   BLOCK     CODE     NEAR LAB  LVL=2
      0000005BH   SYMBOL    DATA     ---       tmp
      0000005BH   SYMBOL    DATA     ---       tmp
      ---         BLOCKEND  ---      ---       LVL=2
      01002BB1H   BLOCK     CODE     NEAR LAB  LVL=2
      0000005BH   SYMBOL    DATA     ---       tmp
      ---         BLOCKEND  ---      ---       LVL=2
      01002BD7H   BLOCK     CODE     NEAR LAB  LVL=2
      0000005BH   SYMBOL    DATA     ---       tmp
      0000005BH   SYMBOL    DATA     ---       tmp
      ---         BLOCKEND  ---      ---       LVL=2
      01002BDEH   BLOCK     CODE     NEAR LAB  LVL=2
      0000005BH   SYMBOL    DATA     ---       tmp
      ---         BLOCKEND  ---      ---       LVL=2
      ---         BLOCKEND  ---      ---       LVL=1
      01002B5AH   LINE      CODE     ---       #28
      01002B62H   LINE      CODE     ---       #29
      01002B62H   LINE      CODE     ---       #35
      01002B66H   LINE      CODE     ---       #36
      01002B7EH   LINE      CODE     ---       #38
      01002B7EH   LINE      CODE     ---       #40
      01002B82H   LINE      CODE     ---       #41
      01002B8CH   LINE      CODE     ---       #43
      01002BF9H   LINE      CODE     ---       #45
      01002C04H   LINE      CODE     ---       #52
      01002C09H   LINE      CODE     ---       #53
      01002C14H   LINE      CODE     ---       #54
      01002C1CH   LINE      CODE     ---       #55
      01002C27H   LINE      CODE     ---       #56
      01002C30H   LINE      CODE     ---       #58
      01002C34H   LINE      CODE     ---       #60
      01002C39H   LINE      CODE     ---       #66
      01002C53H   LINE      CODE     ---       #67
      01002C5EH   LINE      CODE     ---       #68
      01002C60H   LINE      CODE     ---       #69
      01002C63H   LINE      CODE     ---       #70
LX51 LINKER/LOCATER V4.66.30.0                                                        07/27/2019  23:22:19  PAGE 87


      01002C6EH   LINE      CODE     ---       #71
      01002C7BH   LINE      CODE     ---       #72
      01002C7BH   LINE      CODE     ---       #73
      01002C7DH   LINE      CODE     ---       #79
      01002C88H   LINE      CODE     ---       #80
      01002C93H   LINE      CODE     ---       #81
      01002C95H   LINE      CODE     ---       #82
      01002C98H   LINE      CODE     ---       #83
      01002CA3H   LINE      CODE     ---       #84
      01002CB0H   LINE      CODE     ---       #85
      01002CB9H   LINE      CODE     ---       #92
      01002CB9H   LINE      CODE     ---       #93
      ---         BLOCKEND  ---      ---       LVL=0

      ---         MODULE    ---      ---       RGBLED
      00000071H   PUBLIC    IDATA    ---       hsv
      00000065H   PUBLIC    IDATA    ---       rgb
      01002E07H   PUBLIC    CODE     ---       _rgbled_update
      000000A2H   SFRSYM    DATA     BYTE      SPI0CKR
      00000080H   SFRSYM    DATA     BYTE      P0
      000000D0H.2 SFRSYM    DATA     BIT       PSW_OV
      000000B1H   SFRSYM    DATA     BYTE      XOSC0CN
      00000090H   SFRSYM    DATA     BYTE      P1
      000000A0H   SFRSYM    DATA     BYTE      P2
      000000B0H   SFRSYM    DATA     BYTE      P3
      000000BCH   SFRSYM    DATA     BYTE      ADC0CF
      000000C8H   SFRSYM    DATA     BIT       TMR2CN0_T2XCLK
      000000C7H   SFRSYM    DATA     BYTE      P4
      000000C0H.7 SFRSYM    DATA     BIT       SMB0CN0_MASTER
      000000F9H   SFRSYM    DATA     WORD      PCA0
      000000E6H   SFRSYM    DATA     BYTE      EIE1
      000000C0H.7 SFRSYM    DATA     BIT       SMB1CN0_MASTER
      000000C0H.1 SFRSYM    DATA     BIT       SMB0CN0_ACK
      000000D7H   SFRSYM    DATA     BYTE      USB0XCN
      000000E7H   SFRSYM    DATA     BYTE      EIE2
      000000C0H.1 SFRSYM    DATA     BIT       SMB1CN0_ACK
      0000008FH   SFRSYM    DATA     BYTE      PSCTL
      000000E4H   SFRSYM    DATA     BYTE      IT01CF
      000000C8H   SFRSYM    DATA     BIT       TMR5CN0_T5XCLK
      000000C0H.6 SFRSYM    DATA     BIT       SMB0CN0_TXMODE
      000000C0H.6 SFRSYM    DATA     BIT       SMB1CN0_TXMODE
      000000BFH   SFRSYM    DATA     BYTE      SFRPAGE
      000000A4H   SFRSYM    DATA     BYTE      P0MDOUT
      000000A5H   SFRSYM    DATA     BYTE      P1MDOUT
      000000E8H.5 SFRSYM    DATA     BIT       ADC0CN0_ADINT
      000000CBH   SFRSYM    DATA     BYTE      TMR2RLH
      000000A6H   SFRSYM    DATA     BYTE      P2MDOUT
      000000A8H   SFRSYM    DATA     BYTE      IE
      00000093H   SFRSYM    DATA     BYTE      TMR3RLH
      000000A7H   SFRSYM    DATA     BYTE      P3MDOUT
      00000093H   SFRSYM    DATA     BYTE      TMR4RLH
      000000AEH   SFRSYM    DATA     BYTE      P4MDOUT
      000000F6H   SFRSYM    DATA     BYTE      EIP1
      000000CBH   SFRSYM    DATA     BYTE      TMR5RLH
      000000F7H   SFRSYM    DATA     BYTE      EIP2
      00000098H.2 SFRSYM    DATA     BIT       SCON0_RB8
      000000CAH   SFRSYM    DATA     BYTE      TMR2RLL
      000000FCH   SFRSYM    DATA     BYTE      PCA0CPH0
      00000092H   SFRSYM    DATA     BYTE      TMR3RLL
      000000EAH   SFRSYM    DATA     BYTE      PCA0CPH1
      00000098H.3 SFRSYM    DATA     BIT       SCON0_TB8
      000000F0H   SFRSYM    DATA     BIT       B_B0
LX51 LINKER/LOCATER V4.66.30.0                                                        07/27/2019  23:22:19  PAGE 88


      00000082H   SFRSYM    DATA     WORD      DP
      00000092H   SFRSYM    DATA     BYTE      TMR4RLL
      000000ECH   SFRSYM    DATA     BYTE      PCA0CPH2
      000000F0H.1 SFRSYM    DATA     BIT       B_B1
      000000C3H   SFRSYM    DATA     WORD      ADC0GT
      000000CAH   SFRSYM    DATA     BYTE      TMR5RLL
      000000EEH   SFRSYM    DATA     BYTE      PCA0CPH3
      000000F0H.2 SFRSYM    DATA     BIT       B_B2
      000000FBH   SFRSYM    DATA     BYTE      PCA0CPL0
      000000FEH   SFRSYM    DATA     BYTE      PCA0CPH4
      00000085H   SFRSYM    DATA     BYTE      EMI0CF
      000000F0H.3 SFRSYM    DATA     BIT       B_B3
      000000D9H   SFRSYM    DATA     BYTE      PCA0MD
      000000DAH   SFRSYM    DATA     BYTE      PCA0CPM0
      000000E9H   SFRSYM    DATA     BYTE      PCA0CPL1
      000000F0H.4 SFRSYM    DATA     BIT       B_B4
      000000DBH   SFRSYM    DATA     BYTE      PCA0CPM1
      000000EBH   SFRSYM    DATA     BYTE      PCA0CPL2
      000000F0H.5 SFRSYM    DATA     BIT       B_B5
      000000DCH   SFRSYM    DATA     BYTE      PCA0CPM2
      000000EDH   SFRSYM    DATA     BYTE      PCA0CPL3
      000000B8H   SFRSYM    DATA     BYTE      IP
      000000F0H.6 SFRSYM    DATA     BIT       B_B6
      000000C5H   SFRSYM    DATA     WORD      ADC0LT
      000000DDH   SFRSYM    DATA     BYTE      PCA0CPM3
      000000FDH   SFRSYM    DATA     BYTE      PCA0CPL4
      00000098H.5 SFRSYM    DATA     BIT       SCON0_MCE
      000000F0H.7 SFRSYM    DATA     BIT       B_B7
      000000DEH   SFRSYM    DATA     BYTE      PCA0CPM4
      000000E1H   SFRSYM    DATA     BYTE      XBR0
      000000C1H   SFRSYM    DATA     BYTE      SMB0CF
      000000E2H   SFRSYM    DATA     BYTE      XBR1
      000000C1H   SFRSYM    DATA     BYTE      SMB1CF
      000000AFH   SFRSYM    DATA     BYTE      PFE0CN
      000000AAH   SFRSYM    DATA     BYTE      EMI0CN
      000000C0H.5 SFRSYM    DATA     BIT       SMB0CN0_STA
      000000E3H   SFRSYM    DATA     BYTE      XBR2
      000000C0H.5 SFRSYM    DATA     BIT       SMB1CN0_STA
      000000E0H   SFRSYM    DATA     BIT       ACC_ACC0
      000000D1H   SFRSYM    DATA     BYTE      REF0CN
      000000B2H   SFRSYM    DATA     BYTE      HFO0CN
      0000008EH   SFRSYM    DATA     BYTE      CKCON0
      000000E0H.1 SFRSYM    DATA     BIT       ACC_ACC1
      000000E4H   SFRSYM    DATA     BYTE      CKCON1
      000000C8H.2 SFRSYM    DATA     BIT       TMR2CN0_TR2
      000000E0H.2 SFRSYM    DATA     BIT       ACC_ACC2
      000000E0H.3 SFRSYM    DATA     BIT       ACC_ACC3
      00000081H   SFRSYM    DATA     BYTE      SP
      0000009DH   SFRSYM    DATA     BYTE      CMP0MD
      000000E0H.4 SFRSYM    DATA     BIT       ACC_ACC4
      00000086H   SFRSYM    DATA     BYTE      LFO0CN
      00000084H   SFRSYM    DATA     BYTE      EMI0TC
      0000009CH   SFRSYM    DATA     BYTE      CMP1MD
      000000D8H   SFRSYM    DATA     BIT       PCA0CN0_CCF0
      000000E0H.5 SFRSYM    DATA     BIT       ACC_ACC5
      000000D8H.1 SFRSYM    DATA     BIT       PCA0CN0_CCF1
      000000E0H.6 SFRSYM    DATA     BIT       ACC_ACC6
      000000CCH   SFRSYM    DATA     WORD      TMR2
      000000D8H.2 SFRSYM    DATA     BIT       PCA0CN0_CCF2
      000000E0H.7 SFRSYM    DATA     BIT       ACC_ACC7
      00000094H   SFRSYM    DATA     WORD      TMR3
      000000C8H.2 SFRSYM    DATA     BIT       TMR5CN0_TR5
LX51 LINKER/LOCATER V4.66.30.0                                                        07/27/2019  23:22:19  PAGE 89


      000000D8H.3 SFRSYM    DATA     BIT       PCA0CN0_CCF3
      00000094H   SFRSYM    DATA     WORD      TMR4
      000000ACH   SFRSYM    DATA     BYTE      SBCON1
      000000D8H.4 SFRSYM    DATA     BIT       PCA0CN0_CCF4
      000000CCH   SFRSYM    DATA     WORD      TMR5
      000000C0H.3 SFRSYM    DATA     BIT       SMB0CN0_ACKRQ
      000000FFH   SFRSYM    DATA     BYTE      VDM0CN
      000000F1H   SFRSYM    DATA     BYTE      P0MDIN
      000000C0H.3 SFRSYM    DATA     BIT       SMB1CN0_ACKRQ
      00000098H.4 SFRSYM    DATA     BIT       SCON0_REN
      000000F2H   SFRSYM    DATA     BYTE      P1MDIN
      000000F3H   SFRSYM    DATA     BYTE      P2MDIN
      000000C0H.4 SFRSYM    DATA     BIT       SMB0CN0_STO
      000000F4H   SFRSYM    DATA     BYTE      P3MDIN
      000000C0H.4 SFRSYM    DATA     BIT       SMB1CN0_STO
      000000B5H   SFRSYM    DATA     BYTE      SBRLH1
      000000F5H   SFRSYM    DATA     BYTE      P4MDIN
      000000D0H.3 SFRSYM    DATA     BIT       PSW_RS0
      000000D8H.7 SFRSYM    DATA     BIT       PCA0CN0_CF
      000000F8H.4 SFRSYM    DATA     BIT       SPI0CN0_RXOVRN
      000000D0H.4 SFRSYM    DATA     BIT       PSW_RS1
      000000B4H   SFRSYM    DATA     BYTE      SBRLL1
      000000E8H.7 SFRSYM    DATA     BIT       ADC0CN0_ADEN
      00000089H   SFRSYM    DATA     BYTE      TMOD
      00000088H   SFRSYM    DATA     BYTE      TCON
      000000D0H   SFRSYM    DATA     BIT       PSW_PARITY
      000000A8H.4 SFRSYM    DATA     BIT       IE_ES0
      0000009FH   SFRSYM    DATA     BYTE      CMP0MX
      000000A8H.1 SFRSYM    DATA     BIT       IE_ET0
      0000009EH   SFRSYM    DATA     BYTE      CMP1MX
      000000A8H.3 SFRSYM    DATA     BIT       IE_ET1
      000000D4H   SFRSYM    DATA     BYTE      P0SKIP
      000000C8H.1 SFRSYM    DATA     BIT       TMR2CN0_T2CSS
      000000A8H.5 SFRSYM    DATA     BIT       IE_ET2
      000000D5H   SFRSYM    DATA     BYTE      P1SKIP
      000000D6H   SFRSYM    DATA     BYTE      P2SKIP
      000000E8H   SFRSYM    DATA     BYTE      ADC0CN0
      000000A8H   SFRSYM    DATA     BIT       IE_EX0
      000000DFH   SFRSYM    DATA     BYTE      P3SKIP
      000000D8H.6 SFRSYM    DATA     BIT       PCA0CN0_CR
      000000A8H.2 SFRSYM    DATA     BIT       IE_EX1
      00000098H.7 SFRSYM    DATA     BIT       SCON0_SMODE
      000000A9H   SFRSYM    DATA     BYTE      CLKSEL
      000000F8H   SFRSYM    DATA     BIT       SPI0CN0_SPIEN
      000000F0H   SFRSYM    DATA     BYTE      B
      000000BEH   SFRSYM    DATA     BYTE      ADC0H
      000000E8H.6 SFRSYM    DATA     BIT       ADC0CN0_ADTM
      000000CAH   SFRSYM    DATA     WORD      TMR2RL
      000000BDH   SFRSYM    DATA     BYTE      ADC0L
      00000092H   SFRSYM    DATA     WORD      TMR3RL
      00000092H   SFRSYM    DATA     WORD      TMR4RL
      000000D8H   SFRSYM    DATA     BYTE      PCA0CN0
      000000E0H   SFRSYM    DATA     BYTE      ACC
      000000CAH   SFRSYM    DATA     WORD      TMR5RL
      000000FBH   SFRSYM    DATA     WORD      PCA0CP0
      000000E9H   SFRSYM    DATA     WORD      PCA0CP1
      000000EBH   SFRSYM    DATA     WORD      PCA0CP2
      000000EDH   SFRSYM    DATA     WORD      PCA0CP3
      0000008CH   SFRSYM    DATA     BYTE      TH0
      000000B8H.4 SFRSYM    DATA     BIT       IP_PS0
      000000FDH   SFRSYM    DATA     WORD      PCA0CP4
      0000008DH   SFRSYM    DATA     BYTE      TH1
LX51 LINKER/LOCATER V4.66.30.0                                                        07/27/2019  23:22:19  PAGE 90


      000000FAH   SFRSYM    DATA     BYTE      PCA0H
      000000B8H.1 SFRSYM    DATA     BIT       IP_PT0
      000000B8H.3 SFRSYM    DATA     BIT       IP_PT1
      000000C0H.2 SFRSYM    DATA     BIT       SMB0CN0_ARBLOST
      000000B8H.5 SFRSYM    DATA     BIT       IP_PT2
      0000008AH   SFRSYM    DATA     BYTE      TL0
      000000F8H.1 SFRSYM    DATA     BIT       SPI0CN0_TXBMT
      000000C0H.2 SFRSYM    DATA     BIT       SMB1CN0_ARBLOST
      000000D0H.5 SFRSYM    DATA     BIT       PSW_F0
      000000A8H.6 SFRSYM    DATA     BIT       IE_ESPI0
      0000008BH   SFRSYM    DATA     BYTE      TL1
      000000F9H   SFRSYM    DATA     BYTE      PCA0L
      000000C0H   SFRSYM    DATA     BIT       SMB0CN0_SI
      000000D0H.1 SFRSYM    DATA     BIT       PSW_F1
      00000080H   SFRSYM    DATA     BIT       P0_B0
      000000B8H   SFRSYM    DATA     BIT       IP_PX0
      000000C9H   SFRSYM    DATA     BYTE      REG01CN
      000000C0H   SFRSYM    DATA     BIT       SMB1CN0_SI
      00000090H   SFRSYM    DATA     BIT       P1_B0
      00000080H.1 SFRSYM    DATA     BIT       P0_B1
      000000B8H.2 SFRSYM    DATA     BIT       IP_PX1
      0000009BH   SFRSYM    DATA     BYTE      CMP0CN0
      00000088H.1 SFRSYM    DATA     BIT       TCON_IE0
      000000A0H   SFRSYM    DATA     BIT       P2_B0
      00000090H.1 SFRSYM    DATA     BIT       P1_B1
      00000080H.2 SFRSYM    DATA     BIT       P0_B2
      0000009AH   SFRSYM    DATA     BYTE      CMP1CN0
      00000088H.3 SFRSYM    DATA     BIT       TCON_IE1
      000000B0H   SFRSYM    DATA     BIT       P3_B0
      000000A0H.1 SFRSYM    DATA     BIT       P2_B1
      00000090H.2 SFRSYM    DATA     BIT       P1_B2
      00000080H.3 SFRSYM    DATA     BIT       P0_B3
      000000C0H   SFRSYM    DATA     BYTE      SMB0CN0
      000000B0H.1 SFRSYM    DATA     BIT       P3_B1
      000000A0H.2 SFRSYM    DATA     BIT       P2_B2
      00000090H.3 SFRSYM    DATA     BIT       P1_B3
      00000080H.4 SFRSYM    DATA     BIT       P0_B4
      000000C0H   SFRSYM    DATA     BYTE      SMB1CN0
      000000B0H.2 SFRSYM    DATA     BIT       P3_B2
      000000A0H.3 SFRSYM    DATA     BIT       P2_B3
      00000090H.4 SFRSYM    DATA     BIT       P1_B4
      00000080H.5 SFRSYM    DATA     BIT       P0_B5
      000000B0H.3 SFRSYM    DATA     BIT       P3_B3
      000000A0H.4 SFRSYM    DATA     BIT       P2_B4
      00000090H.5 SFRSYM    DATA     BIT       P1_B5
      00000080H.6 SFRSYM    DATA     BIT       P0_B6
      000000B0H.4 SFRSYM    DATA     BIT       P3_B4
      000000A0H.5 SFRSYM    DATA     BIT       P2_B5
      00000090H.6 SFRSYM    DATA     BIT       P1_B6
      00000080H.7 SFRSYM    DATA     BIT       P0_B7
      000000B0H.5 SFRSYM    DATA     BIT       P3_B5
      000000A0H.6 SFRSYM    DATA     BIT       P2_B6
      00000090H.7 SFRSYM    DATA     BIT       P1_B7
      000000B0H.6 SFRSYM    DATA     BIT       P3_B6
      000000A0H.7 SFRSYM    DATA     BIT       P2_B7
      000000B0H.7 SFRSYM    DATA     BIT       P3_B7
      00000083H   SFRSYM    DATA     BYTE      DPH
      000000C4H   SFRSYM    DATA     BYTE      ADC0GTH
      000000C8H.7 SFRSYM    DATA     BIT       TMR2CN0_TF2H
      000000C8H.3 SFRSYM    DATA     BIT       TMR2CN0_T2SPLIT
      000000D0H.6 SFRSYM    DATA     BIT       PSW_AC
      000000F8H   SFRSYM    DATA     BYTE      SPI0CN0
LX51 LINKER/LOCATER V4.66.30.0                                                        07/27/2019  23:22:19  PAGE 91


      000000B3H   SFRSYM    DATA     BYTE      HFO0CAL
      00000088H.5 SFRSYM    DATA     BIT       TCON_TF0
      00000098H   SFRSYM    DATA     BIT       SCON0_RI
      00000082H   SFRSYM    DATA     BYTE      DPL
      00000088H.7 SFRSYM    DATA     BIT       TCON_TF1
      00000099H   SFRSYM    DATA     BYTE      SBUF0
      00000087H   SFRSYM    DATA     BYTE      PCON0
      000000C3H   SFRSYM    DATA     BYTE      ADC0GTL
      000000C8H.6 SFRSYM    DATA     BIT       TMR2CN0_TF2L
      00000098H.1 SFRSYM    DATA     BIT       SCON0_TI
      000000E8H   SFRSYM    DATA     BIT       ADC0CN0_ADCM0
      000000D3H   SFRSYM    DATA     BYTE      SBUF1
      000000C6H   SFRSYM    DATA     BYTE      ADC0LTH
      00000088H   SFRSYM    DATA     BIT       TCON_IT0
      000000E8H.1 SFRSYM    DATA     BIT       ADC0CN0_ADCM1
      000000EFH   SFRSYM    DATA     BYTE      RSTSRC
      000000C8H.7 SFRSYM    DATA     BIT       TMR5CN0_TF5H
      000000C8H.3 SFRSYM    DATA     BIT       TMR5CN0_T5SPLIT
      00000088H.2 SFRSYM    DATA     BIT       TCON_IT1
      000000E8H.2 SFRSYM    DATA     BIT       ADC0CN0_ADCM2
      00000098H   SFRSYM    DATA     BYTE      SCON0
      000000E8H.3 SFRSYM    DATA     BIT       ADC0CN0_ADWINT
      000000B4H   SFRSYM    DATA     WORD      SBRL1
      000000E5H   SFRSYM    DATA     BYTE      SMOD1
      000000D2H   SFRSYM    DATA     BYTE      SCON1
      000000BAH   SFRSYM    DATA     BYTE      AMX0N
      000000E8H.4 SFRSYM    DATA     BIT       ADC0CN0_ADBUSY
      000000CEH   SFRSYM    DATA     BYTE      SMB0ADM
      000000C5H   SFRSYM    DATA     BYTE      ADC0LTL
      000000F8H.5 SFRSYM    DATA     BIT       SPI0CN0_MODF
      000000B8H.6 SFRSYM    DATA     BIT       IP_PSPI0
      000000CEH   SFRSYM    DATA     BYTE      SMB1ADM
      000000BBH   SFRSYM    DATA     BYTE      AMX0P
      000000C8H.6 SFRSYM    DATA     BIT       TMR5CN0_TF5L
      000000C8H   SFRSYM    DATA     BYTE      TMR2CN0
      00000091H   SFRSYM    DATA     BYTE      TMR3CN0
      00000091H   SFRSYM    DATA     BYTE      TMR4CN0
      000000C8H   SFRSYM    DATA     BYTE      TMR5CN0
      000000CFH   SFRSYM    DATA     BYTE      SMB0ADR
      00000088H.4 SFRSYM    DATA     BIT       TCON_TR0
      000000CFH   SFRSYM    DATA     BYTE      SMB1ADR
      000000C8H.4 SFRSYM    DATA     BIT       TMR2CN0_TF2CEN
      00000088H.6 SFRSYM    DATA     BIT       TCON_TR1
      000000C2H   SFRSYM    DATA     BYTE      SMB0DAT
      000000CDH   SFRSYM    DATA     BYTE      TMR2H
      000000A1H   SFRSYM    DATA     BYTE      SPI0CFG
      000000C2H   SFRSYM    DATA     BYTE      SMB1DAT
      00000095H   SFRSYM    DATA     BYTE      TMR3H
      00000095H   SFRSYM    DATA     BYTE      TMR4H
      000000CDH   SFRSYM    DATA     BYTE      TMR5H
      000000CCH   SFRSYM    DATA     BYTE      TMR2L
      000000F8H.7 SFRSYM    DATA     BIT       SPI0CN0_SPIF
      00000096H   SFRSYM    DATA     BYTE      USB0ADR
      00000094H   SFRSYM    DATA     BYTE      TMR3L
      000000A8H.7 SFRSYM    DATA     BIT       IE_EA
      00000094H   SFRSYM    DATA     BYTE      TMR4L
      00000097H   SFRSYM    DATA     BYTE      USB0DAT
      000000CCH   SFRSYM    DATA     BYTE      TMR5L
      000000B6H   SFRSYM    DATA     BYTE      FLSCL
      000000C8H.5 SFRSYM    DATA     BIT       TMR2CN0_TF2LEN
      000000F8H.6 SFRSYM    DATA     BIT       SPI0CN0_WCOL
      000000F8H.2 SFRSYM    DATA     BIT       SPI0CN0_NSSMD0
LX51 LINKER/LOCATER V4.66.30.0                                                        07/27/2019  23:22:19  PAGE 92


      000000D0H.7 SFRSYM    DATA     BIT       PSW_CY
      000000A3H   SFRSYM    DATA     BYTE      SPI0DAT
      000000F8H.3 SFRSYM    DATA     BIT       SPI0CN0_NSSMD1
      000000BDH   SFRSYM    DATA     WORD      ADC0
      000000B9H   SFRSYM    DATA     BYTE      SMBTC
      000000D0H   SFRSYM    DATA     BYTE      PSW
      000000C8H.5 SFRSYM    DATA     BIT       TMR5CN0_TF5LEN
      000000B7H   SFRSYM    DATA     BYTE      FLKEY

      01002E07H   BLOCK     CODE     ---       LVL=0
      00000007H   SYMBOL    DATA     BYTE      idx
      01002E07H   BLOCK     CODE     NEAR LAB  LVL=1
      00000043H   SYMBOL    DATA     BYTE      i
      00000044H   SYMBOL    DATA     ---       p
      00000045H   SYMBOL    DATA     ---       pwm
      00000007H   SYMBOL    DATA     BYTE      sfrsave
      ---         BLOCKEND  ---      ---       LVL=1
      01002E07H   LINE      CODE     ---       #16
      01002E07H   LINE      CODE     ---       #23
      01002E15H   LINE      CODE     ---       #24
      01002E15H   LINE      CODE     ---       #25
      01002E18H   LINE      CODE     ---       #26
      01002E76H   LINE      CODE     ---       #27
      01002E80H   LINE      CODE     ---       #29
      01002E80H   LINE      CODE     ---       #30
      01002E85H   LINE      CODE     ---       #31
      01002E8AH   LINE      CODE     ---       #32
      01002E8DH   LINE      CODE     ---       #33
      01002E8DH   LINE      CODE     ---       #36
      01002E90H   LINE      CODE     ---       #38
      01002E99H   LINE      CODE     ---       #39
      01002E9BH   LINE      CODE     ---       #40
      01002E9BH   LINE      CODE     ---       #42
      01002EA6H   LINE      CODE     ---       #43
      01002EACH   LINE      CODE     ---       #44
      01002EB3H   LINE      CODE     ---       #47
      01002EB5H   LINE      CODE     ---       #48
      01002EB8H   LINE      CODE     ---       #58
      01002EBBH   LINE      CODE     ---       #59
      01002EC4H   LINE      CODE     ---       #60
      01002EC7H   LINE      CODE     ---       #61
      01002ECAH   LINE      CODE     ---       #62
      01002ECDH   LINE      CODE     ---       #63
      01002ECDH   LINE      CODE     ---       #65
      01002ED6H   LINE      CODE     ---       #66
      01002ED9H   LINE      CODE     ---       #67
      01002EDCH   LINE      CODE     ---       #68
      01002EDFH   LINE      CODE     ---       #69
      01002EDFH   LINE      CODE     ---       #71
      01002EE8H   LINE      CODE     ---       #72
      01002EEBH   LINE      CODE     ---       #73
      01002EEEH   LINE      CODE     ---       #74
      01002EF1H   LINE      CODE     ---       #75
      01002EF1H   LINE      CODE     ---       #77
      01002EF6H   LINE      CODE     ---       #78
      01002EF9H   LINE      CODE     ---       #79
      01002EFCH   LINE      CODE     ---       #80
      01002EFFH   LINE      CODE     ---       #81
      01002EFFH   LINE      CODE     ---       #84
      01002F02H   LINE      CODE     ---       #85
      01002F08H   LINE      CODE     ---       #86
      01002F0EH   LINE      CODE     ---       #87
LX51 LINKER/LOCATER V4.66.30.0                                                        07/27/2019  23:22:19  PAGE 93


      01002F10H   LINE      CODE     ---       #88
      01002F13H   LINE      CODE     ---       #89
      01002F13H   LINE      CODE     ---       #91
      01002F15H   LINE      CODE     ---       #92
      01002F1BH   LINE      CODE     ---       #93
      01002F21H   LINE      CODE     ---       #94
      01002F23H   LINE      CODE     ---       #95
      01002F26H   LINE      CODE     ---       #96
      01002F26H   LINE      CODE     ---       #98
      01002F28H   LINE      CODE     ---       #99
      01002F2EH   LINE      CODE     ---       #100
      01002F34H   LINE      CODE     ---       #101
      01002F36H   LINE      CODE     ---       #102
      01002F39H   LINE      CODE     ---       #103
      01002F39H   LINE      CODE     ---       #105
      01002F3BH   LINE      CODE     ---       #106
      01002F41H   LINE      CODE     ---       #107
      01002F47H   LINE      CODE     ---       #108
      01002F49H   LINE      CODE     ---       #109
      01002F4CH   LINE      CODE     ---       #110
      01002F4CH   LINE      CODE     ---       #112
      01002F4EH   LINE      CODE     ---       #113
      ---         BLOCKEND  ---      ---       LVL=0

      ---         MODULE    ---      ---       FONT
      0100B6E0H   PUBLIC    CONST    ---       font_Orbitron_28
      0100A794H   PUBLIC    CONST    ---       font_Nimbus_Sans_L_25
      01009994H   PUBLIC    CONST    ---       font_Crushed_25
      010089C4H   PUBLIC    CONST    ---       font_Chewy_24
      01007670H   PUBLIC    CONST    ---       font_DialogInput_Bold_24
      01006636H   PUBLIC    CONST    ---       font_Nimbus_Mono_L_Bold_20
      0100601EH   PUBLIC    CONST    ---       font_DejaVu_Sans_Mono_Bold_11
      01005BB3H   PUBLIC    CONST    ---       font_Dialog_plain_8

      ---         MODULE    ---      ---       PWR
      01005A89H   PUBLIC    CODE     ---       PWR_enterIdle
      000000A2H   SFRSYM    DATA     BYTE      SPI0CKR
      00000080H   SFRSYM    DATA     BYTE      P0
      000000D0H.2 SFRSYM    DATA     BIT       PSW_OV
      000000B1H   SFRSYM    DATA     BYTE      XOSC0CN
      00000090H   SFRSYM    DATA     BYTE      P1
      000000A0H   SFRSYM    DATA     BYTE      P2
      000000B0H   SFRSYM    DATA     BYTE      P3
      000000BCH   SFRSYM    DATA     BYTE      ADC0CF
      000000C8H   SFRSYM    DATA     BIT       TMR2CN0_T2XCLK
      000000C7H   SFRSYM    DATA     BYTE      P4
      000000C0H.7 SFRSYM    DATA     BIT       SMB0CN0_MASTER
      000000F9H   SFRSYM    DATA     WORD      PCA0
      000000E6H   SFRSYM    DATA     BYTE      EIE1
      000000C0H.7 SFRSYM    DATA     BIT       SMB1CN0_MASTER
      000000C0H.1 SFRSYM    DATA     BIT       SMB0CN0_ACK
      000000D7H   SFRSYM    DATA     BYTE      USB0XCN
      000000E7H   SFRSYM    DATA     BYTE      EIE2
      000000C0H.1 SFRSYM    DATA     BIT       SMB1CN0_ACK
      0000008FH   SFRSYM    DATA     BYTE      PSCTL
      000000E4H   SFRSYM    DATA     BYTE      IT01CF
      000000C8H   SFRSYM    DATA     BIT       TMR5CN0_T5XCLK
      000000C0H.6 SFRSYM    DATA     BIT       SMB0CN0_TXMODE
      000000C0H.6 SFRSYM    DATA     BIT       SMB1CN0_TXMODE
      000000BFH   SFRSYM    DATA     BYTE      SFRPAGE
      000000A4H   SFRSYM    DATA     BYTE      P0MDOUT
      000000A5H   SFRSYM    DATA     BYTE      P1MDOUT
LX51 LINKER/LOCATER V4.66.30.0                                                        07/27/2019  23:22:19  PAGE 94


      000000E8H.5 SFRSYM    DATA     BIT       ADC0CN0_ADINT
      000000CBH   SFRSYM    DATA     BYTE      TMR2RLH
      000000A6H   SFRSYM    DATA     BYTE      P2MDOUT
      000000A8H   SFRSYM    DATA     BYTE      IE
      00000093H   SFRSYM    DATA     BYTE      TMR3RLH
      000000A7H   SFRSYM    DATA     BYTE      P3MDOUT
      00000093H   SFRSYM    DATA     BYTE      TMR4RLH
      000000AEH   SFRSYM    DATA     BYTE      P4MDOUT
      000000F6H   SFRSYM    DATA     BYTE      EIP1
      000000CBH   SFRSYM    DATA     BYTE      TMR5RLH
      000000F7H   SFRSYM    DATA     BYTE      EIP2
      00000098H.2 SFRSYM    DATA     BIT       SCON0_RB8
      000000CAH   SFRSYM    DATA     BYTE      TMR2RLL
      000000FCH   SFRSYM    DATA     BYTE      PCA0CPH0
      00000092H   SFRSYM    DATA     BYTE      TMR3RLL
      000000EAH   SFRSYM    DATA     BYTE      PCA0CPH1
      00000098H.3 SFRSYM    DATA     BIT       SCON0_TB8
      000000F0H   SFRSYM    DATA     BIT       B_B0
      00000082H   SFRSYM    DATA     WORD      DP
      00000092H   SFRSYM    DATA     BYTE      TMR4RLL
      000000ECH   SFRSYM    DATA     BYTE      PCA0CPH2
      000000F0H.1 SFRSYM    DATA     BIT       B_B1
      000000C3H   SFRSYM    DATA     WORD      ADC0GT
      000000CAH   SFRSYM    DATA     BYTE      TMR5RLL
      000000EEH   SFRSYM    DATA     BYTE      PCA0CPH3
      000000F0H.2 SFRSYM    DATA     BIT       B_B2
      000000FBH   SFRSYM    DATA     BYTE      PCA0CPL0
      000000FEH   SFRSYM    DATA     BYTE      PCA0CPH4
      00000085H   SFRSYM    DATA     BYTE      EMI0CF
      000000F0H.3 SFRSYM    DATA     BIT       B_B3
      000000D9H   SFRSYM    DATA     BYTE      PCA0MD
      000000DAH   SFRSYM    DATA     BYTE      PCA0CPM0
      000000E9H   SFRSYM    DATA     BYTE      PCA0CPL1
      000000F0H.4 SFRSYM    DATA     BIT       B_B4
      000000DBH   SFRSYM    DATA     BYTE      PCA0CPM1
      000000EBH   SFRSYM    DATA     BYTE      PCA0CPL2
      000000F0H.5 SFRSYM    DATA     BIT       B_B5
      000000DCH   SFRSYM    DATA     BYTE      PCA0CPM2
      000000EDH   SFRSYM    DATA     BYTE      PCA0CPL3
      000000B8H   SFRSYM    DATA     BYTE      IP
      000000F0H.6 SFRSYM    DATA     BIT       B_B6
      000000C5H   SFRSYM    DATA     WORD      ADC0LT
      000000DDH   SFRSYM    DATA     BYTE      PCA0CPM3
      000000FDH   SFRSYM    DATA     BYTE      PCA0CPL4
      00000098H.5 SFRSYM    DATA     BIT       SCON0_MCE
      000000F0H.7 SFRSYM    DATA     BIT       B_B7
      000000DEH   SFRSYM    DATA     BYTE      PCA0CPM4
      000000E1H   SFRSYM    DATA     BYTE      XBR0
      000000C1H   SFRSYM    DATA     BYTE      SMB0CF
      000000E2H   SFRSYM    DATA     BYTE      XBR1
      000000C1H   SFRSYM    DATA     BYTE      SMB1CF
      000000AFH   SFRSYM    DATA     BYTE      PFE0CN
      000000AAH   SFRSYM    DATA     BYTE      EMI0CN
      000000C0H.5 SFRSYM    DATA     BIT       SMB0CN0_STA
      000000E3H   SFRSYM    DATA     BYTE      XBR2
      000000C0H.5 SFRSYM    DATA     BIT       SMB1CN0_STA
      000000E0H   SFRSYM    DATA     BIT       ACC_ACC0
      000000D1H   SFRSYM    DATA     BYTE      REF0CN
      000000B2H   SFRSYM    DATA     BYTE      HFO0CN
      0000008EH   SFRSYM    DATA     BYTE      CKCON0
      000000E0H.1 SFRSYM    DATA     BIT       ACC_ACC1
      000000E4H   SFRSYM    DATA     BYTE      CKCON1
LX51 LINKER/LOCATER V4.66.30.0                                                        07/27/2019  23:22:19  PAGE 95


      000000C8H.2 SFRSYM    DATA     BIT       TMR2CN0_TR2
      000000E0H.2 SFRSYM    DATA     BIT       ACC_ACC2
      000000E0H.3 SFRSYM    DATA     BIT       ACC_ACC3
      00000081H   SFRSYM    DATA     BYTE      SP
      0000009DH   SFRSYM    DATA     BYTE      CMP0MD
      000000E0H.4 SFRSYM    DATA     BIT       ACC_ACC4
      00000086H   SFRSYM    DATA     BYTE      LFO0CN
      00000084H   SFRSYM    DATA     BYTE      EMI0TC
      0000009CH   SFRSYM    DATA     BYTE      CMP1MD
      000000D8H   SFRSYM    DATA     BIT       PCA0CN0_CCF0
      000000E0H.5 SFRSYM    DATA     BIT       ACC_ACC5
      000000D8H.1 SFRSYM    DATA     BIT       PCA0CN0_CCF1
      000000E0H.6 SFRSYM    DATA     BIT       ACC_ACC6
      000000CCH   SFRSYM    DATA     WORD      TMR2
      000000D8H.2 SFRSYM    DATA     BIT       PCA0CN0_CCF2
      000000E0H.7 SFRSYM    DATA     BIT       ACC_ACC7
      00000094H   SFRSYM    DATA     WORD      TMR3
      000000C8H.2 SFRSYM    DATA     BIT       TMR5CN0_TR5
      000000D8H.3 SFRSYM    DATA     BIT       PCA0CN0_CCF3
      00000094H   SFRSYM    DATA     WORD      TMR4
      000000ACH   SFRSYM    DATA     BYTE      SBCON1
      000000D8H.4 SFRSYM    DATA     BIT       PCA0CN0_CCF4
      000000CCH   SFRSYM    DATA     WORD      TMR5
      000000C0H.3 SFRSYM    DATA     BIT       SMB0CN0_ACKRQ
      000000FFH   SFRSYM    DATA     BYTE      VDM0CN
      000000F1H   SFRSYM    DATA     BYTE      P0MDIN
      000000C0H.3 SFRSYM    DATA     BIT       SMB1CN0_ACKRQ
      00000098H.4 SFRSYM    DATA     BIT       SCON0_REN
      000000F2H   SFRSYM    DATA     BYTE      P1MDIN
      000000F3H   SFRSYM    DATA     BYTE      P2MDIN
      000000C0H.4 SFRSYM    DATA     BIT       SMB0CN0_STO
      000000F4H   SFRSYM    DATA     BYTE      P3MDIN
      000000C0H.4 SFRSYM    DATA     BIT       SMB1CN0_STO
      000000B5H   SFRSYM    DATA     BYTE      SBRLH1
      000000F5H   SFRSYM    DATA     BYTE      P4MDIN
      000000D0H.3 SFRSYM    DATA     BIT       PSW_RS0
      000000D8H.7 SFRSYM    DATA     BIT       PCA0CN0_CF
      000000F8H.4 SFRSYM    DATA     BIT       SPI0CN0_RXOVRN
      000000D0H.4 SFRSYM    DATA     BIT       PSW_RS1
      000000B4H   SFRSYM    DATA     BYTE      SBRLL1
      000000E8H.7 SFRSYM    DATA     BIT       ADC0CN0_ADEN
      00000089H   SFRSYM    DATA     BYTE      TMOD
      00000088H   SFRSYM    DATA     BYTE      TCON
      000000D0H   SFRSYM    DATA     BIT       PSW_PARITY
      000000A8H.4 SFRSYM    DATA     BIT       IE_ES0
      0000009FH   SFRSYM    DATA     BYTE      CMP0MX
      000000A8H.1 SFRSYM    DATA     BIT       IE_ET0
      0000009EH   SFRSYM    DATA     BYTE      CMP1MX
      000000A8H.3 SFRSYM    DATA     BIT       IE_ET1
      000000D4H   SFRSYM    DATA     BYTE      P0SKIP
      000000C8H.1 SFRSYM    DATA     BIT       TMR2CN0_T2CSS
      000000A8H.5 SFRSYM    DATA     BIT       IE_ET2
      000000D5H   SFRSYM    DATA     BYTE      P1SKIP
      000000D6H   SFRSYM    DATA     BYTE      P2SKIP
      000000E8H   SFRSYM    DATA     BYTE      ADC0CN0
      000000A8H   SFRSYM    DATA     BIT       IE_EX0
      000000DFH   SFRSYM    DATA     BYTE      P3SKIP
      000000D8H.6 SFRSYM    DATA     BIT       PCA0CN0_CR
      000000A8H.2 SFRSYM    DATA     BIT       IE_EX1
      00000098H.7 SFRSYM    DATA     BIT       SCON0_SMODE
      000000A9H   SFRSYM    DATA     BYTE      CLKSEL
      000000F8H   SFRSYM    DATA     BIT       SPI0CN0_SPIEN
LX51 LINKER/LOCATER V4.66.30.0                                                        07/27/2019  23:22:19  PAGE 96


      000000F0H   SFRSYM    DATA     BYTE      B
      000000BEH   SFRSYM    DATA     BYTE      ADC0H
      000000E8H.6 SFRSYM    DATA     BIT       ADC0CN0_ADTM
      000000CAH   SFRSYM    DATA     WORD      TMR2RL
      000000BDH   SFRSYM    DATA     BYTE      ADC0L
      00000092H   SFRSYM    DATA     WORD      TMR3RL
      00000092H   SFRSYM    DATA     WORD      TMR4RL
      000000D8H   SFRSYM    DATA     BYTE      PCA0CN0
      000000E0H   SFRSYM    DATA     BYTE      ACC
      000000CAH   SFRSYM    DATA     WORD      TMR5RL
      000000FBH   SFRSYM    DATA     WORD      PCA0CP0
      000000E9H   SFRSYM    DATA     WORD      PCA0CP1
      000000EBH   SFRSYM    DATA     WORD      PCA0CP2
      000000EDH   SFRSYM    DATA     WORD      PCA0CP3
      0000008CH   SFRSYM    DATA     BYTE      TH0
      000000B8H.4 SFRSYM    DATA     BIT       IP_PS0
      000000FDH   SFRSYM    DATA     WORD      PCA0CP4
      0000008DH   SFRSYM    DATA     BYTE      TH1
      000000FAH   SFRSYM    DATA     BYTE      PCA0H
      000000B8H.1 SFRSYM    DATA     BIT       IP_PT0
      000000B8H.3 SFRSYM    DATA     BIT       IP_PT1
      000000C0H.2 SFRSYM    DATA     BIT       SMB0CN0_ARBLOST
      000000B8H.5 SFRSYM    DATA     BIT       IP_PT2
      0000008AH   SFRSYM    DATA     BYTE      TL0
      000000F8H.1 SFRSYM    DATA     BIT       SPI0CN0_TXBMT
      000000C0H.2 SFRSYM    DATA     BIT       SMB1CN0_ARBLOST
      000000D0H.5 SFRSYM    DATA     BIT       PSW_F0
      000000A8H.6 SFRSYM    DATA     BIT       IE_ESPI0
      0000008BH   SFRSYM    DATA     BYTE      TL1
      000000F9H   SFRSYM    DATA     BYTE      PCA0L
      000000C0H   SFRSYM    DATA     BIT       SMB0CN0_SI
      000000D0H.1 SFRSYM    DATA     BIT       PSW_F1
      00000080H   SFRSYM    DATA     BIT       P0_B0
      000000B8H   SFRSYM    DATA     BIT       IP_PX0
      000000C9H   SFRSYM    DATA     BYTE      REG01CN
      000000C0H   SFRSYM    DATA     BIT       SMB1CN0_SI
      00000090H   SFRSYM    DATA     BIT       P1_B0
      00000080H.1 SFRSYM    DATA     BIT       P0_B1
      000000B8H.2 SFRSYM    DATA     BIT       IP_PX1
      0000009BH   SFRSYM    DATA     BYTE      CMP0CN0
      00000088H.1 SFRSYM    DATA     BIT       TCON_IE0
      000000A0H   SFRSYM    DATA     BIT       P2_B0
      00000090H.1 SFRSYM    DATA     BIT       P1_B1
      00000080H.2 SFRSYM    DATA     BIT       P0_B2
      0000009AH   SFRSYM    DATA     BYTE      CMP1CN0
      00000088H.3 SFRSYM    DATA     BIT       TCON_IE1
      000000B0H   SFRSYM    DATA     BIT       P3_B0
      000000A0H.1 SFRSYM    DATA     BIT       P2_B1
      00000090H.2 SFRSYM    DATA     BIT       P1_B2
      00000080H.3 SFRSYM    DATA     BIT       P0_B3
      000000C0H   SFRSYM    DATA     BYTE      SMB0CN0
      000000B0H.1 SFRSYM    DATA     BIT       P3_B1
      000000A0H.2 SFRSYM    DATA     BIT       P2_B2
      00000090H.3 SFRSYM    DATA     BIT       P1_B3
      00000080H.4 SFRSYM    DATA     BIT       P0_B4
      000000C0H   SFRSYM    DATA     BYTE      SMB1CN0
      000000B0H.2 SFRSYM    DATA     BIT       P3_B2
      000000A0H.3 SFRSYM    DATA     BIT       P2_B3
      00000090H.4 SFRSYM    DATA     BIT       P1_B4
      00000080H.5 SFRSYM    DATA     BIT       P0_B5
      000000B0H.3 SFRSYM    DATA     BIT       P3_B3
      000000A0H.4 SFRSYM    DATA     BIT       P2_B4
LX51 LINKER/LOCATER V4.66.30.0                                                        07/27/2019  23:22:19  PAGE 97


      00000090H.5 SFRSYM    DATA     BIT       P1_B5
      00000080H.6 SFRSYM    DATA     BIT       P0_B6
      000000B0H.4 SFRSYM    DATA     BIT       P3_B4
      000000A0H.5 SFRSYM    DATA     BIT       P2_B5
      00000090H.6 SFRSYM    DATA     BIT       P1_B6
      00000080H.7 SFRSYM    DATA     BIT       P0_B7
      000000B0H.5 SFRSYM    DATA     BIT       P3_B5
      000000A0H.6 SFRSYM    DATA     BIT       P2_B6
      00000090H.7 SFRSYM    DATA     BIT       P1_B7
      000000B0H.6 SFRSYM    DATA     BIT       P3_B6
      000000A0H.7 SFRSYM    DATA     BIT       P2_B7
      000000B0H.7 SFRSYM    DATA     BIT       P3_B7
      00000083H   SFRSYM    DATA     BYTE      DPH
      000000C4H   SFRSYM    DATA     BYTE      ADC0GTH
      000000C8H.7 SFRSYM    DATA     BIT       TMR2CN0_TF2H
      000000C8H.3 SFRSYM    DATA     BIT       TMR2CN0_T2SPLIT
      000000D0H.6 SFRSYM    DATA     BIT       PSW_AC
      000000F8H   SFRSYM    DATA     BYTE      SPI0CN0
      000000B3H   SFRSYM    DATA     BYTE      HFO0CAL
      00000088H.5 SFRSYM    DATA     BIT       TCON_TF0
      00000098H   SFRSYM    DATA     BIT       SCON0_RI
      00000082H   SFRSYM    DATA     BYTE      DPL
      00000088H.7 SFRSYM    DATA     BIT       TCON_TF1
      00000099H   SFRSYM    DATA     BYTE      SBUF0
      00000087H   SFRSYM    DATA     BYTE      PCON0
      000000C3H   SFRSYM    DATA     BYTE      ADC0GTL
      000000C8H.6 SFRSYM    DATA     BIT       TMR2CN0_TF2L
      00000098H.1 SFRSYM    DATA     BIT       SCON0_TI
      000000E8H   SFRSYM    DATA     BIT       ADC0CN0_ADCM0
      000000D3H   SFRSYM    DATA     BYTE      SBUF1
      000000C6H   SFRSYM    DATA     BYTE      ADC0LTH
      00000088H   SFRSYM    DATA     BIT       TCON_IT0
      000000E8H.1 SFRSYM    DATA     BIT       ADC0CN0_ADCM1
      000000EFH   SFRSYM    DATA     BYTE      RSTSRC
      000000C8H.7 SFRSYM    DATA     BIT       TMR5CN0_TF5H
      000000C8H.3 SFRSYM    DATA     BIT       TMR5CN0_T5SPLIT
      00000088H.2 SFRSYM    DATA     BIT       TCON_IT1
      000000E8H.2 SFRSYM    DATA     BIT       ADC0CN0_ADCM2
      00000098H   SFRSYM    DATA     BYTE      SCON0
      000000E8H.3 SFRSYM    DATA     BIT       ADC0CN0_ADWINT
      000000B4H   SFRSYM    DATA     WORD      SBRL1
      000000E5H   SFRSYM    DATA     BYTE      SMOD1
      000000D2H   SFRSYM    DATA     BYTE      SCON1
      000000BAH   SFRSYM    DATA     BYTE      AMX0N
      000000E8H.4 SFRSYM    DATA     BIT       ADC0CN0_ADBUSY
      000000CEH   SFRSYM    DATA     BYTE      SMB0ADM
      000000C5H   SFRSYM    DATA     BYTE      ADC0LTL
      000000F8H.5 SFRSYM    DATA     BIT       SPI0CN0_MODF
      000000B8H.6 SFRSYM    DATA     BIT       IP_PSPI0
      000000CEH   SFRSYM    DATA     BYTE      SMB1ADM
      000000BBH   SFRSYM    DATA     BYTE      AMX0P
      000000C8H.6 SFRSYM    DATA     BIT       TMR5CN0_TF5L
      000000C8H   SFRSYM    DATA     BYTE      TMR2CN0
      00000091H   SFRSYM    DATA     BYTE      TMR3CN0
      00000091H   SFRSYM    DATA     BYTE      TMR4CN0
      000000C8H   SFRSYM    DATA     BYTE      TMR5CN0
      000000CFH   SFRSYM    DATA     BYTE      SMB0ADR
      00000088H.4 SFRSYM    DATA     BIT       TCON_TR0
      000000CFH   SFRSYM    DATA     BYTE      SMB1ADR
      000000C8H.4 SFRSYM    DATA     BIT       TMR2CN0_TF2CEN
      00000088H.6 SFRSYM    DATA     BIT       TCON_TR1
      000000C2H   SFRSYM    DATA     BYTE      SMB0DAT
LX51 LINKER/LOCATER V4.66.30.0                                                        07/27/2019  23:22:19  PAGE 98


      000000CDH   SFRSYM    DATA     BYTE      TMR2H
      000000A1H   SFRSYM    DATA     BYTE      SPI0CFG
      000000C2H   SFRSYM    DATA     BYTE      SMB1DAT
      00000095H   SFRSYM    DATA     BYTE      TMR3H
      00000095H   SFRSYM    DATA     BYTE      TMR4H
      000000CDH   SFRSYM    DATA     BYTE      TMR5H
      000000CCH   SFRSYM    DATA     BYTE      TMR2L
      000000F8H.7 SFRSYM    DATA     BIT       SPI0CN0_SPIF
      00000096H   SFRSYM    DATA     BYTE      USB0ADR
      00000094H   SFRSYM    DATA     BYTE      TMR3L
      000000A8H.7 SFRSYM    DATA     BIT       IE_EA
      00000094H   SFRSYM    DATA     BYTE      TMR4L
      00000097H   SFRSYM    DATA     BYTE      USB0DAT
      000000CCH   SFRSYM    DATA     BYTE      TMR5L
      000000B6H   SFRSYM    DATA     BYTE      FLSCL
      000000C8H.5 SFRSYM    DATA     BIT       TMR2CN0_TF2LEN
      000000F8H.6 SFRSYM    DATA     BIT       SPI0CN0_WCOL
      000000F8H.2 SFRSYM    DATA     BIT       SPI0CN0_NSSMD0
      000000D0H.7 SFRSYM    DATA     BIT       PSW_CY
      000000A3H   SFRSYM    DATA     BYTE      SPI0DAT
      000000F8H.3 SFRSYM    DATA     BIT       SPI0CN0_NSSMD1
      000000BDH   SFRSYM    DATA     WORD      ADC0
      000000B9H   SFRSYM    DATA     BYTE      SMBTC
      000000D0H   SFRSYM    DATA     BYTE      PSW
      000000C8H.5 SFRSYM    DATA     BIT       TMR5CN0_TF5LEN
      000000B7H   SFRSYM    DATA     BYTE      FLKEY

      01005A89H   BLOCK     CODE     ---       LVL=0
      01005A89H   BLOCK     CODE     NEAR LAB  LVL=1
      00000007H   SYMBOL    DATA     BYTE      save_sfrpage
      ---         BLOCKEND  ---      ---       LVL=1
      01005A89H   LINE      CODE     ---       #17
      01005A89H   LINE      CODE     ---       #18
      01005A89H   LINE      CODE     ---       #19
      01005A8BH   LINE      CODE     ---       #20
      01005A8EH   LINE      CODE     ---       #24
      01005A91H   LINE      CODE     ---       #25
      01005A94H   LINE      CODE     ---       #27
      01005A96H   LINE      CODE     ---       #28
      ---         BLOCKEND  ---      ---       LVL=0
      00000006H   SYMBOL    DATA     BYTE      save_ie
      00000005H   SYMBOL    DATA     BYTE      save_clksel
      00000007H   SYMBOL    DATA     BYTE      save_sfrpage

      ---         MODULE    ---      ---       ASSERT

      ---         MODULE    ---      ---       USER_CONFIG
      0000001FH   PUBLIC    DATA     BYTE      sysflags
      00000085H   PUBLIC    IDATA    BYTE      last_empty_offset
      02000393H   PUBLIC    XDATA    ---       uconf
      00000084H   PUBLIC    IDATA    BYTE      last_valid_offset
      01003D71H   PUBLIC    CODE     ---       uconf_write
      01004D48H   PUBLIC    CODE     ---       uconf_load
      000000A2H   SFRSYM    DATA     BYTE      SPI0CKR
      00000080H   SFRSYM    DATA     BYTE      P0
      000000D0H.2 SFRSYM    DATA     BIT       PSW_OV
      000000B1H   SFRSYM    DATA     BYTE      XOSC0CN
      00000090H   SFRSYM    DATA     BYTE      P1
      000000A0H   SFRSYM    DATA     BYTE      P2
      000000B0H   SFRSYM    DATA     BYTE      P3
      000000BCH   SFRSYM    DATA     BYTE      ADC0CF
      000000C8H   SFRSYM    DATA     BIT       TMR2CN0_T2XCLK
LX51 LINKER/LOCATER V4.66.30.0                                                        07/27/2019  23:22:19  PAGE 99


      000000C7H   SFRSYM    DATA     BYTE      P4
      000000C0H.7 SFRSYM    DATA     BIT       SMB0CN0_MASTER
      000000F9H   SFRSYM    DATA     WORD      PCA0
      000000E6H   SFRSYM    DATA     BYTE      EIE1
      000000C0H.7 SFRSYM    DATA     BIT       SMB1CN0_MASTER
      000000C0H.1 SFRSYM    DATA     BIT       SMB0CN0_ACK
      000000D7H   SFRSYM    DATA     BYTE      USB0XCN
      000000E7H   SFRSYM    DATA     BYTE      EIE2
      000000C0H.1 SFRSYM    DATA     BIT       SMB1CN0_ACK
      0000008FH   SFRSYM    DATA     BYTE      PSCTL
      000000E4H   SFRSYM    DATA     BYTE      IT01CF
      000000C8H   SFRSYM    DATA     BIT       TMR5CN0_T5XCLK
      000000C0H.6 SFRSYM    DATA     BIT       SMB0CN0_TXMODE
      000000C0H.6 SFRSYM    DATA     BIT       SMB1CN0_TXMODE
      000000BFH   SFRSYM    DATA     BYTE      SFRPAGE
      000000A4H   SFRSYM    DATA     BYTE      P0MDOUT
      000000A5H   SFRSYM    DATA     BYTE      P1MDOUT
      000000E8H.5 SFRSYM    DATA     BIT       ADC0CN0_ADINT
      000000CBH   SFRSYM    DATA     BYTE      TMR2RLH
      000000A6H   SFRSYM    DATA     BYTE      P2MDOUT
      000000A8H   SFRSYM    DATA     BYTE      IE
      00000093H   SFRSYM    DATA     BYTE      TMR3RLH
      000000A7H   SFRSYM    DATA     BYTE      P3MDOUT
      00000093H   SFRSYM    DATA     BYTE      TMR4RLH
      000000AEH   SFRSYM    DATA     BYTE      P4MDOUT
      000000F6H   SFRSYM    DATA     BYTE      EIP1
      000000CBH   SFRSYM    DATA     BYTE      TMR5RLH
      000000F7H   SFRSYM    DATA     BYTE      EIP2
      00000098H.2 SFRSYM    DATA     BIT       SCON0_RB8
      000000CAH   SFRSYM    DATA     BYTE      TMR2RLL
      000000FCH   SFRSYM    DATA     BYTE      PCA0CPH0
      00000092H   SFRSYM    DATA     BYTE      TMR3RLL
      000000EAH   SFRSYM    DATA     BYTE      PCA0CPH1
      00000098H.3 SFRSYM    DATA     BIT       SCON0_TB8
      000000F0H   SFRSYM    DATA     BIT       B_B0
      00000082H   SFRSYM    DATA     WORD      DP
      00000092H   SFRSYM    DATA     BYTE      TMR4RLL
      000000ECH   SFRSYM    DATA     BYTE      PCA0CPH2
      000000F0H.1 SFRSYM    DATA     BIT       B_B1
      000000C3H   SFRSYM    DATA     WORD      ADC0GT
      000000CAH   SFRSYM    DATA     BYTE      TMR5RLL
      000000EEH   SFRSYM    DATA     BYTE      PCA0CPH3
      000000F0H.2 SFRSYM    DATA     BIT       B_B2
      000000FBH   SFRSYM    DATA     BYTE      PCA0CPL0
      000000FEH   SFRSYM    DATA     BYTE      PCA0CPH4
      00000085H   SFRSYM    DATA     BYTE      EMI0CF
      000000F0H.3 SFRSYM    DATA     BIT       B_B3
      000000D9H   SFRSYM    DATA     BYTE      PCA0MD
      000000DAH   SFRSYM    DATA     BYTE      PCA0CPM0
      000000E9H   SFRSYM    DATA     BYTE      PCA0CPL1
      000000F0H.4 SFRSYM    DATA     BIT       B_B4
      000000DBH   SFRSYM    DATA     BYTE      PCA0CPM1
      000000EBH   SFRSYM    DATA     BYTE      PCA0CPL2
      000000F0H.5 SFRSYM    DATA     BIT       B_B5
      000000DCH   SFRSYM    DATA     BYTE      PCA0CPM2
      000000EDH   SFRSYM    DATA     BYTE      PCA0CPL3
      000000B8H   SFRSYM    DATA     BYTE      IP
      000000F0H.6 SFRSYM    DATA     BIT       B_B6
      000000C5H   SFRSYM    DATA     WORD      ADC0LT
      000000DDH   SFRSYM    DATA     BYTE      PCA0CPM3
      000000FDH   SFRSYM    DATA     BYTE      PCA0CPL4
      00000098H.5 SFRSYM    DATA     BIT       SCON0_MCE
LX51 LINKER/LOCATER V4.66.30.0                                                        07/27/2019  23:22:19  PAGE 100


      000000F0H.7 SFRSYM    DATA     BIT       B_B7
      000000DEH   SFRSYM    DATA     BYTE      PCA0CPM4
      000000E1H   SFRSYM    DATA     BYTE      XBR0
      000000C1H   SFRSYM    DATA     BYTE      SMB0CF
      000000E2H   SFRSYM    DATA     BYTE      XBR1
      000000C1H   SFRSYM    DATA     BYTE      SMB1CF
      000000AFH   SFRSYM    DATA     BYTE      PFE0CN
      000000AAH   SFRSYM    DATA     BYTE      EMI0CN
      000000C0H.5 SFRSYM    DATA     BIT       SMB0CN0_STA
      000000E3H   SFRSYM    DATA     BYTE      XBR2
      000000C0H.5 SFRSYM    DATA     BIT       SMB1CN0_STA
      000000E0H   SFRSYM    DATA     BIT       ACC_ACC0
      000000D1H   SFRSYM    DATA     BYTE      REF0CN
      000000B2H   SFRSYM    DATA     BYTE      HFO0CN
      0000008EH   SFRSYM    DATA     BYTE      CKCON0
      000000E0H.1 SFRSYM    DATA     BIT       ACC_ACC1
      000000E4H   SFRSYM    DATA     BYTE      CKCON1
      000000C8H.2 SFRSYM    DATA     BIT       TMR2CN0_TR2
      000000E0H.2 SFRSYM    DATA     BIT       ACC_ACC2
      000000E0H.3 SFRSYM    DATA     BIT       ACC_ACC3
      00000081H   SFRSYM    DATA     BYTE      SP
      0000009DH   SFRSYM    DATA     BYTE      CMP0MD
      000000E0H.4 SFRSYM    DATA     BIT       ACC_ACC4
      00000086H   SFRSYM    DATA     BYTE      LFO0CN
      00000084H   SFRSYM    DATA     BYTE      EMI0TC
      0000009CH   SFRSYM    DATA     BYTE      CMP1MD
      000000D8H   SFRSYM    DATA     BIT       PCA0CN0_CCF0
      000000E0H.5 SFRSYM    DATA     BIT       ACC_ACC5
      000000D8H.1 SFRSYM    DATA     BIT       PCA0CN0_CCF1
      000000E0H.6 SFRSYM    DATA     BIT       ACC_ACC6
      000000CCH   SFRSYM    DATA     WORD      TMR2
      000000D8H.2 SFRSYM    DATA     BIT       PCA0CN0_CCF2
      000000E0H.7 SFRSYM    DATA     BIT       ACC_ACC7
      00000094H   SFRSYM    DATA     WORD      TMR3
      000000C8H.2 SFRSYM    DATA     BIT       TMR5CN0_TR5
      000000D8H.3 SFRSYM    DATA     BIT       PCA0CN0_CCF3
      00000094H   SFRSYM    DATA     WORD      TMR4
      000000ACH   SFRSYM    DATA     BYTE      SBCON1
      000000D8H.4 SFRSYM    DATA     BIT       PCA0CN0_CCF4
      000000CCH   SFRSYM    DATA     WORD      TMR5
      000000C0H.3 SFRSYM    DATA     BIT       SMB0CN0_ACKRQ
      000000FFH   SFRSYM    DATA     BYTE      VDM0CN
      000000F1H   SFRSYM    DATA     BYTE      P0MDIN
      000000C0H.3 SFRSYM    DATA     BIT       SMB1CN0_ACKRQ
      00000098H.4 SFRSYM    DATA     BIT       SCON0_REN
      000000F2H   SFRSYM    DATA     BYTE      P1MDIN
      000000F3H   SFRSYM    DATA     BYTE      P2MDIN
      000000C0H.4 SFRSYM    DATA     BIT       SMB0CN0_STO
      000000F4H   SFRSYM    DATA     BYTE      P3MDIN
      000000C0H.4 SFRSYM    DATA     BIT       SMB1CN0_STO
      000000B5H   SFRSYM    DATA     BYTE      SBRLH1
      000000F5H   SFRSYM    DATA     BYTE      P4MDIN
      000000D0H.3 SFRSYM    DATA     BIT       PSW_RS0
      000000D8H.7 SFRSYM    DATA     BIT       PCA0CN0_CF
      000000F8H.4 SFRSYM    DATA     BIT       SPI0CN0_RXOVRN
      000000D0H.4 SFRSYM    DATA     BIT       PSW_RS1
      000000B4H   SFRSYM    DATA     BYTE      SBRLL1
      000000E8H.7 SFRSYM    DATA     BIT       ADC0CN0_ADEN
      00000089H   SFRSYM    DATA     BYTE      TMOD
      00000088H   SFRSYM    DATA     BYTE      TCON
      000000D0H   SFRSYM    DATA     BIT       PSW_PARITY
      000000A8H.4 SFRSYM    DATA     BIT       IE_ES0
LX51 LINKER/LOCATER V4.66.30.0                                                        07/27/2019  23:22:19  PAGE 101


      0000009FH   SFRSYM    DATA     BYTE      CMP0MX
      000000A8H.1 SFRSYM    DATA     BIT       IE_ET0
      0000009EH   SFRSYM    DATA     BYTE      CMP1MX
      000000A8H.3 SFRSYM    DATA     BIT       IE_ET1
      000000D4H   SFRSYM    DATA     BYTE      P0SKIP
      000000C8H.1 SFRSYM    DATA     BIT       TMR2CN0_T2CSS
      000000A8H.5 SFRSYM    DATA     BIT       IE_ET2
      000000D5H   SFRSYM    DATA     BYTE      P1SKIP
      000000D6H   SFRSYM    DATA     BYTE      P2SKIP
      000000E8H   SFRSYM    DATA     BYTE      ADC0CN0
      000000A8H   SFRSYM    DATA     BIT       IE_EX0
      000000DFH   SFRSYM    DATA     BYTE      P3SKIP
      000000D8H.6 SFRSYM    DATA     BIT       PCA0CN0_CR
      000000A8H.2 SFRSYM    DATA     BIT       IE_EX1
      00000098H.7 SFRSYM    DATA     BIT       SCON0_SMODE
      000000A9H   SFRSYM    DATA     BYTE      CLKSEL
      000000F8H   SFRSYM    DATA     BIT       SPI0CN0_SPIEN
      000000F0H   SFRSYM    DATA     BYTE      B
      000000BEH   SFRSYM    DATA     BYTE      ADC0H
      000000E8H.6 SFRSYM    DATA     BIT       ADC0CN0_ADTM
      000000CAH   SFRSYM    DATA     WORD      TMR2RL
      000000BDH   SFRSYM    DATA     BYTE      ADC0L
      00000092H   SFRSYM    DATA     WORD      TMR3RL
      00000092H   SFRSYM    DATA     WORD      TMR4RL
      000000D8H   SFRSYM    DATA     BYTE      PCA0CN0
      000000E0H   SFRSYM    DATA     BYTE      ACC
      000000CAH   SFRSYM    DATA     WORD      TMR5RL
      000000FBH   SFRSYM    DATA     WORD      PCA0CP0
      000000E9H   SFRSYM    DATA     WORD      PCA0CP1
      000000EBH   SFRSYM    DATA     WORD      PCA0CP2
      000000EDH   SFRSYM    DATA     WORD      PCA0CP3
      0000008CH   SFRSYM    DATA     BYTE      TH0
      000000B8H.4 SFRSYM    DATA     BIT       IP_PS0
      000000FDH   SFRSYM    DATA     WORD      PCA0CP4
      0000008DH   SFRSYM    DATA     BYTE      TH1
      000000FAH   SFRSYM    DATA     BYTE      PCA0H
      000000B8H.1 SFRSYM    DATA     BIT       IP_PT0
      000000B8H.3 SFRSYM    DATA     BIT       IP_PT1
      000000C0H.2 SFRSYM    DATA     BIT       SMB0CN0_ARBLOST
      000000B8H.5 SFRSYM    DATA     BIT       IP_PT2
      0000008AH   SFRSYM    DATA     BYTE      TL0
      000000F8H.1 SFRSYM    DATA     BIT       SPI0CN0_TXBMT
      000000C0H.2 SFRSYM    DATA     BIT       SMB1CN0_ARBLOST
      000000D0H.5 SFRSYM    DATA     BIT       PSW_F0
      000000A8H.6 SFRSYM    DATA     BIT       IE_ESPI0
      0000008BH   SFRSYM    DATA     BYTE      TL1
      000000F9H   SFRSYM    DATA     BYTE      PCA0L
      000000C0H   SFRSYM    DATA     BIT       SMB0CN0_SI
      000000D0H.1 SFRSYM    DATA     BIT       PSW_F1
      00000080H   SFRSYM    DATA     BIT       P0_B0
      000000B8H   SFRSYM    DATA     BIT       IP_PX0
      000000C9H   SFRSYM    DATA     BYTE      REG01CN
      000000C0H   SFRSYM    DATA     BIT       SMB1CN0_SI
      00000090H   SFRSYM    DATA     BIT       P1_B0
      00000080H.1 SFRSYM    DATA     BIT       P0_B1
      000000B8H.2 SFRSYM    DATA     BIT       IP_PX1
      0000009BH   SFRSYM    DATA     BYTE      CMP0CN0
      00000088H.1 SFRSYM    DATA     BIT       TCON_IE0
      000000A0H   SFRSYM    DATA     BIT       P2_B0
      00000090H.1 SFRSYM    DATA     BIT       P1_B1
      00000080H.2 SFRSYM    DATA     BIT       P0_B2
      0000009AH   SFRSYM    DATA     BYTE      CMP1CN0
LX51 LINKER/LOCATER V4.66.30.0                                                        07/27/2019  23:22:19  PAGE 102


      00000088H.3 SFRSYM    DATA     BIT       TCON_IE1
      000000B0H   SFRSYM    DATA     BIT       P3_B0
      000000A0H.1 SFRSYM    DATA     BIT       P2_B1
      00000090H.2 SFRSYM    DATA     BIT       P1_B2
      00000080H.3 SFRSYM    DATA     BIT       P0_B3
      000000C0H   SFRSYM    DATA     BYTE      SMB0CN0
      000000B0H.1 SFRSYM    DATA     BIT       P3_B1
      000000A0H.2 SFRSYM    DATA     BIT       P2_B2
      00000090H.3 SFRSYM    DATA     BIT       P1_B3
      00000080H.4 SFRSYM    DATA     BIT       P0_B4
      000000C0H   SFRSYM    DATA     BYTE      SMB1CN0
      000000B0H.2 SFRSYM    DATA     BIT       P3_B2
      000000A0H.3 SFRSYM    DATA     BIT       P2_B3
      00000090H.4 SFRSYM    DATA     BIT       P1_B4
      00000080H.5 SFRSYM    DATA     BIT       P0_B5
      000000B0H.3 SFRSYM    DATA     BIT       P3_B3
      000000A0H.4 SFRSYM    DATA     BIT       P2_B4
      00000090H.5 SFRSYM    DATA     BIT       P1_B5
      00000080H.6 SFRSYM    DATA     BIT       P0_B6
      000000B0H.4 SFRSYM    DATA     BIT       P3_B4
      000000A0H.5 SFRSYM    DATA     BIT       P2_B5
      00000090H.6 SFRSYM    DATA     BIT       P1_B6
      00000080H.7 SFRSYM    DATA     BIT       P0_B7
      000000B0H.5 SFRSYM    DATA     BIT       P3_B5
      000000A0H.6 SFRSYM    DATA     BIT       P2_B6
      00000090H.7 SFRSYM    DATA     BIT       P1_B7
      000000B0H.6 SFRSYM    DATA     BIT       P3_B6
      000000A0H.7 SFRSYM    DATA     BIT       P2_B7
      000000B0H.7 SFRSYM    DATA     BIT       P3_B7
      00000083H   SFRSYM    DATA     BYTE      DPH
      000000C4H   SFRSYM    DATA     BYTE      ADC0GTH
      000000C8H.7 SFRSYM    DATA     BIT       TMR2CN0_TF2H
      000000C8H.3 SFRSYM    DATA     BIT       TMR2CN0_T2SPLIT
      000000D0H.6 SFRSYM    DATA     BIT       PSW_AC
      000000F8H   SFRSYM    DATA     BYTE      SPI0CN0
      000000B3H   SFRSYM    DATA     BYTE      HFO0CAL
      00000088H.5 SFRSYM    DATA     BIT       TCON_TF0
      00000098H   SFRSYM    DATA     BIT       SCON0_RI
      00000082H   SFRSYM    DATA     BYTE      DPL
      00000088H.7 SFRSYM    DATA     BIT       TCON_TF1
      00000099H   SFRSYM    DATA     BYTE      SBUF0
      00000087H   SFRSYM    DATA     BYTE      PCON0
      000000C3H   SFRSYM    DATA     BYTE      ADC0GTL
      000000C8H.6 SFRSYM    DATA     BIT       TMR2CN0_TF2L
      00000098H.1 SFRSYM    DATA     BIT       SCON0_TI
      000000E8H   SFRSYM    DATA     BIT       ADC0CN0_ADCM0
      000000D3H   SFRSYM    DATA     BYTE      SBUF1
      000000C6H   SFRSYM    DATA     BYTE      ADC0LTH
      00000088H   SFRSYM    DATA     BIT       TCON_IT0
      000000E8H.1 SFRSYM    DATA     BIT       ADC0CN0_ADCM1
      000000EFH   SFRSYM    DATA     BYTE      RSTSRC
      000000C8H.7 SFRSYM    DATA     BIT       TMR5CN0_TF5H
      000000C8H.3 SFRSYM    DATA     BIT       TMR5CN0_T5SPLIT
      00000088H.2 SFRSYM    DATA     BIT       TCON_IT1
      000000E8H.2 SFRSYM    DATA     BIT       ADC0CN0_ADCM2
      00000098H   SFRSYM    DATA     BYTE      SCON0
      000000E8H.3 SFRSYM    DATA     BIT       ADC0CN0_ADWINT
      000000B4H   SFRSYM    DATA     WORD      SBRL1
      000000E5H   SFRSYM    DATA     BYTE      SMOD1
      000000D2H   SFRSYM    DATA     BYTE      SCON1
      000000BAH   SFRSYM    DATA     BYTE      AMX0N
      000000E8H.4 SFRSYM    DATA     BIT       ADC0CN0_ADBUSY
LX51 LINKER/LOCATER V4.66.30.0                                                        07/27/2019  23:22:19  PAGE 103


      000000CEH   SFRSYM    DATA     BYTE      SMB0ADM
      000000C5H   SFRSYM    DATA     BYTE      ADC0LTL
      000000F8H.5 SFRSYM    DATA     BIT       SPI0CN0_MODF
      000000B8H.6 SFRSYM    DATA     BIT       IP_PSPI0
      000000CEH   SFRSYM    DATA     BYTE      SMB1ADM
      000000BBH   SFRSYM    DATA     BYTE      AMX0P
      000000C8H.6 SFRSYM    DATA     BIT       TMR5CN0_TF5L
      000000C8H   SFRSYM    DATA     BYTE      TMR2CN0
      00000091H   SFRSYM    DATA     BYTE      TMR3CN0
      00000091H   SFRSYM    DATA     BYTE      TMR4CN0
      000000C8H   SFRSYM    DATA     BYTE      TMR5CN0
      000000CFH   SFRSYM    DATA     BYTE      SMB0ADR
      00000088H.4 SFRSYM    DATA     BIT       TCON_TR0
      000000CFH   SFRSYM    DATA     BYTE      SMB1ADR
      000000C8H.4 SFRSYM    DATA     BIT       TMR2CN0_TF2CEN
      00000088H.6 SFRSYM    DATA     BIT       TCON_TR1
      000000C2H   SFRSYM    DATA     BYTE      SMB0DAT
      000000CDH   SFRSYM    DATA     BYTE      TMR2H
      000000A1H   SFRSYM    DATA     BYTE      SPI0CFG
      000000C2H   SFRSYM    DATA     BYTE      SMB1DAT
      00000095H   SFRSYM    DATA     BYTE      TMR3H
      00000095H   SFRSYM    DATA     BYTE      TMR4H
      000000CDH   SFRSYM    DATA     BYTE      TMR5H
      000000CCH   SFRSYM    DATA     BYTE      TMR2L
      000000F8H.7 SFRSYM    DATA     BIT       SPI0CN0_SPIF
      00000096H   SFRSYM    DATA     BYTE      USB0ADR
      00000094H   SFRSYM    DATA     BYTE      TMR3L
      000000A8H.7 SFRSYM    DATA     BIT       IE_EA
      00000094H   SFRSYM    DATA     BYTE      TMR4L
      00000097H   SFRSYM    DATA     BYTE      USB0DAT
      000000CCH   SFRSYM    DATA     BYTE      TMR5L
      000000B6H   SFRSYM    DATA     BYTE      FLSCL
      000000C8H.5 SFRSYM    DATA     BIT       TMR2CN0_TF2LEN
      000000F8H.6 SFRSYM    DATA     BIT       SPI0CN0_WCOL
      000000F8H.2 SFRSYM    DATA     BIT       SPI0CN0_NSSMD0
      000000D0H.7 SFRSYM    DATA     BIT       PSW_CY
      000000A3H   SFRSYM    DATA     BYTE      SPI0DAT
      000000F8H.3 SFRSYM    DATA     BIT       SPI0CN0_NSSMD1
      000000BDH   SFRSYM    DATA     WORD      ADC0
      000000B9H   SFRSYM    DATA     BYTE      SMBTC
      000000D0H   SFRSYM    DATA     BYTE      PSW
      000000C8H.5 SFRSYM    DATA     BIT       TMR5CN0_TF5LEN
      000000B7H   SFRSYM    DATA     BYTE      FLKEY
      0100515AH   SYMBOL    CODE     ---       _uconf_validate
      01004EBEH   SYMBOL    CODE     ---       uconf_defaults

      01004EBEH   BLOCK     CODE     ---       LVL=0
      01004EBEH   LINE      CODE     ---       #21
      01004EBEH   LINE      CODE     ---       #22
      01004EBEH   LINE      CODE     ---       #23
      01004EC4H   LINE      CODE     ---       #24
      01004EC9H   LINE      CODE     ---       #25
      01004ECDH   LINE      CODE     ---       #26
      01004ED1H   LINE      CODE     ---       #27
      01004ED5H   LINE      CODE     ---       #28
      01004ED9H   LINE      CODE     ---       #29
      01004EDCH   LINE      CODE     ---       #31
      01004EEBH   LINE      CODE     ---       #33
      01004EF1H   LINE      CODE     ---       #34
      01004EF5H   LINE      CODE     ---       #35
      01004EF9H   LINE      CODE     ---       #37
      01004EFCH   LINE      CODE     ---       #38
LX51 LINKER/LOCATER V4.66.30.0                                                        07/27/2019  23:22:19  PAGE 104


      01004F00H   LINE      CODE     ---       #39
      01004F04H   LINE      CODE     ---       #41
      01004F08H   LINE      CODE     ---       #43
      01004F18H   LINE      CODE     ---       #44
      ---         BLOCKEND  ---      ---       LVL=0

      0100515AH   BLOCK     CODE     ---       LVL=0
      00000028H   SYMBOL    DATA     BYTE      offset
      0100515CH   BLOCK     CODE     NEAR LAB  LVL=1
      00000007H   SYMBOL    DATA     BYTE      c
      00000029H   SYMBOL    DATA     ---       flash
      ---         BLOCKEND  ---      ---       LVL=1
      0100515AH   LINE      CODE     ---       #46
      0100515CH   LINE      CODE     ---       #47
      0100515CH   LINE      CODE     ---       #51
      01005172H   LINE      CODE     ---       #54
      0100517CH   LINE      CODE     ---       #55
      0100517EH   LINE      CODE     ---       #56
      0100517EH   LINE      CODE     ---       #59
      01005189H   LINE      CODE     ---       #60
      01005195H   LINE      CODE     ---       #61
      01005199H   LINE      CODE     ---       #62
      01005199H   LINE      CODE     ---       #64
      010051A7H   LINE      CODE     ---       #65
      ---         BLOCKEND  ---      ---       LVL=0

      01004D48H   BLOCK     CODE     ---       LVL=0
      01004D48H   BLOCK     CODE     NEAR LAB  LVL=1
      00000022H   SYMBOL    DATA     BYTE      i
      00000006H   SYMBOL    DATA     WORD      test_iter
      00000023H   SYMBOL    DATA     BYTE      valid_offset
      00000024H   SYMBOL    DATA     WORD      valid_iter
      00000026H   SYMBOL    DATA     WORD      base
      ---         BLOCKEND  ---      ---       LVL=1
      01004D48H   LINE      CODE     ---       #67
      01004D48H   LINE      CODE     ---       #68
      01004D48H   LINE      CODE     ---       #78
      01004D4BH   LINE      CODE     ---       #79
      01004D4FH   LINE      CODE     ---       #82
      01004D58H   LINE      CODE     ---       #86
      01004D5BH   LINE      CODE     ---       #87
      01004D60H   LINE      CODE     ---       #88
      01004D6DH   LINE      CODE     ---       #89
      01004D73H   LINE      CODE     ---       #90
      01004D77H   LINE      CODE     ---       #91
      01004D77H   LINE      CODE     ---       #92
      01004D80H   LINE      CODE     ---       #94
      01004D84H   LINE      CODE     ---       #95
      01004D87H   LINE      CODE     ---       #96
      01004D8BH   LINE      CODE     ---       #97
      01004DA2H   LINE      CODE     ---       #98
      01004DA2H   LINE      CODE     ---       #99
      01004DA5H   LINE      CODE     ---       #100
      01004DA5H   LINE      CODE     ---       #101
      ---         BLOCKEND  ---      ---       LVL=0

      01003D71H   BLOCK     CODE     ---       LVL=0
      01003D71H   BLOCK     CODE     NEAR LAB  LVL=1
      00000026H   SYMBOL    DATA     BYTE      offset
      00000027H   SYMBOL    DATA     WORD      base
      ---         BLOCKEND  ---      ---       LVL=1
      01003D71H   LINE      CODE     ---       #103
LX51 LINKER/LOCATER V4.66.30.0                                                        07/27/2019  23:22:19  PAGE 105


      01003D71H   LINE      CODE     ---       #104
      01003D71H   LINE      CODE     ---       #108
      01003D78H   LINE      CODE     ---       #112
      01003D7CH   LINE      CODE     ---       #113
      01003D8AH   LINE      CODE     ---       #114
      01003DA0H   LINE      CODE     ---       #115
      01003DA4H   LINE      CODE     ---       #116
      01003DA6H   LINE      CODE     ---       #117
      01003DA6H   LINE      CODE     ---       #118
      01003DAAH   LINE      CODE     ---       #120
      01003DB1H   LINE      CODE     ---       #122
      01003DB4H   LINE      CODE     ---       #123
      01003DB6H   LINE      CODE     ---       #124
      01003DB8H   LINE      CODE     ---       #125
      01003DB8H   LINE      CODE     ---       #128
      01003DC2H   LINE      CODE     ---       #129
      01003DCCH   LINE      CODE     ---       #131
      01003DCEH   LINE      CODE     ---       #132
      01003DE0H   LINE      CODE     ---       #133
      01003DE9H   LINE      CODE     ---       #135
      01003DF1H   LINE      CODE     ---       #136
      01003DF4H   LINE      CODE     ---       #137
      01003DF6H   LINE      CODE     ---       #139
      01003DFCH   LINE      CODE     ---       #140
      01003E12H   LINE      CODE     ---       #141
      01003E12H   LINE      CODE     ---       #142
      01003E12H   LINE      CODE     ---       #145
      01003E22H   LINE      CODE     ---       #146
      ---         BLOCKEND  ---      ---       LVL=0

      ---         MODULE    ---      ---       FONT_TABLE
      01004B23H   PUBLIC    CODE     ---       font_table

      ---         MODULE    ---      ---       EFM8_SPI
      00000046H   PUBLIC    DATA     BYTE      ?_spi0_xfer?BYTE
      010052D1H   PUBLIC    CODE     ---       _spi0_xfer
      01005ABFH   PUBLIC    CODE     ---       _spi0_xfer_byte
      000000A2H   SFRSYM    DATA     BYTE      SPI0CKR
      00000080H   SFRSYM    DATA     BYTE      P0
      000000D0H.2 SFRSYM    DATA     BIT       PSW_OV
      000000B1H   SFRSYM    DATA     BYTE      XOSC0CN
      00000090H   SFRSYM    DATA     BYTE      P1
      000000A0H   SFRSYM    DATA     BYTE      P2
      000000B0H   SFRSYM    DATA     BYTE      P3
      000000BCH   SFRSYM    DATA     BYTE      ADC0CF
      000000C8H   SFRSYM    DATA     BIT       TMR2CN0_T2XCLK
      000000C7H   SFRSYM    DATA     BYTE      P4
      000000C0H.7 SFRSYM    DATA     BIT       SMB0CN0_MASTER
      000000F9H   SFRSYM    DATA     WORD      PCA0
      000000E6H   SFRSYM    DATA     BYTE      EIE1
      000000C0H.7 SFRSYM    DATA     BIT       SMB1CN0_MASTER
      000000C0H.1 SFRSYM    DATA     BIT       SMB0CN0_ACK
      000000D7H   SFRSYM    DATA     BYTE      USB0XCN
      000000E7H   SFRSYM    DATA     BYTE      EIE2
      000000C0H.1 SFRSYM    DATA     BIT       SMB1CN0_ACK
      0000008FH   SFRSYM    DATA     BYTE      PSCTL
      000000E4H   SFRSYM    DATA     BYTE      IT01CF
      000000C8H   SFRSYM    DATA     BIT       TMR5CN0_T5XCLK
      000000C0H.6 SFRSYM    DATA     BIT       SMB0CN0_TXMODE
      000000C0H.6 SFRSYM    DATA     BIT       SMB1CN0_TXMODE
      000000BFH   SFRSYM    DATA     BYTE      SFRPAGE
      000000A4H   SFRSYM    DATA     BYTE      P0MDOUT
LX51 LINKER/LOCATER V4.66.30.0                                                        07/27/2019  23:22:19  PAGE 106


      000000A5H   SFRSYM    DATA     BYTE      P1MDOUT
      000000E8H.5 SFRSYM    DATA     BIT       ADC0CN0_ADINT
      000000CBH   SFRSYM    DATA     BYTE      TMR2RLH
      000000A6H   SFRSYM    DATA     BYTE      P2MDOUT
      000000A8H   SFRSYM    DATA     BYTE      IE
      00000093H   SFRSYM    DATA     BYTE      TMR3RLH
      000000A7H   SFRSYM    DATA     BYTE      P3MDOUT
      00000093H   SFRSYM    DATA     BYTE      TMR4RLH
      000000AEH   SFRSYM    DATA     BYTE      P4MDOUT
      000000F6H   SFRSYM    DATA     BYTE      EIP1
      000000CBH   SFRSYM    DATA     BYTE      TMR5RLH
      000000F7H   SFRSYM    DATA     BYTE      EIP2
      00000098H.2 SFRSYM    DATA     BIT       SCON0_RB8
      000000CAH   SFRSYM    DATA     BYTE      TMR2RLL
      000000FCH   SFRSYM    DATA     BYTE      PCA0CPH0
      00000092H   SFRSYM    DATA     BYTE      TMR3RLL
      000000EAH   SFRSYM    DATA     BYTE      PCA0CPH1
      00000098H.3 SFRSYM    DATA     BIT       SCON0_TB8
      000000F0H   SFRSYM    DATA     BIT       B_B0
      00000082H   SFRSYM    DATA     WORD      DP
      00000092H   SFRSYM    DATA     BYTE      TMR4RLL
      000000ECH   SFRSYM    DATA     BYTE      PCA0CPH2
      000000F0H.1 SFRSYM    DATA     BIT       B_B1
      000000C3H   SFRSYM    DATA     WORD      ADC0GT
      000000CAH   SFRSYM    DATA     BYTE      TMR5RLL
      000000EEH   SFRSYM    DATA     BYTE      PCA0CPH3
      000000F0H.2 SFRSYM    DATA     BIT       B_B2
      000000FBH   SFRSYM    DATA     BYTE      PCA0CPL0
      000000FEH   SFRSYM    DATA     BYTE      PCA0CPH4
      00000085H   SFRSYM    DATA     BYTE      EMI0CF
      000000F0H.3 SFRSYM    DATA     BIT       B_B3
      000000D9H   SFRSYM    DATA     BYTE      PCA0MD
      000000DAH   SFRSYM    DATA     BYTE      PCA0CPM0
      000000E9H   SFRSYM    DATA     BYTE      PCA0CPL1
      000000F0H.4 SFRSYM    DATA     BIT       B_B4
      000000DBH   SFRSYM    DATA     BYTE      PCA0CPM1
      000000EBH   SFRSYM    DATA     BYTE      PCA0CPL2
      000000F0H.5 SFRSYM    DATA     BIT       B_B5
      000000DCH   SFRSYM    DATA     BYTE      PCA0CPM2
      000000EDH   SFRSYM    DATA     BYTE      PCA0CPL3
      000000B8H   SFRSYM    DATA     BYTE      IP
      000000F0H.6 SFRSYM    DATA     BIT       B_B6
      000000C5H   SFRSYM    DATA     WORD      ADC0LT
      000000DDH   SFRSYM    DATA     BYTE      PCA0CPM3
      000000FDH   SFRSYM    DATA     BYTE      PCA0CPL4
      00000098H.5 SFRSYM    DATA     BIT       SCON0_MCE
      000000F0H.7 SFRSYM    DATA     BIT       B_B7
      000000DEH   SFRSYM    DATA     BYTE      PCA0CPM4
      000000E1H   SFRSYM    DATA     BYTE      XBR0
      000000C1H   SFRSYM    DATA     BYTE      SMB0CF
      000000E2H   SFRSYM    DATA     BYTE      XBR1
      000000C1H   SFRSYM    DATA     BYTE      SMB1CF
      000000AFH   SFRSYM    DATA     BYTE      PFE0CN
      000000AAH   SFRSYM    DATA     BYTE      EMI0CN
      000000C0H.5 SFRSYM    DATA     BIT       SMB0CN0_STA
      000000E3H   SFRSYM    DATA     BYTE      XBR2
      000000C0H.5 SFRSYM    DATA     BIT       SMB1CN0_STA
      000000E0H   SFRSYM    DATA     BIT       ACC_ACC0
      000000D1H   SFRSYM    DATA     BYTE      REF0CN
      000000B2H   SFRSYM    DATA     BYTE      HFO0CN
      0000008EH   SFRSYM    DATA     BYTE      CKCON0
      000000E0H.1 SFRSYM    DATA     BIT       ACC_ACC1
LX51 LINKER/LOCATER V4.66.30.0                                                        07/27/2019  23:22:19  PAGE 107


      000000E4H   SFRSYM    DATA     BYTE      CKCON1
      000000C8H.2 SFRSYM    DATA     BIT       TMR2CN0_TR2
      000000E0H.2 SFRSYM    DATA     BIT       ACC_ACC2
      000000E0H.3 SFRSYM    DATA     BIT       ACC_ACC3
      00000081H   SFRSYM    DATA     BYTE      SP
      0000009DH   SFRSYM    DATA     BYTE      CMP0MD
      000000E0H.4 SFRSYM    DATA     BIT       ACC_ACC4
      00000086H   SFRSYM    DATA     BYTE      LFO0CN
      00000084H   SFRSYM    DATA     BYTE      EMI0TC
      0000009CH   SFRSYM    DATA     BYTE      CMP1MD
      000000D8H   SFRSYM    DATA     BIT       PCA0CN0_CCF0
      000000E0H.5 SFRSYM    DATA     BIT       ACC_ACC5
      000000D8H.1 SFRSYM    DATA     BIT       PCA0CN0_CCF1
      000000E0H.6 SFRSYM    DATA     BIT       ACC_ACC6
      000000CCH   SFRSYM    DATA     WORD      TMR2
      000000D8H.2 SFRSYM    DATA     BIT       PCA0CN0_CCF2
      000000E0H.7 SFRSYM    DATA     BIT       ACC_ACC7
      00000094H   SFRSYM    DATA     WORD      TMR3
      000000C8H.2 SFRSYM    DATA     BIT       TMR5CN0_TR5
      000000D8H.3 SFRSYM    DATA     BIT       PCA0CN0_CCF3
      00000094H   SFRSYM    DATA     WORD      TMR4
      000000ACH   SFRSYM    DATA     BYTE      SBCON1
      000000D8H.4 SFRSYM    DATA     BIT       PCA0CN0_CCF4
      000000CCH   SFRSYM    DATA     WORD      TMR5
      000000C0H.3 SFRSYM    DATA     BIT       SMB0CN0_ACKRQ
      000000FFH   SFRSYM    DATA     BYTE      VDM0CN
      000000F1H   SFRSYM    DATA     BYTE      P0MDIN
      000000C0H.3 SFRSYM    DATA     BIT       SMB1CN0_ACKRQ
      00000098H.4 SFRSYM    DATA     BIT       SCON0_REN
      000000F2H   SFRSYM    DATA     BYTE      P1MDIN
      000000F3H   SFRSYM    DATA     BYTE      P2MDIN
      000000C0H.4 SFRSYM    DATA     BIT       SMB0CN0_STO
      000000F4H   SFRSYM    DATA     BYTE      P3MDIN
      000000C0H.4 SFRSYM    DATA     BIT       SMB1CN0_STO
      000000B5H   SFRSYM    DATA     BYTE      SBRLH1
      000000F5H   SFRSYM    DATA     BYTE      P4MDIN
      000000D0H.3 SFRSYM    DATA     BIT       PSW_RS0
      000000D8H.7 SFRSYM    DATA     BIT       PCA0CN0_CF
      000000F8H.4 SFRSYM    DATA     BIT       SPI0CN0_RXOVRN
      000000D0H.4 SFRSYM    DATA     BIT       PSW_RS1
      000000B4H   SFRSYM    DATA     BYTE      SBRLL1
      000000E8H.7 SFRSYM    DATA     BIT       ADC0CN0_ADEN
      00000089H   SFRSYM    DATA     BYTE      TMOD
      00000088H   SFRSYM    DATA     BYTE      TCON
      000000D0H   SFRSYM    DATA     BIT       PSW_PARITY
      000000A8H.4 SFRSYM    DATA     BIT       IE_ES0
      0000009FH   SFRSYM    DATA     BYTE      CMP0MX
      000000A8H.1 SFRSYM    DATA     BIT       IE_ET0
      0000009EH   SFRSYM    DATA     BYTE      CMP1MX
      000000A8H.3 SFRSYM    DATA     BIT       IE_ET1
      000000D4H   SFRSYM    DATA     BYTE      P0SKIP
      000000C8H.1 SFRSYM    DATA     BIT       TMR2CN0_T2CSS
      000000A8H.5 SFRSYM    DATA     BIT       IE_ET2
      000000D5H   SFRSYM    DATA     BYTE      P1SKIP
      000000D6H   SFRSYM    DATA     BYTE      P2SKIP
      000000E8H   SFRSYM    DATA     BYTE      ADC0CN0
      000000A8H   SFRSYM    DATA     BIT       IE_EX0
      000000DFH   SFRSYM    DATA     BYTE      P3SKIP
      000000D8H.6 SFRSYM    DATA     BIT       PCA0CN0_CR
      000000A8H.2 SFRSYM    DATA     BIT       IE_EX1
      00000098H.7 SFRSYM    DATA     BIT       SCON0_SMODE
      000000A9H   SFRSYM    DATA     BYTE      CLKSEL
LX51 LINKER/LOCATER V4.66.30.0                                                        07/27/2019  23:22:19  PAGE 108


      000000F8H   SFRSYM    DATA     BIT       SPI0CN0_SPIEN
      000000F0H   SFRSYM    DATA     BYTE      B
      000000BEH   SFRSYM    DATA     BYTE      ADC0H
      000000E8H.6 SFRSYM    DATA     BIT       ADC0CN0_ADTM
      000000CAH   SFRSYM    DATA     WORD      TMR2RL
      000000BDH   SFRSYM    DATA     BYTE      ADC0L
      00000092H   SFRSYM    DATA     WORD      TMR3RL
      00000092H   SFRSYM    DATA     WORD      TMR4RL
      000000D8H   SFRSYM    DATA     BYTE      PCA0CN0
      000000E0H   SFRSYM    DATA     BYTE      ACC
      000000CAH   SFRSYM    DATA     WORD      TMR5RL
      000000FBH   SFRSYM    DATA     WORD      PCA0CP0
      000000E9H   SFRSYM    DATA     WORD      PCA0CP1
      000000EBH   SFRSYM    DATA     WORD      PCA0CP2
      000000EDH   SFRSYM    DATA     WORD      PCA0CP3
      0000008CH   SFRSYM    DATA     BYTE      TH0
      000000B8H.4 SFRSYM    DATA     BIT       IP_PS0
      000000FDH   SFRSYM    DATA     WORD      PCA0CP4
      0000008DH   SFRSYM    DATA     BYTE      TH1
      000000FAH   SFRSYM    DATA     BYTE      PCA0H
      000000B8H.1 SFRSYM    DATA     BIT       IP_PT0
      000000B8H.3 SFRSYM    DATA     BIT       IP_PT1
      000000C0H.2 SFRSYM    DATA     BIT       SMB0CN0_ARBLOST
      000000B8H.5 SFRSYM    DATA     BIT       IP_PT2
      0000008AH   SFRSYM    DATA     BYTE      TL0
      000000F8H.1 SFRSYM    DATA     BIT       SPI0CN0_TXBMT
      000000C0H.2 SFRSYM    DATA     BIT       SMB1CN0_ARBLOST
      000000D0H.5 SFRSYM    DATA     BIT       PSW_F0
      000000A8H.6 SFRSYM    DATA     BIT       IE_ESPI0
      0000008BH   SFRSYM    DATA     BYTE      TL1
      000000F9H   SFRSYM    DATA     BYTE      PCA0L
      000000C0H   SFRSYM    DATA     BIT       SMB0CN0_SI
      000000D0H.1 SFRSYM    DATA     BIT       PSW_F1
      00000080H   SFRSYM    DATA     BIT       P0_B0
      000000B8H   SFRSYM    DATA     BIT       IP_PX0
      000000C9H   SFRSYM    DATA     BYTE      REG01CN
      000000C0H   SFRSYM    DATA     BIT       SMB1CN0_SI
      00000090H   SFRSYM    DATA     BIT       P1_B0
      00000080H.1 SFRSYM    DATA     BIT       P0_B1
      000000B8H.2 SFRSYM    DATA     BIT       IP_PX1
      0000009BH   SFRSYM    DATA     BYTE      CMP0CN0
      00000088H.1 SFRSYM    DATA     BIT       TCON_IE0
      000000A0H   SFRSYM    DATA     BIT       P2_B0
      00000090H.1 SFRSYM    DATA     BIT       P1_B1
      00000080H.2 SFRSYM    DATA     BIT       P0_B2
      0000009AH   SFRSYM    DATA     BYTE      CMP1CN0
      00000088H.3 SFRSYM    DATA     BIT       TCON_IE1
      000000B0H   SFRSYM    DATA     BIT       P3_B0
      000000A0H.1 SFRSYM    DATA     BIT       P2_B1
      00000090H.2 SFRSYM    DATA     BIT       P1_B2
      00000080H.3 SFRSYM    DATA     BIT       P0_B3
      000000C0H   SFRSYM    DATA     BYTE      SMB0CN0
      000000B0H.1 SFRSYM    DATA     BIT       P3_B1
      000000A0H.2 SFRSYM    DATA     BIT       P2_B2
      00000090H.3 SFRSYM    DATA     BIT       P1_B3
      00000080H.4 SFRSYM    DATA     BIT       P0_B4
      000000C0H   SFRSYM    DATA     BYTE      SMB1CN0
      000000B0H.2 SFRSYM    DATA     BIT       P3_B2
      000000A0H.3 SFRSYM    DATA     BIT       P2_B3
      00000090H.4 SFRSYM    DATA     BIT       P1_B4
      00000080H.5 SFRSYM    DATA     BIT       P0_B5
      000000B0H.3 SFRSYM    DATA     BIT       P3_B3
LX51 LINKER/LOCATER V4.66.30.0                                                        07/27/2019  23:22:19  PAGE 109


      000000A0H.4 SFRSYM    DATA     BIT       P2_B4
      00000090H.5 SFRSYM    DATA     BIT       P1_B5
      00000080H.6 SFRSYM    DATA     BIT       P0_B6
      000000B0H.4 SFRSYM    DATA     BIT       P3_B4
      000000A0H.5 SFRSYM    DATA     BIT       P2_B5
      00000090H.6 SFRSYM    DATA     BIT       P1_B6
      00000080H.7 SFRSYM    DATA     BIT       P0_B7
      000000B0H.5 SFRSYM    DATA     BIT       P3_B5
      000000A0H.6 SFRSYM    DATA     BIT       P2_B6
      00000090H.7 SFRSYM    DATA     BIT       P1_B7
      000000B0H.6 SFRSYM    DATA     BIT       P3_B6
      000000A0H.7 SFRSYM    DATA     BIT       P2_B7
      000000B0H.7 SFRSYM    DATA     BIT       P3_B7
      00000083H   SFRSYM    DATA     BYTE      DPH
      000000C4H   SFRSYM    DATA     BYTE      ADC0GTH
      000000C8H.7 SFRSYM    DATA     BIT       TMR2CN0_TF2H
      000000C8H.3 SFRSYM    DATA     BIT       TMR2CN0_T2SPLIT
      000000D0H.6 SFRSYM    DATA     BIT       PSW_AC
      000000F8H   SFRSYM    DATA     BYTE      SPI0CN0
      000000B3H   SFRSYM    DATA     BYTE      HFO0CAL
      00000088H.5 SFRSYM    DATA     BIT       TCON_TF0
      00000098H   SFRSYM    DATA     BIT       SCON0_RI
      00000082H   SFRSYM    DATA     BYTE      DPL
      00000088H.7 SFRSYM    DATA     BIT       TCON_TF1
      00000099H   SFRSYM    DATA     BYTE      SBUF0
      00000087H   SFRSYM    DATA     BYTE      PCON0
      000000C3H   SFRSYM    DATA     BYTE      ADC0GTL
      000000C8H.6 SFRSYM    DATA     BIT       TMR2CN0_TF2L
      00000098H.1 SFRSYM    DATA     BIT       SCON0_TI
      000000E8H   SFRSYM    DATA     BIT       ADC0CN0_ADCM0
      000000D3H   SFRSYM    DATA     BYTE      SBUF1
      000000C6H   SFRSYM    DATA     BYTE      ADC0LTH
      00000088H   SFRSYM    DATA     BIT       TCON_IT0
      000000E8H.1 SFRSYM    DATA     BIT       ADC0CN0_ADCM1
      000000EFH   SFRSYM    DATA     BYTE      RSTSRC
      000000C8H.7 SFRSYM    DATA     BIT       TMR5CN0_TF5H
      000000C8H.3 SFRSYM    DATA     BIT       TMR5CN0_T5SPLIT
      00000088H.2 SFRSYM    DATA     BIT       TCON_IT1
      000000E8H.2 SFRSYM    DATA     BIT       ADC0CN0_ADCM2
      00000098H   SFRSYM    DATA     BYTE      SCON0
      000000E8H.3 SFRSYM    DATA     BIT       ADC0CN0_ADWINT
      000000B4H   SFRSYM    DATA     WORD      SBRL1
      000000E5H   SFRSYM    DATA     BYTE      SMOD1
      000000D2H   SFRSYM    DATA     BYTE      SCON1
      000000BAH   SFRSYM    DATA     BYTE      AMX0N
      000000E8H.4 SFRSYM    DATA     BIT       ADC0CN0_ADBUSY
      000000CEH   SFRSYM    DATA     BYTE      SMB0ADM
      000000C5H   SFRSYM    DATA     BYTE      ADC0LTL
      000000F8H.5 SFRSYM    DATA     BIT       SPI0CN0_MODF
      000000B8H.6 SFRSYM    DATA     BIT       IP_PSPI0
      000000CEH   SFRSYM    DATA     BYTE      SMB1ADM
      000000BBH   SFRSYM    DATA     BYTE      AMX0P
      000000C8H.6 SFRSYM    DATA     BIT       TMR5CN0_TF5L
      000000C8H   SFRSYM    DATA     BYTE      TMR2CN0
      00000091H   SFRSYM    DATA     BYTE      TMR3CN0
      00000091H   SFRSYM    DATA     BYTE      TMR4CN0
      000000C8H   SFRSYM    DATA     BYTE      TMR5CN0
      000000CFH   SFRSYM    DATA     BYTE      SMB0ADR
      00000088H.4 SFRSYM    DATA     BIT       TCON_TR0
      000000CFH   SFRSYM    DATA     BYTE      SMB1ADR
      000000C8H.4 SFRSYM    DATA     BIT       TMR2CN0_TF2CEN
      00000088H.6 SFRSYM    DATA     BIT       TCON_TR1
LX51 LINKER/LOCATER V4.66.30.0                                                        07/27/2019  23:22:19  PAGE 110


      000000C2H   SFRSYM    DATA     BYTE      SMB0DAT
      000000CDH   SFRSYM    DATA     BYTE      TMR2H
      000000A1H   SFRSYM    DATA     BYTE      SPI0CFG
      000000C2H   SFRSYM    DATA     BYTE      SMB1DAT
      00000095H   SFRSYM    DATA     BYTE      TMR3H
      00000095H   SFRSYM    DATA     BYTE      TMR4H
      000000CDH   SFRSYM    DATA     BYTE      TMR5H
      000000CCH   SFRSYM    DATA     BYTE      TMR2L
      000000F8H.7 SFRSYM    DATA     BIT       SPI0CN0_SPIF
      00000096H   SFRSYM    DATA     BYTE      USB0ADR
      00000094H   SFRSYM    DATA     BYTE      TMR3L
      000000A8H.7 SFRSYM    DATA     BIT       IE_EA
      00000094H   SFRSYM    DATA     BYTE      TMR4L
      00000097H   SFRSYM    DATA     BYTE      USB0DAT
      000000CCH   SFRSYM    DATA     BYTE      TMR5L
      000000B6H   SFRSYM    DATA     BYTE      FLSCL
      000000C8H.5 SFRSYM    DATA     BIT       TMR2CN0_TF2LEN
      000000F8H.6 SFRSYM    DATA     BIT       SPI0CN0_WCOL
      000000F8H.2 SFRSYM    DATA     BIT       SPI0CN0_NSSMD0
      000000D0H.7 SFRSYM    DATA     BIT       PSW_CY
      000000A3H   SFRSYM    DATA     BYTE      SPI0DAT
      000000F8H.3 SFRSYM    DATA     BIT       SPI0CN0_NSSMD1
      000000BDH   SFRSYM    DATA     WORD      ADC0
      000000B9H   SFRSYM    DATA     BYTE      SMBTC
      000000D0H   SFRSYM    DATA     BYTE      PSW
      000000C8H.5 SFRSYM    DATA     BIT       TMR5CN0_TF5LEN
      000000B7H   SFRSYM    DATA     BYTE      FLKEY

      01005ABFH   BLOCK     CODE     ---       LVL=0
      00000007H   SYMBOL    DATA     BYTE      byte
      01005ABFH   LINE      CODE     ---       #12
      01005ABFH   LINE      CODE     ---       #13
      01005ABFH   LINE      CODE     ---       #14
      01005AC2H   LINE      CODE     ---       #15
      01005AC4H   LINE      CODE     ---       #16
      01005AC7H   LINE      CODE     ---       #17
      01005AC9H   LINE      CODE     ---       #19
      01005ACBH   LINE      CODE     ---       #20
      ---         BLOCKEND  ---      ---       LVL=0

      010052D1H   BLOCK     CODE     ---       LVL=0
      00000046H   SYMBOL    DATA     ---       rbuf
      00000049H   SYMBOL    DATA     ---       wbuf
      0000004CH   SYMBOL    DATA     BYTE      len
      010052D7H   BLOCK     CODE     NEAR LAB  LVL=1
      00000006H   SYMBOL    DATA     BYTE      i
      00000007H   SYMBOL    DATA     BYTE      r
      ---         BLOCKEND  ---      ---       LVL=1
      010052D1H   LINE      CODE     ---       #22
      010052D7H   LINE      CODE     ---       #23
      010052D7H   LINE      CODE     ---       #27
      010052D9H   LINE      CODE     ---       #29
      010052DBH   LINE      CODE     ---       #30
      010052E0H   LINE      CODE     ---       #31
      010052E8H   LINE      CODE     ---       #32
      010052FAH   LINE      CODE     ---       #33
      01005302H   LINE      CODE     ---       #34
      01005311H   LINE      CODE     ---       #35
      01005311H   LINE      CODE     ---       #36
      01005311H   LINE      CODE     ---       #37
      01005312H   LINE      CODE     ---       #38
      01005314H   LINE      CODE     ---       #40
LX51 LINKER/LOCATER V4.66.30.0                                                        07/27/2019  23:22:19  PAGE 111


      01005316H   LINE      CODE     ---       #41
      ---         BLOCKEND  ---      ---       LVL=0

      ---         MODULE    ---      ---       EFM8UB2_HWID
      0000005FH   PUBLIC    DATA     ---       hwid
      01004C26H   PUBLIC    CODE     ---       hwid_get_model
      01005B82H   PUBLIC    CODE     ---       hwid_init
      000000A2H   SFRSYM    DATA     BYTE      SPI0CKR
      00000080H   SFRSYM    DATA     BYTE      P0
      000000D0H.2 SFRSYM    DATA     BIT       PSW_OV
      000000B1H   SFRSYM    DATA     BYTE      XOSC0CN
      00000090H   SFRSYM    DATA     BYTE      P1
      000000A0H   SFRSYM    DATA     BYTE      P2
      000000B0H   SFRSYM    DATA     BYTE      P3
      000000BCH   SFRSYM    DATA     BYTE      ADC0CF
      000000C8H   SFRSYM    DATA     BIT       TMR2CN0_T2XCLK
      000000C7H   SFRSYM    DATA     BYTE      P4
      000000C0H.7 SFRSYM    DATA     BIT       SMB0CN0_MASTER
      000000F9H   SFRSYM    DATA     WORD      PCA0
      000000E6H   SFRSYM    DATA     BYTE      EIE1
      000000C0H.7 SFRSYM    DATA     BIT       SMB1CN0_MASTER
      000000C0H.1 SFRSYM    DATA     BIT       SMB0CN0_ACK
      000000D7H   SFRSYM    DATA     BYTE      USB0XCN
      000000E7H   SFRSYM    DATA     BYTE      EIE2
      000000C0H.1 SFRSYM    DATA     BIT       SMB1CN0_ACK
      0000008FH   SFRSYM    DATA     BYTE      PSCTL
      000000E4H   SFRSYM    DATA     BYTE      IT01CF
      000000C8H   SFRSYM    DATA     BIT       TMR5CN0_T5XCLK
      000000C0H.6 SFRSYM    DATA     BIT       SMB0CN0_TXMODE
      000000C0H.6 SFRSYM    DATA     BIT       SMB1CN0_TXMODE
      000000BFH   SFRSYM    DATA     BYTE      SFRPAGE
      000000A4H   SFRSYM    DATA     BYTE      P0MDOUT
      000000A5H   SFRSYM    DATA     BYTE      P1MDOUT
      000000E8H.5 SFRSYM    DATA     BIT       ADC0CN0_ADINT
      000000CBH   SFRSYM    DATA     BYTE      TMR2RLH
      000000A6H   SFRSYM    DATA     BYTE      P2MDOUT
      000000A8H   SFRSYM    DATA     BYTE      IE
      00000093H   SFRSYM    DATA     BYTE      TMR3RLH
      000000A7H   SFRSYM    DATA     BYTE      P3MDOUT
      00000093H   SFRSYM    DATA     BYTE      TMR4RLH
      000000AEH   SFRSYM    DATA     BYTE      P4MDOUT
      000000F6H   SFRSYM    DATA     BYTE      EIP1
      000000CBH   SFRSYM    DATA     BYTE      TMR5RLH
      000000F7H   SFRSYM    DATA     BYTE      EIP2
      00000098H.2 SFRSYM    DATA     BIT       SCON0_RB8
      000000CAH   SFRSYM    DATA     BYTE      TMR2RLL
      000000FCH   SFRSYM    DATA     BYTE      PCA0CPH0
      00000092H   SFRSYM    DATA     BYTE      TMR3RLL
      000000EAH   SFRSYM    DATA     BYTE      PCA0CPH1
      00000098H.3 SFRSYM    DATA     BIT       SCON0_TB8
      000000F0H   SFRSYM    DATA     BIT       B_B0
      00000082H   SFRSYM    DATA     WORD      DP
      00000092H   SFRSYM    DATA     BYTE      TMR4RLL
      000000ECH   SFRSYM    DATA     BYTE      PCA0CPH2
      000000F0H.1 SFRSYM    DATA     BIT       B_B1
      000000C3H   SFRSYM    DATA     WORD      ADC0GT
      000000CAH   SFRSYM    DATA     BYTE      TMR5RLL
      000000EEH   SFRSYM    DATA     BYTE      PCA0CPH3
      000000F0H.2 SFRSYM    DATA     BIT       B_B2
      000000FBH   SFRSYM    DATA     BYTE      PCA0CPL0
      000000FEH   SFRSYM    DATA     BYTE      PCA0CPH4
      00000085H   SFRSYM    DATA     BYTE      EMI0CF
LX51 LINKER/LOCATER V4.66.30.0                                                        07/27/2019  23:22:19  PAGE 112


      000000F0H.3 SFRSYM    DATA     BIT       B_B3
      000000D9H   SFRSYM    DATA     BYTE      PCA0MD
      000000DAH   SFRSYM    DATA     BYTE      PCA0CPM0
      000000E9H   SFRSYM    DATA     BYTE      PCA0CPL1
      000000F0H.4 SFRSYM    DATA     BIT       B_B4
      000000DBH   SFRSYM    DATA     BYTE      PCA0CPM1
      000000EBH   SFRSYM    DATA     BYTE      PCA0CPL2
      000000F0H.5 SFRSYM    DATA     BIT       B_B5
      000000DCH   SFRSYM    DATA     BYTE      PCA0CPM2
      000000EDH   SFRSYM    DATA     BYTE      PCA0CPL3
      000000B8H   SFRSYM    DATA     BYTE      IP
      000000F0H.6 SFRSYM    DATA     BIT       B_B6
      000000C5H   SFRSYM    DATA     WORD      ADC0LT
      000000DDH   SFRSYM    DATA     BYTE      PCA0CPM3
      000000FDH   SFRSYM    DATA     BYTE      PCA0CPL4
      00000098H.5 SFRSYM    DATA     BIT       SCON0_MCE
      000000F0H.7 SFRSYM    DATA     BIT       B_B7
      000000DEH   SFRSYM    DATA     BYTE      PCA0CPM4
      000000E1H   SFRSYM    DATA     BYTE      XBR0
      000000C1H   SFRSYM    DATA     BYTE      SMB0CF
      000000E2H   SFRSYM    DATA     BYTE      XBR1
      000000C1H   SFRSYM    DATA     BYTE      SMB1CF
      000000AFH   SFRSYM    DATA     BYTE      PFE0CN
      000000AAH   SFRSYM    DATA     BYTE      EMI0CN
      000000C0H.5 SFRSYM    DATA     BIT       SMB0CN0_STA
      000000E3H   SFRSYM    DATA     BYTE      XBR2
      000000C0H.5 SFRSYM    DATA     BIT       SMB1CN0_STA
      000000E0H   SFRSYM    DATA     BIT       ACC_ACC0
      000000D1H   SFRSYM    DATA     BYTE      REF0CN
      000000B2H   SFRSYM    DATA     BYTE      HFO0CN
      0000008EH   SFRSYM    DATA     BYTE      CKCON0
      000000E0H.1 SFRSYM    DATA     BIT       ACC_ACC1
      000000E4H   SFRSYM    DATA     BYTE      CKCON1
      000000C8H.2 SFRSYM    DATA     BIT       TMR2CN0_TR2
      000000E0H.2 SFRSYM    DATA     BIT       ACC_ACC2
      000000E0H.3 SFRSYM    DATA     BIT       ACC_ACC3
      00000081H   SFRSYM    DATA     BYTE      SP
      0000009DH   SFRSYM    DATA     BYTE      CMP0MD
      000000E0H.4 SFRSYM    DATA     BIT       ACC_ACC4
      00000086H   SFRSYM    DATA     BYTE      LFO0CN
      00000084H   SFRSYM    DATA     BYTE      EMI0TC
      0000009CH   SFRSYM    DATA     BYTE      CMP1MD
      000000D8H   SFRSYM    DATA     BIT       PCA0CN0_CCF0
      000000E0H.5 SFRSYM    DATA     BIT       ACC_ACC5
      000000D8H.1 SFRSYM    DATA     BIT       PCA0CN0_CCF1
      000000E0H.6 SFRSYM    DATA     BIT       ACC_ACC6
      000000CCH   SFRSYM    DATA     WORD      TMR2
      000000D8H.2 SFRSYM    DATA     BIT       PCA0CN0_CCF2
      000000E0H.7 SFRSYM    DATA     BIT       ACC_ACC7
      00000094H   SFRSYM    DATA     WORD      TMR3
      000000C8H.2 SFRSYM    DATA     BIT       TMR5CN0_TR5
      000000D8H.3 SFRSYM    DATA     BIT       PCA0CN0_CCF3
      00000094H   SFRSYM    DATA     WORD      TMR4
      000000ACH   SFRSYM    DATA     BYTE      SBCON1
      000000D8H.4 SFRSYM    DATA     BIT       PCA0CN0_CCF4
      000000CCH   SFRSYM    DATA     WORD      TMR5
      000000C0H.3 SFRSYM    DATA     BIT       SMB0CN0_ACKRQ
      000000FFH   SFRSYM    DATA     BYTE      VDM0CN
      000000F1H   SFRSYM    DATA     BYTE      P0MDIN
      000000C0H.3 SFRSYM    DATA     BIT       SMB1CN0_ACKRQ
      00000098H.4 SFRSYM    DATA     BIT       SCON0_REN
      000000F2H   SFRSYM    DATA     BYTE      P1MDIN
LX51 LINKER/LOCATER V4.66.30.0                                                        07/27/2019  23:22:19  PAGE 113


      000000F3H   SFRSYM    DATA     BYTE      P2MDIN
      000000C0H.4 SFRSYM    DATA     BIT       SMB0CN0_STO
      000000F4H   SFRSYM    DATA     BYTE      P3MDIN
      000000C0H.4 SFRSYM    DATA     BIT       SMB1CN0_STO
      000000B5H   SFRSYM    DATA     BYTE      SBRLH1
      000000F5H   SFRSYM    DATA     BYTE      P4MDIN
      000000D0H.3 SFRSYM    DATA     BIT       PSW_RS0
      000000D8H.7 SFRSYM    DATA     BIT       PCA0CN0_CF
      000000F8H.4 SFRSYM    DATA     BIT       SPI0CN0_RXOVRN
      000000D0H.4 SFRSYM    DATA     BIT       PSW_RS1
      000000B4H   SFRSYM    DATA     BYTE      SBRLL1
      000000E8H.7 SFRSYM    DATA     BIT       ADC0CN0_ADEN
      00000089H   SFRSYM    DATA     BYTE      TMOD
      00000088H   SFRSYM    DATA     BYTE      TCON
      000000D0H   SFRSYM    DATA     BIT       PSW_PARITY
      000000A8H.4 SFRSYM    DATA     BIT       IE_ES0
      0000009FH   SFRSYM    DATA     BYTE      CMP0MX
      000000A8H.1 SFRSYM    DATA     BIT       IE_ET0
      0000009EH   SFRSYM    DATA     BYTE      CMP1MX
      000000A8H.3 SFRSYM    DATA     BIT       IE_ET1
      000000D4H   SFRSYM    DATA     BYTE      P0SKIP
      000000C8H.1 SFRSYM    DATA     BIT       TMR2CN0_T2CSS
      000000A8H.5 SFRSYM    DATA     BIT       IE_ET2
      000000D5H   SFRSYM    DATA     BYTE      P1SKIP
      000000D6H   SFRSYM    DATA     BYTE      P2SKIP
      000000E8H   SFRSYM    DATA     BYTE      ADC0CN0
      000000A8H   SFRSYM    DATA     BIT       IE_EX0
      000000DFH   SFRSYM    DATA     BYTE      P3SKIP
      000000D8H.6 SFRSYM    DATA     BIT       PCA0CN0_CR
      000000A8H.2 SFRSYM    DATA     BIT       IE_EX1
      00000098H.7 SFRSYM    DATA     BIT       SCON0_SMODE
      000000A9H   SFRSYM    DATA     BYTE      CLKSEL
      000000F8H   SFRSYM    DATA     BIT       SPI0CN0_SPIEN
      000000F0H   SFRSYM    DATA     BYTE      B
      000000BEH   SFRSYM    DATA     BYTE      ADC0H
      000000E8H.6 SFRSYM    DATA     BIT       ADC0CN0_ADTM
      000000CAH   SFRSYM    DATA     WORD      TMR2RL
      000000BDH   SFRSYM    DATA     BYTE      ADC0L
      00000092H   SFRSYM    DATA     WORD      TMR3RL
      00000092H   SFRSYM    DATA     WORD      TMR4RL
      000000D8H   SFRSYM    DATA     BYTE      PCA0CN0
      000000E0H   SFRSYM    DATA     BYTE      ACC
      000000CAH   SFRSYM    DATA     WORD      TMR5RL
      000000FBH   SFRSYM    DATA     WORD      PCA0CP0
      000000E9H   SFRSYM    DATA     WORD      PCA0CP1
      000000EBH   SFRSYM    DATA     WORD      PCA0CP2
      000000EDH   SFRSYM    DATA     WORD      PCA0CP3
      0000008CH   SFRSYM    DATA     BYTE      TH0
      000000B8H.4 SFRSYM    DATA     BIT       IP_PS0
      000000FDH   SFRSYM    DATA     WORD      PCA0CP4
      0000008DH   SFRSYM    DATA     BYTE      TH1
      000000FAH   SFRSYM    DATA     BYTE      PCA0H
      000000B8H.1 SFRSYM    DATA     BIT       IP_PT0
      000000B8H.3 SFRSYM    DATA     BIT       IP_PT1
      000000C0H.2 SFRSYM    DATA     BIT       SMB0CN0_ARBLOST
      000000B8H.5 SFRSYM    DATA     BIT       IP_PT2
      0000008AH   SFRSYM    DATA     BYTE      TL0
      000000F8H.1 SFRSYM    DATA     BIT       SPI0CN0_TXBMT
      000000C0H.2 SFRSYM    DATA     BIT       SMB1CN0_ARBLOST
      000000D0H.5 SFRSYM    DATA     BIT       PSW_F0
      000000A8H.6 SFRSYM    DATA     BIT       IE_ESPI0
      0000008BH   SFRSYM    DATA     BYTE      TL1
LX51 LINKER/LOCATER V4.66.30.0                                                        07/27/2019  23:22:19  PAGE 114


      000000F9H   SFRSYM    DATA     BYTE      PCA0L
      000000C0H   SFRSYM    DATA     BIT       SMB0CN0_SI
      000000D0H.1 SFRSYM    DATA     BIT       PSW_F1
      00000080H   SFRSYM    DATA     BIT       P0_B0
      000000B8H   SFRSYM    DATA     BIT       IP_PX0
      000000C9H   SFRSYM    DATA     BYTE      REG01CN
      000000C0H   SFRSYM    DATA     BIT       SMB1CN0_SI
      00000090H   SFRSYM    DATA     BIT       P1_B0
      00000080H.1 SFRSYM    DATA     BIT       P0_B1
      000000B8H.2 SFRSYM    DATA     BIT       IP_PX1
      0000009BH   SFRSYM    DATA     BYTE      CMP0CN0
      00000088H.1 SFRSYM    DATA     BIT       TCON_IE0
      000000A0H   SFRSYM    DATA     BIT       P2_B0
      00000090H.1 SFRSYM    DATA     BIT       P1_B1
      00000080H.2 SFRSYM    DATA     BIT       P0_B2
      0000009AH   SFRSYM    DATA     BYTE      CMP1CN0
      00000088H.3 SFRSYM    DATA     BIT       TCON_IE1
      000000B0H   SFRSYM    DATA     BIT       P3_B0
      000000A0H.1 SFRSYM    DATA     BIT       P2_B1
      00000090H.2 SFRSYM    DATA     BIT       P1_B2
      00000080H.3 SFRSYM    DATA     BIT       P0_B3
      000000C0H   SFRSYM    DATA     BYTE      SMB0CN0
      000000B0H.1 SFRSYM    DATA     BIT       P3_B1
      000000A0H.2 SFRSYM    DATA     BIT       P2_B2
      00000090H.3 SFRSYM    DATA     BIT       P1_B3
      00000080H.4 SFRSYM    DATA     BIT       P0_B4
      000000C0H   SFRSYM    DATA     BYTE      SMB1CN0
      000000B0H.2 SFRSYM    DATA     BIT       P3_B2
      000000A0H.3 SFRSYM    DATA     BIT       P2_B3
      00000090H.4 SFRSYM    DATA     BIT       P1_B4
      00000080H.5 SFRSYM    DATA     BIT       P0_B5
      000000B0H.3 SFRSYM    DATA     BIT       P3_B3
      000000A0H.4 SFRSYM    DATA     BIT       P2_B4
      00000090H.5 SFRSYM    DATA     BIT       P1_B5
      00000080H.6 SFRSYM    DATA     BIT       P0_B6
      000000B0H.4 SFRSYM    DATA     BIT       P3_B4
      000000A0H.5 SFRSYM    DATA     BIT       P2_B5
      00000090H.6 SFRSYM    DATA     BIT       P1_B6
      00000080H.7 SFRSYM    DATA     BIT       P0_B7
      000000B0H.5 SFRSYM    DATA     BIT       P3_B5
      000000A0H.6 SFRSYM    DATA     BIT       P2_B6
      00000090H.7 SFRSYM    DATA     BIT       P1_B7
      000000B0H.6 SFRSYM    DATA     BIT       P3_B6
      000000A0H.7 SFRSYM    DATA     BIT       P2_B7
      000000B0H.7 SFRSYM    DATA     BIT       P3_B7
      00000083H   SFRSYM    DATA     BYTE      DPH
      000000C4H   SFRSYM    DATA     BYTE      ADC0GTH
      000000C8H.7 SFRSYM    DATA     BIT       TMR2CN0_TF2H
      000000C8H.3 SFRSYM    DATA     BIT       TMR2CN0_T2SPLIT
      000000D0H.6 SFRSYM    DATA     BIT       PSW_AC
      000000F8H   SFRSYM    DATA     BYTE      SPI0CN0
      000000B3H   SFRSYM    DATA     BYTE      HFO0CAL
      00000088H.5 SFRSYM    DATA     BIT       TCON_TF0
      00000098H   SFRSYM    DATA     BIT       SCON0_RI
      00000082H   SFRSYM    DATA     BYTE      DPL
      00000088H.7 SFRSYM    DATA     BIT       TCON_TF1
      00000099H   SFRSYM    DATA     BYTE      SBUF0
      00000087H   SFRSYM    DATA     BYTE      PCON0
      000000C3H   SFRSYM    DATA     BYTE      ADC0GTL
      000000C8H.6 SFRSYM    DATA     BIT       TMR2CN0_TF2L
      00000098H.1 SFRSYM    DATA     BIT       SCON0_TI
      000000E8H   SFRSYM    DATA     BIT       ADC0CN0_ADCM0
LX51 LINKER/LOCATER V4.66.30.0                                                        07/27/2019  23:22:19  PAGE 115


      000000D3H   SFRSYM    DATA     BYTE      SBUF1
      000000C6H   SFRSYM    DATA     BYTE      ADC0LTH
      00000088H   SFRSYM    DATA     BIT       TCON_IT0
      000000E8H.1 SFRSYM    DATA     BIT       ADC0CN0_ADCM1
      000000EFH   SFRSYM    DATA     BYTE      RSTSRC
      000000C8H.7 SFRSYM    DATA     BIT       TMR5CN0_TF5H
      000000C8H.3 SFRSYM    DATA     BIT       TMR5CN0_T5SPLIT
      00000088H.2 SFRSYM    DATA     BIT       TCON_IT1
      000000E8H.2 SFRSYM    DATA     BIT       ADC0CN0_ADCM2
      00000098H   SFRSYM    DATA     BYTE      SCON0
      000000E8H.3 SFRSYM    DATA     BIT       ADC0CN0_ADWINT
      000000B4H   SFRSYM    DATA     WORD      SBRL1
      000000E5H   SFRSYM    DATA     BYTE      SMOD1
      000000D2H   SFRSYM    DATA     BYTE      SCON1
      000000BAH   SFRSYM    DATA     BYTE      AMX0N
      000000E8H.4 SFRSYM    DATA     BIT       ADC0CN0_ADBUSY
      000000CEH   SFRSYM    DATA     BYTE      SMB0ADM
      000000C5H   SFRSYM    DATA     BYTE      ADC0LTL
      000000F8H.5 SFRSYM    DATA     BIT       SPI0CN0_MODF
      000000B8H.6 SFRSYM    DATA     BIT       IP_PSPI0
      000000CEH   SFRSYM    DATA     BYTE      SMB1ADM
      000000BBH   SFRSYM    DATA     BYTE      AMX0P
      000000C8H.6 SFRSYM    DATA     BIT       TMR5CN0_TF5L
      000000C8H   SFRSYM    DATA     BYTE      TMR2CN0
      00000091H   SFRSYM    DATA     BYTE      TMR3CN0
      00000091H   SFRSYM    DATA     BYTE      TMR4CN0
      000000C8H   SFRSYM    DATA     BYTE      TMR5CN0
      000000CFH   SFRSYM    DATA     BYTE      SMB0ADR
      00000088H.4 SFRSYM    DATA     BIT       TCON_TR0
      000000CFH   SFRSYM    DATA     BYTE      SMB1ADR
      000000C8H.4 SFRSYM    DATA     BIT       TMR2CN0_TF2CEN
      00000088H.6 SFRSYM    DATA     BIT       TCON_TR1
      000000C2H   SFRSYM    DATA     BYTE      SMB0DAT
      000000CDH   SFRSYM    DATA     BYTE      TMR2H
      000000A1H   SFRSYM    DATA     BYTE      SPI0CFG
      000000C2H   SFRSYM    DATA     BYTE      SMB1DAT
      00000095H   SFRSYM    DATA     BYTE      TMR3H
      00000095H   SFRSYM    DATA     BYTE      TMR4H
      000000CDH   SFRSYM    DATA     BYTE      TMR5H
      000000CCH   SFRSYM    DATA     BYTE      TMR2L
      000000F8H.7 SFRSYM    DATA     BIT       SPI0CN0_SPIF
      00000096H   SFRSYM    DATA     BYTE      USB0ADR
      00000094H   SFRSYM    DATA     BYTE      TMR3L
      000000A8H.7 SFRSYM    DATA     BIT       IE_EA
      00000094H   SFRSYM    DATA     BYTE      TMR4L
      00000097H   SFRSYM    DATA     BYTE      USB0DAT
      000000CCH   SFRSYM    DATA     BYTE      TMR5L
      000000B6H   SFRSYM    DATA     BYTE      FLSCL
      000000C8H.5 SFRSYM    DATA     BIT       TMR2CN0_TF2LEN
      000000F8H.6 SFRSYM    DATA     BIT       SPI0CN0_WCOL
      000000F8H.2 SFRSYM    DATA     BIT       SPI0CN0_NSSMD0
      000000D0H.7 SFRSYM    DATA     BIT       PSW_CY
      000000A3H   SFRSYM    DATA     BYTE      SPI0DAT
      000000F8H.3 SFRSYM    DATA     BIT       SPI0CN0_NSSMD1
      000000BDH   SFRSYM    DATA     WORD      ADC0
      000000B9H   SFRSYM    DATA     BYTE      SMBTC
      000000D0H   SFRSYM    DATA     BYTE      PSW
      000000C8H.5 SFRSYM    DATA     BIT       TMR5CN0_TF5LEN
      000000B7H   SFRSYM    DATA     BYTE      FLKEY

      01005B82H   BLOCK     CODE     ---       LVL=0
      01005B82H   LINE      CODE     ---       #12
LX51 LINKER/LOCATER V4.66.30.0                                                        07/27/2019  23:22:19  PAGE 116


      01005B82H   LINE      CODE     ---       #13
      01005B82H   LINE      CODE     ---       #14
      01005B88H   LINE      CODE     ---       #15
      ---         BLOCKEND  ---      ---       LVL=0

      01004C26H   BLOCK     CODE     ---       LVL=0
      01004C26H   BLOCK     CODE     NEAR LAB  LVL=1
      00000029H   SYMBOL    DATA     ---       a
      00000006H   SYMBOL    DATA     WORD      s1
      00000004H   SYMBOL    DATA     WORD      s2
      ---         BLOCKEND  ---      ---       LVL=1
      01004C26H   LINE      CODE     ---       #25
      01004C26H   LINE      CODE     ---       #26
      01004C26H   LINE      CODE     ---       #28
      01004C29H   LINE      CODE     ---       #29
      01004C2BH   LINE      CODE     ---       #31
      01004C31H   LINE      CODE     ---       #32
      01004C3CH   LINE      CODE     ---       #33
      01004C50H   LINE      CODE     ---       #34
      01004C52H   LINE      CODE     ---       #36
      01004C58H   LINE      CODE     ---       #37
      01004C63H   LINE      CODE     ---       #38
      01004C77H   LINE      CODE     ---       #39
      01004C79H   LINE      CODE     ---       #41
      01004C81H   LINE      CODE     ---       #42
      01004C84H   LINE      CODE     ---       #43
      01004C84H   LINE      CODE     ---       #45
      01004C86H   LINE      CODE     ---       #46
      ---         BLOCKEND  ---      ---       LVL=0
      00000007H   SYMBOL    DATA     BYTE      byte

      ---         MODULE    ---      ---       EFM8UB2_USERFLASH
      00000061H   PUBLIC    DATA     WORD      ee_baseaddr
      01005616H   PUBLIC    CODE     ---       _userflash_write
      01005B6CH   PUBLIC    CODE     ---       _userflash_erase_page
      01005808H   PUBLIC    CODE     ---       _userflash_write_byte
      010056FCH   PUBLIC    CODE     ---       _userflash_read
      010058A1H   PUBLIC    CODE     ---       _userflash_reserve_pages
      01005B95H   PUBLIC    CODE     ---       userflash_get_baseaddr
      01005A49H   PUBLIC    CODE     ---       userflash_init
      000000A2H   SFRSYM    DATA     BYTE      SPI0CKR
      00000080H   SFRSYM    DATA     BYTE      P0
      000000D0H.2 SFRSYM    DATA     BIT       PSW_OV
      000000B1H   SFRSYM    DATA     BYTE      XOSC0CN
      00000090H   SFRSYM    DATA     BYTE      P1
      000000A0H   SFRSYM    DATA     BYTE      P2
      000000B0H   SFRSYM    DATA     BYTE      P3
      000000BCH   SFRSYM    DATA     BYTE      ADC0CF
      000000C8H   SFRSYM    DATA     BIT       TMR2CN0_T2XCLK
      000000C7H   SFRSYM    DATA     BYTE      P4
      000000C0H.7 SFRSYM    DATA     BIT       SMB0CN0_MASTER
      000000F9H   SFRSYM    DATA     WORD      PCA0
      000000E6H   SFRSYM    DATA     BYTE      EIE1
      000000C0H.7 SFRSYM    DATA     BIT       SMB1CN0_MASTER
      000000C0H.1 SFRSYM    DATA     BIT       SMB0CN0_ACK
      000000D7H   SFRSYM    DATA     BYTE      USB0XCN
      000000E7H   SFRSYM    DATA     BYTE      EIE2
      000000C0H.1 SFRSYM    DATA     BIT       SMB1CN0_ACK
      0000008FH   SFRSYM    DATA     BYTE      PSCTL
      000000E4H   SFRSYM    DATA     BYTE      IT01CF
      000000C8H   SFRSYM    DATA     BIT       TMR5CN0_T5XCLK
      000000C0H.6 SFRSYM    DATA     BIT       SMB0CN0_TXMODE
LX51 LINKER/LOCATER V4.66.30.0                                                        07/27/2019  23:22:19  PAGE 117


      000000C0H.6 SFRSYM    DATA     BIT       SMB1CN0_TXMODE
      000000BFH   SFRSYM    DATA     BYTE      SFRPAGE
      000000A4H   SFRSYM    DATA     BYTE      P0MDOUT
      000000A5H   SFRSYM    DATA     BYTE      P1MDOUT
      000000E8H.5 SFRSYM    DATA     BIT       ADC0CN0_ADINT
      000000CBH   SFRSYM    DATA     BYTE      TMR2RLH
      000000A6H   SFRSYM    DATA     BYTE      P2MDOUT
      000000A8H   SFRSYM    DATA     BYTE      IE
      00000093H   SFRSYM    DATA     BYTE      TMR3RLH
      000000A7H   SFRSYM    DATA     BYTE      P3MDOUT
      00000093H   SFRSYM    DATA     BYTE      TMR4RLH
      000000AEH   SFRSYM    DATA     BYTE      P4MDOUT
      000000F6H   SFRSYM    DATA     BYTE      EIP1
      000000CBH   SFRSYM    DATA     BYTE      TMR5RLH
      000000F7H   SFRSYM    DATA     BYTE      EIP2
      00000098H.2 SFRSYM    DATA     BIT       SCON0_RB8
      000000CAH   SFRSYM    DATA     BYTE      TMR2RLL
      000000FCH   SFRSYM    DATA     BYTE      PCA0CPH0
      00000092H   SFRSYM    DATA     BYTE      TMR3RLL
      000000EAH   SFRSYM    DATA     BYTE      PCA0CPH1
      00000098H.3 SFRSYM    DATA     BIT       SCON0_TB8
      000000F0H   SFRSYM    DATA     BIT       B_B0
      00000082H   SFRSYM    DATA     WORD      DP
      00000092H   SFRSYM    DATA     BYTE      TMR4RLL
      000000ECH   SFRSYM    DATA     BYTE      PCA0CPH2
      000000F0H.1 SFRSYM    DATA     BIT       B_B1
      000000C3H   SFRSYM    DATA     WORD      ADC0GT
      000000CAH   SFRSYM    DATA     BYTE      TMR5RLL
      000000EEH   SFRSYM    DATA     BYTE      PCA0CPH3
      000000F0H.2 SFRSYM    DATA     BIT       B_B2
      000000FBH   SFRSYM    DATA     BYTE      PCA0CPL0
      000000FEH   SFRSYM    DATA     BYTE      PCA0CPH4
      00000085H   SFRSYM    DATA     BYTE      EMI0CF
      000000F0H.3 SFRSYM    DATA     BIT       B_B3
      000000D9H   SFRSYM    DATA     BYTE      PCA0MD
      000000DAH   SFRSYM    DATA     BYTE      PCA0CPM0
      000000E9H   SFRSYM    DATA     BYTE      PCA0CPL1
      000000F0H.4 SFRSYM    DATA     BIT       B_B4
      000000DBH   SFRSYM    DATA     BYTE      PCA0CPM1
      000000EBH   SFRSYM    DATA     BYTE      PCA0CPL2
      000000F0H.5 SFRSYM    DATA     BIT       B_B5
      000000DCH   SFRSYM    DATA     BYTE      PCA0CPM2
      000000EDH   SFRSYM    DATA     BYTE      PCA0CPL3
      000000B8H   SFRSYM    DATA     BYTE      IP
      000000F0H.6 SFRSYM    DATA     BIT       B_B6
      000000C5H   SFRSYM    DATA     WORD      ADC0LT
      000000DDH   SFRSYM    DATA     BYTE      PCA0CPM3
      000000FDH   SFRSYM    DATA     BYTE      PCA0CPL4
      00000098H.5 SFRSYM    DATA     BIT       SCON0_MCE
      000000F0H.7 SFRSYM    DATA     BIT       B_B7
      000000DEH   SFRSYM    DATA     BYTE      PCA0CPM4
      000000E1H   SFRSYM    DATA     BYTE      XBR0
      000000C1H   SFRSYM    DATA     BYTE      SMB0CF
      000000E2H   SFRSYM    DATA     BYTE      XBR1
      000000C1H   SFRSYM    DATA     BYTE      SMB1CF
      000000AFH   SFRSYM    DATA     BYTE      PFE0CN
      000000AAH   SFRSYM    DATA     BYTE      EMI0CN
      000000C0H.5 SFRSYM    DATA     BIT       SMB0CN0_STA
      000000E3H   SFRSYM    DATA     BYTE      XBR2
      000000C0H.5 SFRSYM    DATA     BIT       SMB1CN0_STA
      000000E0H   SFRSYM    DATA     BIT       ACC_ACC0
      000000D1H   SFRSYM    DATA     BYTE      REF0CN
LX51 LINKER/LOCATER V4.66.30.0                                                        07/27/2019  23:22:19  PAGE 118


      000000B2H   SFRSYM    DATA     BYTE      HFO0CN
      0000008EH   SFRSYM    DATA     BYTE      CKCON0
      000000E0H.1 SFRSYM    DATA     BIT       ACC_ACC1
      000000E4H   SFRSYM    DATA     BYTE      CKCON1
      000000C8H.2 SFRSYM    DATA     BIT       TMR2CN0_TR2
      000000E0H.2 SFRSYM    DATA     BIT       ACC_ACC2
      000000E0H.3 SFRSYM    DATA     BIT       ACC_ACC3
      00000081H   SFRSYM    DATA     BYTE      SP
      0000009DH   SFRSYM    DATA     BYTE      CMP0MD
      000000E0H.4 SFRSYM    DATA     BIT       ACC_ACC4
      00000086H   SFRSYM    DATA     BYTE      LFO0CN
      00000084H   SFRSYM    DATA     BYTE      EMI0TC
      0000009CH   SFRSYM    DATA     BYTE      CMP1MD
      000000D8H   SFRSYM    DATA     BIT       PCA0CN0_CCF0
      000000E0H.5 SFRSYM    DATA     BIT       ACC_ACC5
      000000D8H.1 SFRSYM    DATA     BIT       PCA0CN0_CCF1
      000000E0H.6 SFRSYM    DATA     BIT       ACC_ACC6
      000000CCH   SFRSYM    DATA     WORD      TMR2
      000000D8H.2 SFRSYM    DATA     BIT       PCA0CN0_CCF2
      000000E0H.7 SFRSYM    DATA     BIT       ACC_ACC7
      00000094H   SFRSYM    DATA     WORD      TMR3
      000000C8H.2 SFRSYM    DATA     BIT       TMR5CN0_TR5
      000000D8H.3 SFRSYM    DATA     BIT       PCA0CN0_CCF3
      00000094H   SFRSYM    DATA     WORD      TMR4
      000000ACH   SFRSYM    DATA     BYTE      SBCON1
      000000D8H.4 SFRSYM    DATA     BIT       PCA0CN0_CCF4
      000000CCH   SFRSYM    DATA     WORD      TMR5
      000000C0H.3 SFRSYM    DATA     BIT       SMB0CN0_ACKRQ
      000000FFH   SFRSYM    DATA     BYTE      VDM0CN
      000000F1H   SFRSYM    DATA     BYTE      P0MDIN
      000000C0H.3 SFRSYM    DATA     BIT       SMB1CN0_ACKRQ
      00000098H.4 SFRSYM    DATA     BIT       SCON0_REN
      000000F2H   SFRSYM    DATA     BYTE      P1MDIN
      000000F3H   SFRSYM    DATA     BYTE      P2MDIN
      000000C0H.4 SFRSYM    DATA     BIT       SMB0CN0_STO
      000000F4H   SFRSYM    DATA     BYTE      P3MDIN
      000000C0H.4 SFRSYM    DATA     BIT       SMB1CN0_STO
      000000B5H   SFRSYM    DATA     BYTE      SBRLH1
      000000F5H   SFRSYM    DATA     BYTE      P4MDIN
      000000D0H.3 SFRSYM    DATA     BIT       PSW_RS0
      000000D8H.7 SFRSYM    DATA     BIT       PCA0CN0_CF
      000000F8H.4 SFRSYM    DATA     BIT       SPI0CN0_RXOVRN
      000000D0H.4 SFRSYM    DATA     BIT       PSW_RS1
      000000B4H   SFRSYM    DATA     BYTE      SBRLL1
      000000E8H.7 SFRSYM    DATA     BIT       ADC0CN0_ADEN
      00000089H   SFRSYM    DATA     BYTE      TMOD
      00000088H   SFRSYM    DATA     BYTE      TCON
      000000D0H   SFRSYM    DATA     BIT       PSW_PARITY
      000000A8H.4 SFRSYM    DATA     BIT       IE_ES0
      0000009FH   SFRSYM    DATA     BYTE      CMP0MX
      000000A8H.1 SFRSYM    DATA     BIT       IE_ET0
      0000009EH   SFRSYM    DATA     BYTE      CMP1MX
      000000A8H.3 SFRSYM    DATA     BIT       IE_ET1
      000000D4H   SFRSYM    DATA     BYTE      P0SKIP
      000000C8H.1 SFRSYM    DATA     BIT       TMR2CN0_T2CSS
      000000A8H.5 SFRSYM    DATA     BIT       IE_ET2
      000000D5H   SFRSYM    DATA     BYTE      P1SKIP
      000000D6H   SFRSYM    DATA     BYTE      P2SKIP
      000000E8H   SFRSYM    DATA     BYTE      ADC0CN0
      000000A8H   SFRSYM    DATA     BIT       IE_EX0
      000000DFH   SFRSYM    DATA     BYTE      P3SKIP
      000000D8H.6 SFRSYM    DATA     BIT       PCA0CN0_CR
LX51 LINKER/LOCATER V4.66.30.0                                                        07/27/2019  23:22:19  PAGE 119


      000000A8H.2 SFRSYM    DATA     BIT       IE_EX1
      00000098H.7 SFRSYM    DATA     BIT       SCON0_SMODE
      000000A9H   SFRSYM    DATA     BYTE      CLKSEL
      000000F8H   SFRSYM    DATA     BIT       SPI0CN0_SPIEN
      000000F0H   SFRSYM    DATA     BYTE      B
      000000BEH   SFRSYM    DATA     BYTE      ADC0H
      000000E8H.6 SFRSYM    DATA     BIT       ADC0CN0_ADTM
      000000CAH   SFRSYM    DATA     WORD      TMR2RL
      000000BDH   SFRSYM    DATA     BYTE      ADC0L
      00000092H   SFRSYM    DATA     WORD      TMR3RL
      00000092H   SFRSYM    DATA     WORD      TMR4RL
      000000D8H   SFRSYM    DATA     BYTE      PCA0CN0
      000000E0H   SFRSYM    DATA     BYTE      ACC
      000000CAH   SFRSYM    DATA     WORD      TMR5RL
      000000FBH   SFRSYM    DATA     WORD      PCA0CP0
      000000E9H   SFRSYM    DATA     WORD      PCA0CP1
      000000EBH   SFRSYM    DATA     WORD      PCA0CP2
      000000EDH   SFRSYM    DATA     WORD      PCA0CP3
      0000008CH   SFRSYM    DATA     BYTE      TH0
      000000B8H.4 SFRSYM    DATA     BIT       IP_PS0
      000000FDH   SFRSYM    DATA     WORD      PCA0CP4
      0000008DH   SFRSYM    DATA     BYTE      TH1
      000000FAH   SFRSYM    DATA     BYTE      PCA0H
      000000B8H.1 SFRSYM    DATA     BIT       IP_PT0
      000000B8H.3 SFRSYM    DATA     BIT       IP_PT1
      000000C0H.2 SFRSYM    DATA     BIT       SMB0CN0_ARBLOST
      000000B8H.5 SFRSYM    DATA     BIT       IP_PT2
      0000008AH   SFRSYM    DATA     BYTE      TL0
      000000F8H.1 SFRSYM    DATA     BIT       SPI0CN0_TXBMT
      000000C0H.2 SFRSYM    DATA     BIT       SMB1CN0_ARBLOST
      000000D0H.5 SFRSYM    DATA     BIT       PSW_F0
      000000A8H.6 SFRSYM    DATA     BIT       IE_ESPI0
      0000008BH   SFRSYM    DATA     BYTE      TL1
      000000F9H   SFRSYM    DATA     BYTE      PCA0L
      000000C0H   SFRSYM    DATA     BIT       SMB0CN0_SI
      000000D0H.1 SFRSYM    DATA     BIT       PSW_F1
      00000080H   SFRSYM    DATA     BIT       P0_B0
      000000B8H   SFRSYM    DATA     BIT       IP_PX0
      000000C9H   SFRSYM    DATA     BYTE      REG01CN
      000000C0H   SFRSYM    DATA     BIT       SMB1CN0_SI
      00000090H   SFRSYM    DATA     BIT       P1_B0
      00000080H.1 SFRSYM    DATA     BIT       P0_B1
      000000B8H.2 SFRSYM    DATA     BIT       IP_PX1
      0000009BH   SFRSYM    DATA     BYTE      CMP0CN0
      00000088H.1 SFRSYM    DATA     BIT       TCON_IE0
      000000A0H   SFRSYM    DATA     BIT       P2_B0
      00000090H.1 SFRSYM    DATA     BIT       P1_B1
      00000080H.2 SFRSYM    DATA     BIT       P0_B2
      0000009AH   SFRSYM    DATA     BYTE      CMP1CN0
      00000088H.3 SFRSYM    DATA     BIT       TCON_IE1
      000000B0H   SFRSYM    DATA     BIT       P3_B0
      000000A0H.1 SFRSYM    DATA     BIT       P2_B1
      00000090H.2 SFRSYM    DATA     BIT       P1_B2
      00000080H.3 SFRSYM    DATA     BIT       P0_B3
      000000C0H   SFRSYM    DATA     BYTE      SMB0CN0
      000000B0H.1 SFRSYM    DATA     BIT       P3_B1
      000000A0H.2 SFRSYM    DATA     BIT       P2_B2
      00000090H.3 SFRSYM    DATA     BIT       P1_B3
      00000080H.4 SFRSYM    DATA     BIT       P0_B4
      000000C0H   SFRSYM    DATA     BYTE      SMB1CN0
      000000B0H.2 SFRSYM    DATA     BIT       P3_B2
      000000A0H.3 SFRSYM    DATA     BIT       P2_B3
LX51 LINKER/LOCATER V4.66.30.0                                                        07/27/2019  23:22:19  PAGE 120


      00000090H.4 SFRSYM    DATA     BIT       P1_B4
      00000080H.5 SFRSYM    DATA     BIT       P0_B5
      000000B0H.3 SFRSYM    DATA     BIT       P3_B3
      000000A0H.4 SFRSYM    DATA     BIT       P2_B4
      00000090H.5 SFRSYM    DATA     BIT       P1_B5
      00000080H.6 SFRSYM    DATA     BIT       P0_B6
      000000B0H.4 SFRSYM    DATA     BIT       P3_B4
      000000A0H.5 SFRSYM    DATA     BIT       P2_B5
      00000090H.6 SFRSYM    DATA     BIT       P1_B6
      00000080H.7 SFRSYM    DATA     BIT       P0_B7
      000000B0H.5 SFRSYM    DATA     BIT       P3_B5
      000000A0H.6 SFRSYM    DATA     BIT       P2_B6
      00000090H.7 SFRSYM    DATA     BIT       P1_B7
      000000B0H.6 SFRSYM    DATA     BIT       P3_B6
      000000A0H.7 SFRSYM    DATA     BIT       P2_B7
      000000B0H.7 SFRSYM    DATA     BIT       P3_B7
      00000083H   SFRSYM    DATA     BYTE      DPH
      000000C4H   SFRSYM    DATA     BYTE      ADC0GTH
      000000C8H.7 SFRSYM    DATA     BIT       TMR2CN0_TF2H
      000000C8H.3 SFRSYM    DATA     BIT       TMR2CN0_T2SPLIT
      000000D0H.6 SFRSYM    DATA     BIT       PSW_AC
      000000F8H   SFRSYM    DATA     BYTE      SPI0CN0
      000000B3H   SFRSYM    DATA     BYTE      HFO0CAL
      00000088H.5 SFRSYM    DATA     BIT       TCON_TF0
      00000098H   SFRSYM    DATA     BIT       SCON0_RI
      00000082H   SFRSYM    DATA     BYTE      DPL
      00000088H.7 SFRSYM    DATA     BIT       TCON_TF1
      00000099H   SFRSYM    DATA     BYTE      SBUF0
      00000087H   SFRSYM    DATA     BYTE      PCON0
      000000C3H   SFRSYM    DATA     BYTE      ADC0GTL
      000000C8H.6 SFRSYM    DATA     BIT       TMR2CN0_TF2L
      00000098H.1 SFRSYM    DATA     BIT       SCON0_TI
      000000E8H   SFRSYM    DATA     BIT       ADC0CN0_ADCM0
      000000D3H   SFRSYM    DATA     BYTE      SBUF1
      000000C6H   SFRSYM    DATA     BYTE      ADC0LTH
      00000088H   SFRSYM    DATA     BIT       TCON_IT0
      000000E8H.1 SFRSYM    DATA     BIT       ADC0CN0_ADCM1
      000000EFH   SFRSYM    DATA     BYTE      RSTSRC
      000000C8H.7 SFRSYM    DATA     BIT       TMR5CN0_TF5H
      000000C8H.3 SFRSYM    DATA     BIT       TMR5CN0_T5SPLIT
      00000088H.2 SFRSYM    DATA     BIT       TCON_IT1
      000000E8H.2 SFRSYM    DATA     BIT       ADC0CN0_ADCM2
      00000098H   SFRSYM    DATA     BYTE      SCON0
      000000E8H.3 SFRSYM    DATA     BIT       ADC0CN0_ADWINT
      000000B4H   SFRSYM    DATA     WORD      SBRL1
      000000E5H   SFRSYM    DATA     BYTE      SMOD1
      000000D2H   SFRSYM    DATA     BYTE      SCON1
      000000BAH   SFRSYM    DATA     BYTE      AMX0N
      000000E8H.4 SFRSYM    DATA     BIT       ADC0CN0_ADBUSY
      000000CEH   SFRSYM    DATA     BYTE      SMB0ADM
      000000C5H   SFRSYM    DATA     BYTE      ADC0LTL
      000000F8H.5 SFRSYM    DATA     BIT       SPI0CN0_MODF
      000000B8H.6 SFRSYM    DATA     BIT       IP_PSPI0
      000000CEH   SFRSYM    DATA     BYTE      SMB1ADM
      000000BBH   SFRSYM    DATA     BYTE      AMX0P
      000000C8H.6 SFRSYM    DATA     BIT       TMR5CN0_TF5L
      000000C8H   SFRSYM    DATA     BYTE      TMR2CN0
      00000091H   SFRSYM    DATA     BYTE      TMR3CN0
      00000091H   SFRSYM    DATA     BYTE      TMR4CN0
      000000C8H   SFRSYM    DATA     BYTE      TMR5CN0
      000000CFH   SFRSYM    DATA     BYTE      SMB0ADR
      00000088H.4 SFRSYM    DATA     BIT       TCON_TR0
LX51 LINKER/LOCATER V4.66.30.0                                                        07/27/2019  23:22:19  PAGE 121


      000000CFH   SFRSYM    DATA     BYTE      SMB1ADR
      000000C8H.4 SFRSYM    DATA     BIT       TMR2CN0_TF2CEN
      00000088H.6 SFRSYM    DATA     BIT       TCON_TR1
      000000C2H   SFRSYM    DATA     BYTE      SMB0DAT
      000000CDH   SFRSYM    DATA     BYTE      TMR2H
      000000A1H   SFRSYM    DATA     BYTE      SPI0CFG
      000000C2H   SFRSYM    DATA     BYTE      SMB1DAT
      00000095H   SFRSYM    DATA     BYTE      TMR3H
      00000095H   SFRSYM    DATA     BYTE      TMR4H
      000000CDH   SFRSYM    DATA     BYTE      TMR5H
      000000CCH   SFRSYM    DATA     BYTE      TMR2L
      000000F8H.7 SFRSYM    DATA     BIT       SPI0CN0_SPIF
      00000096H   SFRSYM    DATA     BYTE      USB0ADR
      00000094H   SFRSYM    DATA     BYTE      TMR3L
      000000A8H.7 SFRSYM    DATA     BIT       IE_EA
      00000094H   SFRSYM    DATA     BYTE      TMR4L
      00000097H   SFRSYM    DATA     BYTE      USB0DAT
      000000CCH   SFRSYM    DATA     BYTE      TMR5L
      000000B6H   SFRSYM    DATA     BYTE      FLSCL
      000000C8H.5 SFRSYM    DATA     BIT       TMR2CN0_TF2LEN
      000000F8H.6 SFRSYM    DATA     BIT       SPI0CN0_WCOL
      000000F8H.2 SFRSYM    DATA     BIT       SPI0CN0_NSSMD0
      000000D0H.7 SFRSYM    DATA     BIT       PSW_CY
      000000A3H   SFRSYM    DATA     BYTE      SPI0DAT
      000000F8H.3 SFRSYM    DATA     BIT       SPI0CN0_NSSMD1
      000000BDH   SFRSYM    DATA     WORD      ADC0
      000000B9H   SFRSYM    DATA     BYTE      SMBTC
      000000D0H   SFRSYM    DATA     BYTE      PSW
      000000C8H.5 SFRSYM    DATA     BIT       TMR5CN0_TF5LEN
      000000B7H   SFRSYM    DATA     BYTE      FLKEY

      01005A49H   BLOCK     CODE     ---       LVL=0
      01005A49H   LINE      CODE     ---       #14
      01005A49H   LINE      CODE     ---       #15
      01005A49H   LINE      CODE     ---       #17
      01005A59H   LINE      CODE     ---       #18
      ---         BLOCKEND  ---      ---       LVL=0

      01005B95H   BLOCK     CODE     ---       LVL=0
      01005B95H   LINE      CODE     ---       #20
      01005B95H   LINE      CODE     ---       #21
      01005B95H   LINE      CODE     ---       #22
      01005B99H   LINE      CODE     ---       #23
      ---         BLOCKEND  ---      ---       LVL=0

      010058A1H   BLOCK     CODE     ---       LVL=0
      00000028H   SYMBOL    DATA     BYTE      erasepage_rsvd
      010058A1H   LINE      CODE     ---       #25
      010058A3H   LINE      CODE     ---       #26
      010058A3H   LINE      CODE     ---       #27
      010058A6H   LINE      CODE     ---       #29
      010058AAH   LINE      CODE     ---       #30
      010058B5H   LINE      CODE     ---       #31
      010058B7H   LINE      CODE     ---       #32
      010058B9H   LINE      CODE     ---       #34
      010058BDH   LINE      CODE     ---       #35
      ---         BLOCKEND  ---      ---       LVL=0

      010056FCH   BLOCK     CODE     ---       LVL=0
      00000006H   SYMBOL    DATA     WORD      addr
      00000004H   SYMBOL    DATA     ---       dat
      00000003H   SYMBOL    DATA     BYTE      len
LX51 LINKER/LOCATER V4.66.30.0                                                        07/27/2019  23:22:19  PAGE 122


      010056FCH   BLOCK     CODE     NEAR LAB  LVL=1
      00000007H   SYMBOL    DATA     BYTE      c
      00000028H   SYMBOL    DATA     ---       flash
      ---         BLOCKEND  ---      ---       LVL=1
      010056FCH   LINE      CODE     ---       #37
      010056FCH   LINE      CODE     ---       #38
      010056FCH   LINE      CODE     ---       #42
      01005700H   LINE      CODE     ---       #44
      01005706H   LINE      CODE     ---       #45
      01005718H   LINE      CODE     ---       #46
      01005724H   LINE      CODE     ---       #47
      01005726H   LINE      CODE     ---       #48
      ---         BLOCKEND  ---      ---       LVL=0

      01005808H   BLOCK     CODE     ---       LVL=0
      00000006H   SYMBOL    DATA     WORD      addr
      00000005H   SYMBOL    DATA     BYTE      dat
      01005808H   BLOCK     CODE     NEAR LAB  LVL=1
      00000082H   SYMBOL    DATA     ---       flash
      00000020H.0 SYMBOL    BIT      BIT       ea_save
      ---         BLOCKEND  ---      ---       LVL=1
      01005808H   LINE      CODE     ---       #50
      01005808H   LINE      CODE     ---       #51
      01005808H   LINE      CODE     ---       #55
      0100580CH   LINE      CODE     ---       #58
      01005810H   LINE      CODE     ---       #59
      01005812H   LINE      CODE     ---       #62
      01005815H   LINE      CODE     ---       #63
      01005818H   LINE      CODE     ---       #66
      0100581BH   LINE      CODE     ---       #70
      0100581EH   LINE      CODE     ---       #73
      01005820H   LINE      CODE     ---       #76
      01005823H   LINE      CODE     ---       #79
      01005827H   LINE      CODE     ---       #80
      ---         BLOCKEND  ---      ---       LVL=0

      01005B6CH   BLOCK     CODE     ---       LVL=0
      00000006H   SYMBOL    DATA     WORD      addr
      01005B6CH   LINE      CODE     ---       #82
      01005B6CH   LINE      CODE     ---       #83
      01005B6CH   LINE      CODE     ---       #84
      01005B6FH   LINE      CODE     ---       #85
      ---         BLOCKEND  ---      ---       LVL=0

      01005616H   BLOCK     CODE     ---       LVL=0
      00000029H   SYMBOL    DATA     WORD      addr
      0000002BH   SYMBOL    DATA     ---       dat
      00000003H   SYMBOL    DATA     BYTE      len
      01005616H   LINE      CODE     ---       #88
      0100561EH   LINE      CODE     ---       #89
      0100561EH   LINE      CODE     ---       #90
      01005624H   LINE      CODE     ---       #91
      01005644H   LINE      CODE     ---       #92
      01005646H   LINE      CODE     ---       #93
      ---         BLOCKEND  ---      ---       LVL=0

      ---         MODULE    ---      ---       RGBLED_PROG
      01002971H   PUBLIC    CODE     ---       ledprog
      01003793H   PUBLIC    CODE     ---       _ledprog_rainbow
      01003193H   PUBLIC    CODE     ---       _ledprog_pfade1
      0100429BH   PUBLIC    CODE     ---       _ledprog_calt
      01003F00H   PUBLIC    CODE     ---       _ledprog_cmirror
LX51 LINKER/LOCATER V4.66.30.0                                                        07/27/2019  23:22:19  PAGE 123


      01003FC1H   PUBLIC    CODE     ---       _ledprog_cflip
      01000006H   PUBLIC    CODE     ---       _ledprog_ccross
      010035B6H   PUBLIC    CODE     ---       _ledprog_randomcolor
      01004132H   PUBLIC    CODE     ---       _ledprog_random
      0100471DH   PUBLIC    CODE     ---       _ledprog_circler
      010033B9H   PUBLIC    CODE     ---       _ledprog_flicker
      01005BB2H   PUBLIC    CODE     ---       _ledprog_solid_edit
      0100407AH   PUBLIC    CODE     ---       _ledprog_solid
      000000A2H   SFRSYM    DATA     BYTE      SPI0CKR
      00000080H   SFRSYM    DATA     BYTE      P0
      000000D0H.2 SFRSYM    DATA     BIT       PSW_OV
      000000B1H   SFRSYM    DATA     BYTE      XOSC0CN
      00000090H   SFRSYM    DATA     BYTE      P1
      000000A0H   SFRSYM    DATA     BYTE      P2
      000000B0H   SFRSYM    DATA     BYTE      P3
      000000BCH   SFRSYM    DATA     BYTE      ADC0CF
      000000C8H   SFRSYM    DATA     BIT       TMR2CN0_T2XCLK
      000000C7H   SFRSYM    DATA     BYTE      P4
      000000C0H.7 SFRSYM    DATA     BIT       SMB0CN0_MASTER
      000000F9H   SFRSYM    DATA     WORD      PCA0
      000000E6H   SFRSYM    DATA     BYTE      EIE1
      000000C0H.7 SFRSYM    DATA     BIT       SMB1CN0_MASTER
      000000C0H.1 SFRSYM    DATA     BIT       SMB0CN0_ACK
      000000D7H   SFRSYM    DATA     BYTE      USB0XCN
      000000E7H   SFRSYM    DATA     BYTE      EIE2
      000000C0H.1 SFRSYM    DATA     BIT       SMB1CN0_ACK
      0000008FH   SFRSYM    DATA     BYTE      PSCTL
      000000E4H   SFRSYM    DATA     BYTE      IT01CF
      000000C8H   SFRSYM    DATA     BIT       TMR5CN0_T5XCLK
      000000C0H.6 SFRSYM    DATA     BIT       SMB0CN0_TXMODE
      000000C0H.6 SFRSYM    DATA     BIT       SMB1CN0_TXMODE
      000000BFH   SFRSYM    DATA     BYTE      SFRPAGE
      000000A4H   SFRSYM    DATA     BYTE      P0MDOUT
      000000A5H   SFRSYM    DATA     BYTE      P1MDOUT
      000000E8H.5 SFRSYM    DATA     BIT       ADC0CN0_ADINT
      000000CBH   SFRSYM    DATA     BYTE      TMR2RLH
      000000A6H   SFRSYM    DATA     BYTE      P2MDOUT
      000000A8H   SFRSYM    DATA     BYTE      IE
      00000093H   SFRSYM    DATA     BYTE      TMR3RLH
      000000A7H   SFRSYM    DATA     BYTE      P3MDOUT
      00000093H   SFRSYM    DATA     BYTE      TMR4RLH
      000000AEH   SFRSYM    DATA     BYTE      P4MDOUT
      000000F6H   SFRSYM    DATA     BYTE      EIP1
      000000CBH   SFRSYM    DATA     BYTE      TMR5RLH
      000000F7H   SFRSYM    DATA     BYTE      EIP2
      00000098H.2 SFRSYM    DATA     BIT       SCON0_RB8
      000000CAH   SFRSYM    DATA     BYTE      TMR2RLL
      000000FCH   SFRSYM    DATA     BYTE      PCA0CPH0
      00000092H   SFRSYM    DATA     BYTE      TMR3RLL
      000000EAH   SFRSYM    DATA     BYTE      PCA0CPH1
      00000098H.3 SFRSYM    DATA     BIT       SCON0_TB8
      000000F0H   SFRSYM    DATA     BIT       B_B0
      00000082H   SFRSYM    DATA     WORD      DP
      00000092H   SFRSYM    DATA     BYTE      TMR4RLL
      000000ECH   SFRSYM    DATA     BYTE      PCA0CPH2
      000000F0H.1 SFRSYM    DATA     BIT       B_B1
      000000C3H   SFRSYM    DATA     WORD      ADC0GT
      000000CAH   SFRSYM    DATA     BYTE      TMR5RLL
      000000EEH   SFRSYM    DATA     BYTE      PCA0CPH3
      000000F0H.2 SFRSYM    DATA     BIT       B_B2
      000000FBH   SFRSYM    DATA     BYTE      PCA0CPL0
      000000FEH   SFRSYM    DATA     BYTE      PCA0CPH4
LX51 LINKER/LOCATER V4.66.30.0                                                        07/27/2019  23:22:19  PAGE 124


      00000085H   SFRSYM    DATA     BYTE      EMI0CF
      000000F0H.3 SFRSYM    DATA     BIT       B_B3
      000000D9H   SFRSYM    DATA     BYTE      PCA0MD
      000000DAH   SFRSYM    DATA     BYTE      PCA0CPM0
      000000E9H   SFRSYM    DATA     BYTE      PCA0CPL1
      000000F0H.4 SFRSYM    DATA     BIT       B_B4
      000000DBH   SFRSYM    DATA     BYTE      PCA0CPM1
      000000EBH   SFRSYM    DATA     BYTE      PCA0CPL2
      000000F0H.5 SFRSYM    DATA     BIT       B_B5
      000000DCH   SFRSYM    DATA     BYTE      PCA0CPM2
      000000EDH   SFRSYM    DATA     BYTE      PCA0CPL3
      000000B8H   SFRSYM    DATA     BYTE      IP
      000000F0H.6 SFRSYM    DATA     BIT       B_B6
      000000C5H   SFRSYM    DATA     WORD      ADC0LT
      000000DDH   SFRSYM    DATA     BYTE      PCA0CPM3
      000000FDH   SFRSYM    DATA     BYTE      PCA0CPL4
      00000098H.5 SFRSYM    DATA     BIT       SCON0_MCE
      000000F0H.7 SFRSYM    DATA     BIT       B_B7
      000000DEH   SFRSYM    DATA     BYTE      PCA0CPM4
      000000E1H   SFRSYM    DATA     BYTE      XBR0
      000000C1H   SFRSYM    DATA     BYTE      SMB0CF
      000000E2H   SFRSYM    DATA     BYTE      XBR1
      000000C1H   SFRSYM    DATA     BYTE      SMB1CF
      000000AFH   SFRSYM    DATA     BYTE      PFE0CN
      000000AAH   SFRSYM    DATA     BYTE      EMI0CN
      000000C0H.5 SFRSYM    DATA     BIT       SMB0CN0_STA
      000000E3H   SFRSYM    DATA     BYTE      XBR2
      000000C0H.5 SFRSYM    DATA     BIT       SMB1CN0_STA
      000000E0H   SFRSYM    DATA     BIT       ACC_ACC0
      000000D1H   SFRSYM    DATA     BYTE      REF0CN
      000000B2H   SFRSYM    DATA     BYTE      HFO0CN
      0000008EH   SFRSYM    DATA     BYTE      CKCON0
      000000E0H.1 SFRSYM    DATA     BIT       ACC_ACC1
      000000E4H   SFRSYM    DATA     BYTE      CKCON1
      000000C8H.2 SFRSYM    DATA     BIT       TMR2CN0_TR2
      000000E0H.2 SFRSYM    DATA     BIT       ACC_ACC2
      000000E0H.3 SFRSYM    DATA     BIT       ACC_ACC3
      00000081H   SFRSYM    DATA     BYTE      SP
      0000009DH   SFRSYM    DATA     BYTE      CMP0MD
      000000E0H.4 SFRSYM    DATA     BIT       ACC_ACC4
      00000086H   SFRSYM    DATA     BYTE      LFO0CN
      00000084H   SFRSYM    DATA     BYTE      EMI0TC
      0000009CH   SFRSYM    DATA     BYTE      CMP1MD
      000000D8H   SFRSYM    DATA     BIT       PCA0CN0_CCF0
      000000E0H.5 SFRSYM    DATA     BIT       ACC_ACC5
      000000D8H.1 SFRSYM    DATA     BIT       PCA0CN0_CCF1
      000000E0H.6 SFRSYM    DATA     BIT       ACC_ACC6
      000000CCH   SFRSYM    DATA     WORD      TMR2
      000000D8H.2 SFRSYM    DATA     BIT       PCA0CN0_CCF2
      000000E0H.7 SFRSYM    DATA     BIT       ACC_ACC7
      00000094H   SFRSYM    DATA     WORD      TMR3
      000000C8H.2 SFRSYM    DATA     BIT       TMR5CN0_TR5
      000000D8H.3 SFRSYM    DATA     BIT       PCA0CN0_CCF3
      00000094H   SFRSYM    DATA     WORD      TMR4
      000000ACH   SFRSYM    DATA     BYTE      SBCON1
      000000D8H.4 SFRSYM    DATA     BIT       PCA0CN0_CCF4
      000000CCH   SFRSYM    DATA     WORD      TMR5
      000000C0H.3 SFRSYM    DATA     BIT       SMB0CN0_ACKRQ
      000000FFH   SFRSYM    DATA     BYTE      VDM0CN
      000000F1H   SFRSYM    DATA     BYTE      P0MDIN
      000000C0H.3 SFRSYM    DATA     BIT       SMB1CN0_ACKRQ
      00000098H.4 SFRSYM    DATA     BIT       SCON0_REN
LX51 LINKER/LOCATER V4.66.30.0                                                        07/27/2019  23:22:19  PAGE 125


      000000F2H   SFRSYM    DATA     BYTE      P1MDIN
      000000F3H   SFRSYM    DATA     BYTE      P2MDIN
      000000C0H.4 SFRSYM    DATA     BIT       SMB0CN0_STO
      000000F4H   SFRSYM    DATA     BYTE      P3MDIN
      000000C0H.4 SFRSYM    DATA     BIT       SMB1CN0_STO
      000000B5H   SFRSYM    DATA     BYTE      SBRLH1
      000000F5H   SFRSYM    DATA     BYTE      P4MDIN
      000000D0H.3 SFRSYM    DATA     BIT       PSW_RS0
      000000D8H.7 SFRSYM    DATA     BIT       PCA0CN0_CF
      000000F8H.4 SFRSYM    DATA     BIT       SPI0CN0_RXOVRN
      000000D0H.4 SFRSYM    DATA     BIT       PSW_RS1
      000000B4H   SFRSYM    DATA     BYTE      SBRLL1
      000000E8H.7 SFRSYM    DATA     BIT       ADC0CN0_ADEN
      00000089H   SFRSYM    DATA     BYTE      TMOD
      00000088H   SFRSYM    DATA     BYTE      TCON
      000000D0H   SFRSYM    DATA     BIT       PSW_PARITY
      000000A8H.4 SFRSYM    DATA     BIT       IE_ES0
      0000009FH   SFRSYM    DATA     BYTE      CMP0MX
      000000A8H.1 SFRSYM    DATA     BIT       IE_ET0
      0000009EH   SFRSYM    DATA     BYTE      CMP1MX
      000000A8H.3 SFRSYM    DATA     BIT       IE_ET1
      000000D4H   SFRSYM    DATA     BYTE      P0SKIP
      000000C8H.1 SFRSYM    DATA     BIT       TMR2CN0_T2CSS
      000000A8H.5 SFRSYM    DATA     BIT       IE_ET2
      000000D5H   SFRSYM    DATA     BYTE      P1SKIP
      000000D6H   SFRSYM    DATA     BYTE      P2SKIP
      000000E8H   SFRSYM    DATA     BYTE      ADC0CN0
      000000A8H   SFRSYM    DATA     BIT       IE_EX0
      000000DFH   SFRSYM    DATA     BYTE      P3SKIP
      000000D8H.6 SFRSYM    DATA     BIT       PCA0CN0_CR
      000000A8H.2 SFRSYM    DATA     BIT       IE_EX1
      00000098H.7 SFRSYM    DATA     BIT       SCON0_SMODE
      000000A9H   SFRSYM    DATA     BYTE      CLKSEL
      000000F8H   SFRSYM    DATA     BIT       SPI0CN0_SPIEN
      000000F0H   SFRSYM    DATA     BYTE      B
      000000BEH   SFRSYM    DATA     BYTE      ADC0H
      000000E8H.6 SFRSYM    DATA     BIT       ADC0CN0_ADTM
      000000CAH   SFRSYM    DATA     WORD      TMR2RL
      000000BDH   SFRSYM    DATA     BYTE      ADC0L
      00000092H   SFRSYM    DATA     WORD      TMR3RL
      00000092H   SFRSYM    DATA     WORD      TMR4RL
      000000D8H   SFRSYM    DATA     BYTE      PCA0CN0
      000000E0H   SFRSYM    DATA     BYTE      ACC
      000000CAH   SFRSYM    DATA     WORD      TMR5RL
      000000FBH   SFRSYM    DATA     WORD      PCA0CP0
      000000E9H   SFRSYM    DATA     WORD      PCA0CP1
      000000EBH   SFRSYM    DATA     WORD      PCA0CP2
      000000EDH   SFRSYM    DATA     WORD      PCA0CP3
      0000008CH   SFRSYM    DATA     BYTE      TH0
      000000B8H.4 SFRSYM    DATA     BIT       IP_PS0
      000000FDH   SFRSYM    DATA     WORD      PCA0CP4
      0000008DH   SFRSYM    DATA     BYTE      TH1
      000000FAH   SFRSYM    DATA     BYTE      PCA0H
      000000B8H.1 SFRSYM    DATA     BIT       IP_PT0
      000000B8H.3 SFRSYM    DATA     BIT       IP_PT1
      000000C0H.2 SFRSYM    DATA     BIT       SMB0CN0_ARBLOST
      000000B8H.5 SFRSYM    DATA     BIT       IP_PT2
      0000008AH   SFRSYM    DATA     BYTE      TL0
      000000F8H.1 SFRSYM    DATA     BIT       SPI0CN0_TXBMT
      000000C0H.2 SFRSYM    DATA     BIT       SMB1CN0_ARBLOST
      000000D0H.5 SFRSYM    DATA     BIT       PSW_F0
      000000A8H.6 SFRSYM    DATA     BIT       IE_ESPI0
LX51 LINKER/LOCATER V4.66.30.0                                                        07/27/2019  23:22:19  PAGE 126


      0000008BH   SFRSYM    DATA     BYTE      TL1
      000000F9H   SFRSYM    DATA     BYTE      PCA0L
      000000C0H   SFRSYM    DATA     BIT       SMB0CN0_SI
      000000D0H.1 SFRSYM    DATA     BIT       PSW_F1
      00000080H   SFRSYM    DATA     BIT       P0_B0
      000000B8H   SFRSYM    DATA     BIT       IP_PX0
      000000C9H   SFRSYM    DATA     BYTE      REG01CN
      000000C0H   SFRSYM    DATA     BIT       SMB1CN0_SI
      00000090H   SFRSYM    DATA     BIT       P1_B0
      00000080H.1 SFRSYM    DATA     BIT       P0_B1
      000000B8H.2 SFRSYM    DATA     BIT       IP_PX1
      0000009BH   SFRSYM    DATA     BYTE      CMP0CN0
      00000088H.1 SFRSYM    DATA     BIT       TCON_IE0
      000000A0H   SFRSYM    DATA     BIT       P2_B0
      00000090H.1 SFRSYM    DATA     BIT       P1_B1
      00000080H.2 SFRSYM    DATA     BIT       P0_B2
      0000009AH   SFRSYM    DATA     BYTE      CMP1CN0
      00000088H.3 SFRSYM    DATA     BIT       TCON_IE1
      000000B0H   SFRSYM    DATA     BIT       P3_B0
      000000A0H.1 SFRSYM    DATA     BIT       P2_B1
      00000090H.2 SFRSYM    DATA     BIT       P1_B2
      00000080H.3 SFRSYM    DATA     BIT       P0_B3
      000000C0H   SFRSYM    DATA     BYTE      SMB0CN0
      000000B0H.1 SFRSYM    DATA     BIT       P3_B1
      000000A0H.2 SFRSYM    DATA     BIT       P2_B2
      00000090H.3 SFRSYM    DATA     BIT       P1_B3
      00000080H.4 SFRSYM    DATA     BIT       P0_B4
      000000C0H   SFRSYM    DATA     BYTE      SMB1CN0
      000000B0H.2 SFRSYM    DATA     BIT       P3_B2
      000000A0H.3 SFRSYM    DATA     BIT       P2_B3
      00000090H.4 SFRSYM    DATA     BIT       P1_B4
      00000080H.5 SFRSYM    DATA     BIT       P0_B5
      000000B0H.3 SFRSYM    DATA     BIT       P3_B3
      000000A0H.4 SFRSYM    DATA     BIT       P2_B4
      00000090H.5 SFRSYM    DATA     BIT       P1_B5
      00000080H.6 SFRSYM    DATA     BIT       P0_B6
      000000B0H.4 SFRSYM    DATA     BIT       P3_B4
      000000A0H.5 SFRSYM    DATA     BIT       P2_B5
      00000090H.6 SFRSYM    DATA     BIT       P1_B6
      00000080H.7 SFRSYM    DATA     BIT       P0_B7
      000000B0H.5 SFRSYM    DATA     BIT       P3_B5
      000000A0H.6 SFRSYM    DATA     BIT       P2_B6
      00000090H.7 SFRSYM    DATA     BIT       P1_B7
      000000B0H.6 SFRSYM    DATA     BIT       P3_B6
      000000A0H.7 SFRSYM    DATA     BIT       P2_B7
      000000B0H.7 SFRSYM    DATA     BIT       P3_B7
      00000083H   SFRSYM    DATA     BYTE      DPH
      000000C4H   SFRSYM    DATA     BYTE      ADC0GTH
      000000C8H.7 SFRSYM    DATA     BIT       TMR2CN0_TF2H
      000000C8H.3 SFRSYM    DATA     BIT       TMR2CN0_T2SPLIT
      000000D0H.6 SFRSYM    DATA     BIT       PSW_AC
      000000F8H   SFRSYM    DATA     BYTE      SPI0CN0
      000000B3H   SFRSYM    DATA     BYTE      HFO0CAL
      00000088H.5 SFRSYM    DATA     BIT       TCON_TF0
      00000098H   SFRSYM    DATA     BIT       SCON0_RI
      00000082H   SFRSYM    DATA     BYTE      DPL
      00000088H.7 SFRSYM    DATA     BIT       TCON_TF1
      00000099H   SFRSYM    DATA     BYTE      SBUF0
      00000087H   SFRSYM    DATA     BYTE      PCON0
      000000C3H   SFRSYM    DATA     BYTE      ADC0GTL
      000000C8H.6 SFRSYM    DATA     BIT       TMR2CN0_TF2L
      00000098H.1 SFRSYM    DATA     BIT       SCON0_TI
LX51 LINKER/LOCATER V4.66.30.0                                                        07/27/2019  23:22:19  PAGE 127


      000000E8H   SFRSYM    DATA     BIT       ADC0CN0_ADCM0
      000000D3H   SFRSYM    DATA     BYTE      SBUF1
      000000C6H   SFRSYM    DATA     BYTE      ADC0LTH
      00000088H   SFRSYM    DATA     BIT       TCON_IT0
      000000E8H.1 SFRSYM    DATA     BIT       ADC0CN0_ADCM1
      000000EFH   SFRSYM    DATA     BYTE      RSTSRC
      000000C8H.7 SFRSYM    DATA     BIT       TMR5CN0_TF5H
      000000C8H.3 SFRSYM    DATA     BIT       TMR5CN0_T5SPLIT
      00000088H.2 SFRSYM    DATA     BIT       TCON_IT1
      000000E8H.2 SFRSYM    DATA     BIT       ADC0CN0_ADCM2
      00000098H   SFRSYM    DATA     BYTE      SCON0
      000000E8H.3 SFRSYM    DATA     BIT       ADC0CN0_ADWINT
      000000B4H   SFRSYM    DATA     WORD      SBRL1
      000000E5H   SFRSYM    DATA     BYTE      SMOD1
      000000D2H   SFRSYM    DATA     BYTE      SCON1
      000000BAH   SFRSYM    DATA     BYTE      AMX0N
      000000E8H.4 SFRSYM    DATA     BIT       ADC0CN0_ADBUSY
      000000CEH   SFRSYM    DATA     BYTE      SMB0ADM
      000000C5H   SFRSYM    DATA     BYTE      ADC0LTL
      000000F8H.5 SFRSYM    DATA     BIT       SPI0CN0_MODF
      000000B8H.6 SFRSYM    DATA     BIT       IP_PSPI0
      000000CEH   SFRSYM    DATA     BYTE      SMB1ADM
      000000BBH   SFRSYM    DATA     BYTE      AMX0P
      000000C8H.6 SFRSYM    DATA     BIT       TMR5CN0_TF5L
      000000C8H   SFRSYM    DATA     BYTE      TMR2CN0
      00000091H   SFRSYM    DATA     BYTE      TMR3CN0
      00000091H   SFRSYM    DATA     BYTE      TMR4CN0
      000000C8H   SFRSYM    DATA     BYTE      TMR5CN0
      000000CFH   SFRSYM    DATA     BYTE      SMB0ADR
      00000088H.4 SFRSYM    DATA     BIT       TCON_TR0
      000000CFH   SFRSYM    DATA     BYTE      SMB1ADR
      000000C8H.4 SFRSYM    DATA     BIT       TMR2CN0_TF2CEN
      00000088H.6 SFRSYM    DATA     BIT       TCON_TR1
      000000C2H   SFRSYM    DATA     BYTE      SMB0DAT
      000000CDH   SFRSYM    DATA     BYTE      TMR2H
      000000A1H   SFRSYM    DATA     BYTE      SPI0CFG
      000000C2H   SFRSYM    DATA     BYTE      SMB1DAT
      00000095H   SFRSYM    DATA     BYTE      TMR3H
      00000095H   SFRSYM    DATA     BYTE      TMR4H
      000000CDH   SFRSYM    DATA     BYTE      TMR5H
      000000CCH   SFRSYM    DATA     BYTE      TMR2L
      000000F8H.7 SFRSYM    DATA     BIT       SPI0CN0_SPIF
      00000096H   SFRSYM    DATA     BYTE      USB0ADR
      00000094H   SFRSYM    DATA     BYTE      TMR3L
      000000A8H.7 SFRSYM    DATA     BIT       IE_EA
      00000094H   SFRSYM    DATA     BYTE      TMR4L
      00000097H   SFRSYM    DATA     BYTE      USB0DAT
      000000CCH   SFRSYM    DATA     BYTE      TMR5L
      000000B6H   SFRSYM    DATA     BYTE      FLSCL
      000000C8H.5 SFRSYM    DATA     BIT       TMR2CN0_TF2LEN
      000000F8H.6 SFRSYM    DATA     BIT       SPI0CN0_WCOL
      000000F8H.2 SFRSYM    DATA     BIT       SPI0CN0_NSSMD0
      000000D0H.7 SFRSYM    DATA     BIT       PSW_CY
      000000A3H   SFRSYM    DATA     BYTE      SPI0DAT
      000000F8H.3 SFRSYM    DATA     BIT       SPI0CN0_NSSMD1
      000000BDH   SFRSYM    DATA     WORD      ADC0
      000000B9H   SFRSYM    DATA     BYTE      SMBTC
      000000D0H   SFRSYM    DATA     BYTE      PSW
      000000C8H.5 SFRSYM    DATA     BIT       TMR5CN0_TF5LEN
      000000B7H   SFRSYM    DATA     BYTE      FLKEY
      00000086H   SYMBOL    IDATA    BYTE      led_tick
      00000087H   SYMBOL    IDATA    BYTE      led_idx
LX51 LINKER/LOCATER V4.66.30.0                                                        07/27/2019  23:22:19  PAGE 128


      020004BFH   SYMBOL    XDATA    BYTE      led_aux
      00000000H   SYMBOL    DATA     ---       prog

      0100407AH   BLOCK     CODE     ---       LVL=0
      00000043H   SYMBOL    DATA     ---       prog
      01004080H   BLOCK     CODE     NEAR LAB  LVL=1
      00000046H   SYMBOL    DATA     BYTE      i
      00000047H   SYMBOL    DATA     BYTE      flags
      ---         BLOCKEND  ---      ---       LVL=1
      0100407AH   LINE      CODE     ---       #32
      01004080H   LINE      CODE     ---       #33
      01004080H   LINE      CODE     ---       #35
      01004088H   LINE      CODE     ---       #43
      0100408BH   LINE      CODE     ---       #44
      01004095H   LINE      CODE     ---       #45
      010040B6H   LINE      CODE     ---       #46
      010040D6H   LINE      CODE     ---       #47
      010040E7H   LINE      CODE     ---       #48
      010040E9H   LINE      CODE     ---       #49
      01004102H   LINE      CODE     ---       #50
      01004114H   LINE      CODE     ---       #51
      01004126H   LINE      CODE     ---       #52
      01004126H   LINE      CODE     ---       #53
      01004131H   LINE      CODE     ---       #54
      ---         BLOCKEND  ---      ---       LVL=0

      01005BB2H   BLOCK     CODE     ---       LVL=0
      00000007H   SYMBOL    DATA     BYTE      state
      01005BB2H   LINE      CODE     ---       #56
      01005BB2H   LINE      CODE     ---       #57
      01005BB2H   LINE      CODE     ---       #58
      01005BB2H   LINE      CODE     ---       #59
      01005BB2H   LINE      CODE     ---       #61
      01005BB2H   LINE      CODE     ---       #62
      01005BB2H   LINE      CODE     ---       #63
      ---         BLOCKEND  ---      ---       LVL=0

      010033B9H   BLOCK     CODE     ---       LVL=0
      00000043H   SYMBOL    DATA     ---       prog
      010033BFH   BLOCK     CODE     NEAR LAB  LVL=1
      00000046H   SYMBOL    DATA     BYTE      i
      00000047H   SYMBOL    DATA     BYTE      flags
      00000048H   SYMBOL    DATA     BYTE      rnd
      00000049H   SYMBOL    DATA     BYTE      rnd_first
      ---         BLOCKEND  ---      ---       LVL=1
      010033B9H   LINE      CODE     ---       #65
      010033BFH   LINE      CODE     ---       #66
      010033BFH   LINE      CODE     ---       #68
      010033C8H   LINE      CODE     ---       #80
      010033CBH   LINE      CODE     ---       #81
      010033D3H   LINE      CODE     ---       #82
      010033DBH   LINE      CODE     ---       #84
      010033DEH   LINE      CODE     ---       #85
      010033FFH   LINE      CODE     ---       #87
      0100341BH   LINE      CODE     ---       #88
      0100343CH   LINE      CODE     ---       #89
      0100345CH   LINE      CODE     ---       #90
      0100346DH   LINE      CODE     ---       #91
      0100346FH   LINE      CODE     ---       #92
      01003488H   LINE      CODE     ---       #93
      0100349AH   LINE      CODE     ---       #94
      010034B0H   LINE      CODE     ---       #95
LX51 LINKER/LOCATER V4.66.30.0                                                        07/27/2019  23:22:19  PAGE 129


      010034B0H   LINE      CODE     ---       #96
      010034BCH   LINE      CODE     ---       #97
      010034BCH   LINE      CODE     ---       #98
      ---         BLOCKEND  ---      ---       LVL=0

      0100471DH   BLOCK     CODE     ---       LVL=0
      00000001H   SYMBOL    DATA     ---       prog
      0100471DH   BLOCK     CODE     NEAR LAB  LVL=1
      00000043H   SYMBOL    DATA     BYTE      i
      00000044H   SYMBOL    DATA     BYTE      offset
      00000007H   SYMBOL    DATA     BYTE      idx
      ---         BLOCKEND  ---      ---       LVL=1
      0100471DH   LINE      CODE     ---       #100
      0100471DH   LINE      CODE     ---       #101
      0100471DH   LINE      CODE     ---       #117
      01004720H   LINE      CODE     ---       #118
      0100472EH   LINE      CODE     ---       #119
      01004730H   LINE      CODE     ---       #121
      01004732H   LINE      CODE     ---       #122
      01004736H   LINE      CODE     ---       #124
      01004739H   LINE      CODE     ---       #125
      0100474CH   LINE      CODE     ---       #128
      01004759H   LINE      CODE     ---       #130
      01004775H   LINE      CODE     ---       #131
      0100478EH   LINE      CODE     ---       #132
      010047A4H   LINE      CODE     ---       #133
      010047ACH   LINE      CODE     ---       #134
      010047ACH   LINE      CODE     ---       #135
      ---         BLOCKEND  ---      ---       LVL=0

      01004132H   BLOCK     CODE     ---       LVL=0
      00000043H   SYMBOL    DATA     ---       prog
      01004138H   BLOCK     CODE     NEAR LAB  LVL=1
      00000046H   SYMBOL    DATA     BYTE      i
      00000047H   SYMBOL    DATA     BYTE      offset
      00000007H   SYMBOL    DATA     BYTE      rnd
      00000048H   SYMBOL    DATA     BYTE      rnd_first
      00000049H   SYMBOL    DATA     BYTE      flags
      ---         BLOCKEND  ---      ---       LVL=1
      01004132H   LINE      CODE     ---       #137
      01004138H   LINE      CODE     ---       #138
      01004138H   LINE      CODE     ---       #143
      01004140H   LINE      CODE     ---       #155
      01004143H   LINE      CODE     ---       #156
      01004154H   LINE      CODE     ---       #157
      01004156H   LINE      CODE     ---       #159
      0100415CH   LINE      CODE     ---       #161
      0100415FH   LINE      CODE     ---       #162
      0100417AH   LINE      CODE     ---       #164
      01004192H   LINE      CODE     ---       #166
      010041AEH   LINE      CODE     ---       #167
      010041C7H   LINE      CODE     ---       #168
      010041DDH   LINE      CODE     ---       #169
      010041E9H   LINE      CODE     ---       #170
      010041E9H   LINE      CODE     ---       #171
      ---         BLOCKEND  ---      ---       LVL=0

      010035B6H   BLOCK     CODE     ---       LVL=0
      00000043H   SYMBOL    DATA     ---       prog
      010035BCH   BLOCK     CODE     NEAR LAB  LVL=1
      00000046H   SYMBOL    DATA     BYTE      i
      00000047H   SYMBOL    DATA     BYTE      valid
LX51 LINKER/LOCATER V4.66.30.0                                                        07/27/2019  23:22:19  PAGE 130


      00000007H   SYMBOL    DATA     BYTE      rnd
      00000048H   SYMBOL    DATA     BYTE      rnd_first
      00000049H   SYMBOL    DATA     BYTE      flags
      ---         BLOCKEND  ---      ---       LVL=1
      010035B6H   LINE      CODE     ---       #173
      010035BCH   LINE      CODE     ---       #174
      010035BCH   LINE      CODE     ---       #179
      010035C4H   LINE      CODE     ---       #189
      010035C7H   LINE      CODE     ---       #190
      010035D8H   LINE      CODE     ---       #191
      010035DAH   LINE      CODE     ---       #193
      010035E0H   LINE      CODE     ---       #195
      010035E3H   LINE      CODE     ---       #196
      010035FEH   LINE      CODE     ---       #198
      01003616H   LINE      CODE     ---       #200
      01003649H   LINE      CODE     ---       #201
      01003670H   LINE      CODE     ---       #202
      01003688H   LINE      CODE     ---       #205
      01003695H   LINE      CODE     ---       #206
      01003698H   LINE      CODE     ---       #207
      01003698H   LINE      CODE     ---       #208
      010036A4H   LINE      CODE     ---       #209
      010036A4H   LINE      CODE     ---       #210
      ---         BLOCKEND  ---      ---       LVL=0

      01000006H   BLOCK     CODE     ---       LVL=0
      00000001H   SYMBOL    DATA     ---       prog
      01000006H   BLOCK     CODE     NEAR LAB  LVL=1
      00000043H   SYMBOL    DATA     BYTE      i
      00000044H   SYMBOL    DATA     BYTE      offset
      00000045H   SYMBOL    DATA     BYTE      flags
      ---         BLOCKEND  ---      ---       LVL=1
      01000006H   LINE      CODE     ---       #212
      01000006H   LINE      CODE     ---       #213
      01000006H   LINE      CODE     ---       #217
      0100000EH   LINE      CODE     ---       #227
      01000011H   LINE      CODE     ---       #228
      0100001FH   LINE      CODE     ---       #229
      01000021H   LINE      CODE     ---       #231
      01000023H   LINE      CODE     ---       #232
      01000027H   LINE      CODE     ---       #234
      0100002AH   LINE      CODE     ---       #235
      01000039H   LINE      CODE     ---       #237
      01000055H   LINE      CODE     ---       #238
      0100006EH   LINE      CODE     ---       #239
      01000084H   LINE      CODE     ---       #240
      0100008BH   LINE      CODE     ---       #241
      0100008BH   LINE      CODE     ---       #242
      ---         BLOCKEND  ---      ---       LVL=0

      01003FC1H   BLOCK     CODE     ---       LVL=0
      00000001H   SYMBOL    DATA     ---       prog
      01003FC1H   BLOCK     CODE     NEAR LAB  LVL=1
      00000043H   SYMBOL    DATA     BYTE      i
      00000044H   SYMBOL    DATA     BYTE      offset
      00000045H   SYMBOL    DATA     BYTE      flags
      ---         BLOCKEND  ---      ---       LVL=1
      01003FC1H   LINE      CODE     ---       #244
      01003FC1H   LINE      CODE     ---       #245
      01003FC1H   LINE      CODE     ---       #249
      01003FC9H   LINE      CODE     ---       #259
      01003FCCH   LINE      CODE     ---       #260
LX51 LINKER/LOCATER V4.66.30.0                                                        07/27/2019  23:22:19  PAGE 131


      01003FDDH   LINE      CODE     ---       #261
      01003FDFH   LINE      CODE     ---       #263
      01003FE1H   LINE      CODE     ---       #264
      01003FE5H   LINE      CODE     ---       #266
      01003FF2H   LINE      CODE     ---       #267
      01004001H   LINE      CODE     ---       #269
      0100402DH   LINE      CODE     ---       #270
      01004051H   LINE      CODE     ---       #271
      01004072H   LINE      CODE     ---       #272
      01004079H   LINE      CODE     ---       #273
      01004079H   LINE      CODE     ---       #274
      ---         BLOCKEND  ---      ---       LVL=0

      01003F00H   BLOCK     CODE     ---       LVL=0
      00000001H   SYMBOL    DATA     ---       prog
      01003F00H   BLOCK     CODE     NEAR LAB  LVL=1
      00000043H   SYMBOL    DATA     BYTE      i
      00000044H   SYMBOL    DATA     BYTE      offset
      00000045H   SYMBOL    DATA     BYTE      flags
      ---         BLOCKEND  ---      ---       LVL=1
      01003F00H   LINE      CODE     ---       #276
      01003F00H   LINE      CODE     ---       #277
      01003F00H   LINE      CODE     ---       #281
      01003F08H   LINE      CODE     ---       #291
      01003F0BH   LINE      CODE     ---       #292
      01003F1CH   LINE      CODE     ---       #293
      01003F1EH   LINE      CODE     ---       #295
      01003F20H   LINE      CODE     ---       #296
      01003F24H   LINE      CODE     ---       #298
      01003F31H   LINE      CODE     ---       #299
      01003F40H   LINE      CODE     ---       #301
      01003F71H   LINE      CODE     ---       #302
      01003F92H   LINE      CODE     ---       #303
      01003FB9H   LINE      CODE     ---       #304
      01003FC0H   LINE      CODE     ---       #305
      01003FC0H   LINE      CODE     ---       #306
      ---         BLOCKEND  ---      ---       LVL=0

      0100429BH   BLOCK     CODE     ---       LVL=0
      00000001H   SYMBOL    DATA     ---       prog
      0100429BH   BLOCK     CODE     NEAR LAB  LVL=1
      00000043H   SYMBOL    DATA     BYTE      i
      00000044H   SYMBOL    DATA     BYTE      offset
      00000045H   SYMBOL    DATA     BYTE      flags
      ---         BLOCKEND  ---      ---       LVL=1
      0100429BH   LINE      CODE     ---       #308
      0100429BH   LINE      CODE     ---       #309
      0100429BH   LINE      CODE     ---       #313
      010042A3H   LINE      CODE     ---       #323
      010042A6H   LINE      CODE     ---       #324
      010042B7H   LINE      CODE     ---       #325
      010042B9H   LINE      CODE     ---       #327
      010042BBH   LINE      CODE     ---       #328
      010042BFH   LINE      CODE     ---       #330
      010042C7H   LINE      CODE     ---       #332
      010042D1H   LINE      CODE     ---       #333
      010042FEH   LINE      CODE     ---       #334
      01004322H   LINE      CODE     ---       #335
      01004343H   LINE      CODE     ---       #336
      01004349H   LINE      CODE     ---       #337
      01004349H   LINE      CODE     ---       #338
      ---         BLOCKEND  ---      ---       LVL=0
LX51 LINKER/LOCATER V4.66.30.0                                                        07/27/2019  23:22:19  PAGE 132



      01003193H   BLOCK     CODE     ---       LVL=0
      00000043H   SYMBOL    DATA     ---       prog
      01003199H   BLOCK     CODE     NEAR LAB  LVL=1
      00000046H   SYMBOL    DATA     BYTE      i
      00000047H   SYMBOL    DATA     BYTE      fade
      00000048H   SYMBOL    DATA     BYTE      flags
      ---         BLOCKEND  ---      ---       LVL=1
      01003193H   LINE      CODE     ---       #340
      01003199H   LINE      CODE     ---       #341
      01003199H   LINE      CODE     ---       #345
      010031A1H   LINE      CODE     ---       #353
      010031A4H   LINE      CODE     ---       #354
      010031B5H   LINE      CODE     ---       #355
      010031B7H   LINE      CODE     ---       #356
      010031B9H   LINE      CODE     ---       #358
      010031BBH   LINE      CODE     ---       #360
      010031C1H   LINE      CODE     ---       #361
      010031C8H   LINE      CODE     ---       #362
      010031D0H   LINE      CODE     ---       #363
      010031D3H   LINE      CODE     ---       #364
      010031DBH   LINE      CODE     ---       #365
      010031E8H   LINE      CODE     ---       #366
      010031F2H   LINE      CODE     ---       #368
      010031F2H   LINE      CODE     ---       #369
      010031F6H   LINE      CODE     ---       #370
      010031F6H   LINE      CODE     ---       #372
      010031F9H   LINE      CODE     ---       #373
      01003203H   LINE      CODE     ---       #374
      01003224H   LINE      CODE     ---       #375
      01003244H   LINE      CODE     ---       #376
      01003255H   LINE      CODE     ---       #377
      01003257H   LINE      CODE     ---       #378
      01003270H   LINE      CODE     ---       #379
      01003282H   LINE      CODE     ---       #380
      0100329AH   LINE      CODE     ---       #381
      0100329AH   LINE      CODE     ---       #382
      010032A5H   LINE      CODE     ---       #383
      010032A5H   LINE      CODE     ---       #384
      ---         BLOCKEND  ---      ---       LVL=0

      01003793H   BLOCK     CODE     ---       LVL=0
      00000001H   SYMBOL    DATA     ---       prog
      01003793H   BLOCK     CODE     NEAR LAB  LVL=1
      00000043H   SYMBOL    DATA     BYTE      i
      00000044H   SYMBOL    DATA     BYTE      hue
      00000045H   SYMBOL    DATA     BYTE      range
      ---         BLOCKEND  ---      ---       LVL=1
      01003793H   LINE      CODE     ---       #386
      01003793H   LINE      CODE     ---       #387
      01003793H   LINE      CODE     ---       #405
      01003796H   LINE      CODE     ---       #406
      010037A7H   LINE      CODE     ---       #407
      010037A9H   LINE      CODE     ---       #408
      010037ABH   LINE      CODE     ---       #410
      010037BDH   LINE      CODE     ---       #411
      010037C1H   LINE      CODE     ---       #412
      010037C4H   LINE      CODE     ---       #413
      010037C6H   LINE      CODE     ---       #414
      010037D8H   LINE      CODE     ---       #415
      010037DBH   LINE      CODE     ---       #416
      010037DBH   LINE      CODE     ---       #418
LX51 LINKER/LOCATER V4.66.30.0                                                        07/27/2019  23:22:19  PAGE 133


      010037E3H   LINE      CODE     ---       #419
      010037E5H   LINE      CODE     ---       #420
      010037F4H   LINE      CODE     ---       #421
      010037F4H   LINE      CODE     ---       #424
      010037FBH   LINE      CODE     ---       #425
      01003801H   LINE      CODE     ---       #427
      01003807H   LINE      CODE     ---       #428
      01003809H   LINE      CODE     ---       #430
      0100380CH   LINE      CODE     ---       #431
      0100380CH   LINE      CODE     ---       #432
      0100380EH   LINE      CODE     ---       #433
      01003812H   LINE      CODE     ---       #435
      01003818H   LINE      CODE     ---       #436
      0100381AH   LINE      CODE     ---       #438
      01003821H   LINE      CODE     ---       #439
      01003821H   LINE      CODE     ---       #440
      01003821H   LINE      CODE     ---       #442
      01003824H   LINE      CODE     ---       #443
      0100384BH   LINE      CODE     ---       #444
      0100385DH   LINE      CODE     ---       #445
      0100386FH   LINE      CODE     ---       #446
      01003876H   LINE      CODE     ---       #447
      01003876H   LINE      CODE     ---       #448
      ---         BLOCKEND  ---      ---       LVL=0

      ---         MODULE    ---      ---       CHECKSUM
      010058BEH   PUBLIC    CODE     ---       _checksum_gen

      010058BEH   BLOCK     CODE     ---       LVL=0
      0000002BH   SYMBOL    DATA     ---       dat
      00000005H   SYMBOL    DATA     BYTE      len
      010058C4H   BLOCK     CODE     NEAR LAB  LVL=1
      00000007H   SYMBOL    DATA     BYTE      r
      ---         BLOCKEND  ---      ---       LVL=1
      010058BEH   LINE      CODE     ---       #12
      010058C4H   LINE      CODE     ---       #13
      010058C4H   LINE      CODE     ---       #14
      010058C6H   LINE      CODE     ---       #16
      010058C9H   LINE      CODE     ---       #17
      010058D7H   LINE      CODE     ---       #18
      010058D8H   LINE      CODE     ---       #19
      010058DAH   LINE      CODE     ---       #21
      010058DAH   LINE      CODE     ---       #22
      ---         BLOCKEND  ---      ---       LVL=0
      00000001H   SYMBOL    DATA     ---       dat
      00000005H   SYMBOL    DATA     BYTE      len

      ---         MODULE    ---      ---       I8ATAN2
      01003BD6H   PUBLIC    CODE     ---       _i8atan2
      010056A5H   SYMBOL    CODE     ---       _iat2

      010056A5H   BLOCK     CODE     ---       LVL=0
      00000007H   SYMBOL    DATA     CHAR      y
      00000005H   SYMBOL    DATA     CHAR      x
      010056A5H   LINE      CODE     ---       #12
      010056A5H   LINE      CODE     ---       #13
      010056A5H   LINE      CODE     ---       #14
      010056D0H   LINE      CODE     ---       #15
      ---         BLOCKEND  ---      ---       LVL=0

      01003BD6H   BLOCK     CODE     ---       LVL=0
      0000002AH   SYMBOL    DATA     CHAR      y
LX51 LINKER/LOCATER V4.66.30.0                                                        07/27/2019  23:22:19  PAGE 134


      00000006H   SYMBOL    DATA     CHAR      x
      01003BD6H   LINE      CODE     ---       #17
      01003BDAH   LINE      CODE     ---       #18
      01003BDAH   LINE      CODE     ---       #20
      01003BE3H   LINE      CODE     ---       #21
      01003BEAH   LINE      CODE     ---       #22
      01003BF6H   LINE      CODE     ---       #23
      01003C06H   LINE      CODE     ---       #24
      01003C06H   LINE      CODE     ---       #25
      01003C0CH   LINE      CODE     ---       #26
      01003C1DH   LINE      CODE     ---       #27
      01003C1DH   LINE      CODE     ---       #28
      01003C1DH   LINE      CODE     ---       #29
      01003C2CH   LINE      CODE     ---       #30
      01003C39H   LINE      CODE     ---       #31
      01003C39H   LINE      CODE     ---       #32
      01003C48H   LINE      CODE     ---       #33
      01003C48H   LINE      CODE     ---       #34
      01003C48H   LINE      CODE     ---       #35
      01003C48H   LINE      CODE     ---       #36
      01003C50H   LINE      CODE     ---       #37
      01003C5CH   LINE      CODE     ---       #38
      01003C6BH   LINE      CODE     ---       #39
      01003C6BH   LINE      CODE     ---       #40
      01003C77H   LINE      CODE     ---       #41
      01003C77H   LINE      CODE     ---       #42
      01003C77H   LINE      CODE     ---       #43
      01003C87H   LINE      CODE     ---       #44
      01003C94H   LINE      CODE     ---       #45
      01003C94H   LINE      CODE     ---       #46
      01003CA4H   LINE      CODE     ---       #47
      01003CA4H   LINE      CODE     ---       #48
      01003CA4H   LINE      CODE     ---       #49
      01003CA4H   LINE      CODE     ---       #50
      ---         BLOCKEND  ---      ---       LVL=0

      ---         MODULE    ---      ---       RAND16
      01005ACCH   PUBLIC    CODE     NEAR LAB  _RAND16_INIT
      010054C8H   PUBLIC    CODE     NEAR LAB  RAND16
      000000F0H   SFRSYM    DATA     BYTE      B
      01005500H   SYMBOL    CODE     NEAR LAB  ?C0001
      010054CBH   SYMBOL    CODE     NEAR LAB  ?RANDOM_LOOP
      010054F7H   SYMBOL    CODE     NEAR LAB  ?RANDOM_X
      020004B8H   SYMBOL    XDATA    BYTE      LFSR

      010054C8H   BLOCK     CODE     NEAR LAB  LVL=0
      010054C8H   LINE      CODE     ---       #152
      010054CBH   LINE      CODE     ---       #160
      010054CCH   LINE      CODE     ---       #162
      010054CFH   LINE      CODE     ---       #164
      010054D0H   LINE      CODE     ---       #166
      010054D1H   LINE      CODE     ---       #168
      010054D2H   LINE      CODE     ---       #170
      010054D3H   LINE      CODE     ---       #172
      010054D4H   LINE      CODE     ---       #174
      010054D5H   LINE      CODE     ---       #176
      010054D6H   LINE      CODE     ---       #178
      010054D7H   LINE      CODE     ---       #180
      010054D8H   LINE      CODE     ---       #182
      010054D9H   LINE      CODE     ---       #184
      010054DAH   LINE      CODE     ---       #186
      010054DBH   LINE      CODE     ---       #188
LX51 LINKER/LOCATER V4.66.30.0                                                        07/27/2019  23:22:19  PAGE 135


      010054DCH   LINE      CODE     ---       #190
      010054DDH   LINE      CODE     ---       #192
      010054DEH   LINE      CODE     ---       #196
      010054E0H   LINE      CODE     ---       #200
      010054E3H   LINE      CODE     ---       #202
      010054E4H   LINE      CODE     ---       #204
      010054E6H   LINE      CODE     ---       #206
      010054E7H   LINE      CODE     ---       #208
      010054E8H   LINE      CODE     ---       #210
      010054E9H   LINE      CODE     ---       #212
      010054EBH   LINE      CODE     ---       #214
      010054ECH   LINE      CODE     ---       #216
      010054EDH   LINE      CODE     ---       #218
      010054EEH   LINE      CODE     ---       #220
      010054F0H   LINE      CODE     ---       #222
      010054F1H   LINE      CODE     ---       #224
      010054F2H   LINE      CODE     ---       #226
      010054F3H   LINE      CODE     ---       #228
      010054F5H   LINE      CODE     ---       #230
      010054F6H   LINE      CODE     ---       #232
      010054F7H   LINE      CODE     ---       #240
      010054FAH   LINE      CODE     ---       #247
      010054FDH   LINE      CODE     ---       #248
      01005500H   LINE      CODE     ---       #252
      ---         BLOCKEND  ---      ---       LVL=0

      01005ACCH   BLOCK     CODE     NEAR LAB  LVL=0
      01005ACCH   LINE      CODE     ---       #266
      01005ACEH   LINE      CODE     ---       #267
      01005ACFH   LINE      CODE     ---       #268
      01005AD0H   LINE      CODE     ---       #269
      01005AD3H   LINE      CODE     ---       #270
      01005AD6H   LINE      CODE     ---       #274
      ---         BLOCKEND  ---      ---       LVL=0

      ---         MODULE    ---      ---       SIN7
      0100D03FH   PUBLIC    CONST    ---       sin90
      0100594FH   PUBLIC    CODE     ---       _cos7
      0100548EH   PUBLIC    CODE     ---       _sin7

      0100548EH   BLOCK     CODE     ---       LVL=0
      00000007H   SYMBOL    DATA     CHAR      angle
      0100548EH   BLOCK     CODE     NEAR LAB  LVL=1
      00000005H   SYMBOL    DATA     CHAR      v0
      00000006H   SYMBOL    DATA     CHAR      v1
      ---         BLOCKEND  ---      ---       LVL=1
      0100548EH   LINE      CODE     ---       #59
      0100548EH   LINE      CODE     ---       #60
      0100548EH   LINE      CODE     ---       #63
      01005496H   LINE      CODE     ---       #64
      0100549AH   LINE      CODE     ---       #65
      0100549BH   LINE      CODE     ---       #66
      0100549BH   LINE      CODE     ---       #68
      0100549DH   LINE      CODE     ---       #70
      010054A1H   LINE      CODE     ---       #71
      010054A4H   LINE      CODE     ---       #72
      010054A4H   LINE      CODE     ---       #73
      010054A6H   LINE      CODE     ---       #74
      010054A6H   LINE      CODE     ---       #75
      010054A6H   LINE      CODE     ---       #77
      010054A9H   LINE      CODE     ---       #79
      010054BDH   LINE      CODE     ---       #81
LX51 LINKER/LOCATER V4.66.30.0                                                        07/27/2019  23:22:19  PAGE 136


      010054C1H   LINE      CODE     ---       #82
      010054C5H   LINE      CODE     ---       #83
      010054C5H   LINE      CODE     ---       #85
      010054C7H   LINE      CODE     ---       #86
      ---         BLOCKEND  ---      ---       LVL=0

      0100594FH   BLOCK     CODE     ---       LVL=0
      00000007H   SYMBOL    DATA     CHAR      angle
      0100594FH   LINE      CODE     ---       #98
      0100594FH   LINE      CODE     ---       #99
      0100594FH   LINE      CODE     ---       #100
      01005957H   LINE      CODE     ---       #101
      0100595BH   LINE      CODE     ---       #102
      0100595CH   LINE      CODE     ---       #103
      0100595CH   LINE      CODE     ---       #105
      01005963H   LINE      CODE     ---       #106
      ---         BLOCKEND  ---      ---       LVL=0

      ---         MODULE    ---      ---       ADXL
      020004B2H   PUBLIC    XDATA    ---       adxl_smoothing
      020004ABH   PUBLIC    XDATA    ---       buf
      020004A5H   PUBLIC    XDATA    ---       adxl
      010057E7H   PUBLIC    CODE     ---       _adxl345_get_rotation
      01004B4BH   PUBLIC    CODE     ---       _adxl345_get_axes
      01004C87H   PUBLIC    CODE     ---       adxl345_tick
      0100535BH   PUBLIC    CODE     ---       adxl345_init
      000000A2H   SFRSYM    DATA     BYTE      SPI0CKR
      00000080H   SFRSYM    DATA     BYTE      P0
      000000D0H.2 SFRSYM    DATA     BIT       PSW_OV
      000000B1H   SFRSYM    DATA     BYTE      XOSC0CN
      00000090H   SFRSYM    DATA     BYTE      P1
      000000A0H   SFRSYM    DATA     BYTE      P2
      000000B0H   SFRSYM    DATA     BYTE      P3
      000000BCH   SFRSYM    DATA     BYTE      ADC0CF
      000000C8H   SFRSYM    DATA     BIT       TMR2CN0_T2XCLK
      000000C7H   SFRSYM    DATA     BYTE      P4
      000000C0H.7 SFRSYM    DATA     BIT       SMB0CN0_MASTER
      000000F9H   SFRSYM    DATA     WORD      PCA0
      000000E6H   SFRSYM    DATA     BYTE      EIE1
      000000C0H.7 SFRSYM    DATA     BIT       SMB1CN0_MASTER
      000000C0H.1 SFRSYM    DATA     BIT       SMB0CN0_ACK
      000000D7H   SFRSYM    DATA     BYTE      USB0XCN
      000000E7H   SFRSYM    DATA     BYTE      EIE2
      000000C0H.1 SFRSYM    DATA     BIT       SMB1CN0_ACK
      0000008FH   SFRSYM    DATA     BYTE      PSCTL
      000000E4H   SFRSYM    DATA     BYTE      IT01CF
      000000C8H   SFRSYM    DATA     BIT       TMR5CN0_T5XCLK
      000000C0H.6 SFRSYM    DATA     BIT       SMB0CN0_TXMODE
      000000C0H.6 SFRSYM    DATA     BIT       SMB1CN0_TXMODE
      000000BFH   SFRSYM    DATA     BYTE      SFRPAGE
      000000A4H   SFRSYM    DATA     BYTE      P0MDOUT
      000000A5H   SFRSYM    DATA     BYTE      P1MDOUT
      000000E8H.5 SFRSYM    DATA     BIT       ADC0CN0_ADINT
      000000CBH   SFRSYM    DATA     BYTE      TMR2RLH
      000000A6H   SFRSYM    DATA     BYTE      P2MDOUT
      000000A8H   SFRSYM    DATA     BYTE      IE
      00000093H   SFRSYM    DATA     BYTE      TMR3RLH
      000000A7H   SFRSYM    DATA     BYTE      P3MDOUT
      00000093H   SFRSYM    DATA     BYTE      TMR4RLH
      000000AEH   SFRSYM    DATA     BYTE      P4MDOUT
      000000F6H   SFRSYM    DATA     BYTE      EIP1
      000000CBH   SFRSYM    DATA     BYTE      TMR5RLH
LX51 LINKER/LOCATER V4.66.30.0                                                        07/27/2019  23:22:19  PAGE 137


      000000F7H   SFRSYM    DATA     BYTE      EIP2
      00000098H.2 SFRSYM    DATA     BIT       SCON0_RB8
      000000CAH   SFRSYM    DATA     BYTE      TMR2RLL
      000000FCH   SFRSYM    DATA     BYTE      PCA0CPH0
      00000092H   SFRSYM    DATA     BYTE      TMR3RLL
      000000EAH   SFRSYM    DATA     BYTE      PCA0CPH1
      00000098H.3 SFRSYM    DATA     BIT       SCON0_TB8
      000000F0H   SFRSYM    DATA     BIT       B_B0
      00000082H   SFRSYM    DATA     WORD      DP
      00000092H   SFRSYM    DATA     BYTE      TMR4RLL
      000000ECH   SFRSYM    DATA     BYTE      PCA0CPH2
      000000F0H.1 SFRSYM    DATA     BIT       B_B1
      000000C3H   SFRSYM    DATA     WORD      ADC0GT
      000000CAH   SFRSYM    DATA     BYTE      TMR5RLL
      000000EEH   SFRSYM    DATA     BYTE      PCA0CPH3
      000000F0H.2 SFRSYM    DATA     BIT       B_B2
      000000FBH   SFRSYM    DATA     BYTE      PCA0CPL0
      000000FEH   SFRSYM    DATA     BYTE      PCA0CPH4
      00000085H   SFRSYM    DATA     BYTE      EMI0CF
      000000F0H.3 SFRSYM    DATA     BIT       B_B3
      000000D9H   SFRSYM    DATA     BYTE      PCA0MD
      000000DAH   SFRSYM    DATA     BYTE      PCA0CPM0
      000000E9H   SFRSYM    DATA     BYTE      PCA0CPL1
      000000F0H.4 SFRSYM    DATA     BIT       B_B4
      000000DBH   SFRSYM    DATA     BYTE      PCA0CPM1
      000000EBH   SFRSYM    DATA     BYTE      PCA0CPL2
      000000F0H.5 SFRSYM    DATA     BIT       B_B5
      000000DCH   SFRSYM    DATA     BYTE      PCA0CPM2
      000000EDH   SFRSYM    DATA     BYTE      PCA0CPL3
      000000B8H   SFRSYM    DATA     BYTE      IP
      000000F0H.6 SFRSYM    DATA     BIT       B_B6
      000000C5H   SFRSYM    DATA     WORD      ADC0LT
      000000DDH   SFRSYM    DATA     BYTE      PCA0CPM3
      000000FDH   SFRSYM    DATA     BYTE      PCA0CPL4
      00000098H.5 SFRSYM    DATA     BIT       SCON0_MCE
      000000F0H.7 SFRSYM    DATA     BIT       B_B7
      000000DEH   SFRSYM    DATA     BYTE      PCA0CPM4
      000000E1H   SFRSYM    DATA     BYTE      XBR0
      000000C1H   SFRSYM    DATA     BYTE      SMB0CF
      000000E2H   SFRSYM    DATA     BYTE      XBR1
      000000C1H   SFRSYM    DATA     BYTE      SMB1CF
      000000AFH   SFRSYM    DATA     BYTE      PFE0CN
      000000AAH   SFRSYM    DATA     BYTE      EMI0CN
      000000C0H.5 SFRSYM    DATA     BIT       SMB0CN0_STA
      000000E3H   SFRSYM    DATA     BYTE      XBR2
      000000C0H.5 SFRSYM    DATA     BIT       SMB1CN0_STA
      000000E0H   SFRSYM    DATA     BIT       ACC_ACC0
      000000D1H   SFRSYM    DATA     BYTE      REF0CN
      000000B2H   SFRSYM    DATA     BYTE      HFO0CN
      0000008EH   SFRSYM    DATA     BYTE      CKCON0
      000000E0H.1 SFRSYM    DATA     BIT       ACC_ACC1
      000000E4H   SFRSYM    DATA     BYTE      CKCON1
      000000C8H.2 SFRSYM    DATA     BIT       TMR2CN0_TR2
      000000E0H.2 SFRSYM    DATA     BIT       ACC_ACC2
      000000E0H.3 SFRSYM    DATA     BIT       ACC_ACC3
      00000081H   SFRSYM    DATA     BYTE      SP
      0000009DH   SFRSYM    DATA     BYTE      CMP0MD
      000000E0H.4 SFRSYM    DATA     BIT       ACC_ACC4
      00000086H   SFRSYM    DATA     BYTE      LFO0CN
      00000084H   SFRSYM    DATA     BYTE      EMI0TC
      0000009CH   SFRSYM    DATA     BYTE      CMP1MD
      000000D8H   SFRSYM    DATA     BIT       PCA0CN0_CCF0
LX51 LINKER/LOCATER V4.66.30.0                                                        07/27/2019  23:22:19  PAGE 138


      000000E0H.5 SFRSYM    DATA     BIT       ACC_ACC5
      000000D8H.1 SFRSYM    DATA     BIT       PCA0CN0_CCF1
      000000E0H.6 SFRSYM    DATA     BIT       ACC_ACC6
      000000CCH   SFRSYM    DATA     WORD      TMR2
      000000D8H.2 SFRSYM    DATA     BIT       PCA0CN0_CCF2
      000000E0H.7 SFRSYM    DATA     BIT       ACC_ACC7
      00000094H   SFRSYM    DATA     WORD      TMR3
      000000C8H.2 SFRSYM    DATA     BIT       TMR5CN0_TR5
      000000D8H.3 SFRSYM    DATA     BIT       PCA0CN0_CCF3
      00000094H   SFRSYM    DATA     WORD      TMR4
      000000ACH   SFRSYM    DATA     BYTE      SBCON1
      000000D8H.4 SFRSYM    DATA     BIT       PCA0CN0_CCF4
      000000CCH   SFRSYM    DATA     WORD      TMR5
      000000C0H.3 SFRSYM    DATA     BIT       SMB0CN0_ACKRQ
      000000FFH   SFRSYM    DATA     BYTE      VDM0CN
      000000F1H   SFRSYM    DATA     BYTE      P0MDIN
      000000C0H.3 SFRSYM    DATA     BIT       SMB1CN0_ACKRQ
      00000098H.4 SFRSYM    DATA     BIT       SCON0_REN
      000000F2H   SFRSYM    DATA     BYTE      P1MDIN
      000000F3H   SFRSYM    DATA     BYTE      P2MDIN
      000000C0H.4 SFRSYM    DATA     BIT       SMB0CN0_STO
      000000F4H   SFRSYM    DATA     BYTE      P3MDIN
      000000C0H.4 SFRSYM    DATA     BIT       SMB1CN0_STO
      000000B5H   SFRSYM    DATA     BYTE      SBRLH1
      000000F5H   SFRSYM    DATA     BYTE      P4MDIN
      000000D0H.3 SFRSYM    DATA     BIT       PSW_RS0
      000000D8H.7 SFRSYM    DATA     BIT       PCA0CN0_CF
      000000F8H.4 SFRSYM    DATA     BIT       SPI0CN0_RXOVRN
      000000D0H.4 SFRSYM    DATA     BIT       PSW_RS1
      000000B4H   SFRSYM    DATA     BYTE      SBRLL1
      000000E8H.7 SFRSYM    DATA     BIT       ADC0CN0_ADEN
      00000089H   SFRSYM    DATA     BYTE      TMOD
      00000088H   SFRSYM    DATA     BYTE      TCON
      000000D0H   SFRSYM    DATA     BIT       PSW_PARITY
      000000A8H.4 SFRSYM    DATA     BIT       IE_ES0
      0000009FH   SFRSYM    DATA     BYTE      CMP0MX
      000000A8H.1 SFRSYM    DATA     BIT       IE_ET0
      0000009EH   SFRSYM    DATA     BYTE      CMP1MX
      000000A8H.3 SFRSYM    DATA     BIT       IE_ET1
      000000D4H   SFRSYM    DATA     BYTE      P0SKIP
      000000C8H.1 SFRSYM    DATA     BIT       TMR2CN0_T2CSS
      000000A8H.5 SFRSYM    DATA     BIT       IE_ET2
      000000D5H   SFRSYM    DATA     BYTE      P1SKIP
      000000D6H   SFRSYM    DATA     BYTE      P2SKIP
      000000E8H   SFRSYM    DATA     BYTE      ADC0CN0
      000000A8H   SFRSYM    DATA     BIT       IE_EX0
      000000DFH   SFRSYM    DATA     BYTE      P3SKIP
      000000D8H.6 SFRSYM    DATA     BIT       PCA0CN0_CR
      000000A8H.2 SFRSYM    DATA     BIT       IE_EX1
      00000098H.7 SFRSYM    DATA     BIT       SCON0_SMODE
      000000A9H   SFRSYM    DATA     BYTE      CLKSEL
      000000F8H   SFRSYM    DATA     BIT       SPI0CN0_SPIEN
      000000F0H   SFRSYM    DATA     BYTE      B
      000000BEH   SFRSYM    DATA     BYTE      ADC0H
      000000E8H.6 SFRSYM    DATA     BIT       ADC0CN0_ADTM
      000000CAH   SFRSYM    DATA     WORD      TMR2RL
      000000BDH   SFRSYM    DATA     BYTE      ADC0L
      00000092H   SFRSYM    DATA     WORD      TMR3RL
      00000092H   SFRSYM    DATA     WORD      TMR4RL
      000000D8H   SFRSYM    DATA     BYTE      PCA0CN0
      000000E0H   SFRSYM    DATA     BYTE      ACC
      000000CAH   SFRSYM    DATA     WORD      TMR5RL
LX51 LINKER/LOCATER V4.66.30.0                                                        07/27/2019  23:22:19  PAGE 139


      000000FBH   SFRSYM    DATA     WORD      PCA0CP0
      000000E9H   SFRSYM    DATA     WORD      PCA0CP1
      000000EBH   SFRSYM    DATA     WORD      PCA0CP2
      000000EDH   SFRSYM    DATA     WORD      PCA0CP3
      0000008CH   SFRSYM    DATA     BYTE      TH0
      000000B8H.4 SFRSYM    DATA     BIT       IP_PS0
      000000FDH   SFRSYM    DATA     WORD      PCA0CP4
      0000008DH   SFRSYM    DATA     BYTE      TH1
      000000FAH   SFRSYM    DATA     BYTE      PCA0H
      000000B8H.1 SFRSYM    DATA     BIT       IP_PT0
      000000B8H.3 SFRSYM    DATA     BIT       IP_PT1
      000000C0H.2 SFRSYM    DATA     BIT       SMB0CN0_ARBLOST
      000000B8H.5 SFRSYM    DATA     BIT       IP_PT2
      0000008AH   SFRSYM    DATA     BYTE      TL0
      000000F8H.1 SFRSYM    DATA     BIT       SPI0CN0_TXBMT
      000000C0H.2 SFRSYM    DATA     BIT       SMB1CN0_ARBLOST
      000000D0H.5 SFRSYM    DATA     BIT       PSW_F0
      000000A8H.6 SFRSYM    DATA     BIT       IE_ESPI0
      0000008BH   SFRSYM    DATA     BYTE      TL1
      000000F9H   SFRSYM    DATA     BYTE      PCA0L
      000000C0H   SFRSYM    DATA     BIT       SMB0CN0_SI
      000000D0H.1 SFRSYM    DATA     BIT       PSW_F1
      00000080H   SFRSYM    DATA     BIT       P0_B0
      000000B8H   SFRSYM    DATA     BIT       IP_PX0
      000000C9H   SFRSYM    DATA     BYTE      REG01CN
      000000C0H   SFRSYM    DATA     BIT       SMB1CN0_SI
      00000090H   SFRSYM    DATA     BIT       P1_B0
      00000080H.1 SFRSYM    DATA     BIT       P0_B1
      000000B8H.2 SFRSYM    DATA     BIT       IP_PX1
      0000009BH   SFRSYM    DATA     BYTE      CMP0CN0
      00000088H.1 SFRSYM    DATA     BIT       TCON_IE0
      000000A0H   SFRSYM    DATA     BIT       P2_B0
      00000090H.1 SFRSYM    DATA     BIT       P1_B1
      00000080H.2 SFRSYM    DATA     BIT       P0_B2
      0000009AH   SFRSYM    DATA     BYTE      CMP1CN0
      00000088H.3 SFRSYM    DATA     BIT       TCON_IE1
      000000B0H   SFRSYM    DATA     BIT       P3_B0
      000000A0H.1 SFRSYM    DATA     BIT       P2_B1
      00000090H.2 SFRSYM    DATA     BIT       P1_B2
      00000080H.3 SFRSYM    DATA     BIT       P0_B3
      000000C0H   SFRSYM    DATA     BYTE      SMB0CN0
      000000B0H.1 SFRSYM    DATA     BIT       P3_B1
      000000A0H.2 SFRSYM    DATA     BIT       P2_B2
      00000090H.3 SFRSYM    DATA     BIT       P1_B3
      00000080H.4 SFRSYM    DATA     BIT       P0_B4
      000000C0H   SFRSYM    DATA     BYTE      SMB1CN0
      000000B0H.2 SFRSYM    DATA     BIT       P3_B2
      000000A0H.3 SFRSYM    DATA     BIT       P2_B3
      00000090H.4 SFRSYM    DATA     BIT       P1_B4
      00000080H.5 SFRSYM    DATA     BIT       P0_B5
      000000B0H.3 SFRSYM    DATA     BIT       P3_B3
      000000A0H.4 SFRSYM    DATA     BIT       P2_B4
      00000090H.5 SFRSYM    DATA     BIT       P1_B5
      00000080H.6 SFRSYM    DATA     BIT       P0_B6
      000000B0H.4 SFRSYM    DATA     BIT       P3_B4
      000000A0H.5 SFRSYM    DATA     BIT       P2_B5
      00000090H.6 SFRSYM    DATA     BIT       P1_B6
      00000080H.7 SFRSYM    DATA     BIT       P0_B7
      000000B0H.5 SFRSYM    DATA     BIT       P3_B5
      000000A0H.6 SFRSYM    DATA     BIT       P2_B6
      00000090H.7 SFRSYM    DATA     BIT       P1_B7
      000000B0H.6 SFRSYM    DATA     BIT       P3_B6
LX51 LINKER/LOCATER V4.66.30.0                                                        07/27/2019  23:22:19  PAGE 140


      000000A0H.7 SFRSYM    DATA     BIT       P2_B7
      000000B0H.7 SFRSYM    DATA     BIT       P3_B7
      00000083H   SFRSYM    DATA     BYTE      DPH
      000000C4H   SFRSYM    DATA     BYTE      ADC0GTH
      000000C8H.7 SFRSYM    DATA     BIT       TMR2CN0_TF2H
      000000C8H.3 SFRSYM    DATA     BIT       TMR2CN0_T2SPLIT
      000000D0H.6 SFRSYM    DATA     BIT       PSW_AC
      000000F8H   SFRSYM    DATA     BYTE      SPI0CN0
      000000B3H   SFRSYM    DATA     BYTE      HFO0CAL
      00000088H.5 SFRSYM    DATA     BIT       TCON_TF0
      00000098H   SFRSYM    DATA     BIT       SCON0_RI
      00000082H   SFRSYM    DATA     BYTE      DPL
      00000088H.7 SFRSYM    DATA     BIT       TCON_TF1
      00000099H   SFRSYM    DATA     BYTE      SBUF0
      00000087H   SFRSYM    DATA     BYTE      PCON0
      000000C3H   SFRSYM    DATA     BYTE      ADC0GTL
      000000C8H.6 SFRSYM    DATA     BIT       TMR2CN0_TF2L
      00000098H.1 SFRSYM    DATA     BIT       SCON0_TI
      000000E8H   SFRSYM    DATA     BIT       ADC0CN0_ADCM0
      000000D3H   SFRSYM    DATA     BYTE      SBUF1
      000000C6H   SFRSYM    DATA     BYTE      ADC0LTH
      00000088H   SFRSYM    DATA     BIT       TCON_IT0
      000000E8H.1 SFRSYM    DATA     BIT       ADC0CN0_ADCM1
      000000EFH   SFRSYM    DATA     BYTE      RSTSRC
      000000C8H.7 SFRSYM    DATA     BIT       TMR5CN0_TF5H
      000000C8H.3 SFRSYM    DATA     BIT       TMR5CN0_T5SPLIT
      00000088H.2 SFRSYM    DATA     BIT       TCON_IT1
      000000E8H.2 SFRSYM    DATA     BIT       ADC0CN0_ADCM2
      00000098H   SFRSYM    DATA     BYTE      SCON0
      000000E8H.3 SFRSYM    DATA     BIT       ADC0CN0_ADWINT
      000000B4H   SFRSYM    DATA     WORD      SBRL1
      000000E5H   SFRSYM    DATA     BYTE      SMOD1
      000000D2H   SFRSYM    DATA     BYTE      SCON1
      000000BAH   SFRSYM    DATA     BYTE      AMX0N
      000000E8H.4 SFRSYM    DATA     BIT       ADC0CN0_ADBUSY
      000000CEH   SFRSYM    DATA     BYTE      SMB0ADM
      000000C5H   SFRSYM    DATA     BYTE      ADC0LTL
      000000F8H.5 SFRSYM    DATA     BIT       SPI0CN0_MODF
      000000B8H.6 SFRSYM    DATA     BIT       IP_PSPI0
      000000CEH   SFRSYM    DATA     BYTE      SMB1ADM
      000000BBH   SFRSYM    DATA     BYTE      AMX0P
      000000C8H.6 SFRSYM    DATA     BIT       TMR5CN0_TF5L
      000000C8H   SFRSYM    DATA     BYTE      TMR2CN0
      00000091H   SFRSYM    DATA     BYTE      TMR3CN0
      00000091H   SFRSYM    DATA     BYTE      TMR4CN0
      000000C8H   SFRSYM    DATA     BYTE      TMR5CN0
      000000CFH   SFRSYM    DATA     BYTE      SMB0ADR
      00000088H.4 SFRSYM    DATA     BIT       TCON_TR0
      000000CFH   SFRSYM    DATA     BYTE      SMB1ADR
      000000C8H.4 SFRSYM    DATA     BIT       TMR2CN0_TF2CEN
      00000088H.6 SFRSYM    DATA     BIT       TCON_TR1
      000000C2H   SFRSYM    DATA     BYTE      SMB0DAT
      000000CDH   SFRSYM    DATA     BYTE      TMR2H
      000000A1H   SFRSYM    DATA     BYTE      SPI0CFG
      000000C2H   SFRSYM    DATA     BYTE      SMB1DAT
      00000095H   SFRSYM    DATA     BYTE      TMR3H
      00000095H   SFRSYM    DATA     BYTE      TMR4H
      000000CDH   SFRSYM    DATA     BYTE      TMR5H
      000000CCH   SFRSYM    DATA     BYTE      TMR2L
      000000F8H.7 SFRSYM    DATA     BIT       SPI0CN0_SPIF
      00000096H   SFRSYM    DATA     BYTE      USB0ADR
      00000094H   SFRSYM    DATA     BYTE      TMR3L
LX51 LINKER/LOCATER V4.66.30.0                                                        07/27/2019  23:22:19  PAGE 141


      000000A8H.7 SFRSYM    DATA     BIT       IE_EA
      00000094H   SFRSYM    DATA     BYTE      TMR4L
      00000097H   SFRSYM    DATA     BYTE      USB0DAT
      000000CCH   SFRSYM    DATA     BYTE      TMR5L
      000000B6H   SFRSYM    DATA     BYTE      FLSCL
      000000C8H.5 SFRSYM    DATA     BIT       TMR2CN0_TF2LEN
      000000F8H.6 SFRSYM    DATA     BIT       SPI0CN0_WCOL
      000000F8H.2 SFRSYM    DATA     BIT       SPI0CN0_NSSMD0
      000000D0H.7 SFRSYM    DATA     BIT       PSW_CY
      000000A3H   SFRSYM    DATA     BYTE      SPI0DAT
      000000F8H.3 SFRSYM    DATA     BIT       SPI0CN0_NSSMD1
      000000BDH   SFRSYM    DATA     WORD      ADC0
      000000B9H   SFRSYM    DATA     BYTE      SMBTC
      000000D0H   SFRSYM    DATA     BYTE      PSW
      000000C8H.5 SFRSYM    DATA     BIT       TMR5CN0_TF5LEN
      000000B7H   SFRSYM    DATA     BYTE      FLKEY

      0100535BH   BLOCK     CODE     ---       LVL=0
      0100535BH   LINE      CODE     ---       #18
      0100535BH   LINE      CODE     ---       #19
      0100535BH   LINE      CODE     ---       #20
      01005361H   LINE      CODE     ---       #21
      01005365H   LINE      CODE     ---       #22
      01005369H   LINE      CODE     ---       #23
      0100537EH   LINE      CODE     ---       #25
      01005384H   LINE      CODE     ---       #26
      01005388H   LINE      CODE     ---       #27
      ---         BLOCKEND  ---      ---       LVL=0

      01004C87H   BLOCK     CODE     ---       LVL=0
      01004C87H   LINE      CODE     ---       #30
      01004C87H   LINE      CODE     ---       #31
      01004C87H   LINE      CODE     ---       #32
      01004C90H   LINE      CODE     ---       #33
      01004CADH   LINE      CODE     ---       #34
      01004CCAH   LINE      CODE     ---       #35
      01004CE7H   LINE      CODE     ---       #36
      ---         BLOCKEND  ---      ---       LVL=0

      01004B4BH   BLOCK     CODE     ---       LVL=0
      00000043H   SYMBOL    DATA     ---       adxl
      01004B4BH   LINE      CODE     ---       #38
      01004B51H   LINE      CODE     ---       #39
      01004B51H   LINE      CODE     ---       #40
      01004B57H   LINE      CODE     ---       #41
      01004B66H   LINE      CODE     ---       #42
      01004B7BH   LINE      CODE     ---       #44
      01004B93H   LINE      CODE     ---       #45
      01004BAEH   LINE      CODE     ---       #46
      ---         BLOCKEND  ---      ---       LVL=0

      010057E7H   BLOCK     CODE     ---       LVL=0
      00000001H   SYMBOL    DATA     ---       adxl
      010057E7H   BLOCK     CODE     NEAR LAB  LVL=1
      00000005H   SYMBOL    DATA     CHAR      nx
      00000007H   SYMBOL    DATA     CHAR      ny
      00000007H   SYMBOL    DATA     CHAR      ret
      ---         BLOCKEND  ---      ---       LVL=1
      010057E7H   LINE      CODE     ---       #49
      010057E7H   LINE      CODE     ---       #50
      010057E7H   LINE      CODE     ---       #53
      010057EDH   LINE      CODE     ---       #54
LX51 LINKER/LOCATER V4.66.30.0                                                        07/27/2019  23:22:19  PAGE 142


      010057F4H   LINE      CODE     ---       #56
      010057FCH   LINE      CODE     ---       #57
      01005803H   LINE      CODE     ---       #58
      01005807H   LINE      CODE     ---       #59
      01005807H   LINE      CODE     ---       #61
      01005807H   LINE      CODE     ---       #62
      ---         BLOCKEND  ---      ---       LVL=0
      00000007H   SYMBOL    DATA     BYTE      interrupt_flags

      ---         MODULE    ---      ---       LIGHTLEVEL
      0000008BH   PUBLIC    IDATA    BYTE      lsens_timeout
      01005A01H   PUBLIC    CODE     ---       lsens_tick
      01005866H   PUBLIC    CODE     ---       _lsens_pulse
      000000A2H   SFRSYM    DATA     BYTE      SPI0CKR
      00000080H   SFRSYM    DATA     BYTE      P0
      000000D0H.2 SFRSYM    DATA     BIT       PSW_OV
      000000B1H   SFRSYM    DATA     BYTE      XOSC0CN
      00000090H   SFRSYM    DATA     BYTE      P1
      000000A0H   SFRSYM    DATA     BYTE      P2
      000000B0H   SFRSYM    DATA     BYTE      P3
      000000BCH   SFRSYM    DATA     BYTE      ADC0CF
      000000C8H   SFRSYM    DATA     BIT       TMR2CN0_T2XCLK
      000000C7H   SFRSYM    DATA     BYTE      P4
      000000C0H.7 SFRSYM    DATA     BIT       SMB0CN0_MASTER
      000000F9H   SFRSYM    DATA     WORD      PCA0
      000000E6H   SFRSYM    DATA     BYTE      EIE1
      000000C0H.7 SFRSYM    DATA     BIT       SMB1CN0_MASTER
      000000C0H.1 SFRSYM    DATA     BIT       SMB0CN0_ACK
      000000D7H   SFRSYM    DATA     BYTE      USB0XCN
      000000E7H   SFRSYM    DATA     BYTE      EIE2
      000000C0H.1 SFRSYM    DATA     BIT       SMB1CN0_ACK
      0000008FH   SFRSYM    DATA     BYTE      PSCTL
      000000E4H   SFRSYM    DATA     BYTE      IT01CF
      000000C8H   SFRSYM    DATA     BIT       TMR5CN0_T5XCLK
      000000C0H.6 SFRSYM    DATA     BIT       SMB0CN0_TXMODE
      000000C0H.6 SFRSYM    DATA     BIT       SMB1CN0_TXMODE
      000000BFH   SFRSYM    DATA     BYTE      SFRPAGE
      000000A4H   SFRSYM    DATA     BYTE      P0MDOUT
      000000A5H   SFRSYM    DATA     BYTE      P1MDOUT
      000000E8H.5 SFRSYM    DATA     BIT       ADC0CN0_ADINT
      000000CBH   SFRSYM    DATA     BYTE      TMR2RLH
      000000A6H   SFRSYM    DATA     BYTE      P2MDOUT
      000000A8H   SFRSYM    DATA     BYTE      IE
      00000093H   SFRSYM    DATA     BYTE      TMR3RLH
      000000A7H   SFRSYM    DATA     BYTE      P3MDOUT
      00000093H   SFRSYM    DATA     BYTE      TMR4RLH
      000000AEH   SFRSYM    DATA     BYTE      P4MDOUT
      000000F6H   SFRSYM    DATA     BYTE      EIP1
      000000CBH   SFRSYM    DATA     BYTE      TMR5RLH
      000000F7H   SFRSYM    DATA     BYTE      EIP2
      00000098H.2 SFRSYM    DATA     BIT       SCON0_RB8
      000000CAH   SFRSYM    DATA     BYTE      TMR2RLL
      000000FCH   SFRSYM    DATA     BYTE      PCA0CPH0
      00000092H   SFRSYM    DATA     BYTE      TMR3RLL
      000000EAH   SFRSYM    DATA     BYTE      PCA0CPH1
      00000098H.3 SFRSYM    DATA     BIT       SCON0_TB8
      000000F0H   SFRSYM    DATA     BIT       B_B0
      00000082H   SFRSYM    DATA     WORD      DP
      00000092H   SFRSYM    DATA     BYTE      TMR4RLL
      000000ECH   SFRSYM    DATA     BYTE      PCA0CPH2
      000000F0H.1 SFRSYM    DATA     BIT       B_B1
      000000C3H   SFRSYM    DATA     WORD      ADC0GT
LX51 LINKER/LOCATER V4.66.30.0                                                        07/27/2019  23:22:19  PAGE 143


      000000CAH   SFRSYM    DATA     BYTE      TMR5RLL
      000000EEH   SFRSYM    DATA     BYTE      PCA0CPH3
      000000F0H.2 SFRSYM    DATA     BIT       B_B2
      000000FBH   SFRSYM    DATA     BYTE      PCA0CPL0
      000000FEH   SFRSYM    DATA     BYTE      PCA0CPH4
      00000085H   SFRSYM    DATA     BYTE      EMI0CF
      000000F0H.3 SFRSYM    DATA     BIT       B_B3
      000000D9H   SFRSYM    DATA     BYTE      PCA0MD
      000000DAH   SFRSYM    DATA     BYTE      PCA0CPM0
      000000E9H   SFRSYM    DATA     BYTE      PCA0CPL1
      000000F0H.4 SFRSYM    DATA     BIT       B_B4
      000000DBH   SFRSYM    DATA     BYTE      PCA0CPM1
      000000EBH   SFRSYM    DATA     BYTE      PCA0CPL2
      000000F0H.5 SFRSYM    DATA     BIT       B_B5
      000000DCH   SFRSYM    DATA     BYTE      PCA0CPM2
      000000EDH   SFRSYM    DATA     BYTE      PCA0CPL3
      000000B8H   SFRSYM    DATA     BYTE      IP
      000000F0H.6 SFRSYM    DATA     BIT       B_B6
      000000C5H   SFRSYM    DATA     WORD      ADC0LT
      000000DDH   SFRSYM    DATA     BYTE      PCA0CPM3
      000000FDH   SFRSYM    DATA     BYTE      PCA0CPL4
      00000098H.5 SFRSYM    DATA     BIT       SCON0_MCE
      000000F0H.7 SFRSYM    DATA     BIT       B_B7
      000000DEH   SFRSYM    DATA     BYTE      PCA0CPM4
      000000E1H   SFRSYM    DATA     BYTE      XBR0
      000000C1H   SFRSYM    DATA     BYTE      SMB0CF
      000000E2H   SFRSYM    DATA     BYTE      XBR1
      000000C1H   SFRSYM    DATA     BYTE      SMB1CF
      000000AFH   SFRSYM    DATA     BYTE      PFE0CN
      000000AAH   SFRSYM    DATA     BYTE      EMI0CN
      000000C0H.5 SFRSYM    DATA     BIT       SMB0CN0_STA
      000000E3H   SFRSYM    DATA     BYTE      XBR2
      000000C0H.5 SFRSYM    DATA     BIT       SMB1CN0_STA
      000000E0H   SFRSYM    DATA     BIT       ACC_ACC0
      000000D1H   SFRSYM    DATA     BYTE      REF0CN
      000000B2H   SFRSYM    DATA     BYTE      HFO0CN
      0000008EH   SFRSYM    DATA     BYTE      CKCON0
      000000E0H.1 SFRSYM    DATA     BIT       ACC_ACC1
      000000E4H   SFRSYM    DATA     BYTE      CKCON1
      000000C8H.2 SFRSYM    DATA     BIT       TMR2CN0_TR2
      000000E0H.2 SFRSYM    DATA     BIT       ACC_ACC2
      000000E0H.3 SFRSYM    DATA     BIT       ACC_ACC3
      00000081H   SFRSYM    DATA     BYTE      SP
      0000009DH   SFRSYM    DATA     BYTE      CMP0MD
      000000E0H.4 SFRSYM    DATA     BIT       ACC_ACC4
      00000086H   SFRSYM    DATA     BYTE      LFO0CN
      00000084H   SFRSYM    DATA     BYTE      EMI0TC
      0000009CH   SFRSYM    DATA     BYTE      CMP1MD
      000000D8H   SFRSYM    DATA     BIT       PCA0CN0_CCF0
      000000E0H.5 SFRSYM    DATA     BIT       ACC_ACC5
      000000D8H.1 SFRSYM    DATA     BIT       PCA0CN0_CCF1
      000000E0H.6 SFRSYM    DATA     BIT       ACC_ACC6
      000000CCH   SFRSYM    DATA     WORD      TMR2
      000000D8H.2 SFRSYM    DATA     BIT       PCA0CN0_CCF2
      000000E0H.7 SFRSYM    DATA     BIT       ACC_ACC7
      00000094H   SFRSYM    DATA     WORD      TMR3
      000000C8H.2 SFRSYM    DATA     BIT       TMR5CN0_TR5
      000000D8H.3 SFRSYM    DATA     BIT       PCA0CN0_CCF3
      00000094H   SFRSYM    DATA     WORD      TMR4
      000000ACH   SFRSYM    DATA     BYTE      SBCON1
      000000D8H.4 SFRSYM    DATA     BIT       PCA0CN0_CCF4
      000000CCH   SFRSYM    DATA     WORD      TMR5
LX51 LINKER/LOCATER V4.66.30.0                                                        07/27/2019  23:22:19  PAGE 144


      000000C0H.3 SFRSYM    DATA     BIT       SMB0CN0_ACKRQ
      000000FFH   SFRSYM    DATA     BYTE      VDM0CN
      000000F1H   SFRSYM    DATA     BYTE      P0MDIN
      000000C0H.3 SFRSYM    DATA     BIT       SMB1CN0_ACKRQ
      00000098H.4 SFRSYM    DATA     BIT       SCON0_REN
      000000F2H   SFRSYM    DATA     BYTE      P1MDIN
      000000F3H   SFRSYM    DATA     BYTE      P2MDIN
      000000C0H.4 SFRSYM    DATA     BIT       SMB0CN0_STO
      000000F4H   SFRSYM    DATA     BYTE      P3MDIN
      000000C0H.4 SFRSYM    DATA     BIT       SMB1CN0_STO
      000000B5H   SFRSYM    DATA     BYTE      SBRLH1
      000000F5H   SFRSYM    DATA     BYTE      P4MDIN
      000000D0H.3 SFRSYM    DATA     BIT       PSW_RS0
      000000D8H.7 SFRSYM    DATA     BIT       PCA0CN0_CF
      000000F8H.4 SFRSYM    DATA     BIT       SPI0CN0_RXOVRN
      000000D0H.4 SFRSYM    DATA     BIT       PSW_RS1
      000000B4H   SFRSYM    DATA     BYTE      SBRLL1
      000000E8H.7 SFRSYM    DATA     BIT       ADC0CN0_ADEN
      00000089H   SFRSYM    DATA     BYTE      TMOD
      00000088H   SFRSYM    DATA     BYTE      TCON
      000000D0H   SFRSYM    DATA     BIT       PSW_PARITY
      000000A8H.4 SFRSYM    DATA     BIT       IE_ES0
      0000009FH   SFRSYM    DATA     BYTE      CMP0MX
      000000A8H.1 SFRSYM    DATA     BIT       IE_ET0
      0000009EH   SFRSYM    DATA     BYTE      CMP1MX
      000000A8H.3 SFRSYM    DATA     BIT       IE_ET1
      000000D4H   SFRSYM    DATA     BYTE      P0SKIP
      000000C8H.1 SFRSYM    DATA     BIT       TMR2CN0_T2CSS
      000000A8H.5 SFRSYM    DATA     BIT       IE_ET2
      000000D5H   SFRSYM    DATA     BYTE      P1SKIP
      000000D6H   SFRSYM    DATA     BYTE      P2SKIP
      000000E8H   SFRSYM    DATA     BYTE      ADC0CN0
      000000A8H   SFRSYM    DATA     BIT       IE_EX0
      000000DFH   SFRSYM    DATA     BYTE      P3SKIP
      000000D8H.6 SFRSYM    DATA     BIT       PCA0CN0_CR
      000000A8H.2 SFRSYM    DATA     BIT       IE_EX1
      00000098H.7 SFRSYM    DATA     BIT       SCON0_SMODE
      000000A9H   SFRSYM    DATA     BYTE      CLKSEL
      000000F8H   SFRSYM    DATA     BIT       SPI0CN0_SPIEN
      000000F0H   SFRSYM    DATA     BYTE      B
      000000BEH   SFRSYM    DATA     BYTE      ADC0H
      000000E8H.6 SFRSYM    DATA     BIT       ADC0CN0_ADTM
      000000CAH   SFRSYM    DATA     WORD      TMR2RL
      000000BDH   SFRSYM    DATA     BYTE      ADC0L
      00000092H   SFRSYM    DATA     WORD      TMR3RL
      00000092H   SFRSYM    DATA     WORD      TMR4RL
      000000D8H   SFRSYM    DATA     BYTE      PCA0CN0
      000000E0H   SFRSYM    DATA     BYTE      ACC
      000000CAH   SFRSYM    DATA     WORD      TMR5RL
      000000FBH   SFRSYM    DATA     WORD      PCA0CP0
      000000E9H   SFRSYM    DATA     WORD      PCA0CP1
      000000EBH   SFRSYM    DATA     WORD      PCA0CP2
      000000EDH   SFRSYM    DATA     WORD      PCA0CP3
      0000008CH   SFRSYM    DATA     BYTE      TH0
      000000B8H.4 SFRSYM    DATA     BIT       IP_PS0
      000000FDH   SFRSYM    DATA     WORD      PCA0CP4
      0000008DH   SFRSYM    DATA     BYTE      TH1
      000000FAH   SFRSYM    DATA     BYTE      PCA0H
      000000B8H.1 SFRSYM    DATA     BIT       IP_PT0
      000000B8H.3 SFRSYM    DATA     BIT       IP_PT1
      000000C0H.2 SFRSYM    DATA     BIT       SMB0CN0_ARBLOST
      000000B8H.5 SFRSYM    DATA     BIT       IP_PT2
LX51 LINKER/LOCATER V4.66.30.0                                                        07/27/2019  23:22:19  PAGE 145


      0000008AH   SFRSYM    DATA     BYTE      TL0
      000000F8H.1 SFRSYM    DATA     BIT       SPI0CN0_TXBMT
      000000C0H.2 SFRSYM    DATA     BIT       SMB1CN0_ARBLOST
      000000D0H.5 SFRSYM    DATA     BIT       PSW_F0
      000000A8H.6 SFRSYM    DATA     BIT       IE_ESPI0
      0000008BH   SFRSYM    DATA     BYTE      TL1
      000000F9H   SFRSYM    DATA     BYTE      PCA0L
      000000C0H   SFRSYM    DATA     BIT       SMB0CN0_SI
      000000D0H.1 SFRSYM    DATA     BIT       PSW_F1
      00000080H   SFRSYM    DATA     BIT       P0_B0
      000000B8H   SFRSYM    DATA     BIT       IP_PX0
      000000C9H   SFRSYM    DATA     BYTE      REG01CN
      000000C0H   SFRSYM    DATA     BIT       SMB1CN0_SI
      00000090H   SFRSYM    DATA     BIT       P1_B0
      00000080H.1 SFRSYM    DATA     BIT       P0_B1
      000000B8H.2 SFRSYM    DATA     BIT       IP_PX1
      0000009BH   SFRSYM    DATA     BYTE      CMP0CN0
      00000088H.1 SFRSYM    DATA     BIT       TCON_IE0
      000000A0H   SFRSYM    DATA     BIT       P2_B0
      00000090H.1 SFRSYM    DATA     BIT       P1_B1
      00000080H.2 SFRSYM    DATA     BIT       P0_B2
      0000009AH   SFRSYM    DATA     BYTE      CMP1CN0
      00000088H.3 SFRSYM    DATA     BIT       TCON_IE1
      000000B0H   SFRSYM    DATA     BIT       P3_B0
      000000A0H.1 SFRSYM    DATA     BIT       P2_B1
      00000090H.2 SFRSYM    DATA     BIT       P1_B2
      00000080H.3 SFRSYM    DATA     BIT       P0_B3
      000000C0H   SFRSYM    DATA     BYTE      SMB0CN0
      000000B0H.1 SFRSYM    DATA     BIT       P3_B1
      000000A0H.2 SFRSYM    DATA     BIT       P2_B2
      00000090H.3 SFRSYM    DATA     BIT       P1_B3
      00000080H.4 SFRSYM    DATA     BIT       P0_B4
      000000C0H   SFRSYM    DATA     BYTE      SMB1CN0
      000000B0H.2 SFRSYM    DATA     BIT       P3_B2
      000000A0H.3 SFRSYM    DATA     BIT       P2_B3
      00000090H.4 SFRSYM    DATA     BIT       P1_B4
      00000080H.5 SFRSYM    DATA     BIT       P0_B5
      000000B0H.3 SFRSYM    DATA     BIT       P3_B3
      000000A0H.4 SFRSYM    DATA     BIT       P2_B4
      00000090H.5 SFRSYM    DATA     BIT       P1_B5
      00000080H.6 SFRSYM    DATA     BIT       P0_B6
      000000B0H.4 SFRSYM    DATA     BIT       P3_B4
      000000A0H.5 SFRSYM    DATA     BIT       P2_B5
      00000090H.6 SFRSYM    DATA     BIT       P1_B6
      00000080H.7 SFRSYM    DATA     BIT       P0_B7
      000000B0H.5 SFRSYM    DATA     BIT       P3_B5
      000000A0H.6 SFRSYM    DATA     BIT       P2_B6
      00000090H.7 SFRSYM    DATA     BIT       P1_B7
      000000B0H.6 SFRSYM    DATA     BIT       P3_B6
      000000A0H.7 SFRSYM    DATA     BIT       P2_B7
      000000B0H.7 SFRSYM    DATA     BIT       P3_B7
      00000083H   SFRSYM    DATA     BYTE      DPH
      000000C4H   SFRSYM    DATA     BYTE      ADC0GTH
      000000C8H.7 SFRSYM    DATA     BIT       TMR2CN0_TF2H
      000000C8H.3 SFRSYM    DATA     BIT       TMR2CN0_T2SPLIT
      000000D0H.6 SFRSYM    DATA     BIT       PSW_AC
      000000F8H   SFRSYM    DATA     BYTE      SPI0CN0
      000000B3H   SFRSYM    DATA     BYTE      HFO0CAL
      00000088H.5 SFRSYM    DATA     BIT       TCON_TF0
      00000098H   SFRSYM    DATA     BIT       SCON0_RI
      00000082H   SFRSYM    DATA     BYTE      DPL
      00000088H.7 SFRSYM    DATA     BIT       TCON_TF1
LX51 LINKER/LOCATER V4.66.30.0                                                        07/27/2019  23:22:19  PAGE 146


      00000099H   SFRSYM    DATA     BYTE      SBUF0
      00000087H   SFRSYM    DATA     BYTE      PCON0
      000000C3H   SFRSYM    DATA     BYTE      ADC0GTL
      000000C8H.6 SFRSYM    DATA     BIT       TMR2CN0_TF2L
      00000098H.1 SFRSYM    DATA     BIT       SCON0_TI
      000000E8H   SFRSYM    DATA     BIT       ADC0CN0_ADCM0
      000000D3H   SFRSYM    DATA     BYTE      SBUF1
      000000C6H   SFRSYM    DATA     BYTE      ADC0LTH
      00000088H   SFRSYM    DATA     BIT       TCON_IT0
      000000E8H.1 SFRSYM    DATA     BIT       ADC0CN0_ADCM1
      000000EFH   SFRSYM    DATA     BYTE      RSTSRC
      000000C8H.7 SFRSYM    DATA     BIT       TMR5CN0_TF5H
      000000C8H.3 SFRSYM    DATA     BIT       TMR5CN0_T5SPLIT
      00000088H.2 SFRSYM    DATA     BIT       TCON_IT1
      000000E8H.2 SFRSYM    DATA     BIT       ADC0CN0_ADCM2
      00000098H   SFRSYM    DATA     BYTE      SCON0
      000000E8H.3 SFRSYM    DATA     BIT       ADC0CN0_ADWINT
      000000B4H   SFRSYM    DATA     WORD      SBRL1
      000000E5H   SFRSYM    DATA     BYTE      SMOD1
      000000D2H   SFRSYM    DATA     BYTE      SCON1
      000000BAH   SFRSYM    DATA     BYTE      AMX0N
      000000E8H.4 SFRSYM    DATA     BIT       ADC0CN0_ADBUSY
      000000CEH   SFRSYM    DATA     BYTE      SMB0ADM
      000000C5H   SFRSYM    DATA     BYTE      ADC0LTL
      000000F8H.5 SFRSYM    DATA     BIT       SPI0CN0_MODF
      000000B8H.6 SFRSYM    DATA     BIT       IP_PSPI0
      000000CEH   SFRSYM    DATA     BYTE      SMB1ADM
      000000BBH   SFRSYM    DATA     BYTE      AMX0P
      000000C8H.6 SFRSYM    DATA     BIT       TMR5CN0_TF5L
      000000C8H   SFRSYM    DATA     BYTE      TMR2CN0
      00000091H   SFRSYM    DATA     BYTE      TMR3CN0
      00000091H   SFRSYM    DATA     BYTE      TMR4CN0
      000000C8H   SFRSYM    DATA     BYTE      TMR5CN0
      000000CFH   SFRSYM    DATA     BYTE      SMB0ADR
      00000088H.4 SFRSYM    DATA     BIT       TCON_TR0
      000000CFH   SFRSYM    DATA     BYTE      SMB1ADR
      000000C8H.4 SFRSYM    DATA     BIT       TMR2CN0_TF2CEN
      00000088H.6 SFRSYM    DATA     BIT       TCON_TR1
      000000C2H   SFRSYM    DATA     BYTE      SMB0DAT
      000000CDH   SFRSYM    DATA     BYTE      TMR2H
      000000A1H   SFRSYM    DATA     BYTE      SPI0CFG
      000000C2H   SFRSYM    DATA     BYTE      SMB1DAT
      00000095H   SFRSYM    DATA     BYTE      TMR3H
      00000095H   SFRSYM    DATA     BYTE      TMR4H
      000000CDH   SFRSYM    DATA     BYTE      TMR5H
      000000CCH   SFRSYM    DATA     BYTE      TMR2L
      000000F8H.7 SFRSYM    DATA     BIT       SPI0CN0_SPIF
      00000096H   SFRSYM    DATA     BYTE      USB0ADR
      00000094H   SFRSYM    DATA     BYTE      TMR3L
      000000A8H.7 SFRSYM    DATA     BIT       IE_EA
      00000094H   SFRSYM    DATA     BYTE      TMR4L
      00000097H   SFRSYM    DATA     BYTE      USB0DAT
      000000CCH   SFRSYM    DATA     BYTE      TMR5L
      000000B6H   SFRSYM    DATA     BYTE      FLSCL
      000000C8H.5 SFRSYM    DATA     BIT       TMR2CN0_TF2LEN
      000000F8H.6 SFRSYM    DATA     BIT       SPI0CN0_WCOL
      000000F8H.2 SFRSYM    DATA     BIT       SPI0CN0_NSSMD0
      000000D0H.7 SFRSYM    DATA     BIT       PSW_CY
      000000A3H   SFRSYM    DATA     BYTE      SPI0DAT
      000000F8H.3 SFRSYM    DATA     BIT       SPI0CN0_NSSMD1
      000000BDH   SFRSYM    DATA     WORD      ADC0
      000000B9H   SFRSYM    DATA     BYTE      SMBTC
LX51 LINKER/LOCATER V4.66.30.0                                                        07/27/2019  23:22:19  PAGE 147


      000000D0H   SFRSYM    DATA     BYTE      PSW
      000000C8H.5 SFRSYM    DATA     BIT       TMR5CN0_TF5LEN
      000000B7H   SFRSYM    DATA     BYTE      FLKEY

      01005866H   BLOCK     CODE     ---       LVL=0
      00000007H   SYMBOL    DATA     BYTE      cnt
      01005866H   LINE      CODE     ---       #14
      01005866H   LINE      CODE     ---       #15
      01005866H   LINE      CODE     ---       #20
      01005868H   LINE      CODE     ---       #21
      0100586AH   LINE      CODE     ---       #22
      0100586DH   LINE      CODE     ---       #23
      01005870H   LINE      CODE     ---       #24
      01005873H   LINE      CODE     ---       #26
      01005877H   LINE      CODE     ---       #28
      01005877H   LINE      CODE     ---       #31
      0100587AH   LINE      CODE     ---       #32
      0100587DH   LINE      CODE     ---       #33
      0100587FH   LINE      CODE     ---       #37
      01005883H   LINE      CODE     ---       #38
      ---         BLOCKEND  ---      ---       LVL=0

      01005A01H   BLOCK     CODE     ---       LVL=0
      01005A01H   LINE      CODE     ---       #45
      01005A01H   LINE      CODE     ---       #46
      01005A01H   LINE      CODE     ---       #47
      01005A06H   LINE      CODE     ---       #48
      01005A07H   LINE      CODE     ---       #49
      01005A0AH   LINE      CODE     ---       #51
      01005A0CH   LINE      CODE     ---       #54
      01005A0FH   LINE      CODE     ---       #55
      01005A12H   LINE      CODE     ---       #56
      01005A12H   LINE      CODE     ---       #57
      01005A12H   LINE      CODE     ---       #58
      ---         BLOCKEND  ---      ---       LVL=0

      ---         MODULE    ---      ---       BTN
      02000461H   PUBLIC    XDATA    ---       btn
      010029F8H   PUBLIC    CODE     ---       btn_callback
      01003072H   PUBLIC    CODE     ---       btn_tick
      0100483CH   PUBLIC    CODE     ---       btn_init
      000000A2H   SFRSYM    DATA     BYTE      SPI0CKR
      00000080H   SFRSYM    DATA     BYTE      P0
      000000D0H.2 SFRSYM    DATA     BIT       PSW_OV
      000000B1H   SFRSYM    DATA     BYTE      XOSC0CN
      00000090H   SFRSYM    DATA     BYTE      P1
      000000A0H   SFRSYM    DATA     BYTE      P2
      000000B0H   SFRSYM    DATA     BYTE      P3
      000000BCH   SFRSYM    DATA     BYTE      ADC0CF
      000000C8H   SFRSYM    DATA     BIT       TMR2CN0_T2XCLK
      000000C7H   SFRSYM    DATA     BYTE      P4
      000000C0H.7 SFRSYM    DATA     BIT       SMB0CN0_MASTER
      000000F9H   SFRSYM    DATA     WORD      PCA0
      000000E6H   SFRSYM    DATA     BYTE      EIE1
      000000C0H.7 SFRSYM    DATA     BIT       SMB1CN0_MASTER
      000000C0H.1 SFRSYM    DATA     BIT       SMB0CN0_ACK
      000000D7H   SFRSYM    DATA     BYTE      USB0XCN
      000000E7H   SFRSYM    DATA     BYTE      EIE2
      000000C0H.1 SFRSYM    DATA     BIT       SMB1CN0_ACK
      0000008FH   SFRSYM    DATA     BYTE      PSCTL
      000000E4H   SFRSYM    DATA     BYTE      IT01CF
      000000C8H   SFRSYM    DATA     BIT       TMR5CN0_T5XCLK
LX51 LINKER/LOCATER V4.66.30.0                                                        07/27/2019  23:22:19  PAGE 148


      000000C0H.6 SFRSYM    DATA     BIT       SMB0CN0_TXMODE
      000000C0H.6 SFRSYM    DATA     BIT       SMB1CN0_TXMODE
      000000BFH   SFRSYM    DATA     BYTE      SFRPAGE
      000000A4H   SFRSYM    DATA     BYTE      P0MDOUT
      000000A5H   SFRSYM    DATA     BYTE      P1MDOUT
      000000E8H.5 SFRSYM    DATA     BIT       ADC0CN0_ADINT
      000000CBH   SFRSYM    DATA     BYTE      TMR2RLH
      000000A6H   SFRSYM    DATA     BYTE      P2MDOUT
      000000A8H   SFRSYM    DATA     BYTE      IE
      00000093H   SFRSYM    DATA     BYTE      TMR3RLH
      000000A7H   SFRSYM    DATA     BYTE      P3MDOUT
      00000093H   SFRSYM    DATA     BYTE      TMR4RLH
      000000AEH   SFRSYM    DATA     BYTE      P4MDOUT
      000000F6H   SFRSYM    DATA     BYTE      EIP1
      000000CBH   SFRSYM    DATA     BYTE      TMR5RLH
      000000F7H   SFRSYM    DATA     BYTE      EIP2
      00000098H.2 SFRSYM    DATA     BIT       SCON0_RB8
      000000CAH   SFRSYM    DATA     BYTE      TMR2RLL
      000000FCH   SFRSYM    DATA     BYTE      PCA0CPH0
      00000092H   SFRSYM    DATA     BYTE      TMR3RLL
      000000EAH   SFRSYM    DATA     BYTE      PCA0CPH1
      00000098H.3 SFRSYM    DATA     BIT       SCON0_TB8
      000000F0H   SFRSYM    DATA     BIT       B_B0
      00000082H   SFRSYM    DATA     WORD      DP
      00000092H   SFRSYM    DATA     BYTE      TMR4RLL
      000000ECH   SFRSYM    DATA     BYTE      PCA0CPH2
      000000F0H.1 SFRSYM    DATA     BIT       B_B1
      000000C3H   SFRSYM    DATA     WORD      ADC0GT
      000000CAH   SFRSYM    DATA     BYTE      TMR5RLL
      000000EEH   SFRSYM    DATA     BYTE      PCA0CPH3
      000000F0H.2 SFRSYM    DATA     BIT       B_B2
      000000FBH   SFRSYM    DATA     BYTE      PCA0CPL0
      000000FEH   SFRSYM    DATA     BYTE      PCA0CPH4
      00000085H   SFRSYM    DATA     BYTE      EMI0CF
      000000F0H.3 SFRSYM    DATA     BIT       B_B3
      000000D9H   SFRSYM    DATA     BYTE      PCA0MD
      000000DAH   SFRSYM    DATA     BYTE      PCA0CPM0
      000000E9H   SFRSYM    DATA     BYTE      PCA0CPL1
      000000F0H.4 SFRSYM    DATA     BIT       B_B4
      000000DBH   SFRSYM    DATA     BYTE      PCA0CPM1
      000000EBH   SFRSYM    DATA     BYTE      PCA0CPL2
      000000F0H.5 SFRSYM    DATA     BIT       B_B5
      000000DCH   SFRSYM    DATA     BYTE      PCA0CPM2
      000000EDH   SFRSYM    DATA     BYTE      PCA0CPL3
      000000B8H   SFRSYM    DATA     BYTE      IP
      000000F0H.6 SFRSYM    DATA     BIT       B_B6
      000000C5H   SFRSYM    DATA     WORD      ADC0LT
      000000DDH   SFRSYM    DATA     BYTE      PCA0CPM3
      000000FDH   SFRSYM    DATA     BYTE      PCA0CPL4
      00000098H.5 SFRSYM    DATA     BIT       SCON0_MCE
      000000F0H.7 SFRSYM    DATA     BIT       B_B7
      000000DEH   SFRSYM    DATA     BYTE      PCA0CPM4
      000000E1H   SFRSYM    DATA     BYTE      XBR0
      000000C1H   SFRSYM    DATA     BYTE      SMB0CF
      000000E2H   SFRSYM    DATA     BYTE      XBR1
      000000C1H   SFRSYM    DATA     BYTE      SMB1CF
      000000AFH   SFRSYM    DATA     BYTE      PFE0CN
      000000AAH   SFRSYM    DATA     BYTE      EMI0CN
      000000C0H.5 SFRSYM    DATA     BIT       SMB0CN0_STA
      000000E3H   SFRSYM    DATA     BYTE      XBR2
      000000C0H.5 SFRSYM    DATA     BIT       SMB1CN0_STA
      000000E0H   SFRSYM    DATA     BIT       ACC_ACC0
LX51 LINKER/LOCATER V4.66.30.0                                                        07/27/2019  23:22:19  PAGE 149


      000000D1H   SFRSYM    DATA     BYTE      REF0CN
      000000B2H   SFRSYM    DATA     BYTE      HFO0CN
      0000008EH   SFRSYM    DATA     BYTE      CKCON0
      000000E0H.1 SFRSYM    DATA     BIT       ACC_ACC1
      000000E4H   SFRSYM    DATA     BYTE      CKCON1
      000000C8H.2 SFRSYM    DATA     BIT       TMR2CN0_TR2
      000000E0H.2 SFRSYM    DATA     BIT       ACC_ACC2
      000000E0H.3 SFRSYM    DATA     BIT       ACC_ACC3
      00000081H   SFRSYM    DATA     BYTE      SP
      0000009DH   SFRSYM    DATA     BYTE      CMP0MD
      000000E0H.4 SFRSYM    DATA     BIT       ACC_ACC4
      00000086H   SFRSYM    DATA     BYTE      LFO0CN
      00000084H   SFRSYM    DATA     BYTE      EMI0TC
      0000009CH   SFRSYM    DATA     BYTE      CMP1MD
      000000D8H   SFRSYM    DATA     BIT       PCA0CN0_CCF0
      000000E0H.5 SFRSYM    DATA     BIT       ACC_ACC5
      000000D8H.1 SFRSYM    DATA     BIT       PCA0CN0_CCF1
      000000E0H.6 SFRSYM    DATA     BIT       ACC_ACC6
      000000CCH   SFRSYM    DATA     WORD      TMR2
      000000D8H.2 SFRSYM    DATA     BIT       PCA0CN0_CCF2
      000000E0H.7 SFRSYM    DATA     BIT       ACC_ACC7
      00000094H   SFRSYM    DATA     WORD      TMR3
      000000C8H.2 SFRSYM    DATA     BIT       TMR5CN0_TR5
      000000D8H.3 SFRSYM    DATA     BIT       PCA0CN0_CCF3
      00000094H   SFRSYM    DATA     WORD      TMR4
      000000ACH   SFRSYM    DATA     BYTE      SBCON1
      000000D8H.4 SFRSYM    DATA     BIT       PCA0CN0_CCF4
      000000CCH   SFRSYM    DATA     WORD      TMR5
      000000C0H.3 SFRSYM    DATA     BIT       SMB0CN0_ACKRQ
      000000FFH   SFRSYM    DATA     BYTE      VDM0CN
      000000F1H   SFRSYM    DATA     BYTE      P0MDIN
      000000C0H.3 SFRSYM    DATA     BIT       SMB1CN0_ACKRQ
      00000098H.4 SFRSYM    DATA     BIT       SCON0_REN
      000000F2H   SFRSYM    DATA     BYTE      P1MDIN
      000000F3H   SFRSYM    DATA     BYTE      P2MDIN
      000000C0H.4 SFRSYM    DATA     BIT       SMB0CN0_STO
      000000F4H   SFRSYM    DATA     BYTE      P3MDIN
      000000C0H.4 SFRSYM    DATA     BIT       SMB1CN0_STO
      000000B5H   SFRSYM    DATA     BYTE      SBRLH1
      000000F5H   SFRSYM    DATA     BYTE      P4MDIN
      000000D0H.3 SFRSYM    DATA     BIT       PSW_RS0
      000000D8H.7 SFRSYM    DATA     BIT       PCA0CN0_CF
      000000F8H.4 SFRSYM    DATA     BIT       SPI0CN0_RXOVRN
      000000D0H.4 SFRSYM    DATA     BIT       PSW_RS1
      000000B4H   SFRSYM    DATA     BYTE      SBRLL1
      000000E8H.7 SFRSYM    DATA     BIT       ADC0CN0_ADEN
      00000089H   SFRSYM    DATA     BYTE      TMOD
      00000088H   SFRSYM    DATA     BYTE      TCON
      000000D0H   SFRSYM    DATA     BIT       PSW_PARITY
      000000A8H.4 SFRSYM    DATA     BIT       IE_ES0
      0000009FH   SFRSYM    DATA     BYTE      CMP0MX
      000000A8H.1 SFRSYM    DATA     BIT       IE_ET0
      0000009EH   SFRSYM    DATA     BYTE      CMP1MX
      000000A8H.3 SFRSYM    DATA     BIT       IE_ET1
      000000D4H   SFRSYM    DATA     BYTE      P0SKIP
      000000C8H.1 SFRSYM    DATA     BIT       TMR2CN0_T2CSS
      000000A8H.5 SFRSYM    DATA     BIT       IE_ET2
      000000D5H   SFRSYM    DATA     BYTE      P1SKIP
      000000D6H   SFRSYM    DATA     BYTE      P2SKIP
      000000E8H   SFRSYM    DATA     BYTE      ADC0CN0
      000000A8H   SFRSYM    DATA     BIT       IE_EX0
      000000DFH   SFRSYM    DATA     BYTE      P3SKIP
LX51 LINKER/LOCATER V4.66.30.0                                                        07/27/2019  23:22:19  PAGE 150


      000000D8H.6 SFRSYM    DATA     BIT       PCA0CN0_CR
      000000A8H.2 SFRSYM    DATA     BIT       IE_EX1
      00000098H.7 SFRSYM    DATA     BIT       SCON0_SMODE
      000000A9H   SFRSYM    DATA     BYTE      CLKSEL
      000000F8H   SFRSYM    DATA     BIT       SPI0CN0_SPIEN
      000000F0H   SFRSYM    DATA     BYTE      B
      000000BEH   SFRSYM    DATA     BYTE      ADC0H
      000000E8H.6 SFRSYM    DATA     BIT       ADC0CN0_ADTM
      000000CAH   SFRSYM    DATA     WORD      TMR2RL
      000000BDH   SFRSYM    DATA     BYTE      ADC0L
      00000092H   SFRSYM    DATA     WORD      TMR3RL
      00000092H   SFRSYM    DATA     WORD      TMR4RL
      000000D8H   SFRSYM    DATA     BYTE      PCA0CN0
      000000E0H   SFRSYM    DATA     BYTE      ACC
      000000CAH   SFRSYM    DATA     WORD      TMR5RL
      000000FBH   SFRSYM    DATA     WORD      PCA0CP0
      000000E9H   SFRSYM    DATA     WORD      PCA0CP1
      000000EBH   SFRSYM    DATA     WORD      PCA0CP2
      000000EDH   SFRSYM    DATA     WORD      PCA0CP3
      0000008CH   SFRSYM    DATA     BYTE      TH0
      000000B8H.4 SFRSYM    DATA     BIT       IP_PS0
      000000FDH   SFRSYM    DATA     WORD      PCA0CP4
      0000008DH   SFRSYM    DATA     BYTE      TH1
      000000FAH   SFRSYM    DATA     BYTE      PCA0H
      000000B8H.1 SFRSYM    DATA     BIT       IP_PT0
      000000B8H.3 SFRSYM    DATA     BIT       IP_PT1
      000000C0H.2 SFRSYM    DATA     BIT       SMB0CN0_ARBLOST
      000000B8H.5 SFRSYM    DATA     BIT       IP_PT2
      0000008AH   SFRSYM    DATA     BYTE      TL0
      000000F8H.1 SFRSYM    DATA     BIT       SPI0CN0_TXBMT
      000000C0H.2 SFRSYM    DATA     BIT       SMB1CN0_ARBLOST
      000000D0H.5 SFRSYM    DATA     BIT       PSW_F0
      000000A8H.6 SFRSYM    DATA     BIT       IE_ESPI0
      0000008BH   SFRSYM    DATA     BYTE      TL1
      000000F9H   SFRSYM    DATA     BYTE      PCA0L
      000000C0H   SFRSYM    DATA     BIT       SMB0CN0_SI
      000000D0H.1 SFRSYM    DATA     BIT       PSW_F1
      00000080H   SFRSYM    DATA     BIT       P0_B0
      000000B8H   SFRSYM    DATA     BIT       IP_PX0
      000000C9H   SFRSYM    DATA     BYTE      REG01CN
      000000C0H   SFRSYM    DATA     BIT       SMB1CN0_SI
      00000090H   SFRSYM    DATA     BIT       P1_B0
      00000080H.1 SFRSYM    DATA     BIT       P0_B1
      000000B8H.2 SFRSYM    DATA     BIT       IP_PX1
      0000009BH   SFRSYM    DATA     BYTE      CMP0CN0
      00000088H.1 SFRSYM    DATA     BIT       TCON_IE0
      000000A0H   SFRSYM    DATA     BIT       P2_B0
      00000090H.1 SFRSYM    DATA     BIT       P1_B1
      00000080H.2 SFRSYM    DATA     BIT       P0_B2
      0000009AH   SFRSYM    DATA     BYTE      CMP1CN0
      00000088H.3 SFRSYM    DATA     BIT       TCON_IE1
      000000B0H   SFRSYM    DATA     BIT       P3_B0
      000000A0H.1 SFRSYM    DATA     BIT       P2_B1
      00000090H.2 SFRSYM    DATA     BIT       P1_B2
      00000080H.3 SFRSYM    DATA     BIT       P0_B3
      000000C0H   SFRSYM    DATA     BYTE      SMB0CN0
      000000B0H.1 SFRSYM    DATA     BIT       P3_B1
      000000A0H.2 SFRSYM    DATA     BIT       P2_B2
      00000090H.3 SFRSYM    DATA     BIT       P1_B3
      00000080H.4 SFRSYM    DATA     BIT       P0_B4
      000000C0H   SFRSYM    DATA     BYTE      SMB1CN0
      000000B0H.2 SFRSYM    DATA     BIT       P3_B2
LX51 LINKER/LOCATER V4.66.30.0                                                        07/27/2019  23:22:19  PAGE 151


      000000A0H.3 SFRSYM    DATA     BIT       P2_B3
      00000090H.4 SFRSYM    DATA     BIT       P1_B4
      00000080H.5 SFRSYM    DATA     BIT       P0_B5
      000000B0H.3 SFRSYM    DATA     BIT       P3_B3
      000000A0H.4 SFRSYM    DATA     BIT       P2_B4
      00000090H.5 SFRSYM    DATA     BIT       P1_B5
      00000080H.6 SFRSYM    DATA     BIT       P0_B6
      000000B0H.4 SFRSYM    DATA     BIT       P3_B4
      000000A0H.5 SFRSYM    DATA     BIT       P2_B5
      00000090H.6 SFRSYM    DATA     BIT       P1_B6
      00000080H.7 SFRSYM    DATA     BIT       P0_B7
      000000B0H.5 SFRSYM    DATA     BIT       P3_B5
      000000A0H.6 SFRSYM    DATA     BIT       P2_B6
      00000090H.7 SFRSYM    DATA     BIT       P1_B7
      000000B0H.6 SFRSYM    DATA     BIT       P3_B6
      000000A0H.7 SFRSYM    DATA     BIT       P2_B7
      000000B0H.7 SFRSYM    DATA     BIT       P3_B7
      00000083H   SFRSYM    DATA     BYTE      DPH
      000000C4H   SFRSYM    DATA     BYTE      ADC0GTH
      000000C8H.7 SFRSYM    DATA     BIT       TMR2CN0_TF2H
      000000C8H.3 SFRSYM    DATA     BIT       TMR2CN0_T2SPLIT
      000000D0H.6 SFRSYM    DATA     BIT       PSW_AC
      000000F8H   SFRSYM    DATA     BYTE      SPI0CN0
      000000B3H   SFRSYM    DATA     BYTE      HFO0CAL
      00000088H.5 SFRSYM    DATA     BIT       TCON_TF0
      00000098H   SFRSYM    DATA     BIT       SCON0_RI
      00000082H   SFRSYM    DATA     BYTE      DPL
      00000088H.7 SFRSYM    DATA     BIT       TCON_TF1
      00000099H   SFRSYM    DATA     BYTE      SBUF0
      00000087H   SFRSYM    DATA     BYTE      PCON0
      000000C3H   SFRSYM    DATA     BYTE      ADC0GTL
      000000C8H.6 SFRSYM    DATA     BIT       TMR2CN0_TF2L
      00000098H.1 SFRSYM    DATA     BIT       SCON0_TI
      000000E8H   SFRSYM    DATA     BIT       ADC0CN0_ADCM0
      000000D3H   SFRSYM    DATA     BYTE      SBUF1
      000000C6H   SFRSYM    DATA     BYTE      ADC0LTH
      00000088H   SFRSYM    DATA     BIT       TCON_IT0
      000000E8H.1 SFRSYM    DATA     BIT       ADC0CN0_ADCM1
      000000EFH   SFRSYM    DATA     BYTE      RSTSRC
      000000C8H.7 SFRSYM    DATA     BIT       TMR5CN0_TF5H
      000000C8H.3 SFRSYM    DATA     BIT       TMR5CN0_T5SPLIT
      00000088H.2 SFRSYM    DATA     BIT       TCON_IT1
      000000E8H.2 SFRSYM    DATA     BIT       ADC0CN0_ADCM2
      00000098H   SFRSYM    DATA     BYTE      SCON0
      000000E8H.3 SFRSYM    DATA     BIT       ADC0CN0_ADWINT
      000000B4H   SFRSYM    DATA     WORD      SBRL1
      000000E5H   SFRSYM    DATA     BYTE      SMOD1
      000000D2H   SFRSYM    DATA     BYTE      SCON1
      000000BAH   SFRSYM    DATA     BYTE      AMX0N
      000000E8H.4 SFRSYM    DATA     BIT       ADC0CN0_ADBUSY
      000000CEH   SFRSYM    DATA     BYTE      SMB0ADM
      000000C5H   SFRSYM    DATA     BYTE      ADC0LTL
      000000F8H.5 SFRSYM    DATA     BIT       SPI0CN0_MODF
      000000B8H.6 SFRSYM    DATA     BIT       IP_PSPI0
      000000CEH   SFRSYM    DATA     BYTE      SMB1ADM
      000000BBH   SFRSYM    DATA     BYTE      AMX0P
      000000C8H.6 SFRSYM    DATA     BIT       TMR5CN0_TF5L
      000000C8H   SFRSYM    DATA     BYTE      TMR2CN0
      00000091H   SFRSYM    DATA     BYTE      TMR3CN0
      00000091H   SFRSYM    DATA     BYTE      TMR4CN0
      000000C8H   SFRSYM    DATA     BYTE      TMR5CN0
      000000CFH   SFRSYM    DATA     BYTE      SMB0ADR
LX51 LINKER/LOCATER V4.66.30.0                                                        07/27/2019  23:22:19  PAGE 152


      00000088H.4 SFRSYM    DATA     BIT       TCON_TR0
      000000CFH   SFRSYM    DATA     BYTE      SMB1ADR
      000000C8H.4 SFRSYM    DATA     BIT       TMR2CN0_TF2CEN
      00000088H.6 SFRSYM    DATA     BIT       TCON_TR1
      000000C2H   SFRSYM    DATA     BYTE      SMB0DAT
      000000CDH   SFRSYM    DATA     BYTE      TMR2H
      000000A1H   SFRSYM    DATA     BYTE      SPI0CFG
      000000C2H   SFRSYM    DATA     BYTE      SMB1DAT
      00000095H   SFRSYM    DATA     BYTE      TMR3H
      00000095H   SFRSYM    DATA     BYTE      TMR4H
      000000CDH   SFRSYM    DATA     BYTE      TMR5H
      000000CCH   SFRSYM    DATA     BYTE      TMR2L
      000000F8H.7 SFRSYM    DATA     BIT       SPI0CN0_SPIF
      00000096H   SFRSYM    DATA     BYTE      USB0ADR
      00000094H   SFRSYM    DATA     BYTE      TMR3L
      000000A8H.7 SFRSYM    DATA     BIT       IE_EA
      00000094H   SFRSYM    DATA     BYTE      TMR4L
      00000097H   SFRSYM    DATA     BYTE      USB0DAT
      000000CCH   SFRSYM    DATA     BYTE      TMR5L
      000000B6H   SFRSYM    DATA     BYTE      FLSCL
      000000C8H.5 SFRSYM    DATA     BIT       TMR2CN0_TF2LEN
      000000F8H.6 SFRSYM    DATA     BIT       SPI0CN0_WCOL
      000000F8H.2 SFRSYM    DATA     BIT       SPI0CN0_NSSMD0
      000000D0H.7 SFRSYM    DATA     BIT       PSW_CY
      000000A3H   SFRSYM    DATA     BYTE      SPI0DAT
      000000F8H.3 SFRSYM    DATA     BIT       SPI0CN0_NSSMD1
      000000BDH   SFRSYM    DATA     WORD      ADC0
      000000B9H   SFRSYM    DATA     BYTE      SMBTC
      000000D0H   SFRSYM    DATA     BYTE      PSW
      000000C8H.5 SFRSYM    DATA     BIT       TMR5CN0_TF5LEN
      000000B7H   SFRSYM    DATA     BYTE      FLKEY
      010051F5H   SYMBOL    CODE     ---       _btn_check

      0100483CH   BLOCK     CODE     ---       LVL=0
      0100483CH   BLOCK     CODE     NEAR LAB  LVL=1
      00000007H   SYMBOL    DATA     BYTE      i
      ---         BLOCKEND  ---      ---       LVL=1
      0100483CH   LINE      CODE     ---       #14
      0100483CH   LINE      CODE     ---       #15
      0100483CH   LINE      CODE     ---       #18
      0100483EH   LINE      CODE     ---       #19
      0100484EH   LINE      CODE     ---       #20
      01004860H   LINE      CODE     ---       #21
      01004870H   LINE      CODE     ---       #22
      01004884H   LINE      CODE     ---       #23
      01004895H   LINE      CODE     ---       #24
      010048A6H   LINE      CODE     ---       #25
      010048AAH   LINE      CODE     ---       #30
      010048ADH   LINE      CODE     ---       #31
      010048B0H   LINE      CODE     ---       #32
      010048B3H   LINE      CODE     ---       #33
      010048B6H   LINE      CODE     ---       #36
      010048B9H   LINE      CODE     ---       #37
      010048BCH   LINE      CODE     ---       #38
      010048BFH   LINE      CODE     ---       #39
      010048C2H   LINE      CODE     ---       #42
      010048C4H   LINE      CODE     ---       #43
      010048C6H   LINE      CODE     ---       #44
      010048C8H   LINE      CODE     ---       #45
      010048CAH   LINE      CODE     ---       #46
      ---         BLOCKEND  ---      ---       LVL=0

LX51 LINKER/LOCATER V4.66.30.0                                                        07/27/2019  23:22:19  PAGE 153


      010051F5H   BLOCK     CODE     ---       LVL=0
      00000007H   SYMBOL    DATA     BYTE      idx
      00000005H   SYMBOL    DATA     BYTE      state
      010051F5H   LINE      CODE     ---       #48
      010051F5H   LINE      CODE     ---       #49
      010051F5H   LINE      CODE     ---       #50
      010051FAH   LINE      CODE     ---       #51
      010051FCH   LINE      CODE     ---       #52
      010051FFH   LINE      CODE     ---       #53
      010051FFH   LINE      CODE     ---       #55
      01005202H   LINE      CODE     ---       #56
      01005218H   LINE      CODE     ---       #57
      0100522DH   LINE      CODE     ---       #58
      0100522DH   LINE      CODE     ---       #59
      0100522DH   LINE      CODE     ---       #60
      0100523FH   LINE      CODE     ---       #61
      0100523FH   LINE      CODE     ---       #62
      ---         BLOCKEND  ---      ---       LVL=0

      01003072H   BLOCK     CODE     ---       LVL=0
      01003072H   BLOCK     CODE     NEAR LAB  LVL=1
      00000005H   SYMBOL    DATA     BYTE      i
      ---         BLOCKEND  ---      ---       LVL=1
      01003072H   LINE      CODE     ---       #64
      01003072H   LINE      CODE     ---       #65
      01003072H   LINE      CODE     ---       #69
      0100307CH   LINE      CODE     ---       #70
      01003086H   LINE      CODE     ---       #71
      01003090H   LINE      CODE     ---       #72
      0100309AH   LINE      CODE     ---       #75
      0100309CH   LINE      CODE     ---       #77
      010030B5H   LINE      CODE     ---       #79
      010030CAH   LINE      CODE     ---       #81
      010030DBH   LINE      CODE     ---       #84
      01003116H   LINE      CODE     ---       #86
      01003128H   LINE      CODE     ---       #87
      01003139H   LINE      CODE     ---       #88
      0100315FH   LINE      CODE     ---       #89
      0100315FH   LINE      CODE     ---       #90
      0100315FH   LINE      CODE     ---       #91
      01003161H   LINE      CODE     ---       #93
      01003178H   LINE      CODE     ---       #94
      01003189H   LINE      CODE     ---       #95
      01003189H   LINE      CODE     ---       #96
      01003189H   LINE      CODE     ---       #97
      01003192H   LINE      CODE     ---       #98
      ---         BLOCKEND  ---      ---       LVL=0

      010029F8H   BLOCK     CODE     ---       LVL=0
      010029F8H   BLOCK     CODE     NEAR LAB  LVL=1
      00000022H   SYMBOL    DATA     BYTE      i
      00000023H   SYMBOL    DATA     BYTE      s
      ---         BLOCKEND  ---      ---       LVL=1
      010029F8H   LINE      CODE     ---       #100
      010029F8H   LINE      CODE     ---       #101
      010029F8H   LINE      CODE     ---       #105
      010029FBH   LINE      CODE     ---       #106
      01002A0EH   LINE      CODE     ---       #108
      01002A14H   LINE      CODE     ---       #109
      01002A27H   LINE      CODE     ---       #110
      01002A3EH   LINE      CODE     ---       #111
      01002A53H   LINE      CODE     ---       #112
LX51 LINKER/LOCATER V4.66.30.0                                                        07/27/2019  23:22:19  PAGE 154


      01002A53H   LINE      CODE     ---       #113
      01002A53H   LINE      CODE     ---       #115
      01002A6AH   LINE      CODE     ---       #116
      01002A80H   LINE      CODE     ---       #117
      01002A96H   LINE      CODE     ---       #118
      01002A98H   LINE      CODE     ---       #119
      01002AACH   LINE      CODE     ---       #120
      01002ABFH   LINE      CODE     ---       #121
      01002ABFH   LINE      CODE     ---       #122
      01002ABFH   LINE      CODE     ---       #124
      01002AC7H   LINE      CODE     ---       #125
      01002ADAH   LINE      CODE     ---       #126
      01002AF1H   LINE      CODE     ---       #127
      01002B06H   LINE      CODE     ---       #128
      01002B06H   LINE      CODE     ---       #129
      01002B06H   LINE      CODE     ---       #131
      01002B0EH   LINE      CODE     ---       #132
      01002B21H   LINE      CODE     ---       #133
      01002B38H   LINE      CODE     ---       #134
      01002B4DH   LINE      CODE     ---       #135
      01002B4DH   LINE      CODE     ---       #136
      01002B4DH   LINE      CODE     ---       #137
      01002B59H   LINE      CODE     ---       #138
      ---         BLOCKEND  ---      ---       LVL=0

      ---         MODULE    ---      ---       MENU
      0000001BH   PUBLIC    DATA     BYTE      menu_idx
      00000019H   PUBLIC    DATA     ---       menu
      00000018H   PUBLIC    DATA     BYTE      mtick
      01004A51H   PUBLIC    CODE     ---       _menu_draw_tabs
      01001E7AH   PUBLIC    CODE     ---       _menu_draw_buttons
      01005677H   PUBLIC    CODE     ---       menu_btn_use_none
      0100468AH   PUBLIC    CODE     ---       menu_btn_use_std
      010055ABH   PUBLIC    CODE     ---       menu_btn_exit
      01005727H   PUBLIC    CODE     ---       menu_btn_enter
      01005A25H   PUBLIC    CODE     ---       menu_btn_prev
      01005964H   PUBLIC    CODE     ---       menu_btn_next
      01005B5BH   PUBLIC    CODE     ---       _menu_stop
      01005A13H   PUBLIC    CODE     ---       _menu_start
      01004DA6H   PUBLIC    CODE     ---       menu_tick
      000000A2H   SFRSYM    DATA     BYTE      SPI0CKR
      00000080H   SFRSYM    DATA     BYTE      P0
      000000D0H.2 SFRSYM    DATA     BIT       PSW_OV
      000000B1H   SFRSYM    DATA     BYTE      XOSC0CN
      00000090H   SFRSYM    DATA     BYTE      P1
      000000A0H   SFRSYM    DATA     BYTE      P2
      000000B0H   SFRSYM    DATA     BYTE      P3
      000000BCH   SFRSYM    DATA     BYTE      ADC0CF
      000000C8H   SFRSYM    DATA     BIT       TMR2CN0_T2XCLK
      000000C7H   SFRSYM    DATA     BYTE      P4
      000000C0H.7 SFRSYM    DATA     BIT       SMB0CN0_MASTER
      000000F9H   SFRSYM    DATA     WORD      PCA0
      000000E6H   SFRSYM    DATA     BYTE      EIE1
      000000C0H.7 SFRSYM    DATA     BIT       SMB1CN0_MASTER
      000000C0H.1 SFRSYM    DATA     BIT       SMB0CN0_ACK
      000000D7H   SFRSYM    DATA     BYTE      USB0XCN
      000000E7H   SFRSYM    DATA     BYTE      EIE2
      000000C0H.1 SFRSYM    DATA     BIT       SMB1CN0_ACK
      0000008FH   SFRSYM    DATA     BYTE      PSCTL
      000000E4H   SFRSYM    DATA     BYTE      IT01CF
      000000C8H   SFRSYM    DATA     BIT       TMR5CN0_T5XCLK
      000000C0H.6 SFRSYM    DATA     BIT       SMB0CN0_TXMODE
LX51 LINKER/LOCATER V4.66.30.0                                                        07/27/2019  23:22:19  PAGE 155


      000000C0H.6 SFRSYM    DATA     BIT       SMB1CN0_TXMODE
      000000BFH   SFRSYM    DATA     BYTE      SFRPAGE
      000000A4H   SFRSYM    DATA     BYTE      P0MDOUT
      000000A5H   SFRSYM    DATA     BYTE      P1MDOUT
      000000E8H.5 SFRSYM    DATA     BIT       ADC0CN0_ADINT
      000000CBH   SFRSYM    DATA     BYTE      TMR2RLH
      000000A6H   SFRSYM    DATA     BYTE      P2MDOUT
      000000A8H   SFRSYM    DATA     BYTE      IE
      00000093H   SFRSYM    DATA     BYTE      TMR3RLH
      000000A7H   SFRSYM    DATA     BYTE      P3MDOUT
      00000093H   SFRSYM    DATA     BYTE      TMR4RLH
      000000AEH   SFRSYM    DATA     BYTE      P4MDOUT
      000000F6H   SFRSYM    DATA     BYTE      EIP1
      000000CBH   SFRSYM    DATA     BYTE      TMR5RLH
      000000F7H   SFRSYM    DATA     BYTE      EIP2
      00000098H.2 SFRSYM    DATA     BIT       SCON0_RB8
      000000CAH   SFRSYM    DATA     BYTE      TMR2RLL
      000000FCH   SFRSYM    DATA     BYTE      PCA0CPH0
      00000092H   SFRSYM    DATA     BYTE      TMR3RLL
      000000EAH   SFRSYM    DATA     BYTE      PCA0CPH1
      00000098H.3 SFRSYM    DATA     BIT       SCON0_TB8
      000000F0H   SFRSYM    DATA     BIT       B_B0
      00000082H   SFRSYM    DATA     WORD      DP
      00000092H   SFRSYM    DATA     BYTE      TMR4RLL
      000000ECH   SFRSYM    DATA     BYTE      PCA0CPH2
      000000F0H.1 SFRSYM    DATA     BIT       B_B1
      000000C3H   SFRSYM    DATA     WORD      ADC0GT
      000000CAH   SFRSYM    DATA     BYTE      TMR5RLL
      000000EEH   SFRSYM    DATA     BYTE      PCA0CPH3
      000000F0H.2 SFRSYM    DATA     BIT       B_B2
      000000FBH   SFRSYM    DATA     BYTE      PCA0CPL0
      000000FEH   SFRSYM    DATA     BYTE      PCA0CPH4
      00000085H   SFRSYM    DATA     BYTE      EMI0CF
      000000F0H.3 SFRSYM    DATA     BIT       B_B3
      000000D9H   SFRSYM    DATA     BYTE      PCA0MD
      000000DAH   SFRSYM    DATA     BYTE      PCA0CPM0
      000000E9H   SFRSYM    DATA     BYTE      PCA0CPL1
      000000F0H.4 SFRSYM    DATA     BIT       B_B4
      000000DBH   SFRSYM    DATA     BYTE      PCA0CPM1
      000000EBH   SFRSYM    DATA     BYTE      PCA0CPL2
      000000F0H.5 SFRSYM    DATA     BIT       B_B5
      000000DCH   SFRSYM    DATA     BYTE      PCA0CPM2
      000000EDH   SFRSYM    DATA     BYTE      PCA0CPL3
      000000B8H   SFRSYM    DATA     BYTE      IP
      000000F0H.6 SFRSYM    DATA     BIT       B_B6
      000000C5H   SFRSYM    DATA     WORD      ADC0LT
      000000DDH   SFRSYM    DATA     BYTE      PCA0CPM3
      000000FDH   SFRSYM    DATA     BYTE      PCA0CPL4
      00000098H.5 SFRSYM    DATA     BIT       SCON0_MCE
      000000F0H.7 SFRSYM    DATA     BIT       B_B7
      000000DEH   SFRSYM    DATA     BYTE      PCA0CPM4
      000000E1H   SFRSYM    DATA     BYTE      XBR0
      000000C1H   SFRSYM    DATA     BYTE      SMB0CF
      000000E2H   SFRSYM    DATA     BYTE      XBR1
      000000C1H   SFRSYM    DATA     BYTE      SMB1CF
      000000AFH   SFRSYM    DATA     BYTE      PFE0CN
      000000AAH   SFRSYM    DATA     BYTE      EMI0CN
      000000C0H.5 SFRSYM    DATA     BIT       SMB0CN0_STA
      000000E3H   SFRSYM    DATA     BYTE      XBR2
      000000C0H.5 SFRSYM    DATA     BIT       SMB1CN0_STA
      000000E0H   SFRSYM    DATA     BIT       ACC_ACC0
      000000D1H   SFRSYM    DATA     BYTE      REF0CN
LX51 LINKER/LOCATER V4.66.30.0                                                        07/27/2019  23:22:19  PAGE 156


      000000B2H   SFRSYM    DATA     BYTE      HFO0CN
      0000008EH   SFRSYM    DATA     BYTE      CKCON0
      000000E0H.1 SFRSYM    DATA     BIT       ACC_ACC1
      000000E4H   SFRSYM    DATA     BYTE      CKCON1
      000000C8H.2 SFRSYM    DATA     BIT       TMR2CN0_TR2
      000000E0H.2 SFRSYM    DATA     BIT       ACC_ACC2
      000000E0H.3 SFRSYM    DATA     BIT       ACC_ACC3
      00000081H   SFRSYM    DATA     BYTE      SP
      0000009DH   SFRSYM    DATA     BYTE      CMP0MD
      000000E0H.4 SFRSYM    DATA     BIT       ACC_ACC4
      00000086H   SFRSYM    DATA     BYTE      LFO0CN
      00000084H   SFRSYM    DATA     BYTE      EMI0TC
      0000009CH   SFRSYM    DATA     BYTE      CMP1MD
      000000D8H   SFRSYM    DATA     BIT       PCA0CN0_CCF0
      000000E0H.5 SFRSYM    DATA     BIT       ACC_ACC5
      000000D8H.1 SFRSYM    DATA     BIT       PCA0CN0_CCF1
      000000E0H.6 SFRSYM    DATA     BIT       ACC_ACC6
      000000CCH   SFRSYM    DATA     WORD      TMR2
      000000D8H.2 SFRSYM    DATA     BIT       PCA0CN0_CCF2
      000000E0H.7 SFRSYM    DATA     BIT       ACC_ACC7
      00000094H   SFRSYM    DATA     WORD      TMR3
      000000C8H.2 SFRSYM    DATA     BIT       TMR5CN0_TR5
      000000D8H.3 SFRSYM    DATA     BIT       PCA0CN0_CCF3
      00000094H   SFRSYM    DATA     WORD      TMR4
      000000ACH   SFRSYM    DATA     BYTE      SBCON1
      000000D8H.4 SFRSYM    DATA     BIT       PCA0CN0_CCF4
      000000CCH   SFRSYM    DATA     WORD      TMR5
      000000C0H.3 SFRSYM    DATA     BIT       SMB0CN0_ACKRQ
      000000FFH   SFRSYM    DATA     BYTE      VDM0CN
      000000F1H   SFRSYM    DATA     BYTE      P0MDIN
      000000C0H.3 SFRSYM    DATA     BIT       SMB1CN0_ACKRQ
      00000098H.4 SFRSYM    DATA     BIT       SCON0_REN
      000000F2H   SFRSYM    DATA     BYTE      P1MDIN
      000000F3H   SFRSYM    DATA     BYTE      P2MDIN
      000000C0H.4 SFRSYM    DATA     BIT       SMB0CN0_STO
      000000F4H   SFRSYM    DATA     BYTE      P3MDIN
      000000C0H.4 SFRSYM    DATA     BIT       SMB1CN0_STO
      000000B5H   SFRSYM    DATA     BYTE      SBRLH1
      000000F5H   SFRSYM    DATA     BYTE      P4MDIN
      000000D0H.3 SFRSYM    DATA     BIT       PSW_RS0
      000000D8H.7 SFRSYM    DATA     BIT       PCA0CN0_CF
      000000F8H.4 SFRSYM    DATA     BIT       SPI0CN0_RXOVRN
      000000D0H.4 SFRSYM    DATA     BIT       PSW_RS1
      000000B4H   SFRSYM    DATA     BYTE      SBRLL1
      000000E8H.7 SFRSYM    DATA     BIT       ADC0CN0_ADEN
      00000089H   SFRSYM    DATA     BYTE      TMOD
      00000088H   SFRSYM    DATA     BYTE      TCON
      000000D0H   SFRSYM    DATA     BIT       PSW_PARITY
      000000A8H.4 SFRSYM    DATA     BIT       IE_ES0
      0000009FH   SFRSYM    DATA     BYTE      CMP0MX
      000000A8H.1 SFRSYM    DATA     BIT       IE_ET0
      0000009EH   SFRSYM    DATA     BYTE      CMP1MX
      000000A8H.3 SFRSYM    DATA     BIT       IE_ET1
      000000D4H   SFRSYM    DATA     BYTE      P0SKIP
      000000C8H.1 SFRSYM    DATA     BIT       TMR2CN0_T2CSS
      000000A8H.5 SFRSYM    DATA     BIT       IE_ET2
      000000D5H   SFRSYM    DATA     BYTE      P1SKIP
      000000D6H   SFRSYM    DATA     BYTE      P2SKIP
      000000E8H   SFRSYM    DATA     BYTE      ADC0CN0
      000000A8H   SFRSYM    DATA     BIT       IE_EX0
      000000DFH   SFRSYM    DATA     BYTE      P3SKIP
      000000D8H.6 SFRSYM    DATA     BIT       PCA0CN0_CR
LX51 LINKER/LOCATER V4.66.30.0                                                        07/27/2019  23:22:19  PAGE 157


      000000A8H.2 SFRSYM    DATA     BIT       IE_EX1
      00000098H.7 SFRSYM    DATA     BIT       SCON0_SMODE
      000000A9H   SFRSYM    DATA     BYTE      CLKSEL
      000000F8H   SFRSYM    DATA     BIT       SPI0CN0_SPIEN
      000000F0H   SFRSYM    DATA     BYTE      B
      000000BEH   SFRSYM    DATA     BYTE      ADC0H
      000000E8H.6 SFRSYM    DATA     BIT       ADC0CN0_ADTM
      000000CAH   SFRSYM    DATA     WORD      TMR2RL
      000000BDH   SFRSYM    DATA     BYTE      ADC0L
      00000092H   SFRSYM    DATA     WORD      TMR3RL
      00000092H   SFRSYM    DATA     WORD      TMR4RL
      000000D8H   SFRSYM    DATA     BYTE      PCA0CN0
      000000E0H   SFRSYM    DATA     BYTE      ACC
      000000CAH   SFRSYM    DATA     WORD      TMR5RL
      000000FBH   SFRSYM    DATA     WORD      PCA0CP0
      000000E9H   SFRSYM    DATA     WORD      PCA0CP1
      000000EBH   SFRSYM    DATA     WORD      PCA0CP2
      000000EDH   SFRSYM    DATA     WORD      PCA0CP3
      0000008CH   SFRSYM    DATA     BYTE      TH0
      000000B8H.4 SFRSYM    DATA     BIT       IP_PS0
      000000FDH   SFRSYM    DATA     WORD      PCA0CP4
      0000008DH   SFRSYM    DATA     BYTE      TH1
      000000FAH   SFRSYM    DATA     BYTE      PCA0H
      000000B8H.1 SFRSYM    DATA     BIT       IP_PT0
      000000B8H.3 SFRSYM    DATA     BIT       IP_PT1
      000000C0H.2 SFRSYM    DATA     BIT       SMB0CN0_ARBLOST
      000000B8H.5 SFRSYM    DATA     BIT       IP_PT2
      0000008AH   SFRSYM    DATA     BYTE      TL0
      000000F8H.1 SFRSYM    DATA     BIT       SPI0CN0_TXBMT
      000000C0H.2 SFRSYM    DATA     BIT       SMB1CN0_ARBLOST
      000000D0H.5 SFRSYM    DATA     BIT       PSW_F0
      000000A8H.6 SFRSYM    DATA     BIT       IE_ESPI0
      0000008BH   SFRSYM    DATA     BYTE      TL1
      000000F9H   SFRSYM    DATA     BYTE      PCA0L
      000000C0H   SFRSYM    DATA     BIT       SMB0CN0_SI
      000000D0H.1 SFRSYM    DATA     BIT       PSW_F1
      00000080H   SFRSYM    DATA     BIT       P0_B0
      000000B8H   SFRSYM    DATA     BIT       IP_PX0
      000000C9H   SFRSYM    DATA     BYTE      REG01CN
      000000C0H   SFRSYM    DATA     BIT       SMB1CN0_SI
      00000090H   SFRSYM    DATA     BIT       P1_B0
      00000080H.1 SFRSYM    DATA     BIT       P0_B1
      000000B8H.2 SFRSYM    DATA     BIT       IP_PX1
      0000009BH   SFRSYM    DATA     BYTE      CMP0CN0
      00000088H.1 SFRSYM    DATA     BIT       TCON_IE0
      000000A0H   SFRSYM    DATA     BIT       P2_B0
      00000090H.1 SFRSYM    DATA     BIT       P1_B1
      00000080H.2 SFRSYM    DATA     BIT       P0_B2
      0000009AH   SFRSYM    DATA     BYTE      CMP1CN0
      00000088H.3 SFRSYM    DATA     BIT       TCON_IE1
      000000B0H   SFRSYM    DATA     BIT       P3_B0
      000000A0H.1 SFRSYM    DATA     BIT       P2_B1
      00000090H.2 SFRSYM    DATA     BIT       P1_B2
      00000080H.3 SFRSYM    DATA     BIT       P0_B3
      000000C0H   SFRSYM    DATA     BYTE      SMB0CN0
      000000B0H.1 SFRSYM    DATA     BIT       P3_B1
      000000A0H.2 SFRSYM    DATA     BIT       P2_B2
      00000090H.3 SFRSYM    DATA     BIT       P1_B3
      00000080H.4 SFRSYM    DATA     BIT       P0_B4
      000000C0H   SFRSYM    DATA     BYTE      SMB1CN0
      000000B0H.2 SFRSYM    DATA     BIT       P3_B2
      000000A0H.3 SFRSYM    DATA     BIT       P2_B3
LX51 LINKER/LOCATER V4.66.30.0                                                        07/27/2019  23:22:19  PAGE 158


      00000090H.4 SFRSYM    DATA     BIT       P1_B4
      00000080H.5 SFRSYM    DATA     BIT       P0_B5
      000000B0H.3 SFRSYM    DATA     BIT       P3_B3
      000000A0H.4 SFRSYM    DATA     BIT       P2_B4
      00000090H.5 SFRSYM    DATA     BIT       P1_B5
      00000080H.6 SFRSYM    DATA     BIT       P0_B6
      000000B0H.4 SFRSYM    DATA     BIT       P3_B4
      000000A0H.5 SFRSYM    DATA     BIT       P2_B5
      00000090H.6 SFRSYM    DATA     BIT       P1_B6
      00000080H.7 SFRSYM    DATA     BIT       P0_B7
      000000B0H.5 SFRSYM    DATA     BIT       P3_B5
      000000A0H.6 SFRSYM    DATA     BIT       P2_B6
      00000090H.7 SFRSYM    DATA     BIT       P1_B7
      000000B0H.6 SFRSYM    DATA     BIT       P3_B6
      000000A0H.7 SFRSYM    DATA     BIT       P2_B7
      000000B0H.7 SFRSYM    DATA     BIT       P3_B7
      00000083H   SFRSYM    DATA     BYTE      DPH
      000000C4H   SFRSYM    DATA     BYTE      ADC0GTH
      000000C8H.7 SFRSYM    DATA     BIT       TMR2CN0_TF2H
      000000C8H.3 SFRSYM    DATA     BIT       TMR2CN0_T2SPLIT
      000000D0H.6 SFRSYM    DATA     BIT       PSW_AC
      000000F8H   SFRSYM    DATA     BYTE      SPI0CN0
      000000B3H   SFRSYM    DATA     BYTE      HFO0CAL
      00000088H.5 SFRSYM    DATA     BIT       TCON_TF0
      00000098H   SFRSYM    DATA     BIT       SCON0_RI
      00000082H   SFRSYM    DATA     BYTE      DPL
      00000088H.7 SFRSYM    DATA     BIT       TCON_TF1
      00000099H   SFRSYM    DATA     BYTE      SBUF0
      00000087H   SFRSYM    DATA     BYTE      PCON0
      000000C3H   SFRSYM    DATA     BYTE      ADC0GTL
      000000C8H.6 SFRSYM    DATA     BIT       TMR2CN0_TF2L
      00000098H.1 SFRSYM    DATA     BIT       SCON0_TI
      000000E8H   SFRSYM    DATA     BIT       ADC0CN0_ADCM0
      000000D3H   SFRSYM    DATA     BYTE      SBUF1
      000000C6H   SFRSYM    DATA     BYTE      ADC0LTH
      00000088H   SFRSYM    DATA     BIT       TCON_IT0
      000000E8H.1 SFRSYM    DATA     BIT       ADC0CN0_ADCM1
      000000EFH   SFRSYM    DATA     BYTE      RSTSRC
      000000C8H.7 SFRSYM    DATA     BIT       TMR5CN0_TF5H
      000000C8H.3 SFRSYM    DATA     BIT       TMR5CN0_T5SPLIT
      00000088H.2 SFRSYM    DATA     BIT       TCON_IT1
      000000E8H.2 SFRSYM    DATA     BIT       ADC0CN0_ADCM2
      00000098H   SFRSYM    DATA     BYTE      SCON0
      000000E8H.3 SFRSYM    DATA     BIT       ADC0CN0_ADWINT
      000000B4H   SFRSYM    DATA     WORD      SBRL1
      000000E5H   SFRSYM    DATA     BYTE      SMOD1
      000000D2H   SFRSYM    DATA     BYTE      SCON1
      000000BAH   SFRSYM    DATA     BYTE      AMX0N
      000000E8H.4 SFRSYM    DATA     BIT       ADC0CN0_ADBUSY
      000000CEH   SFRSYM    DATA     BYTE      SMB0ADM
      000000C5H   SFRSYM    DATA     BYTE      ADC0LTL
      000000F8H.5 SFRSYM    DATA     BIT       SPI0CN0_MODF
      000000B8H.6 SFRSYM    DATA     BIT       IP_PSPI0
      000000CEH   SFRSYM    DATA     BYTE      SMB1ADM
      000000BBH   SFRSYM    DATA     BYTE      AMX0P
      000000C8H.6 SFRSYM    DATA     BIT       TMR5CN0_TF5L
      000000C8H   SFRSYM    DATA     BYTE      TMR2CN0
      00000091H   SFRSYM    DATA     BYTE      TMR3CN0
      00000091H   SFRSYM    DATA     BYTE      TMR4CN0
      000000C8H   SFRSYM    DATA     BYTE      TMR5CN0
      000000CFH   SFRSYM    DATA     BYTE      SMB0ADR
      00000088H.4 SFRSYM    DATA     BIT       TCON_TR0
LX51 LINKER/LOCATER V4.66.30.0                                                        07/27/2019  23:22:19  PAGE 159


      000000CFH   SFRSYM    DATA     BYTE      SMB1ADR
      000000C8H.4 SFRSYM    DATA     BIT       TMR2CN0_TF2CEN
      00000088H.6 SFRSYM    DATA     BIT       TCON_TR1
      000000C2H   SFRSYM    DATA     BYTE      SMB0DAT
      000000CDH   SFRSYM    DATA     BYTE      TMR2H
      000000A1H   SFRSYM    DATA     BYTE      SPI0CFG
      000000C2H   SFRSYM    DATA     BYTE      SMB1DAT
      00000095H   SFRSYM    DATA     BYTE      TMR3H
      00000095H   SFRSYM    DATA     BYTE      TMR4H
      000000CDH   SFRSYM    DATA     BYTE      TMR5H
      000000CCH   SFRSYM    DATA     BYTE      TMR2L
      000000F8H.7 SFRSYM    DATA     BIT       SPI0CN0_SPIF
      00000096H   SFRSYM    DATA     BYTE      USB0ADR
      00000094H   SFRSYM    DATA     BYTE      TMR3L
      000000A8H.7 SFRSYM    DATA     BIT       IE_EA
      00000094H   SFRSYM    DATA     BYTE      TMR4L
      00000097H   SFRSYM    DATA     BYTE      USB0DAT
      000000CCH   SFRSYM    DATA     BYTE      TMR5L
      000000B6H   SFRSYM    DATA     BYTE      FLSCL
      000000C8H.5 SFRSYM    DATA     BIT       TMR2CN0_TF2LEN
      000000F8H.6 SFRSYM    DATA     BIT       SPI0CN0_WCOL
      000000F8H.2 SFRSYM    DATA     BIT       SPI0CN0_NSSMD0
      000000D0H.7 SFRSYM    DATA     BIT       PSW_CY
      000000A3H   SFRSYM    DATA     BYTE      SPI0DAT
      000000F8H.3 SFRSYM    DATA     BIT       SPI0CN0_NSSMD1
      000000BDH   SFRSYM    DATA     WORD      ADC0
      000000B9H   SFRSYM    DATA     BYTE      SMBTC
      000000D0H   SFRSYM    DATA     BYTE      PSW
      000000C8H.5 SFRSYM    DATA     BIT       TMR5CN0_TF5LEN
      000000B7H   SFRSYM    DATA     BYTE      FLKEY

      01004DA6H   BLOCK     CODE     ---       LVL=0
      01004DA6H   LINE      CODE     ---       #19
      01004DA6H   LINE      CODE     ---       #20
      01004DA6H   LINE      CODE     ---       #21
      01004DACH   LINE      CODE     ---       #23
      01004DBFH   LINE      CODE     ---       #24
      01004DD6H   LINE      CODE     ---       #27
      01004DE5H   LINE      CODE     ---       #28
      01004DE5H   LINE      CODE     ---       #29
      01004DF3H   LINE      CODE     ---       #30
      01004DF8H   LINE      CODE     ---       #31
      01004DFAH   LINE      CODE     ---       #32
      01004DFCH   LINE      CODE     ---       #33
      01004E01H   LINE      CODE     ---       #34
      01004E01H   LINE      CODE     ---       #35
      01004E01H   LINE      CODE     ---       #36
      01004E01H   LINE      CODE     ---       #37
      01004E01H   LINE      CODE     ---       #39
      01004E03H   LINE      CODE     ---       #40
      ---         BLOCKEND  ---      ---       LVL=0

      01005A13H   BLOCK     CODE     ---       LVL=0
      00000007H   SYMBOL    DATA     BYTE      x
      01005A13H   LINE      CODE     ---       #42
      01005A13H   LINE      CODE     ---       #43
      01005A13H   LINE      CODE     ---       #44
      01005A13H   LINE      CODE     ---       #46
      01005A19H   LINE      CODE     ---       #47
      01005A1CH   LINE      CODE     ---       #49
      01005A22H   LINE      CODE     ---       #51
      ---         BLOCKEND  ---      ---       LVL=0
LX51 LINKER/LOCATER V4.66.30.0                                                        07/27/2019  23:22:19  PAGE 160



      01005B5BH   BLOCK     CODE     ---       LVL=0
      00000007H   SYMBOL    DATA     BYTE      x
      01005B5BH   LINE      CODE     ---       #54
      01005B5BH   LINE      CODE     ---       #55
      01005B5BH   LINE      CODE     ---       #56
      01005B5BH   LINE      CODE     ---       #58
      01005B61H   LINE      CODE     ---       #60
      ---         BLOCKEND  ---      ---       LVL=0

      01005964H   BLOCK     CODE     ---       LVL=0
      01005964H   LINE      CODE     ---       #64
      01005964H   LINE      CODE     ---       #65
      01005964H   LINE      CODE     ---       #66
      01005966H   LINE      CODE     ---       #67
      01005975H   LINE      CODE     ---       #68
      01005978H   LINE      CODE     ---       #69
      01005978H   LINE      CODE     ---       #70
      ---         BLOCKEND  ---      ---       LVL=0

      01005A25H   BLOCK     CODE     ---       LVL=0
      01005A25H   LINE      CODE     ---       #72
      01005A25H   LINE      CODE     ---       #73
      01005A25H   LINE      CODE     ---       #74
      01005A29H   LINE      CODE     ---       #75
      01005A33H   LINE      CODE     ---       #76
      01005A34H   LINE      CODE     ---       #77
      01005A36H   LINE      CODE     ---       #78
      01005A36H   LINE      CODE     ---       #79
      ---         BLOCKEND  ---      ---       LVL=0

      01005727H   BLOCK     CODE     ---       LVL=0
      01005727H   LINE      CODE     ---       #81
      01005727H   LINE      CODE     ---       #82
      01005727H   LINE      CODE     ---       #83
      0100573AH   LINE      CODE     ---       #84
      01005751H   LINE      CODE     ---       #85
      01005751H   LINE      CODE     ---       #86
      ---         BLOCKEND  ---      ---       LVL=0

      010055ABH   BLOCK     CODE     ---       LVL=0
      010055ABH   LINE      CODE     ---       #88
      010055ABH   LINE      CODE     ---       #89
      010055ABH   LINE      CODE     ---       #90
      010055BBH   LINE      CODE     ---       #92
      010055C7H   LINE      CODE     ---       #93
      010055CAH   LINE      CODE     ---       #94
      010055CAH   LINE      CODE     ---       #97
      010055D5H   LINE      CODE     ---       #98
      010055E0H   LINE      CODE     ---       #99
      010055E0H   LINE      CODE     ---       #100
      ---         BLOCKEND  ---      ---       LVL=0

      0100468AH   BLOCK     CODE     ---       LVL=0
      0100468AH   LINE      CODE     ---       #102
      0100468AH   LINE      CODE     ---       #103
      0100468AH   LINE      CODE     ---       #104
      01004696H   LINE      CODE     ---       #105
      0100469CH   LINE      CODE     ---       #106
      010046A8H   LINE      CODE     ---       #107
      010046AEH   LINE      CODE     ---       #108
      010046B5H   LINE      CODE     ---       #110
LX51 LINKER/LOCATER V4.66.30.0                                                        07/27/2019  23:22:19  PAGE 161


      010046C1H   LINE      CODE     ---       #111
      010046CDH   LINE      CODE     ---       #112
      010046D3H   LINE      CODE     ---       #114
      010046DFH   LINE      CODE     ---       #115
      010046EBH   LINE      CODE     ---       #116
      010046F1H   LINE      CODE     ---       #118
      010046FDH   LINE      CODE     ---       #119
      01004703H   LINE      CODE     ---       #120
      0100470FH   LINE      CODE     ---       #121
      01004715H   LINE      CODE     ---       #122
      0100471CH   LINE      CODE     ---       #123
      ---         BLOCKEND  ---      ---       LVL=0

      01005677H   BLOCK     CODE     ---       LVL=0
      01005677H   BLOCK     CODE     NEAR LAB  LVL=1
      00000007H   SYMBOL    DATA     BYTE      i
      ---         BLOCKEND  ---      ---       LVL=1
      01005677H   LINE      CODE     ---       #125
      01005677H   LINE      CODE     ---       #126
      01005677H   LINE      CODE     ---       #129
      01005679H   LINE      CODE     ---       #130
      01005690H   LINE      CODE     ---       #131
      010056A0H   LINE      CODE     ---       #132
      010056A4H   LINE      CODE     ---       #133
      ---         BLOCKEND  ---      ---       LVL=0

      01001E7AH   BLOCK     CODE     ---       LVL=0
      00000026H   SYMBOL    DATA     BYTE      mode
      00000027H   SYMBOL    DATA     BYTE      mask
      01001E7EH   BLOCK     CODE     NEAR LAB  LVL=1
      00000007H   SYMBOL    DATA     BYTE      w
      00000028H   SYMBOL    DATA     BYTE      i
      00000029H   SYMBOL    DATA     BYTE      j
      02000423H   SYMBOL    XDATA    ---       button_txt
      ---         BLOCKEND  ---      ---       LVL=1
      01001E7AH   LINE      CODE     ---       #136
      01001E7EH   LINE      CODE     ---       #137
      01001E7EH   LINE      CODE     ---       #144
      01001E8AH   LINE      CODE     ---       #145
      01001E99H   LINE      CODE     ---       #146
      01001EA8H   LINE      CODE     ---       #147
      01001EAAH   LINE      CODE     ---       #148
      01001EAFH   LINE      CODE     ---       #149
      01001EB3H   LINE      CODE     ---       #150
      01001EB3H   LINE      CODE     ---       #152
      01001ED1H   LINE      CODE     ---       #153
      01001ED1H   LINE      CODE     ---       #154
      01001EDEH   LINE      CODE     ---       #155
      01001EECH   LINE      CODE     ---       #156
      01001EECH   LINE      CODE     ---       #157
      01001EFAH   LINE      CODE     ---       #158
      01001F09H   LINE      CODE     ---       #159
      01001F09H   LINE      CODE     ---       #160
      01001F18H   LINE      CODE     ---       #162
      01001F1BH   LINE      CODE     ---       #164
      01001F1EH   LINE      CODE     ---       #165
      01001F1EH   LINE      CODE     ---       #167
      01001F1EH   LINE      CODE     ---       #168
      01001F2DH   LINE      CODE     ---       #169
      01001F2DH   LINE      CODE     ---       #170
      01001F30H   LINE      CODE     ---       #171
      01001F30H   LINE      CODE     ---       #173
LX51 LINKER/LOCATER V4.66.30.0                                                        07/27/2019  23:22:19  PAGE 162


      01001F30H   LINE      CODE     ---       #174
      01001F3FH   LINE      CODE     ---       #175
      01001F4EH   LINE      CODE     ---       #176
      01001F5DH   LINE      CODE     ---       #177
      01001F69H   LINE      CODE     ---       #178
      01001F6CH   LINE      CODE     ---       #179
      01001F6CH   LINE      CODE     ---       #181
      01001F6CH   LINE      CODE     ---       #182
      01001F7BH   LINE      CODE     ---       #183
      01001F8AH   LINE      CODE     ---       #184
      01001F99H   LINE      CODE     ---       #185
      01001FA5H   LINE      CODE     ---       #186
      01001FA7H   LINE      CODE     ---       #187
      01001FA7H   LINE      CODE     ---       #189
      01001FA7H   LINE      CODE     ---       #190
      01001FA7H   LINE      CODE     ---       #191
      01001FB6H   LINE      CODE     ---       #192
      01001FC5H   LINE      CODE     ---       #193
      01001FD4H   LINE      CODE     ---       #194
      01001FE0H   LINE      CODE     ---       #195
      01001FE2H   LINE      CODE     ---       #196
      01001FE2H   LINE      CODE     ---       #198
      01001FE2H   LINE      CODE     ---       #199
      01001FE5H   LINE      CODE     ---       #200
      01001FF7H   LINE      CODE     ---       #201
      01002008H   LINE      CODE     ---       #202
      0100200FH   LINE      CODE     ---       #203
      01002014H   LINE      CODE     ---       #204
      01002023H   LINE      CODE     ---       #205
      01002023H   LINE      CODE     ---       #206
      01002023H   LINE      CODE     ---       #207
      01002023H   LINE      CODE     ---       #208
      01002023H   LINE      CODE     ---       #210
      01002026H   LINE      CODE     ---       #211
      01002038H   LINE      CODE     ---       #212
      01002053H   LINE      CODE     ---       #213
      01002053H   LINE      CODE     ---       #214
      0100205AH   LINE      CODE     ---       #216
      01002061H   LINE      CODE     ---       #217
      01002071H   LINE      CODE     ---       #219
      0100208CH   LINE      CODE     ---       #220
      01002096H   LINE      CODE     ---       #221
      010020A6H   LINE      CODE     ---       #223
      010020ADH   LINE      CODE     ---       #224
      010020BDH   LINE      CODE     ---       #226
      010020D8H   LINE      CODE     ---       #227
      010020E2H   LINE      CODE     ---       #228
      010020F2H   LINE      CODE     ---       #231
      010020F8H   LINE      CODE     ---       #232
      010020F8H   LINE      CODE     ---       #233
      0100210AH   LINE      CODE     ---       #234
      01002118H   LINE      CODE     ---       #235
      0100211CH   LINE      CODE     ---       #236
      01002123H   LINE      CODE     ---       #238
      01002129H   LINE      CODE     ---       #239
      01002129H   LINE      CODE     ---       #240
      0100213BH   LINE      CODE     ---       #241
      01002149H   LINE      CODE     ---       #242
      0100214DH   LINE      CODE     ---       #243
      01002154H   LINE      CODE     ---       #244
      ---         BLOCKEND  ---      ---       LVL=0

LX51 LINKER/LOCATER V4.66.30.0                                                        07/27/2019  23:22:19  PAGE 163


      01004A51H   BLOCK     CODE     ---       LVL=0
      00000026H   SYMBOL    DATA     BYTE      active_idx
      01004A53H   BLOCK     CODE     NEAR LAB  LVL=1
      00000027H   SYMBOL    DATA     BYTE      h
      00000028H   SYMBOL    DATA     BYTE      i
      00000029H   SYMBOL    DATA     BYTE      x
      0000002AH   SYMBOL    DATA     BYTE      y
      0000002BH   SYMBOL    DATA     BYTE      s
      0000002CH   SYMBOL    DATA     BYTE      count
      ---         BLOCKEND  ---      ---       LVL=1
      01004A51H   LINE      CODE     ---       #246
      01004A53H   LINE      CODE     ---       #247
      01004A53H   LINE      CODE     ---       #253
      01004A5DH   LINE      CODE     ---       #255
      01004A65H   LINE      CODE     ---       #256
      01004A72H   LINE      CODE     ---       #257
      01004A74H   LINE      CODE     ---       #259
      01004A7EH   LINE      CODE     ---       #260
      01004A89H   LINE      CODE     ---       #262
      01004A90H   LINE      CODE     ---       #263
      01004A9CH   LINE      CODE     ---       #265
      01004AA2H   LINE      CODE     ---       #267
      01004AA7H   LINE      CODE     ---       #268
      01004AB0H   LINE      CODE     ---       #269
      01004AB0H   LINE      CODE     ---       #271
      01004AB7H   LINE      CODE     ---       #272
      01004ABAH   LINE      CODE     ---       #273
      01004ABAH   LINE      CODE     ---       #274
      01004ABEH   LINE      CODE     ---       #276
      01004AC7H   LINE      CODE     ---       #278
      ---         BLOCKEND  ---      ---       LVL=0

      ---         MODULE    ---      ---       MENU_0_FN
      020002F2H   PUBLIC    XDATA    ---       rotdst_fb
      02000251H   PUBLIC    XDATA    ---       rotsrc_fb
      02000245H   PUBLIC    XDATA    ---       rotdst
      02000239H   PUBLIC    XDATA    ---       rotsrc
      0000008CH   PUBLIC    IDATA    BYTE      wiggle
      01003BB5H   PUBLIC    CODE     ---       err_namelong_3
      01003B9BH   PUBLIC    CODE     ---       err_namelong_2
      01003B8DH   PUBLIC    CODE     ---       err_namelong_1
      01003B6EH   PUBLIC    CODE     ---       err_namewide_3
      01003B55H   PUBLIC    CODE     ---       err_namewide_2
      01003B47H   PUBLIC    CODE     ---       err_namewide_1
      0100553AH   PUBLIC    CODE     ---       _menu_0_enter
      010034BDH   PUBLIC    CODE     ---       _menu_0_disp
      01000AF5H   PUBLIC    CODE     ---       _menu_none_disp
      000000A2H   SFRSYM    DATA     BYTE      SPI0CKR
      00000080H   SFRSYM    DATA     BYTE      P0
      000000D0H.2 SFRSYM    DATA     BIT       PSW_OV
      000000B1H   SFRSYM    DATA     BYTE      XOSC0CN
      00000090H   SFRSYM    DATA     BYTE      P1
      000000A0H   SFRSYM    DATA     BYTE      P2
      000000B0H   SFRSYM    DATA     BYTE      P3
      000000BCH   SFRSYM    DATA     BYTE      ADC0CF
      000000C8H   SFRSYM    DATA     BIT       TMR2CN0_T2XCLK
      000000C7H   SFRSYM    DATA     BYTE      P4
      000000C0H.7 SFRSYM    DATA     BIT       SMB0CN0_MASTER
      000000F9H   SFRSYM    DATA     WORD      PCA0
      000000E6H   SFRSYM    DATA     BYTE      EIE1
      000000C0H.7 SFRSYM    DATA     BIT       SMB1CN0_MASTER
      000000C0H.1 SFRSYM    DATA     BIT       SMB0CN0_ACK
LX51 LINKER/LOCATER V4.66.30.0                                                        07/27/2019  23:22:19  PAGE 164


      000000D7H   SFRSYM    DATA     BYTE      USB0XCN
      000000E7H   SFRSYM    DATA     BYTE      EIE2
      000000C0H.1 SFRSYM    DATA     BIT       SMB1CN0_ACK
      0000008FH   SFRSYM    DATA     BYTE      PSCTL
      000000E4H   SFRSYM    DATA     BYTE      IT01CF
      000000C8H   SFRSYM    DATA     BIT       TMR5CN0_T5XCLK
      000000C0H.6 SFRSYM    DATA     BIT       SMB0CN0_TXMODE
      000000C0H.6 SFRSYM    DATA     BIT       SMB1CN0_TXMODE
      000000BFH   SFRSYM    DATA     BYTE      SFRPAGE
      000000A4H   SFRSYM    DATA     BYTE      P0MDOUT
      000000A5H   SFRSYM    DATA     BYTE      P1MDOUT
      000000E8H.5 SFRSYM    DATA     BIT       ADC0CN0_ADINT
      000000CBH   SFRSYM    DATA     BYTE      TMR2RLH
      000000A6H   SFRSYM    DATA     BYTE      P2MDOUT
      000000A8H   SFRSYM    DATA     BYTE      IE
      00000093H   SFRSYM    DATA     BYTE      TMR3RLH
      000000A7H   SFRSYM    DATA     BYTE      P3MDOUT
      00000093H   SFRSYM    DATA     BYTE      TMR4RLH
      000000AEH   SFRSYM    DATA     BYTE      P4MDOUT
      000000F6H   SFRSYM    DATA     BYTE      EIP1
      000000CBH   SFRSYM    DATA     BYTE      TMR5RLH
      000000F7H   SFRSYM    DATA     BYTE      EIP2
      00000098H.2 SFRSYM    DATA     BIT       SCON0_RB8
      000000CAH   SFRSYM    DATA     BYTE      TMR2RLL
      000000FCH   SFRSYM    DATA     BYTE      PCA0CPH0
      00000092H   SFRSYM    DATA     BYTE      TMR3RLL
      000000EAH   SFRSYM    DATA     BYTE      PCA0CPH1
      00000098H.3 SFRSYM    DATA     BIT       SCON0_TB8
      000000F0H   SFRSYM    DATA     BIT       B_B0
      00000082H   SFRSYM    DATA     WORD      DP
      00000092H   SFRSYM    DATA     BYTE      TMR4RLL
      000000ECH   SFRSYM    DATA     BYTE      PCA0CPH2
      000000F0H.1 SFRSYM    DATA     BIT       B_B1
      000000C3H   SFRSYM    DATA     WORD      ADC0GT
      000000CAH   SFRSYM    DATA     BYTE      TMR5RLL
      000000EEH   SFRSYM    DATA     BYTE      PCA0CPH3
      000000F0H.2 SFRSYM    DATA     BIT       B_B2
      000000FBH   SFRSYM    DATA     BYTE      PCA0CPL0
      000000FEH   SFRSYM    DATA     BYTE      PCA0CPH4
      00000085H   SFRSYM    DATA     BYTE      EMI0CF
      000000F0H.3 SFRSYM    DATA     BIT       B_B3
      000000D9H   SFRSYM    DATA     BYTE      PCA0MD
      000000DAH   SFRSYM    DATA     BYTE      PCA0CPM0
      000000E9H   SFRSYM    DATA     BYTE      PCA0CPL1
      000000F0H.4 SFRSYM    DATA     BIT       B_B4
      000000DBH   SFRSYM    DATA     BYTE      PCA0CPM1
      000000EBH   SFRSYM    DATA     BYTE      PCA0CPL2
      000000F0H.5 SFRSYM    DATA     BIT       B_B5
      000000DCH   SFRSYM    DATA     BYTE      PCA0CPM2
      000000EDH   SFRSYM    DATA     BYTE      PCA0CPL3
      000000B8H   SFRSYM    DATA     BYTE      IP
      000000F0H.6 SFRSYM    DATA     BIT       B_B6
      000000C5H   SFRSYM    DATA     WORD      ADC0LT
      000000DDH   SFRSYM    DATA     BYTE      PCA0CPM3
      000000FDH   SFRSYM    DATA     BYTE      PCA0CPL4
      00000098H.5 SFRSYM    DATA     BIT       SCON0_MCE
      000000F0H.7 SFRSYM    DATA     BIT       B_B7
      000000DEH   SFRSYM    DATA     BYTE      PCA0CPM4
      000000E1H   SFRSYM    DATA     BYTE      XBR0
      000000C1H   SFRSYM    DATA     BYTE      SMB0CF
      000000E2H   SFRSYM    DATA     BYTE      XBR1
      000000C1H   SFRSYM    DATA     BYTE      SMB1CF
LX51 LINKER/LOCATER V4.66.30.0                                                        07/27/2019  23:22:19  PAGE 165


      000000AFH   SFRSYM    DATA     BYTE      PFE0CN
      000000AAH   SFRSYM    DATA     BYTE      EMI0CN
      000000C0H.5 SFRSYM    DATA     BIT       SMB0CN0_STA
      000000E3H   SFRSYM    DATA     BYTE      XBR2
      000000C0H.5 SFRSYM    DATA     BIT       SMB1CN0_STA
      000000E0H   SFRSYM    DATA     BIT       ACC_ACC0
      000000D1H   SFRSYM    DATA     BYTE      REF0CN
      000000B2H   SFRSYM    DATA     BYTE      HFO0CN
      0000008EH   SFRSYM    DATA     BYTE      CKCON0
      000000E0H.1 SFRSYM    DATA     BIT       ACC_ACC1
      000000E4H   SFRSYM    DATA     BYTE      CKCON1
      000000C8H.2 SFRSYM    DATA     BIT       TMR2CN0_TR2
      000000E0H.2 SFRSYM    DATA     BIT       ACC_ACC2
      000000E0H.3 SFRSYM    DATA     BIT       ACC_ACC3
      00000081H   SFRSYM    DATA     BYTE      SP
      0000009DH   SFRSYM    DATA     BYTE      CMP0MD
      000000E0H.4 SFRSYM    DATA     BIT       ACC_ACC4
      00000086H   SFRSYM    DATA     BYTE      LFO0CN
      00000084H   SFRSYM    DATA     BYTE      EMI0TC
      0000009CH   SFRSYM    DATA     BYTE      CMP1MD
      000000D8H   SFRSYM    DATA     BIT       PCA0CN0_CCF0
      000000E0H.5 SFRSYM    DATA     BIT       ACC_ACC5
      000000D8H.1 SFRSYM    DATA     BIT       PCA0CN0_CCF1
      000000E0H.6 SFRSYM    DATA     BIT       ACC_ACC6
      000000CCH   SFRSYM    DATA     WORD      TMR2
      000000D8H.2 SFRSYM    DATA     BIT       PCA0CN0_CCF2
      000000E0H.7 SFRSYM    DATA     BIT       ACC_ACC7
      00000094H   SFRSYM    DATA     WORD      TMR3
      000000C8H.2 SFRSYM    DATA     BIT       TMR5CN0_TR5
      000000D8H.3 SFRSYM    DATA     BIT       PCA0CN0_CCF3
      00000094H   SFRSYM    DATA     WORD      TMR4
      000000ACH   SFRSYM    DATA     BYTE      SBCON1
      000000D8H.4 SFRSYM    DATA     BIT       PCA0CN0_CCF4
      000000CCH   SFRSYM    DATA     WORD      TMR5
      000000C0H.3 SFRSYM    DATA     BIT       SMB0CN0_ACKRQ
      000000FFH   SFRSYM    DATA     BYTE      VDM0CN
      000000F1H   SFRSYM    DATA     BYTE      P0MDIN
      000000C0H.3 SFRSYM    DATA     BIT       SMB1CN0_ACKRQ
      00000098H.4 SFRSYM    DATA     BIT       SCON0_REN
      000000F2H   SFRSYM    DATA     BYTE      P1MDIN
      000000F3H   SFRSYM    DATA     BYTE      P2MDIN
      000000C0H.4 SFRSYM    DATA     BIT       SMB0CN0_STO
      000000F4H   SFRSYM    DATA     BYTE      P3MDIN
      000000C0H.4 SFRSYM    DATA     BIT       SMB1CN0_STO
      000000B5H   SFRSYM    DATA     BYTE      SBRLH1
      000000F5H   SFRSYM    DATA     BYTE      P4MDIN
      000000D0H.3 SFRSYM    DATA     BIT       PSW_RS0
      000000D8H.7 SFRSYM    DATA     BIT       PCA0CN0_CF
      000000F8H.4 SFRSYM    DATA     BIT       SPI0CN0_RXOVRN
      000000D0H.4 SFRSYM    DATA     BIT       PSW_RS1
      000000B4H   SFRSYM    DATA     BYTE      SBRLL1
      000000E8H.7 SFRSYM    DATA     BIT       ADC0CN0_ADEN
      00000089H   SFRSYM    DATA     BYTE      TMOD
      00000088H   SFRSYM    DATA     BYTE      TCON
      000000D0H   SFRSYM    DATA     BIT       PSW_PARITY
      000000A8H.4 SFRSYM    DATA     BIT       IE_ES0
      0000009FH   SFRSYM    DATA     BYTE      CMP0MX
      000000A8H.1 SFRSYM    DATA     BIT       IE_ET0
      0000009EH   SFRSYM    DATA     BYTE      CMP1MX
      000000A8H.3 SFRSYM    DATA     BIT       IE_ET1
      000000D4H   SFRSYM    DATA     BYTE      P0SKIP
      000000C8H.1 SFRSYM    DATA     BIT       TMR2CN0_T2CSS
LX51 LINKER/LOCATER V4.66.30.0                                                        07/27/2019  23:22:19  PAGE 166


      000000A8H.5 SFRSYM    DATA     BIT       IE_ET2
      000000D5H   SFRSYM    DATA     BYTE      P1SKIP
      000000D6H   SFRSYM    DATA     BYTE      P2SKIP
      000000E8H   SFRSYM    DATA     BYTE      ADC0CN0
      000000A8H   SFRSYM    DATA     BIT       IE_EX0
      000000DFH   SFRSYM    DATA     BYTE      P3SKIP
      000000D8H.6 SFRSYM    DATA     BIT       PCA0CN0_CR
      000000A8H.2 SFRSYM    DATA     BIT       IE_EX1
      00000098H.7 SFRSYM    DATA     BIT       SCON0_SMODE
      000000A9H   SFRSYM    DATA     BYTE      CLKSEL
      000000F8H   SFRSYM    DATA     BIT       SPI0CN0_SPIEN
      000000F0H   SFRSYM    DATA     BYTE      B
      000000BEH   SFRSYM    DATA     BYTE      ADC0H
      000000E8H.6 SFRSYM    DATA     BIT       ADC0CN0_ADTM
      000000CAH   SFRSYM    DATA     WORD      TMR2RL
      000000BDH   SFRSYM    DATA     BYTE      ADC0L
      00000092H   SFRSYM    DATA     WORD      TMR3RL
      00000092H   SFRSYM    DATA     WORD      TMR4RL
      000000D8H   SFRSYM    DATA     BYTE      PCA0CN0
      000000E0H   SFRSYM    DATA     BYTE      ACC
      000000CAH   SFRSYM    DATA     WORD      TMR5RL
      000000FBH   SFRSYM    DATA     WORD      PCA0CP0
      000000E9H   SFRSYM    DATA     WORD      PCA0CP1
      000000EBH   SFRSYM    DATA     WORD      PCA0CP2
      000000EDH   SFRSYM    DATA     WORD      PCA0CP3
      0000008CH   SFRSYM    DATA     BYTE      TH0
      000000B8H.4 SFRSYM    DATA     BIT       IP_PS0
      000000FDH   SFRSYM    DATA     WORD      PCA0CP4
      0000008DH   SFRSYM    DATA     BYTE      TH1
      000000FAH   SFRSYM    DATA     BYTE      PCA0H
      000000B8H.1 SFRSYM    DATA     BIT       IP_PT0
      000000B8H.3 SFRSYM    DATA     BIT       IP_PT1
      000000C0H.2 SFRSYM    DATA     BIT       SMB0CN0_ARBLOST
      000000B8H.5 SFRSYM    DATA     BIT       IP_PT2
      0000008AH   SFRSYM    DATA     BYTE      TL0
      000000F8H.1 SFRSYM    DATA     BIT       SPI0CN0_TXBMT
      000000C0H.2 SFRSYM    DATA     BIT       SMB1CN0_ARBLOST
      000000D0H.5 SFRSYM    DATA     BIT       PSW_F0
      000000A8H.6 SFRSYM    DATA     BIT       IE_ESPI0
      0000008BH   SFRSYM    DATA     BYTE      TL1
      000000F9H   SFRSYM    DATA     BYTE      PCA0L
      000000C0H   SFRSYM    DATA     BIT       SMB0CN0_SI
      000000D0H.1 SFRSYM    DATA     BIT       PSW_F1
      00000080H   SFRSYM    DATA     BIT       P0_B0
      000000B8H   SFRSYM    DATA     BIT       IP_PX0
      000000C9H   SFRSYM    DATA     BYTE      REG01CN
      000000C0H   SFRSYM    DATA     BIT       SMB1CN0_SI
      00000090H   SFRSYM    DATA     BIT       P1_B0
      00000080H.1 SFRSYM    DATA     BIT       P0_B1
      000000B8H.2 SFRSYM    DATA     BIT       IP_PX1
      0000009BH   SFRSYM    DATA     BYTE      CMP0CN0
      00000088H.1 SFRSYM    DATA     BIT       TCON_IE0
      000000A0H   SFRSYM    DATA     BIT       P2_B0
      00000090H.1 SFRSYM    DATA     BIT       P1_B1
      00000080H.2 SFRSYM    DATA     BIT       P0_B2
      0000009AH   SFRSYM    DATA     BYTE      CMP1CN0
      00000088H.3 SFRSYM    DATA     BIT       TCON_IE1
      000000B0H   SFRSYM    DATA     BIT       P3_B0
      000000A0H.1 SFRSYM    DATA     BIT       P2_B1
      00000090H.2 SFRSYM    DATA     BIT       P1_B2
      00000080H.3 SFRSYM    DATA     BIT       P0_B3
      000000C0H   SFRSYM    DATA     BYTE      SMB0CN0
LX51 LINKER/LOCATER V4.66.30.0                                                        07/27/2019  23:22:19  PAGE 167


      000000B0H.1 SFRSYM    DATA     BIT       P3_B1
      000000A0H.2 SFRSYM    DATA     BIT       P2_B2
      00000090H.3 SFRSYM    DATA     BIT       P1_B3
      00000080H.4 SFRSYM    DATA     BIT       P0_B4
      000000C0H   SFRSYM    DATA     BYTE      SMB1CN0
      000000B0H.2 SFRSYM    DATA     BIT       P3_B2
      000000A0H.3 SFRSYM    DATA     BIT       P2_B3
      00000090H.4 SFRSYM    DATA     BIT       P1_B4
      00000080H.5 SFRSYM    DATA     BIT       P0_B5
      000000B0H.3 SFRSYM    DATA     BIT       P3_B3
      000000A0H.4 SFRSYM    DATA     BIT       P2_B4
      00000090H.5 SFRSYM    DATA     BIT       P1_B5
      00000080H.6 SFRSYM    DATA     BIT       P0_B6
      000000B0H.4 SFRSYM    DATA     BIT       P3_B4
      000000A0H.5 SFRSYM    DATA     BIT       P2_B5
      00000090H.6 SFRSYM    DATA     BIT       P1_B6
      00000080H.7 SFRSYM    DATA     BIT       P0_B7
      000000B0H.5 SFRSYM    DATA     BIT       P3_B5
      000000A0H.6 SFRSYM    DATA     BIT       P2_B6
      00000090H.7 SFRSYM    DATA     BIT       P1_B7
      000000B0H.6 SFRSYM    DATA     BIT       P3_B6
      000000A0H.7 SFRSYM    DATA     BIT       P2_B7
      000000B0H.7 SFRSYM    DATA     BIT       P3_B7
      00000083H   SFRSYM    DATA     BYTE      DPH
      000000C4H   SFRSYM    DATA     BYTE      ADC0GTH
      000000C8H.7 SFRSYM    DATA     BIT       TMR2CN0_TF2H
      000000C8H.3 SFRSYM    DATA     BIT       TMR2CN0_T2SPLIT
      000000D0H.6 SFRSYM    DATA     BIT       PSW_AC
      000000F8H   SFRSYM    DATA     BYTE      SPI0CN0
      000000B3H   SFRSYM    DATA     BYTE      HFO0CAL
      00000088H.5 SFRSYM    DATA     BIT       TCON_TF0
      00000098H   SFRSYM    DATA     BIT       SCON0_RI
      00000082H   SFRSYM    DATA     BYTE      DPL
      00000088H.7 SFRSYM    DATA     BIT       TCON_TF1
      00000099H   SFRSYM    DATA     BYTE      SBUF0
      00000087H   SFRSYM    DATA     BYTE      PCON0
      000000C3H   SFRSYM    DATA     BYTE      ADC0GTL
      000000C8H.6 SFRSYM    DATA     BIT       TMR2CN0_TF2L
      00000098H.1 SFRSYM    DATA     BIT       SCON0_TI
      000000E8H   SFRSYM    DATA     BIT       ADC0CN0_ADCM0
      000000D3H   SFRSYM    DATA     BYTE      SBUF1
      000000C6H   SFRSYM    DATA     BYTE      ADC0LTH
      00000088H   SFRSYM    DATA     BIT       TCON_IT0
      000000E8H.1 SFRSYM    DATA     BIT       ADC0CN0_ADCM1
      000000EFH   SFRSYM    DATA     BYTE      RSTSRC
      000000C8H.7 SFRSYM    DATA     BIT       TMR5CN0_TF5H
      000000C8H.3 SFRSYM    DATA     BIT       TMR5CN0_T5SPLIT
      00000088H.2 SFRSYM    DATA     BIT       TCON_IT1
      000000E8H.2 SFRSYM    DATA     BIT       ADC0CN0_ADCM2
      00000098H   SFRSYM    DATA     BYTE      SCON0
      000000E8H.3 SFRSYM    DATA     BIT       ADC0CN0_ADWINT
      000000B4H   SFRSYM    DATA     WORD      SBRL1
      000000E5H   SFRSYM    DATA     BYTE      SMOD1
      000000D2H   SFRSYM    DATA     BYTE      SCON1
      000000BAH   SFRSYM    DATA     BYTE      AMX0N
      000000E8H.4 SFRSYM    DATA     BIT       ADC0CN0_ADBUSY
      000000CEH   SFRSYM    DATA     BYTE      SMB0ADM
      000000C5H   SFRSYM    DATA     BYTE      ADC0LTL
      000000F8H.5 SFRSYM    DATA     BIT       SPI0CN0_MODF
      000000B8H.6 SFRSYM    DATA     BIT       IP_PSPI0
      000000CEH   SFRSYM    DATA     BYTE      SMB1ADM
      000000BBH   SFRSYM    DATA     BYTE      AMX0P
LX51 LINKER/LOCATER V4.66.30.0                                                        07/27/2019  23:22:19  PAGE 168


      000000C8H.6 SFRSYM    DATA     BIT       TMR5CN0_TF5L
      000000C8H   SFRSYM    DATA     BYTE      TMR2CN0
      00000091H   SFRSYM    DATA     BYTE      TMR3CN0
      00000091H   SFRSYM    DATA     BYTE      TMR4CN0
      000000C8H   SFRSYM    DATA     BYTE      TMR5CN0
      000000CFH   SFRSYM    DATA     BYTE      SMB0ADR
      00000088H.4 SFRSYM    DATA     BIT       TCON_TR0
      000000CFH   SFRSYM    DATA     BYTE      SMB1ADR
      000000C8H.4 SFRSYM    DATA     BIT       TMR2CN0_TF2CEN
      00000088H.6 SFRSYM    DATA     BIT       TCON_TR1
      000000C2H   SFRSYM    DATA     BYTE      SMB0DAT
      000000CDH   SFRSYM    DATA     BYTE      TMR2H
      000000A1H   SFRSYM    DATA     BYTE      SPI0CFG
      000000C2H   SFRSYM    DATA     BYTE      SMB1DAT
      00000095H   SFRSYM    DATA     BYTE      TMR3H
      00000095H   SFRSYM    DATA     BYTE      TMR4H
      000000CDH   SFRSYM    DATA     BYTE      TMR5H
      000000CCH   SFRSYM    DATA     BYTE      TMR2L
      000000F8H.7 SFRSYM    DATA     BIT       SPI0CN0_SPIF
      00000096H   SFRSYM    DATA     BYTE      USB0ADR
      00000094H   SFRSYM    DATA     BYTE      TMR3L
      000000A8H.7 SFRSYM    DATA     BIT       IE_EA
      00000094H   SFRSYM    DATA     BYTE      TMR4L
      00000097H   SFRSYM    DATA     BYTE      USB0DAT
      000000CCH   SFRSYM    DATA     BYTE      TMR5L
      000000B6H   SFRSYM    DATA     BYTE      FLSCL
      000000C8H.5 SFRSYM    DATA     BIT       TMR2CN0_TF2LEN
      000000F8H.6 SFRSYM    DATA     BIT       SPI0CN0_WCOL
      000000F8H.2 SFRSYM    DATA     BIT       SPI0CN0_NSSMD0
      000000D0H.7 SFRSYM    DATA     BIT       PSW_CY
      000000A3H   SFRSYM    DATA     BYTE      SPI0DAT
      000000F8H.3 SFRSYM    DATA     BIT       SPI0CN0_NSSMD1
      000000BDH   SFRSYM    DATA     WORD      ADC0
      000000B9H   SFRSYM    DATA     BYTE      SMBTC
      000000D0H   SFRSYM    DATA     BYTE      PSW
      000000C8H.5 SFRSYM    DATA     BIT       TMR5CN0_TF5LEN
      000000B7H   SFRSYM    DATA     BYTE      FLKEY
      010058F5H   SYMBOL    CODE     ---       _menu_none_set_halfwidth
      01005847H   SYMBOL    CODE     ---       _menu_none_set_flipmirror
      01005501H   SYMBOL    CODE     ---       menu_none_init
      01005240H   SYMBOL    CODE     ---       _menu_none_print_error

      01005501H   BLOCK     CODE     ---       LVL=0
      01005501H   LINE      CODE     ---       #38
      01005501H   LINE      CODE     ---       #39
      01005501H   LINE      CODE     ---       #40
      0100550BH   LINE      CODE     ---       #41
      01005515H   LINE      CODE     ---       #43
      0100551FH   LINE      CODE     ---       #44
      01005527H   LINE      CODE     ---       #46
      01005531H   LINE      CODE     ---       #47
      01005539H   LINE      CODE     ---       #48
      ---         BLOCKEND  ---      ---       LVL=0

      010058F5H   BLOCK     CODE     ---       LVL=0
      00000006H   SYMBOL    DATA     ---       dst
      010058F5H   LINE      CODE     ---       #50
      010058F5H   LINE      CODE     ---       #51
      010058F5H   LINE      CODE     ---       #52
      010058FCH   LINE      CODE     ---       #53
      01005904H   LINE      CODE     ---       #54
      01005905H   LINE      CODE     ---       #55
LX51 LINKER/LOCATER V4.66.30.0                                                        07/27/2019  23:22:19  PAGE 169


      0100590DH   LINE      CODE     ---       #56
      0100590DH   LINE      CODE     ---       #57
      ---         BLOCKEND  ---      ---       LVL=0

      01005847H   BLOCK     CODE     ---       LVL=0
      00000007H   SYMBOL    DATA     BYTE      flip_flag
      01005847H   LINE      CODE     ---       #59
      01005847H   LINE      CODE     ---       #60
      01005847H   LINE      CODE     ---       #61
      0100584EH   LINE      CODE     ---       #62
      01005853H   LINE      CODE     ---       #63
      01005853H   LINE      CODE     ---       #64
      0100585CH   LINE      CODE     ---       #68
      0100585EH   LINE      CODE     ---       #69
      01005860H   LINE      CODE     ---       #70
      01005865H   LINE      CODE     ---       #71
      01005865H   LINE      CODE     ---       #72
      ---         BLOCKEND  ---      ---       LVL=0

      01005240H   BLOCK     CODE     ---       LVL=0
      0000002AH   SYMBOL    DATA     ---       err1
      0000002DH   SYMBOL    DATA     ---       err2
      00000030H   SYMBOL    DATA     ---       err3
      01005240H   LINE      CODE     ---       #83
      01005246H   LINE      CODE     ---       #84
      01005246H   LINE      CODE     ---       #85
      0100524CH   LINE      CODE     ---       #86
      0100525CH   LINE      CODE     ---       #87
      01005263H   LINE      CODE     ---       #88
      01005273H   LINE      CODE     ---       #89
      0100527AH   LINE      CODE     ---       #90
      0100528AH   LINE      CODE     ---       #92
      ---         BLOCKEND  ---      ---       LVL=0

      01000AF5H   BLOCK     CODE     ---       LVL=0
      00000007H   SYMBOL    DATA     BYTE      idx
      01000AF5H   BLOCK     CODE     NEAR LAB  LVL=1
      00000022H   SYMBOL    DATA     BYTE      i
      00000023H   SYMBOL    DATA     BYTE      j
      00000024H   SYMBOL    DATA     BYTE      o
      00000025H   SYMBOL    DATA     WORD      w
      00000027H   SYMBOL    DATA     CHAR      left
      00000028H   SYMBOL    DATA     CHAR      top
      00000029H   SYMBOL    DATA     CHAR      rot
      02000413H   SYMBOL    XDATA    ---       txt
      01000C52H   SYMBOL    CODE     ---       MENU_0_DISP_CHAR_ROTATE
      ---         BLOCKEND  ---      ---       LVL=1
      01000AF5H   LINE      CODE     ---       #94
      01000AF5H   LINE      CODE     ---       #95
      01000AF5H   LINE      CODE     ---       #105
      01000AF5H   LINE      CODE     ---       #107
      01000AF8H   LINE      CODE     ---       #110
      01000AFFH   LINE      CODE     ---       #111
      01000B08H   LINE      CODE     ---       #113
      01000B47H   LINE      CODE     ---       #118
      01000B5AH   LINE      CODE     ---       #119
      01000B75H   LINE      CODE     ---       #120
      01000B75H   LINE      CODE     ---       #122
      01000B87H   LINE      CODE     ---       #123
      01000BABH   LINE      CODE     ---       #126
      01000BB6H   LINE      CODE     ---       #129
      01000BD2H   LINE      CODE     ---       #130
LX51 LINKER/LOCATER V4.66.30.0                                                        07/27/2019  23:22:19  PAGE 170


      01000BD2H   LINE      CODE     ---       #131
      01000BD7H   LINE      CODE     ---       #133
      01000BDEH   LINE      CODE     ---       #134
      01000BE7H   LINE      CODE     ---       #136
      01000BEEH   LINE      CODE     ---       #137
      01000C15H   LINE      CODE     ---       #138
      01000C18H   LINE      CODE     ---       #139
      01000C18H   LINE      CODE     ---       #141
      01000C18H   LINE      CODE     ---       #142
      01000C1DH   LINE      CODE     ---       #144
      01000C20H   LINE      CODE     ---       #146
      01000C22H   LINE      CODE     ---       #147
      01000C22H   LINE      CODE     ---       #148
      01000C22H   LINE      CODE     ---       #149
      01000C27H   LINE      CODE     ---       #152
      01000C2CH   LINE      CODE     ---       #153
      01000C3CH   LINE      CODE     ---       #155
      01000C4BH   LINE      CODE     ---       #157
      01000C4DH   LINE      CODE     ---       #158
      01000C4DH   LINE      CODE     ---       #159
      01000C4DH   LINE      CODE     ---       #160
      01000C52H   LINE      CODE     ---       #162
      01000C52H   LINE      CODE     ---       #164
      01000C5BH   LINE      CODE     ---       #165
      01000C69H   LINE      CODE     ---       #168
      01000C74H   LINE      CODE     ---       #171
      01000C7BH   LINE      CODE     ---       #172
      01000C82H   LINE      CODE     ---       #173
      01000C9DH   LINE      CODE     ---       #175
      01000C9DH   LINE      CODE     ---       #176
      01000CA3H   LINE      CODE     ---       #177
      01000CA3H   LINE      CODE     ---       #178
      01000CA5H   LINE      CODE     ---       #179
      01000CABH   LINE      CODE     ---       #180
      01000CABH   LINE      CODE     ---       #183
      01000CB4H   LINE      CODE     ---       #184
      01000CB9H   LINE      CODE     ---       #185
      01000CC0H   LINE      CODE     ---       #187
      01000CC5H   LINE      CODE     ---       #189
      01000CDBH   LINE      CODE     ---       #190
      01000CDEH   LINE      CODE     ---       #193
      01000CE6H   LINE      CODE     ---       #195
      01000CEBH   LINE      CODE     ---       #196
      01000CFBH   LINE      CODE     ---       #197
      01000CFBH   LINE      CODE     ---       #198
      01000CFBH   LINE      CODE     ---       #200
      01000D0BH   LINE      CODE     ---       #204
      01000D14H   LINE      CODE     ---       #207
      01000D3DH   LINE      CODE     ---       #208
      01000D52H   LINE      CODE     ---       #211
      01000D59H   LINE      CODE     ---       #212
      01000D60H   LINE      CODE     ---       #215
      01000D67H   LINE      CODE     ---       #216
      01000D8BH   LINE      CODE     ---       #217
      01000DA0H   LINE      CODE     ---       #220
      01000DA9H   LINE      CODE     ---       #221
      01000DCBH   LINE      CODE     ---       #224
      01000DD5H   LINE      CODE     ---       #225
      01000DDAH   LINE      CODE     ---       #227
      01000DDAH   LINE      CODE     ---       #228
      01000DDAH   LINE      CODE     ---       #229
      01000DDAH   LINE      CODE     ---       #231
LX51 LINKER/LOCATER V4.66.30.0                                                        07/27/2019  23:22:19  PAGE 171


      01000DE3H   LINE      CODE     ---       #233
      01000DEAH   LINE      CODE     ---       #234
      01000E07H   LINE      CODE     ---       #235
      01000E0EH   LINE      CODE     ---       #236
      01000E1EH   LINE      CODE     ---       #237
      01000E1EH   LINE      CODE     ---       #239
      01000E25H   LINE      CODE     ---       #240
      01000E3CH   LINE      CODE     ---       #241
      01000E43H   LINE      CODE     ---       #242
      01000E53H   LINE      CODE     ---       #243
      01000E53H   LINE      CODE     ---       #245
      01000E5AH   LINE      CODE     ---       #246
      ---         BLOCKEND  ---      ---       LVL=0

      010034BDH   BLOCK     CODE     ---       LVL=0
      00000022H   SYMBOL    DATA     BYTE      idx
      010034BFH   BLOCK     CODE     NEAR LAB  LVL=1
      02000413H   SYMBOL    XDATA    ---       txt
      00000023H   SYMBOL    DATA     BYTE      w
      ---         BLOCKEND  ---      ---       LVL=1
      010034BDH   LINE      CODE     ---       #248
      010034BFH   LINE      CODE     ---       #249
      010034BFH   LINE      CODE     ---       #253
      010034C4H   LINE      CODE     ---       #256
      010034D4H   LINE      CODE     ---       #259
      010034DBH   LINE      CODE     ---       #260
      010034F9H   LINE      CODE     ---       #261
      01003507H   LINE      CODE     ---       #262
      01003515H   LINE      CODE     ---       #263
      01003523H   LINE      CODE     ---       #264
      01003531H   LINE      CODE     ---       #265
      0100353FH   LINE      CODE     ---       #266
      0100354DH   LINE      CODE     ---       #267
      0100355CH   LINE      CODE     ---       #268
      0100355CH   LINE      CODE     ---       #269
      0100356CH   LINE      CODE     ---       #272
      01003575H   LINE      CODE     ---       #273
      01003575H   LINE      CODE     ---       #274
      01003575H   LINE      CODE     ---       #275
      01003592H   LINE      CODE     ---       #276
      0100359EH   LINE      CODE     ---       #277
      010035AAH   LINE      CODE     ---       #278
      010035AAH   LINE      CODE     ---       #279
      010035AAH   LINE      CODE     ---       #282
      010035AFH   LINE      CODE     ---       #283
      ---         BLOCKEND  ---      ---       LVL=0

      0100553AH   BLOCK     CODE     ---       LVL=0
      00000007H   SYMBOL    DATA     BYTE      idx
      0100553AH   LINE      CODE     ---       #286
      0100553AH   LINE      CODE     ---       #287
      0100553AH   LINE      CODE     ---       #288
      0100554CH   LINE      CODE     ---       #289
      0100554CH   LINE      CODE     ---       #290
      01005551H   LINE      CODE     ---       #292
      01005551H   LINE      CODE     ---       #293
      01005551H   LINE      CODE     ---       #294
      01005557H   LINE      CODE     ---       #295
      01005559H   LINE      CODE     ---       #297
      01005559H   LINE      CODE     ---       #298
      01005559H   LINE      CODE     ---       #299
      0100555FH   LINE      CODE     ---       #300
LX51 LINKER/LOCATER V4.66.30.0                                                        07/27/2019  23:22:19  PAGE 172


      01005561H   LINE      CODE     ---       #302
      01005561H   LINE      CODE     ---       #303
      01005561H   LINE      CODE     ---       #304
      01005561H   LINE      CODE     ---       #306
      01005561H   LINE      CODE     ---       #307
      01005561H   LINE      CODE     ---       #308
      01005567H   LINE      CODE     ---       #309
      01005569H   LINE      CODE     ---       #311
      01005569H   LINE      CODE     ---       #312
      01005569H   LINE      CODE     ---       #313
      0100556FH   LINE      CODE     ---       #314
      01005572H   LINE      CODE     ---       #316
      01005572H   LINE      CODE     ---       #317
      01005572H   LINE      CODE     ---       #318
      ---         BLOCKEND  ---      ---       LVL=0

      ---         MODULE    ---      ---       MENU_1_FN
      010041EAH   PUBLIC    CODE     ---       _menu_1_enter
      01001B7CH   PUBLIC    CODE     ---       _menu_1_disp
      010057C3H   PUBLIC    CODE     ---       menu_1_font_next
      01003953H   PUBLIC    CODE     ---       menu_1_name_edit
      010044A7H   PUBLIC    CODE     ---       menu_1_btn_use
      01004CE8H   PUBLIC    CODE     ---       menu_1_btn_exit
      01005A37H   PUBLIC    CODE     ---       menu_1_btn_enter
      01004554H   PUBLIC    CODE     ---       menu_1_btn_prev
      0100434AH   PUBLIC    CODE     ---       menu_1_btn_next
      000000A2H   SFRSYM    DATA     BYTE      SPI0CKR
      00000080H   SFRSYM    DATA     BYTE      P0
      000000D0H.2 SFRSYM    DATA     BIT       PSW_OV
      000000B1H   SFRSYM    DATA     BYTE      XOSC0CN
      00000090H   SFRSYM    DATA     BYTE      P1
      000000A0H   SFRSYM    DATA     BYTE      P2
      000000B0H   SFRSYM    DATA     BYTE      P3
      000000BCH   SFRSYM    DATA     BYTE      ADC0CF
      000000C8H   SFRSYM    DATA     BIT       TMR2CN0_T2XCLK
      000000C7H   SFRSYM    DATA     BYTE      P4
      000000C0H.7 SFRSYM    DATA     BIT       SMB0CN0_MASTER
      000000F9H   SFRSYM    DATA     WORD      PCA0
      000000E6H   SFRSYM    DATA     BYTE      EIE1
      000000C0H.7 SFRSYM    DATA     BIT       SMB1CN0_MASTER
      000000C0H.1 SFRSYM    DATA     BIT       SMB0CN0_ACK
      000000D7H   SFRSYM    DATA     BYTE      USB0XCN
      000000E7H   SFRSYM    DATA     BYTE      EIE2
      000000C0H.1 SFRSYM    DATA     BIT       SMB1CN0_ACK
      0000008FH   SFRSYM    DATA     BYTE      PSCTL
      000000E4H   SFRSYM    DATA     BYTE      IT01CF
      000000C8H   SFRSYM    DATA     BIT       TMR5CN0_T5XCLK
      000000C0H.6 SFRSYM    DATA     BIT       SMB0CN0_TXMODE
      000000C0H.6 SFRSYM    DATA     BIT       SMB1CN0_TXMODE
      000000BFH   SFRSYM    DATA     BYTE      SFRPAGE
      000000A4H   SFRSYM    DATA     BYTE      P0MDOUT
      000000A5H   SFRSYM    DATA     BYTE      P1MDOUT
      000000E8H.5 SFRSYM    DATA     BIT       ADC0CN0_ADINT
      000000CBH   SFRSYM    DATA     BYTE      TMR2RLH
      000000A6H   SFRSYM    DATA     BYTE      P2MDOUT
      000000A8H   SFRSYM    DATA     BYTE      IE
      00000093H   SFRSYM    DATA     BYTE      TMR3RLH
      000000A7H   SFRSYM    DATA     BYTE      P3MDOUT
      00000093H   SFRSYM    DATA     BYTE      TMR4RLH
      000000AEH   SFRSYM    DATA     BYTE      P4MDOUT
      000000F6H   SFRSYM    DATA     BYTE      EIP1
      000000CBH   SFRSYM    DATA     BYTE      TMR5RLH
LX51 LINKER/LOCATER V4.66.30.0                                                        07/27/2019  23:22:19  PAGE 173


      000000F7H   SFRSYM    DATA     BYTE      EIP2
      00000098H.2 SFRSYM    DATA     BIT       SCON0_RB8
      000000CAH   SFRSYM    DATA     BYTE      TMR2RLL
      000000FCH   SFRSYM    DATA     BYTE      PCA0CPH0
      00000092H   SFRSYM    DATA     BYTE      TMR3RLL
      000000EAH   SFRSYM    DATA     BYTE      PCA0CPH1
      00000098H.3 SFRSYM    DATA     BIT       SCON0_TB8
      000000F0H   SFRSYM    DATA     BIT       B_B0
      00000082H   SFRSYM    DATA     WORD      DP
      00000092H   SFRSYM    DATA     BYTE      TMR4RLL
      000000ECH   SFRSYM    DATA     BYTE      PCA0CPH2
      000000F0H.1 SFRSYM    DATA     BIT       B_B1
      000000C3H   SFRSYM    DATA     WORD      ADC0GT
      000000CAH   SFRSYM    DATA     BYTE      TMR5RLL
      000000EEH   SFRSYM    DATA     BYTE      PCA0CPH3
      000000F0H.2 SFRSYM    DATA     BIT       B_B2
      000000FBH   SFRSYM    DATA     BYTE      PCA0CPL0
      000000FEH   SFRSYM    DATA     BYTE      PCA0CPH4
      00000085H   SFRSYM    DATA     BYTE      EMI0CF
      000000F0H.3 SFRSYM    DATA     BIT       B_B3
      000000D9H   SFRSYM    DATA     BYTE      PCA0MD
      000000DAH   SFRSYM    DATA     BYTE      PCA0CPM0
      000000E9H   SFRSYM    DATA     BYTE      PCA0CPL1
      000000F0H.4 SFRSYM    DATA     BIT       B_B4
      000000DBH   SFRSYM    DATA     BYTE      PCA0CPM1
      000000EBH   SFRSYM    DATA     BYTE      PCA0CPL2
      000000F0H.5 SFRSYM    DATA     BIT       B_B5
      000000DCH   SFRSYM    DATA     BYTE      PCA0CPM2
      000000EDH   SFRSYM    DATA     BYTE      PCA0CPL3
      000000B8H   SFRSYM    DATA     BYTE      IP
      000000F0H.6 SFRSYM    DATA     BIT       B_B6
      000000C5H   SFRSYM    DATA     WORD      ADC0LT
      000000DDH   SFRSYM    DATA     BYTE      PCA0CPM3
      000000FDH   SFRSYM    DATA     BYTE      PCA0CPL4
      00000098H.5 SFRSYM    DATA     BIT       SCON0_MCE
      000000F0H.7 SFRSYM    DATA     BIT       B_B7
      000000DEH   SFRSYM    DATA     BYTE      PCA0CPM4
      000000E1H   SFRSYM    DATA     BYTE      XBR0
      000000C1H   SFRSYM    DATA     BYTE      SMB0CF
      000000E2H   SFRSYM    DATA     BYTE      XBR1
      000000C1H   SFRSYM    DATA     BYTE      SMB1CF
      000000AFH   SFRSYM    DATA     BYTE      PFE0CN
      000000AAH   SFRSYM    DATA     BYTE      EMI0CN
      000000C0H.5 SFRSYM    DATA     BIT       SMB0CN0_STA
      000000E3H   SFRSYM    DATA     BYTE      XBR2
      000000C0H.5 SFRSYM    DATA     BIT       SMB1CN0_STA
      000000E0H   SFRSYM    DATA     BIT       ACC_ACC0
      000000D1H   SFRSYM    DATA     BYTE      REF0CN
      000000B2H   SFRSYM    DATA     BYTE      HFO0CN
      0000008EH   SFRSYM    DATA     BYTE      CKCON0
      000000E0H.1 SFRSYM    DATA     BIT       ACC_ACC1
      000000E4H   SFRSYM    DATA     BYTE      CKCON1
      000000C8H.2 SFRSYM    DATA     BIT       TMR2CN0_TR2
      000000E0H.2 SFRSYM    DATA     BIT       ACC_ACC2
      000000E0H.3 SFRSYM    DATA     BIT       ACC_ACC3
      00000081H   SFRSYM    DATA     BYTE      SP
      0000009DH   SFRSYM    DATA     BYTE      CMP0MD
      000000E0H.4 SFRSYM    DATA     BIT       ACC_ACC4
      00000086H   SFRSYM    DATA     BYTE      LFO0CN
      00000084H   SFRSYM    DATA     BYTE      EMI0TC
      0000009CH   SFRSYM    DATA     BYTE      CMP1MD
      000000D8H   SFRSYM    DATA     BIT       PCA0CN0_CCF0
LX51 LINKER/LOCATER V4.66.30.0                                                        07/27/2019  23:22:19  PAGE 174


      000000E0H.5 SFRSYM    DATA     BIT       ACC_ACC5
      000000D8H.1 SFRSYM    DATA     BIT       PCA0CN0_CCF1
      000000E0H.6 SFRSYM    DATA     BIT       ACC_ACC6
      000000CCH   SFRSYM    DATA     WORD      TMR2
      000000D8H.2 SFRSYM    DATA     BIT       PCA0CN0_CCF2
      000000E0H.7 SFRSYM    DATA     BIT       ACC_ACC7
      00000094H   SFRSYM    DATA     WORD      TMR3
      000000C8H.2 SFRSYM    DATA     BIT       TMR5CN0_TR5
      000000D8H.3 SFRSYM    DATA     BIT       PCA0CN0_CCF3
      00000094H   SFRSYM    DATA     WORD      TMR4
      000000ACH   SFRSYM    DATA     BYTE      SBCON1
      000000D8H.4 SFRSYM    DATA     BIT       PCA0CN0_CCF4
      000000CCH   SFRSYM    DATA     WORD      TMR5
      000000C0H.3 SFRSYM    DATA     BIT       SMB0CN0_ACKRQ
      000000FFH   SFRSYM    DATA     BYTE      VDM0CN
      000000F1H   SFRSYM    DATA     BYTE      P0MDIN
      000000C0H.3 SFRSYM    DATA     BIT       SMB1CN0_ACKRQ
      00000098H.4 SFRSYM    DATA     BIT       SCON0_REN
      000000F2H   SFRSYM    DATA     BYTE      P1MDIN
      000000F3H   SFRSYM    DATA     BYTE      P2MDIN
      000000C0H.4 SFRSYM    DATA     BIT       SMB0CN0_STO
      000000F4H   SFRSYM    DATA     BYTE      P3MDIN
      000000C0H.4 SFRSYM    DATA     BIT       SMB1CN0_STO
      000000B5H   SFRSYM    DATA     BYTE      SBRLH1
      000000F5H   SFRSYM    DATA     BYTE      P4MDIN
      000000D0H.3 SFRSYM    DATA     BIT       PSW_RS0
      000000D8H.7 SFRSYM    DATA     BIT       PCA0CN0_CF
      000000F8H.4 SFRSYM    DATA     BIT       SPI0CN0_RXOVRN
      000000D0H.4 SFRSYM    DATA     BIT       PSW_RS1
      000000B4H   SFRSYM    DATA     BYTE      SBRLL1
      000000E8H.7 SFRSYM    DATA     BIT       ADC0CN0_ADEN
      00000089H   SFRSYM    DATA     BYTE      TMOD
      00000088H   SFRSYM    DATA     BYTE      TCON
      000000D0H   SFRSYM    DATA     BIT       PSW_PARITY
      000000A8H.4 SFRSYM    DATA     BIT       IE_ES0
      0000009FH   SFRSYM    DATA     BYTE      CMP0MX
      000000A8H.1 SFRSYM    DATA     BIT       IE_ET0
      0000009EH   SFRSYM    DATA     BYTE      CMP1MX
      000000A8H.3 SFRSYM    DATA     BIT       IE_ET1
      000000D4H   SFRSYM    DATA     BYTE      P0SKIP
      000000C8H.1 SFRSYM    DATA     BIT       TMR2CN0_T2CSS
      000000A8H.5 SFRSYM    DATA     BIT       IE_ET2
      000000D5H   SFRSYM    DATA     BYTE      P1SKIP
      000000D6H   SFRSYM    DATA     BYTE      P2SKIP
      000000E8H   SFRSYM    DATA     BYTE      ADC0CN0
      000000A8H   SFRSYM    DATA     BIT       IE_EX0
      000000DFH   SFRSYM    DATA     BYTE      P3SKIP
      000000D8H.6 SFRSYM    DATA     BIT       PCA0CN0_CR
      000000A8H.2 SFRSYM    DATA     BIT       IE_EX1
      00000098H.7 SFRSYM    DATA     BIT       SCON0_SMODE
      000000A9H   SFRSYM    DATA     BYTE      CLKSEL
      000000F8H   SFRSYM    DATA     BIT       SPI0CN0_SPIEN
      000000F0H   SFRSYM    DATA     BYTE      B
      000000BEH   SFRSYM    DATA     BYTE      ADC0H
      000000E8H.6 SFRSYM    DATA     BIT       ADC0CN0_ADTM
      000000CAH   SFRSYM    DATA     WORD      TMR2RL
      000000BDH   SFRSYM    DATA     BYTE      ADC0L
      00000092H   SFRSYM    DATA     WORD      TMR3RL
      00000092H   SFRSYM    DATA     WORD      TMR4RL
      000000D8H   SFRSYM    DATA     BYTE      PCA0CN0
      000000E0H   SFRSYM    DATA     BYTE      ACC
      000000CAH   SFRSYM    DATA     WORD      TMR5RL
LX51 LINKER/LOCATER V4.66.30.0                                                        07/27/2019  23:22:19  PAGE 175


      000000FBH   SFRSYM    DATA     WORD      PCA0CP0
      000000E9H   SFRSYM    DATA     WORD      PCA0CP1
      000000EBH   SFRSYM    DATA     WORD      PCA0CP2
      000000EDH   SFRSYM    DATA     WORD      PCA0CP3
      0000008CH   SFRSYM    DATA     BYTE      TH0
      000000B8H.4 SFRSYM    DATA     BIT       IP_PS0
      000000FDH   SFRSYM    DATA     WORD      PCA0CP4
      0000008DH   SFRSYM    DATA     BYTE      TH1
      000000FAH   SFRSYM    DATA     BYTE      PCA0H
      000000B8H.1 SFRSYM    DATA     BIT       IP_PT0
      000000B8H.3 SFRSYM    DATA     BIT       IP_PT1
      000000C0H.2 SFRSYM    DATA     BIT       SMB0CN0_ARBLOST
      000000B8H.5 SFRSYM    DATA     BIT       IP_PT2
      0000008AH   SFRSYM    DATA     BYTE      TL0
      000000F8H.1 SFRSYM    DATA     BIT       SPI0CN0_TXBMT
      000000C0H.2 SFRSYM    DATA     BIT       SMB1CN0_ARBLOST
      000000D0H.5 SFRSYM    DATA     BIT       PSW_F0
      000000A8H.6 SFRSYM    DATA     BIT       IE_ESPI0
      0000008BH   SFRSYM    DATA     BYTE      TL1
      000000F9H   SFRSYM    DATA     BYTE      PCA0L
      000000C0H   SFRSYM    DATA     BIT       SMB0CN0_SI
      000000D0H.1 SFRSYM    DATA     BIT       PSW_F1
      00000080H   SFRSYM    DATA     BIT       P0_B0
      000000B8H   SFRSYM    DATA     BIT       IP_PX0
      000000C9H   SFRSYM    DATA     BYTE      REG01CN
      000000C0H   SFRSYM    DATA     BIT       SMB1CN0_SI
      00000090H   SFRSYM    DATA     BIT       P1_B0
      00000080H.1 SFRSYM    DATA     BIT       P0_B1
      000000B8H.2 SFRSYM    DATA     BIT       IP_PX1
      0000009BH   SFRSYM    DATA     BYTE      CMP0CN0
      00000088H.1 SFRSYM    DATA     BIT       TCON_IE0
      000000A0H   SFRSYM    DATA     BIT       P2_B0
      00000090H.1 SFRSYM    DATA     BIT       P1_B1
      00000080H.2 SFRSYM    DATA     BIT       P0_B2
      0000009AH   SFRSYM    DATA     BYTE      CMP1CN0
      00000088H.3 SFRSYM    DATA     BIT       TCON_IE1
      000000B0H   SFRSYM    DATA     BIT       P3_B0
      000000A0H.1 SFRSYM    DATA     BIT       P2_B1
      00000090H.2 SFRSYM    DATA     BIT       P1_B2
      00000080H.3 SFRSYM    DATA     BIT       P0_B3
      000000C0H   SFRSYM    DATA     BYTE      SMB0CN0
      000000B0H.1 SFRSYM    DATA     BIT       P3_B1
      000000A0H.2 SFRSYM    DATA     BIT       P2_B2
      00000090H.3 SFRSYM    DATA     BIT       P1_B3
      00000080H.4 SFRSYM    DATA     BIT       P0_B4
      000000C0H   SFRSYM    DATA     BYTE      SMB1CN0
      000000B0H.2 SFRSYM    DATA     BIT       P3_B2
      000000A0H.3 SFRSYM    DATA     BIT       P2_B3
      00000090H.4 SFRSYM    DATA     BIT       P1_B4
      00000080H.5 SFRSYM    DATA     BIT       P0_B5
      000000B0H.3 SFRSYM    DATA     BIT       P3_B3
      000000A0H.4 SFRSYM    DATA     BIT       P2_B4
      00000090H.5 SFRSYM    DATA     BIT       P1_B5
      00000080H.6 SFRSYM    DATA     BIT       P0_B6
      000000B0H.4 SFRSYM    DATA     BIT       P3_B4
      000000A0H.5 SFRSYM    DATA     BIT       P2_B5
      00000090H.6 SFRSYM    DATA     BIT       P1_B6
      00000080H.7 SFRSYM    DATA     BIT       P0_B7
      000000B0H.5 SFRSYM    DATA     BIT       P3_B5
      000000A0H.6 SFRSYM    DATA     BIT       P2_B6
      00000090H.7 SFRSYM    DATA     BIT       P1_B7
      000000B0H.6 SFRSYM    DATA     BIT       P3_B6
LX51 LINKER/LOCATER V4.66.30.0                                                        07/27/2019  23:22:19  PAGE 176


      000000A0H.7 SFRSYM    DATA     BIT       P2_B7
      000000B0H.7 SFRSYM    DATA     BIT       P3_B7
      00000083H   SFRSYM    DATA     BYTE      DPH
      000000C4H   SFRSYM    DATA     BYTE      ADC0GTH
      000000C8H.7 SFRSYM    DATA     BIT       TMR2CN0_TF2H
      000000C8H.3 SFRSYM    DATA     BIT       TMR2CN0_T2SPLIT
      000000D0H.6 SFRSYM    DATA     BIT       PSW_AC
      000000F8H   SFRSYM    DATA     BYTE      SPI0CN0
      000000B3H   SFRSYM    DATA     BYTE      HFO0CAL
      00000088H.5 SFRSYM    DATA     BIT       TCON_TF0
      00000098H   SFRSYM    DATA     BIT       SCON0_RI
      00000082H   SFRSYM    DATA     BYTE      DPL
      00000088H.7 SFRSYM    DATA     BIT       TCON_TF1
      00000099H   SFRSYM    DATA     BYTE      SBUF0
      00000087H   SFRSYM    DATA     BYTE      PCON0
      000000C3H   SFRSYM    DATA     BYTE      ADC0GTL
      000000C8H.6 SFRSYM    DATA     BIT       TMR2CN0_TF2L
      00000098H.1 SFRSYM    DATA     BIT       SCON0_TI
      000000E8H   SFRSYM    DATA     BIT       ADC0CN0_ADCM0
      000000D3H   SFRSYM    DATA     BYTE      SBUF1
      000000C6H   SFRSYM    DATA     BYTE      ADC0LTH
      00000088H   SFRSYM    DATA     BIT       TCON_IT0
      000000E8H.1 SFRSYM    DATA     BIT       ADC0CN0_ADCM1
      000000EFH   SFRSYM    DATA     BYTE      RSTSRC
      000000C8H.7 SFRSYM    DATA     BIT       TMR5CN0_TF5H
      000000C8H.3 SFRSYM    DATA     BIT       TMR5CN0_T5SPLIT
      00000088H.2 SFRSYM    DATA     BIT       TCON_IT1
      000000E8H.2 SFRSYM    DATA     BIT       ADC0CN0_ADCM2
      00000098H   SFRSYM    DATA     BYTE      SCON0
      000000E8H.3 SFRSYM    DATA     BIT       ADC0CN0_ADWINT
      000000B4H   SFRSYM    DATA     WORD      SBRL1
      000000E5H   SFRSYM    DATA     BYTE      SMOD1
      000000D2H   SFRSYM    DATA     BYTE      SCON1
      000000BAH   SFRSYM    DATA     BYTE      AMX0N
      000000E8H.4 SFRSYM    DATA     BIT       ADC0CN0_ADBUSY
      000000CEH   SFRSYM    DATA     BYTE      SMB0ADM
      000000C5H   SFRSYM    DATA     BYTE      ADC0LTL
      000000F8H.5 SFRSYM    DATA     BIT       SPI0CN0_MODF
      000000B8H.6 SFRSYM    DATA     BIT       IP_PSPI0
      000000CEH   SFRSYM    DATA     BYTE      SMB1ADM
      000000BBH   SFRSYM    DATA     BYTE      AMX0P
      000000C8H.6 SFRSYM    DATA     BIT       TMR5CN0_TF5L
      000000C8H   SFRSYM    DATA     BYTE      TMR2CN0
      00000091H   SFRSYM    DATA     BYTE      TMR3CN0
      00000091H   SFRSYM    DATA     BYTE      TMR4CN0
      000000C8H   SFRSYM    DATA     BYTE      TMR5CN0
      000000CFH   SFRSYM    DATA     BYTE      SMB0ADR
      00000088H.4 SFRSYM    DATA     BIT       TCON_TR0
      000000CFH   SFRSYM    DATA     BYTE      SMB1ADR
      000000C8H.4 SFRSYM    DATA     BIT       TMR2CN0_TF2CEN
      00000088H.6 SFRSYM    DATA     BIT       TCON_TR1
      000000C2H   SFRSYM    DATA     BYTE      SMB0DAT
      000000CDH   SFRSYM    DATA     BYTE      TMR2H
      000000A1H   SFRSYM    DATA     BYTE      SPI0CFG
      000000C2H   SFRSYM    DATA     BYTE      SMB1DAT
      00000095H   SFRSYM    DATA     BYTE      TMR3H
      00000095H   SFRSYM    DATA     BYTE      TMR4H
      000000CDH   SFRSYM    DATA     BYTE      TMR5H
      000000CCH   SFRSYM    DATA     BYTE      TMR2L
      000000F8H.7 SFRSYM    DATA     BIT       SPI0CN0_SPIF
      00000096H   SFRSYM    DATA     BYTE      USB0ADR
      00000094H   SFRSYM    DATA     BYTE      TMR3L
LX51 LINKER/LOCATER V4.66.30.0                                                        07/27/2019  23:22:19  PAGE 177


      000000A8H.7 SFRSYM    DATA     BIT       IE_EA
      00000094H   SFRSYM    DATA     BYTE      TMR4L
      00000097H   SFRSYM    DATA     BYTE      USB0DAT
      000000CCH   SFRSYM    DATA     BYTE      TMR5L
      000000B6H   SFRSYM    DATA     BYTE      FLSCL
      000000C8H.5 SFRSYM    DATA     BIT       TMR2CN0_TF2LEN
      000000F8H.6 SFRSYM    DATA     BIT       SPI0CN0_WCOL
      000000F8H.2 SFRSYM    DATA     BIT       SPI0CN0_NSSMD0
      000000D0H.7 SFRSYM    DATA     BIT       PSW_CY
      000000A3H   SFRSYM    DATA     BYTE      SPI0DAT
      000000F8H.3 SFRSYM    DATA     BIT       SPI0CN0_NSSMD1
      000000BDH   SFRSYM    DATA     WORD      ADC0
      000000B9H   SFRSYM    DATA     BYTE      SMBTC
      000000D0H   SFRSYM    DATA     BYTE      PSW
      000000C8H.5 SFRSYM    DATA     BIT       TMR5CN0_TF5LEN
      000000B7H   SFRSYM    DATA     BYTE      FLKEY
      020004BCH   SYMBOL    XDATA    BYTE      edit_mode
      020004BDH   SYMBOL    XDATA    BYTE      menu_last
      020004BEH   SYMBOL    XDATA    BYTE      edit_pos
      00000007H   SYMBOL    DATA     BYTE      a

      0100434AH   BLOCK     CODE     ---       LVL=0
      0100434AH   BLOCK     CODE     NEAR LAB  LVL=1
      00000025H   SYMBOL    DATA     BYTE      first
      00000026H   SYMBOL    DATA     BYTE      last
      00000007H   SYMBOL    DATA     BYTE      len
      ---         BLOCKEND  ---      ---       LVL=1
      0100434AH   LINE      CODE     ---       #46
      0100434AH   LINE      CODE     ---       #47
      0100434AH   LINE      CODE     ---       #50
      01004351H   LINE      CODE     ---       #51
      01004357H   LINE      CODE     ---       #52
      01004373H   LINE      CODE     ---       #53
      01004378H   LINE      CODE     ---       #54
      01004378H   LINE      CODE     ---       #55
      01004379H   LINE      CODE     ---       #56
      01004399H   LINE      CODE     ---       #57
      010043A0H   LINE      CODE     ---       #58
      010043A9H   LINE      CODE     ---       #60
      010043B3H   LINE      CODE     ---       #61
      010043C0H   LINE      CODE     ---       #62
      010043D6H   LINE      CODE     ---       #63
      010043E6H   LINE      CODE     ---       #64
      010043E6H   LINE      CODE     ---       #66
      010043EDH   LINE      CODE     ---       #67
      010043F8H   LINE      CODE     ---       #68
      010043F8H   LINE      CODE     ---       #69
      010043F8H   LINE      CODE     ---       #70
      010043F8H   LINE      CODE     ---       #71
      ---         BLOCKEND  ---      ---       LVL=0

      01004554H   BLOCK     CODE     ---       LVL=0
      01004554H   BLOCK     CODE     NEAR LAB  LVL=1
      00000025H   SYMBOL    DATA     BYTE      first
      00000026H   SYMBOL    DATA     BYTE      last
      00000007H   SYMBOL    DATA     BYTE      len
      ---         BLOCKEND  ---      ---       LVL=1
      01004554H   LINE      CODE     ---       #73
      01004554H   LINE      CODE     ---       #74
      01004554H   LINE      CODE     ---       #77
      0100455BH   LINE      CODE     ---       #78
      01004561H   LINE      CODE     ---       #79
LX51 LINKER/LOCATER V4.66.30.0                                                        07/27/2019  23:22:19  PAGE 178


      01004570H   LINE      CODE     ---       #80
      01004570H   LINE      CODE     ---       #81
      01004576H   LINE      CODE     ---       #82
      01004577H   LINE      CODE     ---       #83
      01004597H   LINE      CODE     ---       #84
      0100459EH   LINE      CODE     ---       #85
      010045A7H   LINE      CODE     ---       #87
      010045B1H   LINE      CODE     ---       #88
      010045C1H   LINE      CODE     ---       #89
      010045D1H   LINE      CODE     ---       #90
      010045D1H   LINE      CODE     ---       #91
      010045E2H   LINE      CODE     ---       #93
      010045E6H   LINE      CODE     ---       #94
      010045F1H   LINE      CODE     ---       #95
      010045F1H   LINE      CODE     ---       #96
      010045F1H   LINE      CODE     ---       #97
      010045F1H   LINE      CODE     ---       #98
      ---         BLOCKEND  ---      ---       LVL=0

      01005A37H   BLOCK     CODE     ---       LVL=0
      01005A37H   LINE      CODE     ---       #100
      01005A37H   LINE      CODE     ---       #101
      01005A37H   LINE      CODE     ---       #102
      01005A3EH   LINE      CODE     ---       #103
      01005A41H   LINE      CODE     ---       #104
      01005A42H   LINE      CODE     ---       #105
      01005A48H   LINE      CODE     ---       #106
      01005A48H   LINE      CODE     ---       #107
      ---         BLOCKEND  ---      ---       LVL=0

      01004CE8H   BLOCK     CODE     ---       LVL=0
      01004CE8H   BLOCK     CODE     NEAR LAB  LVL=1
      00000025H   SYMBOL    DATA     BYTE      i
      ---         BLOCKEND  ---      ---       LVL=1
      01004CE8H   LINE      CODE     ---       #109
      01004CE8H   LINE      CODE     ---       #110
      01004CE8H   LINE      CODE     ---       #113
      01004CEFH   LINE      CODE     ---       #114
      01004CF1H   LINE      CODE     ---       #115
      01004CF4H   LINE      CODE     ---       #116
      01004CF4H   LINE      CODE     ---       #129
      01004D01H   LINE      CODE     ---       #130
      01004D16H   LINE      CODE     ---       #131
      01004D30H   LINE      CODE     ---       #132
      01004D34H   LINE      CODE     ---       #133
      01004D41H   LINE      CODE     ---       #134
      01004D47H   LINE      CODE     ---       #135
      01004D47H   LINE      CODE     ---       #136
      01004D47H   LINE      CODE     ---       #137
      ---         BLOCKEND  ---      ---       LVL=0

      010044A7H   BLOCK     CODE     ---       LVL=0
      010044A7H   LINE      CODE     ---       #139
      010044A7H   LINE      CODE     ---       #140
      010044A7H   LINE      CODE     ---       #141
      010044B3H   LINE      CODE     ---       #142
      010044B9H   LINE      CODE     ---       #143
      010044C5H   LINE      CODE     ---       #144
      010044CBH   LINE      CODE     ---       #145
      010044E4H   LINE      CODE     ---       #147
      010044F0H   LINE      CODE     ---       #148
      010044FCH   LINE      CODE     ---       #149
LX51 LINKER/LOCATER V4.66.30.0                                                        07/27/2019  23:22:19  PAGE 179


      01004502H   LINE      CODE     ---       #151
      0100450EH   LINE      CODE     ---       #152
      0100451AH   LINE      CODE     ---       #153
      01004520H   LINE      CODE     ---       #155
      0100452CH   LINE      CODE     ---       #156
      01004532H   LINE      CODE     ---       #157
      0100453EH   LINE      CODE     ---       #158
      01004544H   LINE      CODE     ---       #159
      01004553H   LINE      CODE     ---       #160
      ---         BLOCKEND  ---      ---       LVL=0

      01003953H   BLOCK     CODE     ---       LVL=0
      01003953H   BLOCK     CODE     NEAR LAB  LVL=1
      00000005H   SYMBOL    DATA     BYTE      w
      00000007H   SYMBOL    DATA     BYTE      x
      02000423H   SYMBOL    XDATA    ---       txt
      ---         BLOCKEND  ---      ---       LVL=1
      01003953H   LINE      CODE     ---       #162
      01003953H   LINE      CODE     ---       #163
      01003953H   LINE      CODE     ---       #167
      0100395AH   LINE      CODE     ---       #168
      01003970H   LINE      CODE     ---       #170
      01003988H   LINE      CODE     ---       #173
      0100399BH   LINE      CODE     ---       #174
      010039ABH   LINE      CODE     ---       #175
      010039ADH   LINE      CODE     ---       #177
      010039B6H   LINE      CODE     ---       #178
      010039B9H   LINE      CODE     ---       #179
      010039BBH   LINE      CODE     ---       #181
      010039C3H   LINE      CODE     ---       #182
      010039C3H   LINE      CODE     ---       #186
      010039E3H   LINE      CODE     ---       #187
      01003A17H   LINE      CODE     ---       #188
      ---         BLOCKEND  ---      ---       LVL=0

      010057C3H   BLOCK     CODE     ---       LVL=0
      010057C3H   LINE      CODE     ---       #191
      010057C3H   LINE      CODE     ---       #192
      010057C3H   LINE      CODE     ---       #193
      010057C3H   LINE      CODE     ---       #194
      010057C9H   LINE      CODE     ---       #195
      010057CFH   LINE      CODE     ---       #196
      010057D1H   LINE      CODE     ---       #197
      010057D1H   LINE      CODE     ---       #198
      010057E6H   LINE      CODE     ---       #199
      ---         BLOCKEND  ---      ---       LVL=0

      01001B7CH   BLOCK     CODE     ---       LVL=0
      00000022H   SYMBOL    DATA     BYTE      idx
      01001B7EH   BLOCK     CODE     NEAR LAB  LVL=1
      00000023H   SYMBOL    DATA     CHAR      w
      00000024H   SYMBOL    DATA     CHAR      x
      02000413H   SYMBOL    XDATA    ---       txt
      01001E4FH   SYMBOL    CODE     VOID      MENU_0_DRAW_TEXT_DONE
      01001BD7H   SYMBOL    CODE     VOID      MENU_0_ORIENTATION
      01001CACH   SYMBOL    CODE     VOID      MENU_0_FONT
      ---         BLOCKEND  ---      ---       LVL=1
      01001B7CH   LINE      CODE     ---       #201
      01001B7EH   LINE      CODE     ---       #202
      01001B7EH   LINE      CODE     ---       #206
      01001B84H   LINE      CODE     ---       #207
      01001B87H   LINE      CODE     ---       #208
LX51 LINKER/LOCATER V4.66.30.0                                                        07/27/2019  23:22:19  PAGE 180


      01001B8AH   LINE      CODE     ---       #209
      01001B8DH   LINE      CODE     ---       #210
      01001B8DH   LINE      CODE     ---       #212
      01001B94H   LINE      CODE     ---       #215
      01001BB2H   LINE      CODE     ---       #216
      01001BB2H   LINE      CODE     ---       #217
      01001BC8H   LINE      CODE     ---       #218
      01001BD4H   LINE      CODE     ---       #219
      01001BD7H   LINE      CODE     ---       #220
      01001BD7H   LINE      CODE     ---       #221
      01001BD7H   LINE      CODE     ---       #222
      01001BD7H   LINE      CODE     ---       #223
      01001BEDH   LINE      CODE     ---       #224
      01001C06H   LINE      CODE     ---       #225
      01001C06H   LINE      CODE     ---       #226
      01001C12H   LINE      CODE     ---       #227
      01001C15H   LINE      CODE     ---       #228
      01001C15H   LINE      CODE     ---       #229
      01001C15H   LINE      CODE     ---       #230
      01001C21H   LINE      CODE     ---       #231
      01001C24H   LINE      CODE     ---       #232
      01001C24H   LINE      CODE     ---       #233
      01001C24H   LINE      CODE     ---       #234
      01001C30H   LINE      CODE     ---       #235
      01001C33H   LINE      CODE     ---       #236
      01001C33H   LINE      CODE     ---       #237
      01001C33H   LINE      CODE     ---       #238
      01001C3AH   LINE      CODE     ---       #239
      01001C46H   LINE      CODE     ---       #240
      01001C49H   LINE      CODE     ---       #241
      01001C49H   LINE      CODE     ---       #242
      01001C49H   LINE      CODE     ---       #243
      01001C49H   LINE      CODE     ---       #244
      01001C49H   LINE      CODE     ---       #245
      01001C49H   LINE      CODE     ---       #246
      01001C53H   LINE      CODE     ---       #247
      01001C69H   LINE      CODE     ---       #249
      01001C70H   LINE      CODE     ---       #250
      01001C7CH   LINE      CODE     ---       #251
      01001C8EH   LINE      CODE     ---       #252
      01001C92H   LINE      CODE     ---       #253
      01001C95H   LINE      CODE     ---       #254
      01001C99H   LINE      CODE     ---       #255
      01001C99H   LINE      CODE     ---       #257
      01001C9CH   LINE      CODE     ---       #258
      01001C9CH   LINE      CODE     ---       #259
      01001CA5H   LINE      CODE     ---       #260
      01001CA7H   LINE      CODE     ---       #261
      01001CAAH   LINE      CODE     ---       #262
      01001CAAH   LINE      CODE     ---       #263
      01001CACH   LINE      CODE     ---       #264
      01001CACH   LINE      CODE     ---       #265
      01001CACH   LINE      CODE     ---       #266
      01001CACH   LINE      CODE     ---       #267
      01001CACH   LINE      CODE     ---       #268
      01001CACH   LINE      CODE     ---       #269
      01001CACH   LINE      CODE     ---       #270
      01001CACH   LINE      CODE     ---       #271
      01001CC2H   LINE      CODE     ---       #273
      01001CC9H   LINE      CODE     ---       #274
      01001CF5H   LINE      CODE     ---       #276
      01001D1EH   LINE      CODE     ---       #278
LX51 LINKER/LOCATER V4.66.30.0                                                        07/27/2019  23:22:19  PAGE 181


      01001D42H   LINE      CODE     ---       #280
      01001D45H   LINE      CODE     ---       #281
      01001D45H   LINE      CODE     ---       #282
      01001D45H   LINE      CODE     ---       #283
      01001D45H   LINE      CODE     ---       #284
      01001D5BH   LINE      CODE     ---       #285
      01001D73H   LINE      CODE     ---       #286
      01001D75H   LINE      CODE     ---       #287
      01001D75H   LINE      CODE     ---       #288
      01001D75H   LINE      CODE     ---       #289
      01001D8BH   LINE      CODE     ---       #290
      01001DB0H   LINE      CODE     ---       #291
      01001DB2H   LINE      CODE     ---       #292
      01001DB2H   LINE      CODE     ---       #293
      01001DB2H   LINE      CODE     ---       #294
      01001DC8H   LINE      CODE     ---       #295
      01001DF0H   LINE      CODE     ---       #296
      01001DF0H   LINE      CODE     ---       #297
      01001DF0H   LINE      CODE     ---       #298
      01001DF0H   LINE      CODE     ---       #300
      01001E13H   LINE      CODE     ---       #301
      01001E1FH   LINE      CODE     ---       #302
      01001E25H   LINE      CODE     ---       #303
      01001E3BH   LINE      CODE     ---       #306
      01001E4FH   LINE      CODE     ---       #308
      01001E4FH   LINE      CODE     ---       #309
      01001E56H   LINE      CODE     ---       #312
      01001E5BH   LINE      CODE     ---       #314
      01001E62H   LINE      CODE     ---       #315
      01001E65H   LINE      CODE     ---       #316
      01001E67H   LINE      CODE     ---       #317
      01001E6CH   LINE      CODE     ---       #318
      01001E6CH   LINE      CODE     ---       #320
      01001E73H   LINE      CODE     ---       #323
      01001E79H   LINE      CODE     ---       #324
      ---         BLOCKEND  ---      ---       LVL=0

      010041EAH   BLOCK     CODE     ---       LVL=0
      00000007H   SYMBOL    DATA     BYTE      idx
      010041EAH   BLOCK     CODE     NEAR LAB  LVL=1
      00000006H   SYMBOL    DATA     CHAR      a
      ---         BLOCKEND  ---      ---       LVL=1
      010041EAH   LINE      CODE     ---       #326
      010041EAH   LINE      CODE     ---       #327
      010041EAH   LINE      CODE     ---       #330
      01004207H   LINE      CODE     ---       #331
      01004207H   LINE      CODE     ---       #333
      0100420DH   LINE      CODE     ---       #334
      01004213H   LINE      CODE     ---       #336
      01004213H   LINE      CODE     ---       #337
      01004213H   LINE      CODE     ---       #338
      0100421EH   LINE      CODE     ---       #340
      01004227H   LINE      CODE     ---       #341
      01004229H   LINE      CODE     ---       #342
      01004229H   LINE      CODE     ---       #344
      01004231H   LINE      CODE     ---       #345
      01004238H   LINE      CODE     ---       #348
      01004238H   LINE      CODE     ---       #349
      01004238H   LINE      CODE     ---       #350
      01004243H   LINE      CODE     ---       #351
      01004247H   LINE      CODE     ---       #352
      0100424AH   LINE      CODE     ---       #353
LX51 LINKER/LOCATER V4.66.30.0                                                        07/27/2019  23:22:19  PAGE 182


      01004252H   LINE      CODE     ---       #354
      01004255H   LINE      CODE     ---       #355
      01004258H   LINE      CODE     ---       #356
      01004259H   LINE      CODE     ---       #357
      01004260H   LINE      CODE     ---       #358
      01004260H   LINE      CODE     ---       #359
      01004261H   LINE      CODE     ---       #362
      01004261H   LINE      CODE     ---       #363
      01004261H   LINE      CODE     ---       #364
      01004264H   LINE      CODE     ---       #365
      01004264H   LINE      CODE     ---       #366
      01004264H   LINE      CODE     ---       #367
      01004264H   LINE      CODE     ---       #368
      01004271H   LINE      CODE     ---       #369
      01004274H   LINE      CODE     ---       #370
      01004274H   LINE      CODE     ---       #372
      01004275H   LINE      CODE     ---       #373
      01004275H   LINE      CODE     ---       #374
      01004275H   LINE      CODE     ---       #375
      0100427CH   LINE      CODE     ---       #376
      0100427FH   LINE      CODE     ---       #377
      01004280H   LINE      CODE     ---       #378
      01004287H   LINE      CODE     ---       #379
      01004287H   LINE      CODE     ---       #380
      01004288H   LINE      CODE     ---       #381
      01004288H   LINE      CODE     ---       #382
      01004288H   LINE      CODE     ---       #383
      0100428FH   LINE      CODE     ---       #384
      01004292H   LINE      CODE     ---       #385
      01004293H   LINE      CODE     ---       #386
      0100429AH   LINE      CODE     ---       #387
      0100429AH   LINE      CODE     ---       #388
      0100429AH   LINE      CODE     ---       #389
      0100429AH   LINE      CODE     ---       #390
      0100429AH   LINE      CODE     ---       #391
      ---         BLOCKEND  ---      ---       LVL=0

      ---         MODULE    ---      ---       MENU_2_FN
      01004F73H   PUBLIC    CODE     ---       _menu_2_enter
      01001515H   PUBLIC    CODE     ---       _menu_2_disp
      010043F9H   PUBLIC    CODE     ---       _menu_2_btn_use
      01005B89H   PUBLIC    CODE     ---       menu_2_btn_exit
      0100510BH   PUBLIC    CODE     ---       menu_2_btn_prev
      010050BCH   PUBLIC    CODE     ---       menu_2_btn_next
      000000A2H   SFRSYM    DATA     BYTE      SPI0CKR
      00000080H   SFRSYM    DATA     BYTE      P0
      000000D0H.2 SFRSYM    DATA     BIT       PSW_OV
      000000B1H   SFRSYM    DATA     BYTE      XOSC0CN
      00000090H   SFRSYM    DATA     BYTE      P1
      000000A0H   SFRSYM    DATA     BYTE      P2
      000000B0H   SFRSYM    DATA     BYTE      P3
      000000BCH   SFRSYM    DATA     BYTE      ADC0CF
      000000C8H   SFRSYM    DATA     BIT       TMR2CN0_T2XCLK
      000000C7H   SFRSYM    DATA     BYTE      P4
      000000C0H.7 SFRSYM    DATA     BIT       SMB0CN0_MASTER
      000000F9H   SFRSYM    DATA     WORD      PCA0
      000000E6H   SFRSYM    DATA     BYTE      EIE1
      000000C0H.7 SFRSYM    DATA     BIT       SMB1CN0_MASTER
      000000C0H.1 SFRSYM    DATA     BIT       SMB0CN0_ACK
      000000D7H   SFRSYM    DATA     BYTE      USB0XCN
      000000E7H   SFRSYM    DATA     BYTE      EIE2
      000000C0H.1 SFRSYM    DATA     BIT       SMB1CN0_ACK
LX51 LINKER/LOCATER V4.66.30.0                                                        07/27/2019  23:22:19  PAGE 183


      0000008FH   SFRSYM    DATA     BYTE      PSCTL
      000000E4H   SFRSYM    DATA     BYTE      IT01CF
      000000C8H   SFRSYM    DATA     BIT       TMR5CN0_T5XCLK
      000000C0H.6 SFRSYM    DATA     BIT       SMB0CN0_TXMODE
      000000C0H.6 SFRSYM    DATA     BIT       SMB1CN0_TXMODE
      000000BFH   SFRSYM    DATA     BYTE      SFRPAGE
      000000A4H   SFRSYM    DATA     BYTE      P0MDOUT
      000000A5H   SFRSYM    DATA     BYTE      P1MDOUT
      000000E8H.5 SFRSYM    DATA     BIT       ADC0CN0_ADINT
      000000CBH   SFRSYM    DATA     BYTE      TMR2RLH
      000000A6H   SFRSYM    DATA     BYTE      P2MDOUT
      000000A8H   SFRSYM    DATA     BYTE      IE
      00000093H   SFRSYM    DATA     BYTE      TMR3RLH
      000000A7H   SFRSYM    DATA     BYTE      P3MDOUT
      00000093H   SFRSYM    DATA     BYTE      TMR4RLH
      000000AEH   SFRSYM    DATA     BYTE      P4MDOUT
      000000F6H   SFRSYM    DATA     BYTE      EIP1
      000000CBH   SFRSYM    DATA     BYTE      TMR5RLH
      000000F7H   SFRSYM    DATA     BYTE      EIP2
      00000098H.2 SFRSYM    DATA     BIT       SCON0_RB8
      000000CAH   SFRSYM    DATA     BYTE      TMR2RLL
      000000FCH   SFRSYM    DATA     BYTE      PCA0CPH0
      00000092H   SFRSYM    DATA     BYTE      TMR3RLL
      000000EAH   SFRSYM    DATA     BYTE      PCA0CPH1
      00000098H.3 SFRSYM    DATA     BIT       SCON0_TB8
      000000F0H   SFRSYM    DATA     BIT       B_B0
      00000082H   SFRSYM    DATA     WORD      DP
      00000092H   SFRSYM    DATA     BYTE      TMR4RLL
      000000ECH   SFRSYM    DATA     BYTE      PCA0CPH2
      000000F0H.1 SFRSYM    DATA     BIT       B_B1
      000000C3H   SFRSYM    DATA     WORD      ADC0GT
      000000CAH   SFRSYM    DATA     BYTE      TMR5RLL
      000000EEH   SFRSYM    DATA     BYTE      PCA0CPH3
      000000F0H.2 SFRSYM    DATA     BIT       B_B2
      000000FBH   SFRSYM    DATA     BYTE      PCA0CPL0
      000000FEH   SFRSYM    DATA     BYTE      PCA0CPH4
      00000085H   SFRSYM    DATA     BYTE      EMI0CF
      000000F0H.3 SFRSYM    DATA     BIT       B_B3
      000000D9H   SFRSYM    DATA     BYTE      PCA0MD
      000000DAH   SFRSYM    DATA     BYTE      PCA0CPM0
      000000E9H   SFRSYM    DATA     BYTE      PCA0CPL1
      000000F0H.4 SFRSYM    DATA     BIT       B_B4
      000000DBH   SFRSYM    DATA     BYTE      PCA0CPM1
      000000EBH   SFRSYM    DATA     BYTE      PCA0CPL2
      000000F0H.5 SFRSYM    DATA     BIT       B_B5
      000000DCH   SFRSYM    DATA     BYTE      PCA0CPM2
      000000EDH   SFRSYM    DATA     BYTE      PCA0CPL3
      000000B8H   SFRSYM    DATA     BYTE      IP
      000000F0H.6 SFRSYM    DATA     BIT       B_B6
      000000C5H   SFRSYM    DATA     WORD      ADC0LT
      000000DDH   SFRSYM    DATA     BYTE      PCA0CPM3
      000000FDH   SFRSYM    DATA     BYTE      PCA0CPL4
      00000098H.5 SFRSYM    DATA     BIT       SCON0_MCE
      000000F0H.7 SFRSYM    DATA     BIT       B_B7
      000000DEH   SFRSYM    DATA     BYTE      PCA0CPM4
      000000E1H   SFRSYM    DATA     BYTE      XBR0
      000000C1H   SFRSYM    DATA     BYTE      SMB0CF
      000000E2H   SFRSYM    DATA     BYTE      XBR1
      000000C1H   SFRSYM    DATA     BYTE      SMB1CF
      000000AFH   SFRSYM    DATA     BYTE      PFE0CN
      000000AAH   SFRSYM    DATA     BYTE      EMI0CN
      000000C0H.5 SFRSYM    DATA     BIT       SMB0CN0_STA
LX51 LINKER/LOCATER V4.66.30.0                                                        07/27/2019  23:22:19  PAGE 184


      000000E3H   SFRSYM    DATA     BYTE      XBR2
      000000C0H.5 SFRSYM    DATA     BIT       SMB1CN0_STA
      000000E0H   SFRSYM    DATA     BIT       ACC_ACC0
      000000D1H   SFRSYM    DATA     BYTE      REF0CN
      000000B2H   SFRSYM    DATA     BYTE      HFO0CN
      0000008EH   SFRSYM    DATA     BYTE      CKCON0
      000000E0H.1 SFRSYM    DATA     BIT       ACC_ACC1
      000000E4H   SFRSYM    DATA     BYTE      CKCON1
      000000C8H.2 SFRSYM    DATA     BIT       TMR2CN0_TR2
      000000E0H.2 SFRSYM    DATA     BIT       ACC_ACC2
      000000E0H.3 SFRSYM    DATA     BIT       ACC_ACC3
      00000081H   SFRSYM    DATA     BYTE      SP
      0000009DH   SFRSYM    DATA     BYTE      CMP0MD
      000000E0H.4 SFRSYM    DATA     BIT       ACC_ACC4
      00000086H   SFRSYM    DATA     BYTE      LFO0CN
      00000084H   SFRSYM    DATA     BYTE      EMI0TC
      0000009CH   SFRSYM    DATA     BYTE      CMP1MD
      000000D8H   SFRSYM    DATA     BIT       PCA0CN0_CCF0
      000000E0H.5 SFRSYM    DATA     BIT       ACC_ACC5
      000000D8H.1 SFRSYM    DATA     BIT       PCA0CN0_CCF1
      000000E0H.6 SFRSYM    DATA     BIT       ACC_ACC6
      000000CCH   SFRSYM    DATA     WORD      TMR2
      000000D8H.2 SFRSYM    DATA     BIT       PCA0CN0_CCF2
      000000E0H.7 SFRSYM    DATA     BIT       ACC_ACC7
      00000094H   SFRSYM    DATA     WORD      TMR3
      000000C8H.2 SFRSYM    DATA     BIT       TMR5CN0_TR5
      000000D8H.3 SFRSYM    DATA     BIT       PCA0CN0_CCF3
      00000094H   SFRSYM    DATA     WORD      TMR4
      000000ACH   SFRSYM    DATA     BYTE      SBCON1
      000000D8H.4 SFRSYM    DATA     BIT       PCA0CN0_CCF4
      000000CCH   SFRSYM    DATA     WORD      TMR5
      000000C0H.3 SFRSYM    DATA     BIT       SMB0CN0_ACKRQ
      000000FFH   SFRSYM    DATA     BYTE      VDM0CN
      000000F1H   SFRSYM    DATA     BYTE      P0MDIN
      000000C0H.3 SFRSYM    DATA     BIT       SMB1CN0_ACKRQ
      00000098H.4 SFRSYM    DATA     BIT       SCON0_REN
      000000F2H   SFRSYM    DATA     BYTE      P1MDIN
      000000F3H   SFRSYM    DATA     BYTE      P2MDIN
      000000C0H.4 SFRSYM    DATA     BIT       SMB0CN0_STO
      000000F4H   SFRSYM    DATA     BYTE      P3MDIN
      000000C0H.4 SFRSYM    DATA     BIT       SMB1CN0_STO
      000000B5H   SFRSYM    DATA     BYTE      SBRLH1
      000000F5H   SFRSYM    DATA     BYTE      P4MDIN
      000000D0H.3 SFRSYM    DATA     BIT       PSW_RS0
      000000D8H.7 SFRSYM    DATA     BIT       PCA0CN0_CF
      000000F8H.4 SFRSYM    DATA     BIT       SPI0CN0_RXOVRN
      000000D0H.4 SFRSYM    DATA     BIT       PSW_RS1
      000000B4H   SFRSYM    DATA     BYTE      SBRLL1
      000000E8H.7 SFRSYM    DATA     BIT       ADC0CN0_ADEN
      00000089H   SFRSYM    DATA     BYTE      TMOD
      00000088H   SFRSYM    DATA     BYTE      TCON
      000000D0H   SFRSYM    DATA     BIT       PSW_PARITY
      000000A8H.4 SFRSYM    DATA     BIT       IE_ES0
      0000009FH   SFRSYM    DATA     BYTE      CMP0MX
      000000A8H.1 SFRSYM    DATA     BIT       IE_ET0
      0000009EH   SFRSYM    DATA     BYTE      CMP1MX
      000000A8H.3 SFRSYM    DATA     BIT       IE_ET1
      000000D4H   SFRSYM    DATA     BYTE      P0SKIP
      000000C8H.1 SFRSYM    DATA     BIT       TMR2CN0_T2CSS
      000000A8H.5 SFRSYM    DATA     BIT       IE_ET2
      000000D5H   SFRSYM    DATA     BYTE      P1SKIP
      000000D6H   SFRSYM    DATA     BYTE      P2SKIP
LX51 LINKER/LOCATER V4.66.30.0                                                        07/27/2019  23:22:19  PAGE 185


      000000E8H   SFRSYM    DATA     BYTE      ADC0CN0
      000000A8H   SFRSYM    DATA     BIT       IE_EX0
      000000DFH   SFRSYM    DATA     BYTE      P3SKIP
      000000D8H.6 SFRSYM    DATA     BIT       PCA0CN0_CR
      000000A8H.2 SFRSYM    DATA     BIT       IE_EX1
      00000098H.7 SFRSYM    DATA     BIT       SCON0_SMODE
      000000A9H   SFRSYM    DATA     BYTE      CLKSEL
      000000F8H   SFRSYM    DATA     BIT       SPI0CN0_SPIEN
      000000F0H   SFRSYM    DATA     BYTE      B
      000000BEH   SFRSYM    DATA     BYTE      ADC0H
      000000E8H.6 SFRSYM    DATA     BIT       ADC0CN0_ADTM
      000000CAH   SFRSYM    DATA     WORD      TMR2RL
      000000BDH   SFRSYM    DATA     BYTE      ADC0L
      00000092H   SFRSYM    DATA     WORD      TMR3RL
      00000092H   SFRSYM    DATA     WORD      TMR4RL
      000000D8H   SFRSYM    DATA     BYTE      PCA0CN0
      000000E0H   SFRSYM    DATA     BYTE      ACC
      000000CAH   SFRSYM    DATA     WORD      TMR5RL
      000000FBH   SFRSYM    DATA     WORD      PCA0CP0
      000000E9H   SFRSYM    DATA     WORD      PCA0CP1
      000000EBH   SFRSYM    DATA     WORD      PCA0CP2
      000000EDH   SFRSYM    DATA     WORD      PCA0CP3
      0000008CH   SFRSYM    DATA     BYTE      TH0
      000000B8H.4 SFRSYM    DATA     BIT       IP_PS0
      000000FDH   SFRSYM    DATA     WORD      PCA0CP4
      0000008DH   SFRSYM    DATA     BYTE      TH1
      000000FAH   SFRSYM    DATA     BYTE      PCA0H
      000000B8H.1 SFRSYM    DATA     BIT       IP_PT0
      000000B8H.3 SFRSYM    DATA     BIT       IP_PT1
      000000C0H.2 SFRSYM    DATA     BIT       SMB0CN0_ARBLOST
      000000B8H.5 SFRSYM    DATA     BIT       IP_PT2
      0000008AH   SFRSYM    DATA     BYTE      TL0
      000000F8H.1 SFRSYM    DATA     BIT       SPI0CN0_TXBMT
      000000C0H.2 SFRSYM    DATA     BIT       SMB1CN0_ARBLOST
      000000D0H.5 SFRSYM    DATA     BIT       PSW_F0
      000000A8H.6 SFRSYM    DATA     BIT       IE_ESPI0
      0000008BH   SFRSYM    DATA     BYTE      TL1
      000000F9H   SFRSYM    DATA     BYTE      PCA0L
      000000C0H   SFRSYM    DATA     BIT       SMB0CN0_SI
      000000D0H.1 SFRSYM    DATA     BIT       PSW_F1
      00000080H   SFRSYM    DATA     BIT       P0_B0
      000000B8H   SFRSYM    DATA     BIT       IP_PX0
      000000C9H   SFRSYM    DATA     BYTE      REG01CN
      000000C0H   SFRSYM    DATA     BIT       SMB1CN0_SI
      00000090H   SFRSYM    DATA     BIT       P1_B0
      00000080H.1 SFRSYM    DATA     BIT       P0_B1
      000000B8H.2 SFRSYM    DATA     BIT       IP_PX1
      0000009BH   SFRSYM    DATA     BYTE      CMP0CN0
      00000088H.1 SFRSYM    DATA     BIT       TCON_IE0
      000000A0H   SFRSYM    DATA     BIT       P2_B0
      00000090H.1 SFRSYM    DATA     BIT       P1_B1
      00000080H.2 SFRSYM    DATA     BIT       P0_B2
      0000009AH   SFRSYM    DATA     BYTE      CMP1CN0
      00000088H.3 SFRSYM    DATA     BIT       TCON_IE1
      000000B0H   SFRSYM    DATA     BIT       P3_B0
      000000A0H.1 SFRSYM    DATA     BIT       P2_B1
      00000090H.2 SFRSYM    DATA     BIT       P1_B2
      00000080H.3 SFRSYM    DATA     BIT       P0_B3
      000000C0H   SFRSYM    DATA     BYTE      SMB0CN0
      000000B0H.1 SFRSYM    DATA     BIT       P3_B1
      000000A0H.2 SFRSYM    DATA     BIT       P2_B2
      00000090H.3 SFRSYM    DATA     BIT       P1_B3
LX51 LINKER/LOCATER V4.66.30.0                                                        07/27/2019  23:22:19  PAGE 186


      00000080H.4 SFRSYM    DATA     BIT       P0_B4
      000000C0H   SFRSYM    DATA     BYTE      SMB1CN0
      000000B0H.2 SFRSYM    DATA     BIT       P3_B2
      000000A0H.3 SFRSYM    DATA     BIT       P2_B3
      00000090H.4 SFRSYM    DATA     BIT       P1_B4
      00000080H.5 SFRSYM    DATA     BIT       P0_B5
      000000B0H.3 SFRSYM    DATA     BIT       P3_B3
      000000A0H.4 SFRSYM    DATA     BIT       P2_B4
      00000090H.5 SFRSYM    DATA     BIT       P1_B5
      00000080H.6 SFRSYM    DATA     BIT       P0_B6
      000000B0H.4 SFRSYM    DATA     BIT       P3_B4
      000000A0H.5 SFRSYM    DATA     BIT       P2_B5
      00000090H.6 SFRSYM    DATA     BIT       P1_B6
      00000080H.7 SFRSYM    DATA     BIT       P0_B7
      000000B0H.5 SFRSYM    DATA     BIT       P3_B5
      000000A0H.6 SFRSYM    DATA     BIT       P2_B6
      00000090H.7 SFRSYM    DATA     BIT       P1_B7
      000000B0H.6 SFRSYM    DATA     BIT       P3_B6
      000000A0H.7 SFRSYM    DATA     BIT       P2_B7
      000000B0H.7 SFRSYM    DATA     BIT       P3_B7
      00000083H   SFRSYM    DATA     BYTE      DPH
      000000C4H   SFRSYM    DATA     BYTE      ADC0GTH
      000000C8H.7 SFRSYM    DATA     BIT       TMR2CN0_TF2H
      000000C8H.3 SFRSYM    DATA     BIT       TMR2CN0_T2SPLIT
      000000D0H.6 SFRSYM    DATA     BIT       PSW_AC
      000000F8H   SFRSYM    DATA     BYTE      SPI0CN0
      000000B3H   SFRSYM    DATA     BYTE      HFO0CAL
      00000088H.5 SFRSYM    DATA     BIT       TCON_TF0
      00000098H   SFRSYM    DATA     BIT       SCON0_RI
      00000082H   SFRSYM    DATA     BYTE      DPL
      00000088H.7 SFRSYM    DATA     BIT       TCON_TF1
      00000099H   SFRSYM    DATA     BYTE      SBUF0
      00000087H   SFRSYM    DATA     BYTE      PCON0
      000000C3H   SFRSYM    DATA     BYTE      ADC0GTL
      000000C8H.6 SFRSYM    DATA     BIT       TMR2CN0_TF2L
      00000098H.1 SFRSYM    DATA     BIT       SCON0_TI
      000000E8H   SFRSYM    DATA     BIT       ADC0CN0_ADCM0
      000000D3H   SFRSYM    DATA     BYTE      SBUF1
      000000C6H   SFRSYM    DATA     BYTE      ADC0LTH
      00000088H   SFRSYM    DATA     BIT       TCON_IT0
      000000E8H.1 SFRSYM    DATA     BIT       ADC0CN0_ADCM1
      000000EFH   SFRSYM    DATA     BYTE      RSTSRC
      000000C8H.7 SFRSYM    DATA     BIT       TMR5CN0_TF5H
      000000C8H.3 SFRSYM    DATA     BIT       TMR5CN0_T5SPLIT
      00000088H.2 SFRSYM    DATA     BIT       TCON_IT1
      000000E8H.2 SFRSYM    DATA     BIT       ADC0CN0_ADCM2
      00000098H   SFRSYM    DATA     BYTE      SCON0
      000000E8H.3 SFRSYM    DATA     BIT       ADC0CN0_ADWINT
      000000B4H   SFRSYM    DATA     WORD      SBRL1
      000000E5H   SFRSYM    DATA     BYTE      SMOD1
      000000D2H   SFRSYM    DATA     BYTE      SCON1
      000000BAH   SFRSYM    DATA     BYTE      AMX0N
      000000E8H.4 SFRSYM    DATA     BIT       ADC0CN0_ADBUSY
      000000CEH   SFRSYM    DATA     BYTE      SMB0ADM
      000000C5H   SFRSYM    DATA     BYTE      ADC0LTL
      000000F8H.5 SFRSYM    DATA     BIT       SPI0CN0_MODF
      000000B8H.6 SFRSYM    DATA     BIT       IP_PSPI0
      000000CEH   SFRSYM    DATA     BYTE      SMB1ADM
      000000BBH   SFRSYM    DATA     BYTE      AMX0P
      000000C8H.6 SFRSYM    DATA     BIT       TMR5CN0_TF5L
      000000C8H   SFRSYM    DATA     BYTE      TMR2CN0
      00000091H   SFRSYM    DATA     BYTE      TMR3CN0
LX51 LINKER/LOCATER V4.66.30.0                                                        07/27/2019  23:22:19  PAGE 187


      00000091H   SFRSYM    DATA     BYTE      TMR4CN0
      000000C8H   SFRSYM    DATA     BYTE      TMR5CN0
      000000CFH   SFRSYM    DATA     BYTE      SMB0ADR
      00000088H.4 SFRSYM    DATA     BIT       TCON_TR0
      000000CFH   SFRSYM    DATA     BYTE      SMB1ADR
      000000C8H.4 SFRSYM    DATA     BIT       TMR2CN0_TF2CEN
      00000088H.6 SFRSYM    DATA     BIT       TCON_TR1
      000000C2H   SFRSYM    DATA     BYTE      SMB0DAT
      000000CDH   SFRSYM    DATA     BYTE      TMR2H
      000000A1H   SFRSYM    DATA     BYTE      SPI0CFG
      000000C2H   SFRSYM    DATA     BYTE      SMB1DAT
      00000095H   SFRSYM    DATA     BYTE      TMR3H
      00000095H   SFRSYM    DATA     BYTE      TMR4H
      000000CDH   SFRSYM    DATA     BYTE      TMR5H
      000000CCH   SFRSYM    DATA     BYTE      TMR2L
      000000F8H.7 SFRSYM    DATA     BIT       SPI0CN0_SPIF
      00000096H   SFRSYM    DATA     BYTE      USB0ADR
      00000094H   SFRSYM    DATA     BYTE      TMR3L
      000000A8H.7 SFRSYM    DATA     BIT       IE_EA
      00000094H   SFRSYM    DATA     BYTE      TMR4L
      00000097H   SFRSYM    DATA     BYTE      USB0DAT
      000000CCH   SFRSYM    DATA     BYTE      TMR5L
      000000B6H   SFRSYM    DATA     BYTE      FLSCL
      000000C8H.5 SFRSYM    DATA     BIT       TMR2CN0_TF2LEN
      000000F8H.6 SFRSYM    DATA     BIT       SPI0CN0_WCOL
      000000F8H.2 SFRSYM    DATA     BIT       SPI0CN0_NSSMD0
      000000D0H.7 SFRSYM    DATA     BIT       PSW_CY
      000000A3H   SFRSYM    DATA     BYTE      SPI0DAT
      000000F8H.3 SFRSYM    DATA     BIT       SPI0CN0_NSSMD1
      000000BDH   SFRSYM    DATA     WORD      ADC0
      000000B9H   SFRSYM    DATA     BYTE      SMBTC
      000000D0H   SFRSYM    DATA     BYTE      PSW
      000000C8H.5 SFRSYM    DATA     BIT       TMR5CN0_TF5LEN
      000000B7H   SFRSYM    DATA     BYTE      FLKEY
      01005A7AH   SYMBOL    CODE     ---       _menu_2_val_inc
      00000088H   SYMBOL    IDATA    BYTE      edit_mode
      00000089H   SYMBOL    IDATA    BYTE      edit_idx
      01005A97H   SYMBOL    CODE     ---       _menu_2_val_dec

      01005A7AH   BLOCK     CODE     ---       LVL=0
      00000001H   SYMBOL    DATA     ---       val
      00000005H   SYMBOL    DATA     BYTE      loop
      01005A7AH   LINE      CODE     ---       #23
      01005A7AH   LINE      CODE     ---       #24
      01005A7AH   LINE      CODE     ---       #25
      01005A83H   LINE      CODE     ---       #26
      01005A88H   LINE      CODE     ---       #27
      ---         BLOCKEND  ---      ---       LVL=0

      01005A97H   BLOCK     CODE     ---       LVL=0
      00000001H   SYMBOL    DATA     ---       val
      00000005H   SYMBOL    DATA     BYTE      loop
      01005A97H   LINE      CODE     ---       #29
      01005A97H   LINE      CODE     ---       #30
      01005A97H   LINE      CODE     ---       #31
      01005A9FH   LINE      CODE     ---       #32
      01005AA4H   LINE      CODE     ---       #33
      ---         BLOCKEND  ---      ---       LVL=0

      010050BCH   BLOCK     CODE     ---       LVL=0
      010050BCH   LINE      CODE     ---       #35
      010050BCH   LINE      CODE     ---       #36
LX51 LINKER/LOCATER V4.66.30.0                                                        07/27/2019  23:22:19  PAGE 188


      010050BCH   LINE      CODE     ---       #37
      010050D3H   LINE      CODE     ---       #38
      010050DBH   LINE      CODE     ---       #39
      010050E3H   LINE      CODE     ---       #40
      010050EBH   LINE      CODE     ---       #41
      010050F5H   LINE      CODE     ---       #42
      010050FFH   LINE      CODE     ---       #43
      0100510AH   LINE      CODE     ---       #44
      0100510AH   LINE      CODE     ---       #45
      ---         BLOCKEND  ---      ---       LVL=0

      0100510BH   BLOCK     CODE     ---       LVL=0
      0100510BH   LINE      CODE     ---       #47
      0100510BH   LINE      CODE     ---       #48
      0100510BH   LINE      CODE     ---       #49
      01005122H   LINE      CODE     ---       #50
      0100512AH   LINE      CODE     ---       #51
      01005132H   LINE      CODE     ---       #52
      0100513AH   LINE      CODE     ---       #53
      01005144H   LINE      CODE     ---       #54
      0100514EH   LINE      CODE     ---       #55
      01005159H   LINE      CODE     ---       #56
      01005159H   LINE      CODE     ---       #57
      ---         BLOCKEND  ---      ---       LVL=0

      01005B89H   BLOCK     CODE     ---       LVL=0
      01005B89H   LINE      CODE     ---       #59
      01005B89H   LINE      CODE     ---       #60
      01005B89H   LINE      CODE     ---       #61
      01005B8DH   LINE      CODE     ---       #62
      ---         BLOCKEND  ---      ---       LVL=0

      010043F9H   BLOCK     CODE     ---       LVL=0
      00000007H   SYMBOL    DATA     BYTE      idx
      010043F9H   LINE      CODE     ---       #65
      010043F9H   LINE      CODE     ---       #66
      010043F9H   LINE      CODE     ---       #67
      01004405H   LINE      CODE     ---       #68
      0100440BH   LINE      CODE     ---       #69
      01004417H   LINE      CODE     ---       #70
      0100441DH   LINE      CODE     ---       #71
      01004437H   LINE      CODE     ---       #73
      01004443H   LINE      CODE     ---       #74
      0100444FH   LINE      CODE     ---       #75
      01004455H   LINE      CODE     ---       #77
      01004461H   LINE      CODE     ---       #78
      0100446DH   LINE      CODE     ---       #79
      01004473H   LINE      CODE     ---       #81
      0100447FH   LINE      CODE     ---       #82
      01004485H   LINE      CODE     ---       #83
      01004491H   LINE      CODE     ---       #84
      01004497H   LINE      CODE     ---       #85
      010044A6H   LINE      CODE     ---       #86
      ---         BLOCKEND  ---      ---       LVL=0

      01001515H   BLOCK     CODE     ---       LVL=0
      00000022H   SYMBOL    DATA     BYTE      idx
      01001517H   BLOCK     CODE     NEAR LAB  LVL=1
      00000023H   SYMBOL    DATA     CHAR      w
      00000024H   SYMBOL    DATA     CHAR      x
      00000025H   SYMBOL    DATA     BYTE      f
      02000413H   SYMBOL    XDATA    ---       txt
LX51 LINKER/LOCATER V4.66.30.0                                                        07/27/2019  23:22:19  PAGE 189


      0100184DH   SYMBOL    CODE     VOID      MENU_2_DRAW_TEXT_DONE
      010016D9H   SYMBOL    CODE     VOID      MENU_2_EDIT_COLOR_LINE
      01001696H   SYMBOL    CODE     VOID      MENU_2_PCT_COLOR_TEXT
      ---         BLOCKEND  ---      ---       LVL=1
      01001515H   LINE      CODE     ---       #89
      01001517H   LINE      CODE     ---       #90
      01001517H   LINE      CODE     ---       #95
      0100151DH   LINE      CODE     ---       #96
      01001520H   LINE      CODE     ---       #97
      01001520H   LINE      CODE     ---       #99
      01001527H   LINE      CODE     ---       #101
      01001535H   LINE      CODE     ---       #102
      01001547H   LINE      CODE     ---       #103
      01001567H   LINE      CODE     ---       #104
      01001567H   LINE      CODE     ---       #107
      01001588H   LINE      CODE     ---       #108
      01001588H   LINE      CODE     ---       #109
      0100159EH   LINE      CODE     ---       #110
      010015A5H   LINE      CODE     ---       #111
      010015C8H   LINE      CODE     ---       #113
      010015CBH   LINE      CODE     ---       #114
      010015CBH   LINE      CODE     ---       #115
      010015CBH   LINE      CODE     ---       #116
      010015E1H   LINE      CODE     ---       #117
      01001601H   LINE      CODE     ---       #118
      01001604H   LINE      CODE     ---       #119
      01001604H   LINE      CODE     ---       #120
      01001604H   LINE      CODE     ---       #121
      01001604H   LINE      CODE     ---       #122
      0100161AH   LINE      CODE     ---       #125
      0100162DH   LINE      CODE     ---       #128
      01001636H   LINE      CODE     ---       #129
      0100163FH   LINE      CODE     ---       #131
      01001642H   LINE      CODE     ---       #132
      01001642H   LINE      CODE     ---       #133
      01001642H   LINE      CODE     ---       #134
      01001642H   LINE      CODE     ---       #135
      01001658H   LINE      CODE     ---       #138
      0100166BH   LINE      CODE     ---       #140
      0100166DH   LINE      CODE     ---       #141
      0100166DH   LINE      CODE     ---       #142
      0100166DH   LINE      CODE     ---       #143
      0100166DH   LINE      CODE     ---       #144
      01001683H   LINE      CODE     ---       #147
      01001696H   LINE      CODE     ---       #149
      01001696H   LINE      CODE     ---       #151
      010016BCH   LINE      CODE     ---       #152
      010016C3H   LINE      CODE     ---       #153
      010016D9H   LINE      CODE     ---       #155
      010016D9H   LINE      CODE     ---       #157
      010016E1H   LINE      CODE     ---       #158
      010016E5H   LINE      CODE     ---       #159
      010016EEH   LINE      CODE     ---       #162
      010016F7H   LINE      CODE     ---       #163
      01001700H   LINE      CODE     ---       #166
      0100170FH   LINE      CODE     ---       #167
      0100171EH   LINE      CODE     ---       #168
      0100172DH   LINE      CODE     ---       #170
      01001737H   LINE      CODE     ---       #171
      01001743H   LINE      CODE     ---       #173
      0100174AH   LINE      CODE     ---       #174
      01001760H   LINE      CODE     ---       #176
LX51 LINKER/LOCATER V4.66.30.0                                                        07/27/2019  23:22:19  PAGE 190


      01001766H   LINE      CODE     ---       #177
      0100177CH   LINE      CODE     ---       #179
      01001782H   LINE      CODE     ---       #180
      01001798H   LINE      CODE     ---       #182
      0100179EH   LINE      CODE     ---       #183
      010017B1H   LINE      CODE     ---       #184
      010017B3H   LINE      CODE     ---       #186
      010017BAH   LINE      CODE     ---       #187
      010017D0H   LINE      CODE     ---       #189
      010017D6H   LINE      CODE     ---       #190
      010017ECH   LINE      CODE     ---       #191
      010017ECH   LINE      CODE     ---       #192
      010017ECH   LINE      CODE     ---       #194
      010017EEH   LINE      CODE     ---       #195
      010017EEH   LINE      CODE     ---       #196
      010017EEH   LINE      CODE     ---       #198
      01001811H   LINE      CODE     ---       #199
      0100181DH   LINE      CODE     ---       #200
      01001823H   LINE      CODE     ---       #201
      01001839H   LINE      CODE     ---       #204
      0100184DH   LINE      CODE     ---       #206
      0100184DH   LINE      CODE     ---       #208
      01001852H   LINE      CODE     ---       #210
      ---         BLOCKEND  ---      ---       LVL=0

      01004F73H   BLOCK     CODE     ---       LVL=0
      00000007H   SYMBOL    DATA     BYTE      idx
      01004F73H   BLOCK     CODE     NEAR LAB  LVL=1
      00000022H   SYMBOL    DATA     BYTE      a
      ---         BLOCKEND  ---      ---       LVL=1
      01004F73H   LINE      CODE     ---       #213
      01004F73H   LINE      CODE     ---       #214
      01004F73H   LINE      CODE     ---       #217
      01004F77H   LINE      CODE     ---       #219
      01004F80H   LINE      CODE     ---       #220
      01004F80H   LINE      CODE     ---       #221
      01004F83H   LINE      CODE     ---       #222
      01004F89H   LINE      CODE     ---       #223
      01004F92H   LINE      CODE     ---       #224
      01004F96H   LINE      CODE     ---       #225
      01004F96H   LINE      CODE     ---       #226
      01004F97H   LINE      CODE     ---       #227
      01004F97H   LINE      CODE     ---       #228
      01004F97H   LINE      CODE     ---       #229
      01004FA1H   LINE      CODE     ---       #230
      01004FA3H   LINE      CODE     ---       #231
      01004FAAH   LINE      CODE     ---       #232
      01004FADH   LINE      CODE     ---       #233
      01004FADH   LINE      CODE     ---       #234
      01004FB5H   LINE      CODE     ---       #235
      01004FBCH   LINE      CODE     ---       #236
      01004FBDH   LINE      CODE     ---       #237
      01004FBDH   LINE      CODE     ---       #238
      01004FBDH   LINE      CODE     ---       #239
      01004FC3H   LINE      CODE     ---       #240
      01004FC5H   LINE      CODE     ---       #241
      01004FC8H   LINE      CODE     ---       #242
      01004FC8H   LINE      CODE     ---       #243
      01004FCCH   LINE      CODE     ---       #244
      01004FCCH   LINE      CODE     ---       #245
      01004FCCH   LINE      CODE     ---       #246
      01004FCCH   LINE      CODE     ---       #247
LX51 LINKER/LOCATER V4.66.30.0                                                        07/27/2019  23:22:19  PAGE 191


      ---         BLOCKEND  ---      ---       LVL=0

      ---         MODULE    ---      ---       MENU_5_FN
      01005317H   PUBLIC    CODE     ---       _menu_5_enter
      01002F4FH   PUBLIC    CODE     ---       _menu_5_disp
      000000A2H   SFRSYM    DATA     BYTE      SPI0CKR
      00000080H   SFRSYM    DATA     BYTE      P0
      000000D0H.2 SFRSYM    DATA     BIT       PSW_OV
      000000B1H   SFRSYM    DATA     BYTE      XOSC0CN
      00000090H   SFRSYM    DATA     BYTE      P1
      000000A0H   SFRSYM    DATA     BYTE      P2
      000000B0H   SFRSYM    DATA     BYTE      P3
      000000BCH   SFRSYM    DATA     BYTE      ADC0CF
      000000C8H   SFRSYM    DATA     BIT       TMR2CN0_T2XCLK
      000000C7H   SFRSYM    DATA     BYTE      P4
      000000C0H.7 SFRSYM    DATA     BIT       SMB0CN0_MASTER
      000000F9H   SFRSYM    DATA     WORD      PCA0
      000000E6H   SFRSYM    DATA     BYTE      EIE1
      000000C0H.7 SFRSYM    DATA     BIT       SMB1CN0_MASTER
      000000C0H.1 SFRSYM    DATA     BIT       SMB0CN0_ACK
      000000D7H   SFRSYM    DATA     BYTE      USB0XCN
      000000E7H   SFRSYM    DATA     BYTE      EIE2
      000000C0H.1 SFRSYM    DATA     BIT       SMB1CN0_ACK
      0000008FH   SFRSYM    DATA     BYTE      PSCTL
      000000E4H   SFRSYM    DATA     BYTE      IT01CF
      000000C8H   SFRSYM    DATA     BIT       TMR5CN0_T5XCLK
      000000C0H.6 SFRSYM    DATA     BIT       SMB0CN0_TXMODE
      000000C0H.6 SFRSYM    DATA     BIT       SMB1CN0_TXMODE
      000000BFH   SFRSYM    DATA     BYTE      SFRPAGE
      000000A4H   SFRSYM    DATA     BYTE      P0MDOUT
      000000A5H   SFRSYM    DATA     BYTE      P1MDOUT
      000000E8H.5 SFRSYM    DATA     BIT       ADC0CN0_ADINT
      000000CBH   SFRSYM    DATA     BYTE      TMR2RLH
      000000A6H   SFRSYM    DATA     BYTE      P2MDOUT
      000000A8H   SFRSYM    DATA     BYTE      IE
      00000093H   SFRSYM    DATA     BYTE      TMR3RLH
      000000A7H   SFRSYM    DATA     BYTE      P3MDOUT
      00000093H   SFRSYM    DATA     BYTE      TMR4RLH
      000000AEH   SFRSYM    DATA     BYTE      P4MDOUT
      000000F6H   SFRSYM    DATA     BYTE      EIP1
      000000CBH   SFRSYM    DATA     BYTE      TMR5RLH
      000000F7H   SFRSYM    DATA     BYTE      EIP2
      00000098H.2 SFRSYM    DATA     BIT       SCON0_RB8
      000000CAH   SFRSYM    DATA     BYTE      TMR2RLL
      000000FCH   SFRSYM    DATA     BYTE      PCA0CPH0
      00000092H   SFRSYM    DATA     BYTE      TMR3RLL
      000000EAH   SFRSYM    DATA     BYTE      PCA0CPH1
      00000098H.3 SFRSYM    DATA     BIT       SCON0_TB8
      000000F0H   SFRSYM    DATA     BIT       B_B0
      00000082H   SFRSYM    DATA     WORD      DP
      00000092H   SFRSYM    DATA     BYTE      TMR4RLL
      000000ECH   SFRSYM    DATA     BYTE      PCA0CPH2
      000000F0H.1 SFRSYM    DATA     BIT       B_B1
      000000C3H   SFRSYM    DATA     WORD      ADC0GT
      000000CAH   SFRSYM    DATA     BYTE      TMR5RLL
      000000EEH   SFRSYM    DATA     BYTE      PCA0CPH3
      000000F0H.2 SFRSYM    DATA     BIT       B_B2
      000000FBH   SFRSYM    DATA     BYTE      PCA0CPL0
      000000FEH   SFRSYM    DATA     BYTE      PCA0CPH4
      00000085H   SFRSYM    DATA     BYTE      EMI0CF
      000000F0H.3 SFRSYM    DATA     BIT       B_B3
      000000D9H   SFRSYM    DATA     BYTE      PCA0MD
LX51 LINKER/LOCATER V4.66.30.0                                                        07/27/2019  23:22:19  PAGE 192


      000000DAH   SFRSYM    DATA     BYTE      PCA0CPM0
      000000E9H   SFRSYM    DATA     BYTE      PCA0CPL1
      000000F0H.4 SFRSYM    DATA     BIT       B_B4
      000000DBH   SFRSYM    DATA     BYTE      PCA0CPM1
      000000EBH   SFRSYM    DATA     BYTE      PCA0CPL2
      000000F0H.5 SFRSYM    DATA     BIT       B_B5
      000000DCH   SFRSYM    DATA     BYTE      PCA0CPM2
      000000EDH   SFRSYM    DATA     BYTE      PCA0CPL3
      000000B8H   SFRSYM    DATA     BYTE      IP
      000000F0H.6 SFRSYM    DATA     BIT       B_B6
      000000C5H   SFRSYM    DATA     WORD      ADC0LT
      000000DDH   SFRSYM    DATA     BYTE      PCA0CPM3
      000000FDH   SFRSYM    DATA     BYTE      PCA0CPL4
      00000098H.5 SFRSYM    DATA     BIT       SCON0_MCE
      000000F0H.7 SFRSYM    DATA     BIT       B_B7
      000000DEH   SFRSYM    DATA     BYTE      PCA0CPM4
      000000E1H   SFRSYM    DATA     BYTE      XBR0
      000000C1H   SFRSYM    DATA     BYTE      SMB0CF
      000000E2H   SFRSYM    DATA     BYTE      XBR1
      000000C1H   SFRSYM    DATA     BYTE      SMB1CF
      000000AFH   SFRSYM    DATA     BYTE      PFE0CN
      000000AAH   SFRSYM    DATA     BYTE      EMI0CN
      000000C0H.5 SFRSYM    DATA     BIT       SMB0CN0_STA
      000000E3H   SFRSYM    DATA     BYTE      XBR2
      000000C0H.5 SFRSYM    DATA     BIT       SMB1CN0_STA
      000000E0H   SFRSYM    DATA     BIT       ACC_ACC0
      000000D1H   SFRSYM    DATA     BYTE      REF0CN
      000000B2H   SFRSYM    DATA     BYTE      HFO0CN
      0000008EH   SFRSYM    DATA     BYTE      CKCON0
      000000E0H.1 SFRSYM    DATA     BIT       ACC_ACC1
      000000E4H   SFRSYM    DATA     BYTE      CKCON1
      000000C8H.2 SFRSYM    DATA     BIT       TMR2CN0_TR2
      000000E0H.2 SFRSYM    DATA     BIT       ACC_ACC2
      000000E0H.3 SFRSYM    DATA     BIT       ACC_ACC3
      00000081H   SFRSYM    DATA     BYTE      SP
      0000009DH   SFRSYM    DATA     BYTE      CMP0MD
      000000E0H.4 SFRSYM    DATA     BIT       ACC_ACC4
      00000086H   SFRSYM    DATA     BYTE      LFO0CN
      00000084H   SFRSYM    DATA     BYTE      EMI0TC
      0000009CH   SFRSYM    DATA     BYTE      CMP1MD
      000000D8H   SFRSYM    DATA     BIT       PCA0CN0_CCF0
      000000E0H.5 SFRSYM    DATA     BIT       ACC_ACC5
      000000D8H.1 SFRSYM    DATA     BIT       PCA0CN0_CCF1
      000000E0H.6 SFRSYM    DATA     BIT       ACC_ACC6
      000000CCH   SFRSYM    DATA     WORD      TMR2
      000000D8H.2 SFRSYM    DATA     BIT       PCA0CN0_CCF2
      000000E0H.7 SFRSYM    DATA     BIT       ACC_ACC7
      00000094H   SFRSYM    DATA     WORD      TMR3
      000000C8H.2 SFRSYM    DATA     BIT       TMR5CN0_TR5
      000000D8H.3 SFRSYM    DATA     BIT       PCA0CN0_CCF3
      00000094H   SFRSYM    DATA     WORD      TMR4
      000000ACH   SFRSYM    DATA     BYTE      SBCON1
      000000D8H.4 SFRSYM    DATA     BIT       PCA0CN0_CCF4
      000000CCH   SFRSYM    DATA     WORD      TMR5
      000000C0H.3 SFRSYM    DATA     BIT       SMB0CN0_ACKRQ
      000000FFH   SFRSYM    DATA     BYTE      VDM0CN
      000000F1H   SFRSYM    DATA     BYTE      P0MDIN
      000000C0H.3 SFRSYM    DATA     BIT       SMB1CN0_ACKRQ
      00000098H.4 SFRSYM    DATA     BIT       SCON0_REN
      000000F2H   SFRSYM    DATA     BYTE      P1MDIN
      000000F3H   SFRSYM    DATA     BYTE      P2MDIN
      000000C0H.4 SFRSYM    DATA     BIT       SMB0CN0_STO
LX51 LINKER/LOCATER V4.66.30.0                                                        07/27/2019  23:22:19  PAGE 193


      000000F4H   SFRSYM    DATA     BYTE      P3MDIN
      000000C0H.4 SFRSYM    DATA     BIT       SMB1CN0_STO
      000000B5H   SFRSYM    DATA     BYTE      SBRLH1
      000000F5H   SFRSYM    DATA     BYTE      P4MDIN
      000000D0H.3 SFRSYM    DATA     BIT       PSW_RS0
      000000D8H.7 SFRSYM    DATA     BIT       PCA0CN0_CF
      000000F8H.4 SFRSYM    DATA     BIT       SPI0CN0_RXOVRN
      000000D0H.4 SFRSYM    DATA     BIT       PSW_RS1
      000000B4H   SFRSYM    DATA     BYTE      SBRLL1
      000000E8H.7 SFRSYM    DATA     BIT       ADC0CN0_ADEN
      00000089H   SFRSYM    DATA     BYTE      TMOD
      00000088H   SFRSYM    DATA     BYTE      TCON
      000000D0H   SFRSYM    DATA     BIT       PSW_PARITY
      000000A8H.4 SFRSYM    DATA     BIT       IE_ES0
      0000009FH   SFRSYM    DATA     BYTE      CMP0MX
      000000A8H.1 SFRSYM    DATA     BIT       IE_ET0
      0000009EH   SFRSYM    DATA     BYTE      CMP1MX
      000000A8H.3 SFRSYM    DATA     BIT       IE_ET1
      000000D4H   SFRSYM    DATA     BYTE      P0SKIP
      000000C8H.1 SFRSYM    DATA     BIT       TMR2CN0_T2CSS
      000000A8H.5 SFRSYM    DATA     BIT       IE_ET2
      000000D5H   SFRSYM    DATA     BYTE      P1SKIP
      000000D6H   SFRSYM    DATA     BYTE      P2SKIP
      000000E8H   SFRSYM    DATA     BYTE      ADC0CN0
      000000A8H   SFRSYM    DATA     BIT       IE_EX0
      000000DFH   SFRSYM    DATA     BYTE      P3SKIP
      000000D8H.6 SFRSYM    DATA     BIT       PCA0CN0_CR
      000000A8H.2 SFRSYM    DATA     BIT       IE_EX1
      00000098H.7 SFRSYM    DATA     BIT       SCON0_SMODE
      000000A9H   SFRSYM    DATA     BYTE      CLKSEL
      000000F8H   SFRSYM    DATA     BIT       SPI0CN0_SPIEN
      000000F0H   SFRSYM    DATA     BYTE      B
      000000BEH   SFRSYM    DATA     BYTE      ADC0H
      000000E8H.6 SFRSYM    DATA     BIT       ADC0CN0_ADTM
      000000CAH   SFRSYM    DATA     WORD      TMR2RL
      000000BDH   SFRSYM    DATA     BYTE      ADC0L
      00000092H   SFRSYM    DATA     WORD      TMR3RL
      00000092H   SFRSYM    DATA     WORD      TMR4RL
      000000D8H   SFRSYM    DATA     BYTE      PCA0CN0
      000000E0H   SFRSYM    DATA     BYTE      ACC
      000000CAH   SFRSYM    DATA     WORD      TMR5RL
      000000FBH   SFRSYM    DATA     WORD      PCA0CP0
      000000E9H   SFRSYM    DATA     WORD      PCA0CP1
      000000EBH   SFRSYM    DATA     WORD      PCA0CP2
      000000EDH   SFRSYM    DATA     WORD      PCA0CP3
      0000008CH   SFRSYM    DATA     BYTE      TH0
      000000B8H.4 SFRSYM    DATA     BIT       IP_PS0
      000000FDH   SFRSYM    DATA     WORD      PCA0CP4
      0000008DH   SFRSYM    DATA     BYTE      TH1
      000000FAH   SFRSYM    DATA     BYTE      PCA0H
      000000B8H.1 SFRSYM    DATA     BIT       IP_PT0
      000000B8H.3 SFRSYM    DATA     BIT       IP_PT1
      000000C0H.2 SFRSYM    DATA     BIT       SMB0CN0_ARBLOST
      000000B8H.5 SFRSYM    DATA     BIT       IP_PT2
      0000008AH   SFRSYM    DATA     BYTE      TL0
      000000F8H.1 SFRSYM    DATA     BIT       SPI0CN0_TXBMT
      000000C0H.2 SFRSYM    DATA     BIT       SMB1CN0_ARBLOST
      000000D0H.5 SFRSYM    DATA     BIT       PSW_F0
      000000A8H.6 SFRSYM    DATA     BIT       IE_ESPI0
      0000008BH   SFRSYM    DATA     BYTE      TL1
      000000F9H   SFRSYM    DATA     BYTE      PCA0L
      000000C0H   SFRSYM    DATA     BIT       SMB0CN0_SI
LX51 LINKER/LOCATER V4.66.30.0                                                        07/27/2019  23:22:19  PAGE 194


      000000D0H.1 SFRSYM    DATA     BIT       PSW_F1
      00000080H   SFRSYM    DATA     BIT       P0_B0
      000000B8H   SFRSYM    DATA     BIT       IP_PX0
      000000C9H   SFRSYM    DATA     BYTE      REG01CN
      000000C0H   SFRSYM    DATA     BIT       SMB1CN0_SI
      00000090H   SFRSYM    DATA     BIT       P1_B0
      00000080H.1 SFRSYM    DATA     BIT       P0_B1
      000000B8H.2 SFRSYM    DATA     BIT       IP_PX1
      0000009BH   SFRSYM    DATA     BYTE      CMP0CN0
      00000088H.1 SFRSYM    DATA     BIT       TCON_IE0
      000000A0H   SFRSYM    DATA     BIT       P2_B0
      00000090H.1 SFRSYM    DATA     BIT       P1_B1
      00000080H.2 SFRSYM    DATA     BIT       P0_B2
      0000009AH   SFRSYM    DATA     BYTE      CMP1CN0
      00000088H.3 SFRSYM    DATA     BIT       TCON_IE1
      000000B0H   SFRSYM    DATA     BIT       P3_B0
      000000A0H.1 SFRSYM    DATA     BIT       P2_B1
      00000090H.2 SFRSYM    DATA     BIT       P1_B2
      00000080H.3 SFRSYM    DATA     BIT       P0_B3
      000000C0H   SFRSYM    DATA     BYTE      SMB0CN0
      000000B0H.1 SFRSYM    DATA     BIT       P3_B1
      000000A0H.2 SFRSYM    DATA     BIT       P2_B2
      00000090H.3 SFRSYM    DATA     BIT       P1_B3
      00000080H.4 SFRSYM    DATA     BIT       P0_B4
      000000C0H   SFRSYM    DATA     BYTE      SMB1CN0
      000000B0H.2 SFRSYM    DATA     BIT       P3_B2
      000000A0H.3 SFRSYM    DATA     BIT       P2_B3
      00000090H.4 SFRSYM    DATA     BIT       P1_B4
      00000080H.5 SFRSYM    DATA     BIT       P0_B5
      000000B0H.3 SFRSYM    DATA     BIT       P3_B3
      000000A0H.4 SFRSYM    DATA     BIT       P2_B4
      00000090H.5 SFRSYM    DATA     BIT       P1_B5
      00000080H.6 SFRSYM    DATA     BIT       P0_B6
      000000B0H.4 SFRSYM    DATA     BIT       P3_B4
      000000A0H.5 SFRSYM    DATA     BIT       P2_B5
      00000090H.6 SFRSYM    DATA     BIT       P1_B6
      00000080H.7 SFRSYM    DATA     BIT       P0_B7
      000000B0H.5 SFRSYM    DATA     BIT       P3_B5
      000000A0H.6 SFRSYM    DATA     BIT       P2_B6
      00000090H.7 SFRSYM    DATA     BIT       P1_B7
      000000B0H.6 SFRSYM    DATA     BIT       P3_B6
      000000A0H.7 SFRSYM    DATA     BIT       P2_B7
      000000B0H.7 SFRSYM    DATA     BIT       P3_B7
      00000083H   SFRSYM    DATA     BYTE      DPH
      000000C4H   SFRSYM    DATA     BYTE      ADC0GTH
      000000C8H.7 SFRSYM    DATA     BIT       TMR2CN0_TF2H
      000000C8H.3 SFRSYM    DATA     BIT       TMR2CN0_T2SPLIT
      000000D0H.6 SFRSYM    DATA     BIT       PSW_AC
      000000F8H   SFRSYM    DATA     BYTE      SPI0CN0
      000000B3H   SFRSYM    DATA     BYTE      HFO0CAL
      00000088H.5 SFRSYM    DATA     BIT       TCON_TF0
      00000098H   SFRSYM    DATA     BIT       SCON0_RI
      00000082H   SFRSYM    DATA     BYTE      DPL
      00000088H.7 SFRSYM    DATA     BIT       TCON_TF1
      00000099H   SFRSYM    DATA     BYTE      SBUF0
      00000087H   SFRSYM    DATA     BYTE      PCON0
      000000C3H   SFRSYM    DATA     BYTE      ADC0GTL
      000000C8H.6 SFRSYM    DATA     BIT       TMR2CN0_TF2L
      00000098H.1 SFRSYM    DATA     BIT       SCON0_TI
      000000E8H   SFRSYM    DATA     BIT       ADC0CN0_ADCM0
      000000D3H   SFRSYM    DATA     BYTE      SBUF1
      000000C6H   SFRSYM    DATA     BYTE      ADC0LTH
LX51 LINKER/LOCATER V4.66.30.0                                                        07/27/2019  23:22:19  PAGE 195


      00000088H   SFRSYM    DATA     BIT       TCON_IT0
      000000E8H.1 SFRSYM    DATA     BIT       ADC0CN0_ADCM1
      000000EFH   SFRSYM    DATA     BYTE      RSTSRC
      000000C8H.7 SFRSYM    DATA     BIT       TMR5CN0_TF5H
      000000C8H.3 SFRSYM    DATA     BIT       TMR5CN0_T5SPLIT
      00000088H.2 SFRSYM    DATA     BIT       TCON_IT1
      000000E8H.2 SFRSYM    DATA     BIT       ADC0CN0_ADCM2
      00000098H   SFRSYM    DATA     BYTE      SCON0
      000000E8H.3 SFRSYM    DATA     BIT       ADC0CN0_ADWINT
      000000B4H   SFRSYM    DATA     WORD      SBRL1
      000000E5H   SFRSYM    DATA     BYTE      SMOD1
      000000D2H   SFRSYM    DATA     BYTE      SCON1
      000000BAH   SFRSYM    DATA     BYTE      AMX0N
      000000E8H.4 SFRSYM    DATA     BIT       ADC0CN0_ADBUSY
      000000CEH   SFRSYM    DATA     BYTE      SMB0ADM
      000000C5H   SFRSYM    DATA     BYTE      ADC0LTL
      000000F8H.5 SFRSYM    DATA     BIT       SPI0CN0_MODF
      000000B8H.6 SFRSYM    DATA     BIT       IP_PSPI0
      000000CEH   SFRSYM    DATA     BYTE      SMB1ADM
      000000BBH   SFRSYM    DATA     BYTE      AMX0P
      000000C8H.6 SFRSYM    DATA     BIT       TMR5CN0_TF5L
      000000C8H   SFRSYM    DATA     BYTE      TMR2CN0
      00000091H   SFRSYM    DATA     BYTE      TMR3CN0
      00000091H   SFRSYM    DATA     BYTE      TMR4CN0
      000000C8H   SFRSYM    DATA     BYTE      TMR5CN0
      000000CFH   SFRSYM    DATA     BYTE      SMB0ADR
      00000088H.4 SFRSYM    DATA     BIT       TCON_TR0
      000000CFH   SFRSYM    DATA     BYTE      SMB1ADR
      000000C8H.4 SFRSYM    DATA     BIT       TMR2CN0_TF2CEN
      00000088H.6 SFRSYM    DATA     BIT       TCON_TR1
      000000C2H   SFRSYM    DATA     BYTE      SMB0DAT
      000000CDH   SFRSYM    DATA     BYTE      TMR2H
      000000A1H   SFRSYM    DATA     BYTE      SPI0CFG
      000000C2H   SFRSYM    DATA     BYTE      SMB1DAT
      00000095H   SFRSYM    DATA     BYTE      TMR3H
      00000095H   SFRSYM    DATA     BYTE      TMR4H
      000000CDH   SFRSYM    DATA     BYTE      TMR5H
      000000CCH   SFRSYM    DATA     BYTE      TMR2L
      000000F8H.7 SFRSYM    DATA     BIT       SPI0CN0_SPIF
      00000096H   SFRSYM    DATA     BYTE      USB0ADR
      00000094H   SFRSYM    DATA     BYTE      TMR3L
      000000A8H.7 SFRSYM    DATA     BIT       IE_EA
      00000094H   SFRSYM    DATA     BYTE      TMR4L
      00000097H   SFRSYM    DATA     BYTE      USB0DAT
      000000CCH   SFRSYM    DATA     BYTE      TMR5L
      000000B6H   SFRSYM    DATA     BYTE      FLSCL
      000000C8H.5 SFRSYM    DATA     BIT       TMR2CN0_TF2LEN
      000000F8H.6 SFRSYM    DATA     BIT       SPI0CN0_WCOL
      000000F8H.2 SFRSYM    DATA     BIT       SPI0CN0_NSSMD0
      000000D0H.7 SFRSYM    DATA     BIT       PSW_CY
      000000A3H   SFRSYM    DATA     BYTE      SPI0DAT
      000000F8H.3 SFRSYM    DATA     BIT       SPI0CN0_NSSMD1
      000000BDH   SFRSYM    DATA     WORD      ADC0
      000000B9H   SFRSYM    DATA     BYTE      SMBTC
      000000D0H   SFRSYM    DATA     BYTE      PSW
      000000C8H.5 SFRSYM    DATA     BIT       TMR5CN0_TF5LEN
      000000B7H   SFRSYM    DATA     BYTE      FLKEY

      01002F4FH   BLOCK     CODE     ---       LVL=0
      00000022H   SYMBOL    DATA     BYTE      idx
      01002F51H   BLOCK     CODE     NEAR LAB  LVL=1
      00000023H   SYMBOL    DATA     CHAR      w
LX51 LINKER/LOCATER V4.66.30.0                                                        07/27/2019  23:22:19  PAGE 196


      00000024H   SYMBOL    DATA     CHAR      x
      02000413H   SYMBOL    XDATA    ---       txt
      ---         BLOCKEND  ---      ---       LVL=1
      01002F4FH   LINE      CODE     ---       #17
      01002F51H   LINE      CODE     ---       #18
      01002F51H   LINE      CODE     ---       #22
      01002F58H   LINE      CODE     ---       #25
      01002F67H   LINE      CODE     ---       #26
      01002F67H   LINE      CODE     ---       #27
      01002F7DH   LINE      CODE     ---       #28
      01002F96H   LINE      CODE     ---       #29
      01002F98H   LINE      CODE     ---       #30
      01002F98H   LINE      CODE     ---       #31
      01002F98H   LINE      CODE     ---       #32
      01002FAEH   LINE      CODE     ---       #33
      01002FC7H   LINE      CODE     ---       #34
      01002FC9H   LINE      CODE     ---       #35
      01002FC9H   LINE      CODE     ---       #36
      01002FC9H   LINE      CODE     ---       #37
      01002FDFH   LINE      CODE     ---       #38
      01003007H   LINE      CODE     ---       #39
      01003007H   LINE      CODE     ---       #40
      01003007H   LINE      CODE     ---       #41
      01003007H   LINE      CODE     ---       #43
      0100302AH   LINE      CODE     ---       #44
      01003036H   LINE      CODE     ---       #45
      0100303CH   LINE      CODE     ---       #46
      01003052H   LINE      CODE     ---       #49
      01003066H   LINE      CODE     ---       #52
      0100306BH   LINE      CODE     ---       #54
      ---         BLOCKEND  ---      ---       LVL=0

      01005317H   BLOCK     CODE     ---       LVL=0
      00000007H   SYMBOL    DATA     BYTE      idx
      01005317H   LINE      CODE     ---       #57
      01005317H   LINE      CODE     ---       #58
      01005317H   LINE      CODE     ---       #59
      01005322H   LINE      CODE     ---       #60
      01005322H   LINE      CODE     ---       #61
      01005329H   LINE      CODE     ---       #62
      0100532CH   LINE      CODE     ---       #63
      0100532DH   LINE      CODE     ---       #64
      01005334H   LINE      CODE     ---       #65
      01005334H   LINE      CODE     ---       #66
      01005335H   LINE      CODE     ---       #67
      01005335H   LINE      CODE     ---       #68
      01005335H   LINE      CODE     ---       #69
      0100533CH   LINE      CODE     ---       #70
      0100533FH   LINE      CODE     ---       #71
      01005340H   LINE      CODE     ---       #72
      01005347H   LINE      CODE     ---       #73
      01005347H   LINE      CODE     ---       #74
      01005348H   LINE      CODE     ---       #75
      01005348H   LINE      CODE     ---       #76
      01005348H   LINE      CODE     ---       #77
      0100534FH   LINE      CODE     ---       #78
      01005352H   LINE      CODE     ---       #79
      01005353H   LINE      CODE     ---       #80
      0100535AH   LINE      CODE     ---       #81
      0100535AH   LINE      CODE     ---       #82
      0100535AH   LINE      CODE     ---       #83
      0100535AH   LINE      CODE     ---       #84
LX51 LINKER/LOCATER V4.66.30.0                                                        07/27/2019  23:22:19  PAGE 197


      0100535AH   LINE      CODE     ---       #85
      ---         BLOCKEND  ---      ---       LVL=0

      ---         MODULE    ---      ---       MENU_6_FN
      00000064H   PUBLIC    DATA     BYTE      font_glyph
      00000063H   PUBLIC    DATA     BYTE      font_index
      010000A6H   PUBLIC    CODE     ---       _menu_6_disp
      010053DAH   PUBLIC    CODE     ---       menu_6_btn_use
      010059EEH   PUBLIC    CODE     ---       menu_6_font_prev
      010059DBH   PUBLIC    CODE     ---       menu_6_font_next
      01005573H   PUBLIC    CODE     ---       _menu_6_font_glyph
      010058DBH   PUBLIC    CODE     ---       _menu_6_font_index
      000000A2H   SFRSYM    DATA     BYTE      SPI0CKR
      00000080H   SFRSYM    DATA     BYTE      P0
      000000D0H.2 SFRSYM    DATA     BIT       PSW_OV
      000000B1H   SFRSYM    DATA     BYTE      XOSC0CN
      00000090H   SFRSYM    DATA     BYTE      P1
      000000A0H   SFRSYM    DATA     BYTE      P2
      000000B0H   SFRSYM    DATA     BYTE      P3
      000000BCH   SFRSYM    DATA     BYTE      ADC0CF
      000000C8H   SFRSYM    DATA     BIT       TMR2CN0_T2XCLK
      000000C7H   SFRSYM    DATA     BYTE      P4
      000000C0H.7 SFRSYM    DATA     BIT       SMB0CN0_MASTER
      000000F9H   SFRSYM    DATA     WORD      PCA0
      000000E6H   SFRSYM    DATA     BYTE      EIE1
      000000C0H.7 SFRSYM    DATA     BIT       SMB1CN0_MASTER
      000000C0H.1 SFRSYM    DATA     BIT       SMB0CN0_ACK
      000000D7H   SFRSYM    DATA     BYTE      USB0XCN
      000000E7H   SFRSYM    DATA     BYTE      EIE2
      000000C0H.1 SFRSYM    DATA     BIT       SMB1CN0_ACK
      0000008FH   SFRSYM    DATA     BYTE      PSCTL
      000000E4H   SFRSYM    DATA     BYTE      IT01CF
      000000C8H   SFRSYM    DATA     BIT       TMR5CN0_T5XCLK
      000000C0H.6 SFRSYM    DATA     BIT       SMB0CN0_TXMODE
      000000C0H.6 SFRSYM    DATA     BIT       SMB1CN0_TXMODE
      000000BFH   SFRSYM    DATA     BYTE      SFRPAGE
      000000A4H   SFRSYM    DATA     BYTE      P0MDOUT
      000000A5H   SFRSYM    DATA     BYTE      P1MDOUT
      000000E8H.5 SFRSYM    DATA     BIT       ADC0CN0_ADINT
      000000CBH   SFRSYM    DATA     BYTE      TMR2RLH
      000000A6H   SFRSYM    DATA     BYTE      P2MDOUT
      000000A8H   SFRSYM    DATA     BYTE      IE
      00000093H   SFRSYM    DATA     BYTE      TMR3RLH
      000000A7H   SFRSYM    DATA     BYTE      P3MDOUT
      00000093H   SFRSYM    DATA     BYTE      TMR4RLH
      000000AEH   SFRSYM    DATA     BYTE      P4MDOUT
      000000F6H   SFRSYM    DATA     BYTE      EIP1
      000000CBH   SFRSYM    DATA     BYTE      TMR5RLH
      000000F7H   SFRSYM    DATA     BYTE      EIP2
      00000098H.2 SFRSYM    DATA     BIT       SCON0_RB8
      000000CAH   SFRSYM    DATA     BYTE      TMR2RLL
      000000FCH   SFRSYM    DATA     BYTE      PCA0CPH0
      00000092H   SFRSYM    DATA     BYTE      TMR3RLL
      000000EAH   SFRSYM    DATA     BYTE      PCA0CPH1
      00000098H.3 SFRSYM    DATA     BIT       SCON0_TB8
      000000F0H   SFRSYM    DATA     BIT       B_B0
      00000082H   SFRSYM    DATA     WORD      DP
      00000092H   SFRSYM    DATA     BYTE      TMR4RLL
      000000ECH   SFRSYM    DATA     BYTE      PCA0CPH2
      000000F0H.1 SFRSYM    DATA     BIT       B_B1
      000000C3H   SFRSYM    DATA     WORD      ADC0GT
      000000CAH   SFRSYM    DATA     BYTE      TMR5RLL
LX51 LINKER/LOCATER V4.66.30.0                                                        07/27/2019  23:22:19  PAGE 198


      000000EEH   SFRSYM    DATA     BYTE      PCA0CPH3
      000000F0H.2 SFRSYM    DATA     BIT       B_B2
      000000FBH   SFRSYM    DATA     BYTE      PCA0CPL0
      000000FEH   SFRSYM    DATA     BYTE      PCA0CPH4
      00000085H   SFRSYM    DATA     BYTE      EMI0CF
      000000F0H.3 SFRSYM    DATA     BIT       B_B3
      000000D9H   SFRSYM    DATA     BYTE      PCA0MD
      000000DAH   SFRSYM    DATA     BYTE      PCA0CPM0
      000000E9H   SFRSYM    DATA     BYTE      PCA0CPL1
      000000F0H.4 SFRSYM    DATA     BIT       B_B4
      000000DBH   SFRSYM    DATA     BYTE      PCA0CPM1
      000000EBH   SFRSYM    DATA     BYTE      PCA0CPL2
      000000F0H.5 SFRSYM    DATA     BIT       B_B5
      000000DCH   SFRSYM    DATA     BYTE      PCA0CPM2
      000000EDH   SFRSYM    DATA     BYTE      PCA0CPL3
      000000B8H   SFRSYM    DATA     BYTE      IP
      000000F0H.6 SFRSYM    DATA     BIT       B_B6
      000000C5H   SFRSYM    DATA     WORD      ADC0LT
      000000DDH   SFRSYM    DATA     BYTE      PCA0CPM3
      000000FDH   SFRSYM    DATA     BYTE      PCA0CPL4
      00000098H.5 SFRSYM    DATA     BIT       SCON0_MCE
      000000F0H.7 SFRSYM    DATA     BIT       B_B7
      000000DEH   SFRSYM    DATA     BYTE      PCA0CPM4
      000000E1H   SFRSYM    DATA     BYTE      XBR0
      000000C1H   SFRSYM    DATA     BYTE      SMB0CF
      000000E2H   SFRSYM    DATA     BYTE      XBR1
      000000C1H   SFRSYM    DATA     BYTE      SMB1CF
      000000AFH   SFRSYM    DATA     BYTE      PFE0CN
      000000AAH   SFRSYM    DATA     BYTE      EMI0CN
      000000C0H.5 SFRSYM    DATA     BIT       SMB0CN0_STA
      000000E3H   SFRSYM    DATA     BYTE      XBR2
      000000C0H.5 SFRSYM    DATA     BIT       SMB1CN0_STA
      000000E0H   SFRSYM    DATA     BIT       ACC_ACC0
      000000D1H   SFRSYM    DATA     BYTE      REF0CN
      000000B2H   SFRSYM    DATA     BYTE      HFO0CN
      0000008EH   SFRSYM    DATA     BYTE      CKCON0
      000000E0H.1 SFRSYM    DATA     BIT       ACC_ACC1
      000000E4H   SFRSYM    DATA     BYTE      CKCON1
      000000C8H.2 SFRSYM    DATA     BIT       TMR2CN0_TR2
      000000E0H.2 SFRSYM    DATA     BIT       ACC_ACC2
      000000E0H.3 SFRSYM    DATA     BIT       ACC_ACC3
      00000081H   SFRSYM    DATA     BYTE      SP
      0000009DH   SFRSYM    DATA     BYTE      CMP0MD
      000000E0H.4 SFRSYM    DATA     BIT       ACC_ACC4
      00000086H   SFRSYM    DATA     BYTE      LFO0CN
      00000084H   SFRSYM    DATA     BYTE      EMI0TC
      0000009CH   SFRSYM    DATA     BYTE      CMP1MD
      000000D8H   SFRSYM    DATA     BIT       PCA0CN0_CCF0
      000000E0H.5 SFRSYM    DATA     BIT       ACC_ACC5
      000000D8H.1 SFRSYM    DATA     BIT       PCA0CN0_CCF1
      000000E0H.6 SFRSYM    DATA     BIT       ACC_ACC6
      000000CCH   SFRSYM    DATA     WORD      TMR2
      000000D8H.2 SFRSYM    DATA     BIT       PCA0CN0_CCF2
      000000E0H.7 SFRSYM    DATA     BIT       ACC_ACC7
      00000094H   SFRSYM    DATA     WORD      TMR3
      000000C8H.2 SFRSYM    DATA     BIT       TMR5CN0_TR5
      000000D8H.3 SFRSYM    DATA     BIT       PCA0CN0_CCF3
      00000094H   SFRSYM    DATA     WORD      TMR4
      000000ACH   SFRSYM    DATA     BYTE      SBCON1
      000000D8H.4 SFRSYM    DATA     BIT       PCA0CN0_CCF4
      000000CCH   SFRSYM    DATA     WORD      TMR5
      000000C0H.3 SFRSYM    DATA     BIT       SMB0CN0_ACKRQ
LX51 LINKER/LOCATER V4.66.30.0                                                        07/27/2019  23:22:19  PAGE 199


      000000FFH   SFRSYM    DATA     BYTE      VDM0CN
      000000F1H   SFRSYM    DATA     BYTE      P0MDIN
      000000C0H.3 SFRSYM    DATA     BIT       SMB1CN0_ACKRQ
      00000098H.4 SFRSYM    DATA     BIT       SCON0_REN
      000000F2H   SFRSYM    DATA     BYTE      P1MDIN
      000000F3H   SFRSYM    DATA     BYTE      P2MDIN
      000000C0H.4 SFRSYM    DATA     BIT       SMB0CN0_STO
      000000F4H   SFRSYM    DATA     BYTE      P3MDIN
      000000C0H.4 SFRSYM    DATA     BIT       SMB1CN0_STO
      000000B5H   SFRSYM    DATA     BYTE      SBRLH1
      000000F5H   SFRSYM    DATA     BYTE      P4MDIN
      000000D0H.3 SFRSYM    DATA     BIT       PSW_RS0
      000000D8H.7 SFRSYM    DATA     BIT       PCA0CN0_CF
      000000F8H.4 SFRSYM    DATA     BIT       SPI0CN0_RXOVRN
      000000D0H.4 SFRSYM    DATA     BIT       PSW_RS1
      000000B4H   SFRSYM    DATA     BYTE      SBRLL1
      000000E8H.7 SFRSYM    DATA     BIT       ADC0CN0_ADEN
      00000089H   SFRSYM    DATA     BYTE      TMOD
      00000088H   SFRSYM    DATA     BYTE      TCON
      000000D0H   SFRSYM    DATA     BIT       PSW_PARITY
      000000A8H.4 SFRSYM    DATA     BIT       IE_ES0
      0000009FH   SFRSYM    DATA     BYTE      CMP0MX
      000000A8H.1 SFRSYM    DATA     BIT       IE_ET0
      0000009EH   SFRSYM    DATA     BYTE      CMP1MX
      000000A8H.3 SFRSYM    DATA     BIT       IE_ET1
      000000D4H   SFRSYM    DATA     BYTE      P0SKIP
      000000C8H.1 SFRSYM    DATA     BIT       TMR2CN0_T2CSS
      000000A8H.5 SFRSYM    DATA     BIT       IE_ET2
      000000D5H   SFRSYM    DATA     BYTE      P1SKIP
      000000D6H   SFRSYM    DATA     BYTE      P2SKIP
      000000E8H   SFRSYM    DATA     BYTE      ADC0CN0
      000000A8H   SFRSYM    DATA     BIT       IE_EX0
      000000DFH   SFRSYM    DATA     BYTE      P3SKIP
      000000D8H.6 SFRSYM    DATA     BIT       PCA0CN0_CR
      000000A8H.2 SFRSYM    DATA     BIT       IE_EX1
      00000098H.7 SFRSYM    DATA     BIT       SCON0_SMODE
      000000A9H   SFRSYM    DATA     BYTE      CLKSEL
      000000F8H   SFRSYM    DATA     BIT       SPI0CN0_SPIEN
      000000F0H   SFRSYM    DATA     BYTE      B
      000000BEH   SFRSYM    DATA     BYTE      ADC0H
      000000E8H.6 SFRSYM    DATA     BIT       ADC0CN0_ADTM
      000000CAH   SFRSYM    DATA     WORD      TMR2RL
      000000BDH   SFRSYM    DATA     BYTE      ADC0L
      00000092H   SFRSYM    DATA     WORD      TMR3RL
      00000092H   SFRSYM    DATA     WORD      TMR4RL
      000000D8H   SFRSYM    DATA     BYTE      PCA0CN0
      000000E0H   SFRSYM    DATA     BYTE      ACC
      000000CAH   SFRSYM    DATA     WORD      TMR5RL
      000000FBH   SFRSYM    DATA     WORD      PCA0CP0
      000000E9H   SFRSYM    DATA     WORD      PCA0CP1
      000000EBH   SFRSYM    DATA     WORD      PCA0CP2
      000000EDH   SFRSYM    DATA     WORD      PCA0CP3
      0000008CH   SFRSYM    DATA     BYTE      TH0
      000000B8H.4 SFRSYM    DATA     BIT       IP_PS0
      000000FDH   SFRSYM    DATA     WORD      PCA0CP4
      0000008DH   SFRSYM    DATA     BYTE      TH1
      000000FAH   SFRSYM    DATA     BYTE      PCA0H
      000000B8H.1 SFRSYM    DATA     BIT       IP_PT0
      000000B8H.3 SFRSYM    DATA     BIT       IP_PT1
      000000C0H.2 SFRSYM    DATA     BIT       SMB0CN0_ARBLOST
      000000B8H.5 SFRSYM    DATA     BIT       IP_PT2
      0000008AH   SFRSYM    DATA     BYTE      TL0
LX51 LINKER/LOCATER V4.66.30.0                                                        07/27/2019  23:22:19  PAGE 200


      000000F8H.1 SFRSYM    DATA     BIT       SPI0CN0_TXBMT
      000000C0H.2 SFRSYM    DATA     BIT       SMB1CN0_ARBLOST
      000000D0H.5 SFRSYM    DATA     BIT       PSW_F0
      000000A8H.6 SFRSYM    DATA     BIT       IE_ESPI0
      0000008BH   SFRSYM    DATA     BYTE      TL1
      000000F9H   SFRSYM    DATA     BYTE      PCA0L
      000000C0H   SFRSYM    DATA     BIT       SMB0CN0_SI
      000000D0H.1 SFRSYM    DATA     BIT       PSW_F1
      00000080H   SFRSYM    DATA     BIT       P0_B0
      000000B8H   SFRSYM    DATA     BIT       IP_PX0
      000000C9H   SFRSYM    DATA     BYTE      REG01CN
      000000C0H   SFRSYM    DATA     BIT       SMB1CN0_SI
      00000090H   SFRSYM    DATA     BIT       P1_B0
      00000080H.1 SFRSYM    DATA     BIT       P0_B1
      000000B8H.2 SFRSYM    DATA     BIT       IP_PX1
      0000009BH   SFRSYM    DATA     BYTE      CMP0CN0
      00000088H.1 SFRSYM    DATA     BIT       TCON_IE0
      000000A0H   SFRSYM    DATA     BIT       P2_B0
      00000090H.1 SFRSYM    DATA     BIT       P1_B1
      00000080H.2 SFRSYM    DATA     BIT       P0_B2
      0000009AH   SFRSYM    DATA     BYTE      CMP1CN0
      00000088H.3 SFRSYM    DATA     BIT       TCON_IE1
      000000B0H   SFRSYM    DATA     BIT       P3_B0
      000000A0H.1 SFRSYM    DATA     BIT       P2_B1
      00000090H.2 SFRSYM    DATA     BIT       P1_B2
      00000080H.3 SFRSYM    DATA     BIT       P0_B3
      000000C0H   SFRSYM    DATA     BYTE      SMB0CN0
      000000B0H.1 SFRSYM    DATA     BIT       P3_B1
      000000A0H.2 SFRSYM    DATA     BIT       P2_B2
      00000090H.3 SFRSYM    DATA     BIT       P1_B3
      00000080H.4 SFRSYM    DATA     BIT       P0_B4
      000000C0H   SFRSYM    DATA     BYTE      SMB1CN0
      000000B0H.2 SFRSYM    DATA     BIT       P3_B2
      000000A0H.3 SFRSYM    DATA     BIT       P2_B3
      00000090H.4 SFRSYM    DATA     BIT       P1_B4
      00000080H.5 SFRSYM    DATA     BIT       P0_B5
      000000B0H.3 SFRSYM    DATA     BIT       P3_B3
      000000A0H.4 SFRSYM    DATA     BIT       P2_B4
      00000090H.5 SFRSYM    DATA     BIT       P1_B5
      00000080H.6 SFRSYM    DATA     BIT       P0_B6
      000000B0H.4 SFRSYM    DATA     BIT       P3_B4
      000000A0H.5 SFRSYM    DATA     BIT       P2_B5
      00000090H.6 SFRSYM    DATA     BIT       P1_B6
      00000080H.7 SFRSYM    DATA     BIT       P0_B7
      000000B0H.5 SFRSYM    DATA     BIT       P3_B5
      000000A0H.6 SFRSYM    DATA     BIT       P2_B6
      00000090H.7 SFRSYM    DATA     BIT       P1_B7
      000000B0H.6 SFRSYM    DATA     BIT       P3_B6
      000000A0H.7 SFRSYM    DATA     BIT       P2_B7
      000000B0H.7 SFRSYM    DATA     BIT       P3_B7
      00000083H   SFRSYM    DATA     BYTE      DPH
      000000C4H   SFRSYM    DATA     BYTE      ADC0GTH
      000000C8H.7 SFRSYM    DATA     BIT       TMR2CN0_TF2H
      000000C8H.3 SFRSYM    DATA     BIT       TMR2CN0_T2SPLIT
      000000D0H.6 SFRSYM    DATA     BIT       PSW_AC
      000000F8H   SFRSYM    DATA     BYTE      SPI0CN0
      000000B3H   SFRSYM    DATA     BYTE      HFO0CAL
      00000088H.5 SFRSYM    DATA     BIT       TCON_TF0
      00000098H   SFRSYM    DATA     BIT       SCON0_RI
      00000082H   SFRSYM    DATA     BYTE      DPL
      00000088H.7 SFRSYM    DATA     BIT       TCON_TF1
      00000099H   SFRSYM    DATA     BYTE      SBUF0
LX51 LINKER/LOCATER V4.66.30.0                                                        07/27/2019  23:22:19  PAGE 201


      00000087H   SFRSYM    DATA     BYTE      PCON0
      000000C3H   SFRSYM    DATA     BYTE      ADC0GTL
      000000C8H.6 SFRSYM    DATA     BIT       TMR2CN0_TF2L
      00000098H.1 SFRSYM    DATA     BIT       SCON0_TI
      000000E8H   SFRSYM    DATA     BIT       ADC0CN0_ADCM0
      000000D3H   SFRSYM    DATA     BYTE      SBUF1
      000000C6H   SFRSYM    DATA     BYTE      ADC0LTH
      00000088H   SFRSYM    DATA     BIT       TCON_IT0
      000000E8H.1 SFRSYM    DATA     BIT       ADC0CN0_ADCM1
      000000EFH   SFRSYM    DATA     BYTE      RSTSRC
      000000C8H.7 SFRSYM    DATA     BIT       TMR5CN0_TF5H
      000000C8H.3 SFRSYM    DATA     BIT       TMR5CN0_T5SPLIT
      00000088H.2 SFRSYM    DATA     BIT       TCON_IT1
      000000E8H.2 SFRSYM    DATA     BIT       ADC0CN0_ADCM2
      00000098H   SFRSYM    DATA     BYTE      SCON0
      000000E8H.3 SFRSYM    DATA     BIT       ADC0CN0_ADWINT
      000000B4H   SFRSYM    DATA     WORD      SBRL1
      000000E5H   SFRSYM    DATA     BYTE      SMOD1
      000000D2H   SFRSYM    DATA     BYTE      SCON1
      000000BAH   SFRSYM    DATA     BYTE      AMX0N
      000000E8H.4 SFRSYM    DATA     BIT       ADC0CN0_ADBUSY
      000000CEH   SFRSYM    DATA     BYTE      SMB0ADM
      000000C5H   SFRSYM    DATA     BYTE      ADC0LTL
      000000F8H.5 SFRSYM    DATA     BIT       SPI0CN0_MODF
      000000B8H.6 SFRSYM    DATA     BIT       IP_PSPI0
      000000CEH   SFRSYM    DATA     BYTE      SMB1ADM
      000000BBH   SFRSYM    DATA     BYTE      AMX0P
      000000C8H.6 SFRSYM    DATA     BIT       TMR5CN0_TF5L
      000000C8H   SFRSYM    DATA     BYTE      TMR2CN0
      00000091H   SFRSYM    DATA     BYTE      TMR3CN0
      00000091H   SFRSYM    DATA     BYTE      TMR4CN0
      000000C8H   SFRSYM    DATA     BYTE      TMR5CN0
      000000CFH   SFRSYM    DATA     BYTE      SMB0ADR
      00000088H.4 SFRSYM    DATA     BIT       TCON_TR0
      000000CFH   SFRSYM    DATA     BYTE      SMB1ADR
      000000C8H.4 SFRSYM    DATA     BIT       TMR2CN0_TF2CEN
      00000088H.6 SFRSYM    DATA     BIT       TCON_TR1
      000000C2H   SFRSYM    DATA     BYTE      SMB0DAT
      000000CDH   SFRSYM    DATA     BYTE      TMR2H
      000000A1H   SFRSYM    DATA     BYTE      SPI0CFG
      000000C2H   SFRSYM    DATA     BYTE      SMB1DAT
      00000095H   SFRSYM    DATA     BYTE      TMR3H
      00000095H   SFRSYM    DATA     BYTE      TMR4H
      000000CDH   SFRSYM    DATA     BYTE      TMR5H
      000000CCH   SFRSYM    DATA     BYTE      TMR2L
      000000F8H.7 SFRSYM    DATA     BIT       SPI0CN0_SPIF
      00000096H   SFRSYM    DATA     BYTE      USB0ADR
      00000094H   SFRSYM    DATA     BYTE      TMR3L
      000000A8H.7 SFRSYM    DATA     BIT       IE_EA
      00000094H   SFRSYM    DATA     BYTE      TMR4L
      00000097H   SFRSYM    DATA     BYTE      USB0DAT
      000000CCH   SFRSYM    DATA     BYTE      TMR5L
      000000B6H   SFRSYM    DATA     BYTE      FLSCL
      000000C8H.5 SFRSYM    DATA     BIT       TMR2CN0_TF2LEN
      000000F8H.6 SFRSYM    DATA     BIT       SPI0CN0_WCOL
      000000F8H.2 SFRSYM    DATA     BIT       SPI0CN0_NSSMD0
      000000D0H.7 SFRSYM    DATA     BIT       PSW_CY
      000000A3H   SFRSYM    DATA     BYTE      SPI0DAT
      000000F8H.3 SFRSYM    DATA     BIT       SPI0CN0_NSSMD1
      000000BDH   SFRSYM    DATA     WORD      ADC0
      000000B9H   SFRSYM    DATA     BYTE      SMBTC
      000000D0H   SFRSYM    DATA     BYTE      PSW
LX51 LINKER/LOCATER V4.66.30.0                                                        07/27/2019  23:22:19  PAGE 202


      000000C8H.5 SFRSYM    DATA     BIT       TMR5CN0_TF5LEN
      000000B7H   SFRSYM    DATA     BYTE      FLKEY

      010058DBH   BLOCK     CODE     ---       LVL=0
      00000007H   SYMBOL    DATA     CHAR      dir
      010058DBH   LINE      CODE     ---       #25
      010058DBH   LINE      CODE     ---       #26
      010058DBH   LINE      CODE     ---       #27
      010058E0H   LINE      CODE     ---       #28
      010058E5H   LINE      CODE     ---       #29
      010058EDH   LINE      CODE     ---       #30
      010058F0H   LINE      CODE     ---       #31
      010058F1H   LINE      CODE     ---       #32
      010058F4H   LINE      CODE     ---       #33
      010058F4H   LINE      CODE     ---       #34
      010058F4H   LINE      CODE     ---       #35
      ---         BLOCKEND  ---      ---       LVL=0

      01005573H   BLOCK     CODE     ---       LVL=0
      00000007H   SYMBOL    DATA     CHAR      dir
      01005573H   LINE      CODE     ---       #37
      01005573H   LINE      CODE     ---       #38
      01005573H   LINE      CODE     ---       #39
      01005578H   LINE      CODE     ---       #40
      0100559CH   LINE      CODE     ---       #41
      010055A4H   LINE      CODE     ---       #42
      010055A7H   LINE      CODE     ---       #43
      010055A8H   LINE      CODE     ---       #44
      010055AAH   LINE      CODE     ---       #45
      010055AAH   LINE      CODE     ---       #46
      010055AAH   LINE      CODE     ---       #47
      ---         BLOCKEND  ---      ---       LVL=0

      010059DBH   BLOCK     CODE     ---       LVL=0
      010059DBH   LINE      CODE     ---       #49
      010059DBH   LINE      CODE     ---       #50
      010059DBH   LINE      CODE     ---       #51
      010059E7H   LINE      CODE     ---       #52
      010059EAH   LINE      CODE     ---       #53
      010059EAH   LINE      CODE     ---       #54
      010059EDH   LINE      CODE     ---       #55
      010059EDH   LINE      CODE     ---       #56
      ---         BLOCKEND  ---      ---       LVL=0

      010059EEH   BLOCK     CODE     ---       LVL=0
      010059EEH   LINE      CODE     ---       #58
      010059EEH   LINE      CODE     ---       #59
      010059EEH   LINE      CODE     ---       #60
      010059FAH   LINE      CODE     ---       #61
      010059FDH   LINE      CODE     ---       #62
      010059FDH   LINE      CODE     ---       #63
      01005A00H   LINE      CODE     ---       #64
      01005A00H   LINE      CODE     ---       #65
      ---         BLOCKEND  ---      ---       LVL=0

      010053DAH   BLOCK     CODE     ---       LVL=0
      010053DAH   LINE      CODE     ---       #67
      010053DAH   LINE      CODE     ---       #68
      010053DAH   LINE      CODE     ---       #69
      010053E6H   LINE      CODE     ---       #70
      010053ECH   LINE      CODE     ---       #71
      010053F2H   LINE      CODE     ---       #72
LX51 LINKER/LOCATER V4.66.30.0                                                        07/27/2019  23:22:19  PAGE 203


      010053F9H   LINE      CODE     ---       #74
      01005403H   LINE      CODE     ---       #75
      01005409H   LINE      CODE     ---       #76
      0100540FH   LINE      CODE     ---       #77
      01005416H   LINE      CODE     ---       #78
      ---         BLOCKEND  ---      ---       LVL=0

      010000A6H   BLOCK     CODE     ---       LVL=0
      00000022H   SYMBOL    DATA     BYTE      idx
      010000A8H   BLOCK     CODE     NEAR LAB  LVL=1
      00000023H   SYMBOL    DATA     BYTE      i
      02000413H   SYMBOL    XDATA    ---       txt
      010033B1H   SYMBOL    CODE     ---       led_pos
      ---         BLOCKEND  ---      ---       LVL=1
      010000A6H   LINE      CODE     ---       #80
      010000A8H   LINE      CODE     ---       #81
      010000A8H   LINE      CODE     ---       #93
      010000CFH   LINE      CODE     ---       #94
      010000CFH   LINE      CODE     ---       #95
      010000D6H   LINE      CODE     ---       #96
      010000E6H   LINE      CODE     ---       #97
      010000EDH   LINE      CODE     ---       #98
      010000FDH   LINE      CODE     ---       #99
      01000104H   LINE      CODE     ---       #100
      01000114H   LINE      CODE     ---       #102
      0100012FH   LINE      CODE     ---       #103
      01000136H   LINE      CODE     ---       #104
      01000146H   LINE      CODE     ---       #105
      0100014DH   LINE      CODE     ---       #106
      0100015DH   LINE      CODE     ---       #107
      01000164H   LINE      CODE     ---       #108
      0100016EH   LINE      CODE     ---       #109
      01000171H   LINE      CODE     ---       #110
      01000171H   LINE      CODE     ---       #111
      01000171H   LINE      CODE     ---       #112
      01000178H   LINE      CODE     ---       #113
      01000188H   LINE      CODE     ---       #115
      0100018BH   LINE      CODE     ---       #116
      010001ADH   LINE      CODE     ---       #117
      010001D0H   LINE      CODE     ---       #118
      010001E0H   LINE      CODE     ---       #119
      0100020AH   LINE      CODE     ---       #120
      0100021DH   LINE      CODE     ---       #121
      01000222H   LINE      CODE     ---       #122
      01000232H   LINE      CODE     ---       #123
      01000241H   LINE      CODE     ---       #124
      01000241H   LINE      CODE     ---       #125
      01000241H   LINE      CODE     ---       #126
      01000241H   LINE      CODE     ---       #127
      01000248H   LINE      CODE     ---       #128
      01000258H   LINE      CODE     ---       #130
      01000274H   LINE      CODE     ---       #131
      0100027BH   LINE      CODE     ---       #132
      0100028BH   LINE      CODE     ---       #133
      010002A7H   LINE      CODE     ---       #134
      010002AEH   LINE      CODE     ---       #135
      010002BEH   LINE      CODE     ---       #136
      010002DAH   LINE      CODE     ---       #137
      010002E1H   LINE      CODE     ---       #138
      010002F1H   LINE      CODE     ---       #140
      0100031AH   LINE      CODE     ---       #142
      0100031FH   LINE      CODE     ---       #143
LX51 LINKER/LOCATER V4.66.30.0                                                        07/27/2019  23:22:19  PAGE 204


      01000349H   LINE      CODE     ---       #144
      0100034EH   LINE      CODE     ---       #146
      01000351H   LINE      CODE     ---       #147
      01000351H   LINE      CODE     ---       #148
      01000351H   LINE      CODE     ---       #149
      01000368H   LINE      CODE     ---       #150
      0100036FH   LINE      CODE     ---       #151
      0100037FH   LINE      CODE     ---       #153
      01000396H   LINE      CODE     ---       #154
      0100039DH   LINE      CODE     ---       #155
      010003ADH   LINE      CODE     ---       #157
      010003B4H   LINE      CODE     ---       #161
      0100041AH   LINE      CODE     ---       #162
      01000427H   LINE      CODE     ---       #163
      0100042AH   LINE      CODE     ---       #164
      0100042AH   LINE      CODE     ---       #165
      0100042AH   LINE      CODE     ---       #166
      01000431H   LINE      CODE     ---       #167
      01000441H   LINE      CODE     ---       #168
      01000447H   LINE      CODE     ---       #169
      01000463H   LINE      CODE     ---       #170
      01000473H   LINE      CODE     ---       #172
      0100047AH   LINE      CODE     ---       #173
      0100048AH   LINE      CODE     ---       #174
      01000490H   LINE      CODE     ---       #175
      010004ACH   LINE      CODE     ---       #176
      010004BCH   LINE      CODE     ---       #178
      010004C3H   LINE      CODE     ---       #179
      010004D3H   LINE      CODE     ---       #180
      010004EFH   LINE      CODE     ---       #181
      010004FFH   LINE      CODE     ---       #183
      01000506H   LINE      CODE     ---       #184
      01000516H   LINE      CODE     ---       #185
      01000537H   LINE      CODE     ---       #186
      01000544H   LINE      CODE     ---       #188
      01000547H   LINE      CODE     ---       #189
      01000547H   LINE      CODE     ---       #190
      01000547H   LINE      CODE     ---       #191
      0100054EH   LINE      CODE     ---       #192
      0100055EH   LINE      CODE     ---       #194
      01000573H   LINE      CODE     ---       #195
      0100057AH   LINE      CODE     ---       #196
      0100058AH   LINE      CODE     ---       #198
      010005A2H   LINE      CODE     ---       #199
      010005A9H   LINE      CODE     ---       #200
      010005B9H   LINE      CODE     ---       #202
      010005D1H   LINE      CODE     ---       #203
      010005DDH   LINE      CODE     ---       #204
      010005E4H   LINE      CODE     ---       #205
      01000606H   LINE      CODE     ---       #206
      01000606H   LINE      CODE     ---       #207
      01000606H   LINE      CODE     ---       #208
      01000606H   LINE      CODE     ---       #211
      0100060BH   LINE      CODE     ---       #214
      01000618H   LINE      CODE     ---       #215
      01000618H   LINE      CODE     ---       #216
      01000618H   LINE      CODE     ---       #217
      0100061BH   LINE      CODE     ---       #218
      0100061BH   LINE      CODE     ---       #219
      0100061BH   LINE      CODE     ---       #220
      0100061BH   LINE      CODE     ---       #221
      0100061EH   LINE      CODE     ---       #222
LX51 LINKER/LOCATER V4.66.30.0                                                        07/27/2019  23:22:19  PAGE 205


      01000620H   LINE      CODE     ---       #223
      01000622H   LINE      CODE     ---       #224
      01000622H   LINE      CODE     ---       #225
      01000622H   LINE      CODE     ---       #226
      01000625H   LINE      CODE     ---       #227
      0100062CH   LINE      CODE     ---       #228
      0100062CH   LINE      CODE     ---       #229
      0100062CH   LINE      CODE     ---       #230
      0100062CH   LINE      CODE     ---       #231
      ---         BLOCKEND  ---      ---       LVL=0

      ---         MODULE    ---      ---       MENU_DEF
      0100D033H   PUBLIC    CONST    ---       menu_6
      0100D027H   PUBLIC    CONST    ---       menu_5
      0100D01BH   PUBLIC    CONST    ---       menu_2
      0100D00FH   PUBLIC    CONST    ---       menu_1
      0100D003H   PUBLIC    CONST    ---       menu_0
      0100CFF7H   PUBLIC    CONST    ---       menu_none
      000000A2H   SFRSYM    DATA     BYTE      SPI0CKR
      00000080H   SFRSYM    DATA     BYTE      P0
      000000D0H.2 SFRSYM    DATA     BIT       PSW_OV
      000000B1H   SFRSYM    DATA     BYTE      XOSC0CN
      00000090H   SFRSYM    DATA     BYTE      P1
      000000A0H   SFRSYM    DATA     BYTE      P2
      000000B0H   SFRSYM    DATA     BYTE      P3
      000000BCH   SFRSYM    DATA     BYTE      ADC0CF
      000000C8H   SFRSYM    DATA     BIT       TMR2CN0_T2XCLK
      000000C7H   SFRSYM    DATA     BYTE      P4
      000000C0H.7 SFRSYM    DATA     BIT       SMB0CN0_MASTER
      000000F9H   SFRSYM    DATA     WORD      PCA0
      000000E6H   SFRSYM    DATA     BYTE      EIE1
      000000C0H.7 SFRSYM    DATA     BIT       SMB1CN0_MASTER
      000000C0H.1 SFRSYM    DATA     BIT       SMB0CN0_ACK
      000000D7H   SFRSYM    DATA     BYTE      USB0XCN
      000000E7H   SFRSYM    DATA     BYTE      EIE2
      000000C0H.1 SFRSYM    DATA     BIT       SMB1CN0_ACK
      0000008FH   SFRSYM    DATA     BYTE      PSCTL
      000000E4H   SFRSYM    DATA     BYTE      IT01CF
      000000C8H   SFRSYM    DATA     BIT       TMR5CN0_T5XCLK
      000000C0H.6 SFRSYM    DATA     BIT       SMB0CN0_TXMODE
      000000C0H.6 SFRSYM    DATA     BIT       SMB1CN0_TXMODE
      000000BFH   SFRSYM    DATA     BYTE      SFRPAGE
      000000A4H   SFRSYM    DATA     BYTE      P0MDOUT
      000000A5H   SFRSYM    DATA     BYTE      P1MDOUT
      000000E8H.5 SFRSYM    DATA     BIT       ADC0CN0_ADINT
      000000CBH   SFRSYM    DATA     BYTE      TMR2RLH
      000000A6H   SFRSYM    DATA     BYTE      P2MDOUT
      000000A8H   SFRSYM    DATA     BYTE      IE
      00000093H   SFRSYM    DATA     BYTE      TMR3RLH
      000000A7H   SFRSYM    DATA     BYTE      P3MDOUT
      00000093H   SFRSYM    DATA     BYTE      TMR4RLH
      000000AEH   SFRSYM    DATA     BYTE      P4MDOUT
      000000F6H   SFRSYM    DATA     BYTE      EIP1
      000000CBH   SFRSYM    DATA     BYTE      TMR5RLH
      000000F7H   SFRSYM    DATA     BYTE      EIP2
      00000098H.2 SFRSYM    DATA     BIT       SCON0_RB8
      000000CAH   SFRSYM    DATA     BYTE      TMR2RLL
      000000FCH   SFRSYM    DATA     BYTE      PCA0CPH0
      00000092H   SFRSYM    DATA     BYTE      TMR3RLL
      000000EAH   SFRSYM    DATA     BYTE      PCA0CPH1
      00000098H.3 SFRSYM    DATA     BIT       SCON0_TB8
      000000F0H   SFRSYM    DATA     BIT       B_B0
LX51 LINKER/LOCATER V4.66.30.0                                                        07/27/2019  23:22:19  PAGE 206


      00000082H   SFRSYM    DATA     WORD      DP
      00000092H   SFRSYM    DATA     BYTE      TMR4RLL
      000000ECH   SFRSYM    DATA     BYTE      PCA0CPH2
      000000F0H.1 SFRSYM    DATA     BIT       B_B1
      000000C3H   SFRSYM    DATA     WORD      ADC0GT
      000000CAH   SFRSYM    DATA     BYTE      TMR5RLL
      000000EEH   SFRSYM    DATA     BYTE      PCA0CPH3
      000000F0H.2 SFRSYM    DATA     BIT       B_B2
      000000FBH   SFRSYM    DATA     BYTE      PCA0CPL0
      000000FEH   SFRSYM    DATA     BYTE      PCA0CPH4
      00000085H   SFRSYM    DATA     BYTE      EMI0CF
      000000F0H.3 SFRSYM    DATA     BIT       B_B3
      000000D9H   SFRSYM    DATA     BYTE      PCA0MD
      000000DAH   SFRSYM    DATA     BYTE      PCA0CPM0
      000000E9H   SFRSYM    DATA     BYTE      PCA0CPL1
      000000F0H.4 SFRSYM    DATA     BIT       B_B4
      000000DBH   SFRSYM    DATA     BYTE      PCA0CPM1
      000000EBH   SFRSYM    DATA     BYTE      PCA0CPL2
      000000F0H.5 SFRSYM    DATA     BIT       B_B5
      000000DCH   SFRSYM    DATA     BYTE      PCA0CPM2
      000000EDH   SFRSYM    DATA     BYTE      PCA0CPL3
      000000B8H   SFRSYM    DATA     BYTE      IP
      000000F0H.6 SFRSYM    DATA     BIT       B_B6
      000000C5H   SFRSYM    DATA     WORD      ADC0LT
      000000DDH   SFRSYM    DATA     BYTE      PCA0CPM3
      000000FDH   SFRSYM    DATA     BYTE      PCA0CPL4
      00000098H.5 SFRSYM    DATA     BIT       SCON0_MCE
      000000F0H.7 SFRSYM    DATA     BIT       B_B7
      000000DEH   SFRSYM    DATA     BYTE      PCA0CPM4
      000000E1H   SFRSYM    DATA     BYTE      XBR0
      000000C1H   SFRSYM    DATA     BYTE      SMB0CF
      000000E2H   SFRSYM    DATA     BYTE      XBR1
      000000C1H   SFRSYM    DATA     BYTE      SMB1CF
      000000AFH   SFRSYM    DATA     BYTE      PFE0CN
      000000AAH   SFRSYM    DATA     BYTE      EMI0CN
      000000C0H.5 SFRSYM    DATA     BIT       SMB0CN0_STA
      000000E3H   SFRSYM    DATA     BYTE      XBR2
      000000C0H.5 SFRSYM    DATA     BIT       SMB1CN0_STA
      000000E0H   SFRSYM    DATA     BIT       ACC_ACC0
      000000D1H   SFRSYM    DATA     BYTE      REF0CN
      000000B2H   SFRSYM    DATA     BYTE      HFO0CN
      0000008EH   SFRSYM    DATA     BYTE      CKCON0
      000000E0H.1 SFRSYM    DATA     BIT       ACC_ACC1
      000000E4H   SFRSYM    DATA     BYTE      CKCON1
      000000C8H.2 SFRSYM    DATA     BIT       TMR2CN0_TR2
      000000E0H.2 SFRSYM    DATA     BIT       ACC_ACC2
      000000E0H.3 SFRSYM    DATA     BIT       ACC_ACC3
      00000081H   SFRSYM    DATA     BYTE      SP
      0000009DH   SFRSYM    DATA     BYTE      CMP0MD
      000000E0H.4 SFRSYM    DATA     BIT       ACC_ACC4
      00000086H   SFRSYM    DATA     BYTE      LFO0CN
      00000084H   SFRSYM    DATA     BYTE      EMI0TC
      0000009CH   SFRSYM    DATA     BYTE      CMP1MD
      000000D8H   SFRSYM    DATA     BIT       PCA0CN0_CCF0
      000000E0H.5 SFRSYM    DATA     BIT       ACC_ACC5
      000000D8H.1 SFRSYM    DATA     BIT       PCA0CN0_CCF1
      000000E0H.6 SFRSYM    DATA     BIT       ACC_ACC6
      000000CCH   SFRSYM    DATA     WORD      TMR2
      000000D8H.2 SFRSYM    DATA     BIT       PCA0CN0_CCF2
      000000E0H.7 SFRSYM    DATA     BIT       ACC_ACC7
      00000094H   SFRSYM    DATA     WORD      TMR3
      000000C8H.2 SFRSYM    DATA     BIT       TMR5CN0_TR5
LX51 LINKER/LOCATER V4.66.30.0                                                        07/27/2019  23:22:19  PAGE 207


      000000D8H.3 SFRSYM    DATA     BIT       PCA0CN0_CCF3
      00000094H   SFRSYM    DATA     WORD      TMR4
      000000ACH   SFRSYM    DATA     BYTE      SBCON1
      000000D8H.4 SFRSYM    DATA     BIT       PCA0CN0_CCF4
      000000CCH   SFRSYM    DATA     WORD      TMR5
      000000C0H.3 SFRSYM    DATA     BIT       SMB0CN0_ACKRQ
      000000FFH   SFRSYM    DATA     BYTE      VDM0CN
      000000F1H   SFRSYM    DATA     BYTE      P0MDIN
      000000C0H.3 SFRSYM    DATA     BIT       SMB1CN0_ACKRQ
      00000098H.4 SFRSYM    DATA     BIT       SCON0_REN
      000000F2H   SFRSYM    DATA     BYTE      P1MDIN
      000000F3H   SFRSYM    DATA     BYTE      P2MDIN
      000000C0H.4 SFRSYM    DATA     BIT       SMB0CN0_STO
      000000F4H   SFRSYM    DATA     BYTE      P3MDIN
      000000C0H.4 SFRSYM    DATA     BIT       SMB1CN0_STO
      000000B5H   SFRSYM    DATA     BYTE      SBRLH1
      000000F5H   SFRSYM    DATA     BYTE      P4MDIN
      000000D0H.3 SFRSYM    DATA     BIT       PSW_RS0
      000000D8H.7 SFRSYM    DATA     BIT       PCA0CN0_CF
      000000F8H.4 SFRSYM    DATA     BIT       SPI0CN0_RXOVRN
      000000D0H.4 SFRSYM    DATA     BIT       PSW_RS1
      000000B4H   SFRSYM    DATA     BYTE      SBRLL1
      000000E8H.7 SFRSYM    DATA     BIT       ADC0CN0_ADEN
      00000089H   SFRSYM    DATA     BYTE      TMOD
      00000088H   SFRSYM    DATA     BYTE      TCON
      000000D0H   SFRSYM    DATA     BIT       PSW_PARITY
      000000A8H.4 SFRSYM    DATA     BIT       IE_ES0
      0000009FH   SFRSYM    DATA     BYTE      CMP0MX
      000000A8H.1 SFRSYM    DATA     BIT       IE_ET0
      0000009EH   SFRSYM    DATA     BYTE      CMP1MX
      000000A8H.3 SFRSYM    DATA     BIT       IE_ET1
      000000D4H   SFRSYM    DATA     BYTE      P0SKIP
      000000C8H.1 SFRSYM    DATA     BIT       TMR2CN0_T2CSS
      000000A8H.5 SFRSYM    DATA     BIT       IE_ET2
      000000D5H   SFRSYM    DATA     BYTE      P1SKIP
      000000D6H   SFRSYM    DATA     BYTE      P2SKIP
      000000E8H   SFRSYM    DATA     BYTE      ADC0CN0
      000000A8H   SFRSYM    DATA     BIT       IE_EX0
      000000DFH   SFRSYM    DATA     BYTE      P3SKIP
      000000D8H.6 SFRSYM    DATA     BIT       PCA0CN0_CR
      000000A8H.2 SFRSYM    DATA     BIT       IE_EX1
      00000098H.7 SFRSYM    DATA     BIT       SCON0_SMODE
      000000A9H   SFRSYM    DATA     BYTE      CLKSEL
      000000F8H   SFRSYM    DATA     BIT       SPI0CN0_SPIEN
      000000F0H   SFRSYM    DATA     BYTE      B
      000000BEH   SFRSYM    DATA     BYTE      ADC0H
      000000E8H.6 SFRSYM    DATA     BIT       ADC0CN0_ADTM
      000000CAH   SFRSYM    DATA     WORD      TMR2RL
      000000BDH   SFRSYM    DATA     BYTE      ADC0L
      00000092H   SFRSYM    DATA     WORD      TMR3RL
      00000092H   SFRSYM    DATA     WORD      TMR4RL
      000000D8H   SFRSYM    DATA     BYTE      PCA0CN0
      000000E0H   SFRSYM    DATA     BYTE      ACC
      000000CAH   SFRSYM    DATA     WORD      TMR5RL
      000000FBH   SFRSYM    DATA     WORD      PCA0CP0
      000000E9H   SFRSYM    DATA     WORD      PCA0CP1
      000000EBH   SFRSYM    DATA     WORD      PCA0CP2
      000000EDH   SFRSYM    DATA     WORD      PCA0CP3
      0000008CH   SFRSYM    DATA     BYTE      TH0
      000000B8H.4 SFRSYM    DATA     BIT       IP_PS0
      000000FDH   SFRSYM    DATA     WORD      PCA0CP4
      0000008DH   SFRSYM    DATA     BYTE      TH1
LX51 LINKER/LOCATER V4.66.30.0                                                        07/27/2019  23:22:19  PAGE 208


      000000FAH   SFRSYM    DATA     BYTE      PCA0H
      000000B8H.1 SFRSYM    DATA     BIT       IP_PT0
      000000B8H.3 SFRSYM    DATA     BIT       IP_PT1
      000000C0H.2 SFRSYM    DATA     BIT       SMB0CN0_ARBLOST
      000000B8H.5 SFRSYM    DATA     BIT       IP_PT2
      0000008AH   SFRSYM    DATA     BYTE      TL0
      000000F8H.1 SFRSYM    DATA     BIT       SPI0CN0_TXBMT
      000000C0H.2 SFRSYM    DATA     BIT       SMB1CN0_ARBLOST
      000000D0H.5 SFRSYM    DATA     BIT       PSW_F0
      000000A8H.6 SFRSYM    DATA     BIT       IE_ESPI0
      0000008BH   SFRSYM    DATA     BYTE      TL1
      000000F9H   SFRSYM    DATA     BYTE      PCA0L
      000000C0H   SFRSYM    DATA     BIT       SMB0CN0_SI
      000000D0H.1 SFRSYM    DATA     BIT       PSW_F1
      00000080H   SFRSYM    DATA     BIT       P0_B0
      000000B8H   SFRSYM    DATA     BIT       IP_PX0
      000000C9H   SFRSYM    DATA     BYTE      REG01CN
      000000C0H   SFRSYM    DATA     BIT       SMB1CN0_SI
      00000090H   SFRSYM    DATA     BIT       P1_B0
      00000080H.1 SFRSYM    DATA     BIT       P0_B1
      000000B8H.2 SFRSYM    DATA     BIT       IP_PX1
      0000009BH   SFRSYM    DATA     BYTE      CMP0CN0
      00000088H.1 SFRSYM    DATA     BIT       TCON_IE0
      000000A0H   SFRSYM    DATA     BIT       P2_B0
      00000090H.1 SFRSYM    DATA     BIT       P1_B1
      00000080H.2 SFRSYM    DATA     BIT       P0_B2
      0000009AH   SFRSYM    DATA     BYTE      CMP1CN0
      00000088H.3 SFRSYM    DATA     BIT       TCON_IE1
      000000B0H   SFRSYM    DATA     BIT       P3_B0
      000000A0H.1 SFRSYM    DATA     BIT       P2_B1
      00000090H.2 SFRSYM    DATA     BIT       P1_B2
      00000080H.3 SFRSYM    DATA     BIT       P0_B3
      000000C0H   SFRSYM    DATA     BYTE      SMB0CN0
      000000B0H.1 SFRSYM    DATA     BIT       P3_B1
      000000A0H.2 SFRSYM    DATA     BIT       P2_B2
      00000090H.3 SFRSYM    DATA     BIT       P1_B3
      00000080H.4 SFRSYM    DATA     BIT       P0_B4
      000000C0H   SFRSYM    DATA     BYTE      SMB1CN0
      000000B0H.2 SFRSYM    DATA     BIT       P3_B2
      000000A0H.3 SFRSYM    DATA     BIT       P2_B3
      00000090H.4 SFRSYM    DATA     BIT       P1_B4
      00000080H.5 SFRSYM    DATA     BIT       P0_B5
      000000B0H.3 SFRSYM    DATA     BIT       P3_B3
      000000A0H.4 SFRSYM    DATA     BIT       P2_B4
      00000090H.5 SFRSYM    DATA     BIT       P1_B5
      00000080H.6 SFRSYM    DATA     BIT       P0_B6
      000000B0H.4 SFRSYM    DATA     BIT       P3_B4
      000000A0H.5 SFRSYM    DATA     BIT       P2_B5
      00000090H.6 SFRSYM    DATA     BIT       P1_B6
      00000080H.7 SFRSYM    DATA     BIT       P0_B7
      000000B0H.5 SFRSYM    DATA     BIT       P3_B5
      000000A0H.6 SFRSYM    DATA     BIT       P2_B6
      00000090H.7 SFRSYM    DATA     BIT       P1_B7
      000000B0H.6 SFRSYM    DATA     BIT       P3_B6
      000000A0H.7 SFRSYM    DATA     BIT       P2_B7
      000000B0H.7 SFRSYM    DATA     BIT       P3_B7
      00000083H   SFRSYM    DATA     BYTE      DPH
      000000C4H   SFRSYM    DATA     BYTE      ADC0GTH
      000000C8H.7 SFRSYM    DATA     BIT       TMR2CN0_TF2H
      000000C8H.3 SFRSYM    DATA     BIT       TMR2CN0_T2SPLIT
      000000D0H.6 SFRSYM    DATA     BIT       PSW_AC
      000000F8H   SFRSYM    DATA     BYTE      SPI0CN0
LX51 LINKER/LOCATER V4.66.30.0                                                        07/27/2019  23:22:19  PAGE 209


      000000B3H   SFRSYM    DATA     BYTE      HFO0CAL
      00000088H.5 SFRSYM    DATA     BIT       TCON_TF0
      00000098H   SFRSYM    DATA     BIT       SCON0_RI
      00000082H   SFRSYM    DATA     BYTE      DPL
      00000088H.7 SFRSYM    DATA     BIT       TCON_TF1
      00000099H   SFRSYM    DATA     BYTE      SBUF0
      00000087H   SFRSYM    DATA     BYTE      PCON0
      000000C3H   SFRSYM    DATA     BYTE      ADC0GTL
      000000C8H.6 SFRSYM    DATA     BIT       TMR2CN0_TF2L
      00000098H.1 SFRSYM    DATA     BIT       SCON0_TI
      000000E8H   SFRSYM    DATA     BIT       ADC0CN0_ADCM0
      000000D3H   SFRSYM    DATA     BYTE      SBUF1
      000000C6H   SFRSYM    DATA     BYTE      ADC0LTH
      00000088H   SFRSYM    DATA     BIT       TCON_IT0
      000000E8H.1 SFRSYM    DATA     BIT       ADC0CN0_ADCM1
      000000EFH   SFRSYM    DATA     BYTE      RSTSRC
      000000C8H.7 SFRSYM    DATA     BIT       TMR5CN0_TF5H
      000000C8H.3 SFRSYM    DATA     BIT       TMR5CN0_T5SPLIT
      00000088H.2 SFRSYM    DATA     BIT       TCON_IT1
      000000E8H.2 SFRSYM    DATA     BIT       ADC0CN0_ADCM2
      00000098H   SFRSYM    DATA     BYTE      SCON0
      000000E8H.3 SFRSYM    DATA     BIT       ADC0CN0_ADWINT
      000000B4H   SFRSYM    DATA     WORD      SBRL1
      000000E5H   SFRSYM    DATA     BYTE      SMOD1
      000000D2H   SFRSYM    DATA     BYTE      SCON1
      000000BAH   SFRSYM    DATA     BYTE      AMX0N
      000000E8H.4 SFRSYM    DATA     BIT       ADC0CN0_ADBUSY
      000000CEH   SFRSYM    DATA     BYTE      SMB0ADM
      000000C5H   SFRSYM    DATA     BYTE      ADC0LTL
      000000F8H.5 SFRSYM    DATA     BIT       SPI0CN0_MODF
      000000B8H.6 SFRSYM    DATA     BIT       IP_PSPI0
      000000CEH   SFRSYM    DATA     BYTE      SMB1ADM
      000000BBH   SFRSYM    DATA     BYTE      AMX0P
      000000C8H.6 SFRSYM    DATA     BIT       TMR5CN0_TF5L
      000000C8H   SFRSYM    DATA     BYTE      TMR2CN0
      00000091H   SFRSYM    DATA     BYTE      TMR3CN0
      00000091H   SFRSYM    DATA     BYTE      TMR4CN0
      000000C8H   SFRSYM    DATA     BYTE      TMR5CN0
      000000CFH   SFRSYM    DATA     BYTE      SMB0ADR
      00000088H.4 SFRSYM    DATA     BIT       TCON_TR0
      000000CFH   SFRSYM    DATA     BYTE      SMB1ADR
      000000C8H.4 SFRSYM    DATA     BIT       TMR2CN0_TF2CEN
      00000088H.6 SFRSYM    DATA     BIT       TCON_TR1
      000000C2H   SFRSYM    DATA     BYTE      SMB0DAT
      000000CDH   SFRSYM    DATA     BYTE      TMR2H
      000000A1H   SFRSYM    DATA     BYTE      SPI0CFG
      000000C2H   SFRSYM    DATA     BYTE      SMB1DAT
      00000095H   SFRSYM    DATA     BYTE      TMR3H
      00000095H   SFRSYM    DATA     BYTE      TMR4H
      000000CDH   SFRSYM    DATA     BYTE      TMR5H
      000000CCH   SFRSYM    DATA     BYTE      TMR2L
      000000F8H.7 SFRSYM    DATA     BIT       SPI0CN0_SPIF
      00000096H   SFRSYM    DATA     BYTE      USB0ADR
      00000094H   SFRSYM    DATA     BYTE      TMR3L
      000000A8H.7 SFRSYM    DATA     BIT       IE_EA
      00000094H   SFRSYM    DATA     BYTE      TMR4L
      00000097H   SFRSYM    DATA     BYTE      USB0DAT
      000000CCH   SFRSYM    DATA     BYTE      TMR5L
      000000B6H   SFRSYM    DATA     BYTE      FLSCL
      000000C8H.5 SFRSYM    DATA     BIT       TMR2CN0_TF2LEN
      000000F8H.6 SFRSYM    DATA     BIT       SPI0CN0_WCOL
      000000F8H.2 SFRSYM    DATA     BIT       SPI0CN0_NSSMD0
LX51 LINKER/LOCATER V4.66.30.0                                                        07/27/2019  23:22:19  PAGE 210


      000000D0H.7 SFRSYM    DATA     BIT       PSW_CY
      000000A3H   SFRSYM    DATA     BYTE      SPI0DAT
      000000F8H.3 SFRSYM    DATA     BIT       SPI0CN0_NSSMD1
      000000BDH   SFRSYM    DATA     WORD      ADC0
      000000B9H   SFRSYM    DATA     BYTE      SMBTC
      000000D0H   SFRSYM    DATA     BYTE      PSW
      000000C8H.5 SFRSYM    DATA     BIT       TMR5CN0_TF5LEN
      000000B7H   SFRSYM    DATA     BYTE      FLKEY

      ---         MODULE    ---      ---       ?C_INIT
      010047F7H   PUBLIC    CODE     ---       ?C_START

      ---         MODULE    ---      ---       ?C?CLDPTR
      0100062DH   PUBLIC    CODE     ---       ?C?CLDPTR

      ---         MODULE    ---      ---       ?C?CLDOPTR
      01000646H   PUBLIC    CODE     ---       ?C?CLDOPTR

      ---         MODULE    ---      ---       ?C?CILDPTR
      01000673H   PUBLIC    CODE     ---       ?C?CILDPTR

      ---         MODULE    ---      ---       ?C?CILDOPTR
      01000695H   PUBLIC    CODE     ---       ?C?CILDOPTR

      ---         MODULE    ---      ---       ?C?CSTPTR
      010006C8H   PUBLIC    CODE     ---       ?C?CSTPTR

      ---         MODULE    ---      ---       ?C?CSTOPTR
      010006DAH   PUBLIC    CODE     ---       ?C?CSTOPTR

      ---         MODULE    ---      ---       ?C?IMUL
      010006FCH   PUBLIC    CODE     ---       ?C?IMUL

      ---         MODULE    ---      ---       ?C?UIDIV
      0100070EH   PUBLIC    CODE     ---       ?C?UIDIV

      ---         MODULE    ---      ---       ?C?SIDIV
      01000763H   PUBLIC    CODE     ---       ?C?SIDIV

      ---         MODULE    ---      ---       ?C?IILDX
      01000799H   PUBLIC    CODE     ---       ?C?IILDX

      ---         MODULE    ---      ---       ?C?ILDPTR
      010007AFH   PUBLIC    CODE     ---       ?C?ILDPTR

      ---         MODULE    ---      ---       ?C?ILDOPTR
      010007DAH   PUBLIC    CODE     ---       ?C?ILDOPTR

      ---         MODULE    ---      ---       ?C?ISTPTR
      01000812H   PUBLIC    CODE     ---       ?C?ISTPTR

      ---         MODULE    ---      ---       ?C?ISTOPTR
      01000831H   PUBLIC    CODE     ---       ?C?ISTOPTR

      ---         MODULE    ---      ---       ?C?ULDIV
      0100089AH   PUBLIC    CODE     ---       ?C?ULDIV

      ---         MODULE    ---      ---       ?C?ULCMP
      0100092CH   PUBLIC    CODE     ---       ?C?ULCMP

      ---         MODULE    ---      ---       ?C?ULSHR
      0100093DH   PUBLIC    CODE     ---       ?C?ULSHR
LX51 LINKER/LOCATER V4.66.30.0                                                        07/27/2019  23:22:19  PAGE 211



      ---         MODULE    ---      ---       ?C?LLDXDATA
      01000950H   PUBLIC    CODE     ---       ?C?LLDXDATA

      ---         MODULE    ---      ---       ?C?LSTXDATA
      0100095CH   PUBLIC    CODE     ---       ?C?LSTXDATA

      ---         MODULE    ---      ---       ?C?OFFXADD
      01000968H   PUBLIC    CODE     ---       ?C?OFFXADD

      ---         MODULE    ---      ---       ?C?PLDIIDATA
      01000974H   PUBLIC    CODE     ---       ?C?PLDIIDATA

      ---         MODULE    ---      ---       ?C?PLDXDATA
      01000984H   PUBLIC    CODE     ---       ?C?PLDXDATA

      ---         MODULE    ---      ---       ?C?PSTXDATA
      0100098DH   PUBLIC    CODE     ---       ?C?PSTXDATA

      ---         MODULE    ---      ---       ?C?PLDPDATA
      01000996H   PUBLIC    CODE     ---       ?C?PLDPDATA

      ---         MODULE    ---      ---       ?C?PSTPDATA
      0100099FH   PUBLIC    CODE     ---       ?C?PSTPDATA

      ---         MODULE    ---      ---       ?C?PLDCODE
      010009A8H   PUBLIC    CODE     ---       ?C?PLDCODE

      ---         MODULE    ---      ---       ?C?CCASE
      010009B4H   PUBLIC    CODE     ---       ?C?CCASE

      ---         MODULE    ---      ---       ?C?ICALL
      010009DAH   PUBLIC    CODE     ---       ?C?ICALL
      010009DEH   PUBLIC    CODE     ---       ?C?ICALL2

      ---         MODULE    ---      ---       PRINTF
      0000002AH   PUBLIC    DATA     ---       ?_PRINTF517?BYTE
      0000002AH   PUBLIC    DATA     ---       ?_PRINTF?BYTE
      0000002AH   PUBLIC    DATA     ---       ?_SPRINTF517?BYTE
      0000002AH   PUBLIC    DATA     ---       ?_SPRINTF?BYTE
      0100121BH   PUBLIC    CODE     ---       _PRINTF
      0100121BH   PUBLIC    CODE     ---       _PRINTF517
      01001215H   PUBLIC    CODE     ---       _SPRINTF
      01001215H   PUBLIC    CODE     ---       _SPRINTF517

      ---         MODULE    ---      ---       ABS
      01005AD9H   PUBLIC    CODE     ---       _ABS

      ---         MODULE    ---      ---       ?C?STRCPY
      01000AACH   PUBLIC    CODE     ---       ?C?STRCPY

      ---         MODULE    ---      ---       STRLEN
      01005979H   PUBLIC    CODE     ---       _STRLEN

      ---         MODULE    ---      ---       ?C?MEMSET
      01000AC9H   PUBLIC    CODE     ---       ?C?MEMSET

      ---         MODULE    ---      ---       PUTCHAR
      01005752H   PUBLIC    CODE     ---       _PUTCHAR

Program Size: data=141.4 xdata=1216 const=29908 code=23475
LX51 RUN COMPLETE.  0 WARNING(S),  0 ERROR(S)
